 RylAuthServer

 Timestamp is 421aab5f (Tue Feb 22 12:47:43 2005)

 Preferred load address is 00400000

 Start         Length     Name                   Class
 0001:00000000 000461e0H .text                   CODE
 0001:000461e0 000022c6H .text$x                 CODE
 0001:000484b0 0000046eH .text$yc                CODE
 0001:00048920 000002a6H .text$yd                CODE
 0002:00000000 000002fcH .idata$5                DATA
 0002:00000300 00016d70H .rdata                  DATA
 0002:00017070 00000097H .rdata$debug            DATA
 0002:00017108 000005b0H .rdata$r                DATA
 0002:000176b8 00000004H .rtc$IAA                DATA
 0002:000176bc 00000004H .rtc$IZZ                DATA
 0002:000176c0 00000004H .rtc$TAA                DATA
 0002:000176c4 00000004H .rtc$TZZ                DATA
 0002:000176c8 00002bacH .xdata$x                DATA
 0002:0001a274 00000000H ATL$__a                 DATA
 0002:0001a274 00000000H ATL$__z                 DATA
 0002:0001a274 000000c8H .idata$2                DATA
 0002:0001a33c 00000014H .idata$3                DATA
 0002:0001a350 000002fcH .idata$4                DATA
 0002:0001a64c 00000bb6H .idata$6                DATA
 0002:0001b202 00000000H .edata                  DATA
 0003:00000000 00000004H .CRT$XCA                DATA
 0003:00000004 00000004H .CRT$XCAA               DATA
 0003:00000008 0000001cH .CRT$XCC                DATA
 0003:00000024 00000004H .CRT$XCL                DATA
 0003:00000028 000000a0H .CRT$XCU                DATA
 0003:000000c8 00000004H .CRT$XCZ                DATA
 0003:000000cc 00000004H .CRT$XIA                DATA
 0003:000000d0 0000000cH .CRT$XIC                DATA
 0003:000000dc 00000004H .CRT$XIY                DATA
 0003:000000e0 00000004H .CRT$XIZ                DATA
 0003:000000e4 00000004H .CRT$XLA                DATA
 0003:000000e8 00000004H .CRT$XLZ                DATA
 0003:000000ec 00000004H .CRT$XPA                DATA
 0003:000000f0 00000004H .CRT$XPX                DATA
 0003:000000f4 00000004H .CRT$XPZ                DATA
 0003:000000f8 00000004H .CRT$XTA                DATA
 0003:000000fc 00000004H .CRT$XTB                DATA
 0003:00000100 00000004H .CRT$XTZ                DATA
 0003:00000110 000058dcH .data                   DATA
 0003:00005a00 000443e8H .bss                    DATA
 0004:00000000 00000001H .tls                    DATA
 0004:00000008 00000104H .tls$                   DATA
 0004:0000010c 00000001H .tls$ZZZ                DATA
 0005:00000000 000000e8H .rsrc$01                DATA
 0005:000000f0 00000dd8H .rsrc$02                DATA

  Address         Publics by Value              Rva+Base     Lib:Object

 0000:00000000       ___safe_se_handler_table   00000000     <absolute>
 0000:00000000       ___safe_se_handler_count   00000000     <absolute>
 0000:00000000       __except_list              00000000     <absolute>
 0000:0000002c       __tls_array                0000002c     <absolute>
 0000:00000000       ___ImageBase               00400000     <linker-defined>
 0001:00000000       ?Connected@CPacketDispatch@@UAEXXZ 00401000 f i rylgamelibrary:rylserverdispatch.obj
 0001:00000000       ??1INET_Addr@@QAE@XZ       00401000 f i authagentdispatch.obj
 0001:00000000       ?Disconnected@CPacketDispatch@@UAEXXZ 00401000 f i rylgamelibrary:rylserverdispatch.obj
 0001:00000000       ?GenCode_Assert@@YAXPAUSNode@@W4eRegister@@@Z 00401000 f i rylgamelibrary:imcodegen.obj
 0001:00000000       ??1CBuffer@@QAE@XZ         00401000 f i rylgamelibrary:buffer.obj
 0001:00000000       ??3@YAXPAX0@Z              00401000 f i authorizeuser.obj
 0001:00000000       ?GenCode_Empty@@YAXPAUSNode@@W4eRegister@@@Z 00401000 f i rylgamelibrary:imcodegen.obj
 0001:00000010       ??_H@YGXPAXIHP6EPAX0@Z@Z   00401010 f i authagentdispatch.obj
 0001:00000040       ?SetMoveAddress@CAuthClientDispatch@@QAEXKABVINET_Addr@@@Z 00401040 f i authagentdispatch.obj
 0001:00000080       ??0CAuthAgentDispatch@@QAE@AAVCSession@@@Z 00401080 f   authagentdispatch.obj
 0001:000000a0       ??1CAuthAgentDispatch@@UAE@XZ 004010a0 f   authagentdispatch.obj
 0001:00000110       ?ParseSysChannelUpdate@CAuthAgentDispatch@@AAE_NPAUPktSCInfo@@@Z 00401110 f   authagentdispatch.obj
 0001:00000130       ?ParseSysServerVerUpdate@CAuthAgentDispatch@@AAE_NPAUPktSVU@@@Z 00401130 f   authagentdispatch.obj
 0001:00000160       ?ParseAgentZone@CAuthAgentDispatch@@AAE_NPAUPktDD@@@Z 00401160 f   authagentdispatch.obj
 0001:000003f0       ?SendUserKill@CAuthAgentDispatch@@AAE_NKG@Z 004013f0 f   authagentdispatch.obj
 0001:00000440       ?SendSysServerLogin@CAuthAgentDispatch@@AAE_NK@Z 00401440 f   authagentdispatch.obj
 0001:000004e0       ?ParseBillingTimeoutNotify@CAuthAgentDispatch@@AAE_NPAUPktBTN@@@Z 004014e0 f   authagentdispatch.obj
 0001:000005d0       ?ParseBillingTimeCheckNotify@CAuthAgentDispatch@@AAE_NPAUPktBTN@@@Z 004015d0 f   authagentdispatch.obj
 0001:000006c0       ??$accumulate@PAGH@std@@YAHPAG0H@Z 004016c0 f i authagentdispatch.obj
 0001:000006e0       ??0RylServerInfo@@QAE@XZ   004016e0 f i authagentdispatch.obj
 0001:00000740       ??_ECAuthAgentDispatch@@UAEPAXI@Z 00401740 f i authagentdispatch.obj
 0001:00000740       ??_GCAuthAgentDispatch@@UAEPAXI@Z 00401740 f i authagentdispatch.obj
 0001:00000760       ?GetDispatchTable@CAuthAgentDispatch@@SAAAVCSingleDispatch@@XZ 00401760 f   authagentdispatch.obj
 0001:000007c0       ?Connected@CAuthAgentDispatch@@UAEXXZ 004017c0 f   authagentdispatch.obj
 0001:00000810       ?Disconnected@CAuthAgentDispatch@@UAEXXZ 00401810 f   authagentdispatch.obj
 0001:00000890       ?ParseSysServerLogin@CAuthAgentDispatch@@AAE_NPAUPktSLAck@@@Z 00401890 f   authagentdispatch.obj
 0001:00000980       ?ParseUserKill@CAuthAgentDispatch@@AAE_NPAUPktUK@@@Z 00401980 f   authagentdispatch.obj
 0001:00000a60       ?SendStartSession@CAuthAgentDispatch@@SA_NPAVCAuthClientDispatch@@KPADKG@Z 00401a60 f   authagentdispatch.obj
 0001:00000bd0       ?SendCreateCharEquipItem@CAuthAgentDispatch@@AAE_NKGGG@Z 00401bd0 f   authagentdispatch.obj
 0001:00000d50       ?ParseDBGetData@CAuthAgentDispatch@@AAE_NPAUPktDD@@@Z 00401d50 f   authagentdispatch.obj
 0001:000010f0       ?DispatchPacket@CAuthAgentDispatch@@EAE_NPAUPktBase@@@Z 004020f0 f   authagentdispatch.obj
 0001:00001230       ??0Syncronize@?$CLock@VCCSLock@@@@QAE@AAVCCSLock@@@Z 00402230 f i authagentservertable.obj
 0001:00001250       ??1Syncronize@?$CLock@VCCSLock@@@@QAE@XZ 00402250 f i authagentservertable.obj
 0001:00001260       ?GetPatchServerAddress@CAuthAgentServerTable@@QAEXAAKPADI@Z 00402260 f   authagentservertable.obj
 0001:000012b0       ?UpdateServerData@CAuthAgentServerTable@@QAEXKKPBD@Z 004022b0 f   authagentservertable.obj
 0001:00001300       ?GetServerVersion@CAuthAgentServerTable@@QAEKXZ 00402300 f   authagentservertable.obj
 0001:00001320       ?GetServerChecksum@CAuthAgentServerTable@@QAEKXZ 00402320 f   authagentservertable.obj
 0001:00001340       ?SetAgentServerInfo@CAuthAgentServerTable@@QAEXAAURylServerInfo@@@Z 00402340 f   authagentservertable.obj
 0001:00001370       ?GetAgentServerInfo@CAuthAgentServerTable@@QAEXAAURylServerInfo@@@Z 00402370 f   authagentservertable.obj
 0001:000013a0       ?GetInstance@CAuthAgentServerTable@@SAAAV1@XZ 004023a0 f   authagentservertable.obj
 0001:00001400       ?UpdateChannelUserNum@CAuthAgentServerTable@@QAEXPAGG@Z 00402400 f   authagentservertable.obj
 0001:00001460       ??0INET_Addr@@QAE@XZ       00402460 f i authclientdispath.obj
 0001:00001480       ??1CCSLock@@QAE@XZ         00402480 f i authagentservertable.obj
 0001:00001480       ??1CAuthAgentServerTable@@AAE@XZ 00402480 f i authagentservertable.obj
 0001:00001480       ??1CCheckPing@@QAE@XZ      00402480 f i authclientdispath.obj
 0001:00001490       ??1CAuthClientDispatch@@UAE@XZ 00402490 f   authclientdispath.obj
 0001:00001520       ?Connected@CAuthClientDispatch@@UAEXXZ 00402520 f   authclientdispath.obj
 0001:00001560       ?Dispatch@CAuthClientDispatch@@UAE_NXZ 00402560 f   authclientdispath.obj
 0001:00001630       ?ParseServerZone@CAuthClientDispatch@@AAE_NPAUPktSZ@@@Z 00402630 f   authclientdispath.obj
 0001:000017d0       ?ParseSysPatchAddress@CAuthClientDispatch@@AAE_NPAUPktSPI@@@Z 004027d0 f   authclientdispath.obj
 0001:00001810       ?ParseUserLogin@CAuthClientDispatch@@AAE_NPAUPktULi@@@Z 00402810 f   authclientdispath.obj
 0001:000019c0       ?ParseCharSelect@CAuthClientDispatch@@AAE_NPAUPktCS@@@Z 004029c0 f   authclientdispath.obj
 0001:00001c10       ?SetBlockedID@CAuthClientDispatch@@QAEXEQAPBD@Z 00402c10 f   authclientdispath.obj
 0001:00001c60       ?ParseJapanAuthAccount@CAuthClientDispatch@@AAE_NPAUPktJPAU@@@Z 00402c60 f   authclientdispath.obj
 0001:00001f20       ?SendPartyLeaveToDBAgent@@YA_NAAVCSendStream@@KKPBD@Z 00402f20 f   authclientdispath.obj
 0001:00001fa0       ?SendGuildLeaveToDBAgent@@YA_NAAVCSendStream@@KKPBD@Z 00402fa0 f   authclientdispath.obj
 0001:00002030       ??0CAuthClientDispatch@@QAE@AAVCSession@@@Z 00403030 f   authclientdispath.obj
 0001:000020f0       ??_GCAuthClientDispatch@@UAEPAXI@Z 004030f0 f i authclientdispath.obj
 0001:000020f0       ??_ECAuthClientDispatch@@UAEPAXI@Z 004030f0 f i authclientdispath.obj
 0001:00002110       ?GetDispatchTable@CAuthClientDispatch@@SAAAVCMultiDispatch@@XZ 00403110 f   authclientdispath.obj
 0001:00002170       ?UserLogin@CAuthClientDispatch@@QAEXKK@Z 00403170 f   authclientdispath.obj
 0001:000021a0       ?UserLogout@CAuthClientDispatch@@QAEXXZ 004031a0 f   authclientdispath.obj
 0001:000022c0       ?UserMove@CAuthClientDispatch@@QAEXXZ 004032c0 f   authclientdispath.obj
 0001:000023b0       ?ParseAuthAccount@CAuthClientDispatch@@AAE_NPAUPktAU@@@Z 004033b0 f   authclientdispath.obj
 0001:000026b0       ?ParseCharCreate@CAuthClientDispatch@@AAE_NPAUPktCC@@@Z 004036b0 f   authclientdispath.obj
 0001:000029c0       ?ParseCharDelete@CAuthClientDispatch@@AAE_NPAUPktCD@@@Z 004039c0 f   authclientdispath.obj
 0001:00002bd0       ?Disconnected@CAuthClientDispatch@@UAEXXZ 00403bd0 f   authclientdispath.obj
 0001:00002c10       ?DispatchPacket@CAuthClientDispatch@@EAE_NPAUPktBase@@@Z 00403c10 f   authclientdispath.obj
 0001:00002d70       ?SendCharSelect@CAuthClientDispatch@@SA_NAAVCSendStream@@EPAGG@Z 00403d70 f   authclientsend.obj
 0001:00002dc0       ?SendCharCreate@CAuthClientDispatch@@SA_NAAVCSendStream@@KKPAUCHAR_VIEW@@G@Z 00403dc0 f   authclientsend.obj
 0001:00002e20       ?SendCharDelete@CAuthClientDispatch@@SA_NAAVCSendStream@@KKG@Z 00403e20 f   authclientsend.obj
 0001:00002e80       ??_ECThread@@UAEPAXI@Z     00403e80 f i authorizethread.obj
 0001:00002e80       ??_GCThread@@UAEPAXI@Z     00403e80 f i authorizethread.obj
 0001:00002ea0       ?Initialize@CAuthorizeThread@@QAE_NXZ 00403ea0 f   authorizethread.obj
 0001:00002f80       ?End@CAuthorizeThread@@EAEHXZ 00403f80 f   authorizethread.obj
 0001:00002fa0       ?CheckUserIDAndPass@CAuthorizeThread@@SA_NPBD0@Z 00403fa0 f   authorizethread.obj
 0001:000030d0       ?Authorize@CYouxilandAuthorizeThread@@EAEXPAVCAuthInfo@@@Z 004040d0 f   authorizethread.obj
 0001:000032f0       ?Authorize@CJapanAuthorizeThread@@EAEXPAVCAuthInfo@@@Z 004042f0 f   authorizethread.obj
 0001:00003330       ??1CAuthorizeThread@@UAE@XZ 00404330 f   authorizethread.obj
 0001:000033a0       ?Run@CAuthorizeThread@@EAEIXZ 004043a0 f   authorizethread.obj
 0001:00003460       ?GetInstance@?$CStaticSingleton@VCMasterPassword@@@@SAAAVCMasterPassword@@XZ 00404460 f i authorizethread.obj
 0001:000034c0       ??_ECAuthorizeThread@@UAEPAXI@Z 004044c0 f i authorizethread.obj
 0001:000034c0       ??_GCAuthorizeThread@@UAEPAXI@Z 004044c0 f i authorizethread.obj
 0001:000034e0       ?Create@CAuthorizeThread@@SAPAV1@XZ 004044e0 f   authorizethread.obj
 0001:000035a0       ??_ECJapanAuthorizeThread@@UAEPAXI@Z 004045a0 f i authorizethread.obj
 0001:000035a0       ??_GCYouxilandAuthorizeThread@@UAEPAXI@Z 004045a0 f i authorizethread.obj
 0001:000035a0       ??_GCJapanAuthorizeThread@@UAEPAXI@Z 004045a0 f i authorizethread.obj
 0001:000035a0       ??_ECHangameAuthorizeThread@@UAEPAXI@Z 004045a0 f i authorizethread.obj
 0001:000035a0       ??_GCHangameAuthorizeThread@@UAEPAXI@Z 004045a0 f i authorizethread.obj
 0001:000035a0       ??_ECYouxilandAuthorizeThread@@UAEPAXI@Z 004045a0 f i authorizethread.obj
 0001:000035c0       ??1CHangameAuthorizeThread@@UAE@XZ 004045c0 f i authorizethread.obj
 0001:000035c0       ??1CJapanAuthorizeThread@@UAE@XZ 004045c0 f i authorizethread.obj
 0001:000035c0       ??1CYouxilandAuthorizeThread@@UAE@XZ 004045c0 f i authorizethread.obj
 0001:000035d0       ?Authorize@CHangameAuthorizeThread@@EAEXPAVCAuthInfo@@@Z 004045d0 f   authorizethread.obj
 0001:00003a20       ??1CAuthInfo@@QAE@XZ       00404a20 f   authorizeuser.obj
 0001:00003a30       ?Initialize@CAuthorizeUser@@QAE_NKK@Z 00404a30 f   authorizeuser.obj
 0001:00003a70       ?stop@CSyncronizedObjectQueue@@QAEXXZ 00404a70 f   authorizeuser.obj
 0001:00003aa0       ?is_stopped@CSyncronizedObjectQueue@@QAE_NXZ 00404aa0 f   authorizeuser.obj
 0001:00003ac0       ??0CAuthInfo@@QAE@PAVCAuthClientDispatch@@KPBD1IIGG@Z 00404ac0 f   authorizeuser.obj
 0001:00003b70       ?_Tidy@?$basic_string@DU?$char_traits@D@std@@V?$allocator@D@2@@std@@IAEX_NI@Z 00404b70 f i authorizeuser.obj
 0001:00003bd0       ?_Buynode@?$list@PAVCAuthInfo@@V?$allocator@PAVCAuthInfo@@@std@@@std@@IAEPAU_Node@?$_List_nod@PAVCAuthInfo@@V?$allocator@PAVCAuthInfo@@@std@@@2@XZ 00404bd0 f i authorizeuser.obj
 0001:00003bd0       ?_Buynode@?$list@PAVCListener@@V?$allocator@PAVCListener@@@std@@@std@@IAEPAU_Node@?$_List_nod@PAVCListener@@V?$allocator@PAVCListener@@@std@@@2@XZ 00404bd0 f i rylgamelibrary:iocpnet.obj
 0001:00003bd0       ?_Buynode@?$list@PAVCSession@@V?$allocator@PAVCSession@@@std@@@std@@IAEPAU_Node@?$_List_nod@PAVCSession@@V?$allocator@PAVCSession@@@std@@@2@XZ 00404bd0 f i rylgamelibrary:sessionmgr.obj
 0001:00003bd0       ?_Buynode@?$list@PAVCThread@@V?$allocator@PAVCThread@@@std@@@std@@IAEPAU_Node@?$_List_nod@PAVCThread@@V?$allocator@PAVCThread@@@std@@@2@XZ 00404bd0 f i rylgamelibrary:serverwindowframework.obj
 0001:00003bd0       ?_Buynode@?$list@PAVCCommand@@V?$allocator@PAVCCommand@@@std@@@std@@IAEPAU_Node@?$_List_nod@PAVCCommand@@V?$allocator@PAVCCommand@@@std@@@2@XZ 00404bd0 f i rylgamelibrary:command.obj
 0001:00003bd0       ?_Buynode@?$list@PAULogBuffer@@V?$allocator@PAULogBuffer@@@std@@@std@@IAEPAU_Node@?$_List_nod@PAULogBuffer@@V?$allocator@PAULogBuffer@@@std@@@2@XZ 00404bd0 f i rylgamelibrary:gamelog.obj
 0001:00003bd0       ?_Buynode@?$list@PAVIOPCode@@V?$allocator@PAVIOPCode@@@std@@@std@@IAEPAU_Node@?$_List_nod@PAVIOPCode@@V?$allocator@PAVIOPCode@@@std@@@2@XZ 00404bd0 f i rylgamelibrary:intermediatecode.obj
 0001:00003bf0       ?erase@?$basic_string@DU?$char_traits@D@std@@V?$allocator@D@2@@std@@QAEAAV12@II@Z 00404bf0 f i authorizeuser.obj
 0001:00003c70       ?_Buynode@?$list@PAVCSession@@V?$allocator@PAVCSession@@@std@@@std@@IAEPAU_Node@?$_List_nod@PAVCSession@@V?$allocator@PAVCSession@@@std@@@2@PAU342@0ABQAVCSession@@@Z 00404c70 f i rylgamelibrary:sessionmgr.obj
 0001:00003c70       ?_Buynode@?$list@PAULogBuffer@@V?$allocator@PAULogBuffer@@@std@@@std@@IAEPAU_Node@?$_List_nod@PAULogBuffer@@V?$allocator@PAULogBuffer@@@std@@@2@PAU342@0ABQAULogBuffer@@@Z 00404c70 f i rylgamelibrary:gamelog.obj
 0001:00003c70       ?_Buynode@?$list@PAVIOPCode@@V?$allocator@PAVIOPCode@@@std@@@std@@IAEPAU_Node@?$_List_nod@PAVIOPCode@@V?$allocator@PAVIOPCode@@@std@@@2@PAU342@0ABQAVIOPCode@@@Z 00404c70 f i rylgamelibrary:imcodegen.obj
 0001:00003c70       ?_Buynode@?$list@PAVCCommand@@V?$allocator@PAVCCommand@@@std@@@std@@IAEPAU_Node@?$_List_nod@PAVCCommand@@V?$allocator@PAVCCommand@@@std@@@2@PAU342@0ABQAVCCommand@@@Z 00404c70 f i rylauthserver.obj
 0001:00003c70       ?_Buynode@?$list@PAVCAuthInfo@@V?$allocator@PAVCAuthInfo@@@std@@@std@@IAEPAU_Node@?$_List_nod@PAVCAuthInfo@@V?$allocator@PAVCAuthInfo@@@std@@@2@PAU342@0ABQAVCAuthInfo@@@Z 00404c70 f i authorizeuser.obj
 0001:00003c70       ?_Buynode@?$list@PAVCListener@@V?$allocator@PAVCListener@@@std@@@std@@IAEPAU_Node@?$_List_nod@PAVCListener@@V?$allocator@PAVCListener@@@std@@@2@PAU342@0ABQAVCListener@@@Z 00404c70 f i rylgamelibrary:iocpnet.obj
 0001:00003c70       ?_Buynode@?$list@PAVCThread@@V?$allocator@PAVCThread@@@std@@@std@@IAEPAU_Node@?$_List_nod@PAVCThread@@V?$allocator@PAVCThread@@@std@@@2@PAU342@0ABQAVCThread@@@Z 00404c70 f i rylgamelibrary:serverwindowframework.obj
 0001:00003ca0       ?_Copy@?$basic_string@DU?$char_traits@D@std@@V?$allocator@D@2@@std@@IAEXII@Z 00404ca0 f i authorizeuser.obj
 0001:00003de0       ?remove@CSyncronizedObjectQueue@@QAEXPBD@Z 00404de0 f   authorizeuser.obj
 0001:00003eb0       ?clear@CSyncronizedObjectQueue@@QAEXXZ 00404eb0 f   authorizeuser.obj
 0001:00003f60       ?RemovePending@CAuthorizeUser@@QAEXPBD@Z 00404f60 f   authorizeuser.obj
 0001:00003f70       ??1?$basic_string@DU?$char_traits@D@std@@V?$allocator@D@2@@std@@QAE@XZ 00404f70 f i authorizeuser.obj
 0001:00003fa0       ?pop_front@?$list@PAVCAuthInfo@@V?$allocator@PAVCAuthInfo@@@std@@@std@@QAEXXZ 00404fa0 f i authorizeuser.obj
 0001:00003fd0       ?pop_back@?$list@PAVCAuthInfo@@V?$allocator@PAVCAuthInfo@@@std@@@std@@QAEXXZ 00404fd0 f i authorizeuser.obj
 0001:00004000       ?what@logic_error@std@@UBEPBDXZ 00405000 f i authorizeuser.obj
 0001:00004010       ??1CSyncronizedObjectQueue@@QAE@XZ 00405010 f   authorizeuser.obj
 0001:00004090       ?dequeue@CSyncronizedObjectQueue@@QAEPAVCAuthInfo@@K@Z 00405090 f   authorizeuser.obj
 0001:00004130       ??1CAuthorizeUser@@AAE@XZ  00405130 f   authorizeuser.obj
 0001:000041b0       ?GetAuthorizeInfo@CAuthorizeUser@@QAEPAVCAuthInfo@@K@Z 004051b0 f   authorizeuser.obj
 0001:000041c0       ?assign@?$basic_string@DU?$char_traits@D@std@@V?$allocator@D@2@@std@@QAEAAV12@ABV12@II@Z 004051c0 f i authorizeuser.obj
 0001:000042b0       ?assign@?$basic_string@DU?$char_traits@D@std@@V?$allocator@D@2@@std@@QAEAAV12@PBDI@Z 004052b0 f i authorizeuser.obj
 0001:000043a0       ??0CSyncronizedObjectQueue@@QAE@XZ 004053a0 f   authorizeuser.obj
 0001:00004430       ??0?$basic_string@DU?$char_traits@D@std@@V?$allocator@D@2@@std@@QAE@ABV01@@Z 00405430 f i authorizeuser.obj
 0001:00004460       ?assign@?$basic_string@DU?$char_traits@D@std@@V?$allocator@D@2@@std@@QAEAAV12@PBD@Z 00405460 f i authorizeuser.obj
 0001:00004490       ??0logic_error@std@@QAE@ABV?$basic_string@DU?$char_traits@D@std@@V?$allocator@D@2@@1@@Z 00405490 f i authorizeuser.obj
 0001:000044f0       ??_Elength_error@std@@UAEPAXI@Z 004054f0 f i authorizeuser.obj
 0001:000044f0       ??_Gout_of_range@std@@UAEPAXI@Z 004054f0 f i rylgamelibrary:serverrequest.obj
 0001:000044f0       ??_Glength_error@std@@UAEPAXI@Z 004054f0 f i authorizeuser.obj
 0001:000044f0       ??_Eout_of_range@std@@UAEPAXI@Z 004054f0 f i rylgamelibrary:serverrequest.obj
 0001:000044f0       ??_Glogic_error@std@@UAEPAXI@Z 004054f0 f i authorizeuser.obj
 0001:000044f0       ??_Elogic_error@std@@UAEPAXI@Z 004054f0 f i authorizeuser.obj
 0001:00004510       ??1out_of_range@std@@UAE@XZ 00405510 f i rylgamelibrary:serverrequest.obj
 0001:00004510       ??1length_error@std@@UAE@XZ 00405510 f i authorizeuser.obj
 0001:00004510       ??1logic_error@std@@UAE@XZ 00405510 f i authorizeuser.obj
 0001:00004550       ?GetInstance@CAuthorizeUser@@SAAAV1@XZ 00405550 f   authorizeuser.obj
 0001:000045c0       ??0?$basic_string@DU?$char_traits@D@std@@V?$allocator@D@2@@std@@QAE@PBD@Z 004055c0 f i authorizeuser.obj
 0001:00004600       ?_Incsize@?$list@PAVCAuthInfo@@V?$allocator@PAVCAuthInfo@@@std@@@std@@IAEXI@Z 00405600 f i authorizeuser.obj
 0001:000046a0       ??0logic_error@std@@QAE@ABV01@@Z 004056a0 f i authorizeuser.obj
 0001:00004710       ??0length_error@std@@QAE@ABV01@@Z 00405710 f i authorizeuser.obj
 0001:00004730       ?push_front@?$list@PAVCAuthInfo@@V?$allocator@PAVCAuthInfo@@@std@@@std@@QAEXABQAVCAuthInfo@@@Z 00405730 f i authorizeuser.obj
 0001:00004770       ?push_back@?$list@PAVCAuthInfo@@V?$allocator@PAVCAuthInfo@@@std@@@std@@QAEXABQAVCAuthInfo@@@Z 00405770 f i authorizeuser.obj
 0001:000047b0       ?enqueue@CSyncronizedObjectQueue@@QAE_NPAVCAuthInfo@@_N@Z 004057b0 f   authorizeuser.obj
 0001:000048a0       ?AddAuthorizeUser@CAuthorizeUser@@QAE_NPAVCAuthInfo@@@Z 004058a0 f   authorizeuser.obj
 0001:000048b0       ??1CItemCreator@@QAE@XZ    004058b0 f i itemcreator.obj
 0001:000048d0       ??0CItemCreator@@AAE@XZ    004058d0 f   itemcreator.obj
 0001:000048f0       ?Initialize@CItemCreator@@QAE_NXZ 004058f0 f   itemcreator.obj
 0001:00004950       ?SetUID@CItemCreator@@QAEX_K@Z 00405950 f   itemcreator.obj
 0001:00004990       ?Create@CItemCreator@@QAEPAVCItem@Item@@G@Z 00405990 f   itemcreator.obj
 0001:000049f0       ??$_Ucopy@PAH@?$vector@HV?$allocator@H@std@@@std@@IAEPAHPAH00@Z 004059f0 f i rylgamelibrary:reloctable.obj
 0001:000049f0       ??$_Ucopy@PAPAD@?$vector@PADV?$allocator@PAD@std@@@std@@IAEPAPADPAPAD00@Z 004059f0 f i rylgamelibrary:tokenlizedfile.obj
 0001:000049f0       ??$_Ucopy@PAK@?$vector@KV?$allocator@K@std@@@std@@IAEPAKPAK00@Z 004059f0 f i masterpassword.obj
 0001:000049f0       ??$_Ucopy@PAPAV?$pool@Udefault_user_allocator_new_delete@boost@@@boost@@@?$vector@PAV?$pool@Udefault_user_allocator_new_delete@boost@@@boost@@V?$allocator@PAV?$pool@Udefault_user_allocator_new_delete@boost@@@boost@@@std@@@std@@IAEPAPAV?$pool@Udefault_user_allocator_new_delete@boost@@@boost@@PAPAV23@00@Z 004059f0 f i rylgamelibrary:bufferfactory.obj
 0001:00004a20       ?CheckMasterPassword@CMasterPassword@@QAE_NPBD0ABUsockaddr_in@@@Z 00405a20 f   masterpassword.obj
 0001:00004b70       ??1CMasterPassword@@QAE@XZ 00405b70 f   masterpassword.obj
 0001:00004bb0       ?Init@CMasterPassword@@AAEXXZ 00405bb0 f   masterpassword.obj
 0001:00004c10       ?_Xlen@?$vector@KV?$allocator@K@std@@@std@@IBEXXZ 00405c10 f i masterpassword.obj
 0001:00004c80       ?_Insert_n@?$vector@KV?$allocator@K@std@@@std@@IAEXViterator@12@IABK@Z 00405c80 f i masterpassword.obj
 0001:00004e60       ??0CMasterPassword@@QAE@XZ 00405e60 f   masterpassword.obj
 0001:00004eb0       ?push_back@?$vector@KV?$allocator@K@std@@@std@@QAEXABK@Z 00405eb0 f i masterpassword.obj
 0001:00004f00       ?Process@CMasterPassword@@AAEXPBD0@Z 00405f00 f   masterpassword.obj
 0001:00004fb0       ?LoadMasterPassword@CMasterPassword@@QAE_NPBD@Z 00405fb0 f   masterpassword.obj
 0001:000050c0       ??0CRylAuthServerProcess@@QAE@AAVCRylAuthServer@@K@Z 004060c0 f i rylauthserver.obj
 0001:000050f0       ?End@CProcessThread@@EAEHXZ 004060f0 f i rylauthserver.obj
 0001:00005110       ??_GCRylAuthServerProcess@@UAEPAXI@Z 00406110 f i rylauthserver.obj
 0001:00005110       ??_ECRylAuthServerProcess@@UAEPAXI@Z 00406110 f i rylauthserver.obj
 0001:00005130       ??1CRylAuthServerProcess@@UAE@XZ 00406130 f i rylauthserver.obj
 0001:00005190       ??0CRylAuthServer@@AAE@XZ  00406190 f   rylauthserver.obj
 0001:00005210       ??1CRylAuthServer@@EAE@XZ  00406210 f   rylauthserver.obj
 0001:000052a0       ?PrintStatistics@CRylAuthServer@@QAEXXZ 004062a0 f   rylauthserver.obj
 0001:00005310       ?ReloadSetup@CRylAuthServer@@QAEXXZ 00406310 f   rylauthserver.obj
 0001:00005370       ??_ECRylAuthServer@@EAEPAXI@Z 00406370 f i rylauthserver.obj
 0001:00005370       ??_GCRylAuthServer@@EAEPAXI@Z 00406370 f i rylauthserver.obj
 0001:00005390       ?PrintServerInfo@CRylAuthServer@@QAEXXZ 00406390 f   rylauthserver.obj
 0001:000054f0       ?GetInstance@CRylAuthServer@@SAAAV1@XZ 004064f0 f   rylauthserver.obj
 0001:00005550       ?InternalRun@CRylAuthServerProcess@@UAEXAAVCPulse@@@Z 00406550 f i rylauthserver.obj
 0001:00005600       ?purge_memory@?$pool@Udefault_user_allocator_new_delete@boost@@@boost@@QAE_NXZ 00406600 f i rylauthserver.obj
 0001:00005640       ?CreateDispatch@?$CPoolDispatchFactory@VCAuthClientDispatch@@@@UAEPAVCPacketDispatch@@AAVCSession@@@Z 00406640 f i rylauthserver.obj
 0001:000056b0       ?malloc_need_resize@?$pool@Udefault_user_allocator_new_delete@boost@@@boost@@AAEPAXXZ 004066b0 f i rylauthserver.obj
 0001:00005750       ?alloc_size@?$pool@Udefault_user_allocator_new_delete@boost@@@boost@@IBEIXZ 00406750 f i rylauthserver.obj
 0001:00005780       ?next@?$PODptr@I@details@boost@@QBEXABV123@@Z 00406780 f i rylauthserver.obj
 0001:000057b0       ?DeleteDispatch@?$CPoolDispatchFactory@VCAuthAgentDispatch@@@@UAEXPAVCPacketDispatch@@@Z 004067b0 f i rylauthserver.obj
 0001:000057b0       ?DeleteDispatch@?$CPoolDispatchFactory@VCAuthClientDispatch@@@@UAEXPAVCPacketDispatch@@@Z 004067b0 f i rylauthserver.obj
 0001:000057d0       ?CreateDispatch@?$CPoolDispatchFactory@VCAuthAgentDispatch@@@@UAEPAVCPacketDispatch@@AAVCSession@@@Z 004067d0 f i rylauthserver.obj
 0001:00005840       ??_G?$CPoolDispatchFactory@VCAuthClientDispatch@@@@UAEPAXI@Z 00406840 f i rylauthserver.obj
 0001:00005840       ??_E?$CPoolDispatchFactory@VCAuthClientDispatch@@@@UAEPAXI@Z 00406840 f i rylauthserver.obj
 0001:00005860       ??1?$CPoolDispatchFactory@VCAuthClientDispatch@@@@UAE@XZ 00406860 f i rylauthserver.obj
 0001:00005880       ??_G?$CPoolDispatchFactory@VCAuthAgentDispatch@@@@UAEPAXI@Z 00406880 f i rylauthserver.obj
 0001:00005880       ??_E?$CPoolDispatchFactory@VCAuthAgentDispatch@@@@UAEPAXI@Z 00406880 f i rylauthserver.obj
 0001:000058a0       ??1?$CPoolDispatchFactory@VCAuthAgentDispatch@@@@UAE@XZ 004068a0 f i rylauthserver.obj
 0001:000058c0       ?_Incsize@?$list@PAVCCommand@@V?$allocator@PAVCCommand@@@std@@@std@@IAEXI@Z 004068c0 f i rylauthserver.obj
 0001:00005960       ??$Create@VCTCPFactory@@VCPoolBufferFactory@@V?$CPoolDispatchFactory@VCAuthClientDispatch@@@@VCStreamOverlappedFactory@@@CSessionPolicy@@SAPAV0@XZ 00406960 f i rylauthserver.obj
 0001:00005ab0       ??$Create@VCTCPFactory@@VCPoolBufferFactory@@V?$CPoolDispatchFactory@VCAuthAgentDispatch@@@@VCStreamOverlappedFactory@@@CSessionPolicy@@SAPAV0@XZ 00406ab0 f i rylauthserver.obj
 0001:00005c00       ?InitializeClientListener@CRylAuthServer@@QAEXXZ 00406c00 f   rylauthserver.obj
 0001:00005c90       ?ConnectToDBAgent@CRylAuthServer@@QAEXXZ 00406c90 f   rylauthserver.obj
 0001:00005da0       ?Add@CCommandProcess@@QAEXPAVCCommand@@@Z 00406da0 f i rylauthserver.obj
 0001:00005e20       ?ApplicationSpecificInit@CRylAuthServer@@EAE_NPBD@Z 00406e20 f   rylauthserver.obj
 0001:00005fd0       ?do_always_noconv@codecvt_base@std@@MBE_NXZ 00406fd0 f i rylgamelibrary:regfunctions.obj
 0001:00005fd0       ?Destroy@?$CConsoleCMDSingleton@VCCMDStatLog@@@@UAE_NXZ 00406fd0 f i rylauthservercommands.obj
 0001:00005fd0       ?Destroy@?$CConsoleCMDSingleton@VCCMDPrintLog@@@@UAE_NXZ 00406fd0 f i rylauthservercommands.obj
 0001:00005fd0       ?Destroy@?$CConsoleCMDSingleton@VCCMDShowStatistics@@@@UAE_NXZ 00406fd0 f i rylauthservercommands.obj
 0001:00005fd0       ?Destroy@?$CConsoleCMDSingleton@VCCMDStartServer@@@@UAE_NXZ 00406fd0 f i rylauthservercommands.obj
 0001:00005fd0       ?Destroy@?$CConsoleCMDSingleton@VCCMDFlushLog@@@@UAE_NXZ 00406fd0 f i rylauthservercommands.obj
 0001:00005fd0       ?Destroy@?$CConsoleCMDSingleton@VCCMDMasterPass@@@@UAE_NXZ 00406fd0 f i rylauthservercommands.obj
 0001:00005fd0       ?Destroy@?$CConsoleCMDSingleton@VCCMDStatClear@@@@UAE_NXZ 00406fd0 f i rylauthservercommands.obj
 0001:00005fd0       ?Destroy@?$CConsoleCMDSingleton@VCCMDReloadSetup@@@@UAE_NXZ 00406fd0 f i rylauthservercommands.obj
 0001:00005fe0       ?DoProcess@CCMDStartServer@@MAE_NXZ 00406fe0 f i rylauthservercommands.obj
 0001:00006000       ?DoProcess@CCMDShowStatistics@@MAE_NXZ 00407000 f i rylauthservercommands.obj
 0001:00006020       ?DoProcess@CCMDPrintLog@@MAE_NXZ 00407020 f i rylauthservercommands.obj
 0001:00006080       ?DoProcess@CCMDReloadSetup@@MAE_NXZ 00407080 f i rylauthservercommands.obj
 0001:00006090       ?DoProcess@CCMDFlushLog@@MAE_NXZ 00407090 f i rylauthservercommands.obj
 0001:000060e0       ?DoProcess@CCMDMasterPass@@MAE_NXZ 004070e0 f i rylauthservercommands.obj
 0001:00006130       ?DoProcess@CCMDStatClear@@MAE_NXZ 00407130 f i rylauthservercommands.obj
 0001:00006140       ?DoProcess@CCMDStatLog@@MAE_NXZ 00407140 f i rylauthservercommands.obj
 0001:00006150       ?Clone@?$CConsoleCMDSingleton@VCCMDStatClear@@@@UAEPAVCConsoleCommand@@PBDI@Z 00407150 f i rylauthservercommands.obj
 0001:00006180       ?Clone@?$CConsoleCMDSingleton@VCCMDStatLog@@@@UAEPAVCConsoleCommand@@PBDI@Z 00407180 f i rylauthservercommands.obj
 0001:000061b0       ?Clone@?$CConsoleCMDSingleton@VCCMDStartServer@@@@UAEPAVCConsoleCommand@@PBDI@Z 004071b0 f i rylauthservercommands.obj
 0001:000061e0       ?Clone@?$CConsoleCMDSingleton@VCCMDShowStatistics@@@@UAEPAVCConsoleCommand@@PBDI@Z 004071e0 f i rylauthservercommands.obj
 0001:00006210       ?Clone@?$CConsoleCMDSingleton@VCCMDPrintLog@@@@UAEPAVCConsoleCommand@@PBDI@Z 00407210 f i rylauthservercommands.obj
 0001:00006240       ?Clone@?$CConsoleCMDSingleton@VCCMDFlushLog@@@@UAEPAVCConsoleCommand@@PBDI@Z 00407240 f i rylauthservercommands.obj
 0001:00006270       ?Clone@?$CConsoleCMDSingleton@VCCMDReloadSetup@@@@UAEPAVCConsoleCommand@@PBDI@Z 00407270 f i rylauthservercommands.obj
 0001:000062a0       ?Clone@?$CConsoleCMDSingleton@VCCMDMasterPass@@@@UAEPAVCConsoleCommand@@PBDI@Z 004072a0 f i rylauthservercommands.obj
 0001:000062d0       ?InitializeCommand@CRylAuthServer@@AAE_NXZ 004072d0 f   rylauthservercommands.obj
 0001:000064c0       ?ExceptionUserFunc@@YGHPADH@Z 004074c0 f   rylauthservermain.obj
 0001:00006530       _WinMain@16                00407530 f   rylauthservermain.obj
 0001:000065e0       ??RCProcessRYLAUTH_AUTOSTART@@UAEJPAUHWND__@@IIJ@Z 004075e0 f i rylauthserverwindow.obj
 0001:00006620       ??RCProcessAUTH_CONNECTTOAGENT@@UAEJPAUHWND__@@IIJ@Z 00407620 f i rylauthserverwindow.obj
 0001:00006660       ??1CProcessRYLAUTH_QUIT@@UAE@XZ 00407660 f i rylauthserverwindow.obj
 0001:00006660       ??1CSendDataToManageClient@@UAE@XZ 00407660 f i rylgamelibrary:serverwindowframework.obj
 0001:00006660       ??1CProcessCOMMAND@@UAE@XZ 00407660 f i rylauthserverwindow.obj
 0001:00006660       ??1CProcessAUTH_CONNECTTOAGENT@@UAE@XZ 00407660 f i rylauthserverwindow.obj
 0001:00006660       ??1CProcessRYLAUTH_AUTOSTART@@UAE@XZ 00407660 f i rylauthserverwindow.obj
 0001:00006660       ??1CRecvCommandFromManageClient@@UAE@XZ 00407660 f i rylgamelibrary:serverwindowframework.obj
 0001:00006670       ??RCProcessRYLAUTH_QUIT@@UAEJPAUHWND__@@IIJ@Z 00407670 f i rylauthserverwindow.obj
 0001:00006680       ??_ECProcessRYLAUTH_AUTOSTART@@UAEPAXI@Z 00407680 f i rylauthserverwindow.obj
 0001:00006680       ??_GCProcessAUTH_CONNECTTOAGENT@@UAEPAXI@Z 00407680 f i rylauthserverwindow.obj
 0001:00006680       ??_ECProcessAUTH_CONNECTTOAGENT@@UAEPAXI@Z 00407680 f i rylauthserverwindow.obj
 0001:00006680       ??_GCProcessRYLAUTH_QUIT@@UAEPAXI@Z 00407680 f i rylauthserverwindow.obj
 0001:00006680       ??_ECProcessRYLAUTH_QUIT@@UAEPAXI@Z 00407680 f i rylauthserverwindow.obj
 0001:00006680       ??_GCSendDataToManageClient@@UAEPAXI@Z 00407680 f i rylgamelibrary:serverwindowframework.obj
 0001:00006680       ??_ECProcessCOMMAND@@UAEPAXI@Z 00407680 f i rylauthserverwindow.obj
 0001:00006680       ??_GCProcessCOMMAND@@UAEPAXI@Z 00407680 f i rylauthserverwindow.obj
 0001:00006680       ??_GCRecvCommandFromManageClient@@UAEPAXI@Z 00407680 f i rylgamelibrary:serverwindowframework.obj
 0001:00006680       ??_GCProcessRYLAUTH_AUTOSTART@@UAEPAXI@Z 00407680 f i rylauthserverwindow.obj
 0001:00006680       ??_ECSendDataToManageClient@@UAEPAXI@Z 00407680 f i rylgamelibrary:serverwindowframework.obj
 0001:00006680       ??_ECRecvCommandFromManageClient@@UAEPAXI@Z 00407680 f i rylgamelibrary:serverwindowframework.obj
 0001:000066a0       ?InitializeMsgProc@CRylAuthServer@@AAE_NXZ 004076a0 f   rylauthserverwindow.obj
 0001:00006780       ??RCProcessCOMMAND@@UAEJPAUHWND__@@IIJ@Z 00407780 f i rylauthserverwindow.obj
 0001:00006850       ?SendAuthAccount@AuthSendPacket@@YA_NPAVCAuthClientDispatch@@KG@Z 00407850 f   senduserloginout.obj
 0001:000068a0       ?SendUserLogin@AuthSendPacket@@YA_NAAVCSendStream@@KKPAUCHAR_VIEW@@HGEEEG@Z 004078a0 f   senduserloginout.obj
 0001:00006990       ?SendUserLogout@AuthSendPacket@@YA_NKK@Z 00407990 f   senduserloginout.obj
 0001:00006a50       ?SendUserMove@AuthSendPacket@@YA_NKK@Z 00407a50 f   senduserloginout.obj
 0001:00006b10       ?SendServerZone@AuthSendPacket@@YA_NAAVCSendStream@@KAAUsockaddr_in@@G@Z 00407b10 f   senduserloginout.obj
 0001:00006b70       ?set_addr@INET_Addr@@QAEXPBDG@Z 00407b70 f   rylgamelibrary:inet_addr.obj
 0001:00006be0       ?set_addr@INET_Addr@@QAEXABUsockaddr@@H@Z 00407be0 f   rylgamelibrary:inet_addr.obj
 0001:00006c10       ?set_addr@INET_Addr@@QAEXUin_addr@@G@Z 00407c10 f   rylgamelibrary:inet_addr.obj
 0001:00006c60       ??1CPacketDispatch@@UAE@XZ 00407c60 f i rylgamelibrary:rylserverdispatch.obj
 0001:00006c70       ??_ECPacketDispatch@@UAEPAXI@Z 00407c70 f i rylgamelibrary:rylserverdispatch.obj
 0001:00006c70       ??_GCPacketDispatch@@UAEPAXI@Z 00407c70 f i rylgamelibrary:rylserverdispatch.obj
 0001:00006c90       ??0CRylServerDispatch@@IAE@AAVCSession@@K@Z 00407c90 f   rylgamelibrary:rylserverdispatch.obj
 0001:00006d10       ?GetRemoteAddr@CRylServerDispatch@@QAEAAVINET_Addr@@XZ 00407d10 f   rylgamelibrary:rylserverdispatch.obj
 0001:00006d20       ?Shutdown@CRylServerDispatch@@QAE_NXZ 00407d20 f   rylgamelibrary:rylserverdispatch.obj
 0001:00006d30       ?LogErrorPacket@CRylServerDispatch@@QAEXPBDE@Z 00407d30 f   rylgamelibrary:rylserverdispatch.obj
 0001:00006d80       ?LogErrorPacketCreation@CRylServerDispatch@@QAEXW4CreationResult@1@@Z 00407d80 f   rylgamelibrary:rylserverdispatch.obj
 0001:00006df0       ??$greator_second@U?$pair@KK@std@@@@YA_NABU?$pair@KK@std@@0@Z 00407df0 f i rylgamelibrary:rylserverdispatch.obj
 0001:00006e10       ??$fill@PAU?$pair@W4eStdFunc@@H@std@@U12@@std@@YAXPAU?$pair@W4eStdFunc@@H@0@0ABU10@@Z 00407e10 f i rylgamelibrary:reloctable.obj
 0001:00006e10       ??$fill@PAUParseData@ItemDataParser@@U12@@std@@YAXPAUParseData@ItemDataParser@@0ABU12@@Z 00407e10 f i rylgamelibrary:itemdataparser.obj
 0001:00006e10       ??$fill@PAU?$pair@KK@std@@U12@@std@@YAXPAU?$pair@KK@0@0ABU10@@Z 00407e10 f i rylgamelibrary:rylserverdispatch.obj
 0001:00006e40       ??1CRylServerDispatch@@MAE@XZ 00407e40 f   rylgamelibrary:rylserverdispatch.obj
 0001:00006ed0       ?CreatePacket@CRylServerDispatch@@SA?AW4CreationResult@1@AAVCBufferFactory@@AAVCBufferQueue@@QADPAK@Z 00407ed0 f   rylgamelibrary:rylserverdispatch.obj
 0001:000070a0       ?ParsePacket@CRylServerDispatch@@UAE_NQADPAK@Z 004080a0 f   rylgamelibrary:rylserverdispatch.obj
 0001:00007170       ?Dispatch@CRylServerDispatch@@MAE_NXZ 00408170 f   rylgamelibrary:rylserverdispatch.obj
 0001:00007350       ??$_Uninit_copy@Viterator@?$vector@UParseData@ItemDataParser@@V?$allocator@UParseData@ItemDataParser@@@std@@@std@@PAUParseData@ItemDataParser@@V?$allocator@UParseData@ItemDataParser@@@3@@std@@YAPAUParseData@ItemDataParser@@Viterator@?$vector@UParseData@ItemDataParser@@V?$allocator@UParseData@ItemDataParser@@@std@@@0@0PAU12@AAV?$allocator@UParseData@ItemDataParser@@@0@U_Nonscalar_ptr_iterator_tag@0@@Z 00408350 f i rylgamelibrary:itemdataparser.obj
 0001:00007350       ??$_Uninit_copy@PAU?$pair@KK@std@@PAU12@V?$allocator@U?$pair@KK@std@@@2@@std@@YAPAU?$pair@KK@0@PAU10@00AAV?$allocator@U?$pair@KK@std@@@0@U_Nonscalar_ptr_iterator_tag@0@@Z 00408350 f i rylgamelibrary:rylserverdispatch.obj
 0001:00007350       ??$_Uninit_copy@Viterator@?$vector@U?$pair@KK@std@@V?$allocator@U?$pair@KK@std@@@2@@std@@PAU?$pair@KK@3@V?$allocator@U?$pair@KK@std@@@3@@std@@YAPAU?$pair@KK@0@Viterator@?$vector@U?$pair@KK@std@@V?$allocator@U?$pair@KK@std@@@2@@0@0PAU10@AAV?$allocator@U?$pair@KK@std@@@0@U_Nonscalar_ptr_iterator_tag@0@@Z 00408350 f i rylgamelibrary:rylserverdispatch.obj
 0001:00007350       ??$_Uninit_copy@PAU?$pair@W4eStdFunc@@H@std@@PAU12@V?$allocator@U?$pair@W4eStdFunc@@H@std@@@2@@std@@YAPAU?$pair@W4eStdFunc@@H@0@PAU10@00AAV?$allocator@U?$pair@W4eStdFunc@@H@std@@@0@U_Nonscalar_ptr_iterator_tag@0@@Z 00408350 f i rylgamelibrary:reloctable.obj
 0001:00007350       ??$_Uninit_copy@PAUParseData@ItemDataParser@@PAU12@V?$allocator@UParseData@ItemDataParser@@@std@@@std@@YAPAUParseData@ItemDataParser@@PAU12@00AAV?$allocator@UParseData@ItemDataParser@@@0@U_Nonscalar_ptr_iterator_tag@0@@Z 00408350 f i rylgamelibrary:itemdataparser.obj
 0001:00007380       ??$_Push_heap@Viterator@?$vector@U?$pair@KK@std@@V?$allocator@U?$pair@KK@std@@@2@@std@@HU?$pair@KK@3@P6A_NABU43@0@Z@std@@YAXViterator@?$vector@U?$pair@KK@std@@V?$allocator@U?$pair@KK@std@@@2@@0@HHU?$pair@KK@0@P6A_NABU30@2@Z@Z 00408380 f i rylgamelibrary:rylserverdispatch.obj
 0001:000073f0       ??$_Rotate@Viterator@?$vector@U?$pair@KK@std@@V?$allocator@U?$pair@KK@std@@@2@@std@@HU?$pair@KK@3@@std@@YAXViterator@?$vector@U?$pair@KK@std@@V?$allocator@U?$pair@KK@std@@@2@@0@00PAHPAU?$pair@KK@0@@Z 004083f0 f i rylgamelibrary:rylserverdispatch.obj
 0001:000074d0       ??_ECRylServerDispatch@@MAEPAXI@Z 004084d0 f i rylgamelibrary:rylserverdispatch.obj
 0001:000074d0       ??_GCRylServerDispatch@@MAEPAXI@Z 004084d0 f i rylgamelibrary:rylserverdispatch.obj
 0001:000074f0       ??$_Adjust_heap@Viterator@?$vector@U?$pair@KK@std@@V?$allocator@U?$pair@KK@std@@@2@@std@@HU?$pair@KK@3@P6A_NABU43@0@Z@std@@YAXViterator@?$vector@U?$pair@KK@std@@V?$allocator@U?$pair@KK@std@@@2@@0@HHU?$pair@KK@0@P6A_NABU30@2@Z@Z 004084f0 f i rylgamelibrary:rylserverdispatch.obj
 0001:00007580       ??$_Make_heap@Viterator@?$vector@U?$pair@KK@std@@V?$allocator@U?$pair@KK@std@@@2@@std@@HU?$pair@KK@3@P6A_NABU43@0@Z@std@@YAXViterator@?$vector@U?$pair@KK@std@@V?$allocator@U?$pair@KK@std@@@2@@0@0P6A_NABU?$pair@KK@0@1@ZPAHPAU30@@Z 00408580 f i rylgamelibrary:rylserverdispatch.obj
 0001:000075d0       ??$_Med3@Viterator@?$vector@U?$pair@KK@std@@V?$allocator@U?$pair@KK@std@@@2@@std@@P6A_NABU?$pair@KK@3@0@Z@std@@YAXViterator@?$vector@U?$pair@KK@std@@V?$allocator@U?$pair@KK@std@@@2@@0@00P6A_NABU?$pair@KK@0@1@Z@Z 004085d0 f i rylgamelibrary:rylserverdispatch.obj
 0001:00007650       ??$_Insertion_sort@Viterator@?$vector@U?$pair@KK@std@@V?$allocator@U?$pair@KK@std@@@2@@std@@P6A_NABU?$pair@KK@3@0@Z@std@@YAXViterator@?$vector@U?$pair@KK@std@@V?$allocator@U?$pair@KK@std@@@2@@0@0P6A_NABU?$pair@KK@0@1@Z@Z 00408650 f i rylgamelibrary:rylserverdispatch.obj
 0001:000076f0       ??$_Median@Viterator@?$vector@U?$pair@KK@std@@V?$allocator@U?$pair@KK@std@@@2@@std@@P6A_NABU?$pair@KK@3@0@Z@std@@YAXViterator@?$vector@U?$pair@KK@std@@V?$allocator@U?$pair@KK@std@@@2@@0@00P6A_NABU?$pair@KK@0@1@Z@Z 004086f0 f i rylgamelibrary:rylserverdispatch.obj
 0001:00007790       ??$_Unguarded_partition@Viterator@?$vector@U?$pair@KK@std@@V?$allocator@U?$pair@KK@std@@@2@@std@@P6A_NABU?$pair@KK@3@0@Z@std@@YA?AU?$pair@Viterator@?$vector@U?$pair@KK@std@@V?$allocator@U?$pair@KK@std@@@2@@std@@V123@@0@Viterator@?$vector@U?$pair@KK@std@@V?$allocator@U?$pair@KK@std@@@2@@0@0P6A_NABU?$pair@KK@0@1@Z@Z 00408790 f i rylgamelibrary:rylserverdispatch.obj
 0001:000079a0       ??$sort_heap@Viterator@?$vector@U?$pair@KK@std@@V?$allocator@U?$pair@KK@std@@@2@@std@@P6A_NABU?$pair@KK@3@0@Z@std@@YAXViterator@?$vector@U?$pair@KK@std@@V?$allocator@U?$pair@KK@std@@@2@@0@0P6A_NABU?$pair@KK@0@1@Z@Z 004089a0 f i rylgamelibrary:rylserverdispatch.obj
 0001:00007a00       ??$_Sort@Viterator@?$vector@U?$pair@KK@std@@V?$allocator@U?$pair@KK@std@@@2@@std@@HP6A_NABU?$pair@KK@3@0@Z@std@@YAXViterator@?$vector@U?$pair@KK@std@@V?$allocator@U?$pair@KK@std@@@2@@0@0HP6A_NABU?$pair@KK@0@1@Z@Z 00408a00 f i rylgamelibrary:rylserverdispatch.obj
 0001:00007af0       ?_Xlen@?$vector@U?$pair@KK@std@@V?$allocator@U?$pair@KK@std@@@2@@std@@IBEXXZ 00408af0 f i rylgamelibrary:rylserverdispatch.obj
 0001:00007b60       ?_Insert_n@?$vector@U?$pair@KK@std@@V?$allocator@U?$pair@KK@std@@@2@@std@@IAEXViterator@12@IABU?$pair@KK@2@@Z 00408b60 f i rylgamelibrary:rylserverdispatch.obj
 0001:00007db0       ?reserve@?$vector@U?$pair@KK@std@@V?$allocator@U?$pair@KK@std@@@2@@std@@QAEXI@Z 00408db0 f i rylgamelibrary:rylserverdispatch.obj
 0001:00007e80       ?ProcessTooManyPacket@CRylServerDispatch@@MAEXAAVCBufferQueue@@@Z 00408e80 f   rylgamelibrary:rylserverdispatch.obj
 0001:00008070       ??0CServerLog@@QAE@PBD0@Z  00409070 f   rylgamelibrary:serverlog.obj
 0001:00008160       ?CreateLogFile@CServerLog@@IAEPAXXZ 00409160 f   rylgamelibrary:serverlog.obj
 0001:00008290       ?InternalFlush@CServerLog@@IAEXXZ 00409290 f   rylgamelibrary:serverlog.obj
 0001:00008300       ?SimpleLog@CServerLog@@QAAXW4LOG_TYPE@@PBDZZ 00409300 f   rylgamelibrary:serverlog.obj
 0001:00008450       ?DetailLog@CServerLog@@QAAXW4LOG_TYPE@@PBD1H1ZZ 00409450 f   rylgamelibrary:serverlog.obj
 0001:00008590       ??1CServerLog@@UAE@XZ      00409590 f   rylgamelibrary:serverlog.obj
 0001:00008600       ??_ECServerLog@@UAEPAXI@Z  00409600 f i rylgamelibrary:serverlog.obj
 0001:00008600       ??_GCServerLog@@UAEPAXI@Z  00409600 f i rylgamelibrary:serverlog.obj
 0001:00008620       ??1Result@CServerRequest@@QAE@XZ 00409620 f   rylgamelibrary:serverrequest.obj
 0001:00008640       ?GetSession@Result@CServerRequest@@QAEPAVCSession@@XZ 00409640 f   rylgamelibrary:serverrequest.obj
 0001:00008650       ?_Max@?$_Tree@V?$_Tmap_traits@KURequestInfo@CServerRequest@@U?$less@K@std@@V?$allocator@U?$pair@$$CBKURequestInfo@CServerRequest@@@std@@@4@$0A@@std@@@std@@KAPAU_Node@?$_Tree_nod@V?$_Tmap_traits@KURequestInfo@CServerRequest@@U?$less@K@std@@V?$allocator@U?$pair@$$CBKURequestInfo@CServerRequest@@@std@@@4@$0A@@std@@@2@PAU342@@Z 00409650 f i rylgamelibrary:serverrequest.obj
 0001:00008670       ?_Min@?$_Tree@V?$_Tmap_traits@KURequestInfo@CServerRequest@@U?$less@K@std@@V?$allocator@U?$pair@$$CBKURequestInfo@CServerRequest@@@std@@@4@$0A@@std@@@std@@KAPAU_Node@?$_Tree_nod@V?$_Tmap_traits@KURequestInfo@CServerRequest@@U?$less@K@std@@V?$allocator@U?$pair@$$CBKURequestInfo@CServerRequest@@@std@@@4@$0A@@std@@@2@PAU342@@Z 00409670 f i rylgamelibrary:serverrequest.obj
 0001:00008690       ?_Rrotate@?$_Tree@V?$_Tmap_traits@KURequestInfo@CServerRequest@@U?$less@K@std@@V?$allocator@U?$pair@$$CBKURequestInfo@CServerRequest@@@std@@@4@$0A@@std@@@std@@IAEXPAU_Node@?$_Tree_nod@V?$_Tmap_traits@KURequestInfo@CServerRequest@@U?$less@K@std@@V?$allocator@U?$pair@$$CBKURequestInfo@CServerRequest@@@std@@@4@$0A@@std@@@2@@Z 00409690 f i rylgamelibrary:serverrequest.obj
 0001:000086f0       ?_Inc@const_iterator@?$_Tree@V?$_Tmap_traits@KURequestInfo@CServerRequest@@U?$less@K@std@@V?$allocator@U?$pair@$$CBKURequestInfo@CServerRequest@@@std@@@4@$0A@@std@@@std@@QAEXXZ 004096f0 f i rylgamelibrary:serverrequest.obj
 0001:00008750       ?_Dec@const_iterator@?$_Tree@V?$_Tmap_traits@KURequestInfo@CServerRequest@@U?$less@K@std@@V?$allocator@U?$pair@$$CBKURequestInfo@CServerRequest@@@std@@@4@$0A@@std@@@std@@QAEXXZ 00409750 f i rylgamelibrary:serverrequest.obj
 0001:000087b0       ?RequestOff@CServerRequest@@QAEXXZ 004097b0 f   rylgamelibrary:serverrequest.obj
 0001:000087d0       ?_Lrotate@?$_Tree@V?$_Tmap_traits@KURequestInfo@CServerRequest@@U?$less@K@std@@V?$allocator@U?$pair@$$CBKURequestInfo@CServerRequest@@@std@@@4@$0A@@std@@@std@@IAEXPAU_Node@?$_Tree_nod@V?$_Tmap_traits@KURequestInfo@CServerRequest@@U?$less@K@std@@V?$allocator@U?$pair@$$CBKURequestInfo@CServerRequest@@@std@@@4@$0A@@std@@@2@@Z 004097d0 f i rylgamelibrary:serverrequest.obj
 0001:00008830       ?_Erase@?$_Tree@V?$_Tmap_traits@KURequestInfo@CServerRequest@@U?$less@K@std@@V?$allocator@U?$pair@$$CBKURequestInfo@CServerRequest@@@std@@@4@$0A@@std@@@std@@IAEXPAU_Node@?$_Tree_nod@V?$_Tmap_traits@KURequestInfo@CServerRequest@@U?$less@K@std@@V?$allocator@U?$pair@$$CBKURequestInfo@CServerRequest@@@std@@@4@$0A@@std@@@2@@Z 00409830 f i rylgamelibrary:serverrequest.obj
 0001:00008870       ?_Buynode@?$_Tree@V?$_Tmap_traits@KURequestInfo@CServerRequest@@U?$less@K@std@@V?$allocator@U?$pair@$$CBKURequestInfo@CServerRequest@@@std@@@4@$0A@@std@@@std@@IAEPAU_Node@?$_Tree_nod@V?$_Tmap_traits@KURequestInfo@CServerRequest@@U?$less@K@std@@V?$allocator@U?$pair@$$CBKURequestInfo@CServerRequest@@@std@@@4@$0A@@std@@@2@PAU342@00ABU?$pair@$$CBKURequestInfo@CServerRequest@@@2@D@Z 00409870 f i rylgamelibrary:serverrequest.obj
 0001:000088d0       ?_Buynode@?$_Tree@V?$_Tmap_traits@KURequestInfo@CServerRequest@@U?$less@K@std@@V?$allocator@U?$pair@$$CBKURequestInfo@CServerRequest@@@std@@@4@$0A@@std@@@std@@IAEPAU_Node@?$_Tree_nod@V?$_Tmap_traits@KURequestInfo@CServerRequest@@U?$less@K@std@@V?$allocator@U?$pair@$$CBKURequestInfo@CServerRequest@@@std@@@4@$0A@@std@@@2@XZ 004098d0 f i rylgamelibrary:serverrequest.obj
 0001:00008910       ?find@?$_Tree@V?$_Tmap_traits@KURequestInfo@CServerRequest@@U?$less@K@std@@V?$allocator@U?$pair@$$CBKURequestInfo@CServerRequest@@@std@@@4@$0A@@std@@@std@@QAE?AViterator@12@ABK@Z 00409910 f i rylgamelibrary:serverrequest.obj
 0001:00008980       ?RemoveAllRequest@CServerRequest@@QAEXXZ 00409980 f   rylgamelibrary:serverrequest.obj
 0001:00008a70       ?GetRequest@CServerRequest@@AAEPAVCPacketDispatch@@K@Z 00409a70 f   rylgamelibrary:serverrequest.obj
 0001:00008ac0       ?_Insert@?$_Tree@V?$_Tmap_traits@KURequestInfo@CServerRequest@@U?$less@K@std@@V?$allocator@U?$pair@$$CBKURequestInfo@CServerRequest@@@std@@@4@$0A@@std@@@std@@IAE?AViterator@12@_NPAU_Node@?$_Tree_nod@V?$_Tmap_traits@KURequestInfo@CServerRequest@@U?$less@K@std@@V?$allocator@U?$pair@$$CBKURequestInfo@CServerRequest@@@std@@@4@$0A@@std@@@2@ABU?$pair@$$CBKURequestInfo@CServerRequest@@@2@@Z 00409ac0 f i rylgamelibrary:serverrequest.obj
 0001:00008c70       ?insert@?$_Tree@V?$_Tmap_traits@KURequestInfo@CServerRequest@@U?$less@K@std@@V?$allocator@U?$pair@$$CBKURequestInfo@CServerRequest@@@std@@@4@$0A@@std@@@std@@QAE?AU?$pair@Viterator@?$_Tree@V?$_Tmap_traits@KURequestInfo@CServerRequest@@U?$less@K@std@@V?$allocator@U?$pair@$$CBKURequestInfo@CServerRequest@@@std@@@4@$0A@@std@@@std@@_N@2@ABU?$pair@$$CBKURequestInfo@CServerRequest@@@2@@Z 00409c70 f i rylgamelibrary:serverrequest.obj
 0001:00008d30       ?erase@?$_Tree@V?$_Tmap_traits@KURequestInfo@CServerRequest@@U?$less@K@std@@V?$allocator@U?$pair@$$CBKURequestInfo@CServerRequest@@@std@@@4@$0A@@std@@@std@@QAE?AViterator@12@V312@@Z 00409d30 f i rylgamelibrary:serverrequest.obj
 0001:00008ff0       ??0out_of_range@std@@QAE@ABV01@@Z 00409ff0 f i rylgamelibrary:serverrequest.obj
 0001:00009010       ?erase@?$_Tree@V?$_Tmap_traits@KURequestInfo@CServerRequest@@U?$less@K@std@@V?$allocator@U?$pair@$$CBKURequestInfo@CServerRequest@@@std@@@4@$0A@@std@@@std@@QAE?AViterator@12@V312@0@Z 0040a010 f i rylgamelibrary:serverrequest.obj
 0001:000090d0       ?AddRequest@CServerRequest@@QAEKPAVCPacketDispatch@@0KP6AX0@Z@Z 0040a0d0 f   rylgamelibrary:serverrequest.obj
 0001:00009210       ?RemoveRequest@CServerRequest@@QAEXK@Z 0040a210 f   rylgamelibrary:serverrequest.obj
 0001:000092f0       ?RemoveTimeoutRequest@CServerRequest@@QAEXXZ 0040a2f0 f   rylgamelibrary:serverrequest.obj
 0001:00009400       ?PopRequest@CServerRequest@@AAEPAVCPacketDispatch@@K@Z 0040a400 f   rylgamelibrary:serverrequest.obj
 0001:000094f0       ??1?$map@KURequestInfo@CServerRequest@@U?$less@K@std@@V?$allocator@U?$pair@$$CBKURequestInfo@CServerRequest@@@std@@@4@@std@@QAE@XZ 0040a4f0 f i rylgamelibrary:serverrequest.obj
 0001:00009520       ??1CServerRequest@@AAE@XZ  0040a520 f   rylgamelibrary:serverrequest.obj
 0001:000095c0       ??0CServerRequest@@AAE@XZ  0040a5c0 f   rylgamelibrary:serverrequest.obj
 0001:00009630       ?GetInstance@CServerRequest@@SAAAV1@XZ 0040a630 f   rylgamelibrary:serverrequest.obj
 0001:00009690       ??0Result@CServerRequest@@QAE@K_N@Z 0040a690 f   rylgamelibrary:serverrequest.obj
 0001:000096d0       ??0CSendStream@@QAE@AAVCSession@@@Z 0040a6d0 f   rylgamelibrary:sendstream.obj
 0001:000096f0       ??1CSendStream@@QAE@XZ     0040a6f0 f   rylgamelibrary:sendstream.obj
 0001:00009710       ?GetBuffer@CSendStream@@QAEPADK@Z 0040a710 f   rylgamelibrary:sendstream.obj
 0001:00009790       ?Send@CSession@@QAE_NXZ    0040a790 f i rylgamelibrary:sendstream.obj
 0001:000097e0       ?ForceSend@CSendStream@@AAE_NXZ 0040a7e0 f   rylgamelibrary:sendstream.obj
 0001:00009830       ?WrapHeader@CSendStream@@QAE_NGEGG@Z 0040a830 f   rylgamelibrary:sendstream.obj
 0001:000098a0       ?WrapCrypt@CSendStream@@QAE_NGEGG@Z 0040a8a0 f   rylgamelibrary:sendstream.obj
 0001:00009910       ?StrToHex32@Convert@Math@@YAKPBD@Z 0040a910 f i rylgamelibrary:serversetup.obj
 0001:00009ad0       ?Atoi@Convert@Math@@YAKPBD@Z 0040aad0 f i rylgamelibrary:serversetup.obj
 0001:00009b00       ??_GCSocketFactory@@UAEPAXI@Z 0040ab00 f i rylgamelibrary:serversetup.obj
 0001:00009b00       ??_ECSocketFactory@@UAEPAXI@Z 0040ab00 f i rylgamelibrary:serversetup.obj
 0001:00009b20       ??1CTCPFactory@@UAE@XZ     0040ab20 f i rylgamelibrary:serversetup.obj
 0001:00009b30       ?GetServerID@CServerSetup@@QAEKXZ 0040ab30 f   rylgamelibrary:serversetup.obj
 0001:00009b40       ?GetServerGroup@CServerSetup@@QAEDXZ 0040ab40 f   rylgamelibrary:serversetup.obj
 0001:00009b50       ?InitLoginServer@CServerSetup@@QAE_NXZ 0040ab50 f   rylgamelibrary:serversetup.obj
 0001:00009d60       ?InitAuthServer@CServerSetup@@QAE_NXZ 0040ad60 f   rylgamelibrary:serversetup.obj
 0001:0000a0e0       ?InitAgentServer@CServerSetup@@QAE_NXZ 0040b0e0 f   rylgamelibrary:serversetup.obj
 0001:0000a820       ?InitUIDServer@CServerSetup@@QAE_NXZ 0040b820 f   rylgamelibrary:serversetup.obj
 0001:0000aa30       ?InitChatServer@CServerSetup@@QAE_NXZ 0040ba30 f   rylgamelibrary:serversetup.obj
 0001:0000ac50       ?GetManageClientWindowName@CServerSetup@@SAPBDXZ 0040bc50 f   rylgamelibrary:serversetup.obj
 0001:0000ac60       ?GetGameServerTCPPort@CServerSetup@@SAGK@Z 0040bc60 f   rylgamelibrary:serversetup.obj
 0001:0000ac80       ?GetGameServerUDPPort@CServerSetup@@SAGK@Z 0040bc80 f   rylgamelibrary:serversetup.obj
 0001:0000aca0       ?GetZoneFromCmdLine@CServerSetup@@SADXZ 0040bca0 f   rylgamelibrary:serversetup.obj
 0001:0000adb0       ?GetChannelFromCmdLine@CServerSetup@@SADXZ 0040bdb0 f   rylgamelibrary:serversetup.obj
 0001:0000aec0       ??1CServerSetup@@UAE@XZ    0040bec0 f   rylgamelibrary:serversetup.obj
 0001:0000af20       ??_ECServerSetup@@UAEPAXI@Z 0040bf20 f i rylgamelibrary:serversetup.obj
 0001:0000af20       ??_GCServerSetup@@UAEPAXI@Z 0040bf20 f i rylgamelibrary:serversetup.obj
 0001:0000af40       ??0CServerSetup@@QAE@XZ    0040bf40 f   rylgamelibrary:serversetup.obj
 0001:0000b090       ?GetInstance@CServerSetup@@SAAAV1@XZ 0040c090 f   rylgamelibrary:serversetup.obj
 0001:0000b0f0       ?LoadAdminUID@CServerSetup@@QAE_NXZ 0040c0f0 f   rylgamelibrary:serversetup.obj
 0001:0000b1f0       ?InitGameServer@CServerSetup@@QAE_NXZ 0040c1f0 f   rylgamelibrary:serversetup.obj
 0001:0000b9d0       ?Initialize@CServerSetup@@QAE_NH@Z 0040c9d0 f   rylgamelibrary:serversetup.obj
 0001:0000ba40       ?_Max@?$_Tree@V?$_Tmap_traits@PAVCSessionPolicy@@IU?$less@PAVCSessionPolicy@@@std@@V?$allocator@U?$pair@QAVCSessionPolicy@@I@std@@@3@$0A@@std@@@std@@KAPAU_Node@?$_Tree_nod@V?$_Tmap_traits@PAVCSessionPolicy@@IU?$less@PAVCSessionPolicy@@@std@@V?$allocator@U?$pair@QAVCSessionPolicy@@I@std@@@3@$0A@@std@@@2@PAU342@@Z 0040ca40 f i rylgamelibrary:iocpnet.obj
 0001:0000ba40       ?_Max@?$_Tree@V?$_Tmap_traits@KKU?$less@K@std@@V?$allocator@U?$pair@$$CBKK@std@@@2@$00@std@@@std@@KAPAU_Node@?$_Tree_nod@V?$_Tmap_traits@KKU?$less@K@std@@V?$allocator@U?$pair@$$CBKK@std@@@2@$00@std@@@2@PAU342@@Z 0040ca40 f i rylgamelibrary:friendlist.obj
 0001:0000ba40       ?_Max@?$_Tree@V?$_Tmap_traits@KPAVCCell@@U?$less@K@std@@V?$allocator@U?$pair@$$CBKPAVCCell@@@std@@@3@$0A@@std@@@std@@KAPAU_Node@?$_Tree_nod@V?$_Tmap_traits@KPAVCCell@@U?$less@K@std@@V?$allocator@U?$pair@$$CBKPAVCCell@@@std@@@3@$0A@@std@@@2@PAU342@@Z 0040ca40 f i rylgamelibrary:duelcellmanager.obj
 0001:0000ba40       ?_Max@?$_Tree@V?$_Tmap_traits@KPAVCParty@@U?$less@K@std@@V?$allocator@U?$pair@$$CBKPAVCParty@@@std@@@3@$0A@@std@@@std@@KAPAU_Node@?$_Tree_nod@V?$_Tmap_traits@KPAVCParty@@U?$less@K@std@@V?$allocator@U?$pair@$$CBKPAVCParty@@@std@@@3@$0A@@std@@@2@PAU342@@Z 0040ca40 f i rylgamelibrary:partymgr.obj
 0001:0000ba40       ?_Max@?$_Tree@V?$_Tmap_traits@IPAVCMsgProc@@U?$less@I@std@@V?$allocator@U?$pair@$$CBIPAVCMsgProc@@@std@@@3@$0A@@std@@@std@@KAPAU_Node@?$_Tree_nod@V?$_Tmap_traits@IPAVCMsgProc@@U?$less@I@std@@V?$allocator@U?$pair@$$CBIPAVCMsgProc@@@std@@@3@$0A@@std@@@2@PAU342@@Z 0040ca40 f i rylgamelibrary:msgproc.obj
 0001:0000ba40       ?_Max@?$_Tree@V?$_Tmap_traits@KPAVCPacketDispatch@@U?$less@K@std@@V?$allocator@U?$pair@$$CBKPAVCPacketDispatch@@@std@@@3@$0A@@std@@@std@@KAPAU_Node@?$_Tree_nod@V?$_Tmap_traits@KPAVCPacketDispatch@@U?$less@K@std@@V?$allocator@U?$pair@$$CBKPAVCPacketDispatch@@@std@@@3@$0A@@std@@@2@PAU342@@Z 0040ca40 f i rylgamelibrary:multidispatchstorage.obj
 0001:0000ba40       ?_Max@?$_Tree@V?$_Tmap_traits@KPAVCCharacter@@U?$less@K@std@@V?$allocator@U?$pair@$$CBKPAVCCharacter@@@std@@@3@$0A@@std@@@std@@KAPAU_Node@?$_Tree_nod@V?$_Tmap_traits@KPAVCCharacter@@U?$less@K@std@@V?$allocator@U?$pair@$$CBKPAVCCharacter@@@std@@@3@$0A@@std@@@2@PAU342@@Z 0040ca40 f i rylgamelibrary:partymgr.obj
 0001:0000ba60       ?_Min@?$_Tree@V?$_Tmap_traits@KPAVCCell@@U?$less@K@std@@V?$allocator@U?$pair@$$CBKPAVCCell@@@std@@@3@$0A@@std@@@std@@KAPAU_Node@?$_Tree_nod@V?$_Tmap_traits@KPAVCCell@@U?$less@K@std@@V?$allocator@U?$pair@$$CBKPAVCCell@@@std@@@3@$0A@@std@@@2@PAU342@@Z 0040ca60 f i rylgamelibrary:duelcellmanager.obj
 0001:0000ba60       ?_Min@?$_Tree@V?$_Tmap_traits@PAVCSessionPolicy@@IU?$less@PAVCSessionPolicy@@@std@@V?$allocator@U?$pair@QAVCSessionPolicy@@I@std@@@3@$0A@@std@@@std@@KAPAU_Node@?$_Tree_nod@V?$_Tmap_traits@PAVCSessionPolicy@@IU?$less@PAVCSessionPolicy@@@std@@V?$allocator@U?$pair@QAVCSessionPolicy@@I@std@@@3@$0A@@std@@@2@PAU342@@Z 0040ca60 f i rylgamelibrary:iocpnet.obj
 0001:0000ba60       ?_Min@?$_Tree@V?$_Tmap_traits@KPAVCParty@@U?$less@K@std@@V?$allocator@U?$pair@$$CBKPAVCParty@@@std@@@3@$0A@@std@@@std@@KAPAU_Node@?$_Tree_nod@V?$_Tmap_traits@KPAVCParty@@U?$less@K@std@@V?$allocator@U?$pair@$$CBKPAVCParty@@@std@@@3@$0A@@std@@@2@PAU342@@Z 0040ca60 f i rylgamelibrary:partymgr.obj
 0001:0000ba60       ?_Min@?$_Tree@V?$_Tmap_traits@KPAVCCharacter@@U?$less@K@std@@V?$allocator@U?$pair@$$CBKPAVCCharacter@@@std@@@3@$0A@@std@@@std@@KAPAU_Node@?$_Tree_nod@V?$_Tmap_traits@KPAVCCharacter@@U?$less@K@std@@V?$allocator@U?$pair@$$CBKPAVCCharacter@@@std@@@3@$0A@@std@@@2@PAU342@@Z 0040ca60 f i rylgamelibrary:partymgr.obj
 0001:0000ba60       ?_Min@?$_Tree@V?$_Tmap_traits@KKU?$less@K@std@@V?$allocator@U?$pair@$$CBKK@std@@@2@$00@std@@@std@@KAPAU_Node@?$_Tree_nod@V?$_Tmap_traits@KKU?$less@K@std@@V?$allocator@U?$pair@$$CBKK@std@@@2@$00@std@@@2@PAU342@@Z 0040ca60 f i rylgamelibrary:friendlist.obj
 0001:0000ba60       ?_Min@?$_Tree@V?$_Tmap_traits@IPAVCMsgProc@@U?$less@I@std@@V?$allocator@U?$pair@$$CBIPAVCMsgProc@@@std@@@3@$0A@@std@@@std@@KAPAU_Node@?$_Tree_nod@V?$_Tmap_traits@IPAVCMsgProc@@U?$less@I@std@@V?$allocator@U?$pair@$$CBIPAVCMsgProc@@@std@@@3@$0A@@std@@@2@PAU342@@Z 0040ca60 f i rylgamelibrary:msgproc.obj
 0001:0000ba60       ?_Min@?$_Tree@V?$_Tmap_traits@KPAVCPacketDispatch@@U?$less@K@std@@V?$allocator@U?$pair@$$CBKPAVCPacketDispatch@@@std@@@3@$0A@@std@@@std@@KAPAU_Node@?$_Tree_nod@V?$_Tmap_traits@KPAVCPacketDispatch@@U?$less@K@std@@V?$allocator@U?$pair@$$CBKPAVCPacketDispatch@@@std@@@3@$0A@@std@@@2@PAU342@@Z 0040ca60 f i rylgamelibrary:multidispatchstorage.obj
 0001:0000ba80       ?_Dec@const_iterator@?$_Tree@V?$_Tmap_traits@HPAV?$list@PAVIOPCode@@V?$allocator@PAVIOPCode@@@std@@@std@@U?$less@H@2@V?$allocator@U?$pair@$$CBHPAV?$list@PAVIOPCode@@V?$allocator@PAVIOPCode@@@std@@@std@@@std@@@2@$0A@@std@@@std@@QAEXXZ 0040ca80 f i rylgamelibrary:imcodegen.obj
 0001:0000ba80       ?_Dec@const_iterator@?$_Tree@V?$_Tmap_traits@PAVCSessionPolicy@@IU?$less@PAVCSessionPolicy@@@std@@V?$allocator@U?$pair@QAVCSessionPolicy@@I@std@@@3@$0A@@std@@@std@@QAEXXZ 0040ca80 f i rylgamelibrary:iocpnet.obj
 0001:0000ba80       ?_Dec@const_iterator@?$_Tree@V?$_Tmap_traits@IPAVCMsgProc@@U?$less@I@std@@V?$allocator@U?$pair@$$CBIPAVCMsgProc@@@std@@@3@$0A@@std@@@std@@QAEXXZ 0040ca80 f i rylgamelibrary:msgproc.obj
 0001:0000ba80       ?_Dec@const_iterator@?$_Tree@V?$_Tmap_traits@KPAVCPacketDispatch@@U?$less@K@std@@V?$allocator@U?$pair@$$CBKPAVCPacketDispatch@@@std@@@3@$0A@@std@@@std@@QAEXXZ 0040ca80 f i rylgamelibrary:multidispatchstorage.obj
 0001:0000bae0       ?_Erase@?$_Tree@V?$_Tmap_traits@KPAVCPacketDispatch@@U?$less@K@std@@V?$allocator@U?$pair@$$CBKPAVCPacketDispatch@@@std@@@3@$0A@@std@@@std@@IAEXPAU_Node@?$_Tree_nod@V?$_Tmap_traits@KPAVCPacketDispatch@@U?$less@K@std@@V?$allocator@U?$pair@$$CBKPAVCPacketDispatch@@@std@@@3@$0A@@std@@@2@@Z 0040cae0 f i rylgamelibrary:multidispatchstorage.obj
 0001:0000bb20       ?find@?$_Tree@V?$_Tmap_traits@KPAVCPacketDispatch@@U?$less@K@std@@V?$allocator@U?$pair@$$CBKPAVCPacketDispatch@@@std@@@3@$0A@@std@@@std@@QAE?AViterator@12@ABK@Z 0040cb20 f i rylgamelibrary:multidispatchstorage.obj
 0001:0000bb20       ?find@?$_Tree@V?$_Tmap_traits@IPAVCMsgProc@@U?$less@I@std@@V?$allocator@U?$pair@$$CBIPAVCMsgProc@@@std@@@3@$0A@@std@@@std@@QAE?AViterator@12@ABI@Z 0040cb20 f i rylgamelibrary:msgproc.obj
 0001:0000bb90       ?GetDispatch@CMultiDispatch@@AAEPAVCPacketDispatch@@K@Z 0040cb90 f   rylgamelibrary:multidispatchstorage.obj
 0001:0000bc20       ??0Storage@CMultiDispatch@@QAE@AAV1@K@Z 0040cc20 f   rylgamelibrary:multidispatchstorage.obj
 0001:0000bc40       ?_Insert@?$_Tree@V?$_Tmap_traits@KPAVCPacketDispatch@@U?$less@K@std@@V?$allocator@U?$pair@$$CBKPAVCPacketDispatch@@@std@@@3@$0A@@std@@@std@@IAE?AViterator@12@_NPAU_Node@?$_Tree_nod@V?$_Tmap_traits@KPAVCPacketDispatch@@U?$less@K@std@@V?$allocator@U?$pair@$$CBKPAVCPacketDispatch@@@std@@@3@$0A@@std@@@2@ABU?$pair@$$CBKPAVCPacketDispatch@@@2@@Z 0040cc40 f i rylgamelibrary:multidispatchstorage.obj
 0001:0000bdf0       ?erase@?$_Tree@V?$_Tmap_traits@KPAVCPacketDispatch@@U?$less@K@std@@V?$allocator@U?$pair@$$CBKPAVCPacketDispatch@@@std@@@3@$0A@@std@@@std@@QAE?AViterator@12@V312@@Z 0040cdf0 f i rylgamelibrary:multidispatchstorage.obj
 0001:0000c0b0       ?insert@?$_Tree@V?$_Tmap_traits@KPAVCPacketDispatch@@U?$less@K@std@@V?$allocator@U?$pair@$$CBKPAVCPacketDispatch@@@std@@@3@$0A@@std@@@std@@QAE?AU?$pair@Viterator@?$_Tree@V?$_Tmap_traits@KPAVCPacketDispatch@@U?$less@K@std@@V?$allocator@U?$pair@$$CBKPAVCPacketDispatch@@@std@@@3@$0A@@std@@@std@@_N@2@ABU?$pair@$$CBKPAVCPacketDispatch@@@2@@Z 0040d0b0 f i rylgamelibrary:multidispatchstorage.obj
 0001:0000c170       ?erase@?$_Tree@V?$_Tmap_traits@KPAVCPacketDispatch@@U?$less@K@std@@V?$allocator@U?$pair@$$CBKPAVCPacketDispatch@@@std@@@3@$0A@@std@@@std@@QAE?AViterator@12@V312@0@Z 0040d170 f i rylgamelibrary:multidispatchstorage.obj
 0001:0000c230       ?InternalRemoveDispatch@CMultiDispatch@@AAEXK@Z 0040d230 f   rylgamelibrary:multidispatchstorage.obj
 0001:0000c2d0       ?insert@?$_Tree@V?$_Tmap_traits@KPAVCPacketDispatch@@U?$less@K@std@@V?$allocator@U?$pair@$$CBKPAVCPacketDispatch@@@std@@@3@$0A@@std@@@std@@QAE?AViterator@12@V312@ABU?$pair@$$CBKPAVCPacketDispatch@@@2@@Z 0040d2d0 f i rylgamelibrary:multidispatchstorage.obj
 0001:0000c440       ?SetDispatch@CMultiDispatch@@QAE_NKPAVCPacketDispatch@@@Z 0040d440 f   rylgamelibrary:multidispatchstorage.obj
 0001:0000c570       ?RemoveDispatch@CMultiDispatch@@QAEXK@Z 0040d570 f   rylgamelibrary:multidispatchstorage.obj
 0001:0000c5d0       ??1?$map@KPAVCPacketDispatch@@U?$less@K@std@@V?$allocator@U?$pair@$$CBKPAVCPacketDispatch@@@std@@@3@@std@@QAE@XZ 0040d5d0 f i rylgamelibrary:multidispatchstorage.obj
 0001:0000c600       ??1CMultiDispatch@@QAE@XZ  0040d600 f   rylgamelibrary:multidispatchstorage.obj
 0001:0000c720       ??0CMultiDispatch@@QAE@XZ  0040d720 f   rylgamelibrary:multidispatchstorage.obj
 0001:0000c790       ??0CSingleDispatch@@QAE@XZ 0040d790 f   rylgamelibrary:singledispatchstorage.obj
 0001:0000c7b0       ?InternalRemoveDispatch@CSingleDispatch@@AAEXPAVCPacketDispatch@@@Z 0040d7b0 f   rylgamelibrary:singledispatchstorage.obj
 0001:0000c820       ??1Storage@CMultiDispatch@@QAE@XZ 0040d820 f   rylgamelibrary:multidispatchstorage.obj
 0001:0000c820       ??1Storage@CSingleDispatch@@QAE@XZ 0040d820 f   rylgamelibrary:singledispatchstorage.obj
 0001:0000c840       ?SetDispatch@CSingleDispatch@@QAEXPAVCPacketDispatch@@@Z 0040d840 f   rylgamelibrary:singledispatchstorage.obj
 0001:0000c900       ?RemoveDispatch@CSingleDispatch@@QAEXPAVCPacketDispatch@@@Z 0040d900 f   rylgamelibrary:singledispatchstorage.obj
 0001:0000c960       ?GetDispatchNum@CSingleDispatch@@QAEIXZ 0040d960 f   rylgamelibrary:singledispatchstorage.obj
 0001:0000c990       ??1CSingleDispatch@@QAE@XZ 0040d990 f   rylgamelibrary:singledispatchstorage.obj
 0001:0000ca20       ?GetDispatch@CSingleDispatch@@AAEPAVCPacketDispatch@@XZ 0040da20 f   rylgamelibrary:singledispatchstorage.obj
 0001:0000ca80       ??0Storage@CSingleDispatch@@QAE@AAV1@@Z 0040da80 f   rylgamelibrary:singledispatchstorage.obj
 0001:0000caa0       ??0CComCriticalSection@ATL@@QAE@XZ 0040daa0 f i rylgamelibrary:characterlog.obj
 0001:0000cac0       ?Init@CComCriticalSection@ATL@@QAEJXZ 0040dac0 f i rylgamelibrary:characterlog.obj
 0001:0000cb40       ?LogCharCreateDelete@GAMELOG@@YAXKPBUsockaddr_in@@KEG@Z 0040db40 f   rylgamelibrary:characterlog.obj
 0001:0000cc10       ??0CSession@@QAE@AAVCSessionPolicy@@@Z 0040dc10 f   rylgamelibrary:session.obj
 0001:0000ccf0       ?SetAddress@CSession@@QAEXAAVINET_Addr@@0@Z 0040dcf0 f   rylgamelibrary:session.obj
 0001:0000cd40       ?InternalPrintStatistics@CSession@@AAEHPADH@Z 0040dd40 f   rylgamelibrary:session.obj
 0001:0000cdd0       ??1_Sentry_base@?$basic_ostream@DU?$char_traits@D@std@@@std@@QAE@XZ 0040ddd0 f i rylgamelibrary:session.obj
 0001:0000cdf0       ?InternalCloseSocket@CSession@@AAEXXZ 0040ddf0 f   rylgamelibrary:session.obj
 0001:0000cf20       ?Shutdown@CSession@@QAE_NXZ 0040df20 f   rylgamelibrary:session.obj
 0001:0000cf50       ?AddRef@CSession@@QAEJXZ   0040df50 f   rylgamelibrary:session.obj
 0001:0000cf70       ?Release@CSession@@QAEJXZ  0040df70 f   rylgamelibrary:session.obj
 0001:0000cf90       ?CloseSession@CSession@@QAEXXZ 0040df90 f   rylgamelibrary:session.obj
 0001:0000d020       ?CalledDisconnected@CSession@@QAE_NXZ 0040e020 f   rylgamelibrary:session.obj
 0001:0000d050       ?InternalRecv@CSession@@AAE_NXZ 0040e050 f   rylgamelibrary:session.obj
 0001:0000d180       ?InternalSend@CSession@@AAE_NPAVCBuffer@@@Z 0040e180 f   rylgamelibrary:session.obj
 0001:0000d2b0       ?InternalSendTo@CSession@@AAE_NPAVCBuffer@@@Z 0040e2b0 f   rylgamelibrary:session.obj
 0001:0000d410       ?SendPending@CSession@@QAE_NPAVCBuffer@@@Z 0040e410 f   rylgamelibrary:session.obj
 0001:0000d490       ?InternalSend@CSession@@AAE_NXZ 0040e490 f   rylgamelibrary:session.obj
 0001:0000d4d0       ??1CSession@@QAE@XZ        0040e4d0 f   rylgamelibrary:session.obj
 0001:0000d580       ?Process@CSession@@QAE_NXZ 0040e580 f   rylgamelibrary:session.obj
 0001:0000d830       ?Dispatch@CSession@@QAE_NK@Z 0040e830 f   rylgamelibrary:session.obj
 0001:0000d950       ?SendCompleted@CSession@@QAEXHK@Z 0040e950 f   rylgamelibrary:session.obj
 0001:0000da30       ?flush@?$basic_ostream@DU?$char_traits@D@std@@@std@@QAEAAV12@XZ 0040ea30 f i rylgamelibrary:session.obj
 0001:0000da90       ??0sentry@?$basic_ostream@DU?$char_traits@D@std@@@std@@QAE@AAV12@@Z 0040ea90 f i rylgamelibrary:session.obj
 0001:0000db20       ??1sentry@?$basic_ostream@DU?$char_traits@D@std@@@std@@QAE@XZ 0040eb20 f i rylgamelibrary:session.obj
 0001:0000db90       ??$?6U?$char_traits@D@std@@@std@@YAAAV?$basic_ostream@DU?$char_traits@D@std@@@0@AAV10@PBD@Z 0040eb90 f i rylgamelibrary:session.obj
 0001:0000dda0       ??0CCheckPing@@QAE@XZ      0040eda0 f   rylgamelibrary:checkping.obj
 0001:0000ddc0       ?CheckPing@CCheckPing@@QAE_NK@Z 0040edc0 f   rylgamelibrary:checkping.obj
 0001:0000de50       ?SetLastPingRecvTime@CCheckPing@@QAEXK@Z 0040ee50 f   rylgamelibrary:checkping.obj
 0001:0000de80       ?GetPingData@CCheckPing@@QAEXAAK00@Z 0040ee80 f   rylgamelibrary:checkping.obj
 0001:0000deb0       ?InitFilter@Filter@@YA_NXZ 0040eeb0 f   rylgamelibrary:filter.obj
 0001:0000e090       ?NameCheck@Filter@@YA_NPAD@Z 0040f090 f   rylgamelibrary:filter.obj
 0001:0000e140       ?AccountCheck@Filter@@YA_NPAD@Z 0040f140 f   rylgamelibrary:filter.obj
 0001:0000e1c0       ?CheckCharCreateName@CharCreate@@YA_NPAD_N@Z 0040f1c0 f   rylgamelibrary:charactercreate.obj
 0001:0000e330       ?CheckCharCreateData@CharCreate@@YA_NAAUCHAR_CREATE@@@Z 0040f330 f   rylgamelibrary:charactercreate.obj
 0001:0000e490       ?GetDefaultCharacterPos@CharCreate@@YA?AUPOS@@KK@Z 0040f490 f   rylgamelibrary:charactercreate.obj
 0001:0000e5b0       ??0CDBComponent@@QAE@XZ    0040f5b0 f   rylgamelibrary:dbcomponent.obj
 0001:0000e680       ??1CDBComponent@@UAE@XZ    0040f680 f   rylgamelibrary:dbcomponent.obj
 0001:0000e690       ?LoginAuthMyth@CDBComponent@@QAE_NPBD00PAU_AUTH@@@Z 0040f690 f   rylgamelibrary:dbcomponent.obj
 0001:0000e710       ?LoginAuthHan@CDBComponent@@QAE_NPBD0AAU_HAN_UID@@@Z 0040f710 f   rylgamelibrary:dbcomponent.obj
 0001:0000e7b0       ?RegRylGameHan@CDBComponent@@QAE_NPAD0@Z 0040f7b0 f   rylgamelibrary:dbcomponent.obj
 0001:0000e840       ?GetUIDByAccount@CDBComponent@@QAE_NPAD0@Z 0040f840 f   rylgamelibrary:dbcomponent.obj
 0001:0000e8a0       ?CheckBlockedUser@CDBComponent@@QAE_NKEPAU_RE_CMS_CheckUserBlock@@@Z 0040f8a0 f   rylgamelibrary:dbcomponent.obj
 0001:0000e930       ?LoginBattleAuthHan@CDBComponent@@QAE_NPBD0AAU_HAN_UID@@@Z 0040f930 f   rylgamelibrary:dbcomponent.obj
 0001:0000e9d0       ?RegBattleRylGameHan@CDBComponent@@QAE_NPAD0@Z 0040f9d0 f   rylgamelibrary:dbcomponent.obj
 0001:0000ea60       ?GetBattleUIDByAccount@CDBComponent@@QAE_NPAD0@Z 0040fa60 f   rylgamelibrary:dbcomponent.obj
 0001:0000eac0       ??_ECDBComponent@@UAEPAXI@Z 0040fac0 f i rylgamelibrary:dbcomponent.obj
 0001:0000eac0       ??_GCDBComponent@@UAEPAXI@Z 0040fac0 f i rylgamelibrary:dbcomponent.obj
 0001:0000eae0       ?Connect@CDBComponent@@QAE_NH@Z 0040fae0 f   rylgamelibrary:dbcomponent.obj
 0001:0000f040       ?ThreadFunc@CThread@@KGIPAX@Z 00410040 f i rylgamelibrary:threadmgr.obj
 0001:0000f050       ?Run@CThreadMgr@@SAPAXPAVCThread@@@Z 00410050 f   rylgamelibrary:threadmgr.obj
 0001:0000f080       ?Stop@CThreadMgr@@SA_NPAVCThread@@K@Z 00410080 f   rylgamelibrary:threadmgr.obj
 0001:0000f0c0       ??_9@$B7AE                 004100c0 f i rylgamelibrary:threadmgr.obj
 0001:0000f0d0       ??0CThreadMgr@@QAE@XZ      004100d0 f   rylgamelibrary:threadmgr.obj
 0001:0000f120       ?RegisterAndRun@CThreadMgr@@QAE_NPAVCThread@@@Z 00410120 f   rylgamelibrary:threadmgr.obj
 0001:0000f1c0       ??$for_each@PAPAVCThread@@V?$mem_fun_t@HVCThread@@@std@@@std@@YA?AV?$mem_fun_t@HVCThread@@@0@PAPAVCThread@@0V10@@Z 004101c0 f i rylgamelibrary:threadmgr.obj
 0001:0000f200       ?JoinThread@CThreadMgr@@QAE_NXZ 00410200 f   rylgamelibrary:threadmgr.obj
 0001:0000f2d0       ??1CThreadMgr@@UAE@XZ      004102d0 f   rylgamelibrary:threadmgr.obj
 0001:0000f320       ??_ECThreadMgr@@UAEPAXI@Z  00410320 f i rylgamelibrary:threadmgr.obj
 0001:0000f320       ??_GCThreadMgr@@UAEPAXI@Z  00410320 f i rylgamelibrary:threadmgr.obj
 0001:0000f340       ?GetItemInfo@CItemMgr@Item@@QAEPBUItemInfo@2@G@Z 00410340 f   rylgamelibrary:itemmgr.obj
 0001:0000f3a0       ?size@?$vector@UItemInfo@Item@@V?$allocator@UItemInfo@Item@@@std@@@std@@QBEIXZ 004103a0 f i rylgamelibrary:itemmgr.obj
 0001:0000f3d0       ??$fill@PAUItemInfo@Item@@U12@@std@@YAXPAUItemInfo@Item@@0ABU12@@Z 004103d0 f i rylgamelibrary:itemmgr.obj
 0001:0000f400       ??0CItemMgr@Item@@AAE@XZ   00410400 f   rylgamelibrary:itemmgr.obj
 0001:0000f420       ??1CItemMgr@Item@@QAE@XZ   00410420 f   rylgamelibrary:itemmgr.obj
 0001:0000f460       ??0ItemInfo@Item@@QAE@ABU01@@Z 00410460 f i rylgamelibrary:itemmgr.obj
 0001:0000f540       ??$copy_backward@PAUItemInfo@Item@@PAU12@@std@@YAPAUItemInfo@Item@@PAU12@00@Z 00410540 f i rylgamelibrary:itemmgr.obj
 0001:0000f580       ??$swap@UItemInfo@Item@@@std@@YAXAAUItemInfo@Item@@0@Z 00410580 f i rylgamelibrary:itemmgr.obj
 0001:0000f5e0       ??$_Push_heap@Viterator@?$vector@UItemInfo@Item@@V?$allocator@UItemInfo@Item@@@std@@@std@@HUItemInfo@Item@@@std@@YAXViterator@?$vector@UItemInfo@Item@@V?$allocator@UItemInfo@Item@@@std@@@0@HHUItemInfo@Item@@@Z 004105e0 f i rylgamelibrary:itemmgr.obj
 0001:0000f650       ??$_Rotate@Viterator@?$vector@UItemInfo@Item@@V?$allocator@UItemInfo@Item@@@std@@@std@@HUItemInfo@Item@@@std@@YAXViterator@?$vector@UItemInfo@Item@@V?$allocator@UItemInfo@Item@@@std@@@0@00PAHPAUItemInfo@Item@@@Z 00410650 f i rylgamelibrary:itemmgr.obj
 0001:0000f7c0       ??$copy@Viterator@?$vector@UItemInfo@Item@@V?$allocator@UItemInfo@Item@@@std@@@std@@PAUItemInfo@Item@@@std@@YAPAUItemInfo@Item@@Viterator@?$vector@UItemInfo@Item@@V?$allocator@UItemInfo@Item@@@std@@@0@0PAU12@@Z 004107c0 f i rylgamelibrary:itemmgr.obj
 0001:0000f800       ??$_Uninit_copy@PAUItemInfo@Item@@PAU12@V?$allocator@UItemInfo@Item@@@std@@@std@@YAPAUItemInfo@Item@@PAU12@00AAV?$allocator@UItemInfo@Item@@@0@U_Nonscalar_ptr_iterator_tag@0@@Z 00410800 f i rylgamelibrary:itemmgr.obj
 0001:0000f840       ??$_Adjust_heap@Viterator@?$vector@UItemInfo@Item@@V?$allocator@UItemInfo@Item@@@std@@@std@@HUItemInfo@Item@@@std@@YAXViterator@?$vector@UItemInfo@Item@@V?$allocator@UItemInfo@Item@@@std@@@0@HHUItemInfo@Item@@@Z 00410840 f i rylgamelibrary:itemmgr.obj
 0001:0000f8f0       ??RCParseDelimitedData@@QAE_NAAV?$vector@UParseData@ItemDataParser@@V?$allocator@UParseData@ItemDataParser@@@std@@@std@@AAUItemInfo@Item@@@Z 004108f0 f i rylgamelibrary:itemmgr.obj
 0001:0000f980       ??$_Uninit_fill_n@PAUItemInfo@Item@@IU12@V?$allocator@UItemInfo@Item@@@std@@@std@@YAXPAUItemInfo@Item@@IABU12@AAV?$allocator@UItemInfo@Item@@@0@U_Nonscalar_ptr_iterator_tag@0@@Z 00410980 f i rylgamelibrary:itemmgr.obj
 0001:0000f9b0       ??$_Median@Viterator@?$vector@UItemInfo@Item@@V?$allocator@UItemInfo@Item@@@std@@@std@@@std@@YAXViterator@?$vector@UItemInfo@Item@@V?$allocator@UItemInfo@Item@@@std@@@0@00@Z 004109b0 f i rylgamelibrary:itemmgr.obj
 0001:0000fb40       ??$_Make_heap@Viterator@?$vector@UItemInfo@Item@@V?$allocator@UItemInfo@Item@@@std@@@std@@HUItemInfo@Item@@@std@@YAXViterator@?$vector@UItemInfo@Item@@V?$allocator@UItemInfo@Item@@@std@@@0@0PAHPAUItemInfo@Item@@@Z 00410b40 f i rylgamelibrary:itemmgr.obj
 0001:0000fbb0       ??$_Pop_heap_0@Viterator@?$vector@UItemInfo@Item@@V?$allocator@UItemInfo@Item@@@std@@@std@@UItemInfo@Item@@@std@@YAXViterator@?$vector@UItemInfo@Item@@V?$allocator@UItemInfo@Item@@@std@@@0@0PAUItemInfo@Item@@@Z 00410bb0 f i rylgamelibrary:itemmgr.obj
 0001:0000fc30       ??$_Unguarded_partition@Viterator@?$vector@UItemInfo@Item@@V?$allocator@UItemInfo@Item@@@std@@@std@@@std@@YA?AU?$pair@Viterator@?$vector@UItemInfo@Item@@V?$allocator@UItemInfo@Item@@@std@@@std@@V123@@0@Viterator@?$vector@UItemInfo@Item@@V?$allocator@UItemInfo@Item@@@std@@@0@0@Z 00410c30 f i rylgamelibrary:itemmgr.obj
 0001:0000ff50       ??$_Insertion_sort@Viterator@?$vector@UItemInfo@Item@@V?$allocator@UItemInfo@Item@@@std@@@std@@@std@@YAXViterator@?$vector@UItemInfo@Item@@V?$allocator@UItemInfo@Item@@@std@@@0@0@Z 00410f50 f i rylgamelibrary:itemmgr.obj
 0001:0000ffe0       ?_Ufill@?$vector@UItemInfo@Item@@V?$allocator@UItemInfo@Item@@@std@@@std@@IAEPAUItemInfo@Item@@PAU34@IABU34@@Z 00410fe0 f i rylgamelibrary:itemmgr.obj
 0001:00010010       ??$sort_heap@Viterator@?$vector@UItemInfo@Item@@V?$allocator@UItemInfo@Item@@@std@@@std@@@std@@YAXViterator@?$vector@UItemInfo@Item@@V?$allocator@UItemInfo@Item@@@std@@@0@0@Z 00411010 f i rylgamelibrary:itemmgr.obj
 0001:00010070       ?_Xlen@?$vector@UItemInfo@Item@@V?$allocator@UItemInfo@Item@@@std@@@std@@IBEXXZ 00411070 f i rylgamelibrary:itemmgr.obj
 0001:00010070       ?_Xlen@?$vector@UParseData@ItemDataParser@@V?$allocator@UParseData@ItemDataParser@@@std@@@std@@IBEXXZ 00411070 f i rylgamelibrary:itemmgr.obj
 0001:000100e0       ??$_Sort@Viterator@?$vector@UItemInfo@Item@@V?$allocator@UItemInfo@Item@@@std@@@std@@H@std@@YAXViterator@?$vector@UItemInfo@Item@@V?$allocator@UItemInfo@Item@@@std@@@0@0H@Z 004110e0 f i rylgamelibrary:itemmgr.obj
 0001:00010210       ?_Insert_n@?$vector@UItemInfo@Item@@V?$allocator@UItemInfo@Item@@@std@@@std@@IAEXViterator@12@IABUItemInfo@Item@@@Z 00411210 f i rylgamelibrary:itemmgr.obj
 0001:00010500       ??$sort@Viterator@?$vector@UItemInfo@Item@@V?$allocator@UItemInfo@Item@@@std@@@std@@@std@@YAXViterator@?$vector@UItemInfo@Item@@V?$allocator@UItemInfo@Item@@@std@@@0@0@Z 00411500 f i rylgamelibrary:itemmgr.obj
 0001:00010530       ?insert@?$vector@UItemInfo@Item@@V?$allocator@UItemInfo@Item@@@std@@@std@@QAE?AViterator@12@V312@ABUItemInfo@Item@@@Z 00411530 f i rylgamelibrary:itemmgr.obj
 0001:000105a0       ?push_back@?$vector@UItemInfo@Item@@V?$allocator@UItemInfo@Item@@@std@@@std@@QAEXABUItemInfo@Item@@@Z 004115a0 f i rylgamelibrary:itemmgr.obj
 0001:00010630       ?LoadItemProtoType@CItemMgr@Item@@QAE_NPBD@Z 00411630 f   rylgamelibrary:itemmgr.obj
 0001:00010ac0       ?CreateItem@CItemFactory@Item@@QAEPAVCItem@2@ABUItemInfo@2@@Z 00411ac0 f   rylgamelibrary:itemfactory.obj
 0001:00010c00       ??0CItemFactory@Item@@AAE@XZ 00411c00 f   rylgamelibrary:itemfactory.obj
 0001:00010c20       ??1CItemFactory@Item@@QAE@XZ 00411c20 f   rylgamelibrary:itemfactory.obj
 0001:00010c30       ?CreateItem@CItemFactory@Item@@QAEPAVCItem@2@G@Z 00411c30 f   rylgamelibrary:itemfactory.obj
 0001:00010c80       ??RCSendDataToManageClient@@UAEJPAUHWND__@@IIJ@Z 00411c80 f i rylgamelibrary:serverwindowframework.obj
 0001:00010ce0       ?ServerWindowFrameworkProc@CServerWindowFramework@@KGJPAUHWND__@@IIJ@Z 00411ce0 f   rylgamelibrary:serverwindowframework.obj
 0001:00010db0       ?PrintOutput@CServerWindowFramework@@QAEXPBDH@Z 00411db0 f   rylgamelibrary:serverwindowframework.obj
 0001:00010dc0       ?PrintInfo@CServerWindowFramework@@QAEXPBDH@Z 00411dc0 f   rylgamelibrary:serverwindowframework.obj
 0001:00010dd0       ?SendManageClientPacket@CServerWindowFramework@@QAE_NPBXG@Z 00411dd0 f   rylgamelibrary:serverwindowframework.obj
 0001:00010e50       ??0CProcessThread@@QAE@AAVCServerWindowFramework@@J@Z 00411e50 f   rylgamelibrary:serverwindowframework.obj
 0001:00010e80       ??1CProcessThread@@UAE@XZ  00411e80 f   rylgamelibrary:serverwindowframework.obj
 0001:00010ed0       ?InitializeFramework@CServerWindowFramework@@IAE_NPAUHINSTANCE__@@PBDHH@Z 00411ed0 f   rylgamelibrary:serverwindowframework.obj
 0001:00011140       ?Destroy@CServerWindowFramework@@AAEXXZ 00412140 f   rylgamelibrary:serverwindowframework.obj
 0001:00011220       ?SendManageClientPing@CServerWindowFramework@@QAEXXZ 00412220 f   rylgamelibrary:serverwindowframework.obj
 0001:00011300       ??_ECProcessThread@@UAEPAXI@Z 00412300 f i rylgamelibrary:serverwindowframework.obj
 0001:00011300       ??_GCProcessThread@@UAEPAXI@Z 00412300 f i rylgamelibrary:serverwindowframework.obj
 0001:00011320       ?Run@CProcessThread@@EAEIXZ 00412320 f   rylgamelibrary:serverwindowframework.obj
 0001:000113f0       ?Initialize@CServerWindowFramework@@QAE_NPAUHINSTANCE__@@PBD1HH@Z 004123f0 f   rylgamelibrary:serverwindowframework.obj
 0001:00011510       ?ProcessMessage@CServerWindowFramework@@QAEXXZ 00412510 f   rylgamelibrary:serverwindowframework.obj
 0001:00011680       ??1CServerWindowFramework@@MAE@XZ 00412680 f   rylgamelibrary:serverwindowframework.obj
 0001:000116e0       ??0CServerWindowFramework@@IAE@XZ 004126e0 f   rylgamelibrary:serverwindowframework.obj
 0001:00011850       ??_GCServerWindowFramework@@MAEPAXI@Z 00412850 f i rylgamelibrary:serverwindowframework.obj
 0001:00011850       ??_ECServerWindowFramework@@MAEPAXI@Z 00412850 f i rylgamelibrary:serverwindowframework.obj
 0001:00011870       ?_Incsize@?$list@PAVCThread@@V?$allocator@PAVCThread@@@std@@@std@@IAEXI@Z 00412870 f i rylgamelibrary:serverwindowframework.obj
 0001:00011910       ??RCRecvCommandFromManageClient@@UAEJPAUHWND__@@IIJ@Z 00412910 f i rylgamelibrary:serverwindowframework.obj
 0001:000119e0       ?AddProcessThread@CServerWindowFramework@@IAE_NPAVCThread@@@Z 004129e0 f   rylgamelibrary:serverwindowframework.obj
 0001:00011a60       ??1CValidateConnection@@MAE@XZ 00412a60 f i rylgamelibrary:limituserbyip.obj
 0001:00011a70       ??_ECValidateConnection@@MAEPAXI@Z 00412a70 f i rylgamelibrary:limituserbyip.obj
 0001:00011a70       ??_GCValidateConnection@@MAEPAXI@Z 00412a70 f i rylgamelibrary:limituserbyip.obj
 0001:00011a90       ?OperateMode@CLimitUserByIP@@QAEXW4AllowMode_t@1@@Z 00412a90 f   rylgamelibrary:limituserbyip.obj
 0001:00011ac0       ??$_Uninit_copy@Viterator@?$vector@PADV?$allocator@PAD@std@@@std@@PAPADV?$allocator@PAD@3@@std@@YAPAPADViterator@?$vector@PADV?$allocator@PAD@std@@@0@0PAPADAAV?$allocator@PAD@0@U_Nonscalar_ptr_iterator_tag@0@@Z 00412ac0 f i rylgamelibrary:tokenlizedfile.obj
 0001:00011ac0       ??$_Uninit_copy@Viterator@?$vector@W4Type@ItemType@Item@@V?$allocator@W4Type@ItemType@Item@@@std@@@std@@PAW4Type@ItemType@Item@@V?$allocator@W4Type@ItemType@Item@@@3@@std@@YAPAW4Type@ItemType@Item@@Viterator@?$vector@W4Type@ItemType@Item@@V?$allocator@W4Type@ItemType@Item@@@std@@@0@0PAW4123@AAV?$allocator@W4Type@ItemType@Item@@@0@U_Nonscalar_ptr_iterator_tag@0@@Z 00412ac0 f i rylgamelibrary:itemconstants.obj
 0001:00011ac0       ??$_Uninit_copy@Viterator@?$vector@KV?$allocator@K@std@@@std@@PAKV?$allocator@K@3@@std@@YAPAKViterator@?$vector@KV?$allocator@K@std@@@0@0PAKAAV?$allocator@K@0@U_Nonscalar_ptr_iterator_tag@0@@Z 00412ac0 f i rylgamelibrary:limituserbyip.obj
 0001:00011ac0       ??$_Uninit_copy@PAW4Type@ItemType@Item@@PAW4123@V?$allocator@W4Type@ItemType@Item@@@std@@@std@@YAPAW4Type@ItemType@Item@@PAW4123@00AAV?$allocator@W4Type@ItemType@Item@@@0@U_Nonscalar_ptr_iterator_tag@0@@Z 00412ac0 f i rylgamelibrary:itemconstants.obj
 0001:00011af0       ??$_Median@Viterator@?$vector@KV?$allocator@K@std@@@std@@@std@@YAXViterator@?$vector@KV?$allocator@K@std@@@0@00@Z 00412af0 f i rylgamelibrary:limituserbyip.obj
 0001:00011c30       ??$_Adjust_heap@Viterator@?$vector@KV?$allocator@K@std@@@std@@HK@std@@YAXViterator@?$vector@KV?$allocator@K@std@@@0@HHK@Z 00412c30 f i rylgamelibrary:limituserbyip.obj
 0001:00011cb0       ??$_Lower_bound@Viterator@?$vector@KV?$allocator@K@std@@@std@@KH@std@@YA?AViterator@?$vector@KV?$allocator@K@std@@@0@V120@0ABKPAH@Z 00412cb0 f i rylgamelibrary:limituserbyip.obj
 0001:00011d00       ??$_Unguarded_partition@Viterator@?$vector@KV?$allocator@K@std@@@std@@@std@@YA?AU?$pair@Viterator@?$vector@KV?$allocator@K@std@@@std@@V123@@0@Viterator@?$vector@KV?$allocator@K@std@@@0@0@Z 00412d00 f i rylgamelibrary:limituserbyip.obj
 0001:00011e50       ??$_Make_heap@Viterator@?$vector@KV?$allocator@K@std@@@std@@HK@std@@YAXViterator@?$vector@KV?$allocator@K@std@@@0@0PAHPAK@Z 00412e50 f i rylgamelibrary:limituserbyip.obj
 0001:00011e90       ??1CLimitUserByIP@@UAE@XZ  00412e90 f   rylgamelibrary:limituserbyip.obj
 0001:00011ed0       ??$_Insertion_sort@Viterator@?$vector@KV?$allocator@K@std@@@std@@@std@@YAXViterator@?$vector@KV?$allocator@K@std@@@0@0@Z 00412ed0 f i rylgamelibrary:limituserbyip.obj
 0001:00011f50       ??_ECLimitUserByIP@@UAEPAXI@Z 00412f50 f i rylgamelibrary:limituserbyip.obj
 0001:00011f50       ??_GCLimitUserByIP@@UAEPAXI@Z 00412f50 f i rylgamelibrary:limituserbyip.obj
 0001:00011f70       ??$binary_search@Viterator@?$vector@KV?$allocator@K@std@@@std@@K@std@@YA_NViterator@?$vector@KV?$allocator@K@std@@@0@0ABK@Z 00412f70 f i rylgamelibrary:limituserbyip.obj
 0001:00011fb0       ??$sort_heap@Viterator@?$vector@KV?$allocator@K@std@@@std@@@std@@YAXViterator@?$vector@KV?$allocator@K@std@@@0@0@Z 00412fb0 f i rylgamelibrary:limituserbyip.obj
 0001:00012000       ??RCLimitUserByIP@@UAE_NAAVINET_Addr@@0@Z 00413000 f   rylgamelibrary:limituserbyip.obj
 0001:00012070       ??$_Sort@Viterator@?$vector@KV?$allocator@K@std@@@std@@H@std@@YAXViterator@?$vector@KV?$allocator@K@std@@@0@0H@Z 00413070 f i rylgamelibrary:limituserbyip.obj
 0001:00012140       ?reserve@?$vector@KV?$allocator@K@std@@@std@@QAEXI@Z 00413140 f i rylgamelibrary:limituserbyip.obj
 0001:00012210       ?LoadAllowIPList@CLimitUserByIP@@QAE_NPBD@Z 00413210 f   rylgamelibrary:limituserbyip.obj
 0001:00012390       ??0CLimitUserByIP@@QAE@PBD@Z 00413390 f   rylgamelibrary:limituserbyip.obj
 0001:00012430       ?AttachToHander@CCompletionHandler@@QAE_NPAXK@Z 00413430 f i rylgamelibrary:listener.obj
 0001:00012460       ?InternalCloseListen@CListener@@AAEXXZ 00413460 f   rylgamelibrary:listener.obj
 0001:000124b0       ?Release@CValidateConnection@@QAEJXZ 004134b0 f   rylgamelibrary:listener.obj
 0001:000124e0       ??0CListener@@QAE@AAVCCompletionHandler@@AAVCSessionPolicy@@AAVCSessionMgr@@PAVCValidateConnection@@@Z 004134e0 f   rylgamelibrary:listener.obj
 0001:00012590       ?WaitForPendingComplete@CListener@@AAEXK@Z 00413590 f   rylgamelibrary:listener.obj
 0001:00012600       ?PendingAccept@CListener@@QAE_NXZ 00413600 f   rylgamelibrary:listener.obj
 0001:00012720       ?ProcessAccept@CListener@@QAEXHIPAVCBuffer@@K@Z 00413720 f   rylgamelibrary:listener.obj
 0001:00012900       ?GetPendingAcceptNum@CListener@@QAEKXZ 00413900 f   rylgamelibrary:listener.obj
 0001:00012920       ??1CListener@@UAE@XZ       00413920 f   rylgamelibrary:listener.obj
 0001:00012a00       ?Initialize@CListener@@QAE_NAAVINET_Addr@@K@Z 00413a00 f   rylgamelibrary:listener.obj
 0001:00012bc0       ??_ECListener@@UAEPAXI@Z   00413bc0 f i rylgamelibrary:listener.obj
 0001:00012bc0       ??_GCListener@@UAEPAXI@Z   00413bc0 f i rylgamelibrary:listener.obj
 0001:00012be0       ??0CSessionPolicy@@AAE@PAVCSocketFactory@@PAVCBufferFactory@@PAVCDispatchFactory@@PAVCOverlappedFactory@@@Z 00413be0 f   rylgamelibrary:sessionpolicy.obj
 0001:00012c10       ??1CSessionPolicy@@AAE@XZ  00413c10 f   rylgamelibrary:sessionpolicy.obj
 0001:00012c50       ?AddRef@CSessionPolicy@@QAEJXZ 00413c50 f   rylgamelibrary:sessionpolicy.obj
 0001:00012c60       ?Release@CSessionPolicy@@QAEJXZ 00413c60 f   rylgamelibrary:sessionpolicy.obj
 0001:00012cc0       ??0INET_Addr@@QAE@PBDG@Z   00413cc0 f i rylgamelibrary:iocpnet.obj
 0001:00012ce0       ?Initialize@CListener@@QAE_NPBDGK@Z 00413ce0 f i rylgamelibrary:iocpnet.obj
 0001:00012d20       ?GetOptimalThreadNum@@YAKXZ 00413d20 f   rylgamelibrary:iocpnet.obj
 0001:00012d40       ?Process@CSessionMgr@@QAEXXZ 00413d40 f i rylgamelibrary:iocpnet.obj
 0001:00012d90       ?GetSessionNum@CSessionMgr@@QAEIXZ 00413d90 f i rylgamelibrary:iocpnet.obj
 0001:00012db0       ?Initialize@CIOCPNet@@QAE_NXZ 00413db0 f   rylgamelibrary:iocpnet.obj
 0001:00012ea0       ?Process@CIOCPNet@@QAEXXZ  00413ea0 f   rylgamelibrary:iocpnet.obj
 0001:00012eb0       ?GetSessionNum@CIOCPNet@@QAEKXZ 00413eb0 f   rylgamelibrary:iocpnet.obj
 0001:00012ec0       ?_Erase@?$_Tree@V?$_Tmap_traits@PAVCSessionPolicy@@IU?$less@PAVCSessionPolicy@@@std@@V?$allocator@U?$pair@QAVCSessionPolicy@@I@std@@@3@$0A@@std@@@std@@IAEXPAU_Node@?$_Tree_nod@V?$_Tmap_traits@PAVCSessionPolicy@@IU?$less@PAVCSessionPolicy@@@std@@V?$allocator@U?$pair@QAVCSessionPolicy@@I@std@@@3@$0A@@std@@@2@@Z 00413ec0 f i rylgamelibrary:iocpnet.obj
 0001:00012f00       ?_Buynode@?$_Tree@V?$_Tmap_traits@HPAV?$list@PAVIOPCode@@V?$allocator@PAVIOPCode@@@std@@@std@@U?$less@H@2@V?$allocator@U?$pair@$$CBHPAV?$list@PAVIOPCode@@V?$allocator@PAVIOPCode@@@std@@@std@@@std@@@2@$0A@@std@@@std@@IAEPAU_Node@?$_Tree_nod@V?$_Tmap_traits@HPAV?$list@PAVIOPCode@@V?$allocator@PAVIOPCode@@@std@@@std@@U?$less@H@2@V?$allocator@U?$pair@$$CBHPAV?$list@PAVIOPCode@@V?$allocator@PAVIOPCode@@@std@@@std@@@std@@@2@$0A@@std@@@2@PAU342@00ABU?$pair@$$CBHPAV?$list@PAVIOPCode@@V?$allocator@PAVIOPCode@@@std@@@std@@@2@D@Z 00413f00 f i rylgamelibrary:imcodegen.obj
 0001:00012f00       ?_Buynode@?$_Tree@V?$_Tmap_traits@IPAVCMsgProc@@U?$less@I@std@@V?$allocator@U?$pair@$$CBIPAVCMsgProc@@@std@@@3@$0A@@std@@@std@@IAEPAU_Node@?$_Tree_nod@V?$_Tmap_traits@IPAVCMsgProc@@U?$less@I@std@@V?$allocator@U?$pair@$$CBIPAVCMsgProc@@@std@@@3@$0A@@std@@@2@PAU342@00ABU?$pair@$$CBIPAVCMsgProc@@@2@D@Z 00413f00 f i rylgamelibrary:msgproc.obj
 0001:00012f00       ?_Buynode@?$_Tree@V?$_Tmap_traits@KPAVCPacketDispatch@@U?$less@K@std@@V?$allocator@U?$pair@$$CBKPAVCPacketDispatch@@@std@@@3@$0A@@std@@@std@@IAEPAU_Node@?$_Tree_nod@V?$_Tmap_traits@KPAVCPacketDispatch@@U?$less@K@std@@V?$allocator@U?$pair@$$CBKPAVCPacketDispatch@@@std@@@3@$0A@@std@@@2@PAU342@00ABU?$pair@$$CBKPAVCPacketDispatch@@@2@D@Z 00413f00 f i rylgamelibrary:multidispatchstorage.obj
 0001:00012f00       ?_Buynode@?$_Tree@V?$_Tmap_traits@PAVCSessionPolicy@@IU?$less@PAVCSessionPolicy@@@std@@V?$allocator@U?$pair@QAVCSessionPolicy@@I@std@@@3@$0A@@std@@@std@@IAEPAU_Node@?$_Tree_nod@V?$_Tmap_traits@PAVCSessionPolicy@@IU?$less@PAVCSessionPolicy@@@std@@V?$allocator@U?$pair@QAVCSessionPolicy@@I@std@@@3@$0A@@std@@@2@PAU342@00ABU?$pair@QAVCSessionPolicy@@I@2@D@Z 00413f00 f i rylgamelibrary:iocpnet.obj
 0001:00012f40       ?GetAcceptPendingNum@CIOCPNet@@QAEKXZ 00413f40 f   rylgamelibrary:iocpnet.obj
 0001:00012fb0       ?_Copy@?$_Tree@V?$_Tmap_traits@PAVCSessionPolicy@@IU?$less@PAVCSessionPolicy@@@std@@V?$allocator@U?$pair@QAVCSessionPolicy@@I@std@@@3@$0A@@std@@@std@@IAEPAU_Node@?$_Tree_nod@V?$_Tmap_traits@PAVCSessionPolicy@@IU?$less@PAVCSessionPolicy@@@std@@V?$allocator@U?$pair@QAVCSessionPolicy@@I@std@@@3@$0A@@std@@@2@PAU342@0@Z 00413fb0 f i rylgamelibrary:iocpnet.obj
 0001:00013060       ?_Copy@?$_Tree@V?$_Tmap_traits@PAVCSessionPolicy@@IU?$less@PAVCSessionPolicy@@@std@@V?$allocator@U?$pair@QAVCSessionPolicy@@I@std@@@3@$0A@@std@@@std@@IAEXABV12@@Z 00414060 f i rylgamelibrary:iocpnet.obj
 0001:000130f0       ?erase@?$_Tree@V?$_Tmap_traits@PAVCSessionPolicy@@IU?$less@PAVCSessionPolicy@@@std@@V?$allocator@U?$pair@QAVCSessionPolicy@@I@std@@@3@$0A@@std@@@std@@QAE?AViterator@12@V312@@Z 004140f0 f i rylgamelibrary:iocpnet.obj
 0001:000133b0       ?_Incsize@?$list@PAVCListener@@V?$allocator@PAVCListener@@@std@@@std@@IAEXI@Z 004143b0 f i rylgamelibrary:iocpnet.obj
 0001:00013450       ?erase@?$_Tree@V?$_Tmap_traits@PAVCSessionPolicy@@IU?$less@PAVCSessionPolicy@@@std@@V?$allocator@U?$pair@QAVCSessionPolicy@@I@std@@@3@$0A@@std@@@std@@QAE?AViterator@12@V312@0@Z 00414450 f i rylgamelibrary:iocpnet.obj
 0001:00013510       ?_Insert@?$_Tree@V?$_Tmap_traits@PAVCSessionPolicy@@IU?$less@PAVCSessionPolicy@@@std@@V?$allocator@U?$pair@QAVCSessionPolicy@@I@std@@@3@$0A@@std@@@std@@IAE?AViterator@12@_NPAU_Node@?$_Tree_nod@V?$_Tmap_traits@PAVCSessionPolicy@@IU?$less@PAVCSessionPolicy@@@std@@V?$allocator@U?$pair@QAVCSessionPolicy@@I@std@@@3@$0A@@std@@@2@ABU?$pair@QAVCSessionPolicy@@I@2@@Z 00414510 f i rylgamelibrary:iocpnet.obj
 0001:000136c0       ?insert@?$_Tree@V?$_Tmap_traits@PAVCSessionPolicy@@IU?$less@PAVCSessionPolicy@@@std@@V?$allocator@U?$pair@QAVCSessionPolicy@@I@std@@@3@$0A@@std@@@std@@QAE?AU?$pair@Viterator@?$_Tree@V?$_Tmap_traits@PAVCSessionPolicy@@IU?$less@PAVCSessionPolicy@@@std@@V?$allocator@U?$pair@QAVCSessionPolicy@@I@std@@@3@$0A@@std@@@std@@_N@2@ABU?$pair@QAVCSessionPolicy@@I@2@@Z 004146c0 f i rylgamelibrary:iocpnet.obj
 0001:00013780       ?push_back@?$list@PAVCListener@@V?$allocator@PAVCListener@@@std@@@std@@QAEXABQAVCListener@@@Z 00414780 f i rylgamelibrary:iocpnet.obj
 0001:000137c0       ??0?$_Tree@V?$_Tmap_traits@PAVCSessionPolicy@@IU?$less@PAVCSessionPolicy@@@std@@V?$allocator@U?$pair@QAVCSessionPolicy@@I@std@@@3@$0A@@std@@@std@@QAE@ABV01@@Z 004147c0 f i rylgamelibrary:iocpnet.obj
 0001:00013850       ?insert@?$_Tree@V?$_Tmap_traits@PAVCSessionPolicy@@IU?$less@PAVCSessionPolicy@@@std@@V?$allocator@U?$pair@QAVCSessionPolicy@@I@std@@@3@$0A@@std@@@std@@QAE?AViterator@12@V312@ABU?$pair@QAVCSessionPolicy@@I@2@@Z 00414850 f i rylgamelibrary:iocpnet.obj
 0001:000139c0       ?_Tidy@?$_Tree@V?$_Tmap_traits@PAVCSessionPolicy@@IU?$less@PAVCSessionPolicy@@@std@@V?$allocator@U?$pair@QAVCSessionPolicy@@I@std@@@3@$0A@@std@@@std@@IAEXXZ 004149c0 f i rylgamelibrary:iocpnet.obj
 0001:000139c0       ??1?$map@PAVCSessionPolicy@@IU?$less@PAVCSessionPolicy@@@std@@V?$allocator@U?$pair@QAVCSessionPolicy@@I@std@@@3@@std@@QAE@XZ 004149c0 f i rylgamelibrary:iocpnet.obj
 0001:000139f0       ??A?$map@PAVCSessionPolicy@@IU?$less@PAVCSessionPolicy@@@std@@V?$allocator@U?$pair@QAVCSessionPolicy@@I@std@@@3@@std@@QAEAAIABQAVCSessionPolicy@@@Z 004149f0 f i rylgamelibrary:iocpnet.obj
 0001:00013a70       ?_Splice@?$list@PAVCListener@@V?$allocator@PAVCListener@@@std@@@std@@QAEXViterator@12@AAV12@00I@Z 00414a70 f i rylgamelibrary:iocpnet.obj
 0001:00013ac0       ??0CIOCPNet@@QAE@XZ        00414ac0 f   rylgamelibrary:iocpnet.obj
 0001:00013c10       ?AddListener@CIOCPNet@@QAE_NPAVCSessionPolicy@@PBDGKPAVCValidateConnection@@@Z 00414c10 f   rylgamelibrary:iocpnet.obj
 0001:00013d70       ?Connect@CIOCPNet@@QAE_NPAVCSessionPolicy@@PBDG@Z 00414d70 f   rylgamelibrary:iocpnet.obj
 0001:00013f70       ?DestroyListener@CIOCPNet@@AAEXXZ 00414f70 f   rylgamelibrary:iocpnet.obj
 0001:00014050       ?Destroy@CIOCPNet@@AAE_NXZ 00415050 f   rylgamelibrary:iocpnet.obj
 0001:000141e0       ??1CIOCPNet@@QAE@XZ        004151e0 f   rylgamelibrary:iocpnet.obj
 0001:00014280       ?_Min@?$_Tree@V?$_Tmap_traits@KUInstrument@CPerformanceCheck@@U?$less@K@std@@V?$allocator@U?$pair@$$CBKUInstrument@CPerformanceCheck@@@std@@@4@$00@std@@@std@@KAPAU_Node@?$_Tree_nod@V?$_Tmap_traits@KUInstrument@CPerformanceCheck@@U?$less@K@std@@V?$allocator@U?$pair@$$CBKUInstrument@CPerformanceCheck@@@std@@@4@$00@std@@@2@PAU342@@Z 00415280 f i rylgamelibrary:performancecheck.obj
 0001:000142a0       ?_Max@?$_Tree@V?$_Tmap_traits@KUInstrument@CPerformanceCheck@@U?$less@K@std@@V?$allocator@U?$pair@$$CBKUInstrument@CPerformanceCheck@@@std@@@4@$00@std@@@std@@KAPAU_Node@?$_Tree_nod@V?$_Tmap_traits@KUInstrument@CPerformanceCheck@@U?$less@K@std@@V?$allocator@U?$pair@$$CBKUInstrument@CPerformanceCheck@@@std@@@4@$00@std@@@2@PAU342@@Z 004152a0 f i rylgamelibrary:performancecheck.obj
 0001:000142c0       ?_Inc@const_iterator@?$_Tree@V?$_Tmap_traits@KUInstrument@CPerformanceCheck@@U?$less@K@std@@V?$allocator@U?$pair@$$CBKUInstrument@CPerformanceCheck@@@std@@@4@$00@std@@@std@@QAEXXZ 004152c0 f i rylgamelibrary:performancecheck.obj
 0001:00014320       ?_Lrotate@?$_Tree@V?$_Tmap_traits@KUInstrument@CPerformanceCheck@@U?$less@K@std@@V?$allocator@U?$pair@$$CBKUInstrument@CPerformanceCheck@@@std@@@4@$00@std@@@std@@IAEXPAU_Node@?$_Tree_nod@V?$_Tmap_traits@KUInstrument@CPerformanceCheck@@U?$less@K@std@@V?$allocator@U?$pair@$$CBKUInstrument@CPerformanceCheck@@@std@@@4@$00@std@@@2@@Z 00415320 f i rylgamelibrary:performancecheck.obj
 0001:00014380       ?_Rrotate@?$_Tree@V?$_Tmap_traits@KUInstrument@CPerformanceCheck@@U?$less@K@std@@V?$allocator@U?$pair@$$CBKUInstrument@CPerformanceCheck@@@std@@@4@$00@std@@@std@@IAEXPAU_Node@?$_Tree_nod@V?$_Tmap_traits@KUInstrument@CPerformanceCheck@@U?$less@K@std@@V?$allocator@U?$pair@$$CBKUInstrument@CPerformanceCheck@@@std@@@4@$00@std@@@2@@Z 00415380 f i rylgamelibrary:performancecheck.obj
 0001:000143e0       ?_Erase@?$_Tree@V?$_Tmap_traits@KUInstrument@CPerformanceCheck@@U?$less@K@std@@V?$allocator@U?$pair@$$CBKUInstrument@CPerformanceCheck@@@std@@@4@$00@std@@@std@@IAEXPAU_Node@?$_Tree_nod@V?$_Tmap_traits@KUInstrument@CPerformanceCheck@@U?$less@K@std@@V?$allocator@U?$pair@$$CBKUInstrument@CPerformanceCheck@@@std@@@4@$00@std@@@2@@Z 004153e0 f i rylgamelibrary:performancecheck.obj
 0001:00014420       ?_Buynode@?$_Tree@V?$_Tmap_traits@KUInstrument@CPerformanceCheck@@U?$less@K@std@@V?$allocator@U?$pair@$$CBKUInstrument@CPerformanceCheck@@@std@@@4@$00@std@@@std@@IAEPAU_Node@?$_Tree_nod@V?$_Tmap_traits@KUInstrument@CPerformanceCheck@@U?$less@K@std@@V?$allocator@U?$pair@$$CBKUInstrument@CPerformanceCheck@@@std@@@4@$00@std@@@2@XZ 00415420 f i rylgamelibrary:performancecheck.obj
 0001:00014460       ?PrintAllTime@CPerformanceCheck@@QAE_NPBD_N@Z 00415460 f   rylgamelibrary:performancecheck.obj
 0001:00014740       ?erase@?$_Tree@V?$_Tmap_traits@KUInstrument@CPerformanceCheck@@U?$less@K@std@@V?$allocator@U?$pair@$$CBKUInstrument@CPerformanceCheck@@@std@@@4@$00@std@@@std@@QAE?AViterator@12@V312@@Z 00415740 f i rylgamelibrary:performancecheck.obj
 0001:00014a00       ?erase@?$_Tree@V?$_Tmap_traits@KUInstrument@CPerformanceCheck@@U?$less@K@std@@V?$allocator@U?$pair@$$CBKUInstrument@CPerformanceCheck@@@std@@@4@$00@std@@@std@@QAE?AViterator@12@V312@0@Z 00415a00 f i rylgamelibrary:performancecheck.obj
 0001:00014ac0       ??1?$multimap@KUInstrument@CPerformanceCheck@@U?$less@K@std@@V?$allocator@U?$pair@$$CBKUInstrument@CPerformanceCheck@@@std@@@4@@std@@QAE@XZ 00415ac0 f i rylgamelibrary:performancecheck.obj
 0001:00014af0       ??1CPerformanceCheck@@AAE@XZ 00415af0 f   rylgamelibrary:performancecheck.obj
 0001:00014ba0       ??0CPerformanceCheck@@AAE@XZ 00415ba0 f   rylgamelibrary:performancecheck.obj
 0001:00014c60       ?GetInstance@CPerformanceCheck@@SAAAV1@XZ 00415c60 f   rylgamelibrary:performancecheck.obj
 0001:00014cc0       ?End@CLogSaveThread@@MAEHXZ 00415cc0 f   rylgamelibrary:gamelog.obj
 0001:00014ce0       ?Compress@CLogSaveThread@@IAE_NXZ 00415ce0 f   rylgamelibrary:gamelog.obj
 0001:00014fc0       ??1CLogSaveThread@@UAE@XZ  00415fc0 f   rylgamelibrary:gamelog.obj
 0001:00015020       ?GetBuffer@CGameLog@@AAEPAULogBuffer@@XZ 00416020 f   rylgamelibrary:gamelog.obj
 0001:00015110       ??0CLogSaveThread@@QAE@XZ  00416110 f   rylgamelibrary:gamelog.obj
 0001:00015190       ??_ECLogSaveThread@@UAEPAXI@Z 00416190 f i rylgamelibrary:gamelog.obj
 0001:00015190       ??_GCLogSaveThread@@UAEPAXI@Z 00416190 f i rylgamelibrary:gamelog.obj
 0001:000151b0       ??0CGameLog@@QAE@XZ        004161b0 f   rylgamelibrary:gamelog.obj
 0001:00015240       ?_Incsize@?$list@PAULogBuffer@@V?$allocator@PAULogBuffer@@@std@@@std@@IAEXI@Z 00416240 f i rylgamelibrary:gamelog.obj
 0001:000152e0       ?Initialize@CGameLog@@QAE_NPBD@Z 004162e0 f   rylgamelibrary:gamelog.obj
 0001:00015420       ?PushFullBuffer@CGameLog@@AAEXPAPAULogBuffer@@@Z 00416420 f   rylgamelibrary:gamelog.obj
 0001:000154e0       ?_Splice@?$list@PAULogBuffer@@V?$allocator@PAULogBuffer@@@std@@@std@@QAEXViterator@12@AAV12@00I@Z 004164e0 f i rylgamelibrary:gamelog.obj
 0001:00015530       ?Flush@CGameLog@@QAEHXZ    00416530 f   rylgamelibrary:gamelog.obj
 0001:00015550       ?Destroy@CGameLog@@QAE_NXZ 00416550 f   rylgamelibrary:gamelog.obj
 0001:00015630       ?ReserveBuffer@CGameLog@@QAEPADG@Z 00416630 f   rylgamelibrary:gamelog.obj
 0001:000156c0       ?SpliceOutFullBuffer@CGameLog@@AAEXAAV?$list@PAULogBuffer@@V?$allocator@PAULogBuffer@@@std@@@std@@@Z 004166c0 f   rylgamelibrary:gamelog.obj
 0001:00015750       ?SpliceInFreeBuffer@CGameLog@@AAEXAAV?$list@PAULogBuffer@@V?$allocator@PAULogBuffer@@@std@@@std@@@Z 00416750 f   rylgamelibrary:gamelog.obj
 0001:000157e0       ??1CGameLog@@QAE@XZ        004167e0 f   rylgamelibrary:gamelog.obj
 0001:00015870       ?GetInstance@CGameLog@@SAAAV1@XZ 00416870 f   rylgamelibrary:gamelog.obj
 0001:000158d0       ?SetLogFileName@CLogSaveThread@@IAE_NXZ 004168d0 f   rylgamelibrary:gamelog.obj
 0001:00015a70       ?WriteLog@CLogSaveThread@@IAE_NXZ 00416a70 f   rylgamelibrary:gamelog.obj
 0001:00015b90       ?Run@CLogSaveThread@@MAEIXZ 00416b90 f   rylgamelibrary:gamelog.obj
 0001:00015bf0       ??0CTCPFactory@@QAE@XZ     00416bf0 f   rylgamelibrary:socketfactory.obj
 0001:00015c20       ??_GCTCPFactory@@UAEPAXI@Z 00416c20 f i rylgamelibrary:socketfactory.obj
 0001:00015c20       ??_ECTCPFactory@@UAEPAXI@Z 00416c20 f i rylgamelibrary:socketfactory.obj
 0001:00015c40       ?CreateSocket@CSocketFactory@@UAEIXZ 00416c40 f   rylgamelibrary:socketfactory.obj
 0001:00015c60       ?CreateConnectedSocket@CSocketFactory@@QAEIPBDG@Z 00416c60 f   rylgamelibrary:socketfactory.obj
 0001:00015ce0       ?CreateBindedSocket@CSocketFactory@@QAEIPBDG@Z 00416ce0 f   rylgamelibrary:socketfactory.obj
 0001:00015d80       ?CreateListenSocket@CSocketFactory@@QAEIPBDGH@Z 00416d80 f   rylgamelibrary:socketfactory.obj
 0001:00015dd0       ?SetAddr@CINETFamilyFactory@@UAE_NPAUsockaddr@@PBDG@Z 00416dd0 f   rylgamelibrary:socketfactory.obj
 0001:00015e50       ?GetNetworkInfo@CINETFamilyFactory@@UAE_NPADH@Z 00416e50 f   rylgamelibrary:socketfactory.obj
 0001:00015f30       ??1CBufferFactory@@UAE@XZ  00416f30 f i rylgamelibrary:bufferfactory.obj
 0001:00015f40       ??_ECBufferFactory@@UAEPAXI@Z 00416f40 f i rylgamelibrary:bufferfactory.obj
 0001:00015f40       ??_GCBufferFactory@@UAEPAXI@Z 00416f40 f i rylgamelibrary:bufferfactory.obj
 0001:00015f60       ?Release@CPoolBufferFactory@@UAEXPAVCBuffer@@@Z 00416f60 f   rylgamelibrary:bufferfactory.obj
 0001:00016000       ?_Ufill@?$vector@HV?$allocator@H@std@@@std@@IAEPAHPAHIABH@Z 00417000 f i rylgamelibrary:reloctable.obj
 0001:00016000       ?_Ufill@?$vector@PADV?$allocator@PAD@std@@@std@@IAEPAPADPAPADIABQAD@Z 00417000 f i rylgamelibrary:tokenlizedfile.obj
 0001:00016000       ?_Ufill@?$vector@KV?$allocator@K@std@@@std@@IAEPAKPAKIABK@Z 00417000 f i masterpassword.obj
 0001:00016000       ?_Ufill@?$vector@PAV?$pool@Udefault_user_allocator_new_delete@boost@@@boost@@V?$allocator@PAV?$pool@Udefault_user_allocator_new_delete@boost@@@boost@@@std@@@std@@IAEPAPAV?$pool@Udefault_user_allocator_new_delete@boost@@@boost@@PAPAV34@IABQAV34@@Z 00417000 f i rylgamelibrary:bufferfactory.obj
 0001:00016030       ??1?$vector@UColumnInfo@CTokenlizedFile@@V?$allocator@UColumnInfo@CTokenlizedFile@@@std@@@std@@QAE@XZ 00417030 f i rylgamelibrary:tokenlizedfile.obj
 0001:00016030       ??1?$vector@W4Type@ItemType@Item@@V?$allocator@W4Type@ItemType@Item@@@std@@@std@@QAE@XZ 00417030 f i rylgamelibrary:itemconstants.obj
 0001:00016030       ??1?$vector@KV?$allocator@K@std@@@std@@QAE@XZ 00417030 f i masterpassword.obj
 0001:00016030       ??1?$vector@PAV?$pool@Udefault_user_allocator_new_delete@boost@@@boost@@V?$allocator@PAV?$pool@Udefault_user_allocator_new_delete@boost@@@boost@@@std@@@std@@QAE@XZ 00417030 f i rylgamelibrary:bufferfactory.obj
 0001:00016030       ??1?$vector@UItemInfo@Item@@V?$allocator@UItemInfo@Item@@@std@@@std@@QAE@XZ 00417030 f i rylgamelibrary:itemmgr.obj
 0001:00016030       ??1?$vector@U?$pair@KK@std@@V?$allocator@U?$pair@KK@std@@@2@@std@@QAE@XZ 00417030 f i rylgamelibrary:rylserverdispatch.obj
 0001:00016030       ??1?$vector@UParseData@ItemDataParser@@V?$allocator@UParseData@ItemDataParser@@@std@@@std@@QAE@XZ 00417030 f i rylgamelibrary:itemmgr.obj
 0001:00016030       ??1?$vector@PADV?$allocator@PAD@std@@@std@@QAE@XZ 00417030 f i rylgamelibrary:tokenlizedfile.obj
 0001:00016060       ?Create@CPoolBufferFactory@@UAEPAVCBuffer@@I@Z 00417060 f   rylgamelibrary:bufferfactory.obj
 0001:00016140       ?Destroy@CPoolBufferFactory@@QAEXXZ 00417140 f   rylgamelibrary:bufferfactory.obj
 0001:00016200       ??1CPoolBufferFactory@@UAE@XZ 00417200 f   rylgamelibrary:bufferfactory.obj
 0001:00016250       ?_Xlen@?$vector@PAV?$pool@Udefault_user_allocator_new_delete@boost@@@boost@@V?$allocator@PAV?$pool@Udefault_user_allocator_new_delete@boost@@@boost@@@std@@@std@@IBEXXZ 00417250 f i rylgamelibrary:bufferfactory.obj
 0001:000162c0       ??_ECPoolBufferFactory@@UAEPAXI@Z 004172c0 f i rylgamelibrary:bufferfactory.obj
 0001:000162c0       ??_GCPoolBufferFactory@@UAEPAXI@Z 004172c0 f i rylgamelibrary:bufferfactory.obj
 0001:000162e0       ?_Insert_n@?$vector@PAV?$pool@Udefault_user_allocator_new_delete@boost@@@boost@@V?$allocator@PAV?$pool@Udefault_user_allocator_new_delete@boost@@@boost@@@std@@@std@@IAEXViterator@12@IABQAV?$pool@Udefault_user_allocator_new_delete@boost@@@boost@@@Z 004172e0 f i rylgamelibrary:bufferfactory.obj
 0001:000164c0       ?Initialize@CPoolBufferFactory@@IAE_NXZ 004174c0 f   rylgamelibrary:bufferfactory.obj
 0001:00016650       ??0CPoolBufferFactory@@QAE@XZ 00417650 f   rylgamelibrary:bufferfactory.obj
 0001:000166b0       ??_GCOverlappedFactory@@UAEPAXI@Z 004176b0 f i rylgamelibrary:overlapped.obj
 0001:000166b0       ??_ECOverlappedFactory@@UAEPAXI@Z 004176b0 f i rylgamelibrary:overlapped.obj
 0001:000166d0       ??0CSendOverlapped@@QAE@AAVCOverlappedFactory@@PAVCBuffer@@@Z 004176d0 f i rylgamelibrary:overlapped.obj
 0001:00016700       ?Dispatch@CSendOverlapped@@UAEXHKK@Z 00417700 f i rylgamelibrary:overlapped.obj
 0001:00016730       ??1CAcceptOverlapped@@UAE@XZ 00417730 f i rylgamelibrary:overlapped.obj
 0001:00016730       ??1CStreamRecvOverlapped@@UAE@XZ 00417730 f i rylgamelibrary:overlapped.obj
 0001:00016730       ??1CSendOverlapped@@UAE@XZ 00417730 f i rylgamelibrary:overlapped.obj
 0001:00016760       ??0CStreamRecvOverlapped@@QAE@AAVCOverlappedFactory@@@Z 00417760 f i rylgamelibrary:overlapped.obj
 0001:00016790       ??0CAcceptOverlapped@@QAE@AAVCOverlappedFactory@@AAVCListener@@IPAVCBuffer@@@Z 00417790 f i rylgamelibrary:overlapped.obj
 0001:000167d0       ?Dispatch@CAcceptOverlapped@@UAEXHKK@Z 004177d0 f i rylgamelibrary:overlapped.obj
 0001:00016800       ??_ECStreamRecvOverlapped@@UAEPAXI@Z 00417800 f i rylgamelibrary:overlapped.obj
 0001:00016800       ??_GCStreamRecvOverlapped@@UAEPAXI@Z 00417800 f i rylgamelibrary:overlapped.obj
 0001:00016800       ??_ECAcceptOverlapped@@UAEPAXI@Z 00417800 f i rylgamelibrary:overlapped.obj
 0001:00016800       ??_GCSendOverlapped@@UAEPAXI@Z 00417800 f i rylgamelibrary:overlapped.obj
 0001:00016800       ??_GCAcceptOverlapped@@UAEPAXI@Z 00417800 f i rylgamelibrary:overlapped.obj
 0001:00016800       ??_ECSendOverlapped@@UAEPAXI@Z 00417800 f i rylgamelibrary:overlapped.obj
 0001:00016820       ??_GCOverlapped@@UAEPAXI@Z 00417820 f i rylgamelibrary:overlapped.obj
 0001:00016820       ??_ECOverlapped@@UAEPAXI@Z 00417820 f i rylgamelibrary:overlapped.obj
 0001:00016860       ?Dispatch@CStreamRecvOverlapped@@UAEXHKK@Z 00417860 f i rylgamelibrary:overlapped.obj
 0001:00016890       ?Recv@CSession@@QAE_NXZ    00417890 f i rylgamelibrary:overlapped.obj
 0001:000168e0       ??0CStreamOverlappedFactory@@QAE@XZ 004178e0 f   rylgamelibrary:overlapped.obj
 0001:00016950       ?DeleteOverlapped@CStreamOverlappedFactory@@UAEXPAVCOverlapped@@@Z 00417950 f   rylgamelibrary:overlapped.obj
 0001:000169c0       ?CreateSend@CStreamOverlappedFactory@@UAEPAVCOverlapped@@PAVCSession@@PAVCBuffer@@@Z 004179c0 f   rylgamelibrary:overlapped.obj
 0001:00016a20       ?CreateRecv@CStreamOverlappedFactory@@UAEPAVCOverlapped@@PAVCSession@@PAVCBuffer@@@Z 00417a20 f   rylgamelibrary:overlapped.obj
 0001:00016a80       ?CreateAccept@CStreamOverlappedFactory@@UAEPAVCOverlapped@@PAVCListener@@IPAVCBuffer@@@Z 00417a80 f   rylgamelibrary:overlapped.obj
 0001:00016af0       ??1CStreamOverlappedFactory@@UAE@XZ 00417af0 f   rylgamelibrary:overlapped.obj
 0001:00016b40       ??_GCStreamOverlappedFactory@@UAEPAXI@Z 00417b40 f i rylgamelibrary:overlapped.obj
 0001:00016b40       ??_ECStreamOverlappedFactory@@UAEPAXI@Z 00417b40 f i rylgamelibrary:overlapped.obj
 0001:00016b60       ??0StringCMD@CConsoleCMDFactory@@QAE@PBDPAVCConsoleCommand@@@Z 00417b60 f   rylgamelibrary:consolecmdfactory.obj
 0001:00016ba0       ?size@?$vector@UColumnInfo@CTokenlizedFile@@V?$allocator@UColumnInfo@CTokenlizedFile@@@std@@@std@@QBEIXZ 00417ba0 f i rylgamelibrary:tokenlizedfile.obj
 0001:00016ba0       ?size@?$vector@UStringCMD@CConsoleCMDFactory@@V?$allocator@UStringCMD@CConsoleCMDFactory@@@std@@@std@@QBEIXZ 00417ba0 f i rylgamelibrary:consolecmdfactory.obj
 0001:00016bc0       ??$_Uninit_fill_n@PAUStringCMD@CConsoleCMDFactory@@IU12@V?$allocator@UStringCMD@CConsoleCMDFactory@@@std@@@std@@YAXPAUStringCMD@CConsoleCMDFactory@@IABU12@AAV?$allocator@UStringCMD@CConsoleCMDFactory@@@0@U_Nonscalar_ptr_iterator_tag@0@@Z 00417bc0 f i rylgamelibrary:consolecmdfactory.obj
 0001:00016bc0       ??$_Uninit_fill_n@PAUColumnInfo@CTokenlizedFile@@IU12@V?$allocator@UColumnInfo@CTokenlizedFile@@@std@@@std@@YAXPAUColumnInfo@CTokenlizedFile@@IABU12@AAV?$allocator@UColumnInfo@CTokenlizedFile@@@0@U_Nonscalar_ptr_iterator_tag@0@@Z 00417bc0 f i rylgamelibrary:tokenlizedfile.obj
 0001:00016c00       ?Create@CConsoleCMDFactory@@QAEPAVCConsoleCommand@@PBDI@Z 00417c00 f   rylgamelibrary:consolecmdfactory.obj
 0001:00016c70       ??1CConsoleCMDFactory@@UAE@XZ 00417c70 f   rylgamelibrary:consolecmdfactory.obj
 0001:00016cd0       ?_Xlen@?$vector@UStringCMD@CConsoleCMDFactory@@V?$allocator@UStringCMD@CConsoleCMDFactory@@@std@@@std@@IBEXXZ 00417cd0 f i rylgamelibrary:consolecmdfactory.obj
 0001:00016d40       ??_ECConsoleCMDFactory@@UAEPAXI@Z 00417d40 f i rylgamelibrary:consolecmdfactory.obj
 0001:00016d40       ??_GCConsoleCMDFactory@@UAEPAXI@Z 00417d40 f i rylgamelibrary:consolecmdfactory.obj
 0001:00016d60       ?_Insert_n@?$vector@UStringCMD@CConsoleCMDFactory@@V?$allocator@UStringCMD@CConsoleCMDFactory@@@std@@@std@@IAEXViterator@12@IABUStringCMD@CConsoleCMDFactory@@@Z 00417d60 f i rylgamelibrary:consolecmdfactory.obj
 0001:00017020       ?insert@?$vector@UStringCMD@CConsoleCMDFactory@@V?$allocator@UStringCMD@CConsoleCMDFactory@@@std@@@std@@QAE?AViterator@12@V312@ABUStringCMD@CConsoleCMDFactory@@@Z 00418020 f i rylgamelibrary:consolecmdfactory.obj
 0001:00017090       ??0CConsoleCMDFactory@@QAE@XZ 00418090 f   rylgamelibrary:consolecmdfactory.obj
 0001:000170b0       ?push_back@?$vector@UStringCMD@CConsoleCMDFactory@@V?$allocator@UStringCMD@CConsoleCMDFactory@@@std@@@std@@QAEXABUStringCMD@CConsoleCMDFactory@@@Z 004180b0 f i rylgamelibrary:consolecmdfactory.obj
 0001:00017130       ?AddCommand@CConsoleCMDFactory@@QAE_NPBDPAVCConsoleCommand@@@Z 00418130 f   rylgamelibrary:consolecmdfactory.obj
 0001:00017170       ?Clear@PacketData@CPacketStatistics@@QAEXXZ 00418170 f i rylgamelibrary:packetstatistics.obj
 0001:00017190       ?AddSendPacket@CPacketStatistics@@QAEXEK@Z 00418190 f   rylgamelibrary:packetstatistics.obj
 0001:000171d0       ?AddRecvPacket@CPacketStatistics@@QAEXEK@Z 004181d0 f   rylgamelibrary:packetstatistics.obj
 0001:00017200       ?Log@CPacketStatistics@@QAE_NXZ 00418200 f   rylgamelibrary:packetstatistics.obj
 0001:00017660       ??0CPacketStatistics@@AAE@XZ 00418660 f   rylgamelibrary:packetstatistics.obj
 0001:000176d0       ?GetInstance@CPacketStatistics@@SAAAV1@XZ 004186d0 f   rylgamelibrary:packetstatistics.obj
 0001:00017710       ?Clear@CPacketStatistics@@QAEXXZ 00418710 f   rylgamelibrary:packetstatistics.obj
 0001:00017760       ??_ECDLLModule@@UAEPAXI@Z  00418760 f i rylgamelibrary:exceptionreport.obj
 0001:00017760       ??_GCDLLModule@@UAEPAXI@Z  00418760 f i rylgamelibrary:exceptionreport.obj
 0001:00017790       ?Init@CDBGFuncClass@@UAEHPBD@Z 00418790 f i rylgamelibrary:exceptionreport.obj
 0001:00017990       ??1CDBGFuncClass@@UAE@XZ   00418990 f i rylgamelibrary:exceptionreport.obj
 0001:000179b0       ??_GCDBGFuncClass@@UAEPAXI@Z 004189b0 f i rylgamelibrary:exceptionreport.obj
 0001:000179b0       ??_ECDBGFuncClass@@UAEPAXI@Z 004189b0 f i rylgamelibrary:exceptionreport.obj
 0001:000179d0       ?WriteRegistersInfo@CExceptionReport@@SAHPADHPAU_CONTEXT@@@Z 004189d0 f   rylgamelibrary:exceptionreport.obj
 0001:00017a60       ?GetExceptionString@CExceptionReport@@CAPADK@Z 00418a60 f   rylgamelibrary:exceptionreport.obj
 0001:00017cf0       ?GetLogicalAddress@CExceptionReport@@CAHPAXPADKAAK2@Z 00418cf0 f   rylgamelibrary:exceptionreport.obj
 0001:00017dc0       ?FormatOutputValue@CExceptionReport@@CAHPADHW4BasicType@@_KPAX@Z 00418dc0 f   rylgamelibrary:exceptionreport.obj
 0001:00017f60       ?Dump@CExceptionReport@@SAHPADH_KKH@Z 00418f60 f   rylgamelibrary:exceptionreport.obj
 0001:000181f0       ?UnhandledSecondExceptionFilter@CExceptionReport@@CGJPAU_EXCEPTION_POINTERS@@@Z 004191f0 f i rylgamelibrary:exceptionreport.obj
 0001:00018240       ??1CExceptionReport@@AAE@XZ 00419240 f   rylgamelibrary:exceptionreport.obj
 0001:000182b0       ?WriteBasicInfo@CExceptionReport@@SAHPADHPAU_EXCEPTION_RECORD@@@Z 004192b0 f   rylgamelibrary:exceptionreport.obj
 0001:00018430       ?WriteMemoryDump@CExceptionReport@@SAHPADHPAU_CONTEXT@@II@Z 00419430 f   rylgamelibrary:exceptionreport.obj
 0001:00018510       ?DumpTypeIndex@CExceptionReport@@CAHPADH_KKIKAAH@Z 00419510 f   rylgamelibrary:exceptionreport.obj
 0001:00018820       ?FormatSymbolValue@CExceptionReport@@CAHPAU_SYMBOL_INFO@@PAU_tagSTACKFRAME@@PADI@Z 00419820 f   rylgamelibrary:exceptionreport.obj
 0001:00018930       ?EnumerateSymbolsCallback@CExceptionReport@@CGHPAU_SYMBOL_INFO@@KPAX@Z 00419930 f   rylgamelibrary:exceptionreport.obj
 0001:000189f0       ?WriteStackDetails@CExceptionReport@@SAHPADHPAU_CONTEXT@@HAAHH@Z 004199f0 f   rylgamelibrary:exceptionreport.obj
 0001:00018df0       ?WriteExceptionReport@CExceptionReport@@QAEXPAU_EXCEPTION_POINTERS@@@Z 00419df0 f   rylgamelibrary:exceptionreport.obj
 0001:00018fb0       ?ProcessException@CExceptionReport@@AAEJPAU_EXCEPTION_POINTERS@@@Z 00419fb0 f   rylgamelibrary:exceptionreport.obj
 0001:00019260       ?UnhandledExceptionFilter@CExceptionReport@@CGJPAU_EXCEPTION_POINTERS@@@Z 0041a260 f i rylgamelibrary:exceptionreport.obj
 0001:00019280       ?Enable@CExceptionReport@@QAEXK@Z 0041a280 f   rylgamelibrary:exceptionreport.obj
 0001:000192d0       ??0CExceptionReport@@AAE@XZ 0041a2d0 f   rylgamelibrary:exceptionreport.obj
 0001:000193e0       ?GetInstance@CExceptionReport@@SAAAV1@XZ 0041a3e0 f   rylgamelibrary:exceptionreport.obj
 0001:00019440       ?GetBasicType@CExceptionReport@@CA?AW4BasicType@@K_K@Z 0041a440 f   rylgamelibrary:exceptionreport.obj
 0001:000194d0       ?_Erase@?$_Tree@V?$_Tmap_traits@IPAVCMsgProc@@U?$less@I@std@@V?$allocator@U?$pair@$$CBIPAVCMsgProc@@@std@@@3@$0A@@std@@@std@@IAEXPAU_Node@?$_Tree_nod@V?$_Tmap_traits@IPAVCMsgProc@@U?$less@I@std@@V?$allocator@U?$pair@$$CBIPAVCMsgProc@@@std@@@3@$0A@@std@@@2@@Z 0041a4d0 f i rylgamelibrary:msgproc.obj
 0001:00019510       ?FindMsgProc@CMsgProcessMgr@@QAEPAVCMsgProc@@I@Z 0041a510 f   rylgamelibrary:msgproc.obj
 0001:00019540       ?Clear@CMsgProcessMgr@@QAEXXZ 0041a540 f   rylgamelibrary:msgproc.obj
 0001:000195c0       ?erase@?$_Tree@V?$_Tmap_traits@IPAVCMsgProc@@U?$less@I@std@@V?$allocator@U?$pair@$$CBIPAVCMsgProc@@@std@@@3@$0A@@std@@@std@@QAE?AViterator@12@V312@@Z 0041a5c0 f i rylgamelibrary:msgproc.obj
 0001:00019880       ?erase@?$_Tree@V?$_Tmap_traits@IPAVCMsgProc@@U?$less@I@std@@V?$allocator@U?$pair@$$CBIPAVCMsgProc@@@std@@@3@$0A@@std@@@std@@QAE?AViterator@12@V312@0@Z 0041a880 f i rylgamelibrary:msgproc.obj
 0001:00019940       ?_Insert@?$_Tree@V?$_Tmap_traits@IPAVCMsgProc@@U?$less@I@std@@V?$allocator@U?$pair@$$CBIPAVCMsgProc@@@std@@@3@$0A@@std@@@std@@IAE?AViterator@12@_NPAU_Node@?$_Tree_nod@V?$_Tmap_traits@IPAVCMsgProc@@U?$less@I@std@@V?$allocator@U?$pair@$$CBIPAVCMsgProc@@@std@@@3@$0A@@std@@@2@ABU?$pair@$$CBIPAVCMsgProc@@@2@@Z 0041a940 f i rylgamelibrary:msgproc.obj
 0001:00019af0       ?insert@?$_Tree@V?$_Tmap_traits@IPAVCMsgProc@@U?$less@I@std@@V?$allocator@U?$pair@$$CBIPAVCMsgProc@@@std@@@3@$0A@@std@@@std@@QAE?AU?$pair@Viterator@?$_Tree@V?$_Tmap_traits@IPAVCMsgProc@@U?$less@I@std@@V?$allocator@U?$pair@$$CBIPAVCMsgProc@@@std@@@3@$0A@@std@@@std@@_N@2@ABU?$pair@$$CBIPAVCMsgProc@@@2@@Z 0041aaf0 f i rylgamelibrary:msgproc.obj
 0001:00019bb0       ??1?$map@IPAVCMsgProc@@U?$less@I@std@@V?$allocator@U?$pair@$$CBIPAVCMsgProc@@@std@@@3@@std@@QAE@XZ 0041abb0 f i rylgamelibrary:msgproc.obj
 0001:00019be0       ??1CMsgProcessMgr@@QAE@XZ  0041abe0 f   rylgamelibrary:msgproc.obj
 0001:00019c50       ?Register@CMsgProcessMgr@@QAE_NIPAVCMsgProc@@@Z 0041ac50 f   rylgamelibrary:msgproc.obj
 0001:00019c80       ??0CMsgProcessMgr@@QAE@XZ  0041ac80 f   rylgamelibrary:msgproc.obj
 0001:00019cb0       ?Destroy@CConsoleWindow@@QAE_NXZ 0041acb0 f   rylgamelibrary:consolewindow.obj
 0001:00019d30       ??0CConsoleWindow@@QAE@PAUHINSTANCE__@@PAUHWND__@@AAVCConsoleCMDFactory@@AAVCCommandProcess@@@Z 0041ad30 f   rylgamelibrary:consolewindow.obj
 0001:00019df0       ?ConsoleWindowProc@CConsoleWindow@@CGJPAUHWND__@@IIJ@Z 0041adf0 f   rylgamelibrary:consolewindow.obj
 0001:00019f50       ?PrintOutput@CConsoleWindow@@QAEXPBDH@Z 0041af50 f   rylgamelibrary:consolewindow.obj
 0001:00019fd0       ?PrintInfo@CConsoleWindow@@QAEXPBDH@Z 0041afd0 f   rylgamelibrary:consolewindow.obj
 0001:0001a050       ??1CConsoleWindow@@UAE@XZ  0041b050 f   rylgamelibrary:consolewindow.obj
 0001:0001a090       ??_ECConsoleWindow@@UAEPAXI@Z 0041b090 f i rylgamelibrary:consolewindow.obj
 0001:0001a090       ??_GCConsoleWindow@@UAEPAXI@Z 0041b090 f i rylgamelibrary:consolewindow.obj
 0001:0001a0b0       ?CreateCommand@CConsoleWindow@@AAEXXZ 0041b0b0 f   rylgamelibrary:consolewindow.obj
 0001:0001a150       ?InputWindowProc@CConsoleWindow@@CGJPAUHWND__@@GGJ@Z 0041b150 f   rylgamelibrary:consolewindow.obj
 0001:0001a1d0       ?Initialize@CConsoleWindow@@QAE_NXZ 0041b1d0 f   rylgamelibrary:consolewindow.obj
 0001:0001a430       ??0CBufferQueue@@QAE@XZ    0041b430 f   rylgamelibrary:bufferqueue.obj
 0001:0001a450       ?enqueue@CBufferQueue@@QAE_NPAVCBuffer@@_N@Z 0041b450 f   rylgamelibrary:bufferqueue.obj
 0001:0001a4c0       ?dequeue@CBufferQueue@@QAEPAVCBuffer@@XZ 0041b4c0 f   rylgamelibrary:bufferqueue.obj
 0001:0001a500       ?clear@CBufferQueue@@QAEXXZ 0041b500 f   rylgamelibrary:bufferqueue.obj
 0001:0001a550       ?splice@CBufferQueue@@QAEXAAV1@_N@Z 0041b550 f   rylgamelibrary:bufferqueue.obj
 0001:0001a5d0       ??1CBufferQueue@@UAE@XZ    0041b5d0 f   rylgamelibrary:bufferqueue.obj
 0001:0001a5e0       ??_GCBufferQueue@@UAEPAXI@Z 0041b5e0 f i rylgamelibrary:bufferqueue.obj
 0001:0001a5e0       ??_ECBufferQueue@@UAEPAXI@Z 0041b5e0 f i rylgamelibrary:bufferqueue.obj
 0001:0001a610       ?XORF@CXORCrypt@@AAEXPADHGEE@Z 0041b610 f   rylgamelibrary:xorcrypt.obj
 0001:0001a680       ?XORB@CXORCrypt@@AAEXPADHGEE@Z 0041b680 f   rylgamelibrary:xorcrypt.obj
 0001:0001a6f0       ?InitCodePage@CXORCrypt@@AAEXXZ 0041b6f0 f   rylgamelibrary:xorcrypt.obj
 0001:0001a740       ?GetCodePage@CXORCrypt@@QAEKXZ 0041b740 f   rylgamelibrary:xorcrypt.obj
 0001:0001a780       ?EncodePacket@CXORCrypt@@QAE_NPADHK@Z 0041b780 f   rylgamelibrary:xorcrypt.obj
 0001:0001a7d0       ?DecodePacket@CXORCrypt@@QAE_NPADHK@Z 0041b7d0 f   rylgamelibrary:xorcrypt.obj
 0001:0001a820       ?EncodeHeader@CXORCrypt@@QAEXPADHGE@Z 0041b820 f   rylgamelibrary:xorcrypt.obj
 0001:0001a880       ?DecodeHeader@CXORCrypt@@QAEXPADHGE@Z 0041b880 f   rylgamelibrary:xorcrypt.obj
 0001:0001a8e0       ??0CXORCrypt@@AAE@XZ       0041b8e0 f   rylgamelibrary:xorcrypt.obj
 0001:0001a900       ??1CXORCrypt@@QAE@XZ       0041b900 f   rylgamelibrary:xorcrypt.obj
 0001:0001a910       ?Decompress@CMiniLZO@@YA_NPBDKPADPAK@Z 0041b910 f   rylgamelibrary:minilzowrapper.obj
 0001:0001a940       ?SetProgramName@DbgUtils@@YAXPADH0@Z 0041b940 f   rylgamelibrary:debugutils.obj
 0001:0001aa00       ?WrapHeader@PacketWrap@@YA_NPADGEGG@Z 0041ba00 f   rylgamelibrary:wrappacket.obj
 0001:0001aa50       ?WrapCrypt@PacketWrap@@YA_NPADGEGG@Z 0041ba50 f   rylgamelibrary:wrappacket.obj
 0001:0001aad0       ?_Incref@facet@locale@std@@QAEXXZ 0041bad0 f i rylgamelibrary:regfunctions.obj
 0001:0001ab00       ?_Decref@facet@locale@std@@QAEPAV123@XZ 0041bb00 f i rylgamelibrary:regfunctions.obj
 0001:0001ab40       ??1ctype_base@std@@UAE@XZ  0041bb40 f i rylgamelibrary:regfunctions.obj
 0001:0001ab40       ??1facet@locale@std@@UAE@XZ 0041bb40 f i rylgamelibrary:regfunctions.obj
 0001:0001ab40       ??1?$codecvt@DDH@std@@MAE@XZ 0041bb40 f i rylgamelibrary:regfunctions.obj
 0001:0001ab40       ??1codecvt_base@std@@UAE@XZ 0041bb40 f i rylgamelibrary:regfunctions.obj
 0001:0001ab50       ??1locale@std@@QAE@XZ      0041bb50 f i rylgamelibrary:regfunctions.obj
 0001:0001ab70       ??_Gfacet@locale@std@@UAEPAXI@Z 0041bb70 f i rylgamelibrary:regfunctions.obj
 0001:0001ab70       ??_Efacet@locale@std@@UAEPAXI@Z 0041bb70 f i rylgamelibrary:regfunctions.obj
 0001:0001ab90       ?do_max_length@codecvt_base@std@@MBEHXZ 0041bb90 f i rylgamelibrary:regfunctions.obj
 0001:0001ab90       ?do_encoding@codecvt_base@std@@MBEHXZ 0041bb90 f i rylgamelibrary:regfunctions.obj
 0001:0001aba0       ?getloc@ios_base@std@@QBE?AVlocale@2@XZ 0041bba0 f i rylgamelibrary:regfunctions.obj
 0001:0001abe0       ??_Eios_base@std@@UAEPAXI@Z 0041bbe0 f i rylgamelibrary:regfunctions.obj
 0001:0001abe0       ??_Gios_base@std@@UAEPAXI@Z 0041bbe0 f i rylgamelibrary:regfunctions.obj
 0001:0001ac00       ?ReadInt@Registry@@YAKPBD00@Z 0041bc00 f   rylgamelibrary:regfunctions.obj
 0001:0001ac20       ?ReadString@Registry@@YA_NPBD00PADH@Z 0041bc20 f   rylgamelibrary:regfunctions.obj
 0001:0001ac50       ??1?$basic_ios@DU?$char_traits@D@std@@@std@@UAE@XZ 0041bc50 f i rylgamelibrary:regfunctions.obj
 0001:0001ac60       ??_G?$basic_ios@DU?$char_traits@D@std@@@std@@UAEPAXI@Z 0041bc60 f i rylgamelibrary:regfunctions.obj
 0001:0001ac60       ??_E?$basic_ios@DU?$char_traits@D@std@@@std@@UAEPAXI@Z 0041bc60 f i rylgamelibrary:regfunctions.obj
 0001:0001ac80       ??0?$ctype@D@std@@QAE@PBF_NI@Z 0041bc80 f i rylgamelibrary:regfunctions.obj
 0001:0001ad60       ?do_tolower@?$ctype@D@std@@MBEDD@Z 0041bd60 f i rylgamelibrary:regfunctions.obj
 0001:0001ad80       ?do_tolower@?$ctype@D@std@@MBEPBDPADPBD@Z 0041bd80 f i rylgamelibrary:regfunctions.obj
 0001:0001adb0       ?do_toupper@?$ctype@D@std@@MBEDD@Z 0041bdb0 f i rylgamelibrary:regfunctions.obj
 0001:0001add0       ?do_toupper@?$ctype@D@std@@MBEPBDPADPBD@Z 0041bdd0 f i rylgamelibrary:regfunctions.obj
 0001:0001ae00       ?do_widen@?$ctype@D@std@@MBEDD@Z 0041be00 f i rylgamelibrary:regfunctions.obj
 0001:0001ae10       ?do_widen@?$ctype@D@std@@MBEPBDPBD0PAD@Z 0041be10 f i rylgamelibrary:regfunctions.obj
 0001:0001ae40       ?do_narrow@?$ctype@D@std@@MBEDDD@Z 0041be40 f i rylgamelibrary:regfunctions.obj
 0001:0001ae50       ?do_narrow@?$ctype@D@std@@MBEPBDPBD0DPAD@Z 0041be50 f i rylgamelibrary:regfunctions.obj
 0001:0001ae80       ?_Getcat@?$ctype@D@std@@SAIPAPBVfacet@locale@2@@Z 0041be80 f i rylgamelibrary:regfunctions.obj
 0001:0001aef0       ??_G?$ctype@D@std@@MAEPAXI@Z 0041bef0 f i rylgamelibrary:regfunctions.obj
 0001:0001aef0       ??_E?$ctype@D@std@@MAEPAXI@Z 0041bef0 f i rylgamelibrary:regfunctions.obj
 0001:0001af10       ??1?$ctype@D@std@@MAE@XZ   0041bf10 f i rylgamelibrary:regfunctions.obj
 0001:0001af50       ??1?$basic_streambuf@DU?$char_traits@D@std@@@std@@UAE@XZ 0041bf50 f i rylgamelibrary:regfunctions.obj
 0001:0001afc0       ?pbackfail@?$basic_streambuf@DU?$char_traits@D@std@@@std@@MAEHH@Z 0041bfc0 f i rylgamelibrary:regfunctions.obj
 0001:0001afc0       ?overflow@?$basic_streambuf@DU?$char_traits@D@std@@@std@@MAEHH@Z 0041bfc0 f i rylgamelibrary:regfunctions.obj
 0001:0001afd0       ?sync@?$basic_streambuf@DU?$char_traits@D@std@@@std@@MAEHXZ 0041bfd0 f i rylgamelibrary:regfunctions.obj
 0001:0001afd0       ?GetDefaultStartGold@CharCreate@@YAKXZ 0041bfd0 f i rylgamelibrary:charactercreate.obj
 0001:0001afd0       ?showmanyc@?$basic_streambuf@DU?$char_traits@D@std@@@std@@MAEHXZ 0041bfd0 f i rylgamelibrary:regfunctions.obj
 0001:0001afe0       ?underflow@?$basic_streambuf@DU?$char_traits@D@std@@@std@@MAEHXZ 0041bfe0 f i rylgamelibrary:regfunctions.obj
 0001:0001aff0       ?setbuf@?$basic_streambuf@DU?$char_traits@D@std@@@std@@MAEPAV12@PADH@Z 0041bff0 f i rylgamelibrary:regfunctions.obj
 0001:0001b000       ?imbue@?$basic_streambuf@DU?$char_traits@D@std@@@std@@MAEXABVlocale@2@@Z 0041c000 f i rylgamelibrary:regfunctions.obj
 0001:0001b010       ?uflow@?$basic_streambuf@DU?$char_traits@D@std@@@std@@MAEHXZ 0041c010 f i rylgamelibrary:regfunctions.obj
 0001:0001b040       ?xsgetn@?$basic_streambuf@DU?$char_traits@D@std@@@std@@MAEHPADH@Z 0041c040 f i rylgamelibrary:regfunctions.obj
 0001:0001b0e0       ?xsputn@?$basic_streambuf@DU?$char_traits@D@std@@@std@@MAEHPBDH@Z 0041c0e0 f i rylgamelibrary:regfunctions.obj
 0001:0001b190       ?seekoff@?$basic_streambuf@DU?$char_traits@D@std@@@std@@MAE?AV?$fpos@H@2@JHH@Z 0041c190 f i rylgamelibrary:regfunctions.obj
 0001:0001b1c0       ?seekpos@?$basic_streambuf@DU?$char_traits@D@std@@@std@@MAE?AV?$fpos@H@2@V32@H@Z 0041c1c0 f i rylgamelibrary:regfunctions.obj
 0001:0001b1f0       ??_G?$basic_ostream@DU?$char_traits@D@std@@@std@@UAEPAXI@Z 0041c1f0 f i rylgamelibrary:regfunctions.obj
 0001:0001b1f0       ??_E?$basic_ostream@DU?$char_traits@D@std@@@std@@UAEPAXI@Z 0041c1f0 f i rylgamelibrary:regfunctions.obj
 0001:0001b220       ??_G?$basic_streambuf@DU?$char_traits@D@std@@@std@@UAEPAXI@Z 0041c220 f i rylgamelibrary:regfunctions.obj
 0001:0001b220       ??_E?$basic_streambuf@DU?$char_traits@D@std@@@std@@UAEPAXI@Z 0041c220 f i rylgamelibrary:regfunctions.obj
 0001:0001b240       ?_Init@?$basic_streambuf@DU?$char_traits@D@std@@@std@@IAEXXZ 0041c240 f i rylgamelibrary:regfunctions.obj
 0001:0001b2a0       ??$use_facet@V?$ctype@D@std@@@std@@YAABV?$ctype@D@0@ABVlocale@0@@Z 0041c2a0 f i rylgamelibrary:regfunctions.obj
 0001:0001b3b0       ??0?$codecvt@DDH@std@@QAE@I@Z 0041c3b0 f i rylgamelibrary:regfunctions.obj
 0001:0001b420       ?do_out@?$codecvt@DDH@std@@MBEHAAHPBD1AAPBDPAD3AAPAD@Z 0041c420 f i rylgamelibrary:regfunctions.obj
 0001:0001b420       ?do_in@?$codecvt@DDH@std@@MBEHAAHPBD1AAPBDPAD3AAPAD@Z 0041c420 f i rylgamelibrary:regfunctions.obj
 0001:0001b440       ?do_unshift@?$codecvt@DDH@std@@MBEHAAHPAD1AAPAD@Z 0041c440 f i rylgamelibrary:regfunctions.obj
 0001:0001b450       ?do_length@?$codecvt@DDH@std@@MBEHABHPBD1I@Z 0041c450 f i rylgamelibrary:regfunctions.obj
 0001:0001b470       ??_E?$codecvt@DDH@std@@MAEPAXI@Z 0041c470 f i rylgamelibrary:regfunctions.obj
 0001:0001b470       ??_G?$codecvt@DDH@std@@MAEPAXI@Z 0041c470 f i rylgamelibrary:regfunctions.obj
 0001:0001b490       ??0?$basic_string@DU?$char_traits@D@std@@V?$allocator@D@2@@std@@QAE@XZ 0041c490 f i rylgamelibrary:regfunctions.obj
 0001:0001b4b0       ?_Initcvt@?$basic_filebuf@DU?$char_traits@D@std@@@std@@IAEXPAV?$codecvt@DDH@2@@Z 0041c4b0 f i rylgamelibrary:regfunctions.obj
 0001:0001b520       ??0?$basic_streambuf@DU?$char_traits@D@std@@@std@@IAE@XZ 0041c520 f i rylgamelibrary:regfunctions.obj
 0001:0001b590       ?widen@?$basic_ios@DU?$char_traits@D@std@@@std@@QBEDD@Z 0041c590 f i rylgamelibrary:regfunctions.obj
 0001:0001b640       ?_Getcat@?$codecvt@DDH@std@@SAIPAPBVfacet@locale@2@@Z 0041c640 f i rylgamelibrary:regfunctions.obj
 0001:0001b6b0       ??0?$basic_filebuf@DU?$char_traits@D@std@@@std@@QAE@PAU_iobuf@@@Z 0041c6b0 f i rylgamelibrary:regfunctions.obj
 0001:0001b710       ?setbuf@?$basic_filebuf@DU?$char_traits@D@std@@@std@@MAEPAV?$basic_streambuf@DU?$char_traits@D@std@@@2@PADH@Z 0041c710 f i rylgamelibrary:regfunctions.obj
 0001:0001b760       ?sync@?$basic_filebuf@DU?$char_traits@D@std@@@std@@MAEHXZ 0041c760 f i rylgamelibrary:regfunctions.obj
 0001:0001b790       ?pbackfail@?$basic_filebuf@DU?$char_traits@D@std@@@std@@MAEHH@Z 0041c790 f i rylgamelibrary:regfunctions.obj
 0001:0001b830       ?_Gndec@?$basic_streambuf@DU?$char_traits@D@std@@@std@@IAEPADXZ 0041c830 f i rylgamelibrary:regfunctions.obj
 0001:0001b840       ?underflow@?$basic_filebuf@DU?$char_traits@D@std@@@std@@MAEHXZ 0041c840 f i rylgamelibrary:regfunctions.obj
 0001:0001b890       ?init@?$basic_ios@DU?$char_traits@D@std@@@std@@IAEXPAV?$basic_streambuf@DU?$char_traits@D@std@@@2@_N@Z 0041c890 f i rylgamelibrary:regfunctions.obj
 0001:0001b8f0       ??$use_facet@V?$codecvt@DDH@std@@@std@@YAABV?$codecvt@DDH@0@ABVlocale@0@@Z 0041c8f0 f i rylgamelibrary:regfunctions.obj
 0001:0001ba00       ?imbue@?$basic_filebuf@DU?$char_traits@D@std@@@std@@MAEXABVlocale@2@@Z 0041ca00 f i rylgamelibrary:regfunctions.obj
 0001:0001ba20       ?append@?$basic_string@DU?$char_traits@D@std@@V?$allocator@D@2@@std@@QAEAAV12@ID@Z 0041ca20 f i rylgamelibrary:regfunctions.obj
 0001:0001baf0       ?_Endwrite@?$basic_filebuf@DU?$char_traits@D@std@@@std@@IAE_NXZ 0041caf0 f i rylgamelibrary:regfunctions.obj
 0001:0001bc40       ??0?$basic_ostream@DU?$char_traits@D@std@@@std@@QAE@PAV?$basic_streambuf@DU?$char_traits@D@std@@@1@_N@Z 0041cc40 f i rylgamelibrary:regfunctions.obj
 0001:0001bcc0       ?overflow@?$basic_filebuf@DU?$char_traits@D@std@@@std@@MAEHH@Z 0041ccc0 f i rylgamelibrary:regfunctions.obj
 0001:0001bec0       ?uflow@?$basic_filebuf@DU?$char_traits@D@std@@@std@@MAEHXZ 0041cec0 f i rylgamelibrary:regfunctions.obj
 0001:0001c080       ?seekoff@?$basic_filebuf@DU?$char_traits@D@std@@@std@@MAE?AV?$fpos@H@2@JHH@Z 0041d080 f i rylgamelibrary:regfunctions.obj
 0001:0001c1c0       ?seekpos@?$basic_filebuf@DU?$char_traits@D@std@@@std@@MAE?AV?$fpos@H@2@V32@H@Z 0041d1c0 f i rylgamelibrary:regfunctions.obj
 0001:0001c2d0       ?close@?$basic_filebuf@DU?$char_traits@D@std@@@std@@QAEPAV12@XZ 0041d2d0 f i rylgamelibrary:regfunctions.obj
 0001:0001c330       ??1?$basic_filebuf@DU?$char_traits@D@std@@@std@@UAE@XZ 0041d330 f i rylgamelibrary:regfunctions.obj
 0001:0001c3c0       ??_G?$basic_filebuf@DU?$char_traits@D@std@@@std@@UAEPAXI@Z 0041d3c0 f i rylgamelibrary:regfunctions.obj
 0001:0001c3c0       ??_E?$basic_filebuf@DU?$char_traits@D@std@@@std@@UAEPAXI@Z 0041d3c0 f i rylgamelibrary:regfunctions.obj
 0001:0001c3e0       ?instance@?$singleton_default@Upool_type@?$singleton_pool@Ufast_pool_allocator_tag@boost@@$0M@Udefault_user_allocator_new_delete@2@Vwin32_mutex@pool@details@2@$0CA@@boost@@@pool@details@boost@@SAAAUpool_type@?$singleton_pool@Ufast_pool_allocator_tag@boost@@$0M@Udefault_user_allocator_new_delete@2@Vwin32_mutex@pool@details@2@$0CA@@4@XZ 0041d3e0 f i rylgamelibrary:depositcontainer.obj
 0001:0001c440       ??0CBuffer@@QAE@AAVCBufferFactory@@@Z 0041d440 f   rylgamelibrary:buffer.obj
 0001:0001c470       ?init@CBuffer@@QAEXPADK@Z  0041d470 f   rylgamelibrary:buffer.obj
 0001:0001c4b0       ?pop_read_data@CBuffer@@QAEXXZ 0041d4b0 f   rylgamelibrary:buffer.obj
 0001:0001c4e0       ?ComplexRandom@Random@Math@@YAKHH@Z 0041d4e0 f   rylgamelibrary:math.obj
 0001:0001c5b0       ?SimpleRandom@Random@Math@@YAHKHH@Z 0041d5b0 f   rylgamelibrary:math.obj
 0001:0001c5e0       ??0OleDB@@QAE@XZ           0041d5e0 f   rylgamelibrary:oledb.obj
 0001:0001c640       ??1OleDB@@UAE@XZ           0041d640 f   rylgamelibrary:oledb.obj
 0001:0001c6d0       ?HandleError@OleDB@@AAE_NHJPAD@Z 0041d6d0 f   rylgamelibrary:oledb.obj
 0001:0001c830       ?CreateSession@OleDB@@AAE_NXZ 0041d830 f   rylgamelibrary:oledb.obj
 0001:0001c8e0       ?DBCreateCommand@OleDB@@AAE_NXZ 0041d8e0 f   rylgamelibrary:oledb.obj
 0001:0001c9c0       ?AllocResultCols@OleDB@@AAE_NPAUIUnknown@@AAU_RESULT_COLS@1@@Z 0041d9c0 f   rylgamelibrary:oledb.obj
 0001:0001ca30       ?ReleaseResultCols@OleDB@@AAE_NPAUIUnknown@@AAU_RESULT_COLS@1@@Z 0041da30 f   rylgamelibrary:oledb.obj
 0001:0001cab0       ?SetConnectionProperties@OleDB@@AAE_NPBD000@Z 0041dab0 f   rylgamelibrary:oledb.obj
 0001:0001cf00       ?AllocBindGetData@OleDB@@AAEPAUtagDBBINDING@@HPAUtagDBCOLUMNINFO@@@Z 0041df00 f   rylgamelibrary:oledb.obj
 0001:0001cf80       ?AllocBindParamInputData@OleDB@@AAEPAUtagDBBINDING@@AAU_PARAM_INFO@1@@Z 0041df80 f   rylgamelibrary:oledb.obj
 0001:0001d020       ??_EOleDB@@UAEPAXI@Z       0041e020 f i rylgamelibrary:oledb.obj
 0001:0001d020       ??_GOleDB@@UAEPAXI@Z       0041e020 f i rylgamelibrary:oledb.obj
 0001:0001d040       ?ConnectSQLServer@OleDB@@QAE_NPBD000W4ConnType@1@@Z 0041e040 f   rylgamelibrary:oledb.obj
 0001:0001d1c0       ?ExcuteQueryWithParams@OleDB@@QAE_NPBDPADAAU_PARAM_INFO@1@@Z 0041e1c0 f   rylgamelibrary:oledb.obj
 0001:0001d500       ?ExcuteQueryGetData@OleDB@@QAE_NPBDPAX@Z 0041e500 f   rylgamelibrary:oledb.obj
 0001:0001d950       ?trim_string@@YAPADPAD@Z   0041e950 f   rylgamelibrary:tokenlizedfile.obj
 0001:0001d9a0       ??$fill@PAUStringCMD@CConsoleCMDFactory@@U12@@std@@YAXPAUStringCMD@CConsoleCMDFactory@@0ABU12@@Z 0041e9a0 f i rylgamelibrary:consolecmdfactory.obj
 0001:0001d9a0       ??$fill@PAUColumnInfo@CTokenlizedFile@@U12@@std@@YAXPAUColumnInfo@CTokenlizedFile@@0ABU12@@Z 0041e9a0 f i rylgamelibrary:tokenlizedfile.obj
 0001:0001d9e0       ??$_Copy_backward_opt@PAUColumnInfo@CTokenlizedFile@@PAU12@@std@@YAPAUColumnInfo@CTokenlizedFile@@PAU12@00U_Nonscalar_ptr_iterator_tag@0@@Z 0041e9e0 f i rylgamelibrary:tokenlizedfile.obj
 0001:0001d9e0       ??$_Copy_backward_opt@PAUStringCMD@CConsoleCMDFactory@@PAU12@@std@@YAPAUStringCMD@CConsoleCMDFactory@@PAU12@00U_Nonscalar_ptr_iterator_tag@0@@Z 0041e9e0 f i rylgamelibrary:consolecmdfactory.obj
 0001:0001da20       ??$_Med3@Viterator@?$vector@UColumnInfo@CTokenlizedFile@@V?$allocator@UColumnInfo@CTokenlizedFile@@@std@@@std@@@std@@YAXViterator@?$vector@UColumnInfo@CTokenlizedFile@@V?$allocator@UColumnInfo@CTokenlizedFile@@@std@@@0@00@Z 0041ea20 f i rylgamelibrary:tokenlizedfile.obj
 0001:0001dad0       ??$_Push_heap@Viterator@?$vector@UColumnInfo@CTokenlizedFile@@V?$allocator@UColumnInfo@CTokenlizedFile@@@std@@@std@@HUColumnInfo@CTokenlizedFile@@@std@@YAXViterator@?$vector@UColumnInfo@CTokenlizedFile@@V?$allocator@UColumnInfo@CTokenlizedFile@@@std@@@0@HHUColumnInfo@CTokenlizedFile@@@Z 0041ead0 f i rylgamelibrary:tokenlizedfile.obj
 0001:0001db40       ??$_Rotate@Viterator@?$vector@UColumnInfo@CTokenlizedFile@@V?$allocator@UColumnInfo@CTokenlizedFile@@@std@@@std@@HUColumnInfo@CTokenlizedFile@@@std@@YAXViterator@?$vector@UColumnInfo@CTokenlizedFile@@V?$allocator@UColumnInfo@CTokenlizedFile@@@std@@@0@00PAHPAUColumnInfo@CTokenlizedFile@@@Z 0041eb40 f i rylgamelibrary:tokenlizedfile.obj
 0001:0001dc70       ??$_Uninit_copy@Viterator@?$vector@UColumnInfo@CTokenlizedFile@@V?$allocator@UColumnInfo@CTokenlizedFile@@@std@@@std@@PAUColumnInfo@CTokenlizedFile@@V?$allocator@UColumnInfo@CTokenlizedFile@@@3@@std@@YAPAUColumnInfo@CTokenlizedFile@@Viterator@?$vector@UColumnInfo@CTokenlizedFile@@V?$allocator@UColumnInfo@CTokenlizedFile@@@std@@@0@0PAU12@AAV?$allocator@UColumnInfo@CTokenlizedFile@@@0@U_Nonscalar_ptr_iterator_tag@0@@Z 0041ec70 f i rylgamelibrary:tokenlizedfile.obj
 0001:0001dc70       ??$_Uninit_copy@PAUStringCMD@CConsoleCMDFactory@@PAU12@V?$allocator@UStringCMD@CConsoleCMDFactory@@@std@@@std@@YAPAUStringCMD@CConsoleCMDFactory@@PAU12@00AAV?$allocator@UStringCMD@CConsoleCMDFactory@@@0@U_Nonscalar_ptr_iterator_tag@0@@Z 0041ec70 f i rylgamelibrary:consolecmdfactory.obj
 0001:0001dc70       ??$_Uninit_copy@PAUColumnInfo@CTokenlizedFile@@PAU12@V?$allocator@UColumnInfo@CTokenlizedFile@@@std@@@std@@YAPAUColumnInfo@CTokenlizedFile@@PAU12@00AAV?$allocator@UColumnInfo@CTokenlizedFile@@@0@U_Nonscalar_ptr_iterator_tag@0@@Z 0041ec70 f i rylgamelibrary:tokenlizedfile.obj
 0001:0001dcb0       ??$_Median@Viterator@?$vector@UColumnInfo@CTokenlizedFile@@V?$allocator@UColumnInfo@CTokenlizedFile@@@std@@@std@@@std@@YAXViterator@?$vector@UColumnInfo@CTokenlizedFile@@V?$allocator@UColumnInfo@CTokenlizedFile@@@std@@@0@00@Z 0041ecb0 f i rylgamelibrary:tokenlizedfile.obj
 0001:0001dd50       ??$_Lower_bound@Viterator@?$vector@UColumnInfo@CTokenlizedFile@@V?$allocator@UColumnInfo@CTokenlizedFile@@@std@@@std@@UColumnInfo@CTokenlizedFile@@H@std@@YA?AViterator@?$vector@UColumnInfo@CTokenlizedFile@@V?$allocator@UColumnInfo@CTokenlizedFile@@@std@@@0@V120@0ABUColumnInfo@CTokenlizedFile@@PAH@Z 0041ed50 f i rylgamelibrary:tokenlizedfile.obj
 0001:0001ddb0       ??$_Upper_bound@Viterator@?$vector@UColumnInfo@CTokenlizedFile@@V?$allocator@UColumnInfo@CTokenlizedFile@@@std@@@std@@UColumnInfo@CTokenlizedFile@@H@std@@YA?AViterator@?$vector@UColumnInfo@CTokenlizedFile@@V?$allocator@UColumnInfo@CTokenlizedFile@@@std@@@0@V120@0ABUColumnInfo@CTokenlizedFile@@PAH@Z 0041edb0 f i rylgamelibrary:tokenlizedfile.obj
 0001:0001de10       ??$_Adjust_heap@Viterator@?$vector@UColumnInfo@CTokenlizedFile@@V?$allocator@UColumnInfo@CTokenlizedFile@@@std@@@std@@HUColumnInfo@CTokenlizedFile@@@std@@YAXViterator@?$vector@UColumnInfo@CTokenlizedFile@@V?$allocator@UColumnInfo@CTokenlizedFile@@@std@@@0@HHUColumnInfo@CTokenlizedFile@@@Z 0041ee10 f i rylgamelibrary:tokenlizedfile.obj
 0001:0001dec0       ??$_Unguarded_partition@Viterator@?$vector@UColumnInfo@CTokenlizedFile@@V?$allocator@UColumnInfo@CTokenlizedFile@@@std@@@std@@@std@@YA?AU?$pair@Viterator@?$vector@UColumnInfo@CTokenlizedFile@@V?$allocator@UColumnInfo@CTokenlizedFile@@@std@@@std@@V123@@0@Viterator@?$vector@UColumnInfo@CTokenlizedFile@@V?$allocator@UColumnInfo@CTokenlizedFile@@@std@@@0@0@Z 0041eec0 f i rylgamelibrary:tokenlizedfile.obj
 0001:0001e1a0       ??$_Make_heap@Viterator@?$vector@UColumnInfo@CTokenlizedFile@@V?$allocator@UColumnInfo@CTokenlizedFile@@@std@@@std@@HUColumnInfo@CTokenlizedFile@@@std@@YAXViterator@?$vector@UColumnInfo@CTokenlizedFile@@V?$allocator@UColumnInfo@CTokenlizedFile@@@std@@@0@0PAHPAUColumnInfo@CTokenlizedFile@@@Z 0041f1a0 f i rylgamelibrary:tokenlizedfile.obj
 0001:0001e210       ??$_Equal_range@Viterator@?$vector@UColumnInfo@CTokenlizedFile@@V?$allocator@UColumnInfo@CTokenlizedFile@@@std@@@std@@UColumnInfo@CTokenlizedFile@@H@std@@YA?AU?$pair@Viterator@?$vector@UColumnInfo@CTokenlizedFile@@V?$allocator@UColumnInfo@CTokenlizedFile@@@std@@@std@@V123@@0@Viterator@?$vector@UColumnInfo@CTokenlizedFile@@V?$allocator@UColumnInfo@CTokenlizedFile@@@std@@@0@0ABUColumnInfo@CTokenlizedFile@@PAH@Z 0041f210 f i rylgamelibrary:tokenlizedfile.obj
 0001:0001e2c0       ??$_Insertion_sort@Viterator@?$vector@UColumnInfo@CTokenlizedFile@@V?$allocator@UColumnInfo@CTokenlizedFile@@@std@@@std@@@std@@YAXViterator@?$vector@UColumnInfo@CTokenlizedFile@@V?$allocator@UColumnInfo@CTokenlizedFile@@@std@@@0@0@Z 0041f2c0 f i rylgamelibrary:tokenlizedfile.obj
 0001:0001e340       ?_Ufill@?$vector@UColumnInfo@CTokenlizedFile@@V?$allocator@UColumnInfo@CTokenlizedFile@@@std@@@std@@IAEPAUColumnInfo@CTokenlizedFile@@PAU34@IABU34@@Z 0041f340 f i rylgamelibrary:tokenlizedfile.obj
 0001:0001e340       ?_Ufill@?$vector@UStringCMD@CConsoleCMDFactory@@V?$allocator@UStringCMD@CConsoleCMDFactory@@@std@@@std@@IAEPAUStringCMD@CConsoleCMDFactory@@PAU34@IABU34@@Z 0041f340 f i rylgamelibrary:consolecmdfactory.obj
 0001:0001e370       ??$sort_heap@Viterator@?$vector@UColumnInfo@CTokenlizedFile@@V?$allocator@UColumnInfo@CTokenlizedFile@@@std@@@std@@@std@@YAXViterator@?$vector@UColumnInfo@CTokenlizedFile@@V?$allocator@UColumnInfo@CTokenlizedFile@@@std@@@0@0@Z 0041f370 f i rylgamelibrary:tokenlizedfile.obj
 0001:0001e410       ??1CTokenlizedFile@@QAE@XZ 0041f410 f   rylgamelibrary:tokenlizedfile.obj
 0001:0001e470       ?Close@CTokenlizedFile@@QAEXXZ 0041f470 f   rylgamelibrary:tokenlizedfile.obj
 0001:0001e4e0       ?Open@CTokenlizedFile@@QAE_NPBD0@Z 0041f4e0 f   rylgamelibrary:tokenlizedfile.obj
 0001:0001e510       ?GetStringValue@CTokenlizedFile@@QAEPBDPBD@Z 0041f510 f   rylgamelibrary:tokenlizedfile.obj
 0001:0001e600       ?_Xlen@?$vector@UColumnInfo@CTokenlizedFile@@V?$allocator@UColumnInfo@CTokenlizedFile@@@std@@@std@@IBEXXZ 0041f600 f i rylgamelibrary:tokenlizedfile.obj
 0001:0001e600       ?_Xlen@?$vector@PADV?$allocator@PAD@std@@@std@@IBEXXZ 0041f600 f i rylgamelibrary:tokenlizedfile.obj
 0001:0001e670       ?_Insert_n@?$vector@UColumnInfo@CTokenlizedFile@@V?$allocator@UColumnInfo@CTokenlizedFile@@@std@@@std@@IAEXViterator@12@IABUColumnInfo@CTokenlizedFile@@@Z 0041f670 f i rylgamelibrary:tokenlizedfile.obj
 0001:0001e930       ?_Insert_n@?$vector@PADV?$allocator@PAD@std@@@std@@IAEXViterator@12@IABQAD@Z 0041f930 f i rylgamelibrary:tokenlizedfile.obj
 0001:0001eb10       ??$_Sort@Viterator@?$vector@UColumnInfo@CTokenlizedFile@@V?$allocator@UColumnInfo@CTokenlizedFile@@@std@@@std@@H@std@@YAXViterator@?$vector@UColumnInfo@CTokenlizedFile@@V?$allocator@UColumnInfo@CTokenlizedFile@@@std@@@0@0H@Z 0041fb10 f i rylgamelibrary:tokenlizedfile.obj
 0001:0001ec40       ?reserve@?$vector@UColumnInfo@CTokenlizedFile@@V?$allocator@UColumnInfo@CTokenlizedFile@@@std@@@std@@QAEXI@Z 0041fc40 f i rylgamelibrary:tokenlizedfile.obj
 0001:0001ed30       ?reserve@?$vector@PADV?$allocator@PAD@std@@@std@@QAEXI@Z 0041fd30 f i rylgamelibrary:tokenlizedfile.obj
 0001:0001ee00       ?insert@?$vector@UColumnInfo@CTokenlizedFile@@V?$allocator@UColumnInfo@CTokenlizedFile@@@std@@@std@@QAE?AViterator@12@V312@ABUColumnInfo@CTokenlizedFile@@@Z 0041fe00 f i rylgamelibrary:tokenlizedfile.obj
 0001:0001ee70       ?push_back@?$vector@UColumnInfo@CTokenlizedFile@@V?$allocator@UColumnInfo@CTokenlizedFile@@@std@@@std@@QAEXABUColumnInfo@CTokenlizedFile@@@Z 0041fe70 f i rylgamelibrary:tokenlizedfile.obj
 0001:0001eef0       ??0CTokenlizedFile@@QAE@PBD@Z 0041fef0 f   rylgamelibrary:tokenlizedfile.obj
 0001:0001ef80       ?ReadColumn@CTokenlizedFile@@QAE_NXZ 0041ff80 f   rylgamelibrary:tokenlizedfile.obj
 0001:0001f080       ?ReadLine@CTokenlizedFile@@QAE_NXZ 00420080 f   rylgamelibrary:tokenlizedfile.obj
 0001:0001f180       ?Initialize@SpriteData@Item@@QAEXXZ 00420180 f   rylgamelibrary:itemstructure.obj
 0001:0001f1c0       ?Initialize@StringData@Item@@QAEXXZ 004201c0 f   rylgamelibrary:itemstructure.obj
 0001:0001f240       ??0SpriteData@Item@@QAE@XZ 00420240 f   rylgamelibrary:itemstructure.obj
 0001:0001f280       ?Initialize@ItemInfo@Item@@QAEXXZ 00420280 f   rylgamelibrary:itemstructure.obj
 0001:0001f3b0       ??0ItemInfo@Item@@QAE@XZ   004203b0 f   rylgamelibrary:itemstructure.obj
 0001:0001f500       ??0ItemInfo@Item@@QAE@G@Z  00420500 f   rylgamelibrary:itemstructure.obj
 0001:0001f650       ?SetUseItemTypeFlags@CItemType@Item@@QAEXAAUItemInfo@2@@Z 00420650 f   rylgamelibrary:itemconstants.obj
 0001:0001f6c0       ?SetEtcItemTypeFlags@CItemType@Item@@QAEXAAUItemInfo@2@@Z 004206c0 f   rylgamelibrary:itemconstants.obj
 0001:0001f6e0       ?GetEquipType@@YAFW4Type@ItemType@Item@@@Z 004206e0 f   rylgamelibrary:itemconstants.obj
 0001:0001f750       ?GetInstallGemAttribute@CItemType@Item@@SAXPBEPAUItemAttribute@2@W4Type@ItemType@2@EE@Z 00420750 f   rylgamelibrary:itemconstants.obj
 0001:0001f830       ?GetUpgradeItemAttribute@CItemType@Item@@SAXW4Type@ItemType@2@PAUItemAttribute@2@EE@Z 00420830 f   rylgamelibrary:itemconstants.obj
 0001:0001f890       ??1?$CSingleton@VCItemType@Item@@@@IAE@XZ 00420890 f i rylgamelibrary:itemconstants.obj
 0001:0001f8a0       ??$copy_backward@PAW4Type@ItemType@Item@@PAW4123@@std@@YAPAW4Type@ItemType@Item@@PAW4123@00@Z 004208a0 f i rylgamelibrary:itemconstants.obj
 0001:0001f8d0       ??$_Rotate@Viterator@?$vector@KV?$allocator@K@std@@@std@@HK@std@@YAXViterator@?$vector@KV?$allocator@K@std@@@0@00PAHPAK@Z 004208d0 f i rylgamelibrary:limituserbyip.obj
 0001:0001f8d0       ??$_Rotate@Viterator@?$vector@W4Type@ItemType@Item@@V?$allocator@W4Type@ItemType@Item@@@std@@@std@@HW4Type@ItemType@Item@@@std@@YAXViterator@?$vector@W4Type@ItemType@Item@@V?$allocator@W4Type@ItemType@Item@@@std@@@0@00PAHPAW4Type@ItemType@Item@@@Z 004208d0 f i rylgamelibrary:itemconstants.obj
 0001:0001f990       ??$_Median@Viterator@?$vector@W4Type@ItemType@Item@@V?$allocator@W4Type@ItemType@Item@@@std@@@std@@@std@@YAXViterator@?$vector@W4Type@ItemType@Item@@V?$allocator@W4Type@ItemType@Item@@@std@@@0@00@Z 00420990 f i rylgamelibrary:itemconstants.obj
 0001:0001fad0       ??$_Adjust_heap@Viterator@?$vector@W4Type@ItemType@Item@@V?$allocator@W4Type@ItemType@Item@@@std@@@std@@HW4Type@ItemType@Item@@@std@@YAXViterator@?$vector@W4Type@ItemType@Item@@V?$allocator@W4Type@ItemType@Item@@@std@@@0@HHW4Type@ItemType@Item@@@Z 00420ad0 f i rylgamelibrary:itemconstants.obj
 0001:0001fb50       ??$_Uninit_fill_n@PAW4Type@ItemType@Item@@IW4123@V?$allocator@W4Type@ItemType@Item@@@std@@@std@@YAXPAW4Type@ItemType@Item@@IABW4123@AAV?$allocator@W4Type@ItemType@Item@@@0@U_Nonscalar_ptr_iterator_tag@0@@Z 00420b50 f i rylgamelibrary:itemconstants.obj
 0001:0001fb80       ??$_Unguarded_partition@Viterator@?$vector@W4Type@ItemType@Item@@V?$allocator@W4Type@ItemType@Item@@@std@@@std@@@std@@YA?AU?$pair@Viterator@?$vector@W4Type@ItemType@Item@@V?$allocator@W4Type@ItemType@Item@@@std@@@std@@V123@@0@Viterator@?$vector@W4Type@ItemType@Item@@V?$allocator@W4Type@ItemType@Item@@@std@@@0@0@Z 00420b80 f i rylgamelibrary:itemconstants.obj
 0001:0001fcd0       ??$_Lower_bound@Viterator@?$vector@W4Type@ItemType@Item@@V?$allocator@W4Type@ItemType@Item@@@std@@@std@@EH@std@@YA?AViterator@?$vector@W4Type@ItemType@Item@@V?$allocator@W4Type@ItemType@Item@@@std@@@0@V120@0ABEPAH@Z 00420cd0 f i rylgamelibrary:itemconstants.obj
 0001:0001fd20       ??$_Make_heap@Viterator@?$vector@W4Type@ItemType@Item@@V?$allocator@W4Type@ItemType@Item@@@std@@@std@@HW4Type@ItemType@Item@@@std@@YAXViterator@?$vector@W4Type@ItemType@Item@@V?$allocator@W4Type@ItemType@Item@@@std@@@0@0PAHPAW4Type@ItemType@Item@@@Z 00420d20 f i rylgamelibrary:itemconstants.obj
 0001:0001fd60       ??$_Insertion_sort@Viterator@?$vector@W4Type@ItemType@Item@@V?$allocator@W4Type@ItemType@Item@@@std@@@std@@@std@@YAXViterator@?$vector@W4Type@ItemType@Item@@V?$allocator@W4Type@ItemType@Item@@@std@@@0@0@Z 00420d60 f i rylgamelibrary:itemconstants.obj
 0001:0001fde0       ?_Ufill@?$vector@W4Type@ItemType@Item@@V?$allocator@W4Type@ItemType@Item@@@std@@@std@@IAEPAW4Type@ItemType@Item@@PAW4345@IABW4345@@Z 00420de0 f i rylgamelibrary:itemconstants.obj
 0001:0001fe10       ??$sort_heap@Viterator@?$vector@W4Type@ItemType@Item@@V?$allocator@W4Type@ItemType@Item@@@std@@@std@@@std@@YAXViterator@?$vector@W4Type@ItemType@Item@@V?$allocator@W4Type@ItemType@Item@@@std@@@0@0@Z 00420e10 f i rylgamelibrary:itemconstants.obj
 0001:0001fe60       ??1CItemType@Item@@QAE@XZ  00420e60 f i rylgamelibrary:itemconstants.obj
 0001:0001feb0       ?IsCorrectItemType@CItemType@Item@@QAE_NW4ArrayType@12@E@Z 00420eb0 f   rylgamelibrary:itemconstants.obj
 0001:0001ff00       ?SetEquipTypeFlags@CItemType@Item@@QAEXAAUItemInfo@2@@Z 00420f00 f   rylgamelibrary:itemconstants.obj
 0001:00020010       ?_Xlen@?$vector@W4Type@ItemType@Item@@V?$allocator@W4Type@ItemType@Item@@@std@@@std@@IBEXXZ 00421010 f i rylgamelibrary:itemconstants.obj
 0001:00020080       ?_Insert_n@?$vector@W4Type@ItemType@Item@@V?$allocator@W4Type@ItemType@Item@@@std@@@std@@IAEXViterator@12@IABW4Type@ItemType@Item@@@Z 00421080 f i rylgamelibrary:itemconstants.obj
 0001:000202c0       ??$_Sort@Viterator@?$vector@W4Type@ItemType@Item@@V?$allocator@W4Type@ItemType@Item@@@std@@@std@@H@std@@YAXViterator@?$vector@W4Type@ItemType@Item@@V?$allocator@W4Type@ItemType@Item@@@std@@@0@0H@Z 004212c0 f i rylgamelibrary:itemconstants.obj
 0001:00020390       ?reserve@?$vector@W4Type@ItemType@Item@@V?$allocator@W4Type@ItemType@Item@@@std@@@std@@QAEXI@Z 00421390 f i rylgamelibrary:itemconstants.obj
 0001:00020460       ??0?$vector@W4Type@ItemType@Item@@V?$allocator@W4Type@ItemType@Item@@@std@@@std@@QAE@XZ 00421460 f i rylgamelibrary:itemconstants.obj
 0001:00020470       ?push_back@?$vector@W4Type@ItemType@Item@@V?$allocator@W4Type@ItemType@Item@@@std@@@std@@QAEXABW4Type@ItemType@Item@@@Z 00421470 f i rylgamelibrary:itemconstants.obj
 0001:000204e0       ??0CItemType@Item@@AAE@XZ  004214e0 f   rylgamelibrary:itemconstants.obj
 0001:00021b00       ?StrToHex16@Convert@Math@@YAGPBD@Z 00422b00 f i rylgamelibrary:itemdataparser.obj
 0001:00021be0       ?ReadString@@YA_NPADHPBD@Z 00422be0 f   rylgamelibrary:itemdataparser.obj
 0001:00021c40       ?ReadStringToTypeValue@@YA_NAAEPBVCTypeName@@EPBD@Z 00422c40 f   rylgamelibrary:itemdataparser.obj
 0001:00021cc0       ?ReadID@@YA_NAAUItemInfo@Item@@PBD@Z 00422cc0 f   rylgamelibrary:itemdataparser.obj
 0001:00021d10       ?ReadItemName@@YA_NAAUItemInfo@Item@@PBD@Z 00422d10 f   rylgamelibrary:itemdataparser.obj
 0001:00021d30       ?ReadFieldModelName@@YA_NAAUItemInfo@Item@@PBD@Z 00422d30 f   rylgamelibrary:itemdataparser.obj
 0001:00021d50       ?ReadAttachedModelName@@YA_NAAUItemInfo@Item@@PBD@Z 00422d50 f   rylgamelibrary:itemdataparser.obj
 0001:00021d70       ?ReadSpriteDDS@@YA_NAAUItemInfo@Item@@PBD@Z 00422d70 f   rylgamelibrary:itemdataparser.obj
 0001:00021d90       ?ReadMinX@@YA_NAAUItemInfo@Item@@PBD@Z 00422d90 f   rylgamelibrary:itemdataparser.obj
 0001:00021db0       ?ReadMinY@@YA_NAAUItemInfo@Item@@PBD@Z 00422db0 f   rylgamelibrary:itemdataparser.obj
 0001:00021dd0       ?ReadMaxX@@YA_NAAUItemInfo@Item@@PBD@Z 00422dd0 f   rylgamelibrary:itemdataparser.obj
 0001:00021df0       ?ReadMaxY@@YA_NAAUItemInfo@Item@@PBD@Z 00422df0 f   rylgamelibrary:itemdataparser.obj
 0001:00021e10       ?ReadSizeX@@YA_NAAUItemInfo@Item@@PBD@Z 00422e10 f   rylgamelibrary:itemdataparser.obj
 0001:00021e30       ?ReadSizeY@@YA_NAAUItemInfo@Item@@PBD@Z 00422e30 f   rylgamelibrary:itemdataparser.obj
 0001:00021e50       ?ReadEffectSound@@YA_NAAUItemInfo@Item@@PBD@Z 00422e50 f   rylgamelibrary:itemdataparser.obj
 0001:00021e70       ?ReadItemLevel@@YA_NAAUItemInfo@Item@@PBD@Z 00422e70 f   rylgamelibrary:itemdataparser.obj
 0001:00021eb0       ?ReadTypeName@@YA_NAAUItemInfo@Item@@PBD@Z 00422eb0 f   rylgamelibrary:itemdataparser.obj
 0001:00021ed0       ?ReadPrice@@YA_NAAUItemInfo@Item@@PBD@Z 00422ed0 f   rylgamelibrary:itemdataparser.obj
 0001:00021ef0       ?ReadBlackPrice@@YA_NAAUItemInfo@Item@@PBD@Z 00422ef0 f   rylgamelibrary:itemdataparser.obj
 0001:00021f10       ?ReadMedalPrice@@YA_NAAUItemInfo@Item@@PBD@Z 00422f10 f   rylgamelibrary:itemdataparser.obj
 0001:00021f30       ?ReadOptionLimit@@YA_NAAUItemInfo@Item@@PBD@Z 00422f30 f   rylgamelibrary:itemdataparser.obj
 0001:00021f50       ?ReadDurability@@YA_NAAUItemInfo@Item@@PBD@Z 00422f50 f   rylgamelibrary:itemdataparser.obj
 0001:00021f70       ?ReadMaxDurability@@YA_NAAUItemInfo@Item@@PBD@Z 00422f70 f   rylgamelibrary:itemdataparser.obj
 0001:00021f90       ?ReadClassLimit@@YA_NAAUItemInfo@Item@@PBD@Z 00422f90 f   rylgamelibrary:itemdataparser.obj
 0001:00021fb0       ?ReadSkillLimitType@@YA_NAAUItemInfo@Item@@PBD@Z 00422fb0 f   rylgamelibrary:itemdataparser.obj
 0001:00021fd0       ?ReadSkillLimitLevel@@YA_NAAUItemInfo@Item@@PBD@Z 00422fd0 f   rylgamelibrary:itemdataparser.obj
 0001:00021ff0       ?ReadLevelLimit@@YA_NAAUItemInfo@Item@@PBD@Z 00422ff0 f   rylgamelibrary:itemdataparser.obj
 0001:00022010       ?ReadSTRLimit@@YA_NAAUItemInfo@Item@@PBD@Z 00423010 f   rylgamelibrary:itemdataparser.obj
 0001:00022030       ?ReadDEXLimit@@YA_NAAUItemInfo@Item@@PBD@Z 00423030 f   rylgamelibrary:itemdataparser.obj
 0001:00022050       ?ReadCONLimit@@YA_NAAUItemInfo@Item@@PBD@Z 00423050 f   rylgamelibrary:itemdataparser.obj
 0001:00022070       ?ReadINTLimit@@YA_NAAUItemInfo@Item@@PBD@Z 00423070 f   rylgamelibrary:itemdataparser.obj
 0001:00022090       ?ReadWISLimit@@YA_NAAUItemInfo@Item@@PBD@Z 00423090 f   rylgamelibrary:itemdataparser.obj
 0001:000220b0       ?ReadCraftExp@@YA_NAAUItemInfo@Item@@PBD@Z 004230b0 f   rylgamelibrary:itemdataparser.obj
 0001:000220d0       ?ReadCriticalType@@YA_NAAUItemInfo@Item@@PBD@Z 004230d0 f   rylgamelibrary:itemdataparser.obj
 0001:00022100       ?ReadCriticalPercentage@@YA_NAAUItemInfo@Item@@PBD@Z 00423100 f   rylgamelibrary:itemdataparser.obj
 0001:00022130       ?ReadMinDamage@@YA_NAAUItemInfo@Item@@PBD@Z 00423130 f   rylgamelibrary:itemdataparser.obj
 0001:00022160       ?ReadMaxDamage@@YA_NAAUItemInfo@Item@@PBD@Z 00423160 f   rylgamelibrary:itemdataparser.obj
 0001:00022190       ?ReadDRC@@YA_NAAUItemInfo@Item@@PBD@Z 00423190 f   rylgamelibrary:itemdataparser.obj
 0001:000221c0       ?ReadOffenceRevision@@YA_NAAUItemInfo@Item@@PBD@Z 004231c0 f   rylgamelibrary:itemdataparser.obj
 0001:000221f0       ?ReadDefence@@YA_NAAUItemInfo@Item@@PBD@Z 004231f0 f   rylgamelibrary:itemdataparser.obj
 0001:00022220       ?ReadDefenceRevision@@YA_NAAUItemInfo@Item@@PBD@Z 00423220 f   rylgamelibrary:itemdataparser.obj
 0001:00022250       ?ReadResistance@@YA_NAAUItemInfo@Item@@PBD@Z 00423250 f   rylgamelibrary:itemdataparser.obj
 0001:00022280       ?ReadBlockingPercentage@@YA_NAAUItemInfo@Item@@PBD@Z 00423280 f   rylgamelibrary:itemdataparser.obj
 0001:000222b0       ?ReadAttackSpeed@@YA_NAAUItemInfo@Item@@PBD@Z 004232b0 f   rylgamelibrary:itemdataparser.obj
 0001:000222e0       ?ReadMoveSpeed@@YA_NAAUItemInfo@Item@@PBD@Z 004232e0 f   rylgamelibrary:itemdataparser.obj
 0001:00022310       ?ReadAttackRange@@YA_NAAUItemInfo@Item@@PBD@Z 00423310 f   rylgamelibrary:itemdataparser.obj
 0001:00022340       ?ReadRangedAttack@@YA_NAAUItemInfo@Item@@PBD@Z 00423340 f   rylgamelibrary:itemdataparser.obj
 0001:00022370       ?ReadHpMaxPlus@@YA_NAAUItemInfo@Item@@PBD@Z 00423370 f   rylgamelibrary:itemdataparser.obj
 0001:000223a0       ?ReadMpMaxPlus@@YA_NAAUItemInfo@Item@@PBD@Z 004233a0 f   rylgamelibrary:itemdataparser.obj
 0001:000223d0       ?ReadHPRegen@@YA_NAAUItemInfo@Item@@PBD@Z 004233d0 f   rylgamelibrary:itemdataparser.obj
 0001:00022400       ?ReadMPRegen@@YA_NAAUItemInfo@Item@@PBD@Z 00423400 f   rylgamelibrary:itemdataparser.obj
 0001:00022430       ?ReadFireAttribute@@YA_NAAUItemInfo@Item@@PBD@Z 00423430 f   rylgamelibrary:itemdataparser.obj
 0001:00022460       ?ReadLightingAttribute@@YA_NAAUItemInfo@Item@@PBD@Z 00423460 f   rylgamelibrary:itemdataparser.obj
 0001:00022490       ?ReadColdAttribute@@YA_NAAUItemInfo@Item@@PBD@Z 00423490 f   rylgamelibrary:itemdataparser.obj
 0001:000224c0       ?ReadDrainAttribute@@YA_NAAUItemInfo@Item@@PBD@Z 004234c0 f   rylgamelibrary:itemdataparser.obj
 0001:000224f0       ?ReadPoisonAttribute@@YA_NAAUItemInfo@Item@@PBD@Z 004234f0 f   rylgamelibrary:itemdataparser.obj
 0001:00022520       ?ReadFireResistance@@YA_NAAUItemInfo@Item@@PBD@Z 00423520 f   rylgamelibrary:itemdataparser.obj
 0001:00022550       ?ReadLightningResistance@@YA_NAAUItemInfo@Item@@PBD@Z 00423550 f   rylgamelibrary:itemdataparser.obj
 0001:00022580       ?ReadColdResistance@@YA_NAAUItemInfo@Item@@PBD@Z 00423580 f   rylgamelibrary:itemdataparser.obj
 0001:000225b0       ?ReadDrainResistance@@YA_NAAUItemInfo@Item@@PBD@Z 004235b0 f   rylgamelibrary:itemdataparser.obj
 0001:000225e0       ?ReadPoisonResistance@@YA_NAAUItemInfo@Item@@PBD@Z 004235e0 f   rylgamelibrary:itemdataparser.obj
 0001:00022610       ?ReadSTRAdd@@YA_NAAUItemInfo@Item@@PBD@Z 00423610 f   rylgamelibrary:itemdataparser.obj
 0001:00022640       ?ReadDEXAdd@@YA_NAAUItemInfo@Item@@PBD@Z 00423640 f   rylgamelibrary:itemdataparser.obj
 0001:00022670       ?ReadCONAdd@@YA_NAAUItemInfo@Item@@PBD@Z 00423670 f   rylgamelibrary:itemdataparser.obj
 0001:000226a0       ?ReadINTAdd@@YA_NAAUItemInfo@Item@@PBD@Z 004236a0 f   rylgamelibrary:itemdataparser.obj
 0001:000226d0       ?ReadWISAdd@@YA_NAAUItemInfo@Item@@PBD@Z 004236d0 f   rylgamelibrary:itemdataparser.obj
 0001:00022700       ?ReadMaterialValue@@YA_NAAUItemInfo@Item@@PBD@Z 00423700 f   rylgamelibrary:itemdataparser.obj
 0001:00022720       ?ReadMaxSocketNum@@YA_NAAUItemInfo@Item@@PBD@Z 00423720 f   rylgamelibrary:itemdataparser.obj
 0001:00022740       ?ReadSkill_Level@@YA_NAAUItemInfo@Item@@PBD@Z 00423740 f   rylgamelibrary:itemdataparser.obj
 0001:00022760       ?ReadZone@@YA_NAAUItemInfo@Item@@PBD@Z 00423760 f   rylgamelibrary:itemdataparser.obj
 0001:00022780       ?ReadPositionX@@YA_NAAUItemInfo@Item@@PBD@Z 00423780 f   rylgamelibrary:itemdataparser.obj
 0001:000227a0       ?ReadPositionY@@YA_NAAUItemInfo@Item@@PBD@Z 004237a0 f   rylgamelibrary:itemdataparser.obj
 0001:000227c0       ?ReadPositionZ@@YA_NAAUItemInfo@Item@@PBD@Z 004237c0 f   rylgamelibrary:itemdataparser.obj
 0001:000227e0       ?ReadAmount@@YA_NAAUItemInfo@Item@@PBD@Z 004237e0 f   rylgamelibrary:itemdataparser.obj
 0001:00022800       ?ReadItemDescribe@@YA_NAAUItemInfo@Item@@PBD@Z 00423800 f   rylgamelibrary:itemdataparser.obj
 0001:00022820       ?ReadItemType@@YA_NAAUItemInfo@Item@@PBD@Z 00423820 f   rylgamelibrary:itemdataparser.obj
 0001:00022850       ?ReadSkill_ID@@YA_NAAUItemInfo@Item@@PBD@Z 00423850 f   rylgamelibrary:itemdataparser.obj
 0001:000228a0       ??$_Uninit_fill_n@PAUParseData@ItemDataParser@@IU12@V?$allocator@UParseData@ItemDataParser@@@std@@@std@@YAXPAUParseData@ItemDataParser@@IABU12@AAV?$allocator@UParseData@ItemDataParser@@@0@U_Nonscalar_ptr_iterator_tag@0@@Z 004238a0 f i rylgamelibrary:itemdataparser.obj
 0001:000228a0       ??$_Uninit_fill_n@PAU?$pair@W4eStdFunc@@H@std@@IU12@V?$allocator@U?$pair@W4eStdFunc@@H@std@@@2@@std@@YAXPAU?$pair@W4eStdFunc@@H@0@IABU10@AAV?$allocator@U?$pair@W4eStdFunc@@H@std@@@0@U_Nonscalar_ptr_iterator_tag@0@@Z 004238a0 f i rylgamelibrary:reloctable.obj
 0001:000228a0       ??$_Uninit_fill_n@PAU?$pair@KK@std@@IU12@V?$allocator@U?$pair@KK@std@@@2@@std@@YAXPAU?$pair@KK@0@IABU10@AAV?$allocator@U?$pair@KK@std@@@0@U_Nonscalar_ptr_iterator_tag@0@@Z 004238a0 f i rylgamelibrary:rylserverdispatch.obj
 0001:000228d0       ?_Ufill@?$vector@UParseData@ItemDataParser@@V?$allocator@UParseData@ItemDataParser@@@std@@@std@@IAEPAUParseData@ItemDataParser@@PAU34@IABU34@@Z 004238d0 f i rylgamelibrary:itemdataparser.obj
 0001:000228d0       ?_Ufill@?$vector@U?$pair@KK@std@@V?$allocator@U?$pair@KK@std@@@2@@std@@IAEPAU?$pair@KK@2@PAU32@IABU32@@Z 004238d0 f i rylgamelibrary:rylserverdispatch.obj
 0001:000228d0       ?_Ufill@?$vector@U?$pair@W4eStdFunc@@H@std@@V?$allocator@U?$pair@W4eStdFunc@@H@std@@@2@@std@@IAEPAU?$pair@W4eStdFunc@@H@2@PAU32@IABU32@@Z 004238d0 f i rylgamelibrary:reloctable.obj
 0001:00022900       ?_Insert_n@?$vector@UParseData@ItemDataParser@@V?$allocator@UParseData@ItemDataParser@@@std@@@std@@IAEXViterator@12@IABUParseData@ItemDataParser@@@Z 00423900 f i rylgamelibrary:itemdataparser.obj
 0001:00022b50       ?reserve@?$vector@UParseData@ItemDataParser@@V?$allocator@UParseData@ItemDataParser@@@std@@@std@@QAEXI@Z 00423b50 f i rylgamelibrary:itemdataparser.obj
 0001:00022c20       ?push_back@?$vector@UParseData@ItemDataParser@@V?$allocator@UParseData@ItemDataParser@@@std@@@std@@QAEXABUParseData@ItemDataParser@@@Z 00423c20 f i rylgamelibrary:itemdataparser.obj
 0001:00022c90       ?SetDefaultData@ItemDataParser@@YA_NAAV?$vector@UParseData@ItemDataParser@@V?$allocator@UParseData@ItemDataParser@@@std@@@std@@@Z 00423c90 f   rylgamelibrary:itemdataparser.obj
 0001:00023020       ?SetEquipData@ItemDataParser@@YA_NAAV?$vector@UParseData@ItemDataParser@@V?$allocator@UParseData@ItemDataParser@@@std@@@std@@@Z 00424020 f   rylgamelibrary:itemdataparser.obj
 0001:00023410       ?SetUseItemData@ItemDataParser@@YA_NAAV?$vector@UParseData@ItemDataParser@@V?$allocator@UParseData@ItemDataParser@@@std@@@std@@@Z 00424410 f   rylgamelibrary:itemdataparser.obj
 0001:00023500       ?SetEtcItemData@ItemDataParser@@YA_NAAV?$vector@UParseData@ItemDataParser@@V?$allocator@UParseData@ItemDataParser@@@std@@@std@@@Z 00424500 f   rylgamelibrary:itemdataparser.obj
 0001:00023530       ?InitializeAttribute@CEquipment@Item@@IAEXXZ 00424530 f i rylgamelibrary:item.obj
 0001:000235d0       ??0CItem@Item@@QAE@_KABUItemInfo@1@@Z 004245d0 f   rylgamelibrary:item.obj
 0001:00023640       ?SerializeOut@CItem@Item@@UAE_NPADAAI@Z 00424640 f   rylgamelibrary:item.obj
 0001:00023690       ?SerializeIn@CItem@Item@@UAE_NPBDAAI@Z 00424690 f   rylgamelibrary:item.obj
 0001:00023710       ?SerializeOut@CEquipment@Item@@UAE_NPADAAI@Z 00424710 f   rylgamelibrary:item.obj
 0001:00023a80       ??0CUseItem@Item@@QAE@_KABUItemInfo@1@@Z 00424a80 f   rylgamelibrary:item.obj
 0001:00023ab0       ??1CItem@Item@@UAE@XZ      00424ab0 f   rylgamelibrary:item.obj
 0001:00023ab0       ??1CUseItem@Item@@UAE@XZ   00424ab0 f   rylgamelibrary:item.obj
 0001:00023ab0       ??1CEquipment@Item@@UAE@XZ 00424ab0 f   rylgamelibrary:item.obj
 0001:00023ac0       ??_ECItem@Item@@UAEPAXI@Z  00424ac0 f i rylgamelibrary:item.obj
 0001:00023ac0       ??_GCItem@Item@@UAEPAXI@Z  00424ac0 f i rylgamelibrary:item.obj
 0001:00023ae0       ??0CEquipment@Item@@QAE@_KABUItemInfo@1@@Z 00424ae0 f   rylgamelibrary:item.obj
 0001:00023bb0       ??_ECUseItem@Item@@UAEPAXI@Z 00424bb0 f i rylgamelibrary:item.obj
 0001:00023bb0       ??_GCUseItem@Item@@UAEPAXI@Z 00424bb0 f i rylgamelibrary:item.obj
 0001:00023bb0       ??_GCEquipment@Item@@UAEPAXI@Z 00424bb0 f i rylgamelibrary:item.obj
 0001:00023bb0       ??_ECEquipment@Item@@UAEPAXI@Z 00424bb0 f i rylgamelibrary:item.obj
 0001:00023bd0       ?SerializeIn@CEquipment@Item@@UAE_NPBDAAI@Z 00424bd0 f   rylgamelibrary:item.obj
 0001:00023de0       ?_Max@?$_Tree@V?$_Tmap_traits@IUInternalTimerData@CTimerProcMgr@@U?$less@I@std@@V?$allocator@U?$pair@$$CBIUInternalTimerData@CTimerProcMgr@@@std@@@4@$0A@@std@@@std@@KAPAU_Node@?$_Tree_nod@V?$_Tmap_traits@IUInternalTimerData@CTimerProcMgr@@U?$less@I@std@@V?$allocator@U?$pair@$$CBIUInternalTimerData@CTimerProcMgr@@@std@@@4@$0A@@std@@@2@PAU342@@Z 00424de0 f i rylgamelibrary:timerproc.obj
 0001:00023e00       ?_Min@?$_Tree@V?$_Tmap_traits@IUInternalTimerData@CTimerProcMgr@@U?$less@I@std@@V?$allocator@U?$pair@$$CBIUInternalTimerData@CTimerProcMgr@@@std@@@4@$0A@@std@@@std@@KAPAU_Node@?$_Tree_nod@V?$_Tmap_traits@IUInternalTimerData@CTimerProcMgr@@U?$less@I@std@@V?$allocator@U?$pair@$$CBIUInternalTimerData@CTimerProcMgr@@@std@@@4@$0A@@std@@@2@PAU342@@Z 00424e00 f i rylgamelibrary:timerproc.obj
 0001:00023e20       ?_Rrotate@?$_Tree@V?$_Tmap_traits@IUInternalTimerData@CTimerProcMgr@@U?$less@I@std@@V?$allocator@U?$pair@$$CBIUInternalTimerData@CTimerProcMgr@@@std@@@4@$0A@@std@@@std@@IAEXPAU_Node@?$_Tree_nod@V?$_Tmap_traits@IUInternalTimerData@CTimerProcMgr@@U?$less@I@std@@V?$allocator@U?$pair@$$CBIUInternalTimerData@CTimerProcMgr@@@std@@@4@$0A@@std@@@2@@Z 00424e20 f i rylgamelibrary:timerproc.obj
 0001:00023e80       ?_Inc@const_iterator@?$_Tree@V?$_Tmap_traits@IUInternalTimerData@CTimerProcMgr@@U?$less@I@std@@V?$allocator@U?$pair@$$CBIUInternalTimerData@CTimerProcMgr@@@std@@@4@$0A@@std@@@std@@QAEXXZ 00424e80 f i rylgamelibrary:timerproc.obj
 0001:00023ee0       ?_Lrotate@?$_Tree@V?$_Tmap_traits@IUInternalTimerData@CTimerProcMgr@@U?$less@I@std@@V?$allocator@U?$pair@$$CBIUInternalTimerData@CTimerProcMgr@@@std@@@4@$0A@@std@@@std@@IAEXPAU_Node@?$_Tree_nod@V?$_Tmap_traits@IUInternalTimerData@CTimerProcMgr@@U?$less@I@std@@V?$allocator@U?$pair@$$CBIUInternalTimerData@CTimerProcMgr@@@std@@@4@$0A@@std@@@2@@Z 00424ee0 f i rylgamelibrary:timerproc.obj
 0001:00023f40       ?_Buynode@?$_Tree@V?$_Tmap_traits@IUInternalTimerData@CTimerProcMgr@@U?$less@I@std@@V?$allocator@U?$pair@$$CBIUInternalTimerData@CTimerProcMgr@@@std@@@4@$0A@@std@@@std@@IAEPAU_Node@?$_Tree_nod@V?$_Tmap_traits@IUInternalTimerData@CTimerProcMgr@@U?$less@I@std@@V?$allocator@U?$pair@$$CBIUInternalTimerData@CTimerProcMgr@@@std@@@4@$0A@@std@@@2@XZ 00424f40 f i rylgamelibrary:timerproc.obj
 0001:00023f80       ??1_Node@?$_Tree_nod@V?$_Tmap_traits@IUInternalTimerData@CTimerProcMgr@@U?$less@I@std@@V?$allocator@U?$pair@$$CBIUInternalTimerData@CTimerProcMgr@@@std@@@4@$0A@@std@@@std@@QAE@XZ 00424f80 f i rylgamelibrary:timerproc.obj
 0001:00023fa0       ?erase@?$_Tree@V?$_Tmap_traits@IUInternalTimerData@CTimerProcMgr@@U?$less@I@std@@V?$allocator@U?$pair@$$CBIUInternalTimerData@CTimerProcMgr@@@std@@@4@$0A@@std@@@std@@QAE?AViterator@12@V312@@Z 00424fa0 f i rylgamelibrary:timerproc.obj
 0001:000242a0       ?_Erase@?$_Tree@V?$_Tmap_traits@IUInternalTimerData@CTimerProcMgr@@U?$less@I@std@@V?$allocator@U?$pair@$$CBIUInternalTimerData@CTimerProcMgr@@@std@@@4@$0A@@std@@@std@@IAEXPAU_Node@?$_Tree_nod@V?$_Tmap_traits@IUInternalTimerData@CTimerProcMgr@@U?$less@I@std@@V?$allocator@U?$pair@$$CBIUInternalTimerData@CTimerProcMgr@@@std@@@4@$0A@@std@@@2@@Z 004252a0 f i rylgamelibrary:timerproc.obj
 0001:000242e0       ?erase@?$_Tree@V?$_Tmap_traits@IUInternalTimerData@CTimerProcMgr@@U?$less@I@std@@V?$allocator@U?$pair@$$CBIUInternalTimerData@CTimerProcMgr@@@std@@@4@$0A@@std@@@std@@QAE?AViterator@12@V312@0@Z 004252e0 f i rylgamelibrary:timerproc.obj
 0001:000243a0       ?ClearAll@CTimerProcMgr@@QAEXXZ 004253a0 f   rylgamelibrary:timerproc.obj
 0001:000244a0       ??1?$map@IUInternalTimerData@CTimerProcMgr@@U?$less@I@std@@V?$allocator@U?$pair@$$CBIUInternalTimerData@CTimerProcMgr@@@std@@@4@@std@@QAE@XZ 004254a0 f i rylgamelibrary:timerproc.obj
 0001:000244d0       ??1CTimerProcMgr@@QAE@XZ   004254d0 f   rylgamelibrary:timerproc.obj
 0001:00024540       ??0CTimerProcMgr@@QAE@XZ   00425540 f   rylgamelibrary:timerproc.obj
 0001:00024580       ??0CSysTray@@QAE@PAUHWND__@@PAUHINSTANCE__@@@Z 00425580 f   rylgamelibrary:systray.obj
 0001:000245b0       ?ShowPopupMenu@CSysTray@@QAEXPAUHWND__@@PAUHMENU__@@@Z 004255b0 f   rylgamelibrary:systray.obj
 0001:00024600       ?GetSysTrayNotifyMsg@CSysTray@@SA?BIXZ 00425600 f   rylgamelibrary:systray.obj
 0001:00024640       ??1CSysTray@@QAE@XZ        00425640 f   rylgamelibrary:systray.obj
 0001:00024670       ?AddIcon@CSysTray@@QAEHPBDPAUHICON__@@I@Z 00425670 f   rylgamelibrary:systray.obj
 0001:00024750       ??_9@$BA@AE                00425750 f i rylgamelibrary:command.obj
 0001:00024760       ??_9@$B3AE                 00425760 f i rylgamelibrary:command.obj
 0001:00024770       ??$for_each@Viterator@?$list@PAVCCommand@@V?$allocator@PAVCCommand@@@std@@@std@@V?$mem_fun_t@_NVCCommand@@@3@@std@@YA?AV?$mem_fun_t@_NVCCommand@@@0@Viterator@?$list@PAVCCommand@@V?$allocator@PAVCCommand@@@std@@@0@0V10@@Z 00425770 f i rylgamelibrary:command.obj
 0001:000247b0       ?ClearAll@CCommandProcess@@IAEXXZ 004257b0 f   rylgamelibrary:command.obj
 0001:00024820       ??0CCommandProcess@@QAE@XZ 00425820 f   rylgamelibrary:command.obj
 0001:00024880       ??1CCommandProcess@@QAE@XZ 00425880 f   rylgamelibrary:command.obj
 0001:000248e0       ?_Splice@?$list@PAVCCommand@@V?$allocator@PAVCCommand@@@std@@@std@@QAEXViterator@12@AAV12@00I@Z 004258e0 f i rylgamelibrary:command.obj
 0001:00024930       ?ProcessAll@CCommandProcess@@QAEXXZ 00425930 f   rylgamelibrary:command.obj
 0001:00024a00       ?CheckSleep@CPulse@@QAEKXZ 00425a00 f   rylgamelibrary:pulse.obj
 0001:00024ad0       ?GetInstance@CPulse@@SAAAV1@XZ 00425ad0 f   rylgamelibrary:pulse.obj
 0001:00024b30       ?clear@?$list@PAVCCommand@@V?$allocator@PAVCCommand@@@std@@@std@@QAEXXZ 00425b30 f i rylgamelibrary:command.obj
 0001:00024b30       ?clear@?$list@PAVCThread@@V?$allocator@PAVCThread@@@std@@@std@@QAEXXZ 00425b30 f i rylgamelibrary:serverwindowframework.obj
 0001:00024b30       ?clear@?$list@PAVCSession@@V?$allocator@PAVCSession@@@std@@@std@@QAEXXZ 00425b30 f i rylgamelibrary:sessionmgr.obj
 0001:00024b30       ?clear@?$list@PAVCAuthInfo@@V?$allocator@PAVCAuthInfo@@@std@@@std@@QAEXXZ 00425b30 f i authorizeuser.obj
 0001:00024b30       ?clear@?$list@PAULogBuffer@@V?$allocator@PAULogBuffer@@@std@@@std@@QAEXXZ 00425b30 f i rylgamelibrary:gamelog.obj
 0001:00024b30       ?clear@?$list@UInternalProcessData@CTimerProcMgr@@V?$allocator@UInternalProcessData@CTimerProcMgr@@@std@@@std@@QAEXXZ 00425b30 f i rylgamelibrary:timerproc.obj
 0001:00024b30       ?clear@?$list@PAVCListener@@V?$allocator@PAVCListener@@@std@@@std@@QAEXXZ 00425b30 f i rylgamelibrary:iocpnet.obj
 0001:00024b70       ?DeleteSession@CSessionMgr@@QAEXPAVCSession@@@Z 00425b70 f   rylgamelibrary:sessionmgr.obj
 0001:00024bf0       ??1?$list@PAVCListener@@V?$allocator@PAVCListener@@@std@@@std@@QAE@XZ 00425bf0 f i rylgamelibrary:iocpnet.obj
 0001:00024bf0       ??1?$list@PAVCThread@@V?$allocator@PAVCThread@@@std@@@std@@QAE@XZ 00425bf0 f i rylgamelibrary:serverwindowframework.obj
 0001:00024bf0       ??1?$list@PAVCSession@@V?$allocator@PAVCSession@@@std@@@std@@QAE@XZ 00425bf0 f i rylgamelibrary:sessionmgr.obj
 0001:00024bf0       ??1?$list@PAULogBuffer@@V?$allocator@PAULogBuffer@@@std@@@std@@QAE@XZ 00425bf0 f i rylgamelibrary:gamelog.obj
 0001:00024bf0       ??1?$list@PAVCAuthInfo@@V?$allocator@PAVCAuthInfo@@@std@@@std@@QAE@XZ 00425bf0 f i authorizeuser.obj
 0001:00024bf0       ??1?$list@PAVCCommand@@V?$allocator@PAVCCommand@@@std@@@std@@QAE@XZ 00425bf0 f i rylgamelibrary:command.obj
 0001:00024c10       ??0CSessionMgr@@QAE@XZ     00425c10 f   rylgamelibrary:sessionmgr.obj
 0001:00024cd0       ?CreateSession@CSessionMgr@@QAEPAVCSession@@AAVCSessionPolicy@@@Z 00425cd0 f   rylgamelibrary:sessionmgr.obj
 0001:00024d60       ?_Incsize@?$list@PAVCSession@@V?$allocator@PAVCSession@@@std@@@std@@IAEXI@Z 00425d60 f i rylgamelibrary:sessionmgr.obj
 0001:00024e00       ?Add@CSessionMgr@@QAEXPAVCSession@@@Z 00425e00 f   rylgamelibrary:sessionmgr.obj
 0001:00024e80       ?_Splice@?$list@PAVCSession@@V?$allocator@PAVCSession@@@std@@@std@@QAEXViterator@12@AAV12@00I@Z 00425e80 f i rylgamelibrary:sessionmgr.obj
 0001:00024ed0       ?InternalProcess@CSessionMgr@@AAEXXZ 00425ed0 f   rylgamelibrary:sessionmgr.obj
 0001:00024fb0       ?Destroy@CSessionMgr@@QAEXK@Z 00425fb0 f   rylgamelibrary:sessionmgr.obj
 0001:000250a0       ??1CSessionMgr@@QAE@XZ     004260a0 f   rylgamelibrary:sessionmgr.obj
 0001:00025150       ??0CIOWorker@@QAE@AAVCCompletionHandler@@@Z 00426150 f   rylgamelibrary:ioworker.obj
 0001:00025170       ??1CThread@@UAE@XZ         00426170 f   authorizethread.obj
 0001:00025170       ??1CIOWorker@@UAE@XZ       00426170 f   rylgamelibrary:ioworker.obj
 0001:00025180       ?Run@CIOWorker@@EAEIXZ     00426180 f   rylgamelibrary:ioworker.obj
 0001:00025200       ?End@CIOWorker@@EAEHXZ     00426200 f   rylgamelibrary:ioworker.obj
 0001:00025220       ??_GCIOWorker@@UAEPAXI@Z   00426220 f i rylgamelibrary:ioworker.obj
 0001:00025220       ??_ECIOWorker@@UAEPAXI@Z   00426220 f i rylgamelibrary:ioworker.obj
 0001:00025240       ??0CCompletionHandler@@QAE@XZ 00426240 f   rylgamelibrary:completionhandler.obj
 0001:00025260       ?Initialize@CCompletionHandler@@QAE_NKK@Z 00426260 f   rylgamelibrary:completionhandler.obj
 0001:000252a0       ??_ECCompletionHandler@@UAEPAXI@Z 004262a0 f i rylgamelibrary:completionhandler.obj
 0001:000252a0       ??_GCCompletionHandler@@UAEPAXI@Z 004262a0 f i rylgamelibrary:completionhandler.obj
 0001:000257e0       _gzwrite                   004267e0 f   rylgamelibrary:gzio.obj
 0001:00025970       _gzclose                   00426970 f   rylgamelibrary:gzio.obj
 0001:00025c30       _gzopen                    00426c30 f   rylgamelibrary:gzio.obj
 0001:00025c50       _lzo1x_decompress_safe     00426c50 f   rylgamelibrary:minilzo.obj
 0001:00026010       ??1CNullItem@Item@@UAE@XZ  00427010 f i rylgamelibrary:itemcontainer.obj
 0001:00026030       ??0CNullItem@Item@@AAE@ABUItemInfo@1@@Z 00427030 f i rylgamelibrary:itemcontainer.obj
 0001:00026060       ??_ECNullItem@Item@@UAEPAXI@Z 00427060 f i rylgamelibrary:itemcontainer.obj
 0001:00026060       ??_GCNullItem@Item@@UAEPAXI@Z 00427060 f i rylgamelibrary:itemcontainer.obj
 0001:00026080       ??0CSkillMgr@@AAE@XZ       00427080 f   rylgamelibrary:skillmgr.obj
 0001:000260a0       ??1CSkillMgr@@QAE@XZ       004270a0 f   rylgamelibrary:skillmgr.obj
 0001:00026170       _deflate                   00427170 f   rylgamelibrary:deflate.obj
 0001:00026400       _deflateEnd                00427400 f   rylgamelibrary:deflate.obj
 0001:000271c0       _deflateReset              004281c0 f   rylgamelibrary:deflate.obj
 0001:00027240       _deflateInit2_             00428240 f   rylgamelibrary:deflate.obj
 0001:00027430       _inflateReset              00428430 f   rylgamelibrary:inflate.obj
 0001:00027480       _inflateEnd                00428480 f   rylgamelibrary:inflate.obj
 0001:000274d0       _inflateInit2_             004284d0 f   rylgamelibrary:inflate.obj
 0001:000275d0       _crc32                     004285d0 f   rylgamelibrary:crc32.obj
 0001:00027700       _zcalloc                   00428700 f   rylgamelibrary:zutil.obj
 0001:00027720       _zcfree                    00428720 f   rylgamelibrary:zutil.obj
 0001:00027730       ??_Ebad_alloc@std@@UAEPAXI@Z 00428730 f i rylgamelibrary:creaturemanager.obj
 0001:00027730       ??_Gbad_alloc@std@@UAEPAXI@Z 00428730 f i rylgamelibrary:creaturemanager.obj
 0001:00027750       ??1bad_alloc@std@@UAE@XZ   00428750 f i rylgamelibrary:creaturemanager.obj
 0001:00027760       ??1pool_type@?$singleton_pool@Ufast_pool_allocator_tag@boost@@$0BE@Udefault_user_allocator_new_delete@2@Vwin32_mutex@pool@details@2@$0CA@@boost@@QAE@XZ 00428760 f i rylgamelibrary:creaturemanager.obj
 0001:00027760       ??1pool_type@?$singleton_pool@Ufast_pool_allocator_tag@boost@@$0DI@Udefault_user_allocator_new_delete@2@Vwin32_mutex@pool@details@2@$0CA@@boost@@QAE@XZ 00428760 f i rylgamelibrary:cell.obj
 0001:00027760       ??1pool_type@?$singleton_pool@Ufast_pool_allocator_tag@boost@@$0BI@Udefault_user_allocator_new_delete@2@Vwin32_mutex@pool@details@2@$0CA@@boost@@QAE@XZ 00428760 f i rylgamelibrary:creaturemanager.obj
 0001:00027760       ??1pool_type@?$singleton_pool@Ufast_pool_allocator_tag@boost@@$0M@Udefault_user_allocator_new_delete@2@Vwin32_mutex@pool@details@2@$0CA@@boost@@QAE@XZ 00428760 f i rylgamelibrary:depositcontainer.obj
 0001:00027780       ?instance@?$singleton_default@Upool_type@?$singleton_pool@Ufast_pool_allocator_tag@boost@@$0BI@Udefault_user_allocator_new_delete@2@Vwin32_mutex@pool@details@2@$0CA@@boost@@@pool@details@boost@@SAAAUpool_type@?$singleton_pool@Ufast_pool_allocator_tag@boost@@$0BI@Udefault_user_allocator_new_delete@2@Vwin32_mutex@pool@details@2@$0CA@@4@XZ 00428780 f i rylgamelibrary:creaturemanager.obj
 0001:000277e0       ?instance@?$singleton_default@Upool_type@?$singleton_pool@Ufast_pool_allocator_tag@boost@@$0BE@Udefault_user_allocator_new_delete@2@Vwin32_mutex@pool@details@2@$0CA@@boost@@@pool@details@boost@@SAAAUpool_type@?$singleton_pool@Ufast_pool_allocator_tag@boost@@$0BE@Udefault_user_allocator_new_delete@2@Vwin32_mutex@pool@details@2@$0CA@@4@XZ 004287e0 f i rylgamelibrary:creaturemanager.obj
 0001:00027840       ??0bad_alloc@std@@QAE@ABV01@@Z 00428840 f i rylgamelibrary:creaturemanager.obj
 0001:00027860       ?Initialize@ProtoType@Skill@@QAEXXZ 00428860 f   rylgamelibrary:skillstructure.obj
 0001:00027970       ??0ProtoType@Skill@@QAE@XZ 00428970 f   rylgamelibrary:skillstructure.obj
 0001:00027990       ?instance@?$singleton_default@Upool_type@?$singleton_pool@Ufast_pool_allocator_tag@boost@@$0DI@Udefault_user_allocator_new_delete@2@Vwin32_mutex@pool@details@2@$0CA@@boost@@@pool@details@boost@@SAAAUpool_type@?$singleton_pool@Ufast_pool_allocator_tag@boost@@$0DI@Udefault_user_allocator_new_delete@2@Vwin32_mutex@pool@details@2@$0CA@@4@XZ 00428990 f i rylgamelibrary:cell.obj
 0001:000279f0       ??0CMonsterMgr@@AAE@XZ     004289f0 f   rylgamelibrary:monstermgr.obj
 0001:00027a10       ??1CMonsterMgr@@QAE@XZ     00428a10 f   rylgamelibrary:monstermgr.obj
 0001:00027a30       ??0CProcessTable@Skill@@AAE@XZ 00428a30 f   rylgamelibrary:skilltable.obj
 0001:00027a50       ??1CProcessTable@Skill@@AAE@XZ 00428a50 f   rylgamelibrary:skilltable.obj
 0001:00027a80       ??0CAward@AwardTable@@QAE@XZ 00428a80 f i rylgamelibrary:awardtable.obj
 0001:00027a90       ??1CAward@AwardTable@@QAE@XZ 00428a90 f i rylgamelibrary:awardtable.obj
 0001:00027aa0       ?put@?$basic_ostream@DU?$char_traits@D@std@@@std@@QAEAAV12@D@Z 00428aa0 f i rylgamelibrary:cellmanager.obj
 0001:00027bc0       _adler32                   00428bc0 f   rylgamelibrary:adler32.obj
 0001:00028f00       __tr_init                  00429f00 f   rylgamelibrary:trees.obj
 0001:00029270       __tr_stored_block          0042a270 f   rylgamelibrary:trees.obj
 0001:00029310       __tr_align                 0042a310 f   rylgamelibrary:trees.obj
 0001:00029510       __tr_flush_block           0042a510 f   rylgamelibrary:trees.obj
 0001:00029700       _inflate_blocks_reset      0042a700 f   rylgamelibrary:infblock.obj
 0001:00029780       _inflate_blocks_new        0042a780 f   rylgamelibrary:infblock.obj
 0001:00029820       _inflate_blocks_free       0042a820 f   rylgamelibrary:infblock.obj
 0001:000298b0       ??0CRankingMgr@@QAE@XZ     0042a8b0 f   rylgamelibrary:rankingmgr.obj
 0001:000298f0       ??1CRankingMgr@@QAE@XZ     0042a8f0 f   rylgamelibrary:rankingmgr.obj
 0001:00029900       ??1?$CSingleton@VCPartyMgr@@@@IAE@XZ 0042a900 f i rylgamelibrary:partymgr.obj
 0001:00029910       ?_Erase@?$_Tree@V?$_Tmap_traits@KPAVCCharacter@@U?$less@K@std@@V?$allocator@U?$pair@$$CBKPAVCCharacter@@@std@@@3@$0A@@std@@@std@@IAEXPAU_Node@?$_Tree_nod@V?$_Tmap_traits@KPAVCCharacter@@U?$less@K@std@@V?$allocator@U?$pair@$$CBKPAVCCharacter@@@std@@@3@$0A@@std@@@2@@Z 0042a910 f i rylgamelibrary:partymgr.obj
 0001:00029950       ?_Erase@?$_Tree@V?$_Tmap_traits@KPAVCParty@@U?$less@K@std@@V?$allocator@U?$pair@$$CBKPAVCParty@@@std@@@3@$0A@@std@@@std@@IAEXPAU_Node@?$_Tree_nod@V?$_Tmap_traits@KPAVCParty@@U?$less@K@std@@V?$allocator@U?$pair@$$CBKPAVCParty@@@std@@@3@$0A@@std@@@2@@Z 0042a950 f i rylgamelibrary:partymgr.obj
 0001:00029990       ?_Buynode@?$_Tree@V?$_Tmap_traits@KPAVCCell@@U?$less@K@std@@V?$allocator@U?$pair@$$CBKPAVCCell@@@std@@@3@$0A@@std@@@std@@IAEPAU_Node@?$_Tree_nod@V?$_Tmap_traits@KPAVCCell@@U?$less@K@std@@V?$allocator@U?$pair@$$CBKPAVCCell@@@std@@@3@$0A@@std@@@2@XZ 0042a990 f i rylgamelibrary:duelcellmanager.obj
 0001:00029990       ?_Buynode@?$_Tree@V?$_Tmap_traits@IPAVCMsgProc@@U?$less@I@std@@V?$allocator@U?$pair@$$CBIPAVCMsgProc@@@std@@@3@$0A@@std@@@std@@IAEPAU_Node@?$_Tree_nod@V?$_Tmap_traits@IPAVCMsgProc@@U?$less@I@std@@V?$allocator@U?$pair@$$CBIPAVCMsgProc@@@std@@@3@$0A@@std@@@2@XZ 0042a990 f i rylgamelibrary:msgproc.obj
 0001:00029990       ?_Buynode@?$_Tree@V?$_Tmap_traits@KKU?$less@K@std@@V?$allocator@U?$pair@$$CBKK@std@@@2@$00@std@@@std@@IAEPAU_Node@?$_Tree_nod@V?$_Tmap_traits@KKU?$less@K@std@@V?$allocator@U?$pair@$$CBKK@std@@@2@$00@std@@@2@XZ 0042a990 f i rylgamelibrary:friendlist.obj
 0001:00029990       ?_Buynode@?$_Tree@V?$_Tmap_traits@PAVCSessionPolicy@@IU?$less@PAVCSessionPolicy@@@std@@V?$allocator@U?$pair@QAVCSessionPolicy@@I@std@@@3@$0A@@std@@@std@@IAEPAU_Node@?$_Tree_nod@V?$_Tmap_traits@PAVCSessionPolicy@@IU?$less@PAVCSessionPolicy@@@std@@V?$allocator@U?$pair@QAVCSessionPolicy@@I@std@@@3@$0A@@std@@@2@XZ 0042a990 f i rylgamelibrary:iocpnet.obj
 0001:00029990       ?_Buynode@?$_Tree@V?$_Tmap_traits@KPAVCPacketDispatch@@U?$less@K@std@@V?$allocator@U?$pair@$$CBKPAVCPacketDispatch@@@std@@@3@$0A@@std@@@std@@IAEPAU_Node@?$_Tree_nod@V?$_Tmap_traits@KPAVCPacketDispatch@@U?$less@K@std@@V?$allocator@U?$pair@$$CBKPAVCPacketDispatch@@@std@@@3@$0A@@std@@@2@XZ 0042a990 f i rylgamelibrary:multidispatchstorage.obj
 0001:00029990       ?_Buynode@?$_Tree@V?$_Tmap_traits@KPAVCCharacter@@U?$less@K@std@@V?$allocator@U?$pair@$$CBKPAVCCharacter@@@std@@@3@$0A@@std@@@std@@IAEPAU_Node@?$_Tree_nod@V?$_Tmap_traits@KPAVCCharacter@@U?$less@K@std@@V?$allocator@U?$pair@$$CBKPAVCCharacter@@@std@@@3@$0A@@std@@@2@XZ 0042a990 f i rylgamelibrary:partymgr.obj
 0001:00029990       ?_Buynode@?$_Tree@V?$_Tmap_traits@KPAVCParty@@U?$less@K@std@@V?$allocator@U?$pair@$$CBKPAVCParty@@@std@@@3@$0A@@std@@@std@@IAEPAU_Node@?$_Tree_nod@V?$_Tmap_traits@KPAVCParty@@U?$less@K@std@@V?$allocator@U?$pair@$$CBKPAVCParty@@@std@@@3@$0A@@std@@@2@XZ 0042a990 f i rylgamelibrary:partymgr.obj
 0001:000299d0       ?DestoryPartyList@CPartyMgr@@QAEXXZ 0042a9d0 f   rylgamelibrary:partymgr.obj
 0001:00029a50       ?erase@?$_Tree@V?$_Tmap_traits@KPAVCCharacter@@U?$less@K@std@@V?$allocator@U?$pair@$$CBKPAVCCharacter@@@std@@@3@$0A@@std@@@std@@QAE?AViterator@12@V312@@Z 0042aa50 f i rylgamelibrary:partymgr.obj
 0001:00029a50       ?erase@?$_Tree@V?$_Tmap_traits@KPAVCParty@@U?$less@K@std@@V?$allocator@U?$pair@$$CBKPAVCParty@@@std@@@3@$0A@@std@@@std@@QAE?AViterator@12@V312@@Z 0042aa50 f i rylgamelibrary:partymgr.obj
 0001:00029d10       ?erase@?$_Tree@V?$_Tmap_traits@KPAVCParty@@U?$less@K@std@@V?$allocator@U?$pair@$$CBKPAVCParty@@@std@@@3@$0A@@std@@@std@@QAE?AViterator@12@V312@0@Z 0042ad10 f i rylgamelibrary:partymgr.obj
 0001:00029dd0       ?erase@?$_Tree@V?$_Tmap_traits@KPAVCCharacter@@U?$less@K@std@@V?$allocator@U?$pair@$$CBKPAVCCharacter@@@std@@@3@$0A@@std@@@std@@QAE?AViterator@12@V312@0@Z 0042add0 f i rylgamelibrary:partymgr.obj
 0001:00029e90       ??1?$map@KPAVCParty@@U?$less@K@std@@V?$allocator@U?$pair@$$CBKPAVCParty@@@std@@@3@@std@@QAE@XZ 0042ae90 f i rylgamelibrary:partymgr.obj
 0001:00029ec0       ??1?$map@KPAVCCharacter@@U?$less@K@std@@V?$allocator@U?$pair@$$CBKPAVCCharacter@@@std@@@3@@std@@QAE@XZ 0042aec0 f i rylgamelibrary:partymgr.obj
 0001:00029ef0       ??1CPartyMgr@@QAE@XZ       0042aef0 f   rylgamelibrary:partymgr.obj
 0001:00029fc0       ??0CPartyMgr@@QAE@XZ       0042afc0 f   rylgamelibrary:partymgr.obj
 0001:0002a0c0       ?_Inc@const_iterator@?$_Tree@V?$_Tmap_traits@KPAVCPacketDispatch@@U?$less@K@std@@V?$allocator@U?$pair@$$CBKPAVCPacketDispatch@@@std@@@3@$0A@@std@@@std@@QAEXXZ 0042b0c0 f i rylgamelibrary:multidispatchstorage.obj
 0001:0002a0c0       ?_Inc@const_iterator@?$_Tree@V?$_Tmap_traits@KPAVCParty@@U?$less@K@std@@V?$allocator@U?$pair@$$CBKPAVCParty@@@std@@@3@$0A@@std@@@std@@QAEXXZ 0042b0c0 f i rylgamelibrary:partymgr.obj
 0001:0002a0c0       ?_Inc@const_iterator@?$_Tree@V?$_Tmap_traits@IPAVCMsgProc@@U?$less@I@std@@V?$allocator@U?$pair@$$CBIPAVCMsgProc@@@std@@@3@$0A@@std@@@std@@QAEXXZ 0042b0c0 f i rylgamelibrary:msgproc.obj
 0001:0002a0c0       ?_Inc@const_iterator@?$_Tree@V?$_Tmap_traits@PAVCSessionPolicy@@IU?$less@PAVCSessionPolicy@@@std@@V?$allocator@U?$pair@QAVCSessionPolicy@@I@std@@@3@$0A@@std@@@std@@QAEXXZ 0042b0c0 f i rylgamelibrary:iocpnet.obj
 0001:0002a0c0       ?_Inc@const_iterator@?$_Tree@V?$_Tmap_traits@KPAVCCell@@U?$less@K@std@@V?$allocator@U?$pair@$$CBKPAVCCell@@@std@@@3@$0A@@std@@@std@@QAEXXZ 0042b0c0 f i rylgamelibrary:duelcellmanager.obj
 0001:0002a0c0       ?_Inc@const_iterator@?$_Tree@V?$_Tmap_traits@KKU?$less@K@std@@V?$allocator@U?$pair@$$CBKK@std@@@2@$00@std@@@std@@QAEXXZ 0042b0c0 f i rylgamelibrary:friendlist.obj
 0001:0002a0c0       ?_Inc@const_iterator@?$_Tree@V?$_Tmap_traits@KPAVCCharacter@@U?$less@K@std@@V?$allocator@U?$pair@$$CBKPAVCCharacter@@@std@@@3@$0A@@std@@@std@@QAEXXZ 0042b0c0 f i rylgamelibrary:partymgr.obj
 0001:0002a120       ??1?$CSingleton@VCXRefFriends@@@@IAE@XZ 0042b120 f i rylgamelibrary:friendlist.obj
 0001:0002a130       ?_Erase@?$_Tree@V?$_Tmap_traits@KKU?$less@K@std@@V?$allocator@U?$pair@$$CBKK@std@@@2@$00@std@@@std@@IAEXPAU_Node@?$_Tree_nod@V?$_Tmap_traits@KKU?$less@K@std@@V?$allocator@U?$pair@$$CBKK@std@@@2@$00@std@@@2@@Z 0042b130 f i rylgamelibrary:friendlist.obj
 0001:0002a170       ?erase@?$_Tree@V?$_Tmap_traits@KKU?$less@K@std@@V?$allocator@U?$pair@$$CBKK@std@@@2@$00@std@@@std@@QAE?AViterator@12@V312@@Z 0042b170 f i rylgamelibrary:friendlist.obj
 0001:0002a430       ?erase@?$_Tree@V?$_Tmap_traits@KKU?$less@K@std@@V?$allocator@U?$pair@$$CBKK@std@@@2@$00@std@@@std@@QAE?AViterator@12@V312@0@Z 0042b430 f i rylgamelibrary:friendlist.obj
 0001:0002a4f0       ??0CXRefFriends@@QAE@XZ    0042b4f0 f i rylgamelibrary:friendlist.obj
 0001:0002a560       ??1CXRefFriends@@QAE@XZ    0042b560 f i rylgamelibrary:friendlist.obj
 0001:0002a5d0       ??1?$CSingleton@VCDuelCellManager@@@@IAE@XZ 0042b5d0 f i rylgamelibrary:duelcellmanager.obj
 0001:0002a5e0       ?_Rrotate@?$_Tree@V?$_Tmap_traits@PAVCSessionPolicy@@IU?$less@PAVCSessionPolicy@@@std@@V?$allocator@U?$pair@QAVCSessionPolicy@@I@std@@@3@$0A@@std@@@std@@IAEXPAU_Node@?$_Tree_nod@V?$_Tmap_traits@PAVCSessionPolicy@@IU?$less@PAVCSessionPolicy@@@std@@V?$allocator@U?$pair@QAVCSessionPolicy@@I@std@@@3@$0A@@std@@@2@@Z 0042b5e0 f i rylgamelibrary:iocpnet.obj
 0001:0002a5e0       ?_Rrotate@?$_Tree@V?$_Tmap_traits@KPAVCPacketDispatch@@U?$less@K@std@@V?$allocator@U?$pair@$$CBKPAVCPacketDispatch@@@std@@@3@$0A@@std@@@std@@IAEXPAU_Node@?$_Tree_nod@V?$_Tmap_traits@KPAVCPacketDispatch@@U?$less@K@std@@V?$allocator@U?$pair@$$CBKPAVCPacketDispatch@@@std@@@3@$0A@@std@@@2@@Z 0042b5e0 f i rylgamelibrary:multidispatchstorage.obj
 0001:0002a5e0       ?_Rrotate@?$_Tree@V?$_Tmap_traits@IPAVCMsgProc@@U?$less@I@std@@V?$allocator@U?$pair@$$CBIPAVCMsgProc@@@std@@@3@$0A@@std@@@std@@IAEXPAU_Node@?$_Tree_nod@V?$_Tmap_traits@IPAVCMsgProc@@U?$less@I@std@@V?$allocator@U?$pair@$$CBIPAVCMsgProc@@@std@@@3@$0A@@std@@@2@@Z 0042b5e0 f i rylgamelibrary:msgproc.obj
 0001:0002a5e0       ?_Rrotate@?$_Tree@V?$_Tmap_traits@KPAVCCharacter@@U?$less@K@std@@V?$allocator@U?$pair@$$CBKPAVCCharacter@@@std@@@3@$0A@@std@@@std@@IAEXPAU_Node@?$_Tree_nod@V?$_Tmap_traits@KPAVCCharacter@@U?$less@K@std@@V?$allocator@U?$pair@$$CBKPAVCCharacter@@@std@@@3@$0A@@std@@@2@@Z 0042b5e0 f i rylgamelibrary:partymgr.obj
 0001:0002a5e0       ?_Rrotate@?$_Tree@V?$_Tmap_traits@HPAV?$list@PAVIOPCode@@V?$allocator@PAVIOPCode@@@std@@@std@@U?$less@H@2@V?$allocator@U?$pair@$$CBHPAV?$list@PAVIOPCode@@V?$allocator@PAVIOPCode@@@std@@@std@@@std@@@2@$0A@@std@@@std@@IAEXPAU_Node@?$_Tree_nod@V?$_Tmap_traits@HPAV?$list@PAVIOPCode@@V?$allocator@PAVIOPCode@@@std@@@std@@U?$less@H@2@V?$allocator@U?$pair@$$CBHPAV?$list@PAVIOPCode@@V?$allocator@PAVIOPCode@@@std@@@std@@@std@@@2@$0A@@std@@@2@@Z 0042b5e0 f i rylgamelibrary:intermediatecode.obj
 0001:0002a5e0       ?_Rrotate@?$_Tree@V?$_Tmap_traits@KPAVCCell@@U?$less@K@std@@V?$allocator@U?$pair@$$CBKPAVCCell@@@std@@@3@$0A@@std@@@std@@IAEXPAU_Node@?$_Tree_nod@V?$_Tmap_traits@KPAVCCell@@U?$less@K@std@@V?$allocator@U?$pair@$$CBKPAVCCell@@@std@@@3@$0A@@std@@@2@@Z 0042b5e0 f i rylgamelibrary:duelcellmanager.obj
 0001:0002a5e0       ?_Rrotate@?$_Tree@V?$_Tmap_traits@KKU?$less@K@std@@V?$allocator@U?$pair@$$CBKK@std@@@2@$00@std@@@std@@IAEXPAU_Node@?$_Tree_nod@V?$_Tmap_traits@KKU?$less@K@std@@V?$allocator@U?$pair@$$CBKK@std@@@2@$00@std@@@2@@Z 0042b5e0 f i rylgamelibrary:friendlist.obj
 0001:0002a5e0       ?_Rrotate@?$_Tree@V?$_Tmap_traits@KPAVCParty@@U?$less@K@std@@V?$allocator@U?$pair@$$CBKPAVCParty@@@std@@@3@$0A@@std@@@std@@IAEXPAU_Node@?$_Tree_nod@V?$_Tmap_traits@KPAVCParty@@U?$less@K@std@@V?$allocator@U?$pair@$$CBKPAVCParty@@@std@@@3@$0A@@std@@@2@@Z 0042b5e0 f i rylgamelibrary:partymgr.obj
 0001:0002a640       ?_Erase@?$_Tree@V?$_Tmap_traits@KPAVCCell@@U?$less@K@std@@V?$allocator@U?$pair@$$CBKPAVCCell@@@std@@@3@$0A@@std@@@std@@IAEXPAU_Node@?$_Tree_nod@V?$_Tmap_traits@KPAVCCell@@U?$less@K@std@@V?$allocator@U?$pair@$$CBKPAVCCell@@@std@@@3@$0A@@std@@@2@@Z 0042b640 f i rylgamelibrary:duelcellmanager.obj
 0001:0002a680       ?erase@?$_Tree@V?$_Tmap_traits@KPAVCCell@@U?$less@K@std@@V?$allocator@U?$pair@$$CBKPAVCCell@@@std@@@3@$0A@@std@@@std@@QAE?AViterator@12@V312@@Z 0042b680 f i rylgamelibrary:duelcellmanager.obj
 0001:0002a940       ?erase@?$_Tree@V?$_Tmap_traits@KPAVCCell@@U?$less@K@std@@V?$allocator@U?$pair@$$CBKPAVCCell@@@std@@@3@$0A@@std@@@std@@QAE?AViterator@12@V312@0@Z 0042b940 f i rylgamelibrary:duelcellmanager.obj
 0001:0002aa00       ??1CDuelCellManager@@QAE@XZ 0042ba00 f i rylgamelibrary:duelcellmanager.obj
 0001:0002aa70       ??0CDuelCellManager@@AAE@XZ 0042ba70 f i rylgamelibrary:duelcellmanager.obj
 0001:0002aae0       ??1CFSMState@@QAE@XZ       0042bae0 f   rylgamelibrary:fsmstate.obj
 0001:0002ab20       ??1?$CSingleton@VCFSM@@@@IAE@XZ 0042bb20 f i rylgamelibrary:fsm.obj
 0001:0002ab30       ??0CFSM@@IAE@XZ            0042bb30 f   rylgamelibrary:fsm.obj
 0001:0002ab60       ??1CFSM@@QAE@XZ            0042bb60 f   rylgamelibrary:fsm.obj
 0001:0002abd0       ??1PhaseNode@Quest@@QAE@XZ 0042bbd0 f i rylgamelibrary:npc.obj
 0001:0002ac00       ??1TriggerNode@Quest@@QAE@XZ 0042bc00 f i rylgamelibrary:npc.obj
 0001:0002ac40       _inflate_codes_free        0042bc40 f   rylgamelibrary:infcodes.obj
 0001:0002ac60       ??1?$CSingleton@VCQuestMgr@@@@IAE@XZ 0042bc60 f i rylgamelibrary:questmgr.obj
 0001:0002ac70       ??1QuestNode@Quest@@QAE@XZ 0042bc70 f i rylgamelibrary:questmgr.obj
 0001:0002aca0       ?ClearQuest@CQuestMgr@@AAEXXZ 0042bca0 f   rylgamelibrary:questmgr.obj
 0001:0002aed0       ??1CQuestMgr@@QAE@XZ       0042bed0 f   rylgamelibrary:questmgr.obj
 0001:0002af00       ??0CQuestMgr@@QAE@XZ       0042bf00 f   rylgamelibrary:questmgr.obj
 0001:0002af50       ??0CCrc32@@QAE@XZ          0042bf50 f   rylgamelibrary:Crc32Mem.obj
 0001:0002af90       ??1CCrc32@@QAE@XZ          0042bf90 f   rylgamelibrary:Crc32Mem.obj
 0001:0002afa0       ?CompilerMessage2@@YAXPBDZZ 0042bfa0 f   rylgamelibrary:message.obj
 0001:0002afe0       ?ErrorMessage@@YAXHPBD@Z   0042bfe0 f   rylgamelibrary:message.obj
 0001:0002b000       ?WarningMessage2@@YAXHPBDZZ 0042c000 f   rylgamelibrary:message.obj
 0001:0002b050       ?ScriptSystemError@@YAXPBD@Z 0042c050 f   rylgamelibrary:message.obj
 0001:0002b070       ?DefaultMessageFunction@@YAXPBD@Z 0042c070 f   rylgamelibrary:message.obj
 0001:0002b0a0       ?_Lrotate@?$_Tree@V?$_Tmap_traits@KPAVCCharacter@@U?$less@K@std@@V?$allocator@U?$pair@$$CBKPAVCCharacter@@@std@@@3@$0A@@std@@@std@@IAEXPAU_Node@?$_Tree_nod@V?$_Tmap_traits@KPAVCCharacter@@U?$less@K@std@@V?$allocator@U?$pair@$$CBKPAVCCharacter@@@std@@@3@$0A@@std@@@2@@Z 0042c0a0 f i rylgamelibrary:partymgr.obj
 0001:0002b0a0       ?_Lrotate@?$_Tree@V?$_Tmap_traits@KPAVCCell@@U?$less@K@std@@V?$allocator@U?$pair@$$CBKPAVCCell@@@std@@@3@$0A@@std@@@std@@IAEXPAU_Node@?$_Tree_nod@V?$_Tmap_traits@KPAVCCell@@U?$less@K@std@@V?$allocator@U?$pair@$$CBKPAVCCell@@@std@@@3@$0A@@std@@@2@@Z 0042c0a0 f i rylgamelibrary:duelcellmanager.obj
 0001:0002b0a0       ?_Lrotate@?$_Tree@V?$_Tmap_traits@IPAVCMsgProc@@U?$less@I@std@@V?$allocator@U?$pair@$$CBIPAVCMsgProc@@@std@@@3@$0A@@std@@@std@@IAEXPAU_Node@?$_Tree_nod@V?$_Tmap_traits@IPAVCMsgProc@@U?$less@I@std@@V?$allocator@U?$pair@$$CBIPAVCMsgProc@@@std@@@3@$0A@@std@@@2@@Z 0042c0a0 f i rylgamelibrary:msgproc.obj
 0001:0002b0a0       ?_Lrotate@?$_Tree@V?$_Tmap_traits@PAVCSessionPolicy@@IU?$less@PAVCSessionPolicy@@@std@@V?$allocator@U?$pair@QAVCSessionPolicy@@I@std@@@3@$0A@@std@@@std@@IAEXPAU_Node@?$_Tree_nod@V?$_Tmap_traits@PAVCSessionPolicy@@IU?$less@PAVCSessionPolicy@@@std@@V?$allocator@U?$pair@QAVCSessionPolicy@@I@std@@@3@$0A@@std@@@2@@Z 0042c0a0 f i rylgamelibrary:iocpnet.obj
 0001:0002b0a0       ?_Lrotate@?$_Tree@V?$_Tmap_traits@HPAV?$list@PAVIOPCode@@V?$allocator@PAVIOPCode@@@std@@@std@@U?$less@H@2@V?$allocator@U?$pair@$$CBHPAV?$list@PAVIOPCode@@V?$allocator@PAVIOPCode@@@std@@@std@@@std@@@2@$0A@@std@@@std@@IAEXPAU_Node@?$_Tree_nod@V?$_Tmap_traits@HPAV?$list@PAVIOPCode@@V?$allocator@PAVIOPCode@@@std@@@std@@U?$less@H@2@V?$allocator@U?$pair@$$CBHPAV?$list@PAVIOPCode@@V?$allocator@PAVIOPCode@@@std@@@std@@@std@@@2@$0A@@std@@@2@@Z 0042c0a0 f i rylgamelibrary:intermediatecode.obj
 0001:0002b0a0       ?_Lrotate@?$_Tree@V?$_Tmap_traits@KKU?$less@K@std@@V?$allocator@U?$pair@$$CBKK@std@@@2@$00@std@@@std@@IAEXPAU_Node@?$_Tree_nod@V?$_Tmap_traits@KKU?$less@K@std@@V?$allocator@U?$pair@$$CBKK@std@@@2@$00@std@@@2@@Z 0042c0a0 f i rylgamelibrary:friendlist.obj
 0001:0002b0a0       ?_Lrotate@?$_Tree@V?$_Tmap_traits@KPAVCPacketDispatch@@U?$less@K@std@@V?$allocator@U?$pair@$$CBKPAVCPacketDispatch@@@std@@@3@$0A@@std@@@std@@IAEXPAU_Node@?$_Tree_nod@V?$_Tmap_traits@KPAVCPacketDispatch@@U?$less@K@std@@V?$allocator@U?$pair@$$CBKPAVCPacketDispatch@@@std@@@3@$0A@@std@@@2@@Z 0042c0a0 f i rylgamelibrary:multidispatchstorage.obj
 0001:0002b0a0       ?_Lrotate@?$_Tree@V?$_Tmap_traits@KPAVCParty@@U?$less@K@std@@V?$allocator@U?$pair@$$CBKPAVCParty@@@std@@@3@$0A@@std@@@std@@IAEXPAU_Node@?$_Tree_nod@V?$_Tmap_traits@KPAVCParty@@U?$less@K@std@@V?$allocator@U?$pair@$$CBKPAVCParty@@@std@@@3@$0A@@std@@@2@@Z 0042c0a0 f i rylgamelibrary:partymgr.obj
 0001:0002b100       ??$fill@PAW4Type@ItemType@Item@@W4123@@std@@YAXPAW4Type@ItemType@Item@@0ABW4123@@Z 0042c100 f i rylgamelibrary:itemconstants.obj
 0001:0002b100       ??$fill@PAHH@std@@YAXPAH0ABH@Z 0042c100 f i rylgamelibrary:reloctable.obj
 0001:0002b100       ??$fill@PAKK@std@@YAXPAK0ABK@Z 0042c100 f i masterpassword.obj
 0001:0002b100       ??$fill@PAPAV?$pool@Udefault_user_allocator_new_delete@boost@@@boost@@PAV12@@std@@YAXPAPAV?$pool@Udefault_user_allocator_new_delete@boost@@@boost@@0ABQAV12@@Z 0042c100 f i rylgamelibrary:bufferfactory.obj
 0001:0002b100       ??$fill@PAPADPAD@std@@YAXPAPAD0ABQAD@Z 0042c100 f i rylgamelibrary:tokenlizedfile.obj
 0001:0002b120       ??$copy_backward@PAHPAH@std@@YAPAHPAH00@Z 0042c120 f i rylgamelibrary:reloctable.obj
 0001:0002b120       ??$copy_backward@PAPADPAPAD@std@@YAPAPADPAPAD00@Z 0042c120 f i rylgamelibrary:tokenlizedfile.obj
 0001:0002b120       ??$copy_backward@PAPAV?$pool@Udefault_user_allocator_new_delete@boost@@@boost@@PAPAV12@@std@@YAPAPAV?$pool@Udefault_user_allocator_new_delete@boost@@@boost@@PAPAV12@00@Z 0042c120 f i rylgamelibrary:bufferfactory.obj
 0001:0002b120       ??$copy_backward@PAKPAK@std@@YAPAKPAK00@Z 0042c120 f i masterpassword.obj
 0001:0002b150       ??$copy_backward@PAUParseData@ItemDataParser@@PAU12@@std@@YAPAUParseData@ItemDataParser@@PAU12@00@Z 0042c150 f i rylgamelibrary:itemdataparser.obj
 0001:0002b150       ??$copy_backward@PAU?$pair@KK@std@@PAU12@@std@@YAPAU?$pair@KK@0@PAU10@00@Z 0042c150 f i rylgamelibrary:rylserverdispatch.obj
 0001:0002b150       ??$copy_backward@PAU?$pair@W4eStdFunc@@H@std@@PAU12@@std@@YAPAU?$pair@W4eStdFunc@@H@0@PAU10@00@Z 0042c150 f i rylgamelibrary:reloctable.obj
 0001:0002b180       ?_Xlen@?$vector@U?$pair@W4eStdFunc@@H@std@@V?$allocator@U?$pair@W4eStdFunc@@H@std@@@2@@std@@IBEXXZ 0042c180 f i rylgamelibrary:reloctable.obj
 0001:0002b180       ?_Xlen@?$vector@HV?$allocator@H@std@@@std@@IBEXXZ 0042c180 f i rylgamelibrary:reloctable.obj
 0001:0002b1f0       ?_Insert_n@?$vector@HV?$allocator@H@std@@@std@@IAEXViterator@12@IABH@Z 0042c1f0 f i rylgamelibrary:reloctable.obj
 0001:0002b3d0       ?_Insert_n@?$vector@U?$pair@W4eStdFunc@@H@std@@V?$allocator@U?$pair@W4eStdFunc@@H@std@@@2@@std@@IAEXViterator@12@IABU?$pair@W4eStdFunc@@H@2@@Z 0042c3d0 f i rylgamelibrary:reloctable.obj
 0001:0002b620       ?push_back@?$vector@U?$pair@W4eStdFunc@@H@std@@V?$allocator@U?$pair@W4eStdFunc@@H@std@@@2@@std@@QAEXABU?$pair@W4eStdFunc@@H@2@@Z 0042c620 f i rylgamelibrary:reloctable.obj
 0001:0002b690       ?AddGlobalVar@CRelocTable@@QAEXH@Z 0042c690 f   rylgamelibrary:reloctable.obj
 0001:0002b6e0       ?AddConstString@CRelocTable@@QAEXH@Z 0042c6e0 f   rylgamelibrary:reloctable.obj
 0001:0002b730       ?AddFuncBind@CRelocTable@@QAEXW4eStdFunc@@H@Z 0042c730 f   rylgamelibrary:reloctable.obj
 0001:0002b760       ?GetTypeOfConst@CSymbolTable@@QAE?AW4eDataType@@H@Z 0042c760 f   rylgamelibrary:symboltable.obj
 0001:0002b760       ?GetTypeOfVar@CSymbolTable@@QAE?AW4eDataType@@H@Z 0042c760 f   rylgamelibrary:symboltable.obj
 0001:0002b770       ?GetCountOfVar@CSymbolTable@@QAEHH@Z 0042c770 f   rylgamelibrary:symboltable.obj
 0001:0002b770       ?GetOffsetOfConst@CSymbolTable@@QAEHH@Z 0042c770 f   rylgamelibrary:symboltable.obj
 0001:0002b780       ?GetOffsetOfVar@CSymbolTable@@QAEHH@Z 0042c780 f   rylgamelibrary:symboltable.obj
 0001:0002b790       ?GetTypeOfFunc@CSymbolTable@@QAE?AUSFuncType@@H@Z 0042c790 f   rylgamelibrary:symboltable.obj
 0001:0002b7a0       ?GetArgCount@SFuncType@@QAEHXZ 0042c7a0 f   rylgamelibrary:symboltable.obj
 0001:0002b7c0       ?ToString@SFuncType@@QAEPBDPBD@Z 0042c7c0 f   rylgamelibrary:symboltable.obj
 0001:0002b870       ?GetNameOfVar@CSymbolTable@@QAEPBDH@Z 0042c870 f   rylgamelibrary:symboltable.obj
 0001:0002b870       ?GetNameOfConst@CSymbolTable@@QAEPBDH@Z 0042c870 f   rylgamelibrary:symboltable.obj
 0001:0002b870       ?GetNameOfFunc@CSymbolTable@@QAEPBDH@Z 0042c870 f   rylgamelibrary:symboltable.obj
 0001:0002b890       ?GetTypeStringOfFunc@CSymbolTable@@QAEPBDH@Z 0042c890 f   rylgamelibrary:symboltable.obj
 0001:0002b8d0       ?GetLocalVarSize@CSymbolTable@@QAEHH@Z 0042c8d0 f   rylgamelibrary:symboltable.obj
 0001:0002b980       ?GenCode_Error_Statement@@YAXPAUSNode@@W4eRegister@@@Z 0042c980 f   rylgamelibrary:imcodegen.obj
 0001:0002b9a0       ??_GIOPCode@@UAEPAXI@Z     0042c9a0 f i rylgamelibrary:imcodegen.obj
 0001:0002b9a0       ??_EIOPCode@@UAEPAXI@Z     0042c9a0 f i rylgamelibrary:imcodegen.obj
 0001:0002b9c0       ?GenCode_FirstChild_Generate@@YAXPAUSNode@@W4eRegister@@@Z 0042c9c0 f   rylgamelibrary:imcodegen.obj
 0001:0002b9e0       ?GenCode_SecondChild_Generate@@YAXPAUSNode@@W4eRegister@@@Z 0042c9e0 f   rylgamelibrary:imcodegen.obj
 0001:0002ba00       ?GenCode_TwoChild_Generate@@YAXPAUSNode@@W4eRegister@@@Z 0042ca00 f   rylgamelibrary:imcodegen.obj
 0001:0002ba30       ?HandleMARK@@YAXViterator@?$list@PAVIOPCode@@V?$allocator@PAVIOPCode@@@std@@@std@@0PAVIOPCode@@1@Z 0042ca30 f   rylgamelibrary:imcodegen.obj
 0001:0002bab0       ?_Insert@?$_Tree@V?$_Tmap_traits@HPAV?$list@PAVIOPCode@@V?$allocator@PAVIOPCode@@@std@@@std@@U?$less@H@2@V?$allocator@U?$pair@$$CBHPAV?$list@PAVIOPCode@@V?$allocator@PAVIOPCode@@@std@@@std@@@std@@@2@$0A@@std@@@std@@IAE?AViterator@12@_NPAU_Node@?$_Tree_nod@V?$_Tmap_traits@HPAV?$list@PAVIOPCode@@V?$allocator@PAVIOPCode@@@std@@@std@@U?$less@H@2@V?$allocator@U?$pair@$$CBHPAV?$list@PAVIOPCode@@V?$allocator@PAVIOPCode@@@std@@@std@@@std@@@2@$0A@@std@@@2@ABU?$pair@$$CBHPAV?$list@PAVIOPCode@@V?$allocator@PAVIOPCode@@@std@@@std@@@2@@Z 0042cab0 f i rylgamelibrary:imcodegen.obj
 0001:0002bc60       ?_Incsize@?$list@PAVIOPCode@@V?$allocator@PAVIOPCode@@@std@@@std@@IAEXI@Z 0042cc60 f i rylgamelibrary:imcodegen.obj
 0001:0002bd00       ?insert@?$_Tree@V?$_Tmap_traits@HPAV?$list@PAVIOPCode@@V?$allocator@PAVIOPCode@@@std@@@std@@U?$less@H@2@V?$allocator@U?$pair@$$CBHPAV?$list@PAVIOPCode@@V?$allocator@PAVIOPCode@@@std@@@std@@@std@@@2@$0A@@std@@@std@@QAE?AU?$pair@Viterator@?$_Tree@V?$_Tmap_traits@HPAV?$list@PAVIOPCode@@V?$allocator@PAVIOPCode@@@std@@@std@@U?$less@H@2@V?$allocator@U?$pair@$$CBHPAV?$list@PAVIOPCode@@V?$allocator@PAVIOPCode@@@std@@@std@@@std@@@2@$0A@@std@@@std@@_N@2@ABU?$pair@$$CBHPAV?$list@PAVIOPCode@@V?$allocator@PAVIOPCode@@@std@@@std@@@2@@Z 0042cd00 f i rylgamelibrary:imcodegen.obj
 0001:0002bdc0       ?push_back@?$list@PAVIOPCode@@V?$allocator@PAVIOPCode@@@std@@@std@@QAEXABQAVIOPCode@@@Z 0042cdc0 f i rylgamelibrary:imcodegen.obj
 0001:0002be00       ?GenCode_DataTypeToString@@YAXW4eDataType@@W4eRegister@@@Z 0042ce00 f   rylgamelibrary:imcodegen.obj
 0001:0002c3d0       ?GenCode_If_Statement@@YAXPAUSNode@@W4eRegister@@@Z 0042d3d0 f   rylgamelibrary:imcodegen.obj
 0001:0002c550       ?GenCode_If_Else_Statement@@YAXPAUSNode@@W4eRegister@@@Z 0042d550 f   rylgamelibrary:imcodegen.obj
 0001:0002c7b0       ?GenCode_Switch_Statement@@YAXPAUSNode@@W4eRegister@@@Z 0042d7b0 f   rylgamelibrary:imcodegen.obj
 0001:0002cb90       ?GenCode_For_Statement@@YAXPAUSNode@@W4eRegister@@@Z 0042db90 f   rylgamelibrary:imcodegen.obj
 0001:0002cf60       ?GenCode_While_Statement@@YAXPAUSNode@@W4eRegister@@@Z 0042df60 f   rylgamelibrary:imcodegen.obj
 0001:0002d200       ?GenCode_Break_Statement@@YAXPAUSNode@@W4eRegister@@@Z 0042e200 f   rylgamelibrary:imcodegen.obj
 0001:0002d240       ?GenCode_Continue_Statement@@YAXPAUSNode@@W4eRegister@@@Z 0042e240 f   rylgamelibrary:imcodegen.obj
 0001:0002d280       ?GenCode_Return_Statement@@YAXPAUSNode@@W4eRegister@@@Z 0042e280 f   rylgamelibrary:imcodegen.obj
 0001:0002d2e0       ?GenCode_Variable@@YAXPAUSNode@@W4eRegister@@@Z 0042e2e0 f   rylgamelibrary:imcodegen.obj
 0001:0002d390       ?GenCode_Init_Declaration@@YAXPAUSNode@@W4eRegister@@@Z 0042e390 f   rylgamelibrary:imcodegen.obj
 0001:0002d6f0       ?GenCode_Normal_Declaration@@YAXPAUSNode@@W4eRegister@@@Z 0042e6f0 f   rylgamelibrary:imcodegen.obj
 0001:0002d790       ?GenCode_Array_Init@@YAXPAUSNode@@H@Z 0042e790 f   rylgamelibrary:imcodegen.obj
 0001:0002db70       ?GenCode_Array_Initialize@@YAXPAUSNode@@W4eRegister@@@Z 0042eb70 f   rylgamelibrary:imcodegen.obj
 0001:0002db80       ?GenCode_Array_Initialize2@@YAXPAUSNode@@W4eRegister@@@Z 0042eb80 f   rylgamelibrary:imcodegen.obj
 0001:0002db90       ?GenCode_Function_Declaration@@YAXPAUSNode@@W4eRegister@@@Z 0042eb90 f   rylgamelibrary:imcodegen.obj
 0001:0002de50       ?GenCode_Function_Definition@@YAXPAUSNode@@W4eRegister@@@Z 0042ee50 f   rylgamelibrary:imcodegen.obj
 0001:0002e220       ?GenCode_Constant_Expression@@YAXPAUSNode@@W4eRegister@@@Z 0042f220 f   rylgamelibrary:imcodegen.obj
 0001:0002e2c0       ?GenCode_Assignment_Expression@@YAXPAUSNode@@W4eRegister@@@Z 0042f2c0 f   rylgamelibrary:imcodegen.obj
 0001:0002e780       ?GenCode_OR_Expression@@YAXPAUSNode@@W4eRegister@@@Z 0042f780 f   rylgamelibrary:imcodegen.obj
 0001:0002ebc0       ?GenCode_AND_Expression@@YAXPAUSNode@@W4eRegister@@@Z 0042fbc0 f   rylgamelibrary:imcodegen.obj
 0001:0002f000       ?GenCode_NOT_Expression@@YAXPAUSNode@@W4eRegister@@@Z 00430000 f   rylgamelibrary:imcodegen.obj
 0001:0002f110       ?GenCode_Equality_Expression@@YAXPAUSNode@@W4eRegister@@@Z 00430110 f   rylgamelibrary:imcodegen.obj
 0001:0002f330       ?GenCode_NotEqual_Expression@@YAXPAUSNode@@W4eRegister@@@Z 00430330 f   rylgamelibrary:imcodegen.obj
 0001:0002f550       ?GenCode_LessThan_Expression@@YAXPAUSNode@@W4eRegister@@@Z 00430550 f   rylgamelibrary:imcodegen.obj
 0001:0002f8f0       ?GenCode_MoreThan_Expression@@YAXPAUSNode@@W4eRegister@@@Z 004308f0 f   rylgamelibrary:imcodegen.obj
 0001:0002fc90       ?GenCode_LessThanEqual_Expression@@YAXPAUSNode@@W4eRegister@@@Z 00430c90 f   rylgamelibrary:imcodegen.obj
 0001:00030030       ?GenCode_MoreThanEqual_Expression@@YAXPAUSNode@@W4eRegister@@@Z 00431030 f   rylgamelibrary:imcodegen.obj
 0001:000303d0       ?GenCode_Addition_Expression@@YAXPAUSNode@@W4eRegister@@@Z 004313d0 f   rylgamelibrary:imcodegen.obj
 0001:00030d30       ?GenCode_Subtraction_Expression@@YAXPAUSNode@@W4eRegister@@@Z 00431d30 f   rylgamelibrary:imcodegen.obj
 0001:000310c0       ?GenCode_Multiplication_Expression@@YAXPAUSNode@@W4eRegister@@@Z 004320c0 f   rylgamelibrary:imcodegen.obj
 0001:00031450       ?GenCode_Division_Expression@@YAXPAUSNode@@W4eRegister@@@Z 00432450 f   rylgamelibrary:imcodegen.obj
 0001:000317e0       ?GenCode_Reminder_Expression@@YAXPAUSNode@@W4eRegister@@@Z 004327e0 f   rylgamelibrary:imcodegen.obj
 0001:00031900       ?GenCode_Compound_Addition@@YAXPAUSNode@@W4eRegister@@@Z 00432900 f   rylgamelibrary:imcodegen.obj
 0001:000322e0       ?GenCode_Compound_Subtraction@@YAXPAUSNode@@W4eRegister@@@Z 004332e0 f   rylgamelibrary:imcodegen.obj
 0001:000326e0       ?GenCode_Compound_Multiplication@@YAXPAUSNode@@W4eRegister@@@Z 004336e0 f   rylgamelibrary:imcodegen.obj
 0001:00032ae0       ?GenCode_Compound_Division@@YAXPAUSNode@@W4eRegister@@@Z 00433ae0 f   rylgamelibrary:imcodegen.obj
 0001:00032ee0       ?GenCode_Compound_Reminder@@YAXPAUSNode@@W4eRegister@@@Z 00433ee0 f   rylgamelibrary:imcodegen.obj
 0001:000330c0       ?GenCode_PrefixIncrement@@YAXPAUSNode@@W4eRegister@@@Z 004340c0 f   rylgamelibrary:imcodegen.obj
 0001:00033450       ?GenCode_PrefixDecrement@@YAXPAUSNode@@W4eRegister@@@Z 00434450 f   rylgamelibrary:imcodegen.obj
 0001:000337d0       ?GenCode_Array_Indexing@@YAXPAUSNode@@W4eRegister@@@Z 004347d0 f   rylgamelibrary:imcodegen.obj
 0001:00033950       ?GenCode_Function_Call@@YAXPAUSNode@@W4eRegister@@@Z 00434950 f   rylgamelibrary:imcodegen.obj
 0001:00033be0       ?GenCode_PostfixIncrement@@YAXPAUSNode@@W4eRegister@@@Z 00434be0 f   rylgamelibrary:imcodegen.obj
 0001:00033f80       ?GenCode_PostfixDecrement@@YAXPAUSNode@@W4eRegister@@@Z 00434f80 f   rylgamelibrary:imcodegen.obj
 0001:00034320       ??0Conversion@@QAE@PAU_CONST_@@H@Z 00435320 f i rylgamelibrary:imcodeunits.obj
 0001:000343e0       ?Code_RM32_Offset@@YAHPAEEHHJH@Z 004353e0 f   rylgamelibrary:imcodeunits.obj
 0001:00034480       ?Code_RM32@@YAHPAEEHHHJ@Z  00435480 f i rylgamelibrary:imcodeunits.obj
 0001:000344c0       ?Code_RM32_CodeSize_Offset@@YAJHH@Z 004354c0 f   rylgamelibrary:imcodeunits.obj
 0001:000344e0       ?Show@COP_call@@UAEXP6AXPBDZZ@Z 004354e0 f   rylgamelibrary:imcodeunits.obj
 0001:00034500       ?ToMachineCode@COP_mov@@UAEHPAE@Z 00435500 f   rylgamelibrary:imcodeunits.obj
 0001:00034750       ?Addressing@COP_mov@@UAEJJ@Z 00435750 f   rylgamelibrary:imcodeunits.obj
 0001:00034850       ?Show@COP_mov@@UAEXP6AXPBDZZ@Z 00435850 f   rylgamelibrary:imcodeunits.obj
 0001:000349d0       ?ToMachineCode@COP_nop@@UAEHPAE@Z 004359d0 f   rylgamelibrary:imcodeunits.obj
 0001:000349e0       ?Addressing@COP_nop@@UAEJJ@Z 004359e0 f   rylgamelibrary:imcodeunits.obj
 0001:000349e0       ?Addressing@COP_push@@UAEJJ@Z 004359e0 f   rylgamelibrary:imcodeunits.obj
 0001:000349e0       ?Addressing@COP_ret@@UAEJJ@Z 004359e0 f   rylgamelibrary:imcodeunits.obj
 0001:000349e0       ?Addressing@COP_pop@@UAEJJ@Z 004359e0 f   rylgamelibrary:imcodeunits.obj
 0001:000349f0       ?Show@COP_nop@@UAEXP6AXPBDZZ@Z 004359f0 f   rylgamelibrary:imcodeunits.obj
 0001:00034a00       ?ToMachineCode@COP_add@@UAEHPAE@Z 00435a00 f   rylgamelibrary:imcodeunits.obj
 0001:00034a70       ?Show@COP_add@@UAEXP6AXPBDZZ@Z 00435a70 f   rylgamelibrary:imcodeunits.obj
 0001:00034ae0       ?ToMachineCode@COP_sub@@UAEHPAE@Z 00435ae0 f   rylgamelibrary:imcodeunits.obj
 0001:00034b50       ?Addressing@COP_sub@@UAEJJ@Z 00435b50 f   rylgamelibrary:imcodeunits.obj
 0001:00034b50       ?Addressing@COP_add@@UAEJJ@Z 00435b50 f   rylgamelibrary:imcodeunits.obj
 0001:00034b80       ?Show@COP_sub@@UAEXP6AXPBDZZ@Z 00435b80 f   rylgamelibrary:imcodeunits.obj
 0001:00034bf0       ?ToMachineCode@COP_imul@@UAEHPAE@Z 00435bf0 f   rylgamelibrary:imcodeunits.obj
 0001:00034c20       ?Show@COP_imul@@UAEXP6AXPBDZZ@Z 00435c20 f   rylgamelibrary:imcodeunits.obj
 0001:00034c60       ?ToMachineCode@COP_idiv@@UAEHPAE@Z 00435c60 f   rylgamelibrary:imcodeunits.obj
 0001:00034c80       ?Show@COP_idiv@@UAEXP6AXPBDZZ@Z 00435c80 f   rylgamelibrary:imcodeunits.obj
 0001:00034cb0       ?ToMachineCode@COP_push@@UAEHPAE@Z 00435cb0 f   rylgamelibrary:imcodeunits.obj
 0001:00034cd0       ?Show@COP_push@@UAEXP6AXPBDZZ@Z 00435cd0 f   rylgamelibrary:imcodeunits.obj
 0001:00034cf0       ?ToMachineCode@COP_pop@@UAEHPAE@Z 00435cf0 f   rylgamelibrary:imcodeunits.obj
 0001:00034d10       ?Show@COP_pop@@UAEXP6AXPBDZZ@Z 00435d10 f   rylgamelibrary:imcodeunits.obj
 0001:00034d30       ?ToMachineCode@COP_jmp@@UAEHPAE@Z 00435d30 f   rylgamelibrary:imcodeunits.obj
 0001:00034d70       ?Addressing@COP_call@@UAEJJ@Z 00435d70 f   rylgamelibrary:imcodeunits.obj
 0001:00034d70       ?Addressing@COP_jmp@@UAEJJ@Z 00435d70 f   rylgamelibrary:imcodeunits.obj
 0001:00034d80       ?Show@COP_jmp@@UAEXP6AXPBDZZ@Z 00435d80 f   rylgamelibrary:imcodeunits.obj
 0001:00034da0       ?ToMachineCode@COP_jcc@@UAEHPAE@Z 00435da0 f   rylgamelibrary:imcodeunits.obj
 0001:00034e50       ?Addressing@COP_jcc@@UAEJJ@Z 00435e50 f   rylgamelibrary:imcodeunits.obj
 0001:00034e60       ?Show@COP_jcc@@UAEXP6AXPBDZZ@Z 00435e60 f   rylgamelibrary:imcodeunits.obj
 0001:00034e90       ?ToMachineCode@COP_jmpmark@@UAEHPAE@Z 00435e90 f   rylgamelibrary:imcodeunits.obj
 0001:00034ea0       ?Addressing@COP_jmpmark@@UAEJJ@Z 00435ea0 f   rylgamelibrary:imcodeunits.obj
 0001:00034eb0       ?Show@COP_jmpmark@@UAEXP6AXPBDZZ@Z 00435eb0 f   rylgamelibrary:imcodeunits.obj
 0001:00034ee0       ?ToMachineCode@COP_cmp@@UAEHPAE@Z 00435ee0 f   rylgamelibrary:imcodeunits.obj
 0001:00035020       ?Addressing@COP_cmp@@UAEJJ@Z 00436020 f   rylgamelibrary:imcodeunits.obj
 0001:00035080       ?Show@COP_cmp@@UAEXP6AXPBDZZ@Z 00436080 f   rylgamelibrary:imcodeunits.obj
 0001:00035110       ?ToMachineCode@COP_ret@@UAEHPAE@Z 00436110 f   rylgamelibrary:imcodeunits.obj
 0001:00035120       ?Show@COP_ret@@UAEXP6AXPBDZZ@Z 00436120 f   rylgamelibrary:imcodeunits.obj
 0001:00035130       ?ToMachineCode@COP_setcc@@UAEHPAE@Z 00436130 f   rylgamelibrary:imcodeunits.obj
 0001:00035200       ?Addressing@COP_setcc@@UAEJJ@Z 00436200 f   rylgamelibrary:imcodeunits.obj
 0001:00035210       ?Show@COP_setcc@@UAEXP6AXPBDZZ@Z 00436210 f   rylgamelibrary:imcodeunits.obj
 0001:00035240       ?ToMachineCode@COP_fld@@UAEHPAE@Z 00436240 f   rylgamelibrary:imcodeunits.obj
 0001:00035280       ?Show@COP_fld@@UAEXP6AXPBDZZ@Z 00436280 f   rylgamelibrary:imcodeunits.obj
 0001:000352a0       ?ToMachineCode@COP_fadd@@UAEHPAE@Z 004362a0 f   rylgamelibrary:imcodeunits.obj
 0001:000352e0       ?Show@COP_fadd@@UAEXP6AXPBDZZ@Z 004362e0 f   rylgamelibrary:imcodeunits.obj
 0001:00035300       ?ToMachineCode@COP_fsub@@UAEHPAE@Z 00436300 f   rylgamelibrary:imcodeunits.obj
 0001:00035340       ?Show@COP_fsub@@UAEXP6AXPBDZZ@Z 00436340 f   rylgamelibrary:imcodeunits.obj
 0001:00035360       ?ToMachineCode@COP_fmul@@UAEHPAE@Z 00436360 f   rylgamelibrary:imcodeunits.obj
 0001:000353a0       ?Show@COP_fmul@@UAEXP6AXPBDZZ@Z 004363a0 f   rylgamelibrary:imcodeunits.obj
 0001:000353c0       ?ToMachineCode@COP_fdiv@@UAEHPAE@Z 004363c0 f   rylgamelibrary:imcodeunits.obj
 0001:00035400       ?Show@COP_fdiv@@UAEXP6AXPBDZZ@Z 00436400 f   rylgamelibrary:imcodeunits.obj
 0001:00035420       ?ToMachineCode@COP_fstp@@UAEHPAE@Z 00436420 f   rylgamelibrary:imcodeunits.obj
 0001:00035490       ?Show@COP_fstp@@UAEXP6AXPBDZZ@Z 00436490 f   rylgamelibrary:imcodeunits.obj
 0001:000354b0       ?ToMachineCode@COP_fcomp@@UAEHPAE@Z 004364b0 f   rylgamelibrary:imcodeunits.obj
 0001:000354f0       ?Addressing@COP_fsub@@UAEJJ@Z 004364f0 f   rylgamelibrary:imcodeunits.obj
 0001:000354f0       ?Addressing@COP_fadd@@UAEJJ@Z 004364f0 f   rylgamelibrary:imcodeunits.obj
 0001:000354f0       ?Addressing@COP_fmul@@UAEJJ@Z 004364f0 f   rylgamelibrary:imcodeunits.obj
 0001:000354f0       ?Addressing@COP_fdiv@@UAEJJ@Z 004364f0 f   rylgamelibrary:imcodeunits.obj
 0001:000354f0       ?Addressing@COP_fstp@@UAEJJ@Z 004364f0 f   rylgamelibrary:imcodeunits.obj
 0001:000354f0       ?Addressing@COP_fcomp@@UAEJJ@Z 004364f0 f   rylgamelibrary:imcodeunits.obj
 0001:000354f0       ?Addressing@COP_fld@@UAEJJ@Z 004364f0 f   rylgamelibrary:imcodeunits.obj
 0001:00035530       ?Show@COP_fcomp@@UAEXP6AXPBDZZ@Z 00436530 f   rylgamelibrary:imcodeunits.obj
 0001:00035550       ?ToMachineCode@COP_fnstsw_ax@@UAEHPAE@Z 00436550 f   rylgamelibrary:imcodeunits.obj
 0001:00035570       ?Addressing@COP_fnstsw_ax@@UAEJJ@Z 00436570 f   rylgamelibrary:imcodeunits.obj
 0001:00035580       ?Show@COP_fnstsw_ax@@UAEXP6AXPBDZZ@Z 00436580 f   rylgamelibrary:imcodeunits.obj
 0001:00035590       ?ToMachineCode@COP_test_ah@@UAEHPAE@Z 00436590 f   rylgamelibrary:imcodeunits.obj
 0001:000355b0       ?Addressing@COP_idiv@@UAEJJ@Z 004365b0 f   rylgamelibrary:imcodeunits.obj
 0001:000355b0       ?Addressing@COP_imul@@UAEJJ@Z 004365b0 f   rylgamelibrary:imcodeunits.obj
 0001:000355b0       ?Addressing@COP_test_ah@@UAEJJ@Z 004365b0 f   rylgamelibrary:imcodeunits.obj
 0001:000355c0       ?Show@COP_test_ah@@UAEXP6AXPBDZZ@Z 004365c0 f   rylgamelibrary:imcodeunits.obj
 0001:000355e0       ?ToMachineCode@COP_itoa@@UAEHPAE@Z 004365e0 f   rylgamelibrary:imcodeunits.obj
 0001:000356b0       ?Addressing@COP_itoa@@UAEJJ@Z 004366b0 f   rylgamelibrary:imcodeunits.obj
 0001:000356c0       ?Show@COP_itoa@@UAEXP6AXPBDZZ@Z 004366c0 f   rylgamelibrary:imcodeunits.obj
 0001:000356f0       ?ToMachineCode@COP_ftoa@@UAEHPAE@Z 004366f0 f   rylgamelibrary:imcodeunits.obj
 0001:00035850       ?Addressing@COP_ftoa@@UAEJJ@Z 00436850 f   rylgamelibrary:imcodeunits.obj
 0001:00035870       ?Show@COP_ftoa@@UAEXP6AXPBDZZ@Z 00436870 f   rylgamelibrary:imcodeunits.obj
 0001:000358b0       ?ToMachineCode@COP_malloc@@UAEHPAE@Z 004368b0 f   rylgamelibrary:imcodeunits.obj
 0001:00035970       ?Addressing@COP_malloc@@UAEJJ@Z 00436970 f   rylgamelibrary:imcodeunits.obj
 0001:00035980       ?Show@COP_malloc@@UAEXP6AXPBDZZ@Z 00436980 f   rylgamelibrary:imcodeunits.obj
 0001:000359a0       ?ToMachineCode@COP_free@@UAEHPAE@Z 004369a0 f   rylgamelibrary:imcodeunits.obj
 0001:00035aa0       ?Addressing@COP_free@@UAEJJ@Z 00436aa0 f   rylgamelibrary:imcodeunits.obj
 0001:00035ae0       ?Show@COP_free@@UAEXP6AXPBDZZ@Z 00436ae0 f   rylgamelibrary:imcodeunits.obj
 0001:00035b00       ?ToMachineCode@COP_strcpy@@UAEHPAE@Z 00436b00 f   rylgamelibrary:imcodeunits.obj
 0001:00035bb0       ?Addressing@COP_strcpy@@UAEJJ@Z 00436bb0 f   rylgamelibrary:imcodeunits.obj
 0001:00035c00       ?Show@COP_strcpy@@UAEXP6AXPBDZZ@Z 00436c00 f   rylgamelibrary:imcodeunits.obj
 0001:00035c60       ?ToMachineCode@COP_strcmp@@UAEHPAE@Z 00436c60 f   rylgamelibrary:imcodeunits.obj
 0001:00035cd0       ?Addressing@COP_strcmp@@UAEJJ@Z 00436cd0 f   rylgamelibrary:imcodeunits.obj
 0001:00035ce0       ?Show@COP_strcmp@@UAEXP6AXPBDZZ@Z 00436ce0 f   rylgamelibrary:imcodeunits.obj
 0001:00035d10       ?ToMachineCode@COP_strlen@@UAEHPAE@Z 00436d10 f   rylgamelibrary:imcodeunits.obj
 0001:00035db0       ?Addressing@COP_strlen@@UAEJJ@Z 00436db0 f   rylgamelibrary:imcodeunits.obj
 0001:00035e00       ?Show@COP_strlen@@UAEXP6AXPBDZZ@Z 00436e00 f   rylgamelibrary:imcodeunits.obj
 0001:00035e60       ??0COP_call@@QAE@PAU_FUNC_@@H@Z 00436e60 f   rylgamelibrary:imcodeunits.obj
 0001:00035e80       ??0COP_mov@@QAE@PAU_FUNC_@@PAU_VAR_@@W4eRegister@@@Z 00436e80 f   rylgamelibrary:imcodeunits.obj
 0001:00035eb0       ??0COP_mov@@QAE@W4eRegister@@PAU_FUNC_@@PAU_VAR_@@@Z 00436eb0 f   rylgamelibrary:imcodeunits.obj
 0001:00035ee0       ??0COP_mov@@QAE@W4eRegister@@PAU_CONST_@@@Z 00436ee0 f   rylgamelibrary:imcodeunits.obj
 0001:00035f10       ??0COP_mov@@QAE@PAU_FUNC_@@PAU_VAR_@@M@Z 00436f10 f   rylgamelibrary:imcodeunits.obj
 0001:00035f40       ??0COP_mov@@QAE@W4eRegister@@0@Z 00436f40 f   rylgamelibrary:imcodeunits.obj
 0001:00035f70       ??0COP_mov@@QAE@W4eRegister@@H@Z 00436f70 f   rylgamelibrary:imcodeunits.obj
 0001:00035fa0       ??0COP_mov@@QAE@PAU_FUNC_@@PAU_VAR_@@HW4eRegister@@@Z 00436fa0 f   rylgamelibrary:imcodeunits.obj
 0001:00035fd0       ??0COP_mov@@QAE@W4eRegister@@PAU_FUNC_@@PAU_VAR_@@0@Z 00436fd0 f   rylgamelibrary:imcodeunits.obj
 0001:00036000       ??0COP_add@@QAE@W4eRegister@@H@Z 00437000 f   rylgamelibrary:imcodeunits.obj
 0001:00036020       ??0COP_add@@QAE@W4eRegister@@0@Z 00437020 f   rylgamelibrary:imcodeunits.obj
 0001:00036040       ??0COP_sub@@QAE@W4eRegister@@H@Z 00437040 f   rylgamelibrary:imcodeunits.obj
 0001:00036060       ??0COP_sub@@QAE@W4eRegister@@0@Z 00437060 f   rylgamelibrary:imcodeunits.obj
 0001:00036080       ??0COP_imul@@QAE@W4eRegister@@0@Z 00437080 f   rylgamelibrary:imcodeunits.obj
 0001:000360a0       ??0COP_idiv@@QAE@W4eRegister@@@Z 004370a0 f   rylgamelibrary:imcodeunits.obj
 0001:000360c0       ??0COP_push@@QAE@W4eRegister@@@Z 004370c0 f   rylgamelibrary:imcodeunits.obj
 0001:000360e0       ??0COP_pop@@QAE@W4eRegister@@@Z 004370e0 f   rylgamelibrary:imcodeunits.obj
 0001:00036100       ??0COP_jmp@@QAE@XZ         00437100 f   rylgamelibrary:imcodeunits.obj
 0001:00036110       ??0COP_jmp@@QAE@PAVIOPCode@@@Z 00437110 f   rylgamelibrary:imcodeunits.obj
 0001:00036130       ??1COP_nop@@UAE@XZ         00437130 f   rylgamelibrary:imcodegen.obj
 0001:00036130       ??1IOPCode@@UAE@XZ         00437130 f   rylgamelibrary:imcodegen.obj
 0001:00036130       ??1COP_add@@UAE@XZ         00437130 f   rylgamelibrary:imcodeunits.obj
 0001:00036130       ??1COP_strlen@@UAE@XZ      00437130 f   rylgamelibrary:imcodeunits.obj
 0001:00036130       ??1COP_mov@@UAE@XZ         00437130 f   rylgamelibrary:imcodeunits.obj
 0001:00036130       ??1COP_ftoa@@UAE@XZ        00437130 f   rylgamelibrary:imcodeunits.obj
 0001:00036130       ??1COP_fdiv@@UAE@XZ        00437130 f   rylgamelibrary:imcodeunits.obj
 0001:00036130       ??1COP_call@@UAE@XZ        00437130 f   rylgamelibrary:imcodeunits.obj
 0001:00036130       ??1COP_fld@@UAE@XZ         00437130 f   rylgamelibrary:imcodeunits.obj
 0001:00036130       ??1COP_imul@@UAE@XZ        00437130 f   rylgamelibrary:imcodeunits.obj
 0001:00036130       ??1COP_jcc@@UAE@XZ         00437130 f   rylgamelibrary:imcodeunits.obj
 0001:00036130       ??1COP_free@@UAE@XZ        00437130 f   rylgamelibrary:imcodeunits.obj
 0001:00036130       ??1COP_cmp@@UAE@XZ         00437130 f   rylgamelibrary:imcodeunits.obj
 0001:00036130       ??1COP_fstp@@UAE@XZ        00437130 f   rylgamelibrary:imcodeunits.obj
 0001:00036130       ??1COP_strcpy@@UAE@XZ      00437130 f   rylgamelibrary:imcodeunits.obj
 0001:00036130       ??1COP_idiv@@UAE@XZ        00437130 f   rylgamelibrary:imcodeunits.obj
 0001:00036130       ??1COP_setcc@@UAE@XZ       00437130 f   rylgamelibrary:imcodeunits.obj
 0001:00036130       ??1COP_malloc@@UAE@XZ      00437130 f   rylgamelibrary:imcodeunits.obj
 0001:00036130       ??1COP_jmpmark@@UAE@XZ     00437130 f   rylgamelibrary:imcodeunits.obj
 0001:00036130       ??1COP_jmp@@UAE@XZ         00437130 f   rylgamelibrary:imcodeunits.obj
 0001:00036130       ??1COP_test_ah@@UAE@XZ     00437130 f   rylgamelibrary:imcodeunits.obj
 0001:00036130       ??1COP_fsub@@UAE@XZ        00437130 f   rylgamelibrary:imcodeunits.obj
 0001:00036130       ??1COP_itoa@@UAE@XZ        00437130 f   rylgamelibrary:imcodeunits.obj
 0001:00036130       ??1COP_sub@@UAE@XZ         00437130 f   rylgamelibrary:imcodeunits.obj
 0001:00036130       ??1COP_pop@@UAE@XZ         00437130 f   rylgamelibrary:imcodeunits.obj
 0001:00036130       ??1COP_fadd@@UAE@XZ        00437130 f   rylgamelibrary:imcodeunits.obj
 0001:00036130       ??1COP_ret@@UAE@XZ         00437130 f   rylgamelibrary:imcodegen.obj
 0001:00036130       ??1COP_fmul@@UAE@XZ        00437130 f   rylgamelibrary:imcodeunits.obj
 0001:00036130       ??1COP_fcomp@@UAE@XZ       00437130 f   rylgamelibrary:imcodeunits.obj
 0001:00036130       ??1COP_fnstsw_ax@@UAE@XZ   00437130 f   rylgamelibrary:imcodegen.obj
 0001:00036130       ??1COP_push@@UAE@XZ        00437130 f   rylgamelibrary:imcodeunits.obj
 0001:00036130       ??1COP_strcmp@@UAE@XZ      00437130 f   rylgamelibrary:imcodeunits.obj
 0001:00036140       ??0COP_jcc@@QAE@W4eCondition@@@Z 00437140 f   rylgamelibrary:imcodeunits.obj
 0001:00036160       ??0COP_jmpmark@@QAE@XZ     00437160 f   rylgamelibrary:imcodeunits.obj
 0001:00036170       ??0COP_jmpmark@@QAE@PAVCOP_jmp@@@Z 00437170 f   rylgamelibrary:imcodeunits.obj
 0001:00036190       ??0COP_cmp@@QAE@PAU_FUNC_@@PAU_VAR_@@PAU_CONST_@@@Z 00437190 f   rylgamelibrary:imcodeunits.obj
 0001:000361c0       ??0COP_cmp@@QAE@W4eRegister@@E@Z 004371c0 f   rylgamelibrary:imcodeunits.obj
 0001:000361f0       ??0COP_cmp@@QAE@W4eRegister@@0@Z 004371f0 f   rylgamelibrary:imcodeunits.obj
 0001:00036220       ??0COP_setcc@@QAE@W4eCondition@@W4eRegister@@@Z 00437220 f   rylgamelibrary:imcodeunits.obj
 0001:00036280       ??0COP_fld@@QAE@PAU_FUNC_@@PAU_VAR_@@@Z 00437280 f   rylgamelibrary:imcodeunits.obj
 0001:000362a0       ??0COP_fadd@@QAE@PAU_FUNC_@@PAU_VAR_@@@Z 004372a0 f   rylgamelibrary:imcodeunits.obj
 0001:000362c0       ??0COP_fsub@@QAE@PAU_FUNC_@@PAU_VAR_@@@Z 004372c0 f   rylgamelibrary:imcodeunits.obj
 0001:000362e0       ??0COP_fmul@@QAE@PAU_FUNC_@@PAU_VAR_@@@Z 004372e0 f   rylgamelibrary:imcodeunits.obj
 0001:00036300       ??0COP_fdiv@@QAE@PAU_FUNC_@@PAU_VAR_@@@Z 00437300 f   rylgamelibrary:imcodeunits.obj
 0001:00036320       ??0COP_fstp@@QAE@PAU_FUNC_@@PAU_VAR_@@_N@Z 00437320 f   rylgamelibrary:imcodeunits.obj
 0001:00036340       ??0COP_fcomp@@QAE@PAU_FUNC_@@PAU_VAR_@@@Z 00437340 f   rylgamelibrary:imcodeunits.obj
 0001:00036360       ??0COP_test_ah@@QAE@E@Z    00437360 f   rylgamelibrary:imcodeunits.obj
 0001:00036380       ??0COP_itoa@@QAE@W4eRegister@@PAU_VAR_@@@Z 00437380 f   rylgamelibrary:imcodeunits.obj
 0001:000363a0       ??0COP_ftoa@@QAE@W4eRegister@@PAU_VAR_@@1@Z 004373a0 f   rylgamelibrary:imcodeunits.obj
 0001:000363c0       ??0COP_malloc@@QAE@W4eRegister@@@Z 004373c0 f   rylgamelibrary:imcodeunits.obj
 0001:000363e0       ??0COP_free@@QAE@PAU_FUNC_@@PAU_VAR_@@@Z 004373e0 f   rylgamelibrary:imcodeunits.obj
 0001:00036400       ??0COP_strcpy@@QAE@W4eRegister@@0@Z 00437400 f   rylgamelibrary:imcodeunits.obj
 0001:00036420       ??0COP_strcpy@@QAE@W4eRegister@@PAU_FUNC_@@PAU_VAR_@@@Z 00437420 f   rylgamelibrary:imcodeunits.obj
 0001:00036450       ??0COP_strcmp@@QAE@W4eRegister@@0@Z 00437450 f   rylgamelibrary:imcodeunits.obj
 0001:00036470       ??0COP_strlen@@QAE@W4eRegister@@@Z 00437470 f   rylgamelibrary:imcodeunits.obj
 0001:00036490       ??0COP_strlen@@QAE@PAU_FUNC_@@PAU_VAR_@@@Z 00437490 f   rylgamelibrary:imcodeunits.obj
 0001:000364b0       ??_ECOP_fmul@@UAEPAXI@Z    004374b0 f i rylgamelibrary:imcodeunits.obj
 0001:000364b0       ??_ECOP_strcpy@@UAEPAXI@Z  004374b0 f i rylgamelibrary:imcodeunits.obj
 0001:000364b0       ??_GCOP_setcc@@UAEPAXI@Z   004374b0 f i rylgamelibrary:imcodeunits.obj
 0001:000364b0       ??_GCOP_pop@@UAEPAXI@Z     004374b0 f i rylgamelibrary:imcodeunits.obj
 0001:000364b0       ??_GCOP_jmp@@UAEPAXI@Z     004374b0 f i rylgamelibrary:imcodeunits.obj
 0001:000364b0       ??_GCOP_fdiv@@UAEPAXI@Z    004374b0 f i rylgamelibrary:imcodeunits.obj
 0001:000364b0       ??_ECOP_call@@UAEPAXI@Z    004374b0 f i rylgamelibrary:imcodeunits.obj
 0001:000364b0       ??_ECOP_fstp@@UAEPAXI@Z    004374b0 f i rylgamelibrary:imcodeunits.obj
 0001:000364b0       ??_GCOP_ftoa@@UAEPAXI@Z    004374b0 f i rylgamelibrary:imcodeunits.obj
 0001:000364b0       ??_ECOP_malloc@@UAEPAXI@Z  004374b0 f i rylgamelibrary:imcodeunits.obj
 0001:000364b0       ??_GCOP_push@@UAEPAXI@Z    004374b0 f i rylgamelibrary:imcodeunits.obj
 0001:000364b0       ??_GCOP_itoa@@UAEPAXI@Z    004374b0 f i rylgamelibrary:imcodeunits.obj
 0001:000364b0       ??_GCOP_jmpmark@@UAEPAXI@Z 004374b0 f i rylgamelibrary:imcodeunits.obj
 0001:000364b0       ??_GCOP_strcpy@@UAEPAXI@Z  004374b0 f i rylgamelibrary:imcodeunits.obj
 0001:000364b0       ??_ECOP_add@@UAEPAXI@Z     004374b0 f i rylgamelibrary:imcodeunits.obj
 0001:000364b0       ??_GCOP_cmp@@UAEPAXI@Z     004374b0 f i rylgamelibrary:imcodeunits.obj
 0001:000364b0       ??_ECOP_fdiv@@UAEPAXI@Z    004374b0 f i rylgamelibrary:imcodeunits.obj
 0001:000364b0       ??_GCOP_sub@@UAEPAXI@Z     004374b0 f i rylgamelibrary:imcodeunits.obj
 0001:000364b0       ??_GCOP_fld@@UAEPAXI@Z     004374b0 f i rylgamelibrary:imcodeunits.obj
 0001:000364b0       ??_ECOP_nop@@UAEPAXI@Z     004374b0 f i rylgamelibrary:imcodegen.obj
 0001:000364b0       ??_ECOP_ret@@UAEPAXI@Z     004374b0 f i rylgamelibrary:imcodegen.obj
 0001:000364b0       ??_GCOP_strlen@@UAEPAXI@Z  004374b0 f i rylgamelibrary:imcodeunits.obj
 0001:000364b0       ??_GCOP_test_ah@@UAEPAXI@Z 004374b0 f i rylgamelibrary:imcodeunits.obj
 0001:000364b0       ??_GCOP_fsub@@UAEPAXI@Z    004374b0 f i rylgamelibrary:imcodeunits.obj
 0001:000364b0       ??_ECOP_fld@@UAEPAXI@Z     004374b0 f i rylgamelibrary:imcodeunits.obj
 0001:000364b0       ??_ECOP_push@@UAEPAXI@Z    004374b0 f i rylgamelibrary:imcodeunits.obj
 0001:000364b0       ??_GCOP_fcomp@@UAEPAXI@Z   004374b0 f i rylgamelibrary:imcodeunits.obj
 0001:000364b0       ??_ECOP_jmp@@UAEPAXI@Z     004374b0 f i rylgamelibrary:imcodeunits.obj
 0001:000364b0       ??_ECOP_strcmp@@UAEPAXI@Z  004374b0 f i rylgamelibrary:imcodeunits.obj
 0001:000364b0       ??_GCOP_call@@UAEPAXI@Z    004374b0 f i rylgamelibrary:imcodeunits.obj
 0001:000364b0       ??_GCOP_malloc@@UAEPAXI@Z  004374b0 f i rylgamelibrary:imcodeunits.obj
 0001:000364b0       ??_GCOP_nop@@UAEPAXI@Z     004374b0 f i rylgamelibrary:imcodegen.obj
 0001:000364b0       ??_ECOP_itoa@@UAEPAXI@Z    004374b0 f i rylgamelibrary:imcodeunits.obj
 0001:000364b0       ??_ECOP_jmpmark@@UAEPAXI@Z 004374b0 f i rylgamelibrary:imcodeunits.obj
 0001:000364b0       ??_GCOP_fnstsw_ax@@UAEPAXI@Z 004374b0 f i rylgamelibrary:imcodegen.obj
 0001:000364b0       ??_ECOP_strlen@@UAEPAXI@Z  004374b0 f i rylgamelibrary:imcodeunits.obj
 0001:000364b0       ??_ECOP_pop@@UAEPAXI@Z     004374b0 f i rylgamelibrary:imcodeunits.obj
 0001:000364b0       ??_GCOP_ret@@UAEPAXI@Z     004374b0 f i rylgamelibrary:imcodegen.obj
 0001:000364b0       ??_ECOP_fnstsw_ax@@UAEPAXI@Z 004374b0 f i rylgamelibrary:imcodegen.obj
 0001:000364b0       ??_GCOP_imul@@UAEPAXI@Z    004374b0 f i rylgamelibrary:imcodeunits.obj
 0001:000364b0       ??_GCOP_add@@UAEPAXI@Z     004374b0 f i rylgamelibrary:imcodeunits.obj
 0001:000364b0       ??_ECOP_sub@@UAEPAXI@Z     004374b0 f i rylgamelibrary:imcodeunits.obj
 0001:000364b0       ??_GCOP_free@@UAEPAXI@Z    004374b0 f i rylgamelibrary:imcodeunits.obj
 0001:000364b0       ??_GCOP_fmul@@UAEPAXI@Z    004374b0 f i rylgamelibrary:imcodeunits.obj
 0001:000364b0       ??_ECOP_mov@@UAEPAXI@Z     004374b0 f i rylgamelibrary:imcodeunits.obj
 0001:000364b0       ??_ECOP_idiv@@UAEPAXI@Z    004374b0 f i rylgamelibrary:imcodeunits.obj
 0001:000364b0       ??_ECOP_jcc@@UAEPAXI@Z     004374b0 f i rylgamelibrary:imcodeunits.obj
 0001:000364b0       ??_GCOP_jcc@@UAEPAXI@Z     004374b0 f i rylgamelibrary:imcodeunits.obj
 0001:000364b0       ??_ECOP_free@@UAEPAXI@Z    004374b0 f i rylgamelibrary:imcodeunits.obj
 0001:000364b0       ??_GCOP_idiv@@UAEPAXI@Z    004374b0 f i rylgamelibrary:imcodeunits.obj
 0001:000364b0       ??_ECOP_setcc@@UAEPAXI@Z   004374b0 f i rylgamelibrary:imcodeunits.obj
 0001:000364b0       ??_ECOP_imul@@UAEPAXI@Z    004374b0 f i rylgamelibrary:imcodeunits.obj
 0001:000364b0       ??_GCOP_fadd@@UAEPAXI@Z    004374b0 f i rylgamelibrary:imcodeunits.obj
 0001:000364b0       ??_ECOP_test_ah@@UAEPAXI@Z 004374b0 f i rylgamelibrary:imcodeunits.obj
 0001:000364b0       ??_GCOP_mov@@UAEPAXI@Z     004374b0 f i rylgamelibrary:imcodeunits.obj
 0001:000364b0       ??_ECOP_fcomp@@UAEPAXI@Z   004374b0 f i rylgamelibrary:imcodeunits.obj
 0001:000364b0       ??_ECOP_fsub@@UAEPAXI@Z    004374b0 f i rylgamelibrary:imcodeunits.obj
 0001:000364b0       ??_ECOP_ftoa@@UAEPAXI@Z    004374b0 f i rylgamelibrary:imcodeunits.obj
 0001:000364b0       ??_GCOP_fstp@@UAEPAXI@Z    004374b0 f i rylgamelibrary:imcodeunits.obj
 0001:000364b0       ??_GCOP_strcmp@@UAEPAXI@Z  004374b0 f i rylgamelibrary:imcodeunits.obj
 0001:000364b0       ??_ECOP_fadd@@UAEPAXI@Z    004374b0 f i rylgamelibrary:imcodeunits.obj
 0001:000364b0       ??_ECOP_cmp@@UAEPAXI@Z     004374b0 f i rylgamelibrary:imcodeunits.obj
 0001:000364d0       ?find@?$_Tree@V?$_Tmap_traits@HJU?$less@H@std@@V?$allocator@U?$pair@$$CBHJ@std@@@2@$0A@@std@@@std@@QAE?AViterator@12@ABH@Z 004374d0 f i rylgamelibrary:imcodeunits.obj
 0001:00036540       ?ToMachineCode@COP_call@@UAEHPAE@Z 00437540 f   rylgamelibrary:imcodeunits.obj
 0001:000365c2       ??2@YAPAXI@Z               004375c2 f   libcpmt:newop.obj
 0001:000365e6       ?_Xran@_String_base@std@@QBEXXZ 004375e6 f   libcpmt:string.obj
 0001:00036626       ?_Xlen@_String_base@std@@QBEXXZ 00437626 f   libcpmt:string.obj
 0001:00036666       ?_Callfns@ios_base@std@@AAEXW4event@12@@Z 00437666 f   libcpmt:ios.obj
 0001:00036688       ?_Addstd@ios_base@std@@QAEXXZ 00437688 f   libcpmt:ios.obj
 0001:000366d9       ?_Tidy@ios_base@std@@AAEXXZ 004376d9 f   libcpmt:ios.obj
 0001:0003671b       ??1ios_base@std@@UAE@XZ    0043771b f   libcpmt:ios.obj
 0001:0003675b       ??1runtime_error@std@@UAE@XZ 0043775b f i libcpmt:ios.obj
 0001:00036778       ?what@runtime_error@std@@UBEPBDXZ 00437778 f i libcpmt:ios.obj
 0001:00036786       ??_Eruntime_error@std@@UAEPAXI@Z 00437786 f i libcpmt:ios.obj
 0001:00036786       ??_Gruntime_error@std@@UAEPAXI@Z 00437786 f i libcpmt:ios.obj
 0001:000367a2       ??0runtime_error@std@@QAE@ABV?$basic_string@DU?$char_traits@D@std@@V?$allocator@D@2@@1@@Z 004377a2 f i libcpmt:ios.obj
 0001:000367de       ??_Gfailure@ios_base@std@@UAEPAXI@Z 004377de f i libcpmt:ios.obj
 0001:000367de       ??_Efailure@ios_base@std@@UAEPAXI@Z 004377de f i libcpmt:ios.obj
 0001:000367fa       ??1failure@ios_base@std@@UAE@XZ 004377fa f i libcpmt:ios.obj
 0001:00036805       ?clear@ios_base@std@@QAEXH_N@Z 00437805 f   libcpmt:ios.obj
 0001:000368cb       ??0runtime_error@std@@QAE@ABV01@@Z 004378cb f i libcpmt:ios.obj
 0001:0003690e       ??0failure@ios_base@std@@QAE@ABV012@@Z 0043790e f i libcpmt:ios.obj
 0001:00036926       ?_Init@ios_base@std@@IAEXXZ 00437926 f   libcpmt:ios.obj
 0001:0003696c       ??0_Mutex@std@@QAE@XZ      0043796c f   libcpmt:xmutex.obj
 0001:00036984       ??1_Mutex@std@@QAE@XZ      00437984 f   libcpmt:xmutex.obj
 0001:00036999       ?_Lock@_Mutex@std@@QAEXXZ  00437999 f   libcpmt:xmutex.obj
 0001:000369a2       ?_Unlock@_Mutex@std@@QAEXXZ 004379a2 f   libcpmt:xmutex.obj
 0001:000369ab       ?uncaught_exception@std@@YA_NXZ 004379ab f   libcpmt:uncaught.obj
 0001:000369b0       ??_U@YAPAXI@Z              004379b0 f   libcpmt:newaop.obj
 0001:000369b5       __Tolower_lk               004379b5 f   libcpmt:_tolower.obj
 0001:00036a9e       __Getctype                 00437a9e f   libcpmt:_tolower.obj
 0001:00036b69       __Tolower                  00437b69 f   libcpmt:_tolower.obj
 0001:00036c15       ??0_Init_locks@std@@QAE@XZ 00437c15 f   libcpmt:xlock.obj
 0001:00036c44       ??1_Init_locks@std@@QAE@XZ 00437c44 f   libcpmt:xlock.obj
 0001:00036c6d       ??0_Lockit@std@@QAE@H@Z    00437c6d f   libcpmt:xlock.obj
 0001:00036c90       ??1_Lockit@std@@QAE@XZ     00437c90 f   libcpmt:xlock.obj
 0001:00036ca4       ??1_Fac_node@std@@QAE@XZ   00437ca4 f i libcpmt:locale0.obj
 0001:00036cb9       __Deletegloballocale       00437cb9 f   libcpmt:locale0.obj
 0001:00036cf8       __Setgloballocale          00437cf8 f   libcpmt:locale0.obj
 0001:00036d1d       ?_Getfacet@locale@std@@QBEPBVfacet@12@I@Z 00437d1d f   libcpmt:locale0.obj
 0001:00036d52       __Fac_tidy                 00437d52 f   libcpmt:locale0.obj
 0001:00036d95       ?_Register@facet@locale@std@@QAEXXZ 00437d95 f   libcpmt:locale0.obj
 0001:00036dce       ??1_Locimp@locale@std@@MAE@XZ 00437dce f   libcpmt:locale0.obj
 0001:00036e56       ??1_Locinfo@std@@QAE@XZ    00437e56 f   libcpmt:locale0.obj
 0001:00036ead       ??_E_Locimp@locale@std@@MAEPAXI@Z 00437ead f i libcpmt:locale0.obj
 0001:00036ead       ??_G_Locimp@locale@std@@MAEPAXI@Z 00437ead f i libcpmt:locale0.obj
 0001:00036ec9       ??0_Locimp@locale@std@@AAE@_N@Z 00437ec9 f   libcpmt:locale0.obj
 0001:00036f19       ??0_Locinfo@std@@QAE@PBD@Z 00437f19 f   libcpmt:locale0.obj
 0001:00036fa3       ?_Init@locale@std@@CAPAV_Locimp@12@XZ 00437fa3 f   libcpmt:locale0.obj
 0001:00037045       ??0locale@std@@QAE@XZ      00438045 f   libcpmt:locale0.obj
 0001:0003705e       __Toupper_lk               0043805e f   libcpmt:_toupper.obj
 0001:0003713e       __Toupper                  0043813e f   libcpmt:_toupper.obj
 0001:000371ea       ??0_Init_cout@std@@QAE@XZ  004381ea f i libcpmt:cout.obj
 0001:0003723f       ?_Nomemory@std@@YAXXZ      0043823f f   libcpmt:nomemory.obj
 0001:000372a0       __Mtxinit                  004382a0 f   libcpmt:xmtx.obj
 0001:000372ab       __Mtxdst                   004382ab f   libcpmt:xmtx.obj
 0001:000372b6       __Mtxlock                  004382b6 f   libcpmt:xmtx.obj
 0001:000372c1       __Mtxunlock                004382c1 f   libcpmt:xmtx.obj
 0001:000372cc       __Atexit                   004382cc f   libcpmt:iosptrs.obj
 0001:000372ec       ??1_Init_atexit@@QAE@XZ    004382ec f i libcpmt:iosptrs.obj
 0001:0003730c       ?_JumpToContinuation@@YGXPAXPAUEHRegistrationNode@@@Z 0043830c f   LIBCMT:trnsctrl.obj
 0001:0003733c       ?_CallMemberFunction0@@YGXPAX0@Z 0043833c f   LIBCMT:trnsctrl.obj
 0001:0003733c       ?_CallMemberFunction1@@YGXPAX00@Z 0043833c f   LIBCMT:trnsctrl.obj
 0001:0003733c       ?_CallMemberFunction2@@YGXPAX00H@Z 0043833c f   LIBCMT:trnsctrl.obj
 0001:00037343       ?_UnwindNestedFrames@@YGXPAUEHRegistrationNode@@PAUEHExceptionRecord@@@Z 00438343 f   LIBCMT:trnsctrl.obj
 0001:00037395       ___CxxFrameHandler         00438395 f   LIBCMT:trnsctrl.obj
 0001:00037406       ?_CallSETranslator@@YAHPAUEHExceptionRecord@@PAUEHRegistrationNode@@PAX2PBU_s_FuncInfo@@H1@Z 00438406 f   LIBCMT:trnsctrl.obj
 0001:0003757f       ?_GetRangeOfTrysToCheck@@YAPBU_s_TryBlockMapEntry@@PBU_s_FuncInfo@@HHPAI1@Z 0043857f f   LIBCMT:trnsctrl.obj
 0001:000375f9       ?_CreateFrameInfo@@YAPAUFrameInfo@@PAU1@PAX@Z 004385f9 f   LIBCMT:trnsctrl.obj
 0001:00037621       ?IsExceptionObjectToBeDestroyed@@YAHPAX@Z 00438621 f   LIBCMT:trnsctrl.obj
 0001:00037642       ?_FindAndUnlinkFrame@@YAXPAUFrameInfo@@@Z 00438642 f   LIBCMT:trnsctrl.obj
 0001:0003768e       ?_CallCatchBlock2@@YAPAXPAUEHRegistrationNode@@PBU_s_FuncInfo@@PAXHK@Z 0043868e f   LIBCMT:trnsctrl.obj
 0001:000376e8       __global_unwind2           004386e8 f   LIBCMT:exsup.obj
 0001:0003772a       __local_unwind2            0043872a f   LIBCMT:exsup.obj
 0001:00037782       __NLG_Return2              00438782     LIBCMT:exsup.obj
 0001:00037792       __abnormal_termination     00438792 f   LIBCMT:exsup.obj
 0001:000377b5       __NLG_Notify1              004387b5 f   LIBCMT:exsup.obj
 0001:000377be       __NLG_Notify               004387be f   LIBCMT:exsup.obj
 0001:000377d1       __NLG_Dispatch             004387d1     LIBCMT:exsup.obj
 0001:00037807       @__security_check_cookie@4 00438807 f   LIBCMT:secchk.obj
 0001:00037820       _strncpy                   00438820 f   LIBCMT:strncpy.obj
 0001:00037944       ??3@YAXPAX@Z               00438944 f   LIBCMT:delete.obj
 0001:000379c9       ___onexitinit              004389c9 f   LIBCMT:onexit.obj
 0001:000379f1       __onexit                   004389f1 f   LIBCMT:onexit.obj
 0001:00037a29       _atexit                    00438a29 f   LIBCMT:onexit.obj
 0001:00037a40       _memmove                   00438a40 f   LIBCMT:memmove.obj
 0001:00037d7d       __snprintf                 00438d7d f   LIBCMT:snprintf.obj
 0001:00037de0       _strncmp                   00438de0 f   LIBCMT:strncmp.obj
 0001:00037e19       __purecall                 00438e19 f   LIBCMT:purevirt.obj
 0001:00037e40       _strchr                    00438e40 f   LIBCMT:strchr.obj
 0001:00037e46       ___from_strstr_to_strchr   00438e46     LIBCMT:strchr.obj
 0001:00037efe       _atol                      00438efe f   LIBCMT:atox.obj
 0001:00037f86       _atoi                      00438f86 f   LIBCMT:atox.obj
 0001:00037f8b       __CxxThrowException@8      00438f8b f   LIBCMT:throw.obj
 0001:00037fc5       ??0exception@@QAE@XZ       00438fc5 f   LIBCMT:stdexcpt.obj
 0001:00037fd6       ??0exception@@QAE@ABQBD@Z  00438fd6 f   LIBCMT:stdexcpt.obj
 0001:00038013       ??0exception@@QAE@ABV0@@Z  00439013 f   LIBCMT:stdexcpt.obj
 0001:0003805d       ??1exception@@UAE@XZ       0043905d f   LIBCMT:stdexcpt.obj
 0001:00038073       ?what@exception@@UBEPBDXZ  00439073 f   LIBCMT:stdexcpt.obj
 0001:00038080       ??0bad_cast@@QAE@PBD@Z     00439080 f   LIBCMT:stdexcpt.obj
 0001:00038099       ??0bad_cast@@QAE@ABV0@@Z   00439099 f   LIBCMT:stdexcpt.obj
 0001:000380b1       ??1bad_cast@@UAE@XZ        004390b1 f   LIBCMT:stdexcpt.obj
 0001:000380bc       ??_Eexception@@UAEPAXI@Z   004390bc f i LIBCMT:stdexcpt.obj
 0001:000380bc       ??_Gexception@@UAEPAXI@Z   004390bc f i LIBCMT:stdexcpt.obj
 0001:000380d8       ??_Gbad_cast@@UAEPAXI@Z    004390d8 f i LIBCMT:stdexcpt.obj
 0001:000380d8       ??_Ebad_cast@@UAEPAXI@Z    004390d8 f i LIBCMT:stdexcpt.obj
 0001:000380f4       ??1type_info@@UAE@XZ       004390f4 f   LIBCMT:typinfo.obj
 0001:0003813a       ??_Gtype_info@@UAEPAXI@Z   0043913a f i LIBCMT:typinfo.obj
 0001:0003813a       ??_Etype_info@@UAEPAXI@Z   0043913a f i LIBCMT:typinfo.obj
 0001:00038156       __fclose_lk                00439156 f   LIBCMT:fclose.obj
 0001:000381a2       _fclose                    004391a2 f   LIBCMT:fclose.obj
 0001:000381f3       _strtok                    004391f3 f   LIBCMT:strtok.obj
 0001:000382a8       _fgets                     004392a8 f   LIBCMT:fgets.obj
 0001:0003832e       __fsopen                   0043932e f   LIBCMT:fopen.obj
 0001:0003838a       _fopen                     0043938a f   LIBCMT:fopen.obj
 0001:000383a0       __alloca_probe             004393a0     LIBCMT:chkstk.obj
 0001:000383a0       __chkstk                   004393a0 f   LIBCMT:chkstk.obj
 0001:000383dd       ??_V@YAXPAX@Z              004393dd f   LIBCMT:delete2.obj
 0001:000383e2       _time                      004393e2 f   LIBCMT:time.obj
 0001:0003841b       ??_U@YAPAXIABUnothrow_t@std@@@Z 0043941b f   LIBCMT:newaopnt.obj
 0001:00038420       ??3@YAXPAXABUnothrow_t@std@@@Z 00439420 f   LIBCMT:delopnt.obj
 0001:0003842b       ??2@YAPAXIABUnothrow_t@std@@@Z 0043942b f   LIBCMT:newopnt.obj
 0001:00038469       __amsg_exit                00439469 f   LIBCMT:wincrt0.obj
 0001:000384b2       _WinMainCRTStartup         004394b2 f   LIBCMT:wincrt0.obj
 0001:00038687       __fwrite_lk                00439687 f   LIBCMT:fwrite.obj
 0001:0003878e       _fwrite                    0043978e f   LIBCMT:fwrite.obj
 0001:000387da       _fprintf                   004397da f   LIBCMT:fprintf.obj
 0001:00038840       __except_handler3          00439840 f   LIBCMT:exsup3.obj
 0001:00038926       __seh_longjmp_unwind@4     00439926 f   LIBCMT:exsup3.obj
 0001:00038941       __vsnprintf                00439941 f   LIBCMT:vsnprint.obj
 0001:00038997       __mbsnbcmp                 00439997 f   LIBCMT:mbsnbcmp.obj
 0001:00038a6c       ?__ArrayUnwind@@YGXPAXIHP6EX0@Z@Z 00439a6c f   LIBCMT:ehvecdtr.obj
 0001:00038aca       ??_M@YGXPAXIHP6EX0@Z@Z     00439aca f   LIBCMT:ehvecdtr.obj
 0001:00038b2a       ??_L@YGXPAXIHP6EX0@Z1@Z    00439b2a f   LIBCMT:ehvecctr.obj
 0001:00038b8c       __fpclear                  00439b8c f   LIBCMT:fpinit.obj
 0001:00038b8d       __cfltcvt_init             00439b8d f   LIBCMT:fpinit.obj
 0001:00038bc5       __fpmath                   00439bc5 f   LIBCMT:fpinit.obj
 0001:00038be3       __heap_alloc               00439be3 f   LIBCMT:malloc.obj
 0001:00038c5e       __nh_malloc                00439c5e f   LIBCMT:malloc.obj
 0001:00038c8a       _malloc                    00439c8a f   LIBCMT:malloc.obj
 0001:00038c9c       _free                      00439c9c f   LIBCMT:free.obj
 0001:00038d0d       __resetstkoflw             00439d0d f   LIBCMT:resetstk.obj
 0001:00038df0       __ftol2                    00439df0 f   LIBCMT:ftol2.obj
 0001:00038e65       _difftime                  00439e65 f   LIBCMT:difftime.obj
 0001:00038e80       _strstr                    00439e80 f   LIBCMT:strstr.obj
 0001:00038f06       __strlwr                   00439f06 f   LIBCMT:strlwr.obj
 0001:00038f06       _strlwr                    00439f06 f   LIBCMT:strlwr.obj
 0001:0003901a       _sprintf                   0043a01a f   LIBCMT:sprintf.obj
 0001:00039072       __endthreadex              0043a072 f   LIBCMT:threadex.obj
 0001:00039138       __beginthreadex            0043a138 f   LIBCMT:threadex.obj
 0001:000391c3       __splitpath                0043a1c3 f   LIBCMT:splitpat.obj
 0001:0003930b       ___iob_func                0043a30b f   LIBCMT:_file.obj
 0001:00039311       ___initstdio               0043a311 f   LIBCMT:_file.obj
 0001:000393ba       ___endstdio                0043a3ba f   LIBCMT:_file.obj
 0001:000393ce       __lock_file                0043a3ce f   LIBCMT:_file.obj
 0001:000393fd       __lock_file2               0043a3fd f   LIBCMT:_file.obj
 0001:00039420       __unlock_file              0043a420 f   LIBCMT:_file.obj
 0001:0003944f       __unlock_file2             0043a44f f   LIBCMT:_file.obj
 0001:00039472       _localtime                 0043a472 f   LIBCMT:localtim.obj
 0001:000395f2       __mbsnbcpy                 0043a5f2 f   LIBCMT:mbsnbcpy.obj
 0001:00039685       __mbsrchr                  0043a685 f   LIBCMT:mbsrchr.obj
 0001:0003972e       _itoa                      0043a72e f   LIBCMT:xtoa.obj
 0001:0003972e       __itoa                     0043a72e f   LIBCMT:xtoa.obj
 0001:000397c5       __ui64toa                  0043a7c5 f   LIBCMT:xtoa.obj
 0001:000397e0       _isupper                   0043a7e0 f   LIBCMT:_ctype.obj
 0001:0003981a       _islower                   0043a81a f   LIBCMT:_ctype.obj
 0001:00039854       _isdigit                   0043a854 f   LIBCMT:_ctype.obj
 0001:0003988e       _isspace                   0043a88e f   LIBCMT:_ctype.obj
 0001:000398c8       _isprint                   0043a8c8 f   LIBCMT:_ctype.obj
 0001:00039907       __flush                    0043a907 f   LIBCMT:fflush.obj
 0001:00039964       __fflush_lk                0043a964 f   LIBCMT:fflush.obj
 0001:00039a67       _fflush                    0043aa67 f   LIBCMT:fflush.obj
 0001:00039ab7       __flushall                 0043aab7 f   LIBCMT:fflush.obj
 0001:00039ac0       _fputs                     0043aac0 f   LIBCMT:fputs.obj
 0001:00039b31       _srand                     0043ab31 f   LIBCMT:rand.obj
 0001:00039b3e       _rand                      0043ab3e f   LIBCMT:rand.obj
 0001:00039b60       _memchr                    0043ab60 f   LIBCMT:memchr.obj
 0001:00039c0d       _setvbuf                   0043ac0d f   LIBCMT:setvbuf.obj
 0001:00039ce9       __ungetc_lk                0043ace9 f   LIBCMT:ungetc.obj
 0001:00039d55       _ungetc                    0043ad55 f   LIBCMT:ungetc.obj
 0001:00039d9a       _fputc                     0043ad9a f   LIBCMT:fputc.obj
 0001:00039df2       _fgetc                     0043adf2 f   LIBCMT:fgetc.obj
 0001:00039e42       _fgetpos                   0043ae42 f   LIBCMT:fgetpos.obj
 0001:00039e64       __fseek_lk                 0043ae64 f   LIBCMT:fseek.obj
 0001:00039ef3       _fseek                     0043aef3 f   LIBCMT:fseek.obj
 0001:00039f3c       _fsetpos                   0043af3c f   LIBCMT:fsetpos.obj
 0001:00039f54       _wcslen                    0043af54 f   LIBCMT:wcslen.obj
 0001:00039f6a       _atof                      0043af6a f   LIBCMT:atof.obj
 0001:00039fa2       __fread_lk                 0043afa2 f   LIBCMT:fread.obj
 0001:0003a08b       _fread                     0043b08b f   LIBCMT:fread.obj
 0001:0003a0d7       __errno                    0043b0d7 f   LIBCMT:dosmap.obj
 0001:0003a0e0       ___doserrno                0043b0e0 f   LIBCMT:dosmap.obj
 0001:0003a0e9       __dosmaperr                0043b0e9 f   LIBCMT:dosmap.obj
 0001:0003a15c       _vsprintf                  0043b15c f   LIBCMT:vsprintf.obj
 0001:0003a1b3       __ftell_lk                 0043b1b3 f   LIBCMT:ftell.obj
 0001:0003a315       _ftell                     0043b315 f   LIBCMT:ftell.obj
 0001:0003a356       __fdopen                   0043b356 f   LIBCMT:fdopen.obj
 0001:0003a460       __alldiv                   0043b460 f   LIBCMT:lldiv.obj
 0001:0003a50a       _calloc                    0043b50a f   LIBCMT:calloc.obj
 0001:0003a5d0       __allmul                   0043b5d0 f   LIBCMT:llmul.obj
 0001:0003a610       _strcspn                   0043b610 f   LIBCMT:strcspn.obj
 0001:0003a660       _strncat                   0043b660 f   LIBCMT:strncat.obj
 0001:0003a795       ___crtExitProcess          0043b795 f   LIBCMT:crt0dat.obj
 0001:0003a7c5       __lockexit                 0043b7c5 f   LIBCMT:crt0dat.obj
 0001:0003a7ce       __unlockexit               0043b7ce f   LIBCMT:crt0dat.obj
 0001:0003a7ef       __cinit                    0043b7ef f   LIBCMT:crt0dat.obj
 0001:0003a91c       _exit                      0043b91c f   LIBCMT:crt0dat.obj
 0001:0003a92d       __exit                     0043b92d f   LIBCMT:crt0dat.obj
 0001:0003a93e       __cexit                    0043b93e f   LIBCMT:crt0dat.obj
 0001:0003a94d       __c_exit                   0043b94d f   LIBCMT:crt0dat.obj
 0001:0003a960       _strlen                    0043b960 f   LIBCMT:strlen.obj
 0001:0003a9f0       _strcmp                    0043b9f0 f   LIBCMT:strcmp.obj
 0001:0003aa80       _strcpy                    0043ba80 f   LIBCMT:strcat.obj
 0001:0003aa90       _strcat                    0043ba90 f   LIBCMT:strcat.obj
 0001:0003ad37       _strtol                    0043bd37 f   LIBCMT:strtol.obj
 0001:0003ad4e       _realloc                   0043bd4e f   LIBCMT:realloc.obj
 0001:0003aefb       __callnewh                 0043befb f   LIBCMT:handler.obj
 0001:0003af20       _memcpy                    0043bf20 f   LIBCMT:memcpy.obj
 0001:0003b260       __EH_prolog                0043c260 f   LIBCMT:ehprolog.obj
 0001:0003b2ec       ___FrameUnwindToState      0043c2ec f   LIBCMT:frame.obj
 0001:0003b3ba       ___DestructExceptionObject 0043c3ba f   LIBCMT:frame.obj
 0001:0003b41e       ?__uncaught_exception@@YA_NXZ 0043c41e f   LIBCMT:frame.obj
 0001:0003ba9a       ___InternalCxxFrameHandler 0043ca9a f   LIBCMT:frame.obj
 0001:0003bb3c       ___crtLCMapStringA         0043cb3c f   LIBCMT:a_map.obj
 0001:0003bef8       ___pctype_func             0043cef8 f   LIBCMT:ctype.obj
 0001:0003befe       ___init_ctype              0043cefe f   LIBCMT:initctyp.obj
 0001:0003c0e8       ____lc_codepage_func       0043d0e8 f   LIBCMT:initctyp.obj
 0001:0003c101       ____lc_handle_func         0043d101 f   LIBCMT:initctyp.obj
 0001:0003c11a       __mtinitlocks              0043d11a f   LIBCMT:mlock.obj
 0001:0003c163       __mtdeletelocks            0043d163 f   LIBCMT:mlock.obj
 0001:0003c1b8       __unlock                   0043d1b8 f   LIBCMT:mlock.obj
 0001:0003c1cd       __mtinitlocknum            0043d1cd f   LIBCMT:mlock.obj
 0001:0003c26d       __lock                     0043d26d f   LIBCMT:mlock.obj
 0001:0003c29e       ____setlc_active_func      0043d29e f   LIBCMT:setlocal.obj
 0001:0003c2a4       ____unguarded_readlc_active_add_func 0043d2a4 f   LIBCMT:setlocal.obj
 0001:0003c2aa       ___freetlocinfo            0043d2aa f   LIBCMT:setlocal.obj
 0001:0003c43b       ___init_dummy              0043d43b f   LIBCMT:setlocal.obj
 0001:0003c43b       ___init_collate            0043d43b f   LIBCMT:initcoll.obj
 0001:0003c43e       __strcats                  0043d43e f   LIBCMT:setlocal.obj
 0001:0003c462       ___lc_strtolc              0043d462 f   LIBCMT:setlocal.obj
 0001:0003c53e       ___lc_lctostr              0043d53e f   LIBCMT:setlocal.obj
 0001:0003c58c       ___updatetlocinfo          0043d58c f   LIBCMT:setlocal.obj
 0001:0003c686       __expandlocale             0043d686 f   LIBCMT:setlocal.obj
 0001:0003cc4a       _setlocale                 0043dc4a f   LIBCMT:setlocal.obj
 0001:0003cda4       __SEH_prolog               0043dda4 f   LIBCMT:sehprolg.obj
 0001:0003cddf       __SEH_epilog               0043dddf f   LIBCMT:sehprolg.obj
 0001:0003cdf0       _memcmp                    0043ddf0 f   LIBCMT:memcmp.obj
 0001:0003ceb0       _memset                    0043deb0 f   LIBCMT:memset.obj
 0001:0003cf10       _abort                     0043df10 f   LIBCMT:abort.obj
 0001:0003cf28       ___crtTlsAlloc@4           0043df28 f   LIBCMT:tidtable.obj
 0001:0003cf31       __mtterm                   0043df31 f   LIBCMT:tidtable.obj
 0001:0003cf4e       __initptd                  0043df4e f   LIBCMT:tidtable.obj
 0001:0003cf61       __getptd                   0043df61 f   LIBCMT:tidtable.obj
 0001:0003cfd2       __freefls@4                0043dfd2 f   LIBCMT:tidtable.obj
 0001:0003d119       __freeptd                  0043e119 f   LIBCMT:tidtable.obj
 0001:0003d148       __mtinit                   0043e148 f   LIBCMT:tidtable.obj
 0001:0003d237       ?terminate@@YAXXZ          0043e237 f   LIBCMT:hooks.obj
 0001:0003d26c       ?_inconsistency@@YAXXZ     0043e26c f   LIBCMT:hooks.obj
 0001:0003d2a0       __CallSettingFrame@12      0043e2a0 f   LIBCMT:lowhelpr.obj
 0001:0003d2c7       __NLG_Return               0043e2c7     LIBCMT:lowhelpr.obj
 0001:0003d2ec       ___security_init_cookie    0043e2ec f   LIBCMT:seccinit.obj
 0001:0003d352       ___security_error_handler  0043e352 f   LIBCMT:secfail.obj
 0001:0003d49a       __msize                    0043e49a f   LIBCMT:msize.obj
 0001:0003d510       __flsbuf                   0043e510 f   LIBCMT:_flsbuf.obj
 0001:0003d6b7       __output                   0043e6b7 f   LIBCMT:output.obj
 0001:0003deb1       ___isctype_mt              0043eeb1 f   LIBCMT:isctype.obj
 0001:0003df28       ?__CxxUnhandledExceptionFilter@@YGJPAU_EXCEPTION_POINTERS@@@Z 0043ef28 f   LIBCMT:unhandld.obj
 0001:0003df76       ?__CxxSetUnhandledExceptionFilter@@YAHXZ 0043ef76 f   LIBCMT:unhandld.obj
 0001:0003df89       ?__CxxRestoreUnhandledExceptionFilter@@YAXXZ 0043ef89 f   LIBCMT:unhandld.obj
 0001:0003df96       __close_lk                 0043ef96 f   LIBCMT:close.obj
 0001:0003e019       __close                    0043f019 f   LIBCMT:close.obj
 0001:0003e0b4       __freebuf                  0043f0b4 f   LIBCMT:_freebuf.obj
 0001:0003e0df       __filbuf                   0043f0df f   LIBCMT:_filbuf.obj
 0001:0003e1c0       __openfile                 0043f1c0 f   LIBCMT:_open.obj
 0001:0003e328       __getstream                0043f328 f   LIBCMT:stream.obj
 0001:0003e450       __aulldiv                  0043f450 f   LIBCMT:ulldiv.obj
 0001:0003e4b8       __NMSG_WRITE               0043f4b8 f   LIBCMT:crt0msg.obj
 0001:0003e62f       __FF_MSGBANNER             0043f62f f   LIBCMT:crt0msg.obj
 0001:0003e668       __XcptFilter               0043f668 f   LIBCMT:winxfltr.obj
 0001:0003e7cc       __wincmdln                 0043f7cc f   LIBCMT:wincmdln.obj
 0001:0003e829       __setenvp                  0043f829 f   LIBCMT:stdenvp.obj
 0001:0003ea5c       __setargv                  0043fa5c f   LIBCMT:stdargv.obj
 0001:0003eafe       ___crtGetEnvironmentStringsA 0043fafe f   LIBCMT:a_env.obj
 0001:0003ec20       __ioinit                   0043fc20 f   LIBCMT:ioinit.obj
 0001:0003ee1e       __RTC_Initialize           0043fe1e f   LIBCMT:initsect.obj
 0001:0003ee62       __RTC_Terminate            0043fe62 f   LIBCMT:initsect.obj
 0001:0003eea6       ___heap_select             0043fea6 f   LIBCMT:heapinit.obj
 0001:0003eec0       __heap_init                0043fec0 f   LIBCMT:heapinit.obj
 0001:0003ef11       __write_lk                 0043ff11 f   LIBCMT:write.obj
 0001:0003f0df       __write                    004400df f   LIBCMT:write.obj
 0001:0003f18a       __stbuf                    0044018a f   LIBCMT:_sftbuf.obj
 0001:0003f212       __ftbuf                    00440212 f   LIBCMT:_sftbuf.obj
 0001:0003f23c       __ValidateEH3RN            0044023c f   LIBCMT:eh3valid.obj
 0001:0003f649       ___updatetmbcinfo          00440649 f   LIBCMT:mbctype.obj
 0001:0003f848       __setmbcp                  00440848 f   LIBCMT:mbctype.obj
 0001:0003f998       ___initmbctable            00440998 f   LIBCMT:mbctype.obj
 0001:0003f9b6       __forcdecpt                004409b6 f   LIBCMT:cvt.obj
 0001:0003f9f2       __cropzeros                004409f2 f   LIBCMT:cvt.obj
 0001:0003fa3d       __positive                 00440a3d f   LIBCMT:cvt.obj
 0001:0003fa57       __fassign                  00440a57 f   LIBCMT:cvt.obj
 0001:0003fb60       __cftoe                    00440b60 f   LIBCMT:cvt.obj
 0001:0003fc68       __cftof                    00440c68 f   LIBCMT:cvt.obj
 0001:0003fcca       __cftog                    00440cca f   LIBCMT:cvt.obj
 0001:0003fd64       __cfltcvt                  00440d64 f   LIBCMT:cvt.obj
 0001:0003fdb5       __setdefaultprecision      00440db5 f   LIBCMT:fp8.obj
 0001:0003fdc7       __ms_p5_test_fdiv          00440dc7 f   LIBCMT:testfdiv.obj
 0001:0003fe07       __ms_p5_mp_test_fdiv       00440e07 f   LIBCMT:testfdiv.obj
 0001:0003fe30       ___sbh_heap_init           00440e30 f   LIBCMT:sbheap.obj
 0001:0003fe78       ___sbh_find_block          00440e78 f   LIBCMT:sbheap.obj
 0001:0003fea3       ___sbh_free_block          00440ea3 f   LIBCMT:sbheap.obj
 0001:000401bb       ___sbh_alloc_new_region    004411bb f   LIBCMT:sbheap.obj
 0001:00040272       ___sbh_alloc_new_group     00441272 f   LIBCMT:sbheap.obj
 0001:00040378       ___sbh_resize_block        00441378 f   LIBCMT:sbheap.obj
 0001:00040657       ___sbh_alloc_block         00441657 f   LIBCMT:sbheap.obj
 0001:00040953       __fcloseall                00441953 f   LIBCMT:closeall.obj
 0001:00040fd5       ___tzset                   00441fd5 f   LIBCMT:tzset.obj
 0001:00041021       __isindst                  00442021 f   LIBCMT:tzset.obj
 0001:0004105f       _gmtime                    0044205f f   LIBCMT:gmtime.obj
 0001:00041170       _strrchr                   00442170 f   LIBCMT:strrchr.obj
 0001:000411a0       __aulldvrm                 004421a0 f   LIBCMT:ulldvrm.obj
 0001:00041235       __commit                   00442235 f   LIBCMT:commit.obj
 0001:000412f1       __getbuf                   004422f1 f   LIBCMT:_getbuf.obj
 0001:00041335       __ftelli64_lk              00442335 f   LIBCMT:ftelli64.obj
 0001:000414ca       __ftelli64                 004424ca f   LIBCMT:ftelli64.obj
 0001:00041511       __lseek_lk                 00442511 f   LIBCMT:lseek.obj
 0001:00041585       __lseek                    00442585 f   LIBCMT:lseek.obj
 0001:00041630       __fseeki64_lk              00442630 f   LIBCMT:fseeki64.obj
 0001:000416c3       __fseeki64                 004426c3 f   LIBCMT:fseeki64.obj
 0001:0004170f       __fltin2                   0044270f f   LIBCMT:cfin.obj
 0001:000417a4       __read_lk                  004427a4 f   LIBCMT:read.obj
 0001:0004197f       __read                     0044297f f   LIBCMT:read.obj
 0001:00041a30       __allrem                   00442a30 f   LIBCMT:llrem.obj
 0001:00041ae2       ?_ValidateRead@@YAHPBXI@Z  00442ae2 f   LIBCMT:validate.obj
 0001:00041afe       ?_ValidateWrite@@YAHPAXI@Z 00442afe f   LIBCMT:validate.obj
 0001:00041b1a       ?_ValidateExecute@@YAHP6GHXZ@Z 00442b1a f   LIBCMT:validate.obj
 0001:00041b32       ___ansicp                  00442b32 f   LIBCMT:convrtcp.obj
 0001:00041b75       ___convertcp               00442b75 f   LIBCMT:convrtcp.obj
 0001:00041d3e       ___crtGetStringTypeA       00442d3e f   LIBCMT:a_str.obj
 0001:00041ef8       ___getlocaleinfo           00442ef8 f   LIBCMT:inithelp.obj
 0001:0004202f       ___crtInitCritSecAndSpinCount 0044302f f   LIBCMT:initcrit.obj
 0001:00042421       ___free_lc_time            00443421 f   LIBCMT:inittime.obj
 0001:000425b1       ___init_time               004435b1 f   LIBCMT:inittime.obj
 0001:00042610       ___free_lconv_num          00443610 f   LIBCMT:initnum.obj
 0001:0004266f       ___init_numeric            0044366f f   LIBCMT:initnum.obj
 0001:0004283c       ___free_lconv_mon          0044383c f   LIBCMT:initmon.obj
 0001:00042915       ___init_monetary           00443915 f   LIBCMT:initmon.obj
 0001:00043293       ___get_qualified_locale    00444293 f   LIBCMT:getqloc.obj
 0001:00043450       _strpbrk                   00444450 f   LIBCMT:strpbrk.obj
 0001:000434be       _raise                     004444be f   LIBCMT:winsig.obj
 0001:00043637       ___crtMessageBoxA          00444637 f   LIBCMT:crtmbox.obj
 0001:00043730       __isatty                   00444730 f   LIBCMT:isatty.obj
 0001:00043730       _isatty                    00444730 f   LIBCMT:isatty.obj
 0001:0004375a       ___wctomb_mt               0044475a f   LIBCMT:wctomb.obj
 0001:000437ba       _wctomb                    004447ba f   LIBCMT:wctomb.obj
 0001:000437e1       __set_osfhnd               004447e1 f   LIBCMT:osfinfo.obj
 0001:0004385d       __free_osfhnd              0044485d f   LIBCMT:osfinfo.obj
 0001:000438dc       __get_osfhandle            004448dc f   LIBCMT:osfinfo.obj
 0001:0004391d       __lock_fhandle             0044491d f   LIBCMT:osfinfo.obj
 0001:000439bd       __unlock_fhandle           004449bd f   LIBCMT:osfinfo.obj
 0001:000439df       __alloc_osfhnd             004449df f   LIBCMT:osfinfo.obj
 0001:00043e42       __sopen                    00444e42 f   LIBCMT:open.obj
 0001:00043eca       __ismbblead                00444eca f   LIBCMT:ismbbyte.obj
 0001:00043edb       __lseeki64_lk              00444edb f   LIBCMT:lseeki64.obj
 0001:00043f5e       __lseeki64                 00444f5e f   LIBCMT:lseeki64.obj
 0001:0004401c       ___tolower_mt              0044501c f   LIBCMT:tolower.obj
 0001:000440e4       _tolower                   004450e4 f   LIBCMT:tolower.obj
 0001:00044106       __ZeroTail                 00445106 f   LIBCMT:intrncvt.obj
 0001:00044138       __IncMan                   00445138 f   LIBCMT:intrncvt.obj
 0001:00044185       __RoundMan                 00445185 f   LIBCMT:intrncvt.obj
 0001:000441f7       __CopyMan                  004451f7 f   LIBCMT:intrncvt.obj
 0001:00044212       __IsZeroMan                00445212 f   LIBCMT:intrncvt.obj
 0001:0004422b       __ShrMan                   0044522b f   LIBCMT:intrncvt.obj
 0001:000442a6       __ld12cvt                  004452a6 f   LIBCMT:intrncvt.obj
 0001:000443fe       __ld12tod                  004453fe f   LIBCMT:intrncvt.obj
 0001:00044414       __ld12tof                  00445414 f   LIBCMT:intrncvt.obj
 0001:0004442a       __atodbl                   0044542a f   LIBCMT:intrncvt.obj
 0001:00044467       __atoflt                   00445467 f   LIBCMT:intrncvt.obj
 0001:000444a4       __fptostr                  004454a4 f   LIBCMT:_fptostr.obj
 0001:0004451b       ___dtold                   0044551b f   LIBCMT:cfout.obj
 0001:000445d5       __fltout2                  004455d5 f   LIBCMT:cfout.obj
 0001:00044641       __fptrap                   00445641 f   LIBCMT:crt0fp.obj
 0001:0004476a       __control87                0044576a f   LIBCMT:ieee87.obj
 0001:0004479c       __controlfp                0044579c f   LIBCMT:ieee87.obj
 0001:000447b2       __getenv_lk                004457b2 f   LIBCMT:getenv.obj
 0001:00044833       ___strgtold12              00445833 f   LIBCMT:strgtold.obj
 0001:00044c67       ___crtGetLocaleInfoW       00445c67 f   LIBCMT:w_loc.obj
 0001:00044d97       ___crtGetLocaleInfoA       00445d97 f   LIBCMT:a_loc.obj
 0001:00044ee0       ___ascii_stricmp           00445ee0 f   LIBCMT:_stricmp.obj
 0001:00044f2e       __stricmp                  00445f2e f   LIBCMT:stricmp.obj
 0001:00044f2e       _stricmp                   00445f2e f   LIBCMT:stricmp.obj
 0001:00044f97       __strnicmp                 00445f97 f   LIBCMT:strnicmp.obj
 0001:00045016       __chsize_lk                00446016 f   LIBCMT:chsize.obj
 0001:00045157       ___addl                    00446157 f   LIBCMT:mantold.obj
 0001:00045178       ___add_12                  00446178 f   LIBCMT:mantold.obj
 0001:000451d6       ___shl_12                  004461d6 f   LIBCMT:mantold.obj
 0001:00045204       ___shr_12                  00446204 f   LIBCMT:mantold.obj
 0001:00045231       ___mtold12                 00446231 f   LIBCMT:mantold.obj
 0001:0004530f       _$I10_OUTPUT               0044630f f   LIBCMT:x10fout.obj
 0001:0004559d       __mbsnbicoll               0044659d f   LIBCMT:mbsnbico.obj
 0001:000455eb       ___wtomb_environ           004465eb f   LIBCMT:wtombenv.obj
 0001:0004567b       ___ld12mul                 0044667b f   LIBCMT:tenpow.obj
 0001:000458ad       ___multtenpow12            004468ad f   LIBCMT:tenpow.obj
 0001:00045940       ___ascii_strnicmp          00446940 f   LIBCMT:_strnicm.obj
 0001:000459a1       __setmode_lk               004469a1 f   LIBCMT:setmode.obj
 0001:00045a29       ___crtCompareStringA       00446a29 f   LIBCMT:a_cmp.obj
 0001:00045e5b       ___crtsetenv               00446e5b f   LIBCMT:setenv.obj
 0001:00046030       __strdup                   00447030 f   LIBCMT:strdup.obj
 0001:0004605b       __mbschr                   0044705b f   LIBCMT:mbschr.obj
 0001:000460d6       _AcceptEx@32               004470d6 f   mswsock:MSWSOCK.dll
 0001:000460dc       _GetAcceptExSockaddrs@32   004470dc f   mswsock:MSWSOCK.dll
 0001:000460e2       ?RemoveAll@?$CSimpleArray@PAUHINSTANCE__@@V?$CSimpleArrayEqualHelper@PAUHINSTANCE__@@@ATL@@@ATL@@QAEXXZ 004470e2 f i atls:atlbase.obj
 0001:000460ff       ??0_ATL_BASE_MODULE70@ATL@@QAE@XZ 004470ff f i atls:atlbase.obj
 0001:00046119       ??1CAtlBaseModule@ATL@@QAE@XZ 00447119 f   atls:atlbase.obj
 0001:0004612f       ??0CAtlBaseModule@ATL@@QAE@XZ 0044712f f   atls:atlbase.obj
 0001:000461da       _RtlUnwind@16              004471da f   kernel32:KERNEL32.dll
 0001:00048950       ?Instance@?1??GetInstance@?$CStaticSingleton@VCMasterPassword@@@@SAAAVCMasterPassword@@XZ@$AV2@A 00449950 f i authorizethread.obj
 0001:00048a50       ?obj@?1??instance@?$singleton_default@Upool_type@?$singleton_pool@Ufast_pool_allocator_tag@boost@@$0M@Udefault_user_allocator_new_delete@2@Vwin32_mutex@pool@details@2@$0CA@@boost@@@pool@details@boost@@SAAAUpool_type@?$singleton_pool@Ufast_pool_allocator_tag@boost@@$0M@Udefault_user_allocator_new_delete@2@Vwin32_mutex@pool@details@2@$0CA@@4@XZ@$AU564@A 00449a50 f i rylgamelibrary:depositcontainer.obj
 0001:00048aa0       ?obj@?1??instance@?$singleton_default@Upool_type@?$singleton_pool@Ufast_pool_allocator_tag@boost@@$0BI@Udefault_user_allocator_new_delete@2@Vwin32_mutex@pool@details@2@$0CA@@boost@@@pool@details@boost@@SAAAUpool_type@?$singleton_pool@Ufast_pool_allocator_tag@boost@@$0BI@Udefault_user_allocator_new_delete@2@Vwin32_mutex@pool@details@2@$0CA@@4@XZ@$AU564@A 00449aa0 f i rylgamelibrary:creaturemanager.obj
 0001:00048ab0       ?obj@?1??instance@?$singleton_default@Upool_type@?$singleton_pool@Ufast_pool_allocator_tag@boost@@$0BE@Udefault_user_allocator_new_delete@2@Vwin32_mutex@pool@details@2@$0CA@@boost@@@pool@details@boost@@SAAAUpool_type@?$singleton_pool@Ufast_pool_allocator_tag@boost@@$0BE@Udefault_user_allocator_new_delete@2@Vwin32_mutex@pool@details@2@$0CA@@4@XZ@$AU564@A 00449ab0 f i rylgamelibrary:creaturemanager.obj
 0001:00048ac0       ?obj@?1??instance@?$singleton_default@Upool_type@?$singleton_pool@Ufast_pool_allocator_tag@boost@@$0DI@Udefault_user_allocator_new_delete@2@Vwin32_mutex@pool@details@2@$0CA@@boost@@@pool@details@boost@@SAAAUpool_type@?$singleton_pool@Ufast_pool_allocator_tag@boost@@$0DI@Udefault_user_allocator_new_delete@2@Vwin32_mutex@pool@details@2@$0CA@@4@XZ@$AU564@A 00449ac0 f i rylgamelibrary:cell.obj
 0002:00000000       __imp__GetUserNameA@8      0044a000     advapi32:ADVAPI32.dll
 0002:00000004       \177ADVAPI32_NULL_THUNK_DATA 0044a004     advapi32:ADVAPI32.dll
 0002:00000008       __imp__GetStockObject@4    0044a008     gdi32:GDI32.dll
 0002:0000000c       __imp__CreateFontA@56      0044a00c     gdi32:GDI32.dll
 0002:00000010       __imp__DeleteObject@4      0044a010     gdi32:GDI32.dll
 0002:00000014       __imp__SetBkColor@8        0044a014     gdi32:GDI32.dll
 0002:00000018       \177GDI32_NULL_THUNK_DATA  0044a018     gdi32:GDI32.dll
 0002:0000001c       __imp__GetLastError@0      0044a01c     kernel32:KERNEL32.dll
 0002:00000020       __imp__WaitForMultipleObjects@16 0044a020     kernel32:KERNEL32.dll
 0002:00000024       __imp__CreateSemaphoreA@16 0044a024     kernel32:KERNEL32.dll
 0002:00000028       __imp__CloseHandle@4       0044a028     kernel32:KERNEL32.dll
 0002:0000002c       __imp__ReleaseSemaphore@12 0044a02c     kernel32:KERNEL32.dll
 0002:00000030       __imp__InterlockedExchange@8 0044a030     kernel32:KERNEL32.dll
 0002:00000034       __imp__CreateMutexA@12     0044a034     kernel32:KERNEL32.dll
 0002:00000038       __imp__SetEvent@4          0044a038     kernel32:KERNEL32.dll
 0002:0000003c       __imp__GetCurrentThreadId@0 0044a03c     kernel32:KERNEL32.dll
 0002:00000040       __imp__LeaveCriticalSection@4 0044a040     kernel32:KERNEL32.dll
 0002:00000044       __imp__EnterCriticalSection@4 0044a044     kernel32:KERNEL32.dll
 0002:00000048       __imp__DeleteCriticalSection@4 0044a048     kernel32:KERNEL32.dll
 0002:0000004c       __imp__CreateEventA@16     0044a04c     kernel32:KERNEL32.dll
 0002:00000050       __imp__InitializeCriticalSection@4 0044a050     kernel32:KERNEL32.dll
 0002:00000054       __imp__SetEnvironmentVariableA@8 0044a054     kernel32:KERNEL32.dll
 0002:00000058       __imp__SetEndOfFile@4      0044a058     kernel32:KERNEL32.dll
 0002:0000005c       __imp__GetLocaleInfoW@16   0044a05c     kernel32:KERNEL32.dll
 0002:00000060       __imp__SetStdHandle@8      0044a060     kernel32:KERNEL32.dll
 0002:00000064       __imp__IsValidCodePage@4   0044a064     kernel32:KERNEL32.dll
 0002:00000068       __imp__IsValidLocale@8     0044a068     kernel32:KERNEL32.dll
 0002:0000006c       __imp__EnumSystemLocalesA@8 0044a06c     kernel32:KERNEL32.dll
 0002:00000070       __imp__GetUserDefaultLCID@0 0044a070     kernel32:KERNEL32.dll
 0002:00000074       __imp__GetStringTypeW@16   0044a074     kernel32:KERNEL32.dll
 0002:00000078       __imp__GetStringTypeA@20   0044a078     kernel32:KERNEL32.dll
 0002:0000007c       __imp__IsBadCodePtr@4      0044a07c     kernel32:KERNEL32.dll
 0002:00000080       __imp__IsBadReadPtr@8      0044a080     kernel32:KERNEL32.dll
 0002:00000084       __imp__SetFilePointer@16   0044a084     kernel32:KERNEL32.dll
 0002:00000088       __imp__FlushFileBuffers@4  0044a088     kernel32:KERNEL32.dll
 0002:0000008c       __imp__GetTimeZoneInformation@4 0044a08c     kernel32:KERNEL32.dll
 0002:00000090       __imp__IsBadWritePtr@8     0044a090     kernel32:KERNEL32.dll
 0002:00000094       __imp__GetOEMCP@0          0044a094     kernel32:KERNEL32.dll
 0002:00000098       __imp__VirtualFree@12      0044a098     kernel32:KERNEL32.dll
 0002:0000009c       __imp__HeapCreate@12       0044a09c     kernel32:KERNEL32.dll
 0002:000000a0       __imp__HeapDestroy@4       0044a0a0     kernel32:KERNEL32.dll
 0002:000000a4       __imp__GetFileType@4       0044a0a4     kernel32:KERNEL32.dll
 0002:000000a8       __imp__SetHandleCount@4    0044a0a8     kernel32:KERNEL32.dll
 0002:000000ac       __imp__GetEnvironmentStringsW@0 0044a0ac     kernel32:KERNEL32.dll
 0002:000000b0       __imp__CreateFileA@28      0044a0b0     kernel32:KERNEL32.dll
 0002:000000b4       __imp__GetLocalTime@4      0044a0b4     kernel32:KERNEL32.dll
 0002:000000b8       __imp__CreateDirectoryA@8  0044a0b8     kernel32:KERNEL32.dll
 0002:000000bc       __imp__GetFileAttributesA@4 0044a0bc     kernel32:KERNEL32.dll
 0002:000000c0       __imp__WriteFile@20        0044a0c0     kernel32:KERNEL32.dll
 0002:000000c4       __imp__GetCommandLineA@0   0044a0c4     kernel32:KERNEL32.dll
 0002:000000c8       __imp__GetACP@0            0044a0c8     kernel32:KERNEL32.dll
 0002:000000cc       __imp__GetLocaleInfoA@16   0044a0cc     kernel32:KERNEL32.dll
 0002:000000d0       __imp__GetVersionExA@4     0044a0d0     kernel32:KERNEL32.dll
 0002:000000d4       __imp__MultiByteToWideChar@24 0044a0d4     kernel32:KERNEL32.dll
 0002:000000d8       __imp__WideCharToMultiByte@32 0044a0d8     kernel32:KERNEL32.dll
 0002:000000dc       __imp__RaiseException@16   0044a0dc     kernel32:KERNEL32.dll
 0002:000000e0       __imp__CompareStringA@24   0044a0e0     kernel32:KERNEL32.dll
 0002:000000e4       __imp__CompareStringW@24   0044a0e4     kernel32:KERNEL32.dll
 0002:000000e8       __imp__ReadFile@20         0044a0e8     kernel32:KERNEL32.dll
 0002:000000ec       __imp__GetFileSize@8       0044a0ec     kernel32:KERNEL32.dll
 0002:000000f0       __imp__GetTickCount@0      0044a0f0     kernel32:KERNEL32.dll
 0002:000000f4       __imp__WaitForSingleObject@8 0044a0f4     kernel32:KERNEL32.dll
 0002:000000f8       __imp__InterlockedCompareExchange@12 0044a0f8     kernel32:KERNEL32.dll
 0002:000000fc       __imp__GetCurrentProcessId@0 0044a0fc     kernel32:KERNEL32.dll
 0002:00000100       __imp__GetModuleFileNameA@12 0044a100     kernel32:KERNEL32.dll
 0002:00000104       __imp__CreateIoCompletionPort@16 0044a104     kernel32:KERNEL32.dll
 0002:00000108       __imp__InterlockedIncrement@4 0044a108     kernel32:KERNEL32.dll
 0002:0000010c       __imp__InterlockedDecrement@4 0044a10c     kernel32:KERNEL32.dll
 0002:00000110       __imp__Sleep@4             0044a110     kernel32:KERNEL32.dll
 0002:00000114       __imp__GetSystemInfo@4     0044a114     kernel32:KERNEL32.dll
 0002:00000118       __imp__PulseEvent@4        0044a118     kernel32:KERNEL32.dll
 0002:0000011c       __imp__DeleteFileA@4       0044a11c     kernel32:KERNEL32.dll
 0002:00000120       __imp__FreeLibrary@4       0044a120     kernel32:KERNEL32.dll
 0002:00000124       __imp__GetProcAddress@8    0044a124     kernel32:KERNEL32.dll
 0002:00000128       __imp__LoadLibraryA@4      0044a128     kernel32:KERNEL32.dll
 0002:0000012c       __imp__SetUnhandledExceptionFilter@4 0044a12c     kernel32:KERNEL32.dll
 0002:00000130       __imp__FormatMessageA@28   0044a130     kernel32:KERNEL32.dll
 0002:00000134       __imp__GetModuleHandleA@4  0044a134     kernel32:KERNEL32.dll
 0002:00000138       __imp__VirtualQuery@12     0044a138     kernel32:KERNEL32.dll
 0002:0000013c       __imp__IsBadStringPtrA@8   0044a13c     kernel32:KERNEL32.dll
 0002:00000140       __imp__GetComputerNameA@8  0044a140     kernel32:KERNEL32.dll
 0002:00000144       __imp__LocalFree@4         0044a144     kernel32:KERNEL32.dll
 0002:00000148       __imp__GetCurrentProcess@0 0044a148     kernel32:KERNEL32.dll
 0002:0000014c       __imp__GetCurrentThread@0  0044a14c     kernel32:KERNEL32.dll
 0002:00000150       __imp__GetPrivateProfileIntA@16 0044a150     kernel32:KERNEL32.dll
 0002:00000154       __imp__GetPrivateProfileStringA@24 0044a154     kernel32:KERNEL32.dll
 0002:00000158       __imp__GetQueuedCompletionStatus@20 0044a158     kernel32:KERNEL32.dll
 0002:0000015c       __imp__PostQueuedCompletionStatus@16 0044a15c     kernel32:KERNEL32.dll
 0002:00000160       __imp__RtlUnwind@16        0044a160     kernel32:KERNEL32.dll
 0002:00000164       __imp__ExitProcess@4       0044a164     kernel32:KERNEL32.dll
 0002:00000168       __imp__GetSystemTimeAsFileTime@4 0044a168     kernel32:KERNEL32.dll
 0002:0000016c       __imp__GetStartupInfoA@4   0044a16c     kernel32:KERNEL32.dll
 0002:00000170       __imp__HeapAlloc@12        0044a170     kernel32:KERNEL32.dll
 0002:00000174       __imp__HeapFree@12         0044a174     kernel32:KERNEL32.dll
 0002:00000178       __imp__VirtualProtect@16   0044a178     kernel32:KERNEL32.dll
 0002:0000017c       __imp__VirtualAlloc@16     0044a17c     kernel32:KERNEL32.dll
 0002:00000180       __imp__ExitThread@4        0044a180     kernel32:KERNEL32.dll
 0002:00000184       __imp__CreateThread@24     0044a184     kernel32:KERNEL32.dll
 0002:00000188       __imp__TerminateProcess@8  0044a188     kernel32:KERNEL32.dll
 0002:0000018c       __imp__HeapReAlloc@16      0044a18c     kernel32:KERNEL32.dll
 0002:00000190       __imp__LCMapStringA@24     0044a190     kernel32:KERNEL32.dll
 0002:00000194       __imp__LCMapStringW@24     0044a194     kernel32:KERNEL32.dll
 0002:00000198       __imp__GetCPInfo@8         0044a198     kernel32:KERNEL32.dll
 0002:0000019c       __imp__TlsAlloc@0          0044a19c     kernel32:KERNEL32.dll
 0002:000001a0       __imp__SetLastError@4      0044a1a0     kernel32:KERNEL32.dll
 0002:000001a4       __imp__TlsFree@4           0044a1a4     kernel32:KERNEL32.dll
 0002:000001a8       __imp__TlsSetValue@8       0044a1a8     kernel32:KERNEL32.dll
 0002:000001ac       __imp__TlsGetValue@4       0044a1ac     kernel32:KERNEL32.dll
 0002:000001b0       __imp__QueryPerformanceCounter@4 0044a1b0     kernel32:KERNEL32.dll
 0002:000001b4       __imp__HeapSize@12         0044a1b4     kernel32:KERNEL32.dll
 0002:000001b8       __imp__GetStdHandle@4      0044a1b8     kernel32:KERNEL32.dll
 0002:000001bc       __imp__UnhandledExceptionFilter@4 0044a1bc     kernel32:KERNEL32.dll
 0002:000001c0       __imp__FreeEnvironmentStringsA@4 0044a1c0     kernel32:KERNEL32.dll
 0002:000001c4       __imp__GetEnvironmentStrings@0 0044a1c4     kernel32:KERNEL32.dll
 0002:000001c8       __imp__FreeEnvironmentStringsW@4 0044a1c8     kernel32:KERNEL32.dll
 0002:000001cc       \177KERNEL32_NULL_THUNK_DATA 0044a1cc     kernel32:KERNEL32.dll
 0002:000001d0       __imp__GetAcceptExSockaddrs@32 0044a1d0     mswsock:MSWSOCK.dll
 0002:000001d4       __imp__AcceptEx@32         0044a1d4     mswsock:MSWSOCK.dll
 0002:000001d8       \177MSWSOCK_NULL_THUNK_DATA 0044a1d8     mswsock:MSWSOCK.dll
 0002:000001dc       __imp__SysAllocString@4    0044a1dc     oleaut32:OLEAUT32.dll
 0002:000001e0       __imp__SysFreeString@4     0044a1e0     oleaut32:OLEAUT32.dll
 0002:000001e4       __imp__GetErrorInfo@8      0044a1e4     oleaut32:OLEAUT32.dll
 0002:000001e8       \177OLEAUT32_NULL_THUNK_DATA 0044a1e8     oleaut32:OLEAUT32.dll
 0002:000001ec       __imp__Shell_NotifyIconA@8 0044a1ec     shell32:SHELL32.dll
 0002:000001f0       \177SHELL32_NULL_THUNK_DATA 0044a1f0     shell32:SHELL32.dll
 0002:000001f4       __imp__IsDialogMessageA@8  0044a1f4     user32:USER32.dll
 0002:000001f8       __imp__PostMessageA@16     0044a1f8     user32:USER32.dll
 0002:000001fc       __imp__FindWindowA@8       0044a1fc     user32:USER32.dll
 0002:00000200       __imp__PostQuitMessage@4   0044a200     user32:USER32.dll
 0002:00000204       __imp__GetCursorPos@4      0044a204     user32:USER32.dll
 0002:00000208       __imp__SetForegroundWindow@4 0044a208     user32:USER32.dll
 0002:0000020c       __imp__TrackPopupMenu@28   0044a20c     user32:USER32.dll
 0002:00000210       __imp__DestroyIcon@4       0044a210     user32:USER32.dll
 0002:00000214       __imp__KillTimer@8         0044a214     user32:USER32.dll
 0002:00000218       __imp__GetSystemMetrics@4  0044a218     user32:USER32.dll
 0002:0000021c       __imp__LoadCursorA@8       0044a21c     user32:USER32.dll
 0002:00000220       __imp__CallWindowProcA@20  0044a220     user32:USER32.dll
 0002:00000224       __imp__GetWindowTextA@12   0044a224     user32:USER32.dll
 0002:00000228       __imp__SetWindowTextA@8    0044a228     user32:USER32.dll
 0002:0000022c       __imp__UnregisterClassA@8  0044a22c     user32:USER32.dll
 0002:00000230       __imp__GetPropA@8          0044a230     user32:USER32.dll
 0002:00000234       __imp__SendMessageA@16     0044a234     user32:USER32.dll
 0002:00000238       __imp__DestroyMenu@4       0044a238     user32:USER32.dll
 0002:0000023c       __imp__GetSubMenu@8        0044a23c     user32:USER32.dll
 0002:00000240       __imp__LoadMenuA@8         0044a240     user32:USER32.dll
 0002:00000244       __imp__DefWindowProcA@16   0044a244     user32:USER32.dll
 0002:00000248       __imp__SetPropA@12         0044a248     user32:USER32.dll
 0002:0000024c       __imp__CreateWindowExA@48  0044a24c     user32:USER32.dll
 0002:00000250       __imp__RegisterClassA@4    0044a250     user32:USER32.dll
 0002:00000254       __imp__LoadIconA@8         0044a254     user32:USER32.dll
 0002:00000258       __imp__UpdateWindow@4      0044a258     user32:USER32.dll
 0002:0000025c       __imp__DispatchMessageA@4  0044a25c     user32:USER32.dll
 0002:00000260       __imp__TranslateMessage@4  0044a260     user32:USER32.dll
 0002:00000264       __imp__DestroyWindow@4     0044a264     user32:USER32.dll
 0002:00000268       __imp__GetMessageA@16      0044a268     user32:USER32.dll
 0002:0000026c       __imp__RegisterWindowMessageA@4 0044a26c     user32:USER32.dll
 0002:00000270       __imp__wsprintfA           0044a270     user32:USER32.dll
 0002:00000274       __imp__SetWindowLongA@12   0044a274     user32:USER32.dll
 0002:00000278       __imp__GetSysColorBrush@4  0044a278     user32:USER32.dll
 0002:0000027c       __imp__GetSysColor@4       0044a27c     user32:USER32.dll
 0002:00000280       \177USER32_NULL_THUNK_DATA 0044a280     user32:USER32.dll
 0002:00000284       __imp__timeGetTime@0       0044a284     winmm:WINMM.dll
 0002:00000288       __imp__timeGetDevCaps@8    0044a288     winmm:WINMM.dll
 0002:0000028c       __imp__timeBeginPeriod@4   0044a28c     winmm:WINMM.dll
 0002:00000290       \177WINMM_NULL_THUNK_DATA  0044a290     winmm:WINMM.dll
 0002:00000294       __imp__WSAGetLastError@0   0044a294     ws2_32:WS2_32.dll
 0002:00000298       __imp__shutdown@8          0044a298     ws2_32:WS2_32.dll
 0002:0000029c       __imp__WSARecv@28          0044a29c     ws2_32:WS2_32.dll
 0002:000002a0       __imp__WSASend@28          0044a2a0     ws2_32:WS2_32.dll
 0002:000002a4       __imp__WSASendTo@36        0044a2a4     ws2_32:WS2_32.dll
 0002:000002a8       __imp__setsockopt@20       0044a2a8     ws2_32:WS2_32.dll
 0002:000002ac       __imp__WSAStartup@8        0044a2ac     ws2_32:WS2_32.dll
 0002:000002b0       __imp__closesocket@4       0044a2b0     ws2_32:WS2_32.dll
 0002:000002b4       __imp__ntohs@4             0044a2b4     ws2_32:WS2_32.dll
 0002:000002b8       __imp__inet_ntoa@4         0044a2b8     ws2_32:WS2_32.dll
 0002:000002bc       __imp__inet_addr@4         0044a2bc     ws2_32:WS2_32.dll
 0002:000002c0       __imp__WSASocketA@24       0044a2c0     ws2_32:WS2_32.dll
 0002:000002c4       __imp__connect@12          0044a2c4     ws2_32:WS2_32.dll
 0002:000002c8       __imp__bind@12             0044a2c8     ws2_32:WS2_32.dll
 0002:000002cc       __imp__listen@8            0044a2cc     ws2_32:WS2_32.dll
 0002:000002d0       __imp__gethostbyname@4     0044a2d0     ws2_32:WS2_32.dll
 0002:000002d4       __imp__gethostname@8       0044a2d4     ws2_32:WS2_32.dll
 0002:000002d8       __imp__htonl@4             0044a2d8     ws2_32:WS2_32.dll
 0002:000002dc       __imp__htons@4             0044a2dc     ws2_32:WS2_32.dll
 0002:000002e0       __imp__WSACleanup@0        0044a2e0     ws2_32:WS2_32.dll
 0002:000002e4       \177WS2_32_NULL_THUNK_DATA 0044a2e4     ws2_32:WS2_32.dll
 0002:000002e8       __imp__CoGetMalloc@8       0044a2e8     ole32:ole32.dll
 0002:000002ec       __imp__CoUninitialize@0    0044a2ec     ole32:ole32.dll
 0002:000002f0       __imp__CoInitializeEx@8    0044a2f0     ole32:ole32.dll
 0002:000002f4       __imp__CoCreateInstance@20 0044a2f4     ole32:ole32.dll
 0002:000002f8       \177ole32_NULL_THUNK_DATA  0044a2f8     ole32:ole32.dll
 0002:0000031c       ??_7CAuthAgentDispatch@@6B@ 0044a31c     authagentdispatch.obj
 0002:00000338       ??_C@_0CI@BPBJDGKG@CAuthAgentDispatch?3?3?$HOCAuthAgentD@ 0044a338     authagentdispatch.obj
 0002:00000360       ??_C@_0HF@LEPANALH@D?3?2Work?2RYL?2Source?2v?4538?$FN?5?G?X?$LP?$NM?5?$CI@ 0044a360     authagentdispatch.obj
 0002:000003d8       ??_C@_0CC@DNCMFAED@DP?30x?$CFp?1Destroy?5AuthAgentDispatc@ 0044a3d8     authagentdispatch.obj
 0002:00000400       ??_C@_0EC@ENDKPILN@SS?30x?$CFp?1DP?30x?$CFp?1sCmd?30x?$CF02x?1Requ@ 0044a400     authagentdispatch.obj
 0002:00000448       ??_C@_0FC@GPCDBBLF@DB?$LH?N?$LK?N?E?M?5?$MA?L?$LL?s?G?Q?5?F?P?E?$LG?$MA?L?5?$LF?i?$LO?n?$LP?T?$LN?$MA?$LE@ 0044a448     authagentdispatch.obj
 0002:0000049c       ??_C@_0DN@HDHAKJCG@SS?30x?$CFp?1DP?30x?$CFp?1sCmd?30x?$CF02x?1Requ@ 0044a49c     authagentdispatch.obj
 0002:000004dc       ??_C@_0CO@LJOPDGEG@sCmd?30x?$CF02x?1RequestKey?3?$CFd?1Get?5Se@ 0044a4dc     authagentdispatch.obj
 0002:0000050c       ??_C@_0CD@IGBAOIPL@CAuthAgentDispatch?3?3ParseAgentZo@ 0044a50c     authagentdispatch.obj
 0002:00000530       ??_C@_0CM@BLEAOPMF@sCmd?30x?$CF02x?1RequestKey?3?$CFd?1DBRequ@ 0044a530     authagentdispatch.obj
 0002:0000055c       ??_C@_0CO@DCNHKNJC@CAuthAgentDispatch?3?3ParseBilling@ 0044a55c     authagentdispatch.obj
 0002:0000058c       ??_C@_0BL@JPEHHHLA@UID?30x?$CF08d?5?$MA?$KP?$MA?z?5?$LO?r?$LB?b?5?$LN?G?F?P?4?$AA@ 0044a58c     authagentdispatch.obj
 0002:000005a8       ??_C@_0DA@IOAFGECG@CAuthAgentDispatch?3?3ParseBilling@ 0044a5a8     authagentdispatch.obj
 0002:000005d8       ??_C@_07NGIKAGKG@UnKnown?$AA@ 0044a5d8     authagentdispatch.obj
 0002:000005e0       ??_C@_0BO@NBLAKJEI@CAuthAgentDispatch?3?3Connected?$AA@ 0044a5e0     authagentdispatch.obj
 0002:00000600       ??_C@_0CN@HMJHBFJI@SS?30x?$CFp?1DP?30x?$CFp?1Connected?5CAuthA@ 0044a600     authagentdispatch.obj
 0002:00000630       ??_C@_0DA@LOGNODHO@SS?30x?$CFp?1DP?30x?$CFp?1Disconnected?5CAu@ 0044a630     authagentdispatch.obj
 0002:00000660       ??_C@_0CB@BMIKNJDN@CAuthAgentDispatch?3?3Disconnected@ 0044a660     authagentdispatch.obj
 0002:00000684       ??_C@_0CO@CJNKPPIJ@this?30x?$CFp?1PostMessage?5WM_AGENTAU@ 0044a684     authagentdispatch.obj
 0002:000006b4       ??_C@_0BB@MFDILKBO@RYLMANAGERCLIENT?$AA@ 0044a6b4     authagentdispatch.obj
 0002:000006c8       ??_C@_0CI@DHIKNMFN@CAuthAgentDispatch?3?3ParseSysServ@ 0044a6c8     authagentdispatch.obj
 0002:000006f0       ??_C@_0CL@GJCBMIPC@this?30x?$CFp?1PostMessage?5WM_AGENTAU@ 0044a6f0     authagentdispatch.obj
 0002:0000071c       ??_C@_0CJ@NKFNFIFI@SS?30x?$CFp?1DP?30x?$CFp?1UID?3?$CFu?1Process?5U@ 0044a71c     authagentdispatch.obj
 0002:00000748       ??_C@_0CC@HCLEPAII@CAuthAgentDispatch?3?3ParseUserKil@ 0044a748     authagentdispatch.obj
 0002:0000076c       ??_C@_0BH@KHHIMHAC@UID?3?$CFu?1GetUser?5failed?4?$AA@ 0044a76c     authagentdispatch.obj
 0002:00000784       ??_C@_0CF@FADKNCFI@CAuthAgentDispatch?3?3SendStartSes@ 0044a784     authagentdispatch.obj
 0002:000007ac       ??_C@_0CD@FLNJGIPA@CAuthAgentDispatch?3?3ParseDBGetDa@ 0044a7ac     authagentdispatch.obj
 0002:000007d0       ??_C@_0EE@KLLLKMCO@Invalid?5packet?5command?$CIAuthAgent@ 0044a7d0     authagentdispatch.obj
 0002:00000814       ??_C@_02DKCKIIND@?$CFs?$AA@ 0044a814     authagentservertable.obj
 0002:00000818       ??_C@_0CK@MALNHMOA@CAuthClientDispatch?3?3?$HOCAuthClien@ 0044a818     authclientdispath.obj
 0002:00000848       ??_C@_0HF@MCONOHKH@D?3?2Work?2RYL?2Source?2v?4538?$FN?5?G?X?$LP?$NM?5?$CI@ 0044a848     authclientdispath.obj
 0002:000008c0       ??_C@_0DD@CLLANAGK@SS?30x?$CFp?1DP?30x?$CFp?1IP?3?$CF15s?1Destroy?5@ 0044a8c0     authclientdispath.obj
 0002:000008f4       ??_7CAuthClientDispatch@@6B@ 0044a8f4     authclientdispath.obj
 0002:00000910       ??_C@_0BP@KPIAPNHB@CAuthClientDispatch?3?3Connected?$AA@ 0044a910     authclientdispath.obj
 0002:00000930       ??_C@_0DF@IMMBOEKJ@SS?30x?$CFp?1DP?30x?$CFp?1IP?3?$CF15s?1Connecte@ 0044a930     authclientdispath.obj
 0002:00000968       ??_C@_0GH@HPBMMEBH@UID?3?$CFu?1CurrentTime?3?$CFu?1LastPingTi@ 0044a968     authclientdispath.obj
 0002:000009d0       ??_C@_0BK@LAOEOCIG@Get?5agent?5session?5failed?4?$AA@ 0044a9d0     authclientdispath.obj
 0002:000009ec       ??_C@_0CI@LPACFKFI@SS?30x?$CFp?1DP?30x?$CFp?1Buffer?5allocate?5@ 0044a9ec     authclientdispath.obj
 0002:00000a14       ??_C@_0CF@BACPCBEJ@CAuthClientDispatch?3?3ParseServer@ 0044aa14     authclientdispath.obj
 0002:00000a3c       ??_C@_0CE@CGGJIKND@CAuthClientDispatch?3?3ParseUserLo@ 0044aa3c     authclientdispath.obj
 0002:00000a60       ??_C@_0CH@GCGILAHA@Session?30x?$CFp?5Buffer?5allocation?5f@ 0044aa60     authclientdispath.obj
 0002:00000a88       ??_C@_0CF@JFJNKBDG@CAuthClientDispatch?3?3ParseCharSe@ 0044aa88     authclientdispath.obj
 0002:00000ab0       ??_C@_0CL@FDKAHJMG@Authorize?5user?5limit?5failed?5?9?5Ac@ 0044aab0     authclientdispath.obj
 0002:00000adc       ??_C@_0BN@CAAFDIPN@Authorize?5info?5create?5failed?$AA@ 0044aadc     authclientdispath.obj
 0002:00000afc       ??_C@_0BF@DAAHNEDL@Blocked?5Account?5?3?5?$CFs?$AA@ 0044aafc     authclientdispath.obj
 0002:00000b14       ??_C@_0CM@ODGHEJGK@Version?5error?5?$FL?$CFs?$FN?5?3?5Client?3?$CF3d?0@ 0044ab14     authclientdispath.obj
 0002:00000b40       ??_C@_0DE@LPIPDAID@Checksum?5failed?5?$FL?$CFs?$FN?5?3?5Client?30x@ 0044ab40     authclientdispath.obj
 0002:00000b74       ??_C@_0CL@DHLLJAL@CAuthClientDispatch?3?3ParseJapanA@ 0044ab74     authclientdispath.obj
 0002:00000ba0       ??_C@_0FE@OBNMOMIB@UID?3?$CF10u?1CnFlag?30x?$CF04x?1Disconnec@ 0044aba0     authclientdispath.obj
 0002:00000bf4       ??_C@_04FBIDBDME@?E?$LL?E?p?$AA@ 0044abf4     authclientdispath.obj
 0002:00000bfc       ??_C@_0CA@MGJANALH@CAuthClientDispatch?3?3UserLogout?$AA@ 0044abfc     authclientdispath.obj
 0002:00000c20       ??_C@_0EB@LLNKDKKL@this?30x?$CFp?1UIDDB_DP?30x?$CFp?1Unknown?5@ 0044ac20     authclientdispath.obj
 0002:00000c64       ??_C@_0BO@PKAHBOHO@CAuthClientDispatch?3?3UserMove?$AA@ 0044ac64     authclientdispath.obj
 0002:00000c84       ??_C@_0CO@ECDEAHIM@Can?8t?5over?5authorize?5limit?4?5Acco@ 0044ac84     authclientdispath.obj
 0002:00000cb4       ??_C@_0CC@FHKKCPFA@User?5authorize?5info?5create?5faile@ 0044acb4     authclientdispath.obj
 0002:00000cd8       ??_C@_0BC@BEHAKOAA@Blocked?5user?5?3?5?$CFs?$AA@ 0044acd8     authclientdispath.obj
 0002:00000cec       ??_C@_0CI@KNBJHIOL@Can?8t?5recognize?5account?5name?5?3?5?$FL@ 0044acec     authclientdispath.obj
 0002:00000d14       ??_C@_0DD@IBHBFKKC@Checksum?5error?5?$FL?$CFs?$FN?5?3?5Client?30x?$CF@ 0044ad14     authclientdispath.obj
 0002:00000d48       ??_C@_0CG@HHCHKGCH@CAuthClientDispatch?3?3ParseAuthAc@ 0044ad48     authclientdispath.obj
 0002:00000d70       ??_C@_0CF@EDLPIPFI@Session?30x?$CFp?5Buffer?5allocate?5fai@ 0044ad70     authclientdispath.obj
 0002:00000d98       ??_C@_0CA@KHMGLOPM@UID?30x?$CF08X?5?$MA?$NP?$LI?x?$LF?H?5?D?$LD?$LI?$KP?E?M?5?$LF?$KF?$MA?L?E?M?$AA@ 0044ad98     authclientdispath.obj
 0002:00000db8       ??_C@_0BP@KCKAPJIF@UID?30x?$CF08X?5?$LP?e?$LM?$LD?5?D?$LD?$LI?$KP?E?M?5?$MA?L?$LI?$KH?5?$CFs?$AA@ 0044adb8     authclientdispath.obj
 0002:00000dd8       ??_C@_0CF@CEFCGMBI@CAuthClientDispatch?3?3ParseCharCr@ 0044add8     authclientdispath.obj
 0002:00000e00       ??_C@_0CB@FODDNJM@UID?30x?$CF08X?5?$MA?$NP?$LI?x?$LF?H?5?D?$LD?$LI?$KP?E?M?5?$MA?L?$LI?$KH?5?$CFs@ 0044ae00     authclientdispath.obj
 0002:00000e24       ??_C@_0CF@HNFEJFJD@CAuthClientDispatch?3?3ParseCharDe@ 0044ae24     authclientdispath.obj
 0002:00000e4c       ??_C@_0L@KKCECKBM@SS?30x?$CFp?1?$CFs?$AA@ 0044ae4c     authclientdispath.obj
 0002:00000e58       ??_C@_0BH@PDJDLFOA@Get?5requestkey?5failed?4?$AA@ 0044ae58     authclientdispath.obj
 0002:00000e70       ??_C@_0BC@GKJBMEFI@Get?5agent?5failed?4?$AA@ 0044ae70     authclientdispath.obj
 0002:00000e84       ??_C@_0CC@MPDOKPKA@CAuthClientDispatch?3?3Disconnecte@ 0044ae84     authclientdispath.obj
 0002:00000ea8       ??_C@_0DI@MCBPIBLE@SS?30x?$CFp?1DP?30x?$CFp?1IP?3?$CF15s?1Disconne@ 0044aea8     authclientdispath.obj
 0002:00000ee0       ??_C@_0CK@JNMHJHOG@?F?P?E?$LG?5?G?l?$LE?u?$MA?G?5?F?P?E?$LG?5?D?$LP?$LI?G?$LF?e?$LA?$KB?5?$MA?$NP?$LI?x?$LF?G@ 0044aee0     authclientdispath.obj
 0002:00000f0c       ??_7CThread@@6B@           0044af0c     authorizethread.obj
 0002:00000f18       ??_7CAuthorizeThread@@6B@  0044af18     authorizethread.obj
 0002:00000f28       ??_C@_0BO@EPDLIKJB@DB?5Error?5?3?5?$CFs?5?$CILoginAuthMyth?$CJ?$AA@ 0044af28     authorizethread.obj
 0002:00000f48       ??_C@_0CF@HBGEOCJ@CYouxilandAuthorizeThread?3?3Autho@ 0044af48     authorizethread.obj
 0002:00000f70       ??_C@_0HD@HCAKGHEA@D?3?2Work?2RYL?2Source?2v?4538?$FN?5?G?X?$LP?$NM?5?$CI@ 0044af70     authorizethread.obj
 0002:00000fe4       ??_C@_0DE@DOIJCGAO@?$MA?N?A?u?5?$LP?$MA?$LH?y?4?5Account?3?$CFs?5Password?3?$CF@ 0044afe4     authorizethread.obj
 0002:00001018       ??_C@_0CE@NODJHBPN@TID?30x?$CFp?1Authorize?5thread?5stop?5n@ 0044b018     authorizethread.obj
 0002:0000103c       ??_C@_0BG@GMGMAPCC@CAuthorizeThread?3?3Run?$AA@ 0044b03c     authorizethread.obj
 0002:00001058       ??_C@_0EJ@PPIJPMF@SS?30x?$CFp?1DP?30x?$CFp?1Too?5overhead?5in?5@ 0044b058     authorizethread.obj
 0002:000010a4       ??_7CHangameAuthorizeThread@@6B@ 0044b0a4     authorizethread.obj
 0002:000010b4       ??_7CYouxilandAuthorizeThread@@6B@ 0044b0b4     authorizethread.obj
 0002:000010c4       ??_7CJapanAuthorizeThread@@6B@ 0044b0c4     authorizethread.obj
 0002:000010d4       ??_C@_0DA@DJGIEBCA@?$LP?n?$LP?$LF?$MA?Z?$LA?$KB?5?D?$LD?$LI?$KP?E?M?5?F?m?A?$PN?A?$NP?$LP?$KB?5?$LH?N?$LB?W?$MA?N?5@ 0044b0d4     authorizethread.obj
 0002:00001104       ??_C@_0BH@NEDFEAAC@?$LK?m?$LH?$LA?$LF?H?5?$LA?h?A?$KE?4?5?$LA?h?A?$KE?5?3?5?$CFs?$AA@ 0044b104     authorizethread.obj
 0002:0000111c       ??_C@_0CP@HDPCKJNI@Auth?5Error?5?3?5IP?3?$CFs?1ID?3?$CFs?1Errcode@ 0044b11c     authorizethread.obj
 0002:0000114c       ??_C@_0BD@MIPFABEN@LoginBattleAuthHan?$AA@ 0044b14c     authorizethread.obj
 0002:00001160       ??_C@_0N@MDJLENCL@LoginAuthHan?$AA@ 0044b160     authorizethread.obj
 0002:00001170       ??_C@_0BN@DFEPDCN@DB?5Error?5?3?5?$CFs?5?$CILoginAuthHan?$CJ?$AA@ 0044b170     authorizethread.obj
 0002:00001190       ??_C@_0CD@BFFCIMPG@CHangameAuthorizeThread?3?3Authori@ 0044b190     authorizethread.obj
 0002:000011b4       ??_C@_0BD@GEMJBHGG@DB?5Error?5?3?5?$CFs?5?$CI?$CFs?$CJ?$AA@ 0044b1b4     authorizethread.obj
 0002:000011c8       ??_C@_0BE@GOACJJIB@RegBattleRylGameHan?$AA@ 0044b1c8     authorizethread.obj
 0002:000011dc       ??_C@_0O@DAAECCDF@RegRylGameHan?$AA@ 0044b1dc     authorizethread.obj
 0002:000011ec       ??_C@_01NANMIPIL@N?$AA@    0044b1ec     authorizethread.obj
 0002:000011f0       ??_C@_01NFFPALBN@Y?$AA@    0044b1f0     authorizethread.obj
 0002:000011f4       ??_C@_0CB@PGMJFFCC@CSyncronizedObjectQueue?3?3dequeue@ 0044b1f4     authorizeuser.obj
 0002:00001218       ??_C@_0HB@PHBDJFJC@D?3?2Work?2RYL?2Source?2v?4538?$FN?5?G?X?$LP?$NM?5?$CI@ 0044b218     authorizeuser.obj
 0002:0000128c       ??_C@_0CI@FBDIHGNG@Err?3?$CFd?1Error?5from?5WaitForMultipl@ 0044b28c     authorizeuser.obj
 0002:000012b4       ??_C@_0BB@MOGOBHAF@list?$DMT?$DO?5too?5long?$AA@ 0044b2b4     authorizeuser.obj
 0002:000012c8       ??_C@_0DA@IDJFCCIK@Used?5master?5password?5?3?5UserName?$CI@ 0044b2c8     masterpassword.obj
 0002:000012f8       ??_C@_0CF@KGPOGOGJ@CMasterPassword?3?3CheckMasterPass@ 0044b2f8     masterpassword.obj
 0002:00001320       ??_C@_0HC@ILNFDMBE@D?3?2Work?2RYL?2Source?2v?4538?$FN?5?G?X?$LP?$NM?5?$CI@ 0044b320     masterpassword.obj
 0002:00001398       ??_C@_0FB@FLCNFMGE@Can?8t?5apply?5master?5password?5?3?5Un@ 0044b398     masterpassword.obj
 0002:000013ec       ??_C@_0BA@NEGLFBDA@Unknown?5address?$AA@ 0044b3ec     masterpassword.obj
 0002:000013fc       ??_C@_0BD@OLBABOEK@vector?$DMT?$DO?5too?5long?$AA@ 0044b3fc     masterpassword.obj
 0002:00001410       ??_C@_0L@INCJAJMA@ALLOWED_IP?$AA@ 0044b410     masterpassword.obj
 0002:0000141c       ??_C@_0BA@KIAPELOE@MASTER_PASSWORD?$AA@ 0044b41c     masterpassword.obj
 0002:0000142c       ??_C@_02CBLDBPFN@?1?1?$AA@ 0044b42c     masterpassword.obj
 0002:00001430       ??_C@_05NFBBJDEM@?5?$DN?7?6?$AN?$AA@ 0044b430     masterpassword.obj
 0002:00001438       ??_C@_02BMJICGCB@rt?$AA@   0044b438     masterpassword.obj
 0002:0000143c       ??_7CDispatchFactory@@6B@  0044b43c     rylauthserver.obj
 0002:00001448       ??_7CRylAuthServerProcess@@6B@ 0044b448     rylauthserver.obj
 0002:00001458       ??_7CRylAuthServer@@6B@    0044b458     rylauthserver.obj
 0002:00001460       ??_C@_0CC@GHDGHHHB@Accept?5Pening?5?3?5?$CFd?5?1?5Session?5?3?5?$CF@ 0044b460     rylauthserver.obj
 0002:00001484       ??_C@_0O@IFKIEMFK@RylAuthServer?$AA@ 0044b484     rylauthserver.obj
 0002:00001494       ??_C@_0BM@EPJMLKCP@ServerSetup?5reload?5success?4?$AA@ 0044b494     rylauthserver.obj
 0002:000014b0       ??_C@_0BM@GEKILICG@CRylAuthServer?3?3ReloadSetup?$AA@ 0044b4b0     rylauthserver.obj
 0002:000014d0       ??_C@_0HB@BBMJNBIA@D?3?2Work?2RYL?2Source?2v?4538?$FN?5?G?X?$LP?$NM?5?$CI@ 0044b4d0     rylauthserver.obj
 0002:00001544       ??_C@_0CB@KCMNIKLD@ServerSetup?5reinitialize?5failed?4@ 0044b544     rylauthserver.obj
 0002:00001568       ??_C@_0BN@IGIGLBM@There?5is?5no?5DBAgent?5Server?$AN?6?$AA@ 0044b568     rylauthserver.obj
 0002:00001588       ??_C@_0CH@MMHMDMNI@?5?5Human?3?5?$CF4d?0?5Akhan?3?5?$CF4d?0?5Total?3@ 0044b588     rylauthserver.obj
 0002:000015b0       ??_C@_0DO@PMPNOEOE@Client?5Version?5?3?5?$CFd?0?5CheckSum?5?3?5@ 0044b5b0     rylauthserver.obj
 0002:000015f0       ??_C@_0BJ@BDHGLLIP@?$EA?5Limit?5Players?5?3?5?$CFd?$AN?6?$CFs?$AA@ 0044b5f0     rylauthserver.obj
 0002:0000160c       ??_C@_0BE@OPJMHNEL@?$EA?5Client?5Closed?$AN?6?$AN?6?$AA@ 0044b60c     rylauthserver.obj
 0002:00001620       ??_C@_0BC@NODEFHJG@?$EA?5Client?5Open?$AN?6?$AN?6?$AA@ 0044b620     rylauthserver.obj
 0002:00001634       ??_7?$CPoolDispatchFactory@VCAuthClientDispatch@@@@6B@ 0044b634     rylauthserver.obj
 0002:00001640       ??_7?$CPoolDispatchFactory@VCAuthAgentDispatch@@@@6B@ 0044b640     rylauthserver.obj
 0002:0000164c       ??_C@_0BD@CBOPHNJN@AddListener?5failed?$AA@ 0044b64c     rylauthserver.obj
 0002:00001660       ??_C@_0CJ@JEHLMGFK@CRylAuthServer?3?3InitializeClient@ 0044b660     rylauthserver.obj
 0002:0000168c       ??_C@_0BA@CIAMBDJN@IOCPNet?5is?5null?$AA@ 0044b68c     rylauthserver.obj
 0002:0000169c       ??_C@_0CL@LFPGAEEB@this?30x?$CFp?1Cannot?5connect?5to?5DBAg@ 0044b69c     rylauthserver.obj
 0002:000016c8       ??_C@_0BK@HNAJKOKG@this?30x?$CFp?1IOCPNet?5is?5null?$AA@ 0044b6c8     rylauthserver.obj
 0002:000016e4       ??_C@_0CB@DPDNECFN@CRylAuthServer?3?3ConnectToDBAgent@ 0044b6e4     rylauthserver.obj
 0002:00001708       ??_C@_0CO@ELMEBOGJ@this?30x?$CFp?1Already?5connected?5to?5D@ 0044b708     rylauthserver.obj
 0002:00001738       ??_C@_0M@EKIFFKJN@startserver?$AA@ 0044b738     rylauthserver.obj
 0002:00001744       ??_C@_0CI@MHBCJOH@CRylAuthServer?3?3ApplicationSpeci@ 0044b744     rylauthserver.obj
 0002:0000176c       ??_C@_0N@BPFMMBNO@this?30x?$CFp?1?$CFs?$AA@ 0044b76c     rylauthserver.obj
 0002:00001780       ??_C@_0EE@PIECLFAG@AuthServer?5initialize?5failed?5?9?5A@ 0044b780     rylauthserver.obj
 0002:000017c4       ??_C@_0DJ@FJFDPAIA@AuthServer?5initialize?5failed?5?9?5A@ 0044b7c4     rylauthserver.obj
 0002:00001800       ??_C@_0DP@PADDFMIC@AuthServer?5initialize?5failed?5?9?5S@ 0044b800     rylauthserver.obj
 0002:00001840       ??_C@_0DK@CCEMEGPK@AuthServer?5initialize?5failed?5?9?5S@ 0044b840     rylauthserver.obj
 0002:0000187c       ??_C@_0DH@IFLCKDIA@AuthServer?5initialize?5failed?5?9?5I@ 0044b87c     rylauthserver.obj
 0002:000018b4       ??_C@_0DD@BNIPDPPM@AuthServer?5initialize?5failed?5?9?5G@ 0044b8b4     rylauthserver.obj
 0002:000018e8       ??_C@_0DL@IOHLBOB@AuthServer?5initialize?5failed?5?9?5M@ 0044b8e8     rylauthserver.obj
 0002:00001924       ??_C@_0BP@DIKCFNAP@?4?1Script?1Server?1masterpass?4txt?$AA@ 0044b924     rylauthserver.obj
 0002:00001944       ??_C@_0DC@FDNPJPDL@AuthServer?5initialize?5failed?5?9?5F@ 0044b944     rylauthserver.obj
 0002:00001978       ??_C@_0DH@OAIFDJKE@AuthServer?5initialize?5failed?5?9?5S@ 0044b978     rylauthserver.obj
 0002:000019b0       ??_C@_0DM@NJCEJJMD@AuthServer?5initialize?5failed?5?9?5C@ 0044b9b0     rylauthserver.obj
 0002:000019ec       ??_7CCMDStartServer@@6B@   0044b9ec     rylauthservercommands.obj
 0002:000019f8       ??_7CCMDShowStatistics@@6B@ 0044b9f8     rylauthservercommands.obj
 0002:00001a04       ??_7CCMDPrintLog@@6B@      0044ba04     rylauthservercommands.obj
 0002:00001a10       ??_C@_0BI@CBHOLJIE@CCMDPrintLog?3?3DoProcess?$AA@ 0044ba10     rylauthservercommands.obj
 0002:00001a28       ??_C@_0HJ@JOJFOAIJ@D?3?2Work?2RYL?2Source?2v?4538?$FN?5?G?X?$LP?$NM?5?$CI@ 0044ba28     rylauthservercommands.obj
 0002:00001aa4       ??_C@_0L@POJJOIII@Flush?5Log?4?$AA@ 0044baa4     rylauthservercommands.obj
 0002:00001ab0       ??_7CCMDReloadSetup@@6B@   0044bab0     rylauthservercommands.obj
 0002:00001abc       ??_7CCMDFlushLog@@6B@      0044babc     rylauthservercommands.obj
 0002:00001ac8       ??_C@_0BI@LEBEFAMD@CCMDFlushLog?3?3DoProcess?$AA@ 0044bac8     rylauthservercommands.obj
 0002:00001ae0       ??_7CCMDMasterPass@@6B@    0044bae0     rylauthservercommands.obj
 0002:00001aec       ??_C@_0BK@KCHJLKML@CCMDMasterPass?3?3DoProcess?$AA@ 0044baec     rylauthservercommands.obj
 0002:00001b08       ??_C@_0CI@LLPPDOMC@this?30x?$CFp?1Master?5password?5reload@ 0044bb08     rylauthservercommands.obj
 0002:00001b30       ??_7CCMDStatClear@@6B@     0044bb30     rylauthservercommands.obj
 0002:00001b3c       ??_7CCMDStatLog@@6B@       0044bb3c     rylauthservercommands.obj
 0002:00001b48       ??_C@_0CC@CDJMNDHD@CRylAuthServer?3?3InitializeComman@ 0044bb48     rylauthservercommands.obj
 0002:00001b6c       ??_C@_0CA@HNKOLHOA@Command?5create?5failed?5?9?5statlog?$AA@ 0044bb6c     rylauthservercommands.obj
 0002:00001b8c       ??_C@_07HHBIOBOL@statlog?$AA@ 0044bb8c     rylauthservercommands.obj
 0002:00001b94       ??_C@_0CC@EDJIBCIA@Command?5create?5failed?5?9?5statclea@ 0044bb94     rylauthservercommands.obj
 0002:00001bb8       ??_C@_09CCGEDFDM@statclear?$AA@ 0044bbb8     rylauthservercommands.obj
 0002:00001bc4       ??_C@_0CD@OCJLCPLK@Command?5create?5failed?5?9?5reloadpa@ 0044bbc4     rylauthservercommands.obj
 0002:00001be8       ??_C@_0L@CACNCMDK@reloadpass?$AA@ 0044bbe8     rylauthservercommands.obj
 0002:00001bf4       ??_C@_0BO@PFCBPMGA@Command?5create?5failed?5?9?5flush?$AA@ 0044bbf4     rylauthservercommands.obj
 0002:00001c14       ??_C@_05GLCAEPFP@flush?$AA@ 0044bc14     rylauthservercommands.obj
 0002:00001c1c       ??_C@_0CE@OOCHCICO@Command?5create?5failed?5?9?5reloadse@ 0044bc1c     rylauthservercommands.obj
 0002:00001c40       ??_C@_0M@DFNBNAN@reloadsetup?$AA@ 0044bc40     rylauthservercommands.obj
 0002:00001c4c       ??_C@_0BM@FADJNIHN@Command?5create?5failed?5?9?5log?$AA@ 0044bc4c     rylauthservercommands.obj
 0002:00001c68       ??_C@_03MGHMBJCF@log?$AA@  0044bc68     rylauthservercommands.obj
 0002:00001c6c       ??_C@_0BN@EMKPDLMJ@Command?5create?5failed?5?9?5pool?$AA@ 0044bc6c     rylauthservercommands.obj
 0002:00001c8c       ??_C@_04CJIJKHMO@pool?$AA@ 0044bc8c     rylauthservercommands.obj
 0002:00001c94       ??_C@_0CE@KHPPGPLO@Command?5create?5failed?5?9?5startser@ 0044bc94     rylauthservercommands.obj
 0002:00001cb8       ??_C@_0BK@NBNBDIPB@Userdata?5flush?5completed?4?$AA@ 0044bcb8     rylauthservermain.obj
 0002:00001cd4       ??_C@_0BC@OGJLJPN@ExceptionUserFunc?$AA@ 0044bcd4     rylauthservermain.obj
 0002:00001ce8       ??_C@_0HF@NBGHHNAN@D?3?2Work?2RYL?2Source?2v?4538?$FN?5?G?X?$LP?$NM?5?$CI@ 0044bce8     rylauthservermain.obj
 0002:00001d60       ??_C@_09DBBHFMGJ@Flush?5log?$AA@ 0044bd60     rylauthservermain.obj
 0002:00001d6c       ??_C@_0M@JFKBGLCF@Auth?5Server?$AA@ 0044bd6c     rylauthservermain.obj
 0002:00001d78       ??_C@_07HGGPAHEN@WinMain?$AA@ 0044bd78     rylauthservermain.obj
 0002:00001d80       ??_C@_0DO@JIGHGMEL@AuthServer?5already?5operating?5now@ 0044bd80     rylauthservermain.obj
 0002:00001dc0       ??_7CMsgProc@@6B@          0044bdc0     rylauthserverwindow.obj
 0002:00001dc8       ??_7CProcessRYLAUTH_AUTOSTART@@6B@ 0044bdc8     rylauthserverwindow.obj
 0002:00001dd0       ??_C@_0CI@OJMOEBDE@CProcessRYLAUTH_AUTOSTART?3?3opera@ 0044bdd0     rylauthserverwindow.obj
 0002:00001df8       ??_C@_0HH@PFEPKJCM@D?3?2Work?2RYL?2Source?2v?4538?$FN?5?G?X?$LP?$NM?5?$CI@ 0044bdf8     rylauthserverwindow.obj
 0002:00001e70       ??_C@_0BC@CBOJMGIC@AutoStart?5Started?$AA@ 0044be70     rylauthserverwindow.obj
 0002:00001e84       ??_7CProcessAUTH_CONNECTTOAGENT@@6B@ 0044be84     rylauthserverwindow.obj
 0002:00001e8c       ??_C@_0CK@EMLOOEHG@CProcessAUTH_CONNECTTOAGENT?3?3ope@ 0044be8c     rylauthserverwindow.obj
 0002:00001eb8       ??_C@_0CG@OCLIFEP@?$LA?$PM?$LI?$KO?E?x?$MA?G?5?$LP?d?C?$LL?$MA?$LI?$LH?N?5DBAgent?$LM?$KN?$LJ?v?$LH?N?5@ 0044beb8     rylauthserverwindow.obj
 0002:00001ee0       ??_7CProcessRYLAUTH_QUIT@@6B@ 0044bee0     rylauthserverwindow.obj
 0002:00001ee8       ??_7CProcessCOMMAND@@6B@   0044bee8     rylauthserverwindow.obj
 0002:00001ef0       ??_C@_0BO@DJFPDPNG@CProcessCOMMAND?3?3operator?$GA?$CI?$CJ?8?$AA@ 0044bef0     rylauthserverwindow.obj
 0002:00001f10       ??_C@_0CC@MPCLMNGM@Terminate?5AuthServer?5System?5Tray@ 0044bf10     rylauthserverwindow.obj
 0002:00001f34       ??_7CPacketDispatch@@6B@   0044bf34     rylgamelibrary:rylserverdispatch.obj
 0002:00001f48       ??_7CRylServerDispatch@@6B@ 0044bf48     rylgamelibrary:rylserverdispatch.obj
 0002:00001f64       ??_C@_0CD@HJBDBNNC@CRylServerDispatch?3?3LogErrorPack@ 0044bf64     rylgamelibrary:rylserverdispatch.obj
 0002:00001f88       ??_C@_0IJ@JFBONBOK@D?3?2Work?2RYL?2Source?2v?4538?$FN?5?G?X?$LP?$NM?5?$CI@ 0044bf88     rylgamelibrary:rylserverdispatch.obj
 0002:00002014       ??_C@_0CJ@FJKCIJPG@SP?30x?$CFp?1DP?30x?$CFp?1IP?3?$CF15s?1PktCmd?30@ 0044c014     rylgamelibrary:rylserverdispatch.obj
 0002:00002040       ??_C@_0BI@LKMKHKFB@Invalid?5packet?5startbit?$AA@ 0044c040     rylgamelibrary:rylserverdispatch.obj
 0002:00002058       ??_C@_0BN@GGDFEHIB@Allocate?5packetbuffer?5failed?$AA@ 0044c058     rylgamelibrary:rylserverdispatch.obj
 0002:00002078       ??_C@_0BJ@DMGJDKMK@Decompress?5packet?5failed?$AA@ 0044c078     rylgamelibrary:rylserverdispatch.obj
 0002:00002094       ??_C@_0BG@MCKJHDPO@Unknown?5error?5occured?$AA@ 0044c094     rylgamelibrary:rylserverdispatch.obj
 0002:000020ac       ??_C@_0M@HNDPKJJF@0x?$CF02x?3?$CF5d?1?$AA@ 0044c0ac     rylgamelibrary:rylserverdispatch.obj
 0002:000020b8       ??_C@_0DA@MDFDMJF@Processed?3?$CFd?1Remain?3?$CFd?1Remain?5pa@ 0044c0b8     rylgamelibrary:rylserverdispatch.obj
 0002:000020e8       ??_C@_03IJKDIPKN@WRN?$AA@  0044c0e8     rylgamelibrary:serverlog.obj
 0002:000020ec       ??_C@_03GOLGPOF@DBG?$AA@   0044c0ec     rylgamelibrary:serverlog.obj
 0002:000020f0       ??_C@_03JFMEENOE@ERR?$AA@  0044c0f0     rylgamelibrary:serverlog.obj
 0002:000020f4       ??_C@_03PJNPPAFC@SER?$AA@  0044c0f4     rylgamelibrary:serverlog.obj
 0002:000020f8       ??_C@_03GCELDIPC@DET?$AA@  0044c0f8     rylgamelibrary:serverlog.obj
 0002:000020fc       ??_C@_03OEIAHPBN@INF?$AA@  0044c0fc     rylgamelibrary:serverlog.obj
 0002:00002100       ??_C@_03IJAEALJI@RUL?$AA@  0044c100     rylgamelibrary:serverlog.obj
 0002:00002104       ??_C@_03FGDLPKMG@NOR?$AA@  0044c104     rylgamelibrary:serverlog.obj
 0002:00002108       ??_7CServerLog@@6B@        0044c108     rylgamelibrary:serverlog.obj
 0002:0000210c       ??_C@_0O@EHJCJHP@?$CFs?1?$CFs?$CF04d?4log?$AA@ 0044c10c     rylgamelibrary:serverlog.obj
 0002:0000211c       ??_C@_0CB@MHIBELEH@?$CFs?$CF04d?9?$CF02d?9?$CF02d?5?$CF02d?0?$CF02d?0?$CF02d?9@ 0044c11c     rylgamelibrary:serverlog.obj
 0002:00002140       ??_C@_05GMHOPMGA@?$CFs?$FN?$AN?6?$AA@ 0044c140     rylgamelibrary:serverlog.obj
 0002:00002148       ??_C@_08LHNPNMKM@?$FLTy?9?$CFs?$FN?$FL?$AA@ 0044c148     rylgamelibrary:serverlog.obj
 0002:00002154       ??_C@_0CO@GNLJODDP@?$FLTy?9?$CFs?$FN?$FLTm?9?$CF04d?9?$CF02d?9?$CF02d?5?$CF02d?3?$CF@ 0044c154     rylgamelibrary:serverlog.obj
 0002:00002184       ??_C@_0BL@GBLEAPDO@?$CFs?$FN?$FLRt?9?$CFs?$FN?$FLFN?9?$CFs?$FN?$FLLN?9?$CFd?$FN?$AN?6?$AA@ 0044c184     rylgamelibrary:serverlog.obj
 0002:000021a0       ??_C@_0BB@CCPPGGOJ@?$LH?N?$LB?W?$LI?$KG?5?$LD?$KB?$LD?$MA?$LE?O?$LE?Y?4?$AA@ 0044c1a0     rylgamelibrary:serverlog.obj
 0002:000021b4       ??_C@_08PCOKJLAJ@GuildLog?$AA@ 0044c1b4     rylgamelibrary:serverlog.obj
 0002:000021c0       ??_C@_0L@NAGALIAM@SessionLog?$AA@ 0044c1c0     rylgamelibrary:serverlog.obj
 0002:000021cc       ??_C@_0BE@JONHPENG@map?1set?$DMT?$DO?5too?5long?$AA@ 0044c1cc     rylgamelibrary:serverrequest.obj
 0002:000021e0       ??_C@_0BM@PAPJHAGI@invalid?5map?1set?$DMT?$DO?5iterator?$AA@ 0044c1e0     rylgamelibrary:serverrequest.obj
 0002:000021fc       ??_C@_0BL@BFEIIEIK@CServerRequest?3?3AddRequest?$AA@ 0044c1fc     rylgamelibrary:serverrequest.obj
 0002:00002218       ??_C@_0IA@FALIEKAC@D?3?2Work?2RYL?2Source?2v?4538?$FN?5?G?X?$LP?$NM?5?$CI@ 0044c218     rylgamelibrary:serverrequest.obj
 0002:00002298       ??_C@_0DM@LLHPDMFF@SS?30x?$CFp?1DP?30x?$CFp?1IP?3?$CF15s?1Request?3@ 0044c298     rylgamelibrary:serverrequest.obj
 0002:000022d4       ??_C@_0BO@NNOKFBLO@CServerRequest?3?3RemoveRequest?$AA@ 0044c2d4     rylgamelibrary:serverrequest.obj
 0002:000022f8       ??_C@_0EN@HOINCMFG@SS?30x?$CFp?1DP?30x?$CFp?1IP?3?$CF15s?1Request?3@ 0044c2f8     rylgamelibrary:serverrequest.obj
 0002:00002348       ??_C@_0CF@OKAEIFLM@CServerRequest?3?3RemoveTimeoutReq@ 0044c348     rylgamelibrary:serverrequest.obj
 0002:00002370       ??_C@_0EK@DOJKHOOA@SS?30x?$CFp?1DP?30x?$CFp?1IP?3?$CF15s?1Request?3@ 0044c370     rylgamelibrary:serverrequest.obj
 0002:000023bc       ??_C@_0BL@HDPMHHAL@CServerRequest?3?3PopRequest?$AA@ 0044c3bc     rylgamelibrary:serverrequest.obj
 0002:000023d8       ??_C@_0EO@EFPNKIKK@SS?30x?$CFp?1DP?30x?$CFp?1IP?3?$CF15s?1Request?3@ 0044c3d8     rylgamelibrary:serverrequest.obj
 0002:00002438       ??_C@_02MDDDDAID@0x?$AA@   0044c438     rylgamelibrary:serversetup.obj
 0002:0000243c       ??_7CSocketFactory@@6B@    0044c43c     rylgamelibrary:serversetup.obj
 0002:0000244c       ??_C@_0BO@FFINLNAL@CServerSetup?3?3InitLoginServer?$AA@ 0044c44c     rylgamelibrary:serversetup.obj
 0002:00002470       ??_C@_0IA@FBBBMENB@D?3?2Work?2RYL?2Source?2v?4538?$FN?5?G?X?$LP?$NM?5?$CI@ 0044c470     rylgamelibrary:serversetup.obj
 0002:000024f0       ??_C@_0BF@LBPODEFM@?F?P?D?$KB?5?A?V?$LM?R?5?$LO?r?$LB?b?5?$LN?G?F?P?4?$AA@ 0044c4f0     rylgamelibrary:serversetup.obj
 0002:00002508       ??_C@_09BLJKKJCG@PatchAddr?$AA@ 0044c508     rylgamelibrary:serversetup.obj
 0002:00002514       ??_C@_0BK@CKECKGFA@?E?$KM?$LG?s?$MA?L?$LO?p?F?$KO?5?A?$KG?G?Q?5?$LJ?v?A?$KP?5?$LN?G?F?P?$AA@ 0044c514     rylgamelibrary:serversetup.obj
 0002:00002530       ??_C@_08JKEPNHKL@LimitVer?$AA@ 0044c530     rylgamelibrary:serversetup.obj
 0002:0000253c       ??_C@_0BA@HFOGMKFM@?H?$KF?$MA?Z?5?$LI?p?$LF?e?5?$LN?G?F?P?4?$AA@ 0044c53c     rylgamelibrary:serversetup.obj
 0002:0000254c       ??_C@_05OPHNIDEE@Alone?$AA@ 0044c54c     rylgamelibrary:serversetup.obj
 0002:00002554       ??_C@_0N@CFCNBLML@?G?N?C?$LM?E?$KJ?5?$LN?G?F?P?4?$AA@ 0044c554     rylgamelibrary:serversetup.obj
 0002:00002564       ??_C@_04CPBFGEOK@Ping?$AA@ 0044c564     rylgamelibrary:serversetup.obj
 0002:0000256c       ??_C@_0BO@KHNIAFBH@?$LH?N?$LB?W?$MA?N?5?$LM?$KN?$LJ?v?5?$LO?F?$MA?L?$LF?p?5?$LO?r?$LB?b?5?$LN?G?F?P?4?$AA@ 0044c56c     rylgamelibrary:serversetup.obj
 0002:0000258c       ??_C@_05DHEMANOL@Login?$AA@ 0044c58c     rylgamelibrary:serversetup.obj
 0002:00002594       ??_C@_08BHBELLIH@ServerID?$AA@ 0044c594     rylgamelibrary:serversetup.obj
 0002:000025a0       ??_C@_0BC@NJLKFFAC@SupressCharCreate?$AA@ 0044c5a0     rylgamelibrary:serversetup.obj
 0002:000025b4       ??_C@_0BN@MJLJHDPD@CServerSetup?3?3InitAuthServer?$AA@ 0044c5b4     rylgamelibrary:serversetup.obj
 0002:000025d4       ??_C@_0BN@ODDHOFDH@?$MA?N?A?u?$LM?$KN?$LJ?v?5?$LD?$KK?$MA?L?5?A?$KG?G?Q?5?$MA?P?$LB?b?5?$LN?G?F?P?$AA@ 0044c5d4     rylgamelibrary:serversetup.obj
 0002:000025f4       ??_C@_0P@IIGKFOPF@BattleAgeLimit?$AA@ 0044c5f4     rylgamelibrary:serversetup.obj
 0002:00002604       ??_C@_0CH@IBANHAAC@?$MA?N?A?u?$LM?$KN?$LJ?v?$LA?$KB?5?$LJ?h?F?$LC?$LM?$KN?$LJ?v?$MA?N?A?v?5?$LP?$KJ?$LK?N?5?$MA?P?$LB@ 0044c604     rylgamelibrary:serversetup.obj
 0002:0000262c       ??_C@_0BD@PAFNAPMP@IsAuthBattleServer?$AA@ 0044c62c     rylgamelibrary:serversetup.obj
 0002:00002640       ??_C@_0BJ@GDMBOEFO@?A?$NP?$LA?h?5?$LM?$KN?$LJ?v?5?A?V?$LM?R?5?$MA?P?$LB?b?5?$LN?G?F?P?$AA@ 0044c640     rylgamelibrary:serversetup.obj
 0002:0000265c       ??_C@_09FDOKIOP@AgentAddr?$AA@ 0044c65c     rylgamelibrary:serversetup.obj
 0002:00002668       ??_C@_0BE@OILBKEMB@?$LM?$KN?$LJ?v?5?E?$LI?$MA?T?5?$MA?P?$LB?b?5?$LN?G?F?P?$AA@ 0044c668     rylgamelibrary:serversetup.obj
 0002:0000267c       ??_C@_0L@PODLPHGB@ServerType?$AA@ 0044c67c     rylgamelibrary:serversetup.obj
 0002:00002688       ??_C@_0P@FFCKCGMO@?G?Q?$LB?$NL?C?$LM?E?$KJ?5?$LN?G?F?P?4?$AA@ 0044c688     rylgamelibrary:serversetup.obj
 0002:00002698       ??_C@_08FLJKFJLJ@HanCheck?$AA@ 0044c698     rylgamelibrary:serversetup.obj
 0002:000026a4       ??_C@_0BM@DDMFFPNH@?$MA?N?A?u?5?$LM?$KN?$LJ?v?5?$LO?F?$MA?L?$LF?p?5?$LO?r?$LB?b?5?$LN?G?F?P?4?$AA@ 0044c6a4     rylgamelibrary:serversetup.obj
 0002:000026c0       ??_C@_04POHDAIJG@Auth?$AA@ 0044c6c0     rylgamelibrary:serversetup.obj
 0002:000026c8       ??_C@_0BO@PMAOMNLH@CServerSetup?3?3InitAgentServer?$AA@ 0044c6c8     rylgamelibrary:serversetup.obj
 0002:000026e8       ??_C@_0BM@DHADLFIE@?F?D?F?$KO1?5?E?k?G?UDB?5?$LM?B?$LO?w?5?$MA?P?$LB?b?5?$LN?G?F?P?$AA@ 0044c6e8     rylgamelibrary:serversetup.obj
 0002:00002704       ??_C@_0BD@JDNPCBGA@Part1UnifiedDBPass?$AA@ 0044c704     rylgamelibrary:serversetup.obj
 0002:00002718       ??_C@_0BG@GJHEDOH@Part1UnifiedDBAccount?$AA@ 0044c718     rylgamelibrary:serversetup.obj
 0002:00002730       ??_C@_0BD@EGCPDDCO@Part1UnifiedDBName?$AA@ 0044c730     rylgamelibrary:serversetup.obj
 0002:00002744       ??_C@_0BD@PJPDOLNE@Part1UnifiedDBAddr?$AA@ 0044c744     rylgamelibrary:serversetup.obj
 0002:00002758       ??_C@_0CE@FAENGCCK@?F?D?F?$KO1?5?E?k?G?U?5?A?$NP?$LA?h?5?$LM?$KN?$LJ?v?5?A?V?$LM?R?5?$MA?P?$LB?b?5?$LN@ 0044c758     rylgamelibrary:serversetup.obj
 0002:0000277c       ??_C@_0BG@OHHJPDMP@Part1UnifiedAgentAddr?$AA@ 0044c77c     rylgamelibrary:serversetup.obj
 0002:00002794       ??_C@_0BO@JOPEPMDD@?A?$NP?$LA?h?5?$LM?$KN?$LJ?v?5?$LB?$LJ?$LA?$KB?5?E?$LI?$MA?T?5?$MA?P?$LB?b?5?$LN?G?F?P?$AA@ 0044c794     rylgamelibrary:serversetup.obj
 0002:000027b4       ??_C@_0BA@JBGFEDHO@AgentNationType?$AA@ 0044c7b4     rylgamelibrary:serversetup.obj
 0002:000027c4       ??_C@_0BJ@GBIIDLAL@?A?$NP?$LA?h?5?$LM?$KN?$LJ?v?5?E?$LI?$MA?T?5?$MA?P?$LB?b?5?$LN?G?F?P?$AA@ 0044c7c4     rylgamelibrary:serversetup.obj
 0002:000027e0       ??_C@_0BA@PLAJKNGL@AgentServerType?$AA@ 0044c7e0     rylgamelibrary:serversetup.obj
 0002:000027f0       ??_C@_0CI@OCFOKPFD@?A?$NP?$LA?h?5?$LM?$KN?$LJ?v?$LA?$KB?5?$LJ?h?F?$LC?$LM?$KN?$LJ?v?$MA?N?A?v?5?$LP?$KJ?$LK?N?5?$MA?P@ 0044c7f0     rylgamelibrary:serversetup.obj
 0002:00002818       ??_C@_0BE@NGLMDNHK@IsAgentBattleServer?$AA@ 0044c818     rylgamelibrary:serversetup.obj
 0002:0000282c       ??_C@_0BH@IOGGICOH@?$LA?x?$LM?$LK?5?$LD?$KB?5?$LN?C?$LA?$KD?5?$MA?P?$LB?b?5?$LN?G?F?P?$AA@ 0044c82c     rylgamelibrary:serversetup.obj
 0002:00002844       ??_C@_0N@IOLPJPJD@EndSiegeTime?$AA@ 0044c844     rylgamelibrary:serversetup.obj
 0002:00002854       ??_C@_0BJ@EJBPCCN@?$LA?x?$LM?$LK?5?$LN?C?$MA?$NL?5?$LN?C?$LA?$KD?5?$MA?P?$LB?b?5?$LN?G?F?P?$AA@ 0044c854     rylgamelibrary:serversetup.obj
 0002:00002870       ??_C@_0P@OOBMCNDG@StartSiegeTime?$AA@ 0044c870     rylgamelibrary:serversetup.obj
 0002:00002880       ??_C@_0BI@GIFPHBBE@UID?5?$LM?$KN?$LJ?v?5?A?V?$LM?R?5?$MA?P?$LB?b?5?$LN?G?F?P?$AA@ 0044c880     rylgamelibrary:serversetup.obj
 0002:00002898       ??_C@_07EBEBMMMB@UIDAddr?$AA@ 0044c898     rylgamelibrary:serversetup.obj
 0002:000028a0       ??_C@_0BL@LPMIJJAL@?$LH?N?$LB?W?$MA?N?5?$LM?$KN?$LJ?v?5?A?V?$LM?R?5?$MA?P?$LB?b?5?$LN?G?F?P?$AA@ 0044c8a0     rylgamelibrary:serversetup.obj
 0002:000028bc       ??_C@_09GONHJJEJ@LoginAddr?$AA@ 0044c8bc     rylgamelibrary:serversetup.obj
 0002:000028c8       ??_C@_0BB@EJPMNOHC@?C?$LM?E?$KJ?$LM?$LG?5?$LO?r?$LB?b?5?$LN?G?F?P?$AA@ 0044c8c8     rylgamelibrary:serversetup.obj
 0002:000028dc       ??_C@_08BPDKCIGK@CheckSum?$AA@ 0044c8dc     rylgamelibrary:serversetup.obj
 0002:000028e8       ??_C@_0CC@DHKOBKAP@?$LJ?h?F?$LC?$LB?W?$LG?s?$LP?n?$LF?e?5?A?$KG?G?Q?5?$MA?N?$LP?x?5?$LO?r?$LB?b?5?$LN?G?F?P@ 0044c8e8     rylgamelibrary:serversetup.obj
 0002:0000290c       ??_C@_0M@OMKOIECC@BattleLimit?$AA@ 0044c90c     rylgamelibrary:serversetup.obj
 0002:00002918       ??_C@_0P@OMHNIBOL@?$MA?$KP?$MA?z?5?A?$KG?G?Q?5?$LN?G?F?P?$AA@ 0044c918     rylgamelibrary:serversetup.obj
 0002:00002928       ??_C@_08NOJOAFDF@LimitNum?$AA@ 0044c928     rylgamelibrary:serversetup.obj
 0002:00002934       ??_C@_03GDMIGCCC@Ver?$AA@  0044c934     rylgamelibrary:serversetup.obj
 0002:00002938       ??_C@_0BC@NGPHMKMK@?$LP?$LF?$MA?Z?5IP?C?$LM?E?$KJ?5?$LN?G?F?P?4?$AA@ 0044c938     rylgamelibrary:serversetup.obj
 0002:0000294c       ??_C@_0N@GMDOLMIM@AdminIPCheck?$AA@ 0044c94c     rylgamelibrary:serversetup.obj
 0002:0000295c       ??_C@_0BK@NEKPCPLB@?$LM?$KN?$LJ?v?5?$LA?z?$LB?$NN?5?E?$LI?$MA?T?5?$LO?r?$LB?b?5?$LN?G?F?P?4?$AA@ 0044c95c     rylgamelibrary:serversetup.obj
 0002:00002978       ??_C@_0BM@COOCFGIP@?A?$NP?$LA?h?5?$LM?$KN?$LJ?v?5?$LO?F?$MA?L?$LF?p?5?$LO?r?$LB?b?5?$LN?G?F?P?4?$AA@ 0044c978     rylgamelibrary:serversetup.obj
 0002:00002994       ??_C@_05KEMJHBCB@Agent?$AA@ 0044c994     rylgamelibrary:serversetup.obj
 0002:0000299c       ??_C@_0BF@PGKADKBL@HanUnitedBillingPort?$AA@ 0044c99c     rylgamelibrary:serversetup.obj
 0002:000029b4       ??_C@_0BM@FGNDHECI@CServerSetup?3?3InitUIDServer?$AA@ 0044c9b4     rylgamelibrary:serversetup.obj
 0002:000029d0       ??_C@_0BP@HJHNBJJH@?G?Q?$LA?T?$MA?S?5?E?k?G?U?$LK?t?$LI?$LF?5?A?V?$LM?R?5?$MA?P?$LB?b?5?$LN?G?F?P?$AA@ 0044c9d0     rylgamelibrary:serversetup.obj
 0002:000029f0       ??_C@_0BF@DCNAHLGM@HanUnitedBillingAddr?$AA@ 0044c9f0     rylgamelibrary:serversetup.obj
 0002:00002a08       ??_C@_0BG@MAMOICND@?G?C?$LH?$LJ?$LB?W?5?$LJ?$KL?$LN?C?C?$LM?E?$KJ?5?$LN?G?F?P?4?$AA@ 0044ca08     rylgamelibrary:serversetup.obj
 0002:00002a20       ??_C@_0L@HBAIHIJP@IgnoreFlag?$AA@ 0044ca20     rylgamelibrary:serversetup.obj
 0002:00002a2c       ??_C@_0P@IOEOGKO@?G?A?$LI?$KO?C?$LM?E?$KJ?5?$LN?G?F?P?4?$AA@ 0044ca2c     rylgamelibrary:serversetup.obj
 0002:00002a3c       ??_C@_06BFFONFPF@Keeper?$AA@ 0044ca3c     rylgamelibrary:serversetup.obj
 0002:00002a44       ??_C@_09PAOPECMK@FreeCheck?$AA@ 0044ca44     rylgamelibrary:serversetup.obj
 0002:00002a50       ??_C@_0BN@IOMGODDA@CServerSetup?3?3InitChatServer?$AA@ 0044ca50     rylgamelibrary:serversetup.obj
 0002:00002a70       ??_C@_0BC@LBMEOJMM@?$LP?n?$LP?$LF?5DB?5?$MA?P?$LB?b?5?$LN?G?F?P?$AA@ 0044ca70     rylgamelibrary:serversetup.obj
 0002:00002a84       ??_C@_0M@MFKBHEJP@AdminDBPass?$AA@ 0044ca84     rylgamelibrary:serversetup.obj
 0002:00002a90       ??_C@_0P@MIHOICHG@AdminDBAccount?$AA@ 0044ca90     rylgamelibrary:serversetup.obj
 0002:00002aa0       ??_C@_0M@BAFBGGNB@AdminDBName?$AA@ 0044caa0     rylgamelibrary:serversetup.obj
 0002:00002aac       ??_C@_0M@KPINLOCL@AdminDBAddr?$AA@ 0044caac     rylgamelibrary:serversetup.obj
 0002:00002ab8       ??_C@_0N@FLFMEHNP@AgentAddress?$AA@ 0044cab8     rylgamelibrary:serversetup.obj
 0002:00002ac8       ??_C@_0BG@BEELHFME@?C?$KE?F?C?5?$LM?$KN?$LJ?v?5ID?$MA?P?$LB?b?5?$LN?G?F?P?$AA@ 0044cac8     rylgamelibrary:serversetup.obj
 0002:00002ae0       ??_C@_0L@KOLHEMGH@ChatServer?$AA@ 0044cae0     rylgamelibrary:serversetup.obj
 0002:00002aec       ??_C@_0N@LOEGBABN@ManageClient?$AA@ 0044caec     rylgamelibrary:serversetup.obj
 0002:00002afc       ??_C@_02OFPLGCCC@?9z?$AA@  0044cafc     rylgamelibrary:serversetup.obj
 0002:00002b00       ??_C@_04NGCDMBKE@?5?$AN?6?7?$AA@ 0044cb00     rylgamelibrary:serversetup.obj
 0002:00002b08       ??_C@_0CB@BDGEEPLI@CServerSetup?3?3GetZoneFromCmdLine@ 0044cb08     rylgamelibrary:serversetup.obj
 0002:00002b2c       ??_C@_0CA@MPHFNNKD@CommandLine?5Parse?5failed?5?9?5Zone?$AA@ 0044cb2c     rylgamelibrary:serversetup.obj
 0002:00002b4c       ??_C@_02HOPLMLDK@?9c?$AA@  0044cb4c     rylgamelibrary:serversetup.obj
 0002:00002b50       ??_C@_0CE@MLCFPBDB@CServerSetup?3?3GetChannelFromCmdL@ 0044cb50     rylgamelibrary:serversetup.obj
 0002:00002b74       ??_C@_0CD@LDLPOHAN@CommandLine?5Parse?5failed?5?9?5Chann@ 0044cb74     rylgamelibrary:serversetup.obj
 0002:00002b98       ??_7CServerSetup@@6B@      0044cb98     rylgamelibrary:serversetup.obj
 0002:00002b9c       ??_C@_01EEMJAFIK@?6?$AA@   0044cb9c     rylgamelibrary:serversetup.obj
 0002:00002ba0       ??_C@_0BN@BKOBHDCN@?4?1Script?1Server?1AdminUID?4txt?$AA@ 0044cba0     rylgamelibrary:serversetup.obj
 0002:00002bc0       ??_C@_01KDCPPGHE@r?$AA@    0044cbc0     rylgamelibrary:serversetup.obj
 0002:00002bc4       ??_C@_0BM@JNGCCKNC@?$LJ?h?F?$LC?$LM?$KN?$LJ?v?$MA?N?A?v?5?$LP?$KJ?$LK?N?5?$MA?P?$LB?b?5?$LN?G?F?P?$AA@ 0044cbc4     rylgamelibrary:serversetup.obj
 0002:00002be0       ??_C@_0BE@OIPPDBHL@IsBattleServerGroup?$AA@ 0044cbe0     rylgamelibrary:serversetup.obj
 0002:00002bf4       ??_C@_08NCJJFBEA@Zone_ETC?$AA@ 0044cbf4     rylgamelibrary:serversetup.obj
 0002:00002c00       ??_C@_0BB@OOJPDHGF@GameServerNation?$AA@ 0044cc00     rylgamelibrary:serversetup.obj
 0002:00002c14       ??_C@_0CJ@OOOKNLGB@?$LF?p?$LJ?v?$LB?W?$LP?k?5UID?5?$LI?$KO?$LN?$LK?F?$KO?5?$LL?$PN?$LM?$LK?$LP?$KB?5?$LN?G?F?P?G@ 0044cc14     rylgamelibrary:serversetup.obj
 0002:00002c40       ??_C@_0BO@LIEFIGC@?$LA?T?$MA?S?$LM?$KN?$LJ?v?5UDP?5?A?V?$LM?R?$LI?$KG?5?$LM?$LM?F?C?5?$LN?G?F?P?$AA@ 0044cc40     rylgamelibrary:serversetup.obj
 0002:00002c60       ??_C@_0BJ@DNOGNEHK@?C?$KE?F?C?5?$LM?$KN?$LJ?v?5?A?V?$LM?R?5?$MA?P?$LB?b?5?$LN?G?F?P?$AA@ 0044cc60     rylgamelibrary:serversetup.obj
 0002:00002c7c       ??_C@_0P@MGJLGEKL@ChatServerAddr?$AA@ 0044cc7c     rylgamelibrary:serversetup.obj
 0002:00002c8c       ??_C@_0BJ@MDMBEKLP@?$LH?N?$LB?W?5?$LM?$KN?$LJ?v?5?A?V?$LM?R?5?$MA?P?$LB?b?5?$LN?G?F?P?$AA@ 0044cc8c     rylgamelibrary:serversetup.obj
 0002:00002ca8       ??_C@_0O@EONNMLPA@LogServerAddr?$AA@ 0044cca8     rylgamelibrary:serversetup.obj
 0002:00002cb8       ??_C@_0DD@MBCMCOON@?$CIz?3?$CF02d?0?5c?3?$CF02d?$CJ?5?$LJ?h?F?$LC?$LB?W?$LG?s?$LP?n?$LF?e?5?A?$KG@ 0044ccb8     rylgamelibrary:serversetup.obj
 0002:00002cec       ??_C@_0CI@FLPJFHJP@?$CIz?3?$CF02d?0?5c?3?$CF02d?$CJ?5?C?V?$LE?k?5?$LI?m?$LM?$LK?D?$KB?5?$LO?r?$LB@ 0044ccec     rylgamelibrary:serversetup.obj
 0002:00002d14       ??_C@_07HKNLJKBN@FameMax?$AA@ 0044cd14     rylgamelibrary:serversetup.obj
 0002:00002d1c       ??_C@_0CI@HMINEIDD@?$CIz?3?$CF02d?0?5c?3?$CF02d?$CJ?5?C?V?$LM?R?5?$LI?m?$LM?$LK?D?$KB?5?$LO?r?$LB@ 0044cd1c     rylgamelibrary:serversetup.obj
 0002:00002d44       ??_C@_07GIFAHOHC@FameMin?$AA@ 0044cd44     rylgamelibrary:serversetup.obj
 0002:00002d4c       ??_C@_0CI@MIMOCLJC@?$CIz?3?$CF02d?0?5c?3?$CF02d?$CJ?5?$LF?e?$LG?x?$LH?$PM?5?$LJ?h?$MA?$LC?5?$LO?r?$LB@ 0044cd4c     rylgamelibrary:serversetup.obj
 0002:00002d74       ??_C@_04DJCMGLJH@Drop?$AA@ 0044cd74     rylgamelibrary:serversetup.obj
 0002:00002d7c       ??_C@_0CI@IBFFFLOH@?$CIz?3?$CF02d?0?5c?3?$CF02d?$CJ?5?$LA?f?G?h?D?$KB?5?$LJ?h?$MA?$LC?5?$LO?r?$LB@ 0044cd7c     rylgamelibrary:serversetup.obj
 0002:00002da4       ??_C@_03HKMMIPC@Exp?$AA@   0044cda4     rylgamelibrary:serversetup.obj
 0002:00002da8       ??_C@_0CK@KILDKBJL@?$CIz?3?$CF02d?0?5c?3?$CF02d?$CJ?5?$LH?$LJ?$LK?$KH?$LO?w?5?$MA?L?$LK?$KF?F?$KO?5?C@ 0044cda8     rylgamelibrary:serversetup.obj
 0002:00002dd4       ??_C@_0N@CBAIFBNB@LevelUpEvent?$AA@ 0044cdd4     rylgamelibrary:serversetup.obj
 0002:00002de4       ??_C@_0CI@ICOIKNNO@?$CIz?3?$CF02d?0?5c?3?$CF02d?$CJ?5?$LK?$LJ?$LB?G?5?$MA?L?$LK?$KF?F?$KO?5?C?$LM?E@ 0044cde4     rylgamelibrary:serversetup.obj
 0002:00002e0c       ??_C@_0N@JBLHHCGA@LotteryEvent?$AA@ 0044ce0c     rylgamelibrary:serversetup.obj
 0002:00002e1c       ??_C@_0BO@NOOMNIJI@?$CIz?3?$CF02d?0?5c?3?$CF02d?$CJ?5?G?Y?C?$LM?E?$KJ?5?$LN?G?F?P?4?$AA@ 0044ce1c     rylgamelibrary:serversetup.obj
 0002:00002e3c       ??_C@_09ELJEKNDN@SpeedHack?$AA@ 0044ce3c     rylgamelibrary:serversetup.obj
 0002:00002e48       ??_C@_0BO@KGGMNMOL@?$CIz?3?$CF02d?0?5c?3?$CF02d?$CJ?5?G?N?C?$LM?E?$KJ?5?$LN?G?F?P?4?$AA@ 0044ce48     rylgamelibrary:serversetup.obj
 0002:00002e68       ??_C@_0CN@FGNMNMCE@?$CIz?3?$CF02d?0?5c?3?$CF02d?$CJ?5?$LA?T?$MA?S?5?$LM?$KN?$LJ?v?5?$LO?F?$MA?L?$LF@ 0044ce68     rylgamelibrary:serversetup.obj
 0002:00002e98       ??_C@_0BN@JECPHJNJ@CServerSetup?3?3InitGameServer?$AA@ 0044ce98     rylgamelibrary:serversetup.obj
 0002:00002eb8       ??_C@_0CH@HHNJBCCJ@?$CIz?3?$CF02d?0?5c?3?$CF02d?$CJ?5?D?$LP?$LI?G?$LF?e?5?$LG?s?$MA?N?5?F?D?$LN@ 0044ceb8     rylgamelibrary:serversetup.obj
 0002:00002ee0       ??_C@_0O@GEECGKNC@Zone_?$CF02d?$CF02d?$AA@ 0044cee0     rylgamelibrary:serversetup.obj
 0002:00002ef0       ??_C@_0BP@BPGLAJLF@Reset?5dispatch?$CIKey?3?$CFu?1DP?30x?$CFp?$CJ?$AA@ 0044cef0     rylgamelibrary:multidispatchstorage.obj
 0002:00002f10       ??_C@_0CH@CIACIHNK@CMultiDispatch?3?3InternalRemoveDi@ 0044cf10     rylgamelibrary:multidispatchstorage.obj
 0002:00002f38       ??_C@_0IM@MDJPLBPH@D?3?2Work?2RYL?2Source?2v?4538?$FN?5?G?X?$LP?$NM?5?$CI@ 0044cf38     rylgamelibrary:multidispatchstorage.obj
 0002:00002fc4       ??_C@_0DA@BOOBIBID@Reset?5dispatch?5failed?4?5Invalid?5d@ 0044cfc4     rylgamelibrary:multidispatchstorage.obj
 0002:00002ff4       ??_C@_0DE@COFEJOKG@DP?30x?$CFp?1Already?5dispatch?5exist?4?5@ 0044cff4     rylgamelibrary:multidispatchstorage.obj
 0002:00003028       ??_C@_0CF@MIKOEMOP@Setting?5new?5dispatch?$CIKey?3?$CFu?1DP?30@ 0044d028     rylgamelibrary:multidispatchstorage.obj
 0002:00003050       ??_C@_0BM@OELALPEH@CMultiDispatch?3?3SetDispatch?$AA@ 0044d050     rylgamelibrary:multidispatchstorage.obj
 0002:0000306c       ??_C@_0CA@COMGAILM@this?30x?$CFp?1Setting?5null?5dispatch?$AA@ 0044d06c     rylgamelibrary:multidispatchstorage.obj
 0002:0000308c       ??_C@_0CA@IKFMMHBJ@CMultiDispatch?3?3?$HOCMultiDispatch?$AA@ 0044d08c     rylgamelibrary:multidispatchstorage.obj
 0002:000030ac       ??_C@_0DA@KGOMKKFL@this?30x?$CFp?1Dispatch?5is?5not?5remove@ 0044d0ac     rylgamelibrary:multidispatchstorage.obj
 0002:000030dc       ??_C@_0DI@DKBOPIGL@this?30x?$CFp?1Reset?5dispatch?5failed?4@ 0044d0dc     rylgamelibrary:singledispatchstorage.obj
 0002:00003114       ??_C@_0CI@MOKCGFGL@CSingleDispatch?3?3InternalRemoveD@ 0044d114     rylgamelibrary:singledispatchstorage.obj
 0002:00003140       ??_C@_0IN@IKMLJGPD@D?3?2Work?2RYL?2Source?2v?4538?$FN?5?G?X?$LP?$NM?5?$CI@ 0044d140     rylgamelibrary:singledispatchstorage.obj
 0002:000031d0       ??_C@_0BH@BONJLFGE@DP?30x?$CFp?1Reset?5dispatch?$AA@ 0044d1d0     rylgamelibrary:singledispatchstorage.obj
 0002:000031e8       ??_C@_0CG@GFNJALCG@DP?30x?$CFp?1Setting?5new?5dispatch?$CIDP?3@ 0044d1e8     rylgamelibrary:singledispatchstorage.obj
 0002:00003210       ??_C@_0BN@MDJDKLOC@CSingleDispatch?3?3SetDispatch?$AA@ 0044d210     rylgamelibrary:singledispatchstorage.obj
 0002:00003230       ??_C@_0CM@DEEOFNCG@this?30x?$CFp?1Already?5dispatch?5exist@ 0044d230     rylgamelibrary:singledispatchstorage.obj
 0002:0000325c       ??_C@_0CC@GPMPPAEL@CSingleDispatch?3?3?$HOCSingleDispatc@ 0044d25c     rylgamelibrary:singledispatchstorage.obj
 0002:00003280       ??_C@_0CO@OGAEBOKK@DP?30x?$CFp?1Dispatch?5is?5not?5removed?5@ 0044d280     rylgamelibrary:singledispatchstorage.obj
 0002:000032d0       ??_C@_06JBKGCNBB@Delete?$AA@ 0044d2d0     rylgamelibrary:characterlog.obj
 0002:000032d8       ??_C@_08KAAPDIAN@NoRemove?$AA@ 0044d2d8     rylgamelibrary:characterlog.obj
 0002:000032e4       ??_C@_0M@DBGDLGLL@ForceRemove?$AA@ 0044d2e4     rylgamelibrary:characterlog.obj
 0002:000032f0       ??_C@_03LAIAPFCB@Val?$AA@  0044d2f0     rylgamelibrary:characterlog.obj
 0002:000032f4       ??_C@_01HMGJMAIH@B?$AA@    0044d2f4     rylgamelibrary:characterlog.obj
 0002:000032f8       ??_C@_01CKDDGHAB@D?$AA@    0044d2f8     rylgamelibrary:characterlog.obj
 0002:000032fc       ??_C@_01PLPBNMEI@M?$AA@    0044d2fc     rylgamelibrary:characterlog.obj
 0002:00003300       ??_C@_01CPLAODJH@S?$AA@    0044d300     rylgamelibrary:characterlog.obj
 0002:00003318       ??_C@_0HF@BLFKJEBI@D?3?2Work?2RYL?2Source?2v?4538?$FN?5?G?X?$LP?$NM?5?$CI@ 0044d318     rylgamelibrary:characterlog.obj
 0002:00003390       ??_C@_0BC@ECLHJPIL@?$LO?K?5?$LM?v?5?$LO?x?$LE?B?5?D?$LP?$LI?G?$LF?e?$AA@ 0044d390     rylgamelibrary:characterlog.obj
 0002:000033a4       ??_C@_0BN@GGNKMHLJ@GAMELOG?3?3LogCharCreateDelete?$AA@ 0044d3a4     rylgamelibrary:characterlog.obj
 0002:000033c4       ??_C@_0DI@LCJMAFJC@UID?30x?$CF08x?5CID?30x?$CF08x?5?$MA?G?5?$CFs?3?$CF2d?$LH@ 0044d3c4     rylgamelibrary:characterlog.obj
 0002:000033fc       ??_C@_0M@OOIIEAJK@?D?$LD?$LI?$KP?E?M?5?$LL?$PN?$LM?$LK?$AA@ 0044d3fc     rylgamelibrary:characterlog.obj
 0002:00003408       ??_C@_0M@DDBBEBGJ@?D?$LD?$LI?$KP?E?M?5?$LL?h?A?$KG?$AA@ 0044d408     rylgamelibrary:characterlog.obj
 0002:00003418       ??_C@_0MA@NIPMIOFL@?$FLm_hSocket?30x?$CF08x?$FN?$FL?$CF15s?$FN?$FLDiffTim@ 0044d418     rylgamelibrary:session.obj
 0002:000034d8       ??_C@_09KGBNNNJO@CONNECTED?$AA@ 0044d4d8     rylgamelibrary:session.obj
 0002:000034e4       ??_C@_0N@HLEBDOBD@DISCONNECTED?$AA@ 0044d4e4     rylgamelibrary:session.obj
 0002:000034f4       ??_C@_0N@PEIOMEHH@Unknown?5Mode?$AA@ 0044d4f4     rylgamelibrary:session.obj
 0002:00003504       ??_C@_0DP@LMJLFFNN@SP?30x?$CFp?1DP?30x?$CFp?1IP?3?$CF15s?1?5Interna@ 0044d504     rylgamelibrary:session.obj
 0002:00003548       ??_C@_0EP@HHBDFEIF@SP?30x?$CFp?1DP?30x?$CFp?1IP?3?$CF15s?1SOCKET?30@ 0044d548     rylgamelibrary:session.obj
 0002:00003598       ??_C@_0BO@HPINOBI@CSession?3?3InternalCloseSocket?$AA@ 0044d598     rylgamelibrary:session.obj
 0002:000035b8       ??_C@_0HJ@HKBIMOGG@D?3?2Work?2RYL?2Source?2v?4538?$FN?5?G?X?$LP?$NM?5?$CI@ 0044d5b8     rylgamelibrary:session.obj
 0002:00003638       ??_C@_0EE@BKBLFAJL@SP?30x?$CFp?1DP?30x?$CFp?1IP?3?$CF15s?1SOCKET?30@ 0044d638     rylgamelibrary:session.obj
 0002:0000367c       ??_C@_0BH@LKOMCIHL@CSession?3?3CloseSession?$AA@ 0044d67c     rylgamelibrary:session.obj
 0002:00003698       ??_C@_0EI@KADBPLFF@SP?30x?$CFp?1DP?30x?$CFp?1IP?3?$CF15s?1?5Interna@ 0044d698     rylgamelibrary:session.obj
 0002:000036e0       ??_C@_0HG@EINGGMGK@SP?30x?$CFp?1DP?30x?$CFp?1IP?3?$CF15s?1SOCKET?30@ 0044d6e0     rylgamelibrary:session.obj
 0002:00003758       ??_C@_0FH@COLCJKJF@SP?30x?$CFp?1DP?30x?$CFp?1IP?3?$CF15s?1SOCKET?30@ 0044d758     rylgamelibrary:session.obj
 0002:000037b0       ??_C@_0BH@CGDPEHJK@CSession?3?3InternalRecv?$AA@ 0044d7b0     rylgamelibrary:session.obj
 0002:000037c8       ??_C@_0DG@GLNGJLBC@SP?30x?$CFp?1DP?30x?$CFp?1IP?3?$CF15s?1SOCKET?30@ 0044d7c8     rylgamelibrary:session.obj
 0002:00003800       ??_C@_0BH@GLHDINKK@CSession?3?3InternalSend?$AA@ 0044d800     rylgamelibrary:session.obj
 0002:00003818       ??_C@_0GI@INMDMEII@SP?30x?$CFp?1DP?30x?$CFp?1IP?3?$CF15s?1SOCKET?30@ 0044d818     rylgamelibrary:session.obj
 0002:00003880       ??_C@_0HH@GMFGLPHA@SP?30x?$CFp?1DP?30x?$CFp?1IP?3?$CF15s?1SOCKET?30@ 0044d880     rylgamelibrary:session.obj
 0002:000038f8       ??_C@_0FI@PAIHKOAM@SP?30x?$CFp?1DP?30x?$CFp?1IP?3?$CF15s?1SOCKET?30@ 0044d8f8     rylgamelibrary:session.obj
 0002:00003950       ??_C@_0GK@BPJDPGOO@SP?30x?$CFp?1DP?30x?$CFp?1IP?3?$CF15s?1SOCKET?30@ 0044d950     rylgamelibrary:session.obj
 0002:000039c0       ??_C@_0HJ@MPEEIFIK@SP?30x?$CFp?1DP?30x?$CFp?1IP?3?$CF15s?1SOCKET?30@ 0044d9c0     rylgamelibrary:session.obj
 0002:00003a40       ??_C@_0FK@FEFEHPJH@SP?30x?$CFp?1DP?30x?$CFp?1IP?3?$CF15s?1SOCKET?30@ 0044da40     rylgamelibrary:session.obj
 0002:00003a9c       ??_C@_0BJ@EODBDBIJ@CSession?3?3InternalSendTo?$AA@ 0044da9c     rylgamelibrary:session.obj
 0002:00003ab8       ??_C@_0DI@GPFPFCJ@SP?30x?$CFp?1DP?30x?$CFp?1IP?3?$CF15s?1SOCKET?30@ 0044dab8     rylgamelibrary:session.obj
 0002:00003af0       ??_C@_0EM@HCKIGKMO@SP?30x?$CFp?1DP?30x?$CFp?1IP?3?$CF15s?1SOCKET?30@ 0044daf0     rylgamelibrary:session.obj
 0002:00003b40       ??_C@_0EC@DKBMMJEC@SP?30x?$CFp?1DP?30x?$CFp?1IP?3?$CF15s?1SOCKET?30@ 0044db40     rylgamelibrary:session.obj
 0002:00003b88       ??_C@_0EI@IJGNGOCB@SP?30x?$CFp?1DP?30x?$CFp?1IP?3?$CF15s?1SOCKET?30@ 0044db88     rylgamelibrary:session.obj
 0002:00003bd0       ??_C@_0BC@FBCFPDPA@CSession?3?3Process?$AA@ 0044dbd0     rylgamelibrary:session.obj
 0002:00003be4       ??_C@_0DG@FJFPNDJE@SP?30x?$CFp?1DP?30x?$CFp?1IP?3?$CF15s?1SOCKET?30@ 0044dbe4     rylgamelibrary:session.obj
 0002:00003c1c       ??_C@_0BD@JBHILDMG@CSession?3?3Dispatch?$AA@ 0044dc1c     rylgamelibrary:session.obj
 0002:00003c30       ??_C@_0FF@NOJPKKFH@SP?30x?$CFp?1DP?30x?$CFp?1IP?3?$CF15s?1SOCKET?30@ 0044dc30     rylgamelibrary:session.obj
 0002:00003c88       ??_C@_0BK@IPFJOKOK@Failed?5To?5Dispatch?5Packet?$AA@ 0044dc88     rylgamelibrary:session.obj
 0002:00003ca4       ??_C@_0N@NFBNFHML@Disconnected?$AA@ 0044dca4     rylgamelibrary:session.obj
 0002:00003cb4       ??_C@_0BI@OPMFGCNF@CSession?3?3SendCompleted?$AA@ 0044dcb4     rylgamelibrary:session.obj
 0002:00003cd0       ??_C@_0EK@OHIOMIAB@SP?30x?$CFp?1DP?30x?$CFp?1IP?3?$CF15s?1?5Interna@ 0044dcd0     rylgamelibrary:session.obj
 0002:00003ecd       ??_C@_00CNPNBAHC@?$AA@     0044decd     rylgamelibrary:charactercreate.obj
 0002:00003ee0       ??_7CDBComponent@@6B@      0044dee0     rylgamelibrary:dbcomponent.obj
 0002:00003ee4       ??_C@_0CF@FKAKCHBJ@dbo?4spLoginAuthMyth?5?8?$CFs?8?0?5?8?$CFs?8?0?5@ 0044dee4     rylgamelibrary:dbcomponent.obj
 0002:00003f0c       ??_C@_0BN@EHDIALPB@?$HLcall?5pc_ryl_login?$CI?$DP?0?5?$DP?0?5?$DP?$CJ?$HN?$AA@ 0044df0c     rylgamelibrary:dbcomponent.obj
 0002:00003f2c       ??_C@_0BL@OABDMCNF@?$HLcall?5pc_ryl_login2?$CI?$DP?0?5?$DP?$CJ?$HN?$AA@ 0044df2c     rylgamelibrary:dbcomponent.obj
 0002:00003f48       ??_C@_0CM@JIPEKKB@select?5FC_GETUID_BYMEMBERID?$CI?8?$CFs?8@ 0044df48     rylgamelibrary:dbcomponent.obj
 0002:00003f74       ??_C@_0CF@EDEMAIJM@dbo?4USPCheckRestraintChar?5?8?$CFd?8?0?5@ 0044df74     rylgamelibrary:dbcomponent.obj
 0002:00003f9c       ??_C@_0BP@JBJCLALF@?$HLcall?5pc_rylbl_login?$CI?$DP?0?5?$DP?0?5?$DP?$CJ?$HN?$AA@ 0044df9c     rylgamelibrary:dbcomponent.obj
 0002:00003fbc       ??_C@_0BN@CEFANFBL@?$HLcall?5pc_rylbl_login2?$CI?$DP?0?5?$DP?$CJ?$HN?$AA@ 0044dfbc     rylgamelibrary:dbcomponent.obj
 0002:00003fdc       ??_C@_0DC@NMDBNDDP@select?5FC_RYLBL_GETUID_BYMEMBERI@ 0044dfdc     rylgamelibrary:dbcomponent.obj
 0002:00004010       ??_C@_0DO@CEEHIFGN@?C?$KE?F?C?5?$LM?$KN?$LJ?v?5?$LH?N?$LB?W?$MA?N?5DataSource?5?3?5?$CFs@ 0044e010     rylgamelibrary:dbcomponent.obj
 0002:00004050       ??_C@_0DO@GFFOFDNJ@?E?$LA?F?$NL?5?$LM?$KN?$LJ?v?5?$LH?N?$LB?W?$MA?N?5DataSource?5?3?5?$CFs@ 0044e050     rylgamelibrary:dbcomponent.obj
 0002:00004090       ??_C@_0ED@KEMMMGEL@?A?$NP?$LA?h?5?$LM?$KN?$LJ?v?5?$LH?N?$LB?W?$MA?N?5Server?5?3?5?$CFs?0?5DB@ 0044e090     rylgamelibrary:dbcomponent.obj
 0002:000040d4       ??_C@_06HJGLHJBN@DBPass?$AA@ 0044e0d4     rylgamelibrary:dbcomponent.obj
 0002:000040dc       ??_C@_09OENABIMH@DBAccount?$AA@ 0044e0dc     rylgamelibrary:dbcomponent.obj
 0002:000040e8       ??_C@_06KMJLGLFD@DBName?$AA@ 0044e0e8     rylgamelibrary:dbcomponent.obj
 0002:000040f0       ??_C@_0P@GGHIHMIK@DemonSetup?4ini?$AA@ 0044e0f0     rylgamelibrary:dbcomponent.obj
 0002:00004100       ??_C@_0N@JAKHBCCN@DBServerName?$AA@ 0044e100     rylgamelibrary:dbcomponent.obj
 0002:00004110       ??_C@_0EH@LGHBDHAH@?$MA?N?A?u?5?$LM?$KN?$LJ?v?5?$LH?N?$LB?W?$MA?N?$CIHangame?$CJ?5DataSo@ 0044e110     rylgamelibrary:dbcomponent.obj
 0002:00004158       ??_C@_0BG@DGEJHNAK@CDBComponent?3?3Connect?$AA@ 0044e158     rylgamelibrary:dbcomponent.obj
 0002:00004170       ??_C@_0HF@BJNBKHBH@D?3?2Work?2RYL?2Source?2v?4538?$FN?5?G?X?$LP?$NM?5?$CI@ 0044e170     rylgamelibrary:dbcomponent.obj
 0002:000041e8       ??_C@_0EE@IMELCMCG@?$MA?N?A?u?5?$LM?$KN?$LJ?v?5?$LH?N?$LB?W?$MA?N?$CI?$LE?k?$LI?$LI?$CJ?5DataSourc@ 0044e1e8     rylgamelibrary:dbcomponent.obj
 0002:0000422c       ??_C@_0P@COHJCFID@DataSourcePass?$AA@ 0044e22c     rylgamelibrary:dbcomponent.obj
 0002:0000423c       ??_C@_0BC@PGOKOOHK@DataSourceAccount?$AA@ 0044e23c     rylgamelibrary:dbcomponent.obj
 0002:00004250       ??_C@_0P@PLIJDHMN@DataSourceName?$AA@ 0044e250     rylgamelibrary:dbcomponent.obj
 0002:00004260       ??_7CThreadMgr@@6B@        0044e260     rylgamelibrary:threadmgr.obj
 0002:00004264       ??_C@_0BL@JBKMNPIP@?4?1Script?1Game?1Chemical?4txt?$AA@ 0044e264     rylgamelibrary:itemmgr.obj
 0002:00004280       ??_C@_0BP@JEFODPPL@?4?1Script?1Game?1BGItemScript?4txt?$AA@ 0044e280     rylgamelibrary:itemmgr.obj
 0002:000042a0       ??_C@_0BN@EDFPEEOJ@?4?1Script?1Game?1ItemScript?4txt?$AA@ 0044e2a0     rylgamelibrary:itemmgr.obj
 0002:000042e0       ??_C@_0CC@LCACBJBB@CParseDelimitedData?3?3operator?$GA?$CI?$CJ@ 0044e2e0     rylgamelibrary:itemmgr.obj
 0002:00004308       ??_C@_0HB@LKCPHIJO@D?3?2Work?2RYL?2Source?2v?4538?$FN?5?G?X?$LP?$NM?5?$CI@ 0044e308     rylgamelibrary:itemmgr.obj
 0002:0000437c       ??_C@_0DB@NCJCEFLE@?$LO?K?$LI?B?$MA?$LK?5?$LF?$KF?$MA?L?E?M?$LA?$KB?5?$LO?F?$LE?U?$LE?O?$LE?Y?4?5Line?3?$CF@ 0044e37c     rylgamelibrary:itemmgr.obj
 0002:000043b0       ??_C@_0DE@JFIMJLLN@?$LF?$KF?$MA?L?E?M?$LI?$KG?5?$MA?P?$LO?n?$LP?C?5?$LM?v?5?$LO?x?$LN?$MA?$LE?O?$LE?Y?4?5Lin@ 0044e3b0     rylgamelibrary:itemmgr.obj
 0002:000043e8       ??_C@_0EA@POFHLAIP@?$LO?F?$MA?L?E?$NL?5?$LN?$LK?E?$KJ?$LI?$LD?F?$KO?5?$LD?$LL?$LP?k?$MA?$LL?5?$LK?$LJ?$LL?g?G?R?5?$LM?v@ 0044e3e8     rylgamelibrary:itemmgr.obj
 0002:00004428       ??_C@_0CM@BGIOMBGB@?$LA?c?D?$KB?$LE?B?5?$LO?F?$MA?L?E?$NL?5?A?$LO?$LH?y?5ID?$LA?$KB?5?$MA?V?$LN?$MA?$LE?O?$LE?Y@ 0044e428     rylgamelibrary:itemmgr.obj
 0002:00004454       ??_C@_0DC@LNPLGHFC@?$LO?F?$MA?L?E?$NL?5?$LN?$LK?E?$KJ?$LI?$LD?F?$KO?5?F?D?$MA?O?$MA?$LL?5?$LE?Y?5?$MA?P?A?v?5?$LI@ 0044e454     rylgamelibrary:itemmgr.obj
 0002:00004488       ??_C@_0CC@EDHNDCEA@Item?3?3CItemMgr?3?3LoadItemProtoTyp@ 0044e488     rylgamelibrary:itemmgr.obj
 0002:000044ac       ??_C@_0DB@EPMIKHAO@?$LO?F?$MA?L?E?$NL?5?$LN?$LK?E?$KJ?$LI?$LD?F?$KO?5?D?C?$LH?$LD?$MA?$LL?5?$MA?P?$LO?n?$LP?$MA?$LE?B?5@ 0044e4ac     rylgamelibrary:itemmgr.obj
 0002:000044e0       ??_C@_0CK@EJCJCNDK@?$LO?F?$MA?L?E?$NL?5?$LN?$LK?E?$KJ?$LI?$LD?F?$KO?5?F?D?$MA?O?5?$LH?N?$LF?y?$LP?$KB?5?$LN?G?F?P@ 0044e4e0     rylgamelibrary:itemmgr.obj
 0002:0000450c       ??_C@_01GPOEFGEJ@?7?$AA@   0044e50c     rylgamelibrary:itemmgr.obj
 0002:00004530       ??_C@_0BP@KLHLJNFH@Item?3?3CItemFactory?3?3CreateItem?$AA@ 0044e530     rylgamelibrary:itemfactory.obj
 0002:00004550       ??_C@_0HF@EDHBAPHD@D?3?2Work?2RYL?2Source?2v?4538?$FN?5?G?X?$LP?$NM?5?$CI@ 0044e550     rylgamelibrary:itemfactory.obj
 0002:000045c8       ??_C@_0CG@LGGIFDAG@?$LO?F?$MA?L?E?$NL?5?$LL?$PN?$LM?$LK?$LP?$KB?5?$LN?G?F?P?G?$NP?$LN?$MA?$LE?O?$LE?Y?4?5?A?$LO?$LH?y@ 0044e5c8     rylgamelibrary:itemfactory.obj
 0002:000045f0       ??_C@_0BH@GAAEGJO@CServerWindowFramework?$AA@ 0044e5f0     rylgamelibrary:serverwindowframework.obj
 0002:00004608       ??_7CSendDataToManageClient@@6B@ 0044e608     rylgamelibrary:serverwindowframework.obj
 0002:00004610       ??_7CProcessThread@@6B@    0044e610     rylgamelibrary:serverwindowframework.obj
 0002:00004620       ??_7CRecvCommandFromManageClient@@6B@ 0044e620     rylgamelibrary:serverwindowframework.obj
 0002:00004628       ??_C@_0CM@EBPDCIEH@CServerWindowFramework?3?3Initiali@ 0044e628     rylgamelibrary:serverwindowframework.obj
 0002:00004658       ??_C@_0JH@LBAEFFGD@D?3?2Work?2RYL?2Source?2v?4538?$FN?5?G?X?$LP?$NM?5?$CI@ 0044e658     rylgamelibrary:serverwindowframework.obj
 0002:000046f0       ??_C@_0CC@GELPGGCM@CreateWindow?5failed?4?5ErrorCode?3?$CF@ 0044e6f0     rylgamelibrary:serverwindowframework.obj
 0002:00004714       ??_C@_0CE@HKKFILF@RegisterClass?5failed?4?5ErrorCode?3@ 0044e714     rylgamelibrary:serverwindowframework.obj
 0002:00004738       ??_C@_0CD@DHEGJABM@CServerWindowFramework?3?3Initiali@ 0044e738     rylgamelibrary:serverwindowframework.obj
 0002:00004760       ??_C@_0FA@EAOAIJD@this?30x?$CFp?1ServerWindowFramework?5@ 0044e760     rylgamelibrary:serverwindowframework.obj
 0002:000047b0       ??_C@_0FD@PILJCLLJ@this?30x?$CFp?1ServerWindowFramework?5@ 0044e7b0     rylgamelibrary:serverwindowframework.obj
 0002:00004808       ??_C@_0EO@HBOHJCIJ@this?30x?$CFp?1ServerWindowFramework?5@ 0044e808     rylgamelibrary:serverwindowframework.obj
 0002:00004858       ??_C@_0FA@OOCPMCCG@this?30x?$CFp?1ServerWindowFramework?5@ 0044e858     rylgamelibrary:serverwindowframework.obj
 0002:000048a8       ??_C@_0FA@PDKHOHIC@this?30x?$CFp?1ServerWindowFramework?5@ 0044e8a8     rylgamelibrary:serverwindowframework.obj
 0002:000048f8       ??_C@_0CB@MOKDBCAO@this?30x?$CFp?1finish?5process?5threads@ 0044e8f8     rylgamelibrary:serverwindowframework.obj
 0002:0000491c       ??_C@_0CH@FEJHIEBF@CServerWindowFramework?3?3ProcessM@ 0044e91c     rylgamelibrary:serverwindowframework.obj
 0002:00004944       ??_C@_0BI@LKIKEHME@this?30x?$CFp?1finish?5server?$AA@ 0044e944     rylgamelibrary:serverwindowframework.obj
 0002:0000495c       ??_7CServerWindowFramework@@6B@ 0044e95c     rylgamelibrary:serverwindowframework.obj
 0002:00004964       ??_C@_0CL@ODMEGDJG@CRecvCommandFromManageClient?3?3op@ 0044e964     rylgamelibrary:serverwindowframework.obj
 0002:00004990       ??_C@_0CO@CCFDDCBF@Command?5create?5failed?5from?5Manag@ 0044e990     rylgamelibrary:serverwindowframework.obj
 0002:000049c0       ??_C@_0CJ@NBDDMKBI@CServerWindowFramework?3?3AddProce@ 0044e9c0     rylgamelibrary:serverwindowframework.obj
 0002:000049ec       ??_C@_0CG@OKALPKND@this?30x?$CFp?1Process?5thread?5start?5f@ 0044e9ec     rylgamelibrary:serverwindowframework.obj
 0002:00004a14       ??_C@_0CG@DLAOGCOD@this?30x?$CFp?1Process?5thread?5pointer@ 0044ea14     rylgamelibrary:serverwindowframework.obj
 0002:00004a3c       ??_C@_0BI@BBCBGOCG@Send?5WM_COPYDATAMessage?$AA@ 0044ea3c     rylgamelibrary:serverwindowframework.obj
 0002:00004a54       ??_7CValidateConnection@@6B@ 0044ea54     rylgamelibrary:limituserbyip.obj
 0002:00004a5c       ??_7CLimitUserByIP@@6B@    0044ea5c     rylgamelibrary:limituserbyip.obj
 0002:00004a64       ??_C@_0BP@MFFJEOKK@CListener?3?3InternalCloseListen?$AA@ 0044ea64     rylgamelibrary:listener.obj
 0002:00004a88       ??_C@_0HL@BAPICKGG@D?3?2Work?2RYL?2Source?2v?4538?$FN?5?G?X?$LP?$NM?5?$CI@ 0044ea88     rylgamelibrary:listener.obj
 0002:00004b04       ??_C@_0BI@PPEBEICF@closesocket?5failed?5?3?5?$CFd?$AA@ 0044eb04     rylgamelibrary:listener.obj
 0002:00004b1c       ??_7CListener@@6B@         0044eb1c     rylgamelibrary:listener.obj
 0002:00004b20       ??_C@_0BJ@IENFBCHO@CListener?3?3ProcessAccept?$AA@ 0044eb20     rylgamelibrary:listener.obj
 0002:00004b3c       ??_C@_0DC@JNDGFDEB@SP?30x?$CFp?1DP?30x?$CFp?1IP?3?$CF15s?1?5Accept?5@ 0044eb3c     rylgamelibrary:listener.obj
 0002:00004b70       ??_C@_0DN@ODABFDLE@CListener?5initialized?5failed?5?3?5A@ 0044eb70     rylgamelibrary:listener.obj
 0002:00004bb0       ??_C@_0EA@KDBIKJCF@CListener?5initialized?5failed?5?3?5C@ 0044ebb0     rylgamelibrary:listener.obj
 0002:00004bf0       ??_C@_0BG@LCJFNOIK@CListener?3?3Initialize?$AA@ 0044ebf0     rylgamelibrary:listener.obj
 0002:00004c08       ??_C@_0DF@GBFAGKPG@CListener?5initialized?5failed?5?3?5I@ 0044ec08     rylgamelibrary:listener.obj
 0002:00004c40       ??_C@_0CK@KIEJAKBI@SP?30x?$CFp?1DP?30x?$CFp?1IP?3?$CF15s?1?5Connect@ 0044ec40     rylgamelibrary:iocpnet.obj
 0002:00004c6c       ??_C@_0BC@BGIDFILB@CIOCPNet?3?3Connect?$AA@ 0044ec6c     rylgamelibrary:iocpnet.obj
 0002:00004c80       ??_C@_0HG@KFOLNECG@D?3?2Work?2RYL?2Source?2v?4538?$FN?5?G?X?$LP?$NM?5?$CI@ 0044ec80     rylgamelibrary:iocpnet.obj
 0002:00004cf8       ??_C@_0DK@JNALCIHB@Connected?5socket?5creation?5error?5@ 0044ecf8     rylgamelibrary:iocpnet.obj
 0002:00004d38       __real@0000000000000000    0044ed38     rylgamelibrary:performancecheck.obj
 0002:00004d40       ??_C@_0BM@EMHHDPIF@?6?6?5Total?5AvgTime?5?3?5?$CF3?46f?6?6?6?$AA@ 0044ed40     rylgamelibrary:performancecheck.obj
 0002:00004d5c       ??_C@_0DH@MEHGNGLH@?5?5?5?$CF3?46f?5?5?5?5?5?$CF3?46f?5?5?5?5?5?$CF3?46f?5?5?5?5@ 0044ed5c     rylgamelibrary:performancecheck.obj
 0002:00004d98       __real@41f0000000000000    0044ed98     rylgamelibrary:performancecheck.obj
 0002:00004da0       ??_C@_0LE@GLHPGDJD@?5?5?5?5Average?5?3?5?5?5?5Minimum?5?3?5?5?5?5Ma@ 0044eda0     rylgamelibrary:performancecheck.obj
 0002:00004e54       ??_C@_02CPIDLAI@at?$AA@    0044ee54     rylgamelibrary:performancecheck.obj
 0002:00004e58       ??_C@_0BO@GDJDHKJL@?$CFs?1PerformanceLog?9?$CFs?9?$CF05d?4log?$AA@ 0044ee58     rylgamelibrary:performancecheck.obj
 0002:00004e98       ??_C@_0DH@FGGKAJPC@?$CFd?5?$LP?$KB?$LH?$KP?$LH?N?5?$MA?N?G?X?5?$LO?P?C?$OA?G?O?$LA?m?5?$LD?$KN?5?$LH?N?$LB?W?$LI@ 0044ee98     rylgamelibrary:gamelog.obj
 0002:00004ed0       ??_C@_0CO@HPOHCGIB@?$CFd?5?$LP?$KB?$LH?$KP?$LH?N?5?$MA?N?G?X?5?$LH?N?$LB?W?5?F?D?$MA?O?5?$LO?P?C?$OA?$MA?L?5@ 0044eed0     rylgamelibrary:gamelog.obj
 0002:00004f00       ??_C@_0CM@ENADGJCD@?$LP?$KB?$LH?$KP?$LH?N?5?$MA?N?G?X?5?$LO?P?C?$OA?5?F?D?$MA?O?$LP?$KB?5?$LB?b?$LH?O?G?R?5?$LM@ 0044ef00     rylgamelibrary:gamelog.obj
 0002:00004f2c       ??_C@_0DB@GLFICJKI@?$LA?T?$MA?S?5?$LH?N?$LB?W?$LI?$KG?5?$LO?P?C?$OA?G?X?5?$LD?V?$MA?$LL?5?F?D?$MA?O?$MA?$LL?5?$LI@ 0044ef2c     rylgamelibrary:gamelog.obj
 0002:00004f60       ??_C@_02GMLFBBN@wb?$AA@    0044ef60     rylgamelibrary:gamelog.obj
 0002:00004f64       ??_C@_0CJ@PIGPBOKB@?$CFs?2?$CFs?9?$CF04d?$CF02d?$CF02d?9?$CF02d?$CF02d?$CF02d?9@ 0044ef64     rylgamelibrary:gamelog.obj
 0002:00004f90       ??_C@_0BJ@HBEPCDHM@CLogSaveThread?3?3Compress?$AA@ 0044ef90     rylgamelibrary:gamelog.obj
 0002:00004fb0       ??_C@_0HA@JGIIGFE@D?3?2Work?2RYL?2Source?2v?4538?$FN?5?G?X?$LP?$NM?5?$CI@ 0044efb0     rylgamelibrary:gamelog.obj
 0002:00005020       ??_C@_0CA@HJNHKMNE@?$LA?T?$MA?S?5?$LH?N?$LB?W?$LI?$KG?5?$LO?P?C?$OA?G?R?5?$LM?v?5?$LO?x?$LN?$MA?$LE?O?$LE?Y?4?$AA@ 0044f020     rylgamelibrary:gamelog.obj
 0002:00005040       ??_7CLogSaveThread@@6B@    0044f040     rylgamelibrary:gamelog.obj
 0002:0000504c       ??_C@_0BE@MEFCELLL@CGameLog?3?3GetBuffer?$AA@ 0044f04c     rylgamelibrary:gamelog.obj
 0002:00005060       ??_C@_0BL@LHIEKHKA@?$LJ?v?F?$NL?$LI?$KG?5?G?R?$LE?g?G?R?5?$LM?v?5?$LO?x?$LN?$MA?$LE?O?$LE?Y?4?$AA@ 0044f060     rylgamelibrary:gamelog.obj
 0002:0000507c       ??_C@_0BF@EDEILICD@CGameLog?3?3Initialize?$AA@ 0044f07c     rylgamelibrary:gamelog.obj
 0002:00005094       ??_C@_0CI@LJDGPNMF@Flush?$LN?$LK?$LH?$LJ?$LF?e?$LI?$KG?5?$LL?$PN?$LM?$LK?G?O?$LE?B?5?$LF?$KF?5?$LN?G?F?P?G?$NP@ 0044f094     rylgamelibrary:gamelog.obj
 0002:000050bc       ??_C@_0CL@KLHPEGM@?$LA?T?$MA?S?5?$LH?N?$LB?W?5?$LJ?v?F?$NL?$LI?$KG?5?G?R?$LE?g?G?O?$LE?B?5?$LF?$KF?5?$LN?G?F@ 0044f0bc     rylgamelibrary:gamelog.obj
 0002:000050e8       ??_C@_0BI@BHLAOCND@CGameLog?3?3ReserveBuffer?$AA@ 0044f0e8     rylgamelibrary:gamelog.obj
 0002:00005100       ??_C@_0BG@KMOLIMPD@?$LH?N?$LB?W?5?$LJ?v?F?$NL?$LA?$KB?50?$MA?T?$LE?O?$LE?Y?4?5?$AA@ 0044f100     rylgamelibrary:gamelog.obj
 0002:00005118       ??_C@_0BP@BIJILICJ@CLogSaveThread?3?3SetLogFileName?$AA@ 0044f118     rylgamelibrary:gamelog.obj
 0002:00005138       ??_C@_0DB@DMGFBMOC@?$LA?T?$MA?S?5?$LH?N?$LB?W?$LI?$KG?5?$MA?$KH?G?Q?5?F?D?$MA?O?5?$MA?L?$LI?$KH?$MA?$LL?5?$LL?$PN?$LM@ 0044f138     rylgamelibrary:gamelog.obj
 0002:0000516c       ??_C@_0DA@LFEFLEI@?$CFs?2?$CFsGameLog?9?$CF04d?$CF02d?$CF02d?9?$CF02d?$CF0@ 0044f16c     rylgamelibrary:gamelog.obj
 0002:0000519c       ??_C@_0BJ@DMGLFEJJ@CLogSaveThread?3?3WriteLog?$AA@ 0044f19c     rylgamelibrary:gamelog.obj
 0002:000051b8       ??_C@_0EM@KNDGLINF@?$LH?N?$LB?W?5?F?D?$MA?O?5?$LB?b?$LH?O?$LP?$KB?5?$LN?G?F?P?G?$NP?$LN?$MA?$LE?O?$LE?Y?4?5E@ 0044f1b8     rylgamelibrary:gamelog.obj
 0002:00005204       ??_7CTCPFactory@@6B@       0044f204     rylgamelibrary:socketfactory.obj
 0002:00005214       ??_7CBufferFactory@@6B@    0044f214     rylgamelibrary:bufferfactory.obj
 0002:00005220       ??_C@_02BKFDOEMK@wt?$AA@   0044f220     rylgamelibrary:bufferfactory.obj
 0002:00005224       ??_7CPoolBufferFactory@@6B@ 0044f224     rylgamelibrary:bufferfactory.obj
 0002:00005230       ??_7COverlappedFactory@@6B@ 0044f230     rylgamelibrary:overlapped.obj
 0002:00005244       ??_7COverlapped@@6B@       0044f244     rylgamelibrary:overlapped.obj
 0002:0000524c       ??_7CSendOverlapped@@6B@   0044f24c     rylgamelibrary:overlapped.obj
 0002:00005254       ??_7CStreamRecvOverlapped@@6B@ 0044f254     rylgamelibrary:overlapped.obj
 0002:0000525c       ??_7CAcceptOverlapped@@6B@ 0044f25c     rylgamelibrary:overlapped.obj
 0002:00005264       ??_7CStreamOverlappedFactory@@6B@ 0044f264     rylgamelibrary:overlapped.obj
 0002:00005278       ??_7CConsoleCMDFactory@@6B@ 0044f278     rylgamelibrary:consolecmdfactory.obj
 0002:00005280       __real@3ff0000000000000    0044f280     rylgamelibrary:packetstatistics.obj
 0002:00005288       ??_C@_0HL@EJFDLMGI@?6?5Total?5Data?5Send?5?3?5?$CF16?44fMb?5?1?5?$CF@ 0044f288     rylgamelibrary:packetstatistics.obj
 0002:00005308       ??_C@_0FF@KPLEPIBA@?7?5?$CF3d?$CI0x?$CF02X?$CJ?5?3?5?$CF16?44fCount?5?3?5?$CI?$CF@ 0044f308     rylgamelibrary:packetstatistics.obj
 0002:00005360       ??_C@_0HK@EAONGGKM@?6?5Total?5Data?5Recv?5?3?5?$CF16?44fMb?5?1?5?$CF@ 0044f360     rylgamelibrary:packetstatistics.obj
 0002:000053e0       ??_C@_0FA@CLMEHEPI@?7?5?$CF3d?$CI0x?$CF02X?$CJ?5?3?5?$CF16?44f?5?3?5?$CI?$CF16?44f@ 0044f3e0     rylgamelibrary:packetstatistics.obj
 0002:00005430       __real@3eb0000000000000    0044f430     rylgamelibrary:packetstatistics.obj
 0002:00005438       __real@3f50000000000000    0044f438     rylgamelibrary:packetstatistics.obj
 0002:00005440       ??_C@_0NP@EAIJLCLF@?7?9?9?5Server?5Packet?5Statistics?5?9?9?5@ 0044f440     rylgamelibrary:packetstatistics.obj
 0002:00005520       ??_C@_0BK@JKJJLIBM@?$CFs?1Statistics?9?$CFs?9?$CF05d?4log?$AA@ 0044f520     rylgamelibrary:packetstatistics.obj
 0002:0000553c       ??_7CDLLModule@@6B@        0044f53c     rylgamelibrary:exceptionreport.obj
 0002:00005544       ??_7CDBGFuncClass@@6B@     0044f544     rylgamelibrary:exceptionreport.obj
 0002:0000554c       ??_C@_0P@CICBGLGA@SymGetTypeInfo?$AA@ 0044f54c     rylgamelibrary:exceptionreport.obj
 0002:0000555c       ??_C@_0BB@KAOAIDAF@SymGetModuleBase?$AA@ 0044f55c     rylgamelibrary:exceptionreport.obj
 0002:00005570       ??_C@_0L@GDMHENGB@SymCleanup?$AA@ 0044f570     rylgamelibrary:exceptionreport.obj
 0002:0000557c       ??_C@_0O@LIDFOEPH@SymSetOptions?$AA@ 0044f57c     rylgamelibrary:exceptionreport.obj
 0002:0000558c       ??_C@_0O@MCMFENKA@SymInitialize?$AA@ 0044f58c     rylgamelibrary:exceptionreport.obj
 0002:0000559c       ??_C@_0BD@JCAKOMOK@SymGetModuleBase64?$AA@ 0044f59c     rylgamelibrary:exceptionreport.obj
 0002:000055b0       ??_C@_0BH@PMEMHADK@SymFunctionTableAccess?$AA@ 0044f5b0     rylgamelibrary:exceptionreport.obj
 0002:000055c8       ??_C@_0BF@GMMDJHID@SymGetLineFromAddr64?$AA@ 0044f5c8     rylgamelibrary:exceptionreport.obj
 0002:000055e0       ??_C@_0BD@HHOPHPBF@SymGetLineFromAddr?$AA@ 0044f5e0     rylgamelibrary:exceptionreport.obj
 0002:000055f4       ??_C@_09OJFIDCEK@StackWalk?$AA@ 0044f5f4     rylgamelibrary:exceptionreport.obj
 0002:00005600       ??_C@_0M@GHNAPHBH@SymFromAddr?$AA@ 0044f600     rylgamelibrary:exceptionreport.obj
 0002:0000560c       ??_C@_0O@HMGGMGDA@SymSetContext?$AA@ 0044f60c     rylgamelibrary:exceptionreport.obj
 0002:0000561c       ??_C@_0P@HOFLHHNH@SymEnumSymbols?$AA@ 0044f61c     rylgamelibrary:exceptionreport.obj
 0002:0000562c       ??_C@_0BC@MNIKNFKD@MiniDumpWriteDump?$AA@ 0044f62c     rylgamelibrary:exceptionreport.obj
 0002:00005640       ??_C@_0CI@JBIECDGE@Exception?5occured?5AGAIN?$CB?5EXITING@ 0044f640     rylgamelibrary:exceptionreport.obj
 0002:00005668       ??_C@_0BGD@OBDOHKCI@?9?9?9?9?9?9?9?9?9?9?9?9?9?9?9?9?9?9?9?9?9?9?9?9?9?9?9?9?9?9?9?9@ 0044f668     rylgamelibrary:exceptionreport.obj
 0002:000057cc       ??_C@_09KKJFIDEP@NTDLL?4DLL?$AA@ 0044f7cc     rylgamelibrary:exceptionreport.obj
 0002:000057d8       ??_C@_0P@FOKFNGCC@STACK_OVERFLOW?$AA@ 0044f7d8     rylgamelibrary:exceptionreport.obj
 0002:000057e8       ??_C@_0BB@PLLMBPKL@PRIV_INSTRUCTION?$AA@ 0044f7e8     rylgamelibrary:exceptionreport.obj
 0002:000057fc       ??_C@_0N@NOODLLAE@INT_OVERFLOW?$AA@ 0044f7fc     rylgamelibrary:exceptionreport.obj
 0002:0000580c       ??_C@_0BD@JEAJAPHP@INT_DIVIDE_BY_ZERO?$AA@ 0044f80c     rylgamelibrary:exceptionreport.obj
 0002:00005820       ??_C@_0O@FPLBLLBA@FLT_UNDERFLOW?$AA@ 0044f820     rylgamelibrary:exceptionreport.obj
 0002:00005830       ??_C@_0BA@GJKDALBO@FLT_STACK_CHECK?$AA@ 0044f830     rylgamelibrary:exceptionreport.obj
 0002:00005840       ??_C@_0N@BFKIPAKO@FLT_OVERFLOW?$AA@ 0044f840     rylgamelibrary:exceptionreport.obj
 0002:00005850       ??_C@_0BG@KHLFFMKF@FLT_INVALID_OPERATION?$AA@ 0044f850     rylgamelibrary:exceptionreport.obj
 0002:00005868       ??_C@_0BD@IOJOCCFC@FLT_INEXACT_RESULT?$AA@ 0044f868     rylgamelibrary:exceptionreport.obj
 0002:0000587c       ??_C@_0BD@NCECPCDC@FLT_DIVIDE_BY_ZERO?$AA@ 0044f87c     rylgamelibrary:exceptionreport.obj
 0002:00005890       ??_C@_0BF@DPHAEECF@FLT_DENORMAL_OPERAND?$AA@ 0044f890     rylgamelibrary:exceptionreport.obj
 0002:000058a8       ??_C@_0P@BJHADBBK@INVALID_HANDLE?$AA@ 0044f8a8     rylgamelibrary:exceptionreport.obj
 0002:000058b8       ??_C@_0BE@KNOGEHDH@INVALID_DISPOSITION?$AA@ 0044f8b8     rylgamelibrary:exceptionreport.obj
 0002:000058cc       ??_C@_0BJ@HONCONAA@NONCONTINUABLE_EXCEPTION?$AA@ 0044f8cc     rylgamelibrary:exceptionreport.obj
 0002:000058e8       ??_C@_0BE@PPPKHBFF@ILLEGAL_INSTRUCTION?$AA@ 0044f8e8     rylgamelibrary:exceptionreport.obj
 0002:000058fc       ??_C@_0BG@KDAKIDPK@ARRAY_BOUNDS_EXCEEDED?$AA@ 0044f8fc     rylgamelibrary:exceptionreport.obj
 0002:00005914       ??_C@_0O@EAPDGJDK@IN_PAGE_ERROR?$AA@ 0044f914     rylgamelibrary:exceptionreport.obj
 0002:00005924       ??_C@_0M@DKKFMHBE@SINGLE_STEP?$AA@ 0044f924     rylgamelibrary:exceptionreport.obj
 0002:00005930       ??_C@_0BB@KOKDBDNI@ACCESS_VIOLATION?$AA@ 0044f930     rylgamelibrary:exceptionreport.obj
 0002:00005944       ??_C@_0L@EGBPFLC@BREAKPOINT?$AA@ 0044f944     rylgamelibrary:exceptionreport.obj
 0002:00005950       ??_C@_0L@EECANHFC@GUARD_PAGE?$AA@ 0044f950     rylgamelibrary:exceptionreport.obj
 0002:0000595c       ??_C@_0BG@IKBJODCC@DATATYPE_MISALIGNMENT?$AA@ 0044f95c     rylgamelibrary:exceptionreport.obj
 0002:00005974       ??_C@_07JIINBNKP@?5?$DN?50x?$CFs?$AA@ 0044f974     rylgamelibrary:exceptionreport.obj
 0002:0000597c       ??_C@_06DBINIDAD@?5?$DN?5?$CFlf?$AA@ 0044f97c     rylgamelibrary:exceptionreport.obj
 0002:00005984       ??_C@_0L@EJHLJAAC@?5?$DN?5?$CC?$CF?431s?$CC?$AA@ 0044f984     rylgamelibrary:exceptionreport.obj
 0002:00005990       ??_C@_05LNDDMAEJ@?5?$DN?5?$CFf?$AA@ 0044f990     rylgamelibrary:exceptionreport.obj
 0002:00005998       ??_C@_05PMPGNLDE@?5?$DN?5?$CFX?$AA@ 0044f998     rylgamelibrary:exceptionreport.obj
 0002:000059a0       ??_C@_0CI@PMMCJFDC@?$AN?6?5Dump?5failed?5by?5Exception?5?3?5?$CFd@ 0044f9a0     rylgamelibrary:exceptionreport.obj
 0002:000059c8       ??_C@_02PCIJFNDE@?$AN?6?$AA@ 0044f9c8     rylgamelibrary:exceptionreport.obj
 0002:000059cc       ??_C@_02HAOIJKIC@?$CFc?$AA@ 0044f9cc     rylgamelibrary:exceptionreport.obj
 0002:000059d0       ??_C@_01CLKCMJKC@?5?$AA@   0044f9d0     rylgamelibrary:exceptionreport.obj
 0002:000059d4       ??_C@_05BFHEBJNP@?$CF02X?5?$AA@ 0044f9d4     rylgamelibrary:exceptionreport.obj
 0002:000059dc       ??_C@_03MMEAEOBL@?$DP?$DP?5?$AA@ 0044f9dc     rylgamelibrary:exceptionreport.obj
 0002:000059e0       ??_C@_03NDEAONJP@?5?5?5?$AA@ 0044f9e0     rylgamelibrary:exceptionreport.obj
 0002:000059e4       ??_C@_07IFACJFND@?$CF08lX?3?5?$AA@ 0044f9e4     rylgamelibrary:exceptionreport.obj
 0002:00005a00       ??_C@_0BFI@DGJDBGPB@?9?9?9?9?9?9?9?9?9?9?9?9?9?9?9?9?9?9?9?9?9?9?9?9?9?9?9?9?9?9?9?9@ 0044fa00     rylgamelibrary:exceptionreport.obj
 0002:00005b58       ??_C@_04FMMHFHOO@?$AN?6?$AN?6?$AA@ 0044fb58     rylgamelibrary:exceptionreport.obj
 0002:00005b60       ??_C@_0CO@FHGEDCLH@?$AN?6Stack?3?5?$CFd?5bytes?5starting?5at?5?$CIE@ 0044fb60     rylgamelibrary:exceptionreport.obj
 0002:00005b90       ??_C@_0NO@NFEOBEIG@?9?9?9?9?9?9?9?9?9?9?9?9?9?9?9?9?9?9?9?9?9?9?9?9?9?9?9?9?9?9?9?9@ 0044fb90     rylgamelibrary:exceptionreport.obj
 0002:00005c70       ??_C@_04CKCPGAJL@?5?$CFls?$AA@ 0044fc70     rylgamelibrary:exceptionreport.obj
 0002:00005c78       ??_C@_04FBKCMAJG@?8?$CFs?8?$AA@ 0044fc78     rylgamelibrary:exceptionreport.obj
 0002:00005c80       ??_C@_06JBNLAJBO@Local?5?$AA@ 0044fc80     rylgamelibrary:exceptionreport.obj
 0002:00005c88       ??_C@_0L@GAPENNGB@Parameter?5?$AA@ 0044fc88     rylgamelibrary:exceptionreport.obj
 0002:00005c94       ??_C@_0BH@LHFBFGPP@punting?5on?5symbol?5?$CFs?$AN?6?$AA@ 0044fc94     rylgamelibrary:exceptionreport.obj
 0002:00005cac       ??_C@_05OLKONLEL@?7?$CFs?$AN?6?$AA@ 0044fcac     rylgamelibrary:exceptionreport.obj
 0002:00005cc4       ??_C@_0N@FDKDKIO@?5?5?$CFs?5line?5?$CFu?$AA@ 0044fcc4     rylgamelibrary:exceptionreport.obj
 0002:00005cd4       ??_C@_0BP@MDOCJMHI@?$CF04X?3?$CF08x?5?5?5?5?5?5?5?5?5?5?5?5?5?5?5?5?5?5?5?$CFs?$AA@ 0044fcd4     rylgamelibrary:exceptionreport.obj
 0002:00005cf4       ??_C@_05OCOKLJIG@?$CF?930s?$AA@ 0044fcf4     rylgamelibrary:exceptionreport.obj
 0002:00005cfc       ??_C@_08BNBLKJHB@?$CF?9s?$CL0x?$CFp?$AA@ 0044fcfc     rylgamelibrary:exceptionreport.obj
 0002:00005d08       ??_C@_0N@ENKPPALP@?$CF08x?5?5?$CF08x?5?5?$AA@ 0044fd08     rylgamelibrary:exceptionreport.obj
 0002:00005d18       ??_C@_0PI@KDOGOOIL@?9?9?9?9?9?9?9?9?9?9?9?9?9?9?9?9?9?9?9?9?9?9?9?9?9?9?9?9?9?9?9?9@ 0044fd18     rylgamelibrary:exceptionreport.obj
 0002:00005e10       ??_C@_05BCAGPPBA@Short?$AA@ 0044fe10     rylgamelibrary:exceptionreport.obj
 0002:00005e18       ??_C@_06ILGIONGP@Detail?$AA@ 0044fe18     rylgamelibrary:exceptionreport.obj
 0002:00005e20       ??_C@_0CB@GPFNDMLJ@Failed?5to?5write?5memory?5dump?4?$AN?6?$AN?6@ 0044fe20     rylgamelibrary:exceptionreport.obj
 0002:00005e44       ??_C@_06MHMFDNCL@?$AN?6?$AN?6?$AN?6?$AA@ 0044fe44     rylgamelibrary:exceptionreport.obj
 0002:00005e4c       ??_C@_0CD@FBHEOIAD@Failed?5to?5write?5stack?5details?4?$AN?6@ 0044fe4c     rylgamelibrary:exceptionreport.obj
 0002:00005e70       ??_C@_0CE@LIFIMHE@Failed?5to?5write?5registers?5info?4?$AN@ 0044fe70     rylgamelibrary:exceptionreport.obj
 0002:00005e94       ??_C@_0CA@GFJMECCP@Failed?5to?5write?5basic?5info?4?$AN?6?$AN?6?$AA@ 0044fe94     rylgamelibrary:exceptionreport.obj
 0002:00005eb8       ??_C@_0FD@HBPKOILE@?$DN?$DN?$DN?$DN?$DN?$DN?$DN?$DN?$DN?$DN?$DN?$DN?$DN?$DN?$DN?$DN?$DN?$DN?$DN?$DN?$DN?$DN?$DN?$DN?$DN?$DN?$DN?$DN?$DN?$DN?$DN?$DN@ 0044feb8     rylgamelibrary:exceptionreport.obj
 0002:00005f10       ??_C@_0FF@PNKPFNM@?$AN?6?$AN?6?$DN?$DN?$DN?$DN?$DN?$DN?$DN?$DN?$DN?$DN?$DN?$DN?$DN?$DN?$DN?$DN?$DN?$DN?$DN?$DN?$DN?$DN?$DN?$DN?$DN?$DN?$DN?$DN@ 0044ff10     rylgamelibrary:exceptionreport.obj
 0002:00005f68       ??_C@_0DI@DPEKLHMC@Exception?5occured?5by?5UserFunc?5?3?5@ 0044ff68     rylgamelibrary:exceptionreport.obj
 0002:00005fa0       ??_C@_0MB@EDKIHAPE@?9?9?9?9?9?9?9?9?9?9?9?9?9?9?9?9?9?9?9?9?9?9?9?9?9?9?9?9?9?9?9?9@ 0044ffa0     rylgamelibrary:exceptionreport.obj
 0002:00006064       ??_C@_0CD@LJIHLANN@?5?$CF04d?9?$CF02d?9?$CF02d?5?$CF02d?0?$CF02d?0?$CF02d?4t@ 00450064     rylgamelibrary:exceptionreport.obj
 0002:00006088       ??_C@_0CD@JHBPEDNN@?5?$CF04d?9?$CF02d?9?$CF02d?5?$CF02d?0?$CF02d?0?$CF02d?4d@ 00450088     rylgamelibrary:exceptionreport.obj
 0002:000060bc       ??_C@_0M@IBNEFJCG@DBGHELP?4DLL?$AA@ 004500bc     rylgamelibrary:exceptionreport.obj
 0002:000060c8       ??_C@_04IIAJELJL@this?$AA@ 004500c8     rylgamelibrary:consolewindow.obj
 0002:000060d0       ??_C@_06MFMMLLPC@?$LB?$LM?$LI?$LC?C?$LM?$AA@ 004500d0     rylgamelibrary:consolewindow.obj
 0002:000060d8       ??_C@_0P@IIOHIDHA@window?5console?$AA@ 004500d8     rylgamelibrary:consolewindow.obj
 0002:000060e8       ??_7CConsoleWindow@@6B@    004500e8     rylgamelibrary:consolewindow.obj
 0002:000060ec       ??_C@_0CJ@FPLIJFCB@Can?8t?5recognize?5command?4?5Please?5@ 004500ec     rylgamelibrary:consolewindow.obj
 0002:00006118       ??_C@_07EKEMFJNL@LISTBOX?$AA@ 00450118     rylgamelibrary:consolewindow.obj
 0002:00006120       ??_C@_04BMCEDOKO@EDIT?$AA@ 00450120     rylgamelibrary:consolewindow.obj
 0002:00006128       ??_C@_0DB@EPMOPIA@information?5?$DN?$DN?$DN?$DN?$DN?$DN?$DN?$DN?$DN?$DN?$DN?$DN?$DN?$DN?$DN?$DN?$DN?$DN?$DN?$DN@ 00450128     rylgamelibrary:consolewindow.obj
 0002:0000615c       ??_C@_0BP@JEPDOBJN@ConsoleWindowCustomPrintOutput?$AA@ 0045015c     rylgamelibrary:consolewindow.obj
 0002:0000617c       ??_C@_0BN@PCAPNIHC@ConsoleWindowCustomPrintInfo?$AA@ 0045017c     rylgamelibrary:consolewindow.obj
 0002:0000619c       ??_7CBufferQueue@@6B@      0045019c     rylgamelibrary:bufferqueue.obj
 0002:000061a0       ??_C@_01GFHCPBMG@C?$AA@    004501a0     rylgamelibrary:regfunctions.obj
 0002:000061a4       ??_C@_08EPJLHIJG@bad?5cast?$AA@ 004501a4     rylgamelibrary:regfunctions.obj
 0002:000061b0       ??_8?$basic_ostream@DU?$char_traits@D@std@@@std@@7B@ 004501b0     rylgamelibrary:regfunctions.obj
 0002:000061d8       ?m_FastHeToBi@Convert@Math@@3QBGB 004501d8     rylgamelibrary:math.obj
 0002:000063d8       _CLSID_MSDAORA             004503d8     rylgamelibrary:oledb.obj
 0002:000063e8       _CLSID_MSDAORA_ERROR       004503e8     rylgamelibrary:oledb.obj
 0002:000063f8       _CLSID_MSDAORA8            004503f8     rylgamelibrary:oledb.obj
 0002:00006408       _CLSID_MSDAORA8_ERROR      00450408     rylgamelibrary:oledb.obj
 0002:00006418       ?CLSID_SQLOLEDB@@3U_GUID@@B 00450418     rylgamelibrary:oledb.obj
 0002:00006428       ?CLSID_SQLOLEDB_ERROR@@3U_GUID@@B 00450428     rylgamelibrary:oledb.obj
 0002:00006438       ?CLSID_SQLOLEDB_ENUMERATOR@@3U_GUID@@B 00450438     rylgamelibrary:oledb.obj
 0002:00006448       ?IID_ISQLServerErrorInfo@@3U_GUID@@B 00450448     rylgamelibrary:oledb.obj
 0002:00006458       ?IID_IRowsetFastLoad@@3U_GUID@@B 00450458     rylgamelibrary:oledb.obj
 0002:00006468       ?IID_IUMSInitialize@@3U_GUID@@B 00450468     rylgamelibrary:oledb.obj
 0002:00006478       ?IID_ISchemaLock@@3U_GUID@@B 00450478     rylgamelibrary:oledb.obj
 0002:00006488       ?DBGUID_MSSQLXML@@3U_GUID@@B 00450488     rylgamelibrary:oledb.obj
 0002:00006498       ?DBGUID_XPATH@@3U_GUID@@B  00450498     rylgamelibrary:oledb.obj
 0002:000064a8       ?IID_ISQLXMLHelper@@3U_GUID@@B 004504a8     rylgamelibrary:oledb.obj
 0002:000064b8       ?DBSCHEMA_LINKEDSERVERS@@3U_GUID@@B 004504b8     rylgamelibrary:oledb.obj
 0002:000064c8       ?DBPROPSET_SQLSERVERDATASOURCE@@3U_GUID@@B 004504c8     rylgamelibrary:oledb.obj
 0002:000064d8       ?DBPROPSET_SQLSERVERDATASOURCEINFO@@3U_GUID@@B 004504d8     rylgamelibrary:oledb.obj
 0002:000064e8       ?DBPROPSET_SQLSERVERDBINIT@@3U_GUID@@B 004504e8     rylgamelibrary:oledb.obj
 0002:000064f8       ?DBPROPSET_SQLSERVERROWSET@@3U_GUID@@B 004504f8     rylgamelibrary:oledb.obj
 0002:00006508       ?DBPROPSET_SQLSERVERSESSION@@3U_GUID@@B 00450508     rylgamelibrary:oledb.obj
 0002:00006518       ?DBPROPSET_SQLSERVERCOLUMN@@3U_GUID@@B 00450518     rylgamelibrary:oledb.obj
 0002:00006528       ?DBPROPSET_SQLSERVERSTREAM@@3U_GUID@@B 00450528     rylgamelibrary:oledb.obj
 0002:00006538       ?DBCOLUMN_SS_COMPFLAGS@@3UtagDBID@@B 00450538     rylgamelibrary:oledb.obj
 0002:00006550       ?DBCOLUMN_SS_SORTID@@3UtagDBID@@B 00450550     rylgamelibrary:oledb.obj
 0002:00006568       ?DBCOLUMN_BASETABLEINSTANCE@@3UtagDBID@@B 00450568     rylgamelibrary:oledb.obj
 0002:00006580       ?DBCOLUMN_SS_TDSCOLLATION@@3UtagDBID@@B 00450580     rylgamelibrary:oledb.obj
 0002:00006598       _CLSID_OraOLEDB            00450598     rylgamelibrary:oledb.obj
 0002:000065a8       ?CLSID_MSDASQL@@3U_GUID@@B 004505a8     rylgamelibrary:oledb.obj
 0002:000065b8       _DBGUID_DBSQL              004505b8     rylgamelibrary:oledb.obj
 0002:000065c8       _DBPROPSET_ROWSET          004505c8     rylgamelibrary:oledb.obj
 0002:000065d8       _DBPROPSET_DBINIT          004505d8     rylgamelibrary:oledb.obj
 0002:000065e8       _DB_NULLID                 004505e8     rylgamelibrary:oledb.obj
 0002:00006600       ??_7OleDB@@6B@             00450600     rylgamelibrary:oledb.obj
 0002:00006604       ??_C@_0BH@HIPKANGJ@?$FL?$CF3d?30x?$CF5x?$FN?5?$CFs?5?5?$FLM?3?$CFs?$FN?$AA@ 00450604     rylgamelibrary:oledb.obj
 0002:0000661c       ??_C@_0BD@POPGEBLJ@?$FL?$CF3d?30x?$CF5x?$FN?5?$FLM?3?$CFs?$FN?$AA@ 0045061c     rylgamelibrary:oledb.obj
 0002:00006630       ??_C@_0BO@MKAPGHN@IDBInitialize?3?3QueryInterface?$AA@ 00450630     rylgamelibrary:oledb.obj
 0002:00006650       ??_C@_0EE@DEBMFHML@IDBInitialize?5?$LP?$MA?$LK?j?A?$KH?F?$KO?$MA?G?5QueryIn@ 00450650     rylgamelibrary:oledb.obj
 0002:00006694       ??_C@_0BF@NJNCPLCA@OleDB?3?3CreateSession?$AA@ 00450694     rylgamelibrary:oledb.obj
 0002:000066b0       ??_C@_0GK@ONMIBDEF@D?3?2Work?2RYL?2Source?2v?4538?$FN?5?G?X?$LP?$NM?5?$CI@ 004506b0     rylgamelibrary:oledb.obj
 0002:0000671c       ??_C@_0DA@CNAIOJDO@IDBInitialize?5?$LP?$MA?$LK?j?A?$KH?F?$KO?$LA?$KB?5?C?J?$LB?b?H?$KN?$LF@ 0045071c     rylgamelibrary:oledb.obj
 0002:0000674c       ??_C@_0BH@OHGCFAOM@OleDB?3?3DBCreateCommand?$AA@ 0045074c     rylgamelibrary:oledb.obj
 0002:00006764       ??_C@_0CP@JBHPBEAD@CreateSession?5?$MA?$LL?5?$CFd?5?$MA?G?5?$LP?$KB?$LH?$KP?$LH?N?5?$LN?G@ 00450764     rylgamelibrary:oledb.obj
 0002:00006794       ??_C@_0CA@NDJLAIIO@IDBCreateCommand?3?3CreateSession?$AA@ 00450794     rylgamelibrary:oledb.obj
 0002:000067b4       ??_C@_0BN@PFKDKPCE@IDBProperties?3?3SetProperties?$AA@ 004507b4     rylgamelibrary:oledb.obj
 0002:000067d4       ??_C@_0BK@PPDEINAL@IDBInitialize?3?3Initialize?$AA@ 004507d4     rylgamelibrary:oledb.obj
 0002:000067f0       ??_C@_0CN@JNEJDPFK@?$LM?$LM?$LM?G?$MA?L?5?C?J?$LB?b?H?$KN?5?$LF?G?A?v?5?$LO?J?$LO?R?$LA?E?$LD?$KK?5?D?u?$LI?$KO@ 004507f0     rylgamelibrary:oledb.obj
 0002:00006820       ??_C@_0CN@CNCKLNII@IRowset?3?3Execute?5?$LG?G?$LE?B?5IRowsetCha@ 00450820     rylgamelibrary:oledb.obj
 0002:00006850       ??_C@_0BN@FJADKNCN@ICommandText?3?3SetCommandText?$AA@ 00450850     rylgamelibrary:oledb.obj
 0002:00006870       ??_C@_0CA@NDMFIGLB@IDBCreateCommand?3?3CreateCommand?$AA@ 00450870     rylgamelibrary:oledb.obj
 0002:00006890       ??_C@_0CM@GGGPFOHI@CreateCommand?5?$MA?$LL?5?$CFd?5?$MA?G?5?$LP?$KB?$LH?$KP?$LH?N?5?$LN?G@ 00450890     rylgamelibrary:oledb.obj
 0002:000068bc       ??_C@_0BK@PMLGEMHC@IAccessor?3?3CreateAccessor?$AA@ 004508bc     rylgamelibrary:oledb.obj
 0002:000068d8       ??_C@_0DA@PBNGAFHI@CreateAccessor?5?$LI?$KG?5?$CFd?5?$MA?G?5?$LP?$KB?$LH?$KP?$LH?N?5?$LN@ 004508d8     rylgamelibrary:oledb.obj
 0002:00006908       ??_C@_0BN@LMKICNAA@ICommandText?3?3QueryInterface?$AA@ 00450908     rylgamelibrary:oledb.obj
 0002:00006928       ??_C@_0CN@HEKIFNOO@QueryInterface?5?$LI?$KG?5?$CFd?5?$MA?G?5?$LP?$KB?$LH?$KP?$LH?N?5?$LN@ 00450928     rylgamelibrary:oledb.obj
 0002:00006958       ??_C@_0BN@HPDCFAHA@OleDB?3?3ExcuteQueryWithParams?$AA@ 00450958     rylgamelibrary:oledb.obj
 0002:00006978       ??_C@_0BB@IKGFPMON@IRowset?3?3GetData?$AA@ 00450978     rylgamelibrary:oledb.obj
 0002:0000698c       ??_C@_0BI@CAIJCMKB@?$LA?a?$LA?z?5?$LH?N?$LP?l?$LM?B?$MA?L?5?$LO?x?$LN?$MA?$LE?O?$LE?Y?4?$AA@ 0045098c     rylgamelibrary:oledb.obj
 0002:000069a4       ??_C@_0BF@HMMJLEKL@IRowset?3?3GetNextRows?$AA@ 004509a4     rylgamelibrary:oledb.obj
 0002:000069bc       ??_C@_0BI@GHLCGAJI@IRowset?3?3QueryInterface?$AA@ 004509bc     rylgamelibrary:oledb.obj
 0002:000069d4       ??_C@_0BL@PKCJJLE@?5?D?C?$LH?$LD?$LM?v?$LI?$KG?5?$LB?$LI?G?R?$LM?v?5?$LO?x?$LN?$MA?$LE?O?$LE?Y?4?$AA@ 004509d4     rylgamelibrary:oledb.obj
 0002:000069f0       ??_C@_0BB@IFIDCFBJ@?$LH?N?$LP?l?$LM?B?5?$LO?r?$LB?b?5?$LN?G?F?P?$AA@ 004509f0     rylgamelibrary:oledb.obj
 0002:00006a04       ??_C@_0BG@CIFIMHBD@ICommandText?3?3Execute?$AA@ 00450a04     rylgamelibrary:oledb.obj
 0002:00006a7c       ??_C@_0M@EHIIGJP@AIRSHIP_KIT?$AA@ 00450a7c     rylgamelibrary:itemconstants.obj
 0002:00006a88       ??_C@_0BE@LAGLJLGP@LONG_RANGE_ARMS_KIT?$AA@ 00450a88     rylgamelibrary:itemconstants.obj
 0002:00006a9c       ??_C@_0BF@CNNBECF@SHORT_RANGE_ARMS_KIT?$AA@ 00450a9c     rylgamelibrary:itemconstants.obj
 0002:00006ab4       ??_C@_08GFEGKDJH@CAMP_KIT?$AA@ 00450ab4     rylgamelibrary:itemconstants.obj
 0002:00006ac0       ??_C@_0N@MPEFDFMN@FIRE_CRACKER?$AA@ 00450ac0     rylgamelibrary:itemconstants.obj
 0002:00006ad0       ??_C@_08GDOHHCLK@CASHBOOK?$AA@ 00450ad0     rylgamelibrary:itemconstants.obj
 0002:00006adc       ??_C@_07GOBLFMEJ@EXPBOOK?$AA@ 00450adc     rylgamelibrary:itemconstants.obj
 0002:00006ae4       ??_C@_0O@ENKNOIIA@EVENT_LOTTERY?$AA@ 00450ae4     rylgamelibrary:itemconstants.obj
 0002:00006af4       ??_C@_0L@IDHECKJ@EVENT_DROP?$AA@ 00450af4     rylgamelibrary:itemconstants.obj
 0002:00006b00       ??_C@_06JEGAJCCP@PORTAL?$AA@ 00450b00     rylgamelibrary:itemconstants.obj
 0002:00006b08       ??_C@_04HPMOKHFE@BOLT?$AA@ 00450b08     rylgamelibrary:itemconstants.obj
 0002:00006b10       ??_C@_05CHNCNNHJ@ARROW?$AA@ 00450b10     rylgamelibrary:itemconstants.obj
 0002:00006b18       ??_C@_09JKMMAOP@ACCESSORY?$AA@ 00450b18     rylgamelibrary:itemconstants.obj
 0002:00006b24       ??_C@_0O@NKGMDDJJ@SKILL_A_KNIFE?$AA@ 00450b24     rylgamelibrary:itemconstants.obj
 0002:00006b34       ??_C@_0M@LHAJNCMF@SKILL_A_GUN?$AA@ 00450b34     rylgamelibrary:itemconstants.obj
 0002:00006b40       ??_C@_0P@JNJDLIJG@SKILL_A_ATTACK?$AA@ 00450b40     rylgamelibrary:itemconstants.obj
 0002:00006b50       ??_C@_0O@HNBOEHHD@SKILL_A_GUARD?$AA@ 00450b50     rylgamelibrary:itemconstants.obj
 0002:00006b60       ??_C@_09IJNMMIGE@OPP_SYTHE?$AA@ 00450b60     rylgamelibrary:itemconstants.obj
 0002:00006b6c       ??_C@_09LHFPJEKB@OPP_TALON?$AA@ 00450b6c     rylgamelibrary:itemconstants.obj
 0002:00006b78       ??_C@_0M@HBBCADIC@OPP_SLUSHER?$AA@ 00450b78     rylgamelibrary:itemconstants.obj
 0002:00006b84       ??_C@_07DDHBLCJN@OPP_AXE?$AA@ 00450b84     rylgamelibrary:itemconstants.obj
 0002:00006b8c       ??_C@_0L@BCKJALFM@OPP_HAMMER?$AA@ 00450b8c     rylgamelibrary:itemconstants.obj
 0002:00006b98       ??_C@_09DHKFPIKI@COM_SWORD?$AA@ 00450b98     rylgamelibrary:itemconstants.obj
 0002:00006ba4       ??_C@_09IIEFHALL@COM_BLUNT?$AA@ 00450ba4     rylgamelibrary:itemconstants.obj
 0002:00006bb0       ??_C@_06IDGLAPAH@PELVIS?$AA@ 00450bb0     rylgamelibrary:itemconstants.obj
 0002:00006bb8       ??_C@_09FEMJFDKO@PROTECT_A?$AA@ 00450bb8     rylgamelibrary:itemconstants.obj
 0002:00006bc4       ??_C@_04MEHDIIKB@BODY?$AA@ 00450bc4     rylgamelibrary:itemconstants.obj
 0002:00006bcc       ??_C@_04BINJNOJD@HEAD?$AA@ 00450bcc     rylgamelibrary:itemconstants.obj
 0002:00006bd4       ??_C@_03MCJABCEG@ETC?$AA@  00450bd4     rylgamelibrary:itemconstants.obj
 0002:00006bd8       ??_C@_04DKJDLEKC@AMMO?$AA@ 00450bd8     rylgamelibrary:itemconstants.obj
 0002:00006be0       ??_C@_03PPPKCJBG@ORE?$AA@  00450be0     rylgamelibrary:itemconstants.obj
 0002:00006be4       ??_C@_04HANHHAFD@RUNE?$AA@ 00450be4     rylgamelibrary:itemconstants.obj
 0002:00006bec       ??_C@_03OLPODOAE@GEM?$AA@  00450bec     rylgamelibrary:itemconstants.obj
 0002:00006bf0       ??_C@_09FGHNCELF@SKILLBOOK?$AA@ 00450bf0     rylgamelibrary:itemconstants.obj
 0002:00006bfc       ??_C@_04FOKJBMGD@TRAP?$AA@ 00450bfc     rylgamelibrary:itemconstants.obj
 0002:00006c04       ??_C@_06CGCPEDIN@POISON?$AA@ 00450c04     rylgamelibrary:itemconstants.obj
 0002:00006c0c       ??_C@_06IBPLKHEF@POTION?$AA@ 00450c0c     rylgamelibrary:itemconstants.obj
 0002:00006c14       ??_C@_08DPNOGIMP@NECKLACE?$AA@ 00450c14     rylgamelibrary:itemconstants.obj
 0002:00006c20       ??_C@_04FICOPKPG@RING?$AA@ 00450c20     rylgamelibrary:itemconstants.obj
 0002:00006c28       ??_C@_05PLFAKKIE@CLOAK?$AA@ 00450c28     rylgamelibrary:itemconstants.obj
 0002:00006c30       ??_C@_06IHBJDHDI@SHIELD?$AA@ 00450c30     rylgamelibrary:itemconstants.obj
 0002:00006c38       ??_C@_06EBPDMAC@DAGGER?$AA@ 00450c38     rylgamelibrary:itemconstants.obj
 0002:00006c40       ??_C@_05PICIGLKH@STAFF?$AA@ 00450c40     rylgamelibrary:itemconstants.obj
 0002:00006c48       ??_C@_08BBCBHLCC@CROSSBOW?$AA@ 00450c48     rylgamelibrary:itemconstants.obj
 0002:00006c54       ??_C@_03GBJKLBDL@BOW?$AA@  00450c54     rylgamelibrary:itemconstants.obj
 0002:00006c58       ??_C@_0BA@IGICPGDL@TWOHANDED_SWORD?$AA@ 00450c58     rylgamelibrary:itemconstants.obj
 0002:00006c68       ??_C@_0O@HECJOKAO@TWOHANDED_AXE?$AA@ 00450c68     rylgamelibrary:itemconstants.obj
 0002:00006c78       ??_C@_0BA@DJGCHOCI@TWOHANDED_BLUNT?$AA@ 00450c78     rylgamelibrary:itemconstants.obj
 0002:00006c88       ??_C@_0O@IEAGKJNM@ONEHANDED_AXE?$AA@ 00450c88     rylgamelibrary:itemconstants.obj
 0002:00006c98       ??_C@_0BA@GFLJDJLA@ONEHANDED_BLUNT?$AA@ 00450c98     rylgamelibrary:itemconstants.obj
 0002:00006ca8       ??_C@_0BA@NKFJLBKD@ONEHANDED_SWORD?$AA@ 00450ca8     rylgamelibrary:itemconstants.obj
 0002:00006cb8       ??_C@_05OPFKPKDD@BOOTS?$AA@ 00450cb8     rylgamelibrary:itemconstants.obj
 0002:00006cc0       ??_C@_05OHCLHAOJ@GLOVE?$AA@ 00450cc0     rylgamelibrary:itemconstants.obj
 0002:00006cc8       ??_C@_06EAEHPAKO@ARMOUR?$AA@ 00450cc8     rylgamelibrary:itemconstants.obj
 0002:00006cd0       ??_C@_05PGAFNBIB@TUNIC?$AA@ 00450cd0     rylgamelibrary:itemconstants.obj
 0002:00006cd8       ??_C@_05PLFHECLE@SHIRT?$AA@ 00450cd8     rylgamelibrary:itemconstants.obj
 0002:00006ce0       ??_C@_04MBMDPGIJ@HELM?$AA@ 00450ce0     rylgamelibrary:itemconstants.obj
 0002:00006ce8       ??_C@_06LOOCOLAA@WISAdd?$AA@ 00450ce8     rylgamelibrary:itemconstants.obj
 0002:00006cf0       ??_C@_06CGCGOADL@INTAdd?$AA@ 00450cf0     rylgamelibrary:itemconstants.obj
 0002:00006cf8       ??_C@_06GDFKODPD@CONAdd?$AA@ 00450cf8     rylgamelibrary:itemconstants.obj
 0002:00006d00       ??_C@_06OIMGJMDJ@DEXAdd?$AA@ 00450d00     rylgamelibrary:itemconstants.obj
 0002:00006d08       ??_C@_06MIIFPHOG@STRAdd?$AA@ 00450d08     rylgamelibrary:itemconstants.obj
 0002:00006d10       ??_C@_0BB@PABLDCHP@PoisonResistance?$AA@ 00450d10     rylgamelibrary:itemconstants.obj
 0002:00006d24       ??_C@_0BA@GPBDDKHD@DrainResistance?$AA@ 00450d24     rylgamelibrary:itemconstants.obj
 0002:00006d34       ??_C@_0P@OHOLLMHH@ColdResistance?$AA@ 00450d34     rylgamelibrary:itemconstants.obj
 0002:00006d44       ??_C@_0BE@GPGAPLKE@LightningResistance?$AA@ 00450d44     rylgamelibrary:itemconstants.obj
 0002:00006d58       ??_C@_0P@PJOKKPEP@FireResistance?$AA@ 00450d58     rylgamelibrary:itemconstants.obj
 0002:00006d68       ??_C@_0BA@OEDKABIE@PoisonAttribute?$AA@ 00450d68     rylgamelibrary:itemconstants.obj
 0002:00006d78       ??_C@_0P@FDNGKIMC@DrainAttribute?$AA@ 00450d78     rylgamelibrary:itemconstants.obj
 0002:00006d88       ??_C@_0O@KDAKEKBK@ColdAttribute?$AA@ 00450d88     rylgamelibrary:itemconstants.obj
 0002:00006d98       ??_C@_0BC@PDKFBDII@LightingAttribute?$AA@ 00450d98     rylgamelibrary:itemconstants.obj
 0002:00006dac       ??_C@_0O@KDOLBKII@FireAttribute?$AA@ 00450dac     rylgamelibrary:itemconstants.obj
 0002:00006dbc       ??_C@_07IJHMPIE@MPRegen?$AA@ 00450dbc     rylgamelibrary:itemconstants.obj
 0002:00006dc4       ??_C@_07EAHHMBOA@HPRegen?$AA@ 00450dc4     rylgamelibrary:itemconstants.obj
 0002:00006dcc       ??_C@_09OAHBMAHD@MpMaxPlus?$AA@ 00450dcc     rylgamelibrary:itemconstants.obj
 0002:00006dd8       ??_C@_09GFIALDH@HpMaxPlus?$AA@ 00450dd8     rylgamelibrary:itemconstants.obj
 0002:00006de4       ??_C@_0BA@KHMKMKDF@LongRangeAttack?$AA@ 00450de4     rylgamelibrary:itemconstants.obj
 0002:00006df4       ??_C@_0M@GJIHNJEK@AttackRange?$AA@ 00450df4     rylgamelibrary:itemconstants.obj
 0002:00006e00       ??_C@_09HHOHJEHG@MoveSpeed?$AA@ 00450e00     rylgamelibrary:itemconstants.obj
 0002:00006e0c       ??_C@_0M@DCMFNGPD@AttackSpeed?$AA@ 00450e0c     rylgamelibrary:itemconstants.obj
 0002:00006e18       ??_C@_0BD@KKOCDHPN@BlockingPercentage?$AA@ 00450e18     rylgamelibrary:itemconstants.obj
 0002:00006e2c       ??_C@_0L@OFGNBAHF@Resistance?$AA@ 00450e2c     rylgamelibrary:itemconstants.obj
 0002:00006e38       ??_C@_0BA@OEKPEMHI@DefenceRevision?$AA@ 00450e38     rylgamelibrary:itemconstants.obj
 0002:00006e48       ??_C@_07OIBJPBBC@Defence?$AA@ 00450e48     rylgamelibrary:itemconstants.obj
 0002:00006e50       ??_C@_0BA@KPAJANLM@OffenceRevision?$AA@ 00450e50     rylgamelibrary:itemconstants.obj
 0002:00006e60       ??_C@_03HOKBAJJB@DRC?$AA@  00450e60     rylgamelibrary:itemconstants.obj
 0002:00006e64       ??_C@_09IHFKOIBD@MaxDamage?$AA@ 00450e64     rylgamelibrary:itemconstants.obj
 0002:00006e70       ??_C@_09IGFGHCKH@MinDamage?$AA@ 00450e70     rylgamelibrary:itemconstants.obj
 0002:00006e7c       ??_C@_0BD@NKDHJCOG@CriticalPercentage?$AA@ 00450e7c     rylgamelibrary:itemconstants.obj
 0002:00006e90       ??_C@_0N@IHAKLPFE@CriticalType?$AA@ 00450e90     rylgamelibrary:itemconstants.obj
 0002:00006ea0       ??_C@_04OHJIHAFH@None?$AA@ 00450ea0     rylgamelibrary:itemconstants.obj
 0002:00006ea8       ??_C@_04LKJAOKIP@RARE?$AA@ 00450ea8     rylgamelibrary:itemconstants.obj
 0002:00006eb0       ??_C@_08IOCCELMA@ENHANCED?$AA@ 00450eb0     rylgamelibrary:itemconstants.obj
 0002:00006ebc       ??_C@_06IOJAGNKJ@NORMAL?$AA@ 00450ebc     rylgamelibrary:itemconstants.obj
 0002:00006ee4       ??_C@_0L@LDJKHCPF@ReadString?$AA@ 00450ee4     rylgamelibrary:itemdataparser.obj
 0002:00006ef0       ??_C@_0HI@MDHPFBPL@D?3?2Work?2RYL?2Source?2v?4538?$FN?5?G?X?$LP?$NM?5?$CI@ 00450ef0     rylgamelibrary:itemdataparser.obj
 0002:00006f68       ??_C@_0EA@BFLPDPKF@?$LJ?v?F?$NL?5?$LB?f?$MA?L?$LA?$KB?5?$LI?p?$MA?Z?$LG?s?$LM?$KN?0?5?$LF?$KF?$MA?L?E?M?$LI?$KG?5?$MA@ 00450f68     rylgamelibrary:itemdataparser.obj
 0002:00006fa8       ??_C@_06HFKIEEBB@ReadID?$AA@ 00450fa8     rylgamelibrary:itemdataparser.obj
 0002:00006fb0       ??_C@_0EH@DPNPKBEM@?$LO?F?$MA?L?E?$NL?5ID?$LA?$KB?5?$MA?L?$LL?s?G?U?$LE?O?$LE?Y?4?50?$MA?L?$LD?$KK?50x@ 00450fb0     rylgamelibrary:itemdataparser.obj
 0002:00006ff8       ??_C@_08DGLFEHHG@CraftExp?$AA@ 00450ff8     rylgamelibrary:itemdataparser.obj
 0002:00007004       ??_C@_08CILFBKK@WISLimit?$AA@ 00451004     rylgamelibrary:itemdataparser.obj
 0002:00007010       ??_C@_08KJOLPPNO@INTLimit?$AA@ 00451010     rylgamelibrary:itemdataparser.obj
 0002:0000701c       ??_C@_08DDMBLGFO@CONLimit?$AA@ 0045101c     rylgamelibrary:itemdataparser.obj
 0002:00007028       ??_C@_08MCGOGOKL@DEXLimit?$AA@ 00451028     rylgamelibrary:itemdataparser.obj
 0002:00007034       ??_C@_08BOKOCPOI@STRLimit?$AA@ 00451034     rylgamelibrary:itemdataparser.obj
 0002:00007040       ??_C@_0L@BOBIELG@LevelLimit?$AA@ 00451040     rylgamelibrary:itemdataparser.obj
 0002:0000704c       ??_C@_0BA@JOMCHEKH@SkillLimitLevel?$AA@ 0045104c     rylgamelibrary:itemdataparser.obj
 0002:0000705c       ??_C@_0P@KMDHGBKC@SkillLimitType?$AA@ 0045105c     rylgamelibrary:itemdataparser.obj
 0002:0000706c       ??_C@_0L@INOPKAIJ@ClassLimit?$AA@ 0045106c     rylgamelibrary:itemdataparser.obj
 0002:00007078       ??_C@_0O@BJPKLJCM@MaxDurability?$AA@ 00451078     rylgamelibrary:itemdataparser.obj
 0002:00007088       ??_C@_0L@KEKGACHM@Durability?$AA@ 00451088     rylgamelibrary:itemdataparser.obj
 0002:00007094       ??_C@_0M@MMHOGIPI@OptionLimit?$AA@ 00451094     rylgamelibrary:itemdataparser.obj
 0002:000070a0       ??_C@_0L@HEBLGKJJ@MedalPrice?$AA@ 004510a0     rylgamelibrary:itemdataparser.obj
 0002:000070ac       ??_C@_0L@NGODMJCJ@BlackPrice?$AA@ 004510ac     rylgamelibrary:itemdataparser.obj
 0002:000070b8       ??_C@_05NFJELHBG@Price?$AA@ 004510b8     rylgamelibrary:itemdataparser.obj
 0002:000070c0       ??_C@_08NNKIOIN@TypeName?$AA@ 004510c0     rylgamelibrary:itemdataparser.obj
 0002:000070cc       ??_C@_08LJOGMPAO@ItemType?$AA@ 004510cc     rylgamelibrary:itemdataparser.obj
 0002:000070d8       ??_C@_09EBLHEKMK@ItemLevel?$AA@ 004510d8     rylgamelibrary:itemdataparser.obj
 0002:000070e4       ??_C@_0M@JGIEMEFF@EffectSound?$AA@ 004510e4     rylgamelibrary:itemdataparser.obj
 0002:000070f0       ??_C@_05HBOCJOBH@SizeY?$AA@ 004510f0     rylgamelibrary:itemdataparser.obj
 0002:000070f8       ??_C@_05GIPJKPFG@SizeX?$AA@ 004510f8     rylgamelibrary:itemdataparser.obj
 0002:00007100       ??_C@_04CLLPNLIJ@MaxY?$AA@ 00451100     rylgamelibrary:itemdataparser.obj
 0002:00007108       ??_C@_04DCKEOKMI@MaxX?$AA@ 00451108     rylgamelibrary:itemdataparser.obj
 0002:00007110       ??_C@_04PGKACMKE@MinY?$AA@ 00451110     rylgamelibrary:itemdataparser.obj
 0002:00007118       ??_C@_04OPLLBNOF@MinX?$AA@ 00451118     rylgamelibrary:itemdataparser.obj
 0002:00007120       ??_C@_09HNLMKFMH@SpriteDDS?$AA@ 00451120     rylgamelibrary:itemdataparser.obj
 0002:0000712c       ??_C@_0BC@PIPOFCOB@AttachedModelName?$AA@ 0045112c     rylgamelibrary:itemdataparser.obj
 0002:00007140       ??_C@_0P@BKHEPPBI@FieldModelName?$AA@ 00451140     rylgamelibrary:itemdataparser.obj
 0002:00007150       ??_C@_08BCOFAPHO@ItemName?$AA@ 00451150     rylgamelibrary:itemdataparser.obj
 0002:0000715c       ??_C@_02OLOABKKD@ID?$AA@   0045115c     rylgamelibrary:itemdataparser.obj
 0002:00007160       ??_C@_0N@FGNJFPLJ@MaxSocketNum?$AA@ 00451160     rylgamelibrary:itemdataparser.obj
 0002:00007170       ??_C@_0O@BKEDKOKD@MaterialValue?$AA@ 00451170     rylgamelibrary:itemdataparser.obj
 0002:00007658       ??_7CItem@Item@@6B@        00451658     rylgamelibrary:item.obj
 0002:00007664       ??_C@_0BJ@FIEOEILC@Item?3?3CItem?3?3SerializeIn?$AA@ 00451664     rylgamelibrary:item.obj
 0002:00007680       ??_C@_0GO@FHAJMHEH@D?3?2Work?2RYL?2Source?2v?4538?$FN?5?G?X?$LP?$NM?5?$CI@ 00451680     rylgamelibrary:item.obj
 0002:000076f0       ??_C@_0JF@PBICLFOP@SerializeIn?$LP?$KB?5?$LN?G?F?P?G?$NP?$LN?$MA?$LE?O?$LE?Y?4?5?$LO?F?$MA?L@ 004516f0     rylgamelibrary:item.obj
 0002:00007788       ??_7CUseItem@Item@@6B@     00451788     rylgamelibrary:item.obj
 0002:00007794       __real@3f800000            00451794     rylgamelibrary:item.obj
 0002:00007798       ??_7CEquipment@Item@@6B@   00451798     rylgamelibrary:item.obj
 0002:000077a4       __real@4f800000            004517a4     rylgamelibrary:item.obj
 0002:000077a8       ?INVALID_TIMER_ID@CTimerProcMgr@@2IB 004517a8     rylgamelibrary:timerproc.obj
 0002:000077ac       ?INVALID_PROC_ID@CTimerProcMgr@@2IB 004517ac     rylgamelibrary:timerproc.obj
 0002:000077b0       ??_C@_0O@CNIBGEND@CTimerProcMgr?$AA@ 004517b0     rylgamelibrary:timerproc.obj
 0002:000077c0       ??_C@_0BG@OFMDMFJA@CSysTrayNotifyMessage?$AA@ 004517c0     rylgamelibrary:systray.obj
 0002:000077d8       ??_C@_0BB@PGBHBBCL@Temp?5Application?$AA@ 004517d8     rylgamelibrary:systray.obj
 0002:000077f0       ??_C@_0EJ@MMCFMKJC@Time?5Overflow?5?3?5Elapsed?5time?5is?5@ 004517f0     rylgamelibrary:pulse.obj
 0002:0000783c       ??_C@_0BD@HKCBNPPL@CPulse?3?3CheckSleep?$AA@ 0045183c     rylgamelibrary:pulse.obj
 0002:00007850       ??_C@_0HK@GMPKGEBL@D?3?2Work?2RYL?2Source?2v?4538?$FN?5?G?X?$LP?$NM?5?$CI@ 00451850     rylgamelibrary:pulse.obj
 0002:000078cc       ??_C@_0O@CBEIMIGK@Traffic?5is?5?$CFu?$AA@ 004518cc     rylgamelibrary:pulse.obj
 0002:000078dc       ??_7CIOWorker@@6B@         004518dc     rylgamelibrary:ioworker.obj
 0002:000078e8       ??_7CCompletionHandler@@6B@ 004518e8     rylgamelibrary:completionhandler.obj
 0002:000078ec       ??_C@_0BF@FJABJDFD@?$CFc?$CFc?$CFc?$CFc?$CFc?$CFc?$CFc?$CFc?$CFc?$CFc?$AA@ 004518ec     rylgamelibrary:gzio.obj
 0002:00007904       ??_C@_05DOIEBMOI@1?41?44?$AA@ 00451904     rylgamelibrary:gzio.obj
 0002:00007910       ?BitFields@CXORCrypt@@0QAY19CI@$$CBEA 00451910     rylgamelibrary:xorcryptocodelist.obj
 0002:00007c50       ??_7CNullItem@Item@@6B@    00451c50     rylgamelibrary:itemcontainer.obj
 0002:00007c7c       ??_C@_0BO@MEDEEJIF@?4?1Script?1Game?1SkillScript?4txt?$AA@ 00451c7c     rylgamelibrary:skillmgr.obj
 0002:00008560       ??_C@_0CE@JMLOMCJM@?4?1Script?1Game?1VirtualAreaScript?4@ 00452560     rylgamelibrary:characterfight.obj
 0002:000085a8       _deflate_copyright         004525a8     rylgamelibrary:deflate.obj
 0002:0000865c       ??_C@_0BA@MOKMMFOD@need?5dictionary?$AA@ 0045265c     rylgamelibrary:inflate.obj
 0002:00008a70       ??_C@_0BF@CJFPCCEG@incompatible?5version?$AA@ 00452a70     rylgamelibrary:zutil.obj
 0002:00008a88       ??_C@_0N@DFPGLBGC@buffer?5error?$AA@ 00452a88     rylgamelibrary:zutil.obj
 0002:00008a98       ??_C@_0BE@OGGJBMCE@insufficient?5memory?$AA@ 00452a98     rylgamelibrary:zutil.obj
 0002:00008aac       ??_C@_0L@HAHMBNLP@data?5error?$AA@ 00452aac     rylgamelibrary:zutil.obj
 0002:00008ab8       ??_C@_0N@MKKNPMJD@stream?5error?$AA@ 00452ab8     rylgamelibrary:zutil.obj
 0002:00008ac8       ??_C@_0L@KIJFAKBJ@file?5error?$AA@ 00452ac8     rylgamelibrary:zutil.obj
 0002:00008ad4       ??_C@_0L@FNAOCBOG@stream?5end?$AA@ 00452ad4     rylgamelibrary:zutil.obj
 0002:00008b00       ??_C@_0P@GHFPNOJB@bad?5allocation?$AA@ 00452b00     rylgamelibrary:creaturemanager.obj
 0002:00008b30       ??_C@_04BLNHNEEM@ITEM?$AA@ 00452b30     rylgamelibrary:skillstructure.obj
 0002:00008b38       ??_C@_07IJKAIOLD@ENCHANT?$AA@ 00452b38     rylgamelibrary:skillstructure.obj
 0002:00008b40       ??_C@_05CIAJDCNE@CHANT?$AA@ 00452b40     rylgamelibrary:skillstructure.obj
 0002:00008b48       ??_C@_04LFALBNJK@CAST?$AA@ 00452b48     rylgamelibrary:skillstructure.obj
 0002:00008b50       ??_C@_08DDHIOBDH@INSTANCE?$AA@ 00452b50     rylgamelibrary:skillstructure.obj
 0002:00008b5c       ??_C@_07NLANJMCK@PASSIVE?$AA@ 00452b5c     rylgamelibrary:skillstructure.obj
 0002:00008b64       ??_C@_04OKGDLNCL@NONE?$AA@ 00452b64     rylgamelibrary:skillstructure.obj
 0002:00008b6c       ??_C@_08ENCLJPPP@WITHCLOW?$AA@ 00452b6c     rylgamelibrary:skillstructure.obj
 0002:00008b78       ??_C@_08OIOAFMHI@KNIFEARM?$AA@ 00452b78     rylgamelibrary:skillstructure.obj
 0002:00008b84       ??_C@_06FBPIOANE@GUNARM?$AA@ 00452b84     rylgamelibrary:skillstructure.obj
 0002:00008b8c       ??_C@_09NOALINMI@ATTACKARM?$AA@ 00452b8c     rylgamelibrary:skillstructure.obj
 0002:00008b98       ??_C@_0L@HANBPJDH@WITHWEAPON?$AA@ 00452b98     rylgamelibrary:skillstructure.obj
 0002:00008ba4       ??_C@_08LJMNKFEL@GUARDARM?$AA@ 00452ba4     rylgamelibrary:skillstructure.obj
 0002:00008bb0       ??_C@_07OPAJNJFO@LEFTARM?$AA@ 00452bb0     rylgamelibrary:skillstructure.obj
 0002:00008bb8       ??_C@_06BBJJECFA@RANGED?$AA@ 00452bb8     rylgamelibrary:skillstructure.obj
 0002:00008bc0       ??_C@_0BD@CKPFJJIF@WITHTHROWINGDAGGER?$AA@ 00452bc0     rylgamelibrary:skillstructure.obj
 0002:00008bd4       ??_C@_0L@BEBIHPHP@WITHDAGGER?$AA@ 00452bd4     rylgamelibrary:skillstructure.obj
 0002:00008be0       ??_C@_0O@GIECCIMB@FORALLONEHAND?$AA@ 00452be0     rylgamelibrary:skillstructure.obj
 0002:00008bf0       ??_C@_0BC@IJCNCJKH@FORFIGHTERTWOHAND?$AA@ 00452bf0     rylgamelibrary:skillstructure.obj
 0002:00008c04       ??_C@_0L@JHBOHEEF@WITHSHIELD?$AA@ 00452c04     rylgamelibrary:skillstructure.obj
 0002:00008c10       ??_C@_0L@GHJMJCPG@FORFIGHTER?$AA@ 00452c10     rylgamelibrary:skillstructure.obj
 0002:00008c1c       ??_C@_03GGLMKPCA@WIS?$AA@  00452c1c     rylgamelibrary:skillstructure.obj
 0002:00008c20       ??_C@_03JMHEAPMO@INT?$AA@  00452c20     rylgamelibrary:skillstructure.obj
 0002:00008c24       ??_C@_03ECCGHPEG@CON?$AA@  00452c24     rylgamelibrary:skillstructure.obj
 0002:00008c28       ??_C@_03MOPOHHPO@DEX?$AA@  00452c28     rylgamelibrary:skillstructure.obj
 0002:00008c2c       ??_C@_03OEDLDJBF@STR?$AA@  00452c2c     rylgamelibrary:skillstructure.obj
 0002:00008c30       ??_C@_06PAMMPOIB@SUMMON?$AA@ 00452c30     rylgamelibrary:skillstructure.obj
 0002:00008c38       ??_C@_06MNOHKIDG@ENLINE?$AA@ 00452c38     rylgamelibrary:skillstructure.obj
 0002:00008c40       ??_C@_06GPOIJMJJ@FREXME?$AA@ 00452c40     rylgamelibrary:skillstructure.obj
 0002:00008c48       ??_C@_05EGOIIAAK@PARTY?$AA@ 00452c48     rylgamelibrary:skillstructure.obj
 0002:00008c50       ??_C@_05EMJEJFOB@ENOBJ?$AA@ 00452c50     rylgamelibrary:skillstructure.obj
 0002:00008c58       ??_C@_05GPBAJNMM@FROBJ?$AA@ 00452c58     rylgamelibrary:skillstructure.obj
 0002:00008c60       ??_C@_06KFAGCKDD@ENDEAD?$AA@ 00452c60     rylgamelibrary:skillstructure.obj
 0002:00008c68       ??_C@_06OAPKPCEO@FRDEAD?$AA@ 00452c68     rylgamelibrary:skillstructure.obj
 0002:00008c70       ??_C@_05EJJKHDCK@ENEMY?$AA@ 00452c70     rylgamelibrary:skillstructure.obj
 0002:00008c78       ??_C@_06BDDGHBMC@FRIEND?$AA@ 00452c78     rylgamelibrary:skillstructure.obj
 0002:00008c80       ??_C@_05EHHFIDDJ@MELEE?$AA@ 00452c80     rylgamelibrary:skillstructure.obj
 0002:00008cc8       ?ms_fToAngle@CNetworkPos@@0MB 00452cc8     rylgamelibrary:charmovepacket.obj
 0002:00008ccc       ?ms_fToRadian@CNetworkPos@@0MB 00452ccc     rylgamelibrary:charmovepacket.obj
 0002:00008cd0       ?ms_fPositionDetail@CNetworkPos@@0MB 00452cd0     rylgamelibrary:charmovepacket.obj
 0002:00008cd4       ?ms_fVelocityDetail@CNetworkPos@@0MB 00452cd4     rylgamelibrary:charmovepacket.obj
 0002:00008d64       ??_C@_0CD@OAJLOPEC@?4?1Script?1Game?1MonsterProtoType?4t@ 00452d64     rylgamelibrary:monstermgr.obj
 0002:00008f0c       ??_C@_0BP@OEKBIFBL@?4?1Script?1Game?1LotteryEvent?4txt?$AA@ 00452f0c     rylgamelibrary:lotteryevent.obj
 0002:0000f7ec       ??_C@_04LOAJBDKD@true?$AA@ 004597ec     rylgamelibrary:cellmanager.obj
 0002:0000f7f4       ??_C@_01DDCIFGEA@E?$AA@    004597f4     rylgamelibrary:cellmanager.obj
 0002:0000fe80       __dist_code                00459e80     rylgamelibrary:trees.obj
 0002:00010080       __length_code              0045a080     rylgamelibrary:trees.obj
 0002:00010e60       ??_C@_0BM@FHLLGLAD@?4?1Script?1Game?1NPCScript?4mcf?$AA@ 0045ae60     rylgamelibrary:npc.obj
 0002:00010e7c       ??_C@_0BI@FKDKJABB@?4?1Script?1Game?1Quest?4mcf?$AA@ 0045ae7c     rylgamelibrary:npc.obj
 0002:00010eb8       _inflate_copyright         0045aeb8     rylgamelibrary:inftrees.obj
 0002:000110f8       ??_C@_0BO@HOLEOJEB@?4?1Script?1Game?1MonsterChat?4gsf?$AA@ 0045b0f8     rylgamelibrary:monstershout.obj
 0002:00011258       ??_C@_0BF@PIKDIMG@Error?5?$CIline?5?$CFd?$CJ?5?3?5?$CFs?$AA@ 0045b258     rylgamelibrary:message.obj
 0002:00011270       ??_C@_0BH@CIPFEPIL@Warning?5?$CIline?5?$CFd?$CJ?5?3?5?$CFs?$AA@ 0045b270     rylgamelibrary:message.obj
 0002:00011288       ??_C@_0BJ@BPABAGHJ@Script?5System?5Error?5?3?5?$CFs?$AA@ 0045b288     rylgamelibrary:message.obj
 0002:000112a4       ??_C@_0BG@HHPCJAJP@TYPE_POSTFIXDECREMENT?$AA@ 0045b2a4     rylgamelibrary:syntaxtree.obj
 0002:000112bc       ??_C@_0BG@FJIFPC@TYPE_POSTFIXINCREMENT?$AA@ 0045b2bc     rylgamelibrary:syntaxtree.obj
 0002:000112d4       ??_C@_0BD@MDNHJFGP@TYPE_FUNCTION_CALL?$AA@ 0045b2d4     rylgamelibrary:syntaxtree.obj
 0002:000112e8       ??_C@_0BE@CGKIGJFO@TYPE_ARRAY_INDEXING?$AA@ 0045b2e8     rylgamelibrary:syntaxtree.obj
 0002:000112fc       ??_C@_0BF@MENDOHB@TYPE_PREFIXDECREMENT?$AA@ 0045b2fc     rylgamelibrary:syntaxtree.obj
 0002:00011314       ??_C@_0BF@HLOGCLBM@TYPE_PREFIXINCREMENT?$AA@ 0045b314     rylgamelibrary:syntaxtree.obj
 0002:0001132c       ??_C@_0BH@FDMGKMKA@TYPE_COMPOUND_REMINDER?$AA@ 0045b32c     rylgamelibrary:syntaxtree.obj
 0002:00011344       ??_C@_0BH@DPJABJEF@TYPE_COMPOUND_DIVISION?$AA@ 0045b344     rylgamelibrary:syntaxtree.obj
 0002:0001135c       ??_C@_0BN@KNDGNILD@TYPE_COMPOUND_MULTIPLICATION?$AA@ 0045b35c     rylgamelibrary:syntaxtree.obj
 0002:0001137c       ??_C@_0BK@ODAPBNOD@TYPE_COMPOUND_SUBTRACTION?$AA@ 0045b37c     rylgamelibrary:syntaxtree.obj
 0002:00011398       ??_C@_0BH@KMGDBICM@TYPE_COMPOUND_ADDITION?$AA@ 0045b398     rylgamelibrary:syntaxtree.obj
 0002:000113b0       ??_C@_0BJ@LPIMCONP@TYPE_REMINDER_EXPRESSION?$AA@ 0045b3b0     rylgamelibrary:syntaxtree.obj
 0002:000113cc       ??_C@_0BJ@HDNOMEP@TYPE_DIVISION_EXPRESSION?$AA@ 0045b3cc     rylgamelibrary:syntaxtree.obj
 0002:000113e8       ??_C@_0BP@MMKEKLJF@TYPE_MULTIPLICATION_EXPRESSION?$AA@ 0045b3e8     rylgamelibrary:syntaxtree.obj
 0002:00011408       ??_C@_0BM@IIJHGLN@TYPE_SUBTRACTION_EXPRESSION?$AA@ 0045b408     rylgamelibrary:syntaxtree.obj
 0002:00011424       ??_C@_0BJ@MNBCGDIB@TYPE_ADDITION_EXPRESSION?$AA@ 0045b424     rylgamelibrary:syntaxtree.obj
 0002:00011440       ??_C@_0CA@LJNAKFON@TYPE_MORETHANOREQUAL_EXPRESSION?$AA@ 0045b440     rylgamelibrary:syntaxtree.obj
 0002:00011460       ??_C@_0CA@PNOCGFBM@TYPE_LESSTHANOREQUAL_EXPRESSION?$AA@ 0045b460     rylgamelibrary:syntaxtree.obj
 0002:00011480       ??_C@_0BJ@HDHEMDOC@TYPE_MORETHAN_EXPRESSION?$AA@ 0045b480     rylgamelibrary:syntaxtree.obj
 0002:0001149c       ??_C@_0BJ@DEDBHLEE@TYPE_LESSTHAN_EXPRESSION?$AA@ 0045b49c     rylgamelibrary:syntaxtree.obj
 0002:000114b8       ??_C@_0BJ@MBMIPOOI@TYPE_NOTEQAUL_EXPRESSION?$AA@ 0045b4b8     rylgamelibrary:syntaxtree.obj
 0002:000114d4       ??_C@_0BJ@PMBMJNNN@TYPE_EQUALITY_EXPRESSION?$AA@ 0045b4d4     rylgamelibrary:syntaxtree.obj
 0002:000114f0       ??_C@_0BE@FPMLJAKN@TYPE_NOT_EXPRESSION?$AA@ 0045b4f0     rylgamelibrary:syntaxtree.obj
 0002:00011504       ??_C@_0BE@CCELBEJM@TYPE_AND_EXPRESSION?$AA@ 0045b504     rylgamelibrary:syntaxtree.obj
 0002:00011518       ??_C@_0BD@HCPKMAMO@TYPE_OR_EXPRESSION?$AA@ 0045b518     rylgamelibrary:syntaxtree.obj
 0002:0001152c       ??_C@_0BK@EPOIOJFH@TYPE_ASSIGNMENT_EXPESSION?$AA@ 0045b52c     rylgamelibrary:syntaxtree.obj
 0002:00011548       ??_C@_0BF@FCCKPJMB@TYPE_EXPRESSION_LIST?$AA@ 0045b548     rylgamelibrary:syntaxtree.obj
 0002:00011560       ??_C@_0BJ@EGANOAIH@TYPE_CONSTANT_EXPRESSION?$AA@ 0045b560     rylgamelibrary:syntaxtree.obj
 0002:0001157c       ??_C@_0BJ@DHOAAOJP@TYPE_FUNCTION_DEFINITION?$AA@ 0045b57c     rylgamelibrary:syntaxtree.obj
 0002:00011598       ??_C@_0BK@FLHMADMP@TYPE_ARGUMENT_DECLARATION?$AA@ 0045b598     rylgamelibrary:syntaxtree.obj
 0002:000115b4       ??_C@_0BP@ELLONFCL@TYPE_ARGUMENT_DECLARATION_LIST?$AA@ 0045b5b4     rylgamelibrary:syntaxtree.obj
 0002:000115d4       ??_C@_0BG@DCKOGCDE@TYPE_INITIALIZER_LIST?$AA@ 0045b5d4     rylgamelibrary:syntaxtree.obj
 0002:000115ec       ??_C@_0BK@PBPIKNDD@TYPE_FUNCTION_DECLARATION?$AA@ 0045b5ec     rylgamelibrary:syntaxtree.obj
 0002:00011608       ??_C@_0BH@NKPKNBFC@TYPE_ARRAY_DECLARATION?$AA@ 0045b608     rylgamelibrary:syntaxtree.obj
 0002:00011620       ??_C@_0BH@KMCLBAO@TYPE_ARRAY_INITIALIZE2?$AA@ 0045b620     rylgamelibrary:syntaxtree.obj
 0002:00011638       ??_C@_0BG@KMIHIAO@TYPE_ARRAY_INITIALIZE?$AA@ 0045b638     rylgamelibrary:syntaxtree.obj
 0002:00011650       ??_C@_0BI@CIJCFCOM@TYPE_NORMAL_DECLARATION?$AA@ 0045b650     rylgamelibrary:syntaxtree.obj
 0002:00011668       ??_C@_0BG@EFENOIAJ@TYPE_INIT_DECLARATION?$AA@ 0045b668     rylgamelibrary:syntaxtree.obj
 0002:00011680       ??_C@_0BF@MDONADI@TYPE_DECLARATOR_LIST?$AA@ 0045b680     rylgamelibrary:syntaxtree.obj
 0002:00011698       ??_C@_0O@JFOFLKFN@TYPE_VARIABLE?$AA@ 0045b698     rylgamelibrary:syntaxtree.obj
 0002:000116a8       ??_C@_0BG@LINNFKPA@TYPE_SPECIFIER_STRING?$AA@ 0045b6a8     rylgamelibrary:syntaxtree.obj
 0002:000116c0       ??_C@_0BE@GNAECEIF@TYPE_SPECIFIER_BOOL?$AA@ 0045b6c0     rylgamelibrary:syntaxtree.obj
 0002:000116d4       ??_C@_0BF@JHIBEAEO@TYPE_SPECIFIER_FLOAT?$AA@ 0045b6d4     rylgamelibrary:syntaxtree.obj
 0002:000116ec       ??_C@_0BD@NJFPEFAC@TYPE_SPECIFIER_INT?$AA@ 0045b6ec     rylgamelibrary:syntaxtree.obj
 0002:00011700       ??_C@_0BE@DEDAODHN@TYPE_SPECIFIER_VOID?$AA@ 0045b700     rylgamelibrary:syntaxtree.obj
 0002:00011714       ??_C@_0BB@NMPMMCI@TYPE_DECLARATION?$AA@ 0045b714     rylgamelibrary:syntaxtree.obj
 0002:00011728       ??_C@_0BG@CHFCJKLM@TYPE_RETURN_STATEMENT?$AA@ 0045b728     rylgamelibrary:syntaxtree.obj
 0002:00011740       ??_C@_0BI@DLNGHBJJ@TYPE_CONTINUE_STATEMENT?$AA@ 0045b740     rylgamelibrary:syntaxtree.obj
 0002:00011758       ??_C@_0BF@IKIFFGCM@TYPE_BREAK_STATEMENT?$AA@ 0045b758     rylgamelibrary:syntaxtree.obj
 0002:00011770       ??_C@_0BE@DAKHIDPH@TYPE_FOR_EXPRESSION?$AA@ 0045b770     rylgamelibrary:syntaxtree.obj
 0002:00011784       ??_C@_0BF@LBHOHFLA@TYPE_WHILE_STATEMENT?$AA@ 0045b784     rylgamelibrary:syntaxtree.obj
 0002:0001179c       ??_C@_0BD@JKIGIIPD@TYPE_FOR_STATEMENT?$AA@ 0045b79c     rylgamelibrary:syntaxtree.obj
 0002:000117b0       ??_C@_0N@GJFOAGEF@TYPE_DEFAULT?$AA@ 0045b7b0     rylgamelibrary:syntaxtree.obj
 0002:000117c0       ??_C@_0O@IMDJFDPM@TYPE_CASE_ONE?$AA@ 0045b7c0     rylgamelibrary:syntaxtree.obj
 0002:000117d0       ??_C@_0BC@JHPKLPAK@TYPE_SWITCH_CASES?$AA@ 0045b7d0     rylgamelibrary:syntaxtree.obj
 0002:000117e4       ??_C@_0BG@GCLMJMII@TYPE_SWITCH_STATEMENT?$AA@ 0045b7e4     rylgamelibrary:syntaxtree.obj
 0002:000117fc       ??_C@_0BH@NLKNBBAG@TYPE_IF_ELSE_STATEMENT?$AA@ 0045b7fc     rylgamelibrary:syntaxtree.obj
 0002:00011814       ??_C@_0BC@NKKGNEIE@TYPE_IF_STATEMENT?$AA@ 0045b814     rylgamelibrary:syntaxtree.obj
 0002:00011828       ??_C@_0BA@EGLGADMN@TYPE_EXPRESSION?$AA@ 0045b828     rylgamelibrary:syntaxtree.obj
 0002:00011838       ??_C@_0BF@BPFEODCI@TYPE_ERROR_STATEMENT?$AA@ 0045b838     rylgamelibrary:syntaxtree.obj
 0002:00011850       ??_C@_0BF@MMIMMGCA@TYPE_EMPTY_STATEMENT?$AA@ 0045b850     rylgamelibrary:syntaxtree.obj
 0002:00011868       ??_C@_0BE@OLJJFFMD@TYPE_STATEMENT_LIST?$AA@ 0045b868     rylgamelibrary:syntaxtree.obj
 0002:0001187c       ??_C@_06ICGJLFIM@string?$AA@ 0045b87c     rylgamelibrary:syntaxtree.obj
 0002:00011884       ??_C@_05KNFBNCOH@float?$AA@ 0045b884     rylgamelibrary:syntaxtree.obj
 0002:0001188c       ??_C@_03JBIPMCLC@int?$AA@  0045b88c     rylgamelibrary:syntaxtree.obj
 0002:00011890       ??_C@_04DDKJGDCM@bool?$AA@ 0045b890     rylgamelibrary:syntaxtree.obj
 0002:00011898       ??_C@_04GKJNKENE@void?$AA@ 0045b898     rylgamelibrary:syntaxtree.obj
 0002:000118a0       ??_C@_04KHEKMLOH@?0?5?$CFs?$AA@ 0045b8a0     rylgamelibrary:intermediatecode.obj
 0002:000118a8       ??_C@_03EEBNCBOD@?5?$CFs?$AA@ 0045b8a8     rylgamelibrary:symboltable.obj
 0002:000118ac       ??_C@_06CPGHEBHO@?$CFs?5?$CFs?$CI?$AA@ 0045b8ac     rylgamelibrary:symboltable.obj
 0002:000118b8       ??_C@_0EF@EBPIGFAE@?A?v?A?$KE?G?Q?5?$MA?L?$LI?$KH?5?$LA?x?$LA?$KD?$MA?$LL?5?C?$KD?$MA?$LL?5?$LM?v?5?$LO?x?$LN?$MA?$LE@ 0045b8b8     rylgamelibrary:symboltable.obj
 0002:00012c94       ??_C@_0BD@POMNHADD@primary_expression?$AA@ 0045cc94     rylgamelibrary:parse.obj
 0002:00012ca8       ??_C@_0BD@FCPJEELK@postfix_expression?$AA@ 0045cca8     rylgamelibrary:parse.obj
 0002:00012cbc       ??_C@_0BB@PCNJFDMC@unary_expression?$AA@ 0045ccbc     rylgamelibrary:parse.obj
 0002:00012cd0       ??_C@_0BK@CBMFFKFE@multiplicative_expression?$AA@ 0045ccd0     rylgamelibrary:parse.obj
 0002:00012cec       ??_C@_0BE@HIECFDAC@additive_expression?$AA@ 0045ccec     rylgamelibrary:parse.obj
 0002:00012d00       ??_C@_0BG@PBKNPFNE@relational_expression?$AA@ 0045cd00     rylgamelibrary:parse.obj
 0002:00012d18       ??_C@_0BE@GGGBNBNB@equality_expression?$AA@ 0045cd18     rylgamelibrary:parse.obj
 0002:00012d2c       ??_C@_0BH@FLNJOLOJ@logical_and_expression?$AA@ 0045cd2c     rylgamelibrary:parse.obj
 0002:00012d44       ??_C@_0BG@JJHOGFCA@logical_or_expression?$AA@ 0045cd44     rylgamelibrary:parse.obj
 0002:00012d5c       ??_C@_0BG@EMHAHMJD@assignment_expression?$AA@ 0045cd5c     rylgamelibrary:parse.obj
 0002:00012d74       ??_C@_0L@FKCCBALC@expression?$AA@ 0045cd74     rylgamelibrary:parse.obj
 0002:00012d80       ??_C@_0BE@NMHAKMIL@constant_expression?$AA@ 0045cd80     rylgamelibrary:parse.obj
 0002:00012d94       ??_C@_0BE@KNJNECJD@function_definition?$AA@ 0045cd94     rylgamelibrary:parse.obj
 0002:00012da8       ??_C@_0BD@GCMJGLIN@function_def_start?$AA@ 0045cda8     rylgamelibrary:parse.obj
 0002:00012dbc       ??_C@_0BC@GIJILNMI@function_decl_end?$AA@ 0045cdbc     rylgamelibrary:parse.obj
 0002:00012dd0       ??_C@_0O@CIDAHBFE@function_name?$AA@ 0045cdd0     rylgamelibrary:parse.obj
 0002:00012de0       ??_C@_0BF@MHNEBGAK@argument_declaration?$AA@ 0045cde0     rylgamelibrary:parse.obj
 0002:00012df8       ??_C@_0BK@MLCJDOJL@argument_declaration_list?$AA@ 0045cdf8     rylgamelibrary:parse.obj
 0002:00012e14       ??_C@_0BB@MLADMHHB@initializer_list?$AA@ 0045ce14     rylgamelibrary:parse.obj
 0002:00012e28       ??_C@_0BC@IADHJENI@array_initializer?$AA@ 0045ce28     rylgamelibrary:parse.obj
 0002:00012e3c       ??_C@_0BA@ONFPOLM@init_declarator?$AA@ 0045ce3c     rylgamelibrary:parse.obj
 0002:00012e4c       ??_C@_0BA@OFEHPAFO@declarator_list?$AA@ 0045ce4c     rylgamelibrary:parse.obj
 0002:00012e5c       ??_C@_0N@IMKHKHAH@new_variable?$AA@ 0045ce5c     rylgamelibrary:parse.obj
 0002:00012e6c       ??_C@_08LODIKCGI@variable?$AA@ 0045ce6c     rylgamelibrary:parse.obj
 0002:00012e78       ??_C@_0BA@HHLADBEG@decl_specifiers?$AA@ 0045ce78     rylgamelibrary:parse.obj
 0002:00012e88       ??_C@_0M@FIONBADE@declaration?$AA@ 0045ce88     rylgamelibrary:parse.obj
 0002:00012e94       ??_C@_0P@GNCMIDFA@jump_statement?$AA@ 0045ce94     rylgamelibrary:parse.obj
 0002:00012ea4       ??_C@_0BE@BGCEPEOI@optional_expression?$AA@ 0045cea4     rylgamelibrary:parse.obj
 0002:00012eb8       ??_C@_0BD@IKGAHJDE@for_init_statement?$AA@ 0045ceb8     rylgamelibrary:parse.obj
 0002:00012ecc       ??_C@_0P@MILMAEMF@for_expression?$AA@ 0045cecc     rylgamelibrary:parse.obj
 0002:00012edc       ??_C@_0BE@LHIHOAMA@iteration_statement?$AA@ 0045cedc     rylgamelibrary:parse.obj
 0002:00012ef0       ??_C@_07DLHCIBDH@default?$AA@ 0045cef0     rylgamelibrary:parse.obj
 0002:00012ef8       ??_C@_08GGCFGEMN@case_one?$AA@ 0045cef8     rylgamelibrary:parse.obj
 0002:00012f04       ??_C@_05FHILFBNJ@cases?$AA@ 0045cf04     rylgamelibrary:parse.obj
 0002:00012f0c       ??_C@_0BE@IMJEIIDB@selection_statement?$AA@ 0045cf0c     rylgamelibrary:parse.obj
 0002:00012f20       ??_C@_0BF@HJFNGLOG@expression_statement?$AA@ 0045cf20     rylgamelibrary:parse.obj
 0002:00012f38       ??_C@_0BD@IGPHHKLG@compound_statement?$AA@ 0045cf38     rylgamelibrary:parse.obj
 0002:00012f4c       ??_C@_09JEFLBPCK@statement?$AA@ 0045cf4c     rylgamelibrary:parse.obj
 0002:00012f58       ??_C@_0P@MBPAMDP@statement_list?$AA@ 0045cf58     rylgamelibrary:parse.obj
 0002:00012f68       ??_C@_07MHLKLKDM@program?$AA@ 0045cf68     rylgamelibrary:parse.obj
 0002:00012f70       ??_C@_0BA@OKILGALB@TOKEN_DECREMENT?$AA@ 0045cf70     rylgamelibrary:parse.obj
 0002:00012f80       ??_C@_0BA@JNCAHFNM@TOKEN_INCREMENT?$AA@ 0045cf80     rylgamelibrary:parse.obj
 0002:00012f90       ??_C@_0BA@KNCEAEDH@PREFIXDECREMENT?$AA@ 0045cf90     rylgamelibrary:parse.obj
 0002:00012fa0       ??_C@_0BA@NKIPBBFK@PREFIXINCREMENT?$AA@ 0045cfa0     rylgamelibrary:parse.obj
 0002:00012fb0       ??_C@_09JOKOLHKN@TOKEN_NOT?$AA@ 0045cfb0     rylgamelibrary:parse.obj
 0002:00012fbc       ??_C@_0P@DIHKIMFB@TOKEN_REMINDER?$AA@ 0045cfbc     rylgamelibrary:parse.obj
 0002:00012fcc       ??_C@_0P@FECMDJLE@TOKEN_DIVISION?$AA@ 0045cfcc     rylgamelibrary:parse.obj
 0002:00012fdc       ??_C@_0BF@KBBPOIOI@TOKEN_MULTIPLICATION?$AA@ 0045cfdc     rylgamelibrary:parse.obj
 0002:00012ff4       ??_C@_0BC@FKNPGK@TOKEN_SUBTRACTION?$AA@ 0045cff4     rylgamelibrary:parse.obj
 0002:00013008       ??_C@_0P@MHNPDINN@TOKEN_ADDITION?$AA@ 0045d008     rylgamelibrary:parse.obj
 0002:00013018       ??_C@_0P@LPJHJPDA@TOKEN_NOTEQUAL?$AA@ 0045d018     rylgamelibrary:parse.obj
 0002:00013028       ??_C@_0P@MGPCFHMN@TOKEN_EQUALITY?$AA@ 0045d028     rylgamelibrary:parse.obj
 0002:00013038       ??_C@_0BG@KPAPMAAD@TOKEN_MORETHANOREQUAL?$AA@ 0045d038     rylgamelibrary:parse.obj
 0002:00013050       ??_C@_0P@LNGPPEHP@TOKEN_MORETHAN?$AA@ 0045d050     rylgamelibrary:parse.obj
 0002:00013060       ??_C@_0BG@OPIFLEPF@TOKEN_LESSTHANOREQUAL?$AA@ 0045d060     rylgamelibrary:parse.obj
 0002:00013078       ??_C@_0P@EICMBGMG@TOKEN_LESSTHAN?$AA@ 0045d078     rylgamelibrary:parse.obj
 0002:00013088       ??_C@_08FIIKJNMB@TOKEN_OR?$AA@ 0045d088     rylgamelibrary:parse.obj
 0002:00013094       ??_C@_09INMNNPJN@TOKEN_AND?$AA@ 0045d094     rylgamelibrary:parse.obj
 0002:000130a0       ??_C@_0BH@DPPDDICG@TOKEN_COMPOUNDREMINDER?$AA@ 0045d0a0     rylgamelibrary:parse.obj
 0002:000130b8       ??_C@_0BH@FDKFINMD@TOKEN_COMPOUNDDIVISION?$AA@ 0045d0b8     rylgamelibrary:parse.obj
 0002:000130d0       ??_C@_0BN@MHGBJEHB@TOKEN_COMPOUNDMULTIPLICATION?$AA@ 0045d0d0     rylgamelibrary:parse.obj
 0002:000130f0       ??_C@_0BK@EFCJPBIA@TOKEN_COMPOUNDSUBTRACTION?$AA@ 0045d0f0     rylgamelibrary:parse.obj
 0002:0001310c       ??_C@_0BH@MAFGIMKK@TOKEN_COMPOUNDADDITION?$AA@ 0045d10c     rylgamelibrary:parse.obj
 0002:00013124       ??_C@_0BB@FDGGCLCK@TOKEN_ASSIGNMENT?$AA@ 0045d124     rylgamelibrary:parse.obj
 0002:00013138       ??_C@_0M@HCKDLOPN@TOKEN_COLON?$AA@ 0045d138     rylgamelibrary:parse.obj
 0002:00013144       ??_C@_0M@EOADBBDJ@TOKEN_COMMA?$AA@ 0045d144     rylgamelibrary:parse.obj
 0002:00013150       ??_C@_0M@GKDLHDCC@TOKEN_ERROR?$AA@ 0045d150     rylgamelibrary:parse.obj
 0002:0001315c       ??_C@_0BD@ENFBOEDJ@TOKEN_RIGHTBRACKET?$AA@ 0045d15c     rylgamelibrary:parse.obj
 0002:00013170       ??_C@_0BC@HLPNCDDB@TOKEN_LEFTBRACKET?$AA@ 0045d170     rylgamelibrary:parse.obj
 0002:00013184       ??_C@_0BB@HOFPOKEN@TOKEN_RIGHTBRACE?$AA@ 0045d184     rylgamelibrary:parse.obj
 0002:00013198       ??_C@_0BA@PJLKAMOE@TOKEN_LEFTBRACE?$AA@ 0045d198     rylgamelibrary:parse.obj
 0002:000131a8       ??_C@_0BH@LKJKJIPE@TOKEN_RIGHTPARENTHESIS?$AA@ 0045d1a8     rylgamelibrary:parse.obj
 0002:000131c0       ??_C@_0BG@CGMGFGKC@TOKEN_LEFTPARENTHESIS?$AA@ 0045d1c0     rylgamelibrary:parse.obj
 0002:000131d8       ??_C@_0BD@JDGFOHFG@TOKEN_ENDSTATEMENT?$AA@ 0045d1d8     rylgamelibrary:parse.obj
 0002:000131ec       ??_C@_0N@LHLOMKCE@TOKEN_RETURN?$AA@ 0045d1ec     rylgamelibrary:parse.obj
 0002:000131fc       ??_C@_0M@CLGOKIKO@TOKEN_BREAK?$AA@ 0045d1fc     rylgamelibrary:parse.obj
 0002:00013208       ??_C@_0P@FIJJNGOB@TOKEN_CONTINUE?$AA@ 0045d208     rylgamelibrary:parse.obj
 0002:00013218       ??_C@_0O@BNJKIEOC@TOKEN_DEFAULT?$AA@ 0045d218     rylgamelibrary:parse.obj
 0002:00013228       ??_C@_0L@DIPHGPKF@TOKEN_CASE?$AA@ 0045d228     rylgamelibrary:parse.obj
 0002:00013234       ??_C@_0N@DEKFDIJH@TOKEN_SWITCH?$AA@ 0045d234     rylgamelibrary:parse.obj
 0002:00013244       ??_C@_0L@EFNNECNI@TOKEN_ELSE?$AA@ 0045d244     rylgamelibrary:parse.obj
 0002:00013250       ??_C@_08HCKJDGCG@TOKEN_IF?$AA@ 0045d250     rylgamelibrary:parse.obj
 0002:0001325c       ??_C@_0M@IOKILFMA@TOKEN_WHILE?$AA@ 0045d25c     rylgamelibrary:parse.obj
 0002:00013268       ??_C@_09NEADIME@TOKEN_FOR?$AA@ 0045d268     rylgamelibrary:parse.obj
 0002:00013274       ??_C@_0L@HIICBHID@TOKEN_VOID?$AA@ 0045d274     rylgamelibrary:parse.obj
 0002:00013280       ??_C@_0N@IIDCOMHE@TOKEN_STRING?$AA@ 0045d280     rylgamelibrary:parse.obj
 0002:00013290       ??_C@_0L@CBLGNAHL@TOKEN_BOOL?$AA@ 0045d290     rylgamelibrary:parse.obj
 0002:0001329c       ??_C@_0M@MNMICNKB@TOKEN_FLOAT?$AA@ 0045d29c     rylgamelibrary:parse.obj
 0002:000132a8       ??_C@_09CLLOFCD@TOKEN_INT?$AA@ 0045d2a8     rylgamelibrary:parse.obj
 0002:000132b4       ??_C@_0BC@MNLBLBLP@TOKEN_STRINGVALUE?$AA@ 0045d2b4     rylgamelibrary:parse.obj
 0002:000132c8       ??_C@_0BA@GMOFNFIL@TOKEN_BOOLVALUE?$AA@ 0045d2c8     rylgamelibrary:parse.obj
 0002:000132d8       ??_C@_0BB@HHAIIFLD@TOKEN_FLOATVALUE?$AA@ 0045d2d8     rylgamelibrary:parse.obj
 0002:000132ec       ??_C@_0BD@IBFOJDIC@TOKEN_INTEGERVALUE?$AA@ 0045d2ec     rylgamelibrary:parse.obj
 0002:00013300       ??_C@_08EAJPFEKE@TOKEN_ID?$AA@ 0045d300     rylgamelibrary:parse.obj
 0002:0001330c       ??_C@_0M@OPHMOOJC@$undefined?4?$AA@ 0045d30c     rylgamelibrary:parse.obj
 0002:00013318       ??_C@_05KKCIMGE@error?$AA@ 0045d318     rylgamelibrary:parse.obj
 0002:00013320       ??_C@_01EPMOAMKG@$?$AA@    0045d320     rylgamelibrary:parse.obj
 0002:000140c8       ??_C@_03OFAPEBGM@?$CFs?6?$AA@ 0045e0c8     rylgamelibrary:lex.obj
 0002:000140cc       ??_C@_0BA@ECKFJHDH@Error?5Statement?$AA@ 0045e0cc     rylgamelibrary:imcodegen.obj
 0002:000140dc       ??_7IOPCode@@6B@           0045e0dc     rylgamelibrary:imcodegen.obj
 0002:000140ec       ??_7COP_nop@@6B@           0045e0ec     rylgamelibrary:imcodegen.obj
 0002:000140fc       ??_7COP_ret@@6B@           0045e0fc     rylgamelibrary:imcodegen.obj
 0002:0001410c       ??_7COP_fnstsw_ax@@6B@     0045e10c     rylgamelibrary:imcodegen.obj
 0002:0001411c       ??_C@_0CJ@PHLNAGI@?$LA?$LA?$MA?$LK?5?G?T?$LM?v?$LI?$KG?5?$LF?N?5?$LJ?x?5?$LI?$LI?$LF?i?$LH?A?$LA?m?5?$LN?C?$LF?$LF?G@ 0045e11c     rylgamelibrary:imcodegen.obj
 0002:00014148       ??_C@_02PHLEDNGH@NE?$AA@   0045e148     rylgamelibrary:imcodeunits.obj
 0002:0001414c       ??_C@_02PEDAOJAJ@LE?$AA@   0045e14c     rylgamelibrary:imcodeunits.obj
 0002:00014150       ??_C@_01OCOKONAJ@L?$AA@    0045e150     rylgamelibrary:imcodeunits.obj
 0002:00014154       ??_C@_02PIGFAGOI@GE?$AA@   0045e154     rylgamelibrary:imcodeunits.obj
 0002:00014158       ??_C@_01BBODEMC@G?$AA@     0045e158     rylgamelibrary:imcodeunits.obj
 0002:0001415c       ??_C@_03CEFJFJLM@EDI?$AA@  0045e15c     rylgamelibrary:imcodeunits.obj
 0002:00014160       ??_C@_03DNDAOMEJ@ESI?$AA@  0045e160     rylgamelibrary:imcodeunits.obj
 0002:00014164       ??_C@_03LLNEIMBG@EBP?$AA@  0045e164     rylgamelibrary:imcodeunits.obj
 0002:00014168       ??_C@_03KGDAEFFB@ESP?$AA@  0045e168     rylgamelibrary:imcodeunits.obj
 0002:0001416c       ??_C@_03HDANAGBO@EBX?$AA@  0045e16c     rylgamelibrary:imcodeunits.obj
 0002:00014170       ??_C@_03HHIAHKKM@EDX?$AA@  0045e170     rylgamelibrary:imcodeunits.obj
 0002:00014174       ??_C@_03HCMPGMCJ@ECX?$AA@  0045e174     rylgamelibrary:imcodeunits.obj
 0002:00014178       ??_C@_03HBELLIEH@EAX?$AA@  0045e178     rylgamelibrary:imcodeunits.obj
 0002:0001417c       ??_C@_09EMCDKGPH@CALL?7?7?$CFs?6?$AA@ 0045e17c     rylgamelibrary:imcodeunits.obj
 0002:00014188       ??_C@_0M@FAJHGEKI@?$CFs?0?5?$CFs?$FL?$CFs?$FN?6?$AA@ 0045e188     rylgamelibrary:imcodeunits.obj
 0002:00014194       ??_C@_0M@HGFCLGCJ@?$CFs?$FL?$CFd?$FN?0?5?$CFs?6?$AA@ 0045e194     rylgamelibrary:imcodeunits.obj
 0002:000141a0       ??_C@_07GFLJLICB@?$CFs?0?5?$CFd?6?$AA@ 0045e1a0     rylgamelibrary:imcodeunits.obj
 0002:000141a8       ??_C@_07GGDNGMEP@?$CFs?0?5?$CFf?6?$AA@ 0045e1a8     rylgamelibrary:imcodeunits.obj
 0002:000141b0       ??_C@_07HMNAANNE@?$CFs?0?5?$CFs?6?$AA@ 0045e1b0     rylgamelibrary:imcodeunits.obj
 0002:000141b8       ??_C@_05BHCNFIMO@MOV?7?7?$AA@ 0045e1b8     rylgamelibrary:imcodeunits.obj
 0002:000141c0       ??_C@_04ILDKGAJL@NOP?6?$AA@ 0045e1c0     rylgamelibrary:imcodeunits.obj
 0002:000141c8       ??_C@_05ONCPDGLA@ADD?7?7?$AA@ 0045e1c8     rylgamelibrary:imcodeunits.obj
 0002:000141d0       ??_C@_05NLNKHEMO@SUB?7?7?$AA@ 0045e1d0     rylgamelibrary:imcodeunits.obj
 0002:000141d8       ??_C@_06PPOECOGB@IMUL?7?7?$AA@ 0045e1d8     rylgamelibrary:imcodeunits.obj
 0002:000141e0       ??_C@_06ECFPLCNB@IDIV?7?7?$AA@ 0045e1e0     rylgamelibrary:imcodeunits.obj
 0002:000141e8       ??_C@_09CAECIIPF@PUSH?7?7?$CFs?6?$AA@ 0045e1e8     rylgamelibrary:imcodeunits.obj
 0002:000141f4       ??_C@_08KJGHMBOH@POP?7?7?$CFs?6?$AA@ 0045e1f4     rylgamelibrary:imcodeunits.obj
 0002:00014200       ??_C@_08OGLEKHHE@JMP?7?7?$CFX?6?$AA@ 0045e200     rylgamelibrary:imcodeunits.obj
 0002:0001420c       ??_C@_08BLOPDPHL@J?$CFs?7?7?$CFX?6?$AA@ 0045e20c     rylgamelibrary:imcodeunits.obj
 0002:00014218       ??_C@_0L@PDODHME@JMPMARK?7?7?6?$AA@ 0045e218     rylgamelibrary:imcodeunits.obj
 0002:00014224       ??_C@_0N@HHDKJAJB@JMPMARK?7?7?$CFX?6?$AA@ 0045e224     rylgamelibrary:imcodeunits.obj
 0002:00014234       ??_C@_0N@IJGMCKAE@CMP?7?7?$CFs?0?5?$CFd?6?$AA@ 0045e234     rylgamelibrary:imcodeunits.obj
 0002:00014244       ??_C@_0N@JAAFJPPB@CMP?7?7?$CFs?0?5?$CFs?6?$AA@ 0045e244     rylgamelibrary:imcodeunits.obj
 0002:00014254       ??_C@_04EGJOFCKA@RET?6?$AA@ 0045e254     rylgamelibrary:imcodeunits.obj
 0002:0001425c       ??_C@_0L@FPLENNBK@SET?$CFs?7?7?$CFs?6?$AA@ 0045e25c     rylgamelibrary:imcodeunits.obj
 0002:00014268       ??_C@_08GLKDEFCC@FLD?7?7?$CFs?6?$AA@ 0045e268     rylgamelibrary:imcodeunits.obj
 0002:00014274       ??_C@_09EKAADIGB@FADD?7?7?$CFs?6?$AA@ 0045e274     rylgamelibrary:imcodeunits.obj
 0002:00014280       ??_C@_09BLPHFGBJ@FSUB?7?7?$CFs?6?$AA@ 0045e280     rylgamelibrary:imcodeunits.obj
 0002:0001428c       ??_C@_09CPMKLEKH@FMUL?7?7?$CFs?6?$AA@ 0045e28c     rylgamelibrary:imcodeunits.obj
 0002:00014298       ??_C@_09GLNDOFBI@FDIV?7?7?$CFs?6?$AA@ 0045e298     rylgamelibrary:imcodeunits.obj
 0002:000142a4       ??_C@_09CHBMNLGA@FSTP?7?7?$CFs?6?$AA@ 0045e2a4     rylgamelibrary:imcodeunits.obj
 0002:000142b0       ??_C@_0L@FOMFIBHH@FCOMP?7?7?$CFs?6?$AA@ 0045e2b0     rylgamelibrary:imcodeunits.obj
 0002:000142bc       ??_C@_0M@OPLIMCH@FNSTSW?7?7AX?6?$AA@ 0045e2bc     rylgamelibrary:imcodeunits.obj
 0002:000142c8       ??_C@_0O@GCNEJMJD@TEST?7?7AH?0?5?$CFd?6?$AA@ 0045e2c8     rylgamelibrary:imcodeunits.obj
 0002:000142d8       ??_C@_0EA@GKBKDCDG@?$MA?L?$LA?M?$MA?$LK?5String?5Buffer?$LA?$KB?5?$LO?F?$LE?O?$MA?Z?$LD?$KK?$HM@ 0045e2d8     rylgamelibrary:imcodeunits.obj
 0002:00014318       ??_C@_0O@OLBCINBD@ITOA?7?7?$CFs?0?5?$CFs?6?$AA@ 0045e318     rylgamelibrary:imcodeunits.obj
 0002:00014328       ??_C@_0EA@IJAPDJPP@?$MA?L?$LA?M?$MA?$LK?5String?5Buffer?$LA?$KB?5?$LO?F?$LE?O?$MA?Z?$LD?$KK?$HM@ 0045e328     rylgamelibrary:imcodeunits.obj
 0002:00014368       ??_C@_0O@LNIGDJOF@FTOA?7?7?$CFs?0?5?$CFs?6?$AA@ 0045e368     rylgamelibrary:imcodeunits.obj
 0002:00014378       ??_C@_0M@BFPFLDAP@MALLOC?7?7?$CFs?6?$AA@ 0045e378     rylgamelibrary:imcodeunits.obj
 0002:00014384       ??_C@_09LFJAENPP@FREE?7?7?$CFs?6?$AA@ 0045e384     rylgamelibrary:imcodeunits.obj
 0002:00014390       ??_C@_04MDKIEGGJ@?5?$CFs?6?$AA@ 0045e390     rylgamelibrary:imcodeunits.obj
 0002:00014398       ??_C@_0M@GMEIPIMN@STRCPY?7?7?$CFs?0?$AA@ 0045e398     rylgamelibrary:imcodeunits.obj
 0002:000143a4       ??_C@_0BA@FANLGANB@STRCMP?7?7?$CFs?0?5?$CFs?6?$AA@ 0045e3a4     rylgamelibrary:imcodeunits.obj
 0002:000143b4       ??_C@_08HKFOCBKG@STRLEN?7?7?$AA@ 0045e3b4     rylgamelibrary:imcodeunits.obj
 0002:000143c0       ??_7COP_call@@6B@          0045e3c0     rylgamelibrary:imcodeunits.obj
 0002:000143d0       ??_7COP_mov@@6B@           0045e3d0     rylgamelibrary:imcodeunits.obj
 0002:000143e0       ??_7COP_add@@6B@           0045e3e0     rylgamelibrary:imcodeunits.obj
 0002:000143f0       ??_7COP_sub@@6B@           0045e3f0     rylgamelibrary:imcodeunits.obj
 0002:00014400       ??_7COP_imul@@6B@          0045e400     rylgamelibrary:imcodeunits.obj
 0002:00014410       ??_7COP_idiv@@6B@          0045e410     rylgamelibrary:imcodeunits.obj
 0002:00014420       ??_7COP_push@@6B@          0045e420     rylgamelibrary:imcodeunits.obj
 0002:00014430       ??_7COP_pop@@6B@           0045e430     rylgamelibrary:imcodeunits.obj
 0002:00014440       ??_7COP_jmp@@6B@           0045e440     rylgamelibrary:imcodeunits.obj
 0002:00014450       ??_7COP_jcc@@6B@           0045e450     rylgamelibrary:imcodeunits.obj
 0002:00014460       ??_7COP_jmpmark@@6B@       0045e460     rylgamelibrary:imcodeunits.obj
 0002:00014470       ??_7COP_cmp@@6B@           0045e470     rylgamelibrary:imcodeunits.obj
 0002:00014480       ??_C@_0DN@MEDMEGFA@setcc?5?$LI?m?$LH?I?$LP?$KB?5EAX?0?5ECX?0?5EDX?0?5EBX?$LP@ 0045e480     rylgamelibrary:imcodeunits.obj
 0002:000144c0       ??_7COP_setcc@@6B@         0045e4c0     rylgamelibrary:imcodeunits.obj
 0002:000144d0       ??_7COP_fld@@6B@           0045e4d0     rylgamelibrary:imcodeunits.obj
 0002:000144e0       ??_7COP_fadd@@6B@          0045e4e0     rylgamelibrary:imcodeunits.obj
 0002:000144f0       ??_7COP_fsub@@6B@          0045e4f0     rylgamelibrary:imcodeunits.obj
 0002:00014500       ??_7COP_fmul@@6B@          0045e500     rylgamelibrary:imcodeunits.obj
 0002:00014510       ??_7COP_fdiv@@6B@          0045e510     rylgamelibrary:imcodeunits.obj
 0002:00014520       ??_7COP_fstp@@6B@          0045e520     rylgamelibrary:imcodeunits.obj
 0002:00014530       ??_7COP_fcomp@@6B@         0045e530     rylgamelibrary:imcodeunits.obj
 0002:00014540       ??_7COP_test_ah@@6B@       0045e540     rylgamelibrary:imcodeunits.obj
 0002:00014550       ??_7COP_itoa@@6B@          0045e550     rylgamelibrary:imcodeunits.obj
 0002:00014560       ??_7COP_ftoa@@6B@          0045e560     rylgamelibrary:imcodeunits.obj
 0002:00014570       ??_7COP_malloc@@6B@        0045e570     rylgamelibrary:imcodeunits.obj
 0002:00014580       ??_7COP_free@@6B@          0045e580     rylgamelibrary:imcodeunits.obj
 0002:00014590       ??_7COP_strcpy@@6B@        0045e590     rylgamelibrary:imcodeunits.obj
 0002:000145a0       ??_7COP_strcmp@@6B@        0045e5a0     rylgamelibrary:imcodeunits.obj
 0002:000145b0       ??_7COP_strlen@@6B@        0045e5b0     rylgamelibrary:imcodeunits.obj
 0002:000145c0       ??_C@_0DB@LINNNCKK@?A?$KE?$MA?G?$LF?G?A?v?5?$LO?J?$MA?$LK?5?G?T?$LM?v?$LI?$KG?5?H?$KD?C?b?G?O?$LH?A?5?$LN?C@ 0045e5c0     rylgamelibrary:imcodeunits.obj
 0002:000145f8       ??_7logic_error@std@@6B@   0045e5f8     libcpmt:string.obj
 0002:00014604       ??_7length_error@std@@6B@  0045e604     libcpmt:string.obj
 0002:00014610       ??_7out_of_range@std@@6B@  0045e610     libcpmt:string.obj
 0002:00014618       ??_C@_0BI@CFPLBAOH@invalid?5string?5position?$AA@ 0045e618     libcpmt:string.obj
 0002:00014630       ??_C@_0BA@JFNIOLAK@string?5too?5long?$AA@ 0045e630     libcpmt:string.obj
 0002:00014640       ?_BADOFF@std@@3JB          0045e640     libcpmt:ios.obj
 0002:00014648       ??_7ios_base@std@@6B@      0045e648     libcpmt:ios.obj
 0002:00014650       ??_7runtime_error@std@@6B@ 0045e650     libcpmt:ios.obj
 0002:0001465c       ??_7failure@ios_base@std@@6B@ 0045e65c     libcpmt:ios.obj
 0002:00014664       ??_C@_0BF@OOHOMBOF@ios_base?3?3eofbit?5set?$AA@ 0045e664     libcpmt:ios.obj
 0002:0001467c       ??_C@_0BG@FMKFHCIL@ios_base?3?3failbit?5set?$AA@ 0045e67c     libcpmt:ios.obj
 0002:00014694       ??_C@_0BF@PHHKMMFD@ios_base?3?3badbit?5set?$AA@ 0045e694     libcpmt:ios.obj
 0002:000146cc       ?table_size@?$ctype@D@std@@2IB 0045e6cc     libcpmt:locale0.obj
 0002:000146d4       ??_7facet@locale@std@@6B@  0045e6d4     libcpmt:locale0.obj
 0002:000146dc       ??_7_Locimp@locale@std@@6B@ 0045e6dc     libcpmt:locale0.obj
 0002:000146e0       ??_C@_01NBENCBCI@?$CK?$AA@ 0045e6e0     libcpmt:locale0.obj
 0002:000146f8       ??_7?$basic_ostream@DU?$char_traits@D@std@@@std@@6B@ 0045e6f8     libcpmt:cout.obj
 0002:00014700       ??_7?$basic_ios@DU?$char_traits@D@std@@@std@@6B@ 0045e700     libcpmt:cout.obj
 0002:00014708       ??_7?$ctype@D@std@@6B@     0045e708     libcpmt:cout.obj
 0002:00014730       ??_7?$basic_streambuf@DU?$char_traits@D@std@@@std@@6B@ 0045e730     libcpmt:cout.obj
 0002:00014768       ??_7?$basic_filebuf@DU?$char_traits@D@std@@@std@@6B@ 0045e768     libcpmt:cout.obj
 0002:000147a0       ??_7?$codecvt@DDH@std@@6B@ 0045e7a0     libcpmt:cout.obj
 0002:000147c4       ??_7bad_alloc@std@@6B@     0045e7c4     libcpmt:nomemory.obj
 0002:00014810       ??_7exception@@6B@         0045e810     LIBCMT:stdexcpt.obj
 0002:00014818       ??_C@_0BC@EOODALEL@Unknown?5exception?$AA@ 0045e818     LIBCMT:stdexcpt.obj
 0002:00014830       ??_7bad_cast@@6B@          0045e830     LIBCMT:stdexcpt.obj
 0002:0001483c       ??_7type_info@@6B@         0045e83c     LIBCMT:typinfo.obj
 0002:0001491c       __tls_used                 0045e91c     LIBCMT:tlssup.obj
 0002:000149fc       ??_C@_0P@MIGLKIOC@CorExitProcess?$AA@ 0045e9fc     LIBCMT:crt0dat.obj
 0002:00014a0c       ??_C@_0M@MBOPBNBK@mscoree?4dll?$AA@ 0045ea0c     LIBCMT:crt0dat.obj
 0002:00014a84       ??_C@_13NOLLCAOD@?$AA?$AA?$AA?$AA@ 0045ea84     LIBCMT:a_map.obj
 0002:00014ab0       ___newctype                0045eab0     LIBCMT:ctype.obj
 0002:00014db0       __wctype                   0045edb0     LIBCMT:ctype.obj
 0002:00015148       ??_C@_07LCBHPJJN@LC_TIME?$AA@ 0045f148     LIBCMT:setlocal.obj
 0002:00015150       ??_C@_0L@DLHIECNL@LC_NUMERIC?$AA@ 0045f150     LIBCMT:setlocal.obj
 0002:0001515c       ??_C@_0M@MIENIKLA@LC_MONETARY?$AA@ 0045f15c     LIBCMT:setlocal.obj
 0002:00015168       ??_C@_08EADHIDAD@LC_CTYPE?$AA@ 0045f168     LIBCMT:setlocal.obj
 0002:00015174       ??_C@_0L@KFJHEKIK@LC_COLLATE?$AA@ 0045f174     LIBCMT:setlocal.obj
 0002:00015180       ??_C@_06NEFDFEKB@LC_ALL?$AA@ 0045f180     LIBCMT:setlocal.obj
 0002:00015188       ??_C@_03EGDHDPFD@_?4?0?$AA@ 0045f188     LIBCMT:setlocal.obj
 0002:0001518c       ??_C@_01LFCBOECM@?4?$AA@   0045f18c     LIBCMT:setlocal.obj
 0002:00015190       ??_C@_01IDAFKMJL@_?$AA@    0045f190     LIBCMT:setlocal.obj
 0002:000151a4       ??_C@_01ICJEACDI@?$DL?$AA@ 0045f1a4     LIBCMT:setlocal.obj
 0002:000151a8       ??_C@_01NEMOKFLO@?$DN?$AA@ 0045f1a8     LIBCMT:setlocal.obj
 0002:000151ac       ??_C@_02BALPLPBG@?$DN?$DL?$AA@ 0045f1ac     LIBCMT:setlocal.obj
 0002:000151d8       ??_C@_07PEJMOBNF@FlsFree?$AA@ 0045f1d8     LIBCMT:tidtable.obj
 0002:000151e0       ??_C@_0M@JCPCPOEF@FlsSetValue?$AA@ 0045f1e0     LIBCMT:tidtable.obj
 0002:000151ec       ??_C@_0M@GDNOONDI@FlsGetValue?$AA@ 0045f1ec     LIBCMT:tidtable.obj
 0002:000151f8       ??_C@_08KNHFBNJ@FlsAlloc?$AA@ 0045f1f8     LIBCMT:tidtable.obj
 0002:00015204       ??_C@_0N@MDJJJHMB@kernel32?4dll?$AA@ 0045f204     LIBCMT:tidtable.obj
 0002:00015234       ??_C@_0CF@GOGNBNAK@Microsoft?5Visual?5C?$CL?$CL?5Runtime?5Lib@ 0045f234     LIBCMT:secfail.obj
 0002:0001525c       ??_C@_09KLGCKDOD@Program?3?5?$AA@ 0045f25c     LIBCMT:secfail.obj
 0002:00015268       ??_C@_02PHMGELLB@?6?6?$AA@ 0045f268     LIBCMT:secfail.obj
 0002:0001526c       ??_C@_03KHICJKCI@?4?4?4?$AA@ 0045f26c     LIBCMT:secfail.obj
 0002:00015270       ??_C@_0BH@DNAGHKFM@?$DMprogram?5name?5unknown?$DO?$AA@ 0045f270     LIBCMT:secfail.obj
 0002:00015288       ??_C@_0KA@JEHFIFGP@A?5buffer?5overrun?5has?5been?5detect@ 0045f288     LIBCMT:secfail.obj
 0002:00015328       ??_C@_0BJ@MDEKIEOJ@Buffer?5overrun?5detected?$CB?$AA@ 0045f328     LIBCMT:secfail.obj
 0002:00015348       ??_C@_0LB@BPLHHLFD@A?5security?5error?5of?5unknown?5caus@ 0045f348     LIBCMT:secfail.obj
 0002:000153fc       ??_C@_0CD@GMKACBEK@Unknown?5security?5failure?5detecte@ 0045f3fc     LIBCMT:secfail.obj
 0002:00015440       ___lookuptable             0045f440     LIBCMT:output.obj
 0002:0001549c       ??_C@_1O@CEDCILHN@?$AA?$CI?$AAn?$AAu?$AAl?$AAl?$AA?$CJ?$AA?$AA@ 0045f49c     LIBCMT:output.obj
 0002:000154ac       ??_C@_06OJHGLDPL@?$CInull?$CJ?$AA@ 0045f4ac     LIBCMT:output.obj
 0002:000154d4       ??_C@_0P@GGKDKEEG@runtime?5error?5?$AA@ 0045f4d4     LIBCMT:crt0msg.obj
 0002:000154e4       ??_C@_0O@MJNIPGOH@TLOSS?5error?$AN?6?$AA@ 0045f4e4     LIBCMT:crt0msg.obj
 0002:000154f4       ??_C@_0N@BONNPDHF@SING?5error?$AN?6?$AA@ 0045f4f4     LIBCMT:crt0msg.obj
 0002:00015504       ??_C@_0P@MBDAJNE@DOMAIN?5error?$AN?6?$AA@ 0045f504     LIBCMT:crt0msg.obj
 0002:00015518       ??_C@_0KC@BDDGGBEJ@R6029?$AN?6?9?5This?5application?5cannot@ 0045f518     LIBCMT:crt0msg.obj
 0002:000155bc       ??_C@_0CF@KJDAIALP@R6028?$AN?6?9?5unable?5to?5initialize?5he@ 0045f5bc     LIBCMT:crt0msg.obj
 0002:000155e4       ??_C@_0DF@GAKBPDFP@R6027?$AN?6?9?5not?5enough?5space?5for?5lo@ 0045f5e4     LIBCMT:crt0msg.obj
 0002:0001561c       ??_C@_0DF@IBLNNAIG@R6026?$AN?6?9?5not?5enough?5space?5for?5st@ 0045f61c     LIBCMT:crt0msg.obj
 0002:00015654       ??_C@_0CG@IOHKGFNJ@R6025?$AN?6?9?5pure?5virtual?5function?5c@ 0045f654     LIBCMT:crt0msg.obj
 0002:0001567c       ??_C@_0DF@JIJJFJDC@R6024?$AN?6?9?5not?5enough?5space?5for?5_o@ 0045f67c     LIBCMT:crt0msg.obj
 0002:000156b4       ??_C@_0CJ@EGEJHFME@R6019?$AN?6?9?5unable?5to?5open?5console?5@ 0045f6b4     LIBCMT:crt0msg.obj
 0002:000156e0       ??_C@_0CB@GNHNIELH@R6018?$AN?6?9?5unexpected?5heap?5error?$AN?6@ 0045f6e0     LIBCMT:crt0msg.obj
 0002:00015704       ??_C@_0CN@FOLDKNG@R6017?$AN?6?9?5unexpected?5multithread?5@ 0045f704     LIBCMT:crt0msg.obj
 0002:00015734       ??_C@_0CM@FAHFJNHO@R6016?$AN?6?9?5not?5enough?5space?5for?5th@ 0045f734     LIBCMT:crt0msg.obj
 0002:00015760       ??_C@_0JG@LBKMGKLD@?$AN?6This?5application?5has?5requested@ 0045f760     LIBCMT:crt0msg.obj
 0002:000157f8       ??_C@_0CM@FLCNIPKK@R6009?$AN?6?9?5not?5enough?5space?5for?5en@ 0045f7f8     LIBCMT:crt0msg.obj
 0002:00015824       ??_C@_0CK@KMMJOAPP@R6008?$AN?6?9?5not?5enough?5space?5for?5ar@ 0045f824     LIBCMT:crt0msg.obj
 0002:00015850       ??_C@_0CF@HOHMHDEK@R6002?$AN?6?9?5floating?5point?5not?5load@ 0045f850     LIBCMT:crt0msg.obj
 0002:00015878       ??_C@_0BK@OFGJDLJJ@Runtime?5Error?$CB?6?6Program?3?5?$AA@ 0045f878     LIBCMT:crt0msg.obj
 0002:000158e4       ??_C@_05KLBDPFGC@e?$CL000?$AA@ 0045f8e4     LIBCMT:cvt.obj
 0002:000158f0       __real@4150017ec0000000    0045f8f0     LIBCMT:testfdiv.obj
 0002:000158f8       __real@4147ffff80000000    0045f8f8     LIBCMT:testfdiv.obj
 0002:00015900       ??_C@_0BK@NHEOCAHP@IsProcessorFeaturePresent?$AA@ 0045f900     LIBCMT:testfdiv.obj
 0002:0001591c       ??_C@_08CPNIBGIE@KERNEL32?$AA@ 0045f91c     LIBCMT:testfdiv.obj
 0002:00015934       ___dnames                  0045f934     LIBCMT:timeset.obj
 0002:0001594c       ___mnames                  0045f94c     LIBCMT:timeset.obj
 0002:00015974       ??_C@_02CLFPBFFP@TZ?$AA@   0045f974     LIBCMT:tzset.obj
 0002:00015a14       ??_C@_0CG@PKBDLMEO@InitializeCriticalSectionAndSpin@ 0045fa14     LIBCMT:initcrit.obj
 0002:00015a4c       ??_C@_08JCCMCCIL@HH?3mm?3ss?$AA@ 0045fa4c     LIBCMT:strftime.obj
 0002:00015a58       ??_C@_0BE@CKGJFCPC@dddd?0?5MMMM?5dd?0?5yyyy?$AA@ 0045fa58     LIBCMT:strftime.obj
 0002:00015a6c       ??_C@_08BPBNCDIB@MM?1dd?1yy?$AA@ 0045fa6c     LIBCMT:strftime.obj
 0002:00015a78       ??_C@_02CJNFDJBF@PM?$AA@   0045fa78     LIBCMT:strftime.obj
 0002:00015a7c       ??_C@_02DEDBPAFC@AM?$AA@   0045fa7c     LIBCMT:strftime.obj
 0002:00015a80       ??_C@_08EDHMEBNP@December?$AA@ 0045fa80     LIBCMT:strftime.obj
 0002:00015a8c       ??_C@_08HCHEGEOA@November?$AA@ 0045fa8c     LIBCMT:strftime.obj
 0002:00015a98       ??_C@_07JJNFCEND@October?$AA@ 0045fa98     LIBCMT:strftime.obj
 0002:00015aa0       ??_C@_09BHHEALKD@September?$AA@ 0045faa0     LIBCMT:strftime.obj
 0002:00015aac       ??_C@_06LBBHFDDG@August?$AA@ 0045faac     LIBCMT:strftime.obj
 0002:00015ab4       ??_C@_04MIEPOIFP@July?$AA@ 0045fab4     LIBCMT:strftime.obj
 0002:00015abc       ??_C@_04CNLMGBGM@June?$AA@ 0045fabc     LIBCMT:strftime.obj
 0002:00015ac4       ??_C@_05DMJDNLEJ@April?$AA@ 0045fac4     LIBCMT:strftime.obj
 0002:00015acc       ??_C@_05HPCKOFNC@March?$AA@ 0045facc     LIBCMT:strftime.obj
 0002:00015ad4       ??_C@_08GNJGEPFN@February?$AA@ 0045fad4     LIBCMT:strftime.obj
 0002:00015ae0       ??_C@_07CGJPFGJA@January?$AA@ 0045fae0     LIBCMT:strftime.obj
 0002:00015ae8       ??_C@_03MKABNOCG@Dec?$AA@  0045fae8     LIBCMT:strftime.obj
 0002:00015aec       ??_C@_03JPJOFNIA@Nov?$AA@  0045faec     LIBCMT:strftime.obj
 0002:00015af0       ??_C@_03BMAOKBAD@Oct?$AA@  0045faf0     LIBCMT:strftime.obj
 0002:00015af4       ??_C@_03GGCAPAJC@Sep?$AA@  0045faf4     LIBCMT:strftime.obj
 0002:00015af8       ??_C@_03IFJFEIGA@Aug?$AA@  0045faf8     LIBCMT:strftime.obj
 0002:00015afc       ??_C@_03LBGABGKK@Jul?$AA@  0045fafc     LIBCMT:strftime.obj
 0002:00015b00       ??_C@_03IDFGHECI@Jun?$AA@  0045fb00     LIBCMT:strftime.obj
 0002:00015b04       ??_C@_03CNMDKL@May?$AA@    0045fb04     LIBCMT:strftime.obj
 0002:00015b08       ??_C@_03LEOLGMJP@Apr?$AA@  0045fb08     LIBCMT:strftime.obj
 0002:00015b0c       ??_C@_03ODNJBKGA@Mar?$AA@  0045fb0c     LIBCMT:strftime.obj
 0002:00015b10       ??_C@_03HJBDCHOM@Feb?$AA@  0045fb10     LIBCMT:strftime.obj
 0002:00015b14       ??_C@_03JIHJHPIE@Jan?$AA@  0045fb14     LIBCMT:strftime.obj
 0002:00015b18       ??_C@_08INBOOONO@Saturday?$AA@ 0045fb18     LIBCMT:strftime.obj
 0002:00015b24       ??_C@_06JECMNKMI@Friday?$AA@ 0045fb24     LIBCMT:strftime.obj
 0002:00015b2c       ??_C@_08HACCIKIA@Thursday?$AA@ 0045fb2c     LIBCMT:strftime.obj
 0002:00015b38       ??_C@_09DLIGFAKA@Wednesday?$AA@ 0045fb38     LIBCMT:strftime.obj
 0002:00015b44       ??_C@_07BAAGCFCM@Tuesday?$AA@ 0045fb44     LIBCMT:strftime.obj
 0002:00015b4c       ??_C@_06JLEDEDGH@Monday?$AA@ 0045fb4c     LIBCMT:strftime.obj
 0002:00015b54       ??_C@_06OOPIFAJ@Sunday?$AA@ 0045fb54     LIBCMT:strftime.obj
 0002:00015b5c       ??_C@_03FEFJNEK@Sat?$AA@   0045fb5c     LIBCMT:strftime.obj
 0002:00015b60       ??_C@_03IDIOELNC@Fri?$AA@  0045fb60     LIBCMT:strftime.obj
 0002:00015b64       ??_C@_03IOFIKPDN@Thu?$AA@  0045fb64     LIBCMT:strftime.obj
 0002:00015b68       ??_C@_03MHOMLAJA@Wed?$AA@  0045fb68     LIBCMT:strftime.obj
 0002:00015b6c       ??_C@_03NAGEINEP@Tue?$AA@  0045fb6c     LIBCMT:strftime.obj
 0002:00015b70       ??_C@_03PDAGKDH@Mon?$AA@   0045fb70     LIBCMT:strftime.obj
 0002:00015b74       ??_C@_03KOEHGMDN@Sun?$AA@  0045fb74     LIBCMT:strftime.obj
 0002:00015b78       ___rgLocInfo               0045fb78     LIBCMT:getqloc.obj
 0002:0001601c       ??_C@_08PKBIPKE@Paraguay?$AA@ 0046001c     LIBCMT:getqloc.obj
 0002:00016028       ??_C@_07GHBIBIBP@Uruguay?$AA@ 00460028     LIBCMT:getqloc.obj
 0002:00016030       ??_C@_05HBNKAPDN@Chile?$AA@ 00460030     LIBCMT:getqloc.obj
 0002:00016038       ??_C@_07FEIFIPNF@Ecuador?$AA@ 00460038     LIBCMT:getqloc.obj
 0002:00016040       ??_C@_09PGNFPGME@Argentina?$AA@ 00460040     LIBCMT:getqloc.obj
 0002:0001604c       ??_C@_04IALPBJF@Peru?$AA@  0046004c     LIBCMT:getqloc.obj
 0002:00016054       ??_C@_08IJPLNLKH@Colombia?$AA@ 00460054     LIBCMT:getqloc.obj
 0002:00016060       ??_C@_09IDMFKCN@Venezuela?$AA@ 00460060     LIBCMT:getqloc.obj
 0002:0001606c       ??_C@_0BD@DNEJOGOK@Dominican?5Republic?$AA@ 0046006c     LIBCMT:getqloc.obj
 0002:00016080       ??_C@_0N@LPINDNDB@South?5Africa?$AA@ 00460080     LIBCMT:getqloc.obj
 0002:00016090       ??_C@_06BLJPEOBG@Panama?$AA@ 00460090     LIBCMT:getqloc.obj
 0002:00016098       ??_C@_0L@BOCNDGON@Luxembourg?$AA@ 00460098     LIBCMT:getqloc.obj
 0002:000160a4       ??_C@_0L@CONEHKA@Costa?5Rica?$AA@ 004600a4     LIBCMT:getqloc.obj
 0002:000160b0       ??_C@_0M@KGBPELAM@Switzerland?$AA@ 004600b0     LIBCMT:getqloc.obj
 0002:000160bc       ??_C@_09FJGLIMAG@Guatemala?$AA@ 004600bc     LIBCMT:getqloc.obj
 0002:000160c8       ??_C@_06ECHIPDMK@Canada?$AA@ 004600c8     LIBCMT:getqloc.obj
 0002:000160d0       ??_C@_0BG@CCEBNPGH@Spanish?5?9?5Modern?5Sort?$AA@ 004600d0     LIBCMT:getqloc.obj
 0002:000160e8       ??_C@_09EFGJAPAD@Australia?$AA@ 004600e8     LIBCMT:getqloc.obj
 0002:000160f4       ??_C@_07NEKHPBCG@English?$AA@ 004600f4     LIBCMT:getqloc.obj
 0002:000160fc       ??_C@_07LKIIOGFH@Austria?$AA@ 004600fc     LIBCMT:getqloc.obj
 0002:00016104       ??_C@_06EDDDIONA@German?$AA@ 00460104     LIBCMT:getqloc.obj
 0002:0001610c       ??_C@_07LIIIOFOA@Belgium?$AA@ 0046010c     LIBCMT:getqloc.obj
 0002:00016114       ??_C@_06DIAOLLEH@Mexico?$AA@ 00460114     LIBCMT:getqloc.obj
 0002:0001611c       ??_C@_07PFALJOGE@Spanish?$AA@ 0046011c     LIBCMT:getqloc.obj
 0002:00016124       ??_C@_06FFOOPAJB@Basque?$AA@ 00460124     LIBCMT:getqloc.obj
 0002:0001612c       ??_C@_06DGHNDJFJ@Sweden?$AA@ 0046012c     LIBCMT:getqloc.obj
 0002:00016134       ??_C@_07OBINPKFN@Swedish?$AA@ 00460134     LIBCMT:getqloc.obj
 0002:0001613c       ??_C@_07NCOIHDGC@Iceland?$AA@ 0046013c     LIBCMT:getqloc.obj
 0002:00016144       ??_C@_09JHBBDDIA@Icelandic?$AA@ 00460144     LIBCMT:getqloc.obj
 0002:00016150       ??_C@_06COBCPIFO@France?$AA@ 00460150     LIBCMT:getqloc.obj
 0002:00016158       ??_C@_06GODMCAND@French?$AA@ 00460158     LIBCMT:getqloc.obj
 0002:00016160       ??_C@_07MFHPMOED@Finland?$AA@ 00460160     LIBCMT:getqloc.obj
 0002:00016168       ??_C@_07MCEAMKOD@Finnish?$AA@ 00460168     LIBCMT:getqloc.obj
 0002:00016170       ??_C@_05CBHOCCK@Spain?$AA@ 00460170     LIBCMT:getqloc.obj
 0002:00016178       ??_C@_0BL@GIOEGDHB@Spanish?5?9?5Traditional?5Sort?$AA@ 00460178     LIBCMT:getqloc.obj
 0002:00016194       ___rglangidNotDefault      00460194     LIBCMT:getqloc.obj
 0002:000161a8       ___rg_country              004601a8     LIBCMT:getqloc.obj
 0002:00016260       ??_C@_0O@FMJNFNKE@united?9states?$AA@ 00460260     LIBCMT:getqloc.obj
 0002:00016270       ??_C@_0P@NDHFFKCA@united?9kingdom?$AA@ 00460270     LIBCMT:getqloc.obj
 0002:00016280       ??_C@_0BC@HHDADLGF@trinidad?5?$CG?5tobago?$AA@ 00460280     LIBCMT:getqloc.obj
 0002:00016294       ??_C@_0M@IOAEBDAC@south?9korea?$AA@ 00460294     LIBCMT:getqloc.obj
 0002:000162a0       ??_C@_0N@FIELFKIJ@south?9africa?$AA@ 004602a0     LIBCMT:getqloc.obj
 0002:000162b0       ??_C@_0M@OPNDHCMC@south?5korea?$AA@ 004602b0     LIBCMT:getqloc.obj
 0002:000162bc       ??_C@_0N@MDEOEPFI@south?5africa?$AA@ 004602bc     LIBCMT:getqloc.obj
 0002:000162cc       ??_C@_06FKAPCJLB@slovak?$AA@ 004602cc     LIBCMT:getqloc.obj
 0002:000162d4       ??_C@_0M@EFJANOAL@puerto?9rico?$AA@ 004602d4     LIBCMT:getqloc.obj
 0002:000162e0       ??_C@_08PGOJKDAI@pr?9china?$AA@ 004602e0     LIBCMT:getqloc.obj
 0002:000162ec       ??_C@_08JHDOMCMI@pr?5china?$AA@ 004602ec     LIBCMT:getqloc.obj
 0002:000162f8       ??_C@_02JHCHFBLL@nz?$AA@   004602f8     LIBCMT:getqloc.obj
 0002:000162fc       ??_C@_0M@LINHDHKP@new?9zealand?$AA@ 004602fc     LIBCMT:getqloc.obj
 0002:00016308       ??_C@_09IIIPPBDB@hong?9kong?$AA@ 00460308     LIBCMT:getqloc.obj
 0002:00016314       ??_C@_07HJLCKBG@holland?$AA@ 00460314     LIBCMT:getqloc.obj
 0002:0001631c       ??_C@_0O@LEHGMHAG@great?5britain?$AA@ 0046031c     LIBCMT:getqloc.obj
 0002:0001632c       ??_C@_07FACOMELA@england?$AA@ 0046032c     LIBCMT:getqloc.obj
 0002:00016334       ??_C@_05JIHCEICB@czech?$AA@ 00460334     LIBCMT:getqloc.obj
 0002:0001633c       ??_C@_05BBJOBLGB@china?$AA@ 0046033c     LIBCMT:getqloc.obj
 0002:00016344       ??_C@_07GPKPHICP@britain?$AA@ 00460344     LIBCMT:getqloc.obj
 0002:0001634c       ??_C@_07MHIPBHMG@america?$AA@ 0046034c     LIBCMT:getqloc.obj
 0002:00016358       ___rg_language             00460358     LIBCMT:getqloc.obj
 0002:00016560       ??_C@_03KIALPMKC@usa?$AA@  00460560     LIBCMT:getqloc.obj
 0002:00016564       ??_C@_02FGJGKGGD@us?$AA@   00460564     LIBCMT:getqloc.obj
 0002:00016568       ??_C@_02NEINDODK@uk?$AA@   00460568     LIBCMT:getqloc.obj
 0002:0001656c       ??_C@_05JMPCFJFJ@swiss?$AA@ 0046056c     LIBCMT:getqloc.obj
 0002:00016574       ??_C@_0BA@HLOCPIOD@swedish?9finland?$AA@ 00460574     LIBCMT:getqloc.obj
 0002:00016584       ??_C@_0BC@PKCNIABK@spanish?9venezuela?$AA@ 00460584     LIBCMT:getqloc.obj
 0002:00016598       ??_C@_0BA@GBHHMIJI@spanish?9uruguay?$AA@ 00460598     LIBCMT:getqloc.obj
 0002:000165a8       ??_C@_0BE@BHDOHPMC@spanish?9puerto?5rico?$AA@ 004605a8     LIBCMT:getqloc.obj
 0002:000165bc       ??_C@_0N@KMOIDGGN@spanish?9peru?$AA@ 004605bc     LIBCMT:getqloc.obj
 0002:000165cc       ??_C@_0BB@HMHLPGPH@spanish?9paraguay?$AA@ 004605cc     LIBCMT:getqloc.obj
 0002:000165e0       ??_C@_0P@MCPKNGFD@spanish?9panama?$AA@ 004605e0     LIBCMT:getqloc.obj
 0002:000165f0       ??_C@_0BC@IHOHGAIL@spanish?9nicaragua?$AA@ 004605f0     LIBCMT:getqloc.obj
 0002:00016604       ??_C@_0P@KLMJDNFJ@spanish?9modern?$AA@ 00460604     LIBCMT:getqloc.obj
 0002:00016614       ??_C@_0BA@BPAPGBCM@spanish?9mexican?$AA@ 00460614     LIBCMT:getqloc.obj
 0002:00016624       ??_C@_0BB@PDECHHHE@spanish?9honduras?$AA@ 00460624     LIBCMT:getqloc.obj
 0002:00016638       ??_C@_0BC@KLHKFGDB@spanish?9guatemala?$AA@ 00460638     LIBCMT:getqloc.obj
 0002:0001664c       ??_C@_0BE@MFOOKJAI@spanish?9el?5salvador?$AA@ 0046064c     LIBCMT:getqloc.obj
 0002:00016660       ??_C@_0BA@FCOKFPFC@spanish?9ecuador?$AA@ 00460660     LIBCMT:getqloc.obj
 0002:00016670       ??_C@_0BL@PLMGIMOO@spanish?9dominican?5republic?$AA@ 00460670     LIBCMT:getqloc.obj
 0002:0001668c       ??_C@_0BD@HLGDNMHB@spanish?9costa?5rica?$AA@ 0046068c     LIBCMT:getqloc.obj
 0002:000166a0       ??_C@_0BB@PKCBKCPE@spanish?9colombia?$AA@ 004606a0     LIBCMT:getqloc.obj
 0002:000166b4       ??_C@_0O@MCBIJGNE@spanish?9chile?$AA@ 004606b4     LIBCMT:getqloc.obj
 0002:000166c4       ??_C@_0BA@BEFEIGJJ@spanish?9bolivia?$AA@ 004606c4     LIBCMT:getqloc.obj
 0002:000166d4       ??_C@_0BC@EMECMPD@spanish?9argentina?$AA@ 004606d4     LIBCMT:getqloc.obj
 0002:000166e8       ??_C@_0BF@EALFLENP@portuguese?9brazilian?$AA@ 004606e8     LIBCMT:getqloc.obj
 0002:00016700       ??_C@_0BC@HBLEBLNN@norwegian?9nynorsk?$AA@ 00460700     LIBCMT:getqloc.obj
 0002:00016714       ??_C@_0BB@HMACDDCK@norwegian?9bokmal?$AA@ 00460714     LIBCMT:getqloc.obj
 0002:00016728       ??_C@_09BAFFPPHE@norwegian?$AA@ 00460728     LIBCMT:getqloc.obj
 0002:00016734       ??_C@_0O@EAJFJDFG@italian?9swiss?$AA@ 00460734     LIBCMT:getqloc.obj
 0002:00016744       ??_C@_0O@CNOMPGD@irish?9english?$AA@ 00460744     LIBCMT:getqloc.obj
 0002:00016754       ??_C@_0N@EDHBGCKG@german?9swiss?$AA@ 00460754     LIBCMT:getqloc.obj
 0002:00016764       ??_C@_0BC@JACMHNBP@german?9luxembourg?$AA@ 00460764     LIBCMT:getqloc.obj
 0002:00016778       ??_C@_0BE@HBGMGFEG@german?9lichtenstein?$AA@ 00460778     LIBCMT:getqloc.obj
 0002:0001678c       ??_C@_0BA@HKKBIBKL@german?9austrian?$AA@ 0046078c     LIBCMT:getqloc.obj
 0002:0001679c       ??_C@_0N@GCAEPEBK@french?9swiss?$AA@ 0046079c     LIBCMT:getqloc.obj
 0002:000167ac       ??_C@_0BC@DJFJJCK@french?9luxembourg?$AA@ 004607ac     LIBCMT:getqloc.obj
 0002:000167c0       ??_C@_0BA@NNCEDFIC@french?9canadian?$AA@ 004607c0     LIBCMT:getqloc.obj
 0002:000167d0       ??_C@_0P@CMPOCLM@french?9belgian?$AA@ 004607d0     LIBCMT:getqloc.obj
 0002:000167e0       ??_C@_0M@GHHDJOK@english?9usa?$AA@ 004607e0     LIBCMT:getqloc.obj
 0002:000167ec       ??_C@_0L@PLDJKEIL@english?9us?$AA@ 004607ec     LIBCMT:getqloc.obj
 0002:000167f8       ??_C@_0L@HJCCDMNC@english?9uk?$AA@ 004607f8     LIBCMT:getqloc.obj
 0002:00016804       ??_C@_0BK@CKLIAGJB@english?9trinidad?5y?5tobago?$AA@ 00460804     LIBCMT:getqloc.obj
 0002:00016820       ??_C@_0BF@JMJMGNNF@english?9south?5africa?$AA@ 00460820     LIBCMT:getqloc.obj
 0002:00016838       ??_C@_0L@DKIIFDFD@english?9nz?$AA@ 00460838     LIBCMT:getqloc.obj
 0002:00016844       ??_C@_0BA@ONHGJCLH@english?9jamaica?$AA@ 00460844     LIBCMT:getqloc.obj
 0002:00016854       ??_C@_0M@HJBGHOPO@english?9ire?$AA@ 00460854     LIBCMT:getqloc.obj
 0002:00016860       ??_C@_0BC@LFEKMIFB@english?9caribbean?$AA@ 00460860     LIBCMT:getqloc.obj
 0002:00016874       ??_C@_0M@OLDPFKHI@english?9can?$AA@ 00460874     LIBCMT:getqloc.obj
 0002:00016880       ??_C@_0P@OMDEHBMP@english?9belize?$AA@ 00460880     LIBCMT:getqloc.obj
 0002:00016890       ??_C@_0M@KFHFPFED@english?9aus?$AA@ 00460890     LIBCMT:getqloc.obj
 0002:0001689c       ??_C@_0BB@MNMBKDFE@english?9american?$AA@ 0046089c     LIBCMT:getqloc.obj
 0002:000168b0       ??_C@_0O@KIDLNNBA@dutch?9belgian?$AA@ 004608b0     LIBCMT:getqloc.obj
 0002:000168c0       ??_C@_0BE@JBKABBMH@chinese?9traditional?$AA@ 004608c0     LIBCMT:getqloc.obj
 0002:000168d4       ??_C@_0BC@MJJMPKCG@chinese?9singapore?$AA@ 004608d4     LIBCMT:getqloc.obj
 0002:000168e8       ??_C@_0BD@FDKADDCP@chinese?9simplified?$AA@ 004608e8     LIBCMT:getqloc.obj
 0002:000168fc       ??_C@_0BB@DBEFDDME@chinese?9hongkong?$AA@ 004608fc     LIBCMT:getqloc.obj
 0002:00016910       ??_C@_07DHNMFMCI@chinese?$AA@ 00460910     LIBCMT:getqloc.obj
 0002:00016918       ??_C@_03FNDDCHI@chi?$AA@   00460918     LIBCMT:getqloc.obj
 0002:0001691c       ??_C@_03BMMIADDJ@chh?$AA@  0046091c     LIBCMT:getqloc.obj
 0002:00016920       ??_C@_08OAIPJDGI@canadian?$AA@ 00460920     LIBCMT:getqloc.obj
 0002:0001692c       ??_C@_07HBPMNPNJ@belgian?$AA@ 0046092c     LIBCMT:getqloc.obj
 0002:00016934       ??_C@_0L@OEKOPBEL@australian?$AA@ 00460934     LIBCMT:getqloc.obj
 0002:00016940       ??_C@_0BB@MEIMBEDG@american?9english?$AA@ 00460940     LIBCMT:getqloc.obj
 0002:00016954       ??_C@_0BB@DFMDPDGB@american?5english?$AA@ 00460954     LIBCMT:getqloc.obj
 0002:00016968       ??_C@_08IJLOKOLL@american?$AA@ 00460968     LIBCMT:getqloc.obj
 0002:00016974       ??_C@_03NFKLAGEF@OCP?$AA@  00460974     LIBCMT:getqloc.obj
 0002:00016978       ??_C@_03DFHEHBHG@ACP?$AA@  00460978     LIBCMT:getqloc.obj
 0002:0001697c       ??_C@_0BC@NFIEMBLL@Norwegian?9Nynorsk?$AA@ 0046097c     LIBCMT:getqloc.obj
 0002:0001699c       ??_C@_0BI@DFKBFLJE@GetProcessWindowStation?$AA@ 0046099c     LIBCMT:crtmbox.obj
 0002:000169b4       ??_C@_0BK@CIDNPOGP@GetUserObjectInformationA?$AA@ 004609b4     LIBCMT:crtmbox.obj
 0002:000169d0       ??_C@_0BD@HHGDFDBJ@GetLastActivePopup?$AA@ 004609d0     LIBCMT:crtmbox.obj
 0002:000169e4       ??_C@_0BA@HNOPNCHB@GetActiveWindow?$AA@ 004609e4     LIBCMT:crtmbox.obj
 0002:000169f4       ??_C@_0M@CHKKJDAI@MessageBoxA?$AA@ 004609f4     LIBCMT:crtmbox.obj
 0002:00016a00       ??_C@_0L@GMPLCCII@user32?4dll?$AA@ 00460a00     LIBCMT:crtmbox.obj
 0002:00016a74       ??_C@_06IMKFLFPG@1?$CDQNAN?$AA@ 00460a74     LIBCMT:x10fout.obj
 0002:00016a7c       ??_C@_05DNEBIAHO@1?$CDINF?$AA@ 00460a7c     LIBCMT:x10fout.obj
 0002:00016a84       ??_C@_05PHHOCPM@1?$CDIND?$AA@ 00460a84     LIBCMT:x10fout.obj
 0002:00016a8c       ??_C@_06PGGFOGJG@1?$CDSNAN?$AA@ 00460a8c     LIBCMT:x10fout.obj
 0002:00016ab0       _GUID_ATLVer30             00460ab0     atls:atlbase.obj
 0002:00016ac0       _GUID_ATLVer70             00460ac0     atls:atlbase.obj
 0002:00016ad0       _IID_IAccessor             00460ad0     uuid:oledbiid.obj
 0002:00016ae0       _IID_IRowset               00460ae0     uuid:oledbiid.obj
 0002:00016af0       _IID_IRowsetInfo           00460af0     uuid:oledbiid.obj
 0002:00016b00       _IID_IRowsetLocate         00460b00     uuid:oledbiid.obj
 0002:00016b10       _IID_IRowsetResynch        00460b10     uuid:oledbiid.obj
 0002:00016b20       _IID_IRowsetScroll         00460b20     uuid:oledbiid.obj
 0002:00016b30       _IID_IChapteredRowset      00460b30     uuid:oledbiid.obj
 0002:00016b40       _IID_IRowsetFind           00460b40     uuid:oledbiid.obj
 0002:00016b50       _IID_IRowPosition          00460b50     uuid:oledbiid.obj
 0002:00016b60       _IID_IRowPositionChange    00460b60     uuid:oledbiid.obj
 0002:00016b70       _IID_IViewRowset           00460b70     uuid:oledbiid.obj
 0002:00016b80       _IID_IViewChapter          00460b80     uuid:oledbiid.obj
 0002:00016b90       _IID_IViewSort             00460b90     uuid:oledbiid.obj
 0002:00016ba0       _IID_IViewFilter           00460ba0     uuid:oledbiid.obj
 0002:00016bb0       _IID_IRowsetView           00460bb0     uuid:oledbiid.obj
 0002:00016bc0       _IID_IRowsetExactScroll    00460bc0     uuid:oledbiid.obj
 0002:00016bd0       _IID_IRowsetChange         00460bd0     uuid:oledbiid.obj
 0002:00016be0       _IID_IRowsetUpdate         00460be0     uuid:oledbiid.obj
 0002:00016bf0       _IID_IRowsetIdentity       00460bf0     uuid:oledbiid.obj
 0002:00016c00       _IID_IRowsetNotify         00460c00     uuid:oledbiid.obj
 0002:00016c10       _IID_IRowsetIndex          00460c10     uuid:oledbiid.obj
 0002:00016c20       _IID_ICommand              00460c20     uuid:oledbiid.obj
 0002:00016c30       _IID_IMultipleResults      00460c30     uuid:oledbiid.obj
 0002:00016c40       _IID_IConvertType          00460c40     uuid:oledbiid.obj
 0002:00016c50       _IID_ICommandPrepare       00460c50     uuid:oledbiid.obj
 0002:00016c60       _IID_ICommandProperties    00460c60     uuid:oledbiid.obj
 0002:00016c70       _IID_ICommandText          00460c70     uuid:oledbiid.obj
 0002:00016c80       _IID_ICommandWithParameters 00460c80     uuid:oledbiid.obj
 0002:00016c90       _IID_IColumnsRowset        00460c90     uuid:oledbiid.obj
 0002:00016ca0       _IID_IColumnsInfo          00460ca0     uuid:oledbiid.obj
 0002:00016cb0       _IID_IDBCreateCommand      00460cb0     uuid:oledbiid.obj
 0002:00016cc0       _IID_IDBCreateSession      00460cc0     uuid:oledbiid.obj
 0002:00016cd0       _IID_ISourcesRowset        00460cd0     uuid:oledbiid.obj
 0002:00016ce0       _IID_IDBProperties         00460ce0     uuid:oledbiid.obj
 0002:00016cf0       _IID_IDBInitialize         00460cf0     uuid:oledbiid.obj
 0002:00016d00       _IID_IDBInfo               00460d00     uuid:oledbiid.obj
 0002:00016d10       _IID_IDBDataSourceAdmin    00460d10     uuid:oledbiid.obj
 0002:00016d20       _IID_IDBAsynchNotify       00460d20     uuid:oledbiid.obj
 0002:00016d30       _IID_IDBAsynchStatus       00460d30     uuid:oledbiid.obj
 0002:00016d40       _IID_ISessionProperties    00460d40     uuid:oledbiid.obj
 0002:00016d50       _IID_IIndexDefinition      00460d50     uuid:oledbiid.obj
 0002:00016d60       _IID_ITableDefinition      00460d60     uuid:oledbiid.obj
 0002:00016d70       _IID_IOpenRowset           00460d70     uuid:oledbiid.obj
 0002:00016d80       _IID_IDBSchemaRowset       00460d80     uuid:oledbiid.obj
 0002:00016d90       _IID_IMDDataset            00460d90     uuid:oledbiid.obj
 0002:00016da0       _IID_IMDFind               00460da0     uuid:oledbiid.obj
 0002:00016db0       _IID_IMDRangeRowset        00460db0     uuid:oledbiid.obj
 0002:00016dc0       _IID_IAlterTable           00460dc0     uuid:oledbiid.obj
 0002:00016dd0       _IID_IAlterIndex           00460dd0     uuid:oledbiid.obj
 0002:00016de0       _IID_IRowsetChapterMember  00460de0     uuid:oledbiid.obj
 0002:00016df0       _IID_ICommandPersist       00460df0     uuid:oledbiid.obj
 0002:00016e00       _IID_IRowsetRefresh        00460e00     uuid:oledbiid.obj
 0002:00016e10       _IID_IParentRowset         00460e10     uuid:oledbiid.obj
 0002:00016e20       _IID_IErrorRecords         00460e20     uuid:oledbiid.obj
 0002:00016e30       _IID_IErrorLookup          00460e30     uuid:oledbiid.obj
 0002:00016e40       _IID_ISQLErrorInfo         00460e40     uuid:oledbiid.obj
 0002:00016e50       _IID_IGetDataSource        00460e50     uuid:oledbiid.obj
 0002:00016e60       _IID_ITransactionLocal     00460e60     uuid:oledbiid.obj
 0002:00016e70       _IID_ITransactionJoin      00460e70     uuid:oledbiid.obj
 0002:00016e80       _IID_ITransactionObject    00460e80     uuid:oledbiid.obj
 0002:00016e90       _IID_ITrusteeAdmin         00460e90     uuid:oledbiid.obj
 0002:00016ea0       _IID_ITrusteeGroupAdmin    00460ea0     uuid:oledbiid.obj
 0002:00016eb0       _IID_IObjectAccessControl  00460eb0     uuid:oledbiid.obj
 0002:00016ec0       _IID_ISecurityInfo         00460ec0     uuid:oledbiid.obj
 0002:00016ed0       _IID_ITableCreation        00460ed0     uuid:oledbiid.obj
 0002:00016ee0       _IID_ITableDefinitionWithConstraints 00460ee0     uuid:oledbiid.obj
 0002:00016ef0       _IID_IRow                  00460ef0     uuid:oledbiid.obj
 0002:00016f00       _IID_IRowChange            00460f00     uuid:oledbiid.obj
 0002:00016f10       _IID_IRowSchemaChange      00460f10     uuid:oledbiid.obj
 0002:00016f20       _IID_IGetRow               00460f20     uuid:oledbiid.obj
 0002:00016f30       _IID_IBindResource         00460f30     uuid:oledbiid.obj
 0002:00016f40       _IID_IScopedOperations     00460f40     uuid:oledbiid.obj
 0002:00016f50       _IID_ICreateRow            00460f50     uuid:oledbiid.obj
 0002:00016f60       _IID_IDBBinderProperties   00460f60     uuid:oledbiid.obj
 0002:00016f70       _IID_IColumnsInfo2         00460f70     uuid:oledbiid.obj
 0002:00016f80       _IID_IRegisterProvider     00460f80     uuid:oledbiid.obj
 0002:00016f90       _IID_IGetSession           00460f90     uuid:oledbiid.obj
 0002:00016fa0       _IID_IGetSourceRow         00460fa0     uuid:oledbiid.obj
 0002:00016fb0       _IID_IRowsetCurrentIndex   00460fb0     uuid:oledbiid.obj
 0002:00016fc0       _IID_ICommandStream        00460fc0     uuid:oledbiid.obj
 0002:00016fd0       _IID_IRowsetBookmark       00460fd0     uuid:oledbiid.obj
 0002:00016fe0       _IID_IService              00460fe0     uuid:oledbdat.obj
 0002:00016ff0       _IID_IDBPromptInitialize   00460ff0     uuid:oledbdat.obj
 0002:00017000       _IID_IDataInitialize       00461000     uuid:oledbdat.obj
 0002:00017010       _IID_IDataSourceLocator    00461010     uuid:oledbdat.obj
 0002:00017020       _CLSID_DataLinks           00461020     uuid:oledbdat.obj
 0002:00017030       _CLSID_MSDAINITIALIZE      00461030     uuid:oledbdat.obj
 0002:00017040       _CLSID_PDPO                00461040     uuid:oledbdat.obj
 0002:00017050       _CLSID_RootBinder          00461050     uuid:oledbdat.obj
 0002:00017060       _CLSID_DataConvert         00461060     uuid:oledbdat.obj
 0002:00017108       ??_R1A@?0A@A@exception@@8  00461108     libcpmt:string.obj
 0002:00017120       ??_R1A@?0A@A@logic_error@std@@8 00461120     libcpmt:string.obj
 0002:00017138       ??_R2logic_error@std@@8    00461138     libcpmt:string.obj
 0002:00017144       ??_R3logic_error@std@@8    00461144     libcpmt:string.obj
 0002:00017154       ??_R4logic_error@std@@6B@  00461154     libcpmt:string.obj
 0002:00017168       ??_R1A@?0A@A@length_error@std@@8 00461168     libcpmt:string.obj
 0002:00017180       ??_R2length_error@std@@8   00461180     libcpmt:string.obj
 0002:00017190       ??_R3length_error@std@@8   00461190     libcpmt:string.obj
 0002:000171a0       ??_R4length_error@std@@6B@ 004611a0     libcpmt:string.obj
 0002:000171b4       ??_R1A@?0A@A@out_of_range@std@@8 004611b4     libcpmt:string.obj
 0002:000171cc       ??_R2out_of_range@std@@8   004611cc     libcpmt:string.obj
 0002:000171dc       ??_R3out_of_range@std@@8   004611dc     libcpmt:string.obj
 0002:000171ec       ??_R4out_of_range@std@@6B@ 004611ec     libcpmt:string.obj
 0002:00017200       ??_R13?0A@A@?$_Iosb@H@std@@8 00461200     libcpmt:ios.obj
 0002:00017218       ??_R1A@?0A@A@ios_base@std@@8 00461218     libcpmt:ios.obj
 0002:00017230       ??_R2ios_base@std@@8       00461230     libcpmt:ios.obj
 0002:0001723c       ??_R3ios_base@std@@8       0046123c     libcpmt:ios.obj
 0002:0001724c       ??_R4ios_base@std@@6B@     0046124c     libcpmt:ios.obj
 0002:00017260       ??_R1A@?0A@A@runtime_error@std@@8 00461260     libcpmt:ios.obj
 0002:00017278       ??_R2runtime_error@std@@8  00461278     libcpmt:ios.obj
 0002:00017284       ??_R3runtime_error@std@@8  00461284     libcpmt:ios.obj
 0002:00017294       ??_R4runtime_error@std@@6B@ 00461294     libcpmt:ios.obj
 0002:000172a8       ??_R1A@?0A@A@failure@ios_base@std@@8 004612a8     libcpmt:ios.obj
 0002:000172c0       ??_R2failure@ios_base@std@@8 004612c0     libcpmt:ios.obj
 0002:000172d0       ??_R3failure@ios_base@std@@8 004612d0     libcpmt:ios.obj
 0002:000172e0       ??_R4failure@ios_base@std@@6B@ 004612e0     libcpmt:ios.obj
 0002:000172f4       ??_R1A@?0A@A@facet@locale@std@@8 004612f4     libcpmt:locale0.obj
 0002:0001730c       ??_R2facet@locale@std@@8   0046130c     libcpmt:locale0.obj
 0002:00017314       ??_R3facet@locale@std@@8   00461314     libcpmt:locale0.obj
 0002:00017324       ??_R4facet@locale@std@@6B@ 00461324     libcpmt:locale0.obj
 0002:00017338       ??_R1A@?0A@A@_Locimp@locale@std@@8 00461338     libcpmt:locale0.obj
 0002:00017350       ??_R2_Locimp@locale@std@@8 00461350     libcpmt:locale0.obj
 0002:0001735c       ??_R3_Locimp@locale@std@@8 0046135c     libcpmt:locale0.obj
 0002:0001736c       ??_R4_Locimp@locale@std@@6B@ 0046136c     libcpmt:locale0.obj
 0002:00017380       ??_R1A@?0A@A@ctype_base@std@@8 00461380     libcpmt:cout.obj
 0002:00017398       ??_R13A@3A@?$_Iosb@H@std@@8 00461398     libcpmt:cout.obj
 0002:000173b0       ??_R1A@A@3A@ios_base@std@@8 004613b0     libcpmt:cout.obj
 0002:000173c8       ??_R1A@A@3BA@?$basic_ios@DU?$char_traits@D@std@@@std@@8 004613c8     libcpmt:cout.obj
 0002:000173e0       ??_R1A@?0A@A@?$basic_ostream@DU?$char_traits@D@std@@@std@@8 004613e0     libcpmt:cout.obj
 0002:000173f8       ??_R2?$basic_ostream@DU?$char_traits@D@std@@@std@@8 004613f8     libcpmt:cout.obj
 0002:0001740c       ??_R3?$basic_ostream@DU?$char_traits@D@std@@@std@@8 0046140c     libcpmt:cout.obj
 0002:0001741c       ??_R4?$basic_ostream@DU?$char_traits@D@std@@@std@@6B@ 0046141c     libcpmt:cout.obj
 0002:00017430       ??_R1A@?0A@A@?$basic_ios@DU?$char_traits@D@std@@@std@@8 00461430     libcpmt:cout.obj
 0002:00017448       ??_R2?$basic_ios@DU?$char_traits@D@std@@@std@@8 00461448     libcpmt:cout.obj
 0002:00017458       ??_R3?$basic_ios@DU?$char_traits@D@std@@@std@@8 00461458     libcpmt:cout.obj
 0002:00017468       ??_R4?$basic_ios@DU?$char_traits@D@std@@@std@@6B@ 00461468     libcpmt:cout.obj
 0002:0001747c       ??_R1A@?0A@A@?$ctype@D@std@@8 0046147c     libcpmt:cout.obj
 0002:00017494       ??_R2?$ctype@D@std@@8      00461494     libcpmt:cout.obj
 0002:000174a4       ??_R3?$ctype@D@std@@8      004614a4     libcpmt:cout.obj
 0002:000174b4       ??_R4?$ctype@D@std@@6B@    004614b4     libcpmt:cout.obj
 0002:000174c8       ??_R1A@?0A@A@?$basic_streambuf@DU?$char_traits@D@std@@@std@@8 004614c8     libcpmt:cout.obj
 0002:000174e0       ??_R2?$basic_streambuf@DU?$char_traits@D@std@@@std@@8 004614e0     libcpmt:cout.obj
 0002:000174e8       ??_R3?$basic_streambuf@DU?$char_traits@D@std@@@std@@8 004614e8     libcpmt:cout.obj
 0002:000174f8       ??_R4?$basic_streambuf@DU?$char_traits@D@std@@@std@@6B@ 004614f8     libcpmt:cout.obj
 0002:0001750c       ??_R1A@?0A@A@?$basic_filebuf@DU?$char_traits@D@std@@@std@@8 0046150c     libcpmt:cout.obj
 0002:00017524       ??_R2?$basic_filebuf@DU?$char_traits@D@std@@@std@@8 00461524     libcpmt:cout.obj
 0002:00017530       ??_R3?$basic_filebuf@DU?$char_traits@D@std@@@std@@8 00461530     libcpmt:cout.obj
 0002:00017540       ??_R4?$basic_filebuf@DU?$char_traits@D@std@@@std@@6B@ 00461540     libcpmt:cout.obj
 0002:00017554       ??_R1A@?0A@A@codecvt_base@std@@8 00461554     libcpmt:cout.obj
 0002:0001756c       ??_R1A@?0A@A@?$codecvt@DDH@std@@8 0046156c     libcpmt:cout.obj
 0002:00017584       ??_R2?$codecvt@DDH@std@@8  00461584     libcpmt:cout.obj
 0002:00017594       ??_R3?$codecvt@DDH@std@@8  00461594     libcpmt:cout.obj
 0002:000175a4       ??_R4?$codecvt@DDH@std@@6B@ 004615a4     libcpmt:cout.obj
 0002:000175b8       ??_R1A@?0A@A@bad_alloc@std@@8 004615b8     libcpmt:nomemory.obj
 0002:000175d0       ??_R2bad_alloc@std@@8      004615d0     libcpmt:nomemory.obj
 0002:000175dc       ??_R3bad_alloc@std@@8      004615dc     libcpmt:nomemory.obj
 0002:000175ec       ??_R4bad_alloc@std@@6B@    004615ec     libcpmt:nomemory.obj
 0002:00017600       ??_R2exception@@8          00461600     LIBCMT:stdexcpt.obj
 0002:00017608       ??_R3exception@@8          00461608     LIBCMT:stdexcpt.obj
 0002:00017618       ??_R4exception@@6B@        00461618     LIBCMT:stdexcpt.obj
 0002:0001762c       ??_R1A@?0A@A@bad_cast@@8   0046162c     LIBCMT:stdexcpt.obj
 0002:00017644       ??_R2bad_cast@@8           00461644     LIBCMT:stdexcpt.obj
 0002:00017650       ??_R3bad_cast@@8           00461650     LIBCMT:stdexcpt.obj
 0002:00017660       ??_R4bad_cast@@6B@         00461660     LIBCMT:stdexcpt.obj
 0002:00017674       ??_R1A@?0A@A@type_info@@8  00461674     LIBCMT:typinfo.obj
 0002:0001768c       ??_R2type_info@@8          0046168c     LIBCMT:typinfo.obj
 0002:00017694       ??_R3type_info@@8          00461694     LIBCMT:typinfo.obj
 0002:000176a4       ??_R4type_info@@6B@        004616a4     LIBCMT:typinfo.obj
 0002:000176b8       ___rtc_iaa                 004616b8     LIBCMT:initsect.obj
 0002:000176bc       ___rtc_izz                 004616bc     LIBCMT:initsect.obj
 0002:000176c0       ___rtc_taa                 004616c0     LIBCMT:initsect.obj
 0002:000176c4       ___rtc_tzz                 004616c4     LIBCMT:initsect.obj
 0002:00017a68       __CT??_R0?AVexception@@@8??0exception@@QAE@ABV0@@Z12 00461a68     authorizeuser.obj
 0002:00017a84       __CT??_R0?AVlogic_error@std@@@8??0logic_error@std@@QAE@ABV01@@Z40 00461a84     authorizeuser.obj
 0002:00017aa0       __CT??_R0?AVlength_error@std@@@8??0length_error@std@@QAE@ABV01@@Z40 00461aa0     authorizeuser.obj
 0002:00017abc       __CTA3?AVlength_error@std@@ 00461abc     authorizeuser.obj
 0002:00017acc       __TI3?AVlength_error@std@@ 00461acc     authorizeuser.obj
 0002:00017fd0       __CT??_R0?AVout_of_range@std@@@8??0out_of_range@std@@QAE@ABV01@@Z40 00461fd0     rylgamelibrary:serverrequest.obj
 0002:00017fec       __CTA3?AVout_of_range@std@@ 00461fec     rylgamelibrary:serverrequest.obj
 0002:00017ffc       __TI3?AVout_of_range@std@@ 00461ffc     rylgamelibrary:serverrequest.obj
 0002:00018dd4       __CT??_R0?AVbad_cast@@@8??0bad_cast@@QAE@ABV0@@Z12 00462dd4     rylgamelibrary:regfunctions.obj
 0002:00018df0       __CTA2?AVbad_cast@@        00462df0     rylgamelibrary:regfunctions.obj
 0002:00018dfc       __TI2?AVbad_cast@@         00462dfc     rylgamelibrary:regfunctions.obj
 0002:0001945c       __CT??_R0?AVbad_alloc@std@@@8??0bad_alloc@std@@QAE@ABV01@@Z12 0046345c     rylgamelibrary:creaturemanager.obj
 0002:00019478       __CTA2?AVbad_alloc@std@@   00463478     rylgamelibrary:creaturemanager.obj
 0002:00019484       __TI2?AVbad_alloc@std@@    00463484     rylgamelibrary:creaturemanager.obj
 0002:0001a0ac       __CT??_R0?AVruntime_error@std@@@8??0runtime_error@std@@QAE@ABV01@@Z40 004640ac     libcpmt:ios.obj
 0002:0001a0c8       __CT??_R0?AVfailure@ios_base@std@@@8??0failure@ios_base@std@@QAE@ABV012@@Z40 004640c8     libcpmt:ios.obj
 0002:0001a0e4       __CTA3?AVfailure@ios_base@std@@ 004640e4     libcpmt:ios.obj
 0002:0001a0f4       __TI3?AVfailure@ios_base@std@@ 004640f4     libcpmt:ios.obj
 0002:0001a274       __IMPORT_DESCRIPTOR_KERNEL32 00464274     kernel32:KERNEL32.dll
 0002:0001a288       __IMPORT_DESCRIPTOR_USER32 00464288     user32:USER32.dll
 0002:0001a29c       __IMPORT_DESCRIPTOR_WS2_32 0046429c     ws2_32:WS2_32.dll
 0002:0001a2b0       __IMPORT_DESCRIPTOR_WINMM  004642b0     winmm:WINMM.dll
 0002:0001a2c4       __IMPORT_DESCRIPTOR_MSWSOCK 004642c4     mswsock:MSWSOCK.dll
 0002:0001a2d8       __IMPORT_DESCRIPTOR_GDI32  004642d8     gdi32:GDI32.dll
 0002:0001a2ec       __IMPORT_DESCRIPTOR_ADVAPI32 004642ec     advapi32:ADVAPI32.dll
 0002:0001a300       __IMPORT_DESCRIPTOR_SHELL32 00464300     shell32:SHELL32.dll
 0002:0001a314       __IMPORT_DESCRIPTOR_ole32  00464314     ole32:ole32.dll
 0002:0001a328       __IMPORT_DESCRIPTOR_OLEAUT32 00464328     oleaut32:OLEAUT32.dll
 0002:0001a33c       __NULL_IMPORT_DESCRIPTOR   0046433c     kernel32:KERNEL32.dll
 0003:00000000       ___xc_a                    00466000     LIBCMT:crt0init.obj
 0003:000000c8       ___xc_z                    004660c8     LIBCMT:crt0init.obj
 0003:000000cc       ___xi_a                    004660cc     LIBCMT:crt0init.obj
 0003:000000e0       ___xi_z                    004660e0     LIBCMT:crt0init.obj
 0003:000000e4       ___xl_a                    004660e4     LIBCMT:tlssup.obj
 0003:000000e8       ___xl_z                    004660e8     LIBCMT:tlssup.obj
 0003:000000ec       ___xp_a                    004660ec     LIBCMT:crt0init.obj
 0003:000000f4       ___xp_z                    004660f4     LIBCMT:crt0init.obj
 0003:000000f8       ___xt_a                    004660f8     LIBCMT:crt0init.obj
 0003:00000100       ___xt_z                    00466100     LIBCMT:crt0init.obj
 0003:00000144       ??_R0?AVexception@@@8      00466144     authorizeuser.obj
 0003:0000015c       ??_R0?AVlogic_error@std@@@8 0046615c     authorizeuser.obj
 0003:0000017c       ??_R0?AVlength_error@std@@@8 0046617c     authorizeuser.obj
 0003:000001f0       ??_R0?AVout_of_range@std@@@8 004661f0     rylgamelibrary:serverrequest.obj
 0003:000002b8       ?ms_szItemScriptFileName@CItemMgr@Item@@0PBDB 004662b8     rylgamelibrary:itemmgr.obj
 0003:000002bc       ?ms_szBGItemScriptFileName@CItemMgr@Item@@0PBDB 004662bc     rylgamelibrary:itemmgr.obj
 0003:000002c0       ?ms_szChemicalScriptFileName@CItemMgr@Item@@0PBDB 004662c0     rylgamelibrary:itemmgr.obj
 0003:000002f8       ?ms_this@CServerWindowFramework@@0PBDB 004662f8     rylgamelibrary:serverwindowframework.obj
 0003:00000300       ?WINCONSOLE_NAME@@3PBDB    00466300     rylgamelibrary:consolewindow.obj
 0003:00000304       ?WINCONSOLE_FONTNAME@@3PBDB 00466304     rylgamelibrary:consolewindow.obj
 0003:00000308       ?ms_this@CConsoleWindow@@0PBDB 00466308     rylgamelibrary:consolewindow.obj
 0003:0000030c       ??_R0?AVbad_cast@@@8       0046630c     rylgamelibrary:regfunctions.obj
 0003:000003d8       ?Attributes@Attribute@Item@@3QBVCTypeName@@B 004663d8     rylgamelibrary:itemconstants.obj
 0003:000004f0       ?Grades@Grade@Item@@3QBVCTypeName@@B 004664f0     rylgamelibrary:itemconstants.obj
 0003:00000648       ?ms_this@CTimerProcMgr@@0PBDB 00466648     rylgamelibrary:timerproc.obj
 0003:000006f8       ?ms_szSkillScriptFileName@CSkillMgr@@0PBDB 004666f8     rylgamelibrary:skillmgr.obj
 0003:000008ac       _z_errmsg                  004668ac     rylgamelibrary:zutil.obj
 0003:00000910       ?m_aryNormalAttackable@CCreatureManager@@0PAY0N@EA 00466910     rylgamelibrary:creaturemanager.obj
 0003:000009c0       ?m_arySiegeTimeAttackable@CCreatureManager@@0PAY0N@EA 004669c0     rylgamelibrary:creaturemanager.obj
 0003:00000a6c       ??_R0?AVbad_alloc@std@@@8  00466a6c     rylgamelibrary:creaturemanager.obj
 0003:00000abc       ?SkillTypes@Type@Skill@@3QBVCTypeName@@B 00466abc     rylgamelibrary:skillstructure.obj
 0003:00000af8       ?UseLimits@UseLimit@Skill@@3QBVCTypeName@@B 00466af8     rylgamelibrary:skillstructure.obj
 0003:00000b70       ?StatusLimits@StatusLimit@Skill@@3QBVCTypeName@@B 00466b70     rylgamelibrary:skillstructure.obj
 0003:00000ba0       ?TargetTypes@Target@Skill@@3QBVCTypeName@@B 00466ba0     rylgamelibrary:skillstructure.obj
 0003:00000c38       ?ClassTable@@3PAVCClass@@A 00466c38     rylgamelibrary:characterclass.obj
 0003:00000f58       ?s_arrdwCrc32Table@CCrc32Static@@1PAKA 00466f58     rylgamelibrary:crc32static.obj
 0003:000013f8       ?ms_CellSize@CCell@@2EA    004673f8     rylgamelibrary:cell.obj
 0003:00001468       ?m_szMonsterScriptFileName@CMonsterMgr@@0PBDB 00467468     rylgamelibrary:monstermgr.obj
 0003:00001650       ?ms_szEventScriptFileName@CLotteryEvent@@1PBDB 00467650     rylgamelibrary:lotteryevent.obj
 0003:000032e8       ?szQuestScriptFileName@@3PBDB 004692e8     rylgamelibrary:npc.obj
 0003:000032ec       ?szNPCScriptFileName@@3PBDB 004692ec     rylgamelibrary:npc.obj
 0003:000043f8       _inflate_mask              0046a3f8     rylgamelibrary:infutil.obj
 0003:000044b0       ?ms_DefaultFileName@CMonsterShout@@0PBDB 0046a4b0     rylgamelibrary:monstershout.obj
 0003:000045f0       ?g_pfuncCompilerMessage@@3P6AXPBD@ZA 0046a5f0     rylgamelibrary:message.obj
 0003:000045f8       ?SyntaxTypeName@@3PAPBDA   0046a5f8     rylgamelibrary:syntaxtree.obj
 0003:000046f0       ?DataTypeString@@3PAPBDA   0046a6f0     rylgamelibrary:symboltable.obj
 0003:00004708       ?lineno@@3HA               0046a708     rylgamelibrary:lex.obj
 0003:00004710       ?g_GenCodeFunctions@@3PAP6AXPAUSNode@@W4eRegister@@@ZA 0046a710     rylgamelibrary:imcodegen.obj
 0003:00004844       ?arrReg1@@3PAEA            0046a844     rylgamelibrary:imcodeunits.obj
 0003:0000484c       ?arrReg2@@3PAEA            0046a84c     rylgamelibrary:imcodeunits.obj
 0003:00004854       ?arrReg3@@3PAEA            0046a854     rylgamelibrary:imcodeunits.obj
 0003:0000485c       ?arrReg4@@3PAEA            0046a85c     rylgamelibrary:imcodeunits.obj
 0003:00004864       ?_Sync@ios_base@std@@0_NA  0046a864     libcpmt:ios.obj
 0003:00004868       ??_R0?AV?$_Iosb@H@std@@@8  0046a868     libcpmt:ios.obj
 0003:00004884       ??_R0?AVios_base@std@@@8   0046a884     libcpmt:ios.obj
 0003:000048a0       ??_R0?AVruntime_error@std@@@8 0046a8a0     libcpmt:ios.obj
 0003:000048c0       ??_R0?AVfailure@ios_base@std@@@8 0046a8c0     libcpmt:ios.obj
 0003:000048e8       ??_R0?AVfacet@locale@std@@@8 0046a8e8     libcpmt:locale0.obj
 0003:00004908       ??_R0?AV_Locimp@locale@std@@@8 0046a908     libcpmt:locale0.obj
 0003:0000492c       ??_R0?AUctype_base@std@@@8 0046a92c     libcpmt:cout.obj
 0003:0000494c       ??_R0?AV?$basic_ios@DU?$char_traits@D@std@@@std@@@8 0046a94c     libcpmt:cout.obj
 0003:00004984       ??_R0?AV?$basic_ostream@DU?$char_traits@D@std@@@std@@@8 0046a984     libcpmt:cout.obj
 0003:000049c0       ??_R0?AV?$ctype@D@std@@@8  0046a9c0     libcpmt:cout.obj
 0003:000049dc       ??_R0?AV?$basic_streambuf@DU?$char_traits@D@std@@@std@@@8 0046a9dc     libcpmt:cout.obj
 0003:00004a18       ??_R0?AV?$basic_filebuf@DU?$char_traits@D@std@@@std@@@8 0046aa18     libcpmt:cout.obj
 0003:00004a54       ??_R0?AVcodecvt_base@std@@@8 0046aa54     libcpmt:cout.obj
 0003:00004a74       ??_R0?AV?$codecvt@DDH@std@@@8 0046aa74     libcpmt:cout.obj
 0003:00004aa0       ?_PJP_CPP_Copyright@@3PADA 0046aaa0     libcpmt:iosptrs.obj
 0003:00004afc       __NLG_Destination          0046aafc     LIBCMT:exsup.obj
 0003:00004b0c       ___security_cookie         0046ab0c     LIBCMT:seccook.obj
 0003:00004b10       ?__pMyUnhandledExceptionFilter@@3PAXA 0046ab10     LIBCMT:throw.obj
 0003:00004b14       ??_R0?AVtype_info@@@8      0046ab14     LIBCMT:typinfo.obj
 0003:00004b30       __aexit_rtn                0046ab30     LIBCMT:wincrt0.obj
 0003:00004b34       ___app_type                0046ab34     LIBCMT:wincrt0.obj
 0003:00004b38       __fltused                  0046ab38     LIBCMT:fpinit.obj
 0003:00004b3c       __ldused                   0046ab3c     LIBCMT:fpinit.obj
 0003:00004b40       __FPinit                   0046ab40     LIBCMT:fpinit.obj
 0003:00004b44       __FPmtinit                 0046ab44     LIBCMT:fpinit.obj
 0003:00004b48       __FPmtterm                 0046ab48     LIBCMT:fpinit.obj
 0003:00004b50       __iob                      0046ab50     LIBCMT:_file.obj
 0003:00004f40       ___lconv_static_decimal    0046af40     LIBCMT:lconv.obj
 0003:00004f44       ___lconv_c                 0046af44     LIBCMT:lconv.obj
 0003:00004f74       ___lconv                   0046af74     LIBCMT:lconv.obj
 0003:00004f84       __pctype                   0046af84     LIBCMT:ctype.obj
 0003:00004f88       __pwctype                  0046af88     LIBCMT:ctype.obj
 0003:000050b8       ___initiallocinfo          0046b0b8     LIBCMT:setlocal.obj
 0003:0000510c       ___ptlocinfo               0046b10c     LIBCMT:setlocal.obj
 0003:00005248       ___lc_category             0046b248     LIBCMT:setlocal.obj
 0003:00005290       ___tlsindex                0046b290     LIBCMT:tidtable.obj
 0003:00005294       ?__pInconsistency@@3P6AXXZA 0046b294     LIBCMT:hooks.obj
 0003:000052a0       ___nullstring              0046b2a0     LIBCMT:output.obj
 0003:000052a4       ___wnullstring             0046b2a4     LIBCMT:output.obj
 0003:00005348       __XcptActTab               0046b348     LIBCMT:winxfltr.obj
 0003:000053c0       __First_FPE_Indx           0046b3c0     LIBCMT:winxfltr.obj
 0003:000053c4       __Num_FPE                  0046b3c4     LIBCMT:winxfltr.obj
 0003:000053c8       __XcptActTabSize           0046b3c8     LIBCMT:winxfltr.obj
 0003:000053cc       __XcptActTabCount          0046b3cc     LIBCMT:winxfltr.obj
 0003:000053d0       ___badioinfo               0046b3d0     LIBCMT:ioinit.obj
 0003:000053f4       __amblksiz                 0046b3f4     LIBCMT:heapinit.obj
 0003:000054f0       __cfltcvt_tab              0046b4f0     LIBCMT:cmiscdat.obj
 0003:00005508       __timezone                 0046b508     LIBCMT:timeset.obj
 0003:0000550c       __daylight                 0046b50c     LIBCMT:timeset.obj
 0003:00005510       __dstbias                  0046b510     LIBCMT:timeset.obj
 0003:00005598       __tzname                   0046b598     LIBCMT:timeset.obj
 0003:000055c0       __lpdays                   0046b5c0     LIBCMT:days.obj
 0003:000055f4       __days                     0046b5f4     LIBCMT:days.obj
 0003:00005630       ___lc_clike                0046b630     LIBCMT:nlsdata2.obj
 0003:00005634       ___mb_cur_max              0046b634     LIBCMT:nlsdata1.obj
 0003:00005638       ___decimal_point           0046b638     LIBCMT:nlsdata1.obj
 0003:0000563c       ___decimal_point_length    0046b63c     LIBCMT:nlsdata1.obj
 0003:00005640       ___lc_time_curr            0046b640     LIBCMT:strftime.obj
 0003:00005648       ___lc_time_c               0046b648     LIBCMT:strftime.obj
 0003:00005730       __pow10pos                 0046b730     LIBCMT:constpow.obj
 0003:00005890       __pow10neg                 0046b890     LIBCMT:constpow.obj
 0003:00005a00       ?ms_pSingleton@?$CSingleton@VCItemCreator@@@@0PAVCItemCreator@@A 0046ba00     authagentdispatch.obj
 0003:00005b80       ?Instance@?1??GetInstance@?$CStaticSingleton@VCMasterPassword@@@@SAAAVCMasterPassword@@XZ@4V3@A 0046bb80     authorizethread.obj
 0003:00005bd4       ?$S1@?1??GetInstance@?$CStaticSingleton@VCMasterPassword@@@@SAAAVCMasterPassword@@XZ@4IA 0046bbd4     authorizethread.obj
 0003:00005e2c       ?ms_pSingleton@?$CSingleton@VCItemMgr@Item@@@@0PAVCItemMgr@Item@@A 0046be2c     itemcreator.obj
 0003:00005e30       ?ms_pSingleton@?$CSingleton@VCItemFactory@Item@@@@0PAVCItemFactory@Item@@A 0046be30     itemcreator.obj
 0003:00005e34       ?ms_this@CItemCreator@@0V1@A 0046be34     itemcreator.obj
 0003:00005fac       ?Instance@?1??Clone@?$CConsoleCMDSingleton@VCCMDStatClear@@@@UAEPAVCConsoleCommand@@PBDI@Z@4VCCMDStatClear@@A 0046bfac     rylauthservercommands.obj
 0003:00005fb0       ??_B?1??Clone@?$CConsoleCMDSingleton@VCCMDStatClear@@@@UAEPAVCConsoleCommand@@PBDI@Z@51 0046bfb0     rylauthservercommands.obj
 0003:00005fb4       ?Instance@?1??Clone@?$CConsoleCMDSingleton@VCCMDStatLog@@@@UAEPAVCConsoleCommand@@PBDI@Z@4VCCMDStatLog@@A 0046bfb4     rylauthservercommands.obj
 0003:00005fb8       ??_B?1??Clone@?$CConsoleCMDSingleton@VCCMDStatLog@@@@UAEPAVCConsoleCommand@@PBDI@Z@51 0046bfb8     rylauthservercommands.obj
 0003:00005fbc       ?Instance@?1??Clone@?$CConsoleCMDSingleton@VCCMDStartServer@@@@UAEPAVCConsoleCommand@@PBDI@Z@4VCCMDStartServer@@A 0046bfbc     rylauthservercommands.obj
 0003:00005fc0       ??_B?1??Clone@?$CConsoleCMDSingleton@VCCMDStartServer@@@@UAEPAVCConsoleCommand@@PBDI@Z@51 0046bfc0     rylauthservercommands.obj
 0003:00005fc4       ?Instance@?1??Clone@?$CConsoleCMDSingleton@VCCMDShowStatistics@@@@UAEPAVCConsoleCommand@@PBDI@Z@4VCCMDShowStatistics@@A 0046bfc4     rylauthservercommands.obj
 0003:00005fc8       ??_B?1??Clone@?$CConsoleCMDSingleton@VCCMDShowStatistics@@@@UAEPAVCConsoleCommand@@PBDI@Z@51 0046bfc8     rylauthservercommands.obj
 0003:00005fcc       ?Instance@?1??Clone@?$CConsoleCMDSingleton@VCCMDPrintLog@@@@UAEPAVCConsoleCommand@@PBDI@Z@4VCCMDPrintLog@@A 0046bfcc     rylauthservercommands.obj
 0003:00005fd0       ??_B?1??Clone@?$CConsoleCMDSingleton@VCCMDPrintLog@@@@UAEPAVCConsoleCommand@@PBDI@Z@51 0046bfd0     rylauthservercommands.obj
 0003:00005fd4       ?Instance@?1??Clone@?$CConsoleCMDSingleton@VCCMDFlushLog@@@@UAEPAVCConsoleCommand@@PBDI@Z@4VCCMDFlushLog@@A 0046bfd4     rylauthservercommands.obj
 0003:00005fd8       ??_B?1??Clone@?$CConsoleCMDSingleton@VCCMDFlushLog@@@@UAEPAVCConsoleCommand@@PBDI@Z@51 0046bfd8     rylauthservercommands.obj
 0003:00005fdc       ?Instance@?1??Clone@?$CConsoleCMDSingleton@VCCMDReloadSetup@@@@UAEPAVCConsoleCommand@@PBDI@Z@4VCCMDReloadSetup@@A 0046bfdc     rylauthservercommands.obj
 0003:00005fe0       ??_B?1??Clone@?$CConsoleCMDSingleton@VCCMDReloadSetup@@@@UAEPAVCConsoleCommand@@PBDI@Z@51 0046bfe0     rylauthservercommands.obj
 0003:00005fe4       ?Instance@?1??Clone@?$CConsoleCMDSingleton@VCCMDMasterPass@@@@UAEPAVCConsoleCommand@@PBDI@Z@4VCCMDMasterPass@@A 0046bfe4     rylauthservercommands.obj
 0003:00005fe8       ??_B?1??Clone@?$CConsoleCMDSingleton@VCCMDMasterPass@@@@UAEPAVCConsoleCommand@@PBDI@Z@51 0046bfe8     rylauthservercommands.obj
 0003:00005fec       ?ms_pSingleton@?$CSingleton@VCXORCrypt@@@@0PAVCXORCrypt@@A 0046bfec     rylgamelibrary:rylserverdispatch.obj
 0003:00005ff0       ?g_GuildLog@@3VCServerLog@@A 0046bff0     rylgamelibrary:serverlog.obj
 0003:00006228       ?g_Log@@3VCServerLog@@A    0046c228     rylgamelibrary:serverlog.obj
 0003:00006460       ?g_SessionLog@@3VCServerLog@@A 0046c460     rylgamelibrary:serverlog.obj
 0003:00007110       ?m_bInitFailed@CAtlBaseModule@ATL@@2_NA 0046d110     rylgamelibrary:characterlog.obj
 0003:000245e4       ?ms_pSingleton@?$CSingleton@VCItemType@Item@@@@0PAVCItemType@Item@@A 0048a5e4     rylgamelibrary:itemmgr.obj
 0003:000245e8       ?ms_this@CItemMgr@Item@@0V12@A 0048a5e8     rylgamelibrary:itemmgr.obj
 0003:000245f8       ?ms_this@CItemFactory@Item@@0V12@A 0048a5f8     rylgamelibrary:itemfactory.obj
 0003:00024600       ?ms_SendDataMsg@CServerWindowFramework@@0IB 0048a600     rylgamelibrary:serverwindowframework.obj
 0003:00036f08       ?ms_PrintInfoMsg@CConsoleWindow@@0IB 0049cf08     rylgamelibrary:consolewindow.obj
 0003:00036f10       ?ms_PrintOutputMsg@CConsoleWindow@@0IB 0049cf10     rylgamelibrary:consolewindow.obj
 0003:00036f18       ?ms_this@CXORCrypt@@0V1@A  0049cf18     rylgamelibrary:xorcrypt.obj
 0003:00036f80       ?_Stz@?$fpos@H@std@@0HA    0049cf80     rylgamelibrary:regfunctions.obj
 0003:00036f84       ?_Stinit@?1??_Init@?$basic_filebuf@DU?$char_traits@D@std@@@std@@IAEXPAU_iobuf@@W4_Initfl@23@@Z@4HA 0049cf84     rylgamelibrary:regfunctions.obj
 0003:00036f88       ?_Psave@?$_Facetptr@V?$ctype@D@std@@@std@@2PBVfacet@locale@2@B 0049cf88     rylgamelibrary:regfunctions.obj
 0003:00036f8c       ?_Psave@?$_Facetptr@V?$codecvt@DDH@std@@@std@@2PBVfacet@locale@2@B 0049cf8c     rylgamelibrary:regfunctions.obj
 0003:00036f90       ?id@?$codecvt@DDH@std@@2V0locale@2@A 0049cf90     rylgamelibrary:regfunctions.obj
 0003:00036f94       ?obj@?1??instance@?$singleton_default@Upool_type@?$singleton_pool@Ufast_pool_allocator_tag@boost@@$0M@Udefault_user_allocator_new_delete@2@Vwin32_mutex@pool@details@2@$0CA@@boost@@@pool@details@boost@@SAAAUpool_type@?$singleton_pool@Ufast_pool_allocator_tag@boost@@$0M@Udefault_user_allocator_new_delete@2@Vwin32_mutex@pool@details@2@$0CA@@5@XZ@4U675@A 0049cf94     rylgamelibrary:depositcontainer.obj
 0003:00036fc0       ?$S5@?1??instance@?$singleton_default@Upool_type@?$singleton_pool@Ufast_pool_allocator_tag@boost@@$0M@Udefault_user_allocator_new_delete@2@Vwin32_mutex@pool@details@2@$0CA@@boost@@@pool@details@boost@@SAAAUpool_type@?$singleton_pool@Ufast_pool_allocator_tag@boost@@$0M@Udefault_user_allocator_new_delete@2@Vwin32_mutex@pool@details@2@$0CA@@5@XZ@4IA 0049cfc0     rylgamelibrary:depositcontainer.obj
 0003:00036fc4       ?create_object@?$singleton_default@Upool_type@?$singleton_pool@Ufast_pool_allocator_tag@boost@@$0M@Udefault_user_allocator_new_delete@2@Vwin32_mutex@pool@details@2@$0CA@@boost@@@pool@details@boost@@0Uobject_creator@1234@A 0049cfc4     rylgamelibrary:depositcontainer.obj
 0003:00036fcc       ?ms_pSingleton@?$CSingleton@VCSkillMgr@@@@0PAVCSkillMgr@@A 0049cfcc     rylgamelibrary:itemstructure.obj
 0003:00036fd0       ?ms_this@CItemType@Item@@0V12@A 0049cfd0     rylgamelibrary:itemconstants.obj
 0003:000374ac       ___lzo_init_done           0049d4ac     rylgamelibrary:minilzo.obj
 0003:000374b0       ?ms_pSingleton@?$CSingleton@VCNullItem@Item@@@@0PAVCNullItem@Item@@A 0049d4b0     rylgamelibrary:itemcontainer.obj
 0003:000374b8       ?ms_thisiteminfo@CNullItem@Item@@0UItemInfo@2@A 0049d4b8     rylgamelibrary:itemcontainer.obj
 0003:0003773c       ?ms_this@CNullItem@Item@@0V12@A 0049d73c     rylgamelibrary:itemcontainer.obj
 0003:00037760       ?ms_this@CSkillMgr@@0V1@A  0049d760     rylgamelibrary:skillmgr.obj
 0003:0003776c       ?ms_pSingleton@?$CSingleton@VCMonsterMgr@@@@0PAVCMonsterMgr@@A 0049d76c     rylgamelibrary:sendcharattack.obj
 0003:00037770       ?ms_pSingleton@?$CSingleton@VCAward@AwardTable@@@@0PAVCAward@AwardTable@@A 0049d770     rylgamelibrary:characterstatus.obj
 0003:00037774       ?ms_pSingleton@?$CSingleton@VCProcessTable@Skill@@@@0PAVCProcessTable@Skill@@A 0049d774     rylgamelibrary:characterskill.obj
 0003:00037778       ?obj@?1??instance@?$singleton_default@Upool_type@?$singleton_pool@Ufast_pool_allocator_tag@boost@@$0BI@Udefault_user_allocator_new_delete@2@Vwin32_mutex@pool@details@2@$0CA@@boost@@@pool@details@boost@@SAAAUpool_type@?$singleton_pool@Ufast_pool_allocator_tag@boost@@$0BI@Udefault_user_allocator_new_delete@2@Vwin32_mutex@pool@details@2@$0CA@@5@XZ@4U675@A 0049d778     rylgamelibrary:creaturemanager.obj
 0003:000377a4       ?$S7@?1??instance@?$singleton_default@Upool_type@?$singleton_pool@Ufast_pool_allocator_tag@boost@@$0BI@Udefault_user_allocator_new_delete@2@Vwin32_mutex@pool@details@2@$0CA@@boost@@@pool@details@boost@@SAAAUpool_type@?$singleton_pool@Ufast_pool_allocator_tag@boost@@$0BI@Udefault_user_allocator_new_delete@2@Vwin32_mutex@pool@details@2@$0CA@@5@XZ@4IA 0049d7a4     rylgamelibrary:creaturemanager.obj
 0003:000377a8       ?obj@?1??instance@?$singleton_default@Upool_type@?$singleton_pool@Ufast_pool_allocator_tag@boost@@$0BE@Udefault_user_allocator_new_delete@2@Vwin32_mutex@pool@details@2@$0CA@@boost@@@pool@details@boost@@SAAAUpool_type@?$singleton_pool@Ufast_pool_allocator_tag@boost@@$0BE@Udefault_user_allocator_new_delete@2@Vwin32_mutex@pool@details@2@$0CA@@5@XZ@4U675@A 0049d7a8     rylgamelibrary:creaturemanager.obj
 0003:000377d4       ?$S11@?1??instance@?$singleton_default@Upool_type@?$singleton_pool@Ufast_pool_allocator_tag@boost@@$0BE@Udefault_user_allocator_new_delete@2@Vwin32_mutex@pool@details@2@$0CA@@boost@@@pool@details@boost@@SAAAUpool_type@?$singleton_pool@Ufast_pool_allocator_tag@boost@@$0BE@Udefault_user_allocator_new_delete@2@Vwin32_mutex@pool@details@2@$0CA@@5@XZ@4IA 0049d7d4     rylgamelibrary:creaturemanager.obj
 0003:000377d8       ?create_object@?$singleton_default@Upool_type@?$singleton_pool@Ufast_pool_allocator_tag@boost@@$0BI@Udefault_user_allocator_new_delete@2@Vwin32_mutex@pool@details@2@$0CA@@boost@@@pool@details@boost@@0Uobject_creator@1234@A 0049d7d8     rylgamelibrary:creaturemanager.obj
 0003:000377d9       ?create_object@?$singleton_default@Upool_type@?$singleton_pool@Ufast_pool_allocator_tag@boost@@$0BE@Udefault_user_allocator_new_delete@2@Vwin32_mutex@pool@details@2@$0CA@@boost@@@pool@details@boost@@0Uobject_creator@1234@A 0049d7d9     rylgamelibrary:creaturemanager.obj
 0003:000377dc       ?obj@?1??instance@?$singleton_default@Upool_type@?$singleton_pool@Ufast_pool_allocator_tag@boost@@$0DI@Udefault_user_allocator_new_delete@2@Vwin32_mutex@pool@details@2@$0CA@@boost@@@pool@details@boost@@SAAAUpool_type@?$singleton_pool@Ufast_pool_allocator_tag@boost@@$0DI@Udefault_user_allocator_new_delete@2@Vwin32_mutex@pool@details@2@$0CA@@5@XZ@4U675@A 0049d7dc     rylgamelibrary:cell.obj
 0003:00037808       ?$S5@?1??instance@?$singleton_default@Upool_type@?$singleton_pool@Ufast_pool_allocator_tag@boost@@$0DI@Udefault_user_allocator_new_delete@2@Vwin32_mutex@pool@details@2@$0CA@@boost@@@pool@details@boost@@SAAAUpool_type@?$singleton_pool@Ufast_pool_allocator_tag@boost@@$0DI@Udefault_user_allocator_new_delete@2@Vwin32_mutex@pool@details@2@$0CA@@5@XZ@4IA 0049d808     rylgamelibrary:cell.obj
 0003:0003780c       ?create_object@?$singleton_default@Upool_type@?$singleton_pool@Ufast_pool_allocator_tag@boost@@$0DI@Udefault_user_allocator_new_delete@2@Vwin32_mutex@pool@details@2@$0CA@@boost@@@pool@details@boost@@0Uobject_creator@1234@A 0049d80c     rylgamelibrary:cell.obj
 0003:00037810       ?ms_this@CMonsterMgr@@0V1@A 0049d810     rylgamelibrary:monstermgr.obj
 0003:00037818       ?m_NullProtoType@ProcessInfo@CProcessTable@Skill@@2UProtoType@3@A 0049d818     rylgamelibrary:skilltable.obj
 0003:00037a18       ?ms_this@CProcessTable@Skill@@0V12@A 0049da18     rylgamelibrary:skilltable.obj
 0003:00037a20       ?ms_pSingleton@?$CSingleton@VCRankingMgr@@@@0PAVCRankingMgr@@A 0049da20     rylgamelibrary:sendcharetc.obj
 0003:00037a24       ?ms_pSingleton@?$CSingleton@VCDuelCellManager@@@@0PAVCDuelCellManager@@A 0049da24     rylgamelibrary:aggresivecreature.obj
 0003:00037a28       ?ms_this@CAward@AwardTable@@0V12@A 0049da28     rylgamelibrary:awardtable.obj
 0003:00037a2c       ?ms_pSingleton@?$CSingleton@VCPartyMgr@@@@0PAVCPartyMgr@@A 0049da2c     rylgamelibrary:party.obj
 0003:00037a30       ?ms_pSingleton@?$CSingleton@VCXRefFriends@@@@0PAVCXRefFriends@@A 0049da30     rylgamelibrary:character.obj
 0003:00037a34       ?ms_pSingleton@?$CSingleton@VCFSM@@@@0PAVCFSM@@A 0049da34     rylgamelibrary:cellmanager.obj
 0003:00037a38       ?id@?$num_put@DV?$ostreambuf_iterator@DU?$char_traits@D@std@@@std@@@std@@2V0locale@2@A 0049da38     rylgamelibrary:cellmanager.obj
 0003:00037a3c       ?id@?$numpunct@D@std@@2V0locale@2@A 0049da3c     rylgamelibrary:cellmanager.obj
 0003:00037a40       ?ms_NormalBehaviorSendCount@CMonster@@1JA 0049da40     rylgamelibrary:monster.obj
 0003:00037a44       ?ms_AttackBehaviorSendCount@CMonster@@1JA 0049da44     rylgamelibrary:monster.obj
 0003:00037a48       ?ms_ReturnBehaviorSendCount@CMonster@@1JA 0049da48     rylgamelibrary:monster.obj
 0003:00037a4c       ?ms_EscapeBehaviorSendCount@CMonster@@1JA 0049da4c     rylgamelibrary:monster.obj
 0003:00037a50       ?ms_DeadBehaviorSendCount@CMonster@@1JA 0049da50     rylgamelibrary:monster.obj
 0003:00037a58       ?ms_this@CRankingMgr@@0V1@A 0049da58     rylgamelibrary:rankingmgr.obj
 0003:00045130       ?ms_this@CPartyMgr@@1V1@A  004ab130     rylgamelibrary:partymgr.obj
 0003:00045158       ?ms_pSingleton@?$CSingleton@VCQuestMgr@@@@0PAVCQuestMgr@@A 004ab158     rylgamelibrary:parsecharadmin.obj
 0003:00045794       ?ms_this@CXRefFriends@@0V1@A 004ab794     rylgamelibrary:friendlist.obj
 0003:000457a0       ?ms_this@CDuelCellManager@@0V1@A 004ab7a0     rylgamelibrary:duelcellmanager.obj
 0003:000457ac       ?ms_this@CFSM@@1V1@A       004ab7ac     rylgamelibrary:fsm.obj
 0003:000457d0       ?ms_scQuestScript@CNPC@@0PAVCVirtualMachine@@A 004ab7d0     rylgamelibrary:npc.obj
 0003:000457d8       ?ms_cCurrentGroupNum@CRegularAgentDispatch@@0EA 004ab7d8     rylgamelibrary:regularagentdispatch.obj
 0003:000457e0       ?ms_AgentServerInfo@CRegularAgentDispatch@@0PAURylServerInfo@@A 004ab7e0     rylgamelibrary:regularagentdispatch.obj
 0003:000461b8       ?ms_this@CQuestMgr@@0V1@A  004ac1b8     rylgamelibrary:questmgr.obj
 0003:000461d8       ?pAllocatedPtrs@@3PAV?$set@PAXU?$less@PAX@std@@V?$allocator@PAX@2@@std@@A 004ac1d8     rylgamelibrary:virtualmachine.obj
 0003:000461e0       ?szBuffer@@3PADA           004ac1e0     rylgamelibrary:syntaxtree.obj
 0003:000471e0       ?g_pSynTree@@3PAVCSyntaxTree@@A 004ad1e0     rylgamelibrary:syntaxtree.obj
 0003:000471e4       ?g_pSymbolTable@@3PAVCSymbolTable@@A 004ad1e4     rylgamelibrary:syntaxtree.obj
 0003:00047268       ?yylval@@3TYYSTYPE@@A      004ad268     rylgamelibrary:parse.obj
 0003:00048268       ?yydebug@@3HA              004ae268     rylgamelibrary:parse.obj
 0003:0004826c       ?yychar@@3HA               004ae26c     rylgamelibrary:parse.obj
 0003:00048270       ?yylloc@@3Uyyltype@@A      004ae270     rylgamelibrary:parse.obj
 0003:00048288       ?yynerrs@@3HA              004ae288     rylgamelibrary:parse.obj
 0003:00048294       ?yytext@@3PADA             004ae294     rylgamelibrary:lex.obj
 0003:00048298       ?yyleng@@3HA               004ae298     rylgamelibrary:lex.obj
 0003:000482b4       ?yyin@@3PAU_iobuf@@A       004ae2b4     rylgamelibrary:lex.obj
 0003:000482b8       ?yyout@@3PAU_iobuf@@A      004ae2b8     rylgamelibrary:lex.obj
 0003:000482d0       ?SWITCHTEMPVAR@@3HA        004ae2d0     rylgamelibrary:imcodegen.obj
 0003:000482d4       ?FLOATUNIT@@3HA            004ae2d4     rylgamelibrary:imcodegen.obj
 0003:000482d8       ?FLOATTEMP@@3HA            004ae2d8     rylgamelibrary:imcodegen.obj
 0003:000482dc       ?STRINGTRUE@@3HA           004ae2dc     rylgamelibrary:imcodegen.obj
 0003:000482e0       ?STRINGFALSE@@3HA          004ae2e0     rylgamelibrary:imcodegen.obj
 0003:000482e4       ?CONVERSIONBUFFER@@3HA     004ae2e4     rylgamelibrary:imcodegen.obj
 0003:000482f4       ?nothrow@std@@3Unothrow_t@1@B 004ae2f4     libcpmt:nothrow.obj
 0003:000482f8       ?_Fpz@std@@3_JA            004ae2f8     libcpmt:ios.obj
 0003:00048300       ?_Index@ios_base@std@@0HA  004ae300     libcpmt:ios.obj
 0003:000483a4       ?_Clocptr@_Locimp@locale@std@@0PAV123@A 004ae3a4     libcpmt:locale0.obj
 0003:000483a8       ?_Id_cnt@id@locale@std@@0HA 004ae3a8     libcpmt:locale0.obj
 0003:000483b0       ?id@?$ctype@D@std@@2V0locale@2@A 004ae3b0     libcpmt:locale0.obj
 0003:000483b4       ?id@?$codecvt@GDH@std@@2V0locale@2@A 004ae3b4     libcpmt:locale0.obj
 0003:000483b8       ?id@?$ctype@G@std@@2V0locale@2@A 004ae3b8     libcpmt:locale0.obj
 0003:000483bc       ?id@?$codecvt@_WDH@std@@2V0locale@2@A 004ae3bc     libcpmt:locale0.obj
 0003:000483c0       ?id@?$ctype@_W@std@@2V0locale@2@A 004ae3c0     libcpmt:locale0.obj
 0003:00048428       ?cout@std@@3V?$basic_ostream@DU?$char_traits@D@std@@@1@A 004ae428     libcpmt:cout.obj
 0003:00048470       ?_Ptr_cin@std@@3PAV?$basic_istream@DU?$char_traits@D@std@@@1@A 004ae470     libcpmt:iosptrs.obj
 0003:00048474       ?_Ptr_cout@std@@3PAV?$basic_ostream@DU?$char_traits@D@std@@@1@A 004ae474     libcpmt:iosptrs.obj
 0003:00048478       ?_Ptr_cerr@std@@3PAV?$basic_ostream@DU?$char_traits@D@std@@@1@A 004ae478     libcpmt:iosptrs.obj
 0003:0004847c       ?_Ptr_clog@std@@3PAV?$basic_ostream@DU?$char_traits@D@std@@@1@A 004ae47c     libcpmt:iosptrs.obj
 0003:00048480       ?_Ptr_wcin@std@@3PAV?$basic_istream@_WU?$char_traits@_W@std@@@1@A 004ae480     libcpmt:iosptrs.obj
 0003:00048484       ?_Ptr_wcout@std@@3PAV?$basic_ostream@_WU?$char_traits@_W@std@@@1@A 004ae484     libcpmt:iosptrs.obj
 0003:00048488       ?_Ptr_wcerr@std@@3PAV?$basic_ostream@_WU?$char_traits@_W@std@@@1@A 004ae488     libcpmt:iosptrs.obj
 0003:0004848c       ?_Ptr_wclog@std@@3PAV?$basic_ostream@_WU?$char_traits@_W@std@@@1@A 004ae48c     libcpmt:iosptrs.obj
 0003:000484bc       ___pPurecall               004ae4bc     LIBCMT:purevirt.obj
 0003:000484c0       __aenvptr                  004ae4c0     LIBCMT:wincrt0.obj
 0003:000484c4       __wenvptr                  004ae4c4     LIBCMT:wincrt0.obj
 0003:000484c8       ___error_mode              004ae4c8     LIBCMT:wincrt0.obj
 0003:000484cc       ___fastflag                004ae4cc     LIBCMT:fpinit.obj
 0003:000484d0       __adjust_fdiv              004ae4d0     LIBCMT:fpinit.obj
 0003:000484d4       __cflush                   004ae4d4     LIBCMT:_file.obj
 0003:000484d8       __tls_index                004ae4d8     LIBCMT:tlssup.obj
 0003:000484dc       ___lconv_static_null       004ae4dc     LIBCMT:lconv.obj
 0003:000484e0       __umaskval                 004ae4e0     LIBCMT:crt0dat.obj
 0003:000484e4       __osplatform               004ae4e4     LIBCMT:crt0dat.obj
 0003:000484e8       __osver                    004ae4e8     LIBCMT:crt0dat.obj
 0003:000484ec       __winver                   004ae4ec     LIBCMT:crt0dat.obj
 0003:000484f0       __winmajor                 004ae4f0     LIBCMT:crt0dat.obj
 0003:000484f4       __winminor                 004ae4f4     LIBCMT:crt0dat.obj
 0003:000484f8       ___argc                    004ae4f8     LIBCMT:crt0dat.obj
 0003:000484fc       ___argv                    004ae4fc     LIBCMT:crt0dat.obj
 0003:00048500       ___wargv                   004ae500     LIBCMT:crt0dat.obj
 0003:00048504       __environ                  004ae504     LIBCMT:crt0dat.obj
 0003:00048508       ___initenv                 004ae508     LIBCMT:crt0dat.obj
 0003:0004850c       __wenviron                 004ae50c     LIBCMT:crt0dat.obj
 0003:00048510       ___winitenv                004ae510     LIBCMT:crt0dat.obj
 0003:00048514       __pgmptr                   004ae514     LIBCMT:crt0dat.obj
 0003:00048518       __wpgmptr                  004ae518     LIBCMT:crt0dat.obj
 0003:0004851c       __exitflag                 004ae51c     LIBCMT:crt0dat.obj
 0003:00048520       __C_Termination_Done       004ae520     LIBCMT:crt0dat.obj
 0003:00048524       __C_Exit_Done              004ae524     LIBCMT:crt0dat.obj
 0003:00048528       ?_pnhHeap@@3P6AHI@ZA       004ae528     LIBCMT:handler.obj
 0003:0004868c       _gpFlsAlloc                004ae68c     LIBCMT:tidtable.obj
 0003:00048690       _gpFlsGetValue             004ae690     LIBCMT:tidtable.obj
 0003:00048694       _gpFlsSetValue             004ae694     LIBCMT:tidtable.obj
 0003:00048698       _gpFlsFree                 004ae698     LIBCMT:tidtable.obj
 0003:000486a4       __adbgmsg                  004ae6a4     LIBCMT:crt0msg.obj
 0003:000487b4       __stdbuf                   004ae7b4     LIBCMT:_sftbuf.obj
 0003:00048810       __newmode                  004ae810     LIBCMT:_newmode.obj
 0003:000488f4       __commode                  004ae8f4     LIBCMT:ncommode.obj
 0003:0004891c       ___lc_handle               004ae91c     LIBCMT:nlsdata2.obj
 0003:00048934       ___lc_codepage             004ae934     LIBCMT:nlsdata2.obj
 0003:00048938       ___lc_collate_cp           004ae938     LIBCMT:nlsdata2.obj
 0003:00048948       ___lc_id                   004ae948     LIBCMT:nlsdata3.obj
 0003:00048970       ___lc_time_intl            004ae970     LIBCMT:inittime.obj
 0003:00048974       ___lconv_intl              004ae974     LIBCMT:initmon.obj
 0003:000489cc       __fmode                    004ae9cc     LIBCMT:txtmode.obj
 0003:000489d4       ?_AtlBaseModule@ATL@@3VCAtlBaseModule@1@A 004ae9d4     atls:atlbase.obj
 0003:00048a10       ___lconv_mon_refcount      004aea10     <common>
 0003:00048a14       ___lconv_intl_refcount     004aea14     <common>
 0003:00048a18       ___lconv_num_refcount      004aea18     <common>
 0003:00048a1c       ___sbh_pHeaderDefer        004aea1c     <common>
 0003:00048a20       ___sbh_cntHeaderList       004aea20     <common>
 0003:00048a24       ___sbh_pHeaderList         004aea24     <common>
 0003:00048a28       ___sbh_threshold           004aea28     <common>
 0003:00048a2c       ___sbh_pHeaderScan         004aea2c     <common>
 0003:00048a30       ___sbh_sizeHeaderList      004aea30     <common>
 0003:00048a34       ___sbh_indGroupDefer       004aea34     <common>
 0003:00048a38       ___mblcid                  004aea38     <common>
 0003:00048a3c       ___ptmbcinfo               004aea3c     <common>
 0003:00048a40       ___ismbcodepage            004aea40     <common>
 0003:00048a60       __mbctype                  004aea60     <common>
 0003:00048b64       ___mbcodepage              004aeb64     <common>
 0003:00048b70       ___mbulinfo                004aeb70     <common>
 0003:00048b80       __mbcasemap                004aeb80     <common>
 0003:00048c80       __crtheap                  004aec80     <common>
 0003:00048c84       ___active_heap             004aec84     <common>
 0003:00048c88       __nhandle                  004aec88     <common>
 0003:00048ca0       ___pioinfo                 004aeca0     <common>
 0003:00048da0       ___setlc_active            004aeda0     <common>
 0003:00048da4       ___unguarded_readlc_active 004aeda4     <common>
 0003:00048da8       ___ctype1                  004aeda8     <common>
 0003:00048dac       ___ctype1_refcount         004aedac     <common>
 0003:00048db0       ___env_initialized         004aedb0     <common>
 0003:00048db4       ___onexitend               004aedb4     <common>
 0003:00048db8       ___onexitbegin             004aedb8     <common>
 0003:00048dbc       ___mbctype_initialized     004aedbc     <common>
 0003:00048dc0       ___piob                    004aedc0     <common>
 0003:00048de0       __bufin                    004aede0     <common>
 0003:00049de0       __nstream                  004afde0     <common>
 0003:00049de4       __acmdln                   004afde4     <common>
 0004:00000000       __tls_start                004b0000     LIBCMT:tlssup.obj
 0004:0000010c       __tls_end                  004b010c     LIBCMT:tlssup.obj

 entry point at        0001:000384b2

 Static symbols

 0001:00003d13       $L34802                    00404d13 f i authorizeuser.obj
 0001:00003dab       $L34804                    00404dab f i authorizeuser.obj
 0001:00007cce       $L36084                    00408cce f i rylgamelibrary:rylserverdispatch.obj
 0001:00007cda       $L36086                    00408cda f i rylgamelibrary:rylserverdispatch.obj
 0001:00007e6a       $L36325                    00408e6a f i rylgamelibrary:rylserverdispatch.obj
 0001:0000dd1f       $L35067                    0040ed1f f i rylgamelibrary:session.obj
 0001:000103ee       $L99238                    004113ee f i rylgamelibrary:itemmgr.obj
 0001:000103fd       $L99240                    004113fd f i rylgamelibrary:itemmgr.obj
 0001:000121fa       $L35677                    004131fa f i rylgamelibrary:limituserbyip.obj
 0001:00013048       $L37932                    00414048 f i rylgamelibrary:iocpnet.obj
 0001:00013831       $L41175                    00414831 f i rylgamelibrary:iocpnet.obj
 0001:00016f11       $L32220                    00417f11 f i rylgamelibrary:consolecmdfactory.obj
 0001:00016f1d       $L32222                    00417f1d f i rylgamelibrary:consolecmdfactory.obj
 0001:0001e821       $L91066                    0041f821 f i rylgamelibrary:tokenlizedfile.obj
 0001:0001e82d       $L91068                    0041f82d f i rylgamelibrary:tokenlizedfile.obj
 0001:0001ed11       $L91538                    0041fd11 f i rylgamelibrary:tokenlizedfile.obj
 0001:0001edea       $L91658                    0041fdea f i rylgamelibrary:tokenlizedfile.obj
 0001:000201e8       $L92684                    004211e8 f i rylgamelibrary:itemconstants.obj
 0001:000201f4       $L92686                    004211f4 f i rylgamelibrary:itemconstants.obj
 0001:0002044a       $L92980                    0042144a f i rylgamelibrary:itemconstants.obj
 0001:00022a6e       $L88710                    00423a6e f i rylgamelibrary:itemdataparser.obj
 0001:00022a7a       $L88712                    00423a7a f i rylgamelibrary:itemdataparser.obj
 0001:00022c0a       $L88938                    00423c0a f i rylgamelibrary:itemdataparser.obj
 0001:000252e0       _get_byte                  004262e0 f   rylgamelibrary:gzio.obj
 0001:00025350       _check_header              00426350 f   rylgamelibrary:gzio.obj
 0001:00025730       _destroy                   00426730 f   rylgamelibrary:gzio.obj
 0001:00025880       _do_flush                  00426880 f   rylgamelibrary:gzio.obj
 0001:00025940       _putLong                   00426940 f   rylgamelibrary:gzio.obj
 0001:000259c0       _gz_open                   004269c0 f   rylgamelibrary:gzio.obj
 0001:000260d0       _putShortMSB               004270d0 f   rylgamelibrary:deflate.obj
 0001:00026100       _flush_pending             00427100 f   rylgamelibrary:deflate.obj
 0001:000264c0       _lm_init                   004274c0 f   rylgamelibrary:deflate.obj
 0001:00026550       _longest_match             00427550 f   rylgamelibrary:deflate.obj
 0001:000266c0       _fill_window               004276c0 f   rylgamelibrary:deflate.obj
 0001:00026850       _deflate_stored            00427850 f   rylgamelibrary:deflate.obj
 0001:00026a60       _deflate_fast              00427a60 f   rylgamelibrary:deflate.obj
 0001:00026dd0       _deflate_slow              00427dd0 f   rylgamelibrary:deflate.obj
 0001:00027b3b       $L124449                   00428b3b f i rylgamelibrary:cellmanager.obj
 0001:00027cf0       _init_block                00428cf0 f   rylgamelibrary:trees.obj
 0001:00027d60       _pqdownheap                00428d60 f   rylgamelibrary:trees.obj
 0001:00027e30       _gen_bitlen                00428e30 f   rylgamelibrary:trees.obj
 0001:00028070       _scan_tree                 00429070 f   rylgamelibrary:trees.obj
 0001:00028150       _send_tree                 00429150 f   rylgamelibrary:trees.obj
 0001:00028660       _send_all_trees            00429660 f   rylgamelibrary:trees.obj
 0001:000288d0       _compress_block            004298d0 f   rylgamelibrary:trees.obj
 0001:00028cf0       _set_data_type             00429cf0 f   rylgamelibrary:trees.obj
 0001:00028d80       _bi_flush                  00429d80 f   rylgamelibrary:trees.obj
 0001:00028e00       _bi_windup                 00429e00 f   rylgamelibrary:trees.obj
 0001:00028e70       _copy_block                00429e70 f   rylgamelibrary:trees.obj
 0001:00028f70       _gen_codes                 00429f70 f   rylgamelibrary:trees.obj
 0001:00029000       _build_tree                0042a000 f   rylgamelibrary:trees.obj
 0001:00029200       _build_bl_tree             0042a200 f   rylgamelibrary:trees.obj
 0001:0002a080       _$E4                       0042b080 f   rylgamelibrary:CSAuth.obj
 0001:0002a090       _$E1                       0042b090 f   rylgamelibrary:CSAuth.obj
 0001:0002a0a0       _$E3                       0042b0a0 f   rylgamelibrary:CSAuth.obj
 0001:0002a0b0       _$E2                       0042b0b0 f   rylgamelibrary:CSAuth.obj
 0001:0002b53e       $L74548                    0042c53e f i rylgamelibrary:reloctable.obj
 0001:0002b54a       $L74550                    0042c54a f i rylgamelibrary:reloctable.obj
 0001:00036cd5       _tidy_global               00437cd5 f   libcpmt:locale0.obj
 0001:000373cb       ?CatchGuardHandler@@YA?AW4_EXCEPTION_DISPOSITION@@PAUEHExceptionRecord@@PAUCatchGuardRN@@PAX2@Z 004383cb f   LIBCMT:trnsctrl.obj
 0001:000374cd       ?TranslatorGuardHandler@@YA?AW4_EXCEPTION_DISPOSITION@@PAUEHExceptionRecord@@PAUTranslatorGuardRN@@PAX2@Z 004384cd f   LIBCMT:trnsctrl.obj
 0001:000376e8       $$$00001                   004386e8 f   LIBCMT:exsup.obj
 0001:00037708       __unwind_handler           00438708 f   LIBCMT:exsup.obj
 0001:00037708       $$$00003                   00438708 f   LIBCMT:exsup.obj
 0001:0003772a       $$$00005                   0043872a f   LIBCMT:exsup.obj
 0001:00037792       $$$00007                   00438792 f   LIBCMT:exsup.obj
 0001:000377d6       $$$00011                   004387d6 f   LIBCMT:exsup.obj
 0001:000377d6       _report_failure            004387d6 f   LIBCMT:secchk.obj
 0001:00037949       __onexit_lk                00438949 f   LIBCMT:onexit.obj
 0001:00037e30       _$$$00001                  00438e30 f   LIBCMT:strchr.obj
 0001:0003845f       $L528                      0043945f f   LIBCMT:newopnt.obj
 0001:0003848e       _fast_error_exit           0043948e f   LIBCMT:wincrt0.obj
 0001:00038941       $$$00003                   00439941 f   LIBCMT:exsup3.obj
 0001:000390a3       __threadstartex@4          0043a0a3 f   LIBCMT:threadex.obj
 0001:000396f0       _xtoa                      0043a6f0 f   LIBCMT:xtoa.obj
 0001:00039758       _x64toa@20                 0043a758 f   LIBCMT:xtoa.obj
 0001:00039992       _flsall                    0043a992 f   LIBCMT:fflush.obj
 0001:0003a7d7       __initterm                 0043b7d7 f   LIBCMT:crt0dat.obj
 0001:0003a859       _doexit                    0043b859 f   LIBCMT:crt0dat.obj
 0001:0003ab78       _strtoxl                   0043bb78 f   LIBCMT:strtol.obj
 0001:0003b27f       ?TypeMatch@@YAHPBU_s_HandlerType@@PBU_s_CatchableType@@PBU_s_ThrowInfo@@@Z 0043c27f f   LIBCMT:frame.obj
 0001:0003b2ce       ?FrameUnwindFilter@@YAHPAU_EXCEPTION_POINTERS@@@Z 0043c2ce f   LIBCMT:frame.obj
 0001:0003b3ff       ?AdjustPointer@@YAPAXPAXABUPMD@@@Z 0043c3ff f   LIBCMT:frame.obj
 0001:0003b431       ?CallCatchBlock@@YAPAXPAUEHExceptionRecord@@PAUEHRegistrationNode@@PAU_CONTEXT@@PBU_s_FuncInfo@@PAXHK@Z 0043c431 f   LIBCMT:frame.obj
 0001:0003b5f5       ?BuildCatchObject@@YAXPAUEHExceptionRecord@@PAXPBU_s_HandlerType@@PBU_s_CatchableType@@@Z 0043c5f5 f   LIBCMT:frame.obj
 0001:0003b771       ?CatchIt@@YAXPAUEHExceptionRecord@@PAUEHRegistrationNode@@PAU_CONTEXT@@PAXPBU_s_FuncInfo@@PBU_s_HandlerType@@PBU_s_CatchableType@@PBU_s_TryBlockMapEntry@@H1E@Z 0043c771 f   LIBCMT:frame.obj
 0001:0003b7d8       ?FindHandlerForForeignException@@YAXPAUEHExceptionRecord@@PAUEHRegistrationNode@@PAU_CONTEXT@@PAXPBU_s_FuncInfo@@HH1@Z 0043c7d8 f   LIBCMT:frame.obj
 0001:0003b896       ?FindHandler@@YAXPAUEHExceptionRecord@@PAUEHRegistrationNode@@PAU_CONTEXT@@PAXPBU_s_FuncInfo@@EH1@Z 0043c896 f   LIBCMT:frame.obj
 0001:0003c37a       ___updatetlocinfo_lk       0043d37a f   LIBCMT:setlocal.obj
 0001:0003c5c7       __setlocale_get_all        0043d5c7 f   LIBCMT:setlocal.obj
 0001:0003c7e2       __setlocale_set_cat        0043d7e2 f   LIBCMT:setlocal.obj
 0001:0003ca71       __setlocale_lk             0043da71 f   LIBCMT:setlocal.obj
 0001:0003d629       _write_char                0043e629 f   LIBCMT:output.obj
 0001:0003d65c       _write_multi_char          0043e65c f   LIBCMT:output.obj
 0001:0003d680       _write_string              0043e680 f   LIBCMT:output.obj
 0001:0003e8f0       _parse_cmdline             0043f8f0 f   LIBCMT:stdargv.obj
 0001:0003f465       _CPtoLCID                  00440465 f   LIBCMT:mbctype.obj
 0001:0003f494       _setSBCS                   00440494 f   LIBCMT:mbctype.obj
 0001:0003f4bd       _setSBUpLow                004404bd f   LIBCMT:mbctype.obj
 0001:0003f6b8       __setmbcp_lk               004406b8 f   LIBCMT:mbctype.obj
 0001:0003fa95       __shift                    00440a95 f   LIBCMT:cvt.obj
 0001:0003fab2       __cftoe2                   00440ab2 f   LIBCMT:cvt.obj
 0001:0003fbcc       __cftof2                   00440bcc f   LIBCMT:cvt.obj
 0001:000409ee       __tzset_lk                 004419ee f   LIBCMT:tzset.obj
 0001:00040c96       _cvtdate                   00441c96 f   LIBCMT:tzset.obj
 0001:00040e4e       __isindst_lk               00441e4e f   LIBCMT:tzset.obj
 0001:0004201f       ___crtInitCritSecNoSpinCount@8 0044301f f   LIBCMT:initcrit.obj
 0001:000420ba       __get_lc_time              004430ba f   LIBCMT:inittime.obj
 0001:00042b54       _TranslateName             00443b54 f   LIBCMT:getqloc.obj
 0001:00042bb4       _GetLcidFromDefault        00443bb4 f   LIBCMT:getqloc.obj
 0001:00042bce       _ProcessCodePage           00443bce f   LIBCMT:getqloc.obj
 0001:00042c44       _TestDefaultCountry        00443c44 f   LIBCMT:getqloc.obj
 0001:00042c62       _crtGetLocaleInfoA@16      00443c62 f   LIBCMT:getqloc.obj
 0001:00042d45       _LcidFromHexString         00443d45 f   LIBCMT:getqloc.obj
 0001:00042d7a       _GetPrimaryLen             00443d7a f   LIBCMT:getqloc.obj
 0001:00042d97       _CountryEnumProc@4         00443d97 f   LIBCMT:getqloc.obj
 0001:00042e2b       _TestDefaultLanguage       00443e2b f   LIBCMT:getqloc.obj
 0001:00042e9c       _LangCountryEnumProc@4     00443e9c f   LIBCMT:getqloc.obj
 0001:000430b6       _LanguageEnumProc@4        004440b6 f   LIBCMT:getqloc.obj
 0001:00043181       _GetLcidFromCountry        00444181 f   LIBCMT:getqloc.obj
 0001:000431b8       _GetLcidFromLangCountry    004441b8 f   LIBCMT:getqloc.obj
 0001:0004323e       _GetLcidFromLanguage       0044423e f   LIBCMT:getqloc.obj
 0001:00043490       _siglookup                 00444490 f   LIBCMT:winsig.obj
 0001:00043b5b       __tsopen_lk                00444b5b f   LIBCMT:open.obj
 0001:00043e97       _x_ismbbtype               00444e97 f   LIBCMT:ismbbyte.obj
 0001:0004464a       __abstract_cw              0044564a f   LIBCMT:ieee87.obj
 0001:000446dc       __hw_cw                    004456dc f   LIBCMT:ieee87.obj
 0001:00045a0d       _strncnt                   00446a0d f   LIBCMT:a_cmp.obj
 0001:00045dad       _findenv                   00446dad f   LIBCMT:setenv.obj
 0001:00045dfa       _copy_environ              00446dfa f   LIBCMT:setenv.obj
 0001:000461e0       $L40419                    004471e0 f   authagentdispatch.obj
 0001:000461e8       __ehhandler$??1CAuthAgentDispatch@@UAE@XZ 004471e8 f   authagentdispatch.obj
 0001:00046200       $L40444                    00447200 f   authagentdispatch.obj
 0001:00046208       __ehhandler$?ParseAgentZone@CAuthAgentDispatch@@AAE_NPAUPktDD@@@Z 00447208 f   authagentdispatch.obj
 0001:00046220       $L40643                    00447220 f   authagentdispatch.obj
 0001:0004622e       __ehhandler$?GetDispatchTable@CAuthAgentDispatch@@SAAAVCSingleDispatch@@XZ 0044722e f   authagentdispatch.obj
 0001:00046240       $L40575                    00447240 f   authagentdispatch.obj
 0001:00046240       $L40679                    00447240 f   authagentdispatch.obj
 0001:00046240       $L40593                    00447240 f   authagentdispatch.obj
 0001:00046240       $L40698                    00447240 f   authagentdispatch.obj
 0001:00046248       __ehhandler$?ParseUserKill@CAuthAgentDispatch@@AAE_NPAUPktUK@@@Z 00447248 f   authagentdispatch.obj
 0001:00046248       __ehhandler$?ParseBillingTimeoutNotify@CAuthAgentDispatch@@AAE_NPAUPktBTN@@@Z 00447248 f   authagentdispatch.obj
 0001:00046248       __ehhandler$?ParseBillingTimeCheckNotify@CAuthAgentDispatch@@AAE_NPAUPktBTN@@@Z 00447248 f   authagentdispatch.obj
 0001:00046248       __ehhandler$?SendStartSession@CAuthAgentDispatch@@SA_NPAVCAuthClientDispatch@@KPADKG@Z 00447248 f   authagentdispatch.obj
 0001:00046260       $L40807                    00447260 f   authagentdispatch.obj
 0001:00046268       __ehhandler$?ParseDBGetData@CAuthAgentDispatch@@AAE_NPAUPktDD@@@Z 00447268 f   authagentdispatch.obj
 0001:00046280       $L38088                    00447280 f   authclientdispath.obj
 0001:00046288       $L38089                    00447288 f   authclientdispath.obj
 0001:00046293       __ehhandler$??1CAuthClientDispatch@@UAE@XZ 00447293 f   authclientdispath.obj
 0001:000462a0       $L38316                    004472a0 f   authclientdispath.obj
 0001:000462ab       __ehhandler$?ParseJapanAuthAccount@CAuthClientDispatch@@AAE_NPAUPktJPAU@@@Z 004472ab f   authclientdispath.obj
 0001:000462c0       $L38379                    004472c0 f   authclientdispath.obj
 0001:000462c8       __ehhandler$??0CAuthClientDispatch@@QAE@AAVCSession@@@Z 004472c8 f   authclientdispath.obj
 0001:000462e0       $L38398                    004472e0 f   authclientdispath.obj
 0001:000462ee       __ehhandler$?GetDispatchTable@CAuthClientDispatch@@SAAAVCMultiDispatch@@XZ 004472ee f   authclientdispath.obj
 0001:00046300       $L38449                    00447300 f   authclientdispath.obj
 0001:0004630b       __ehhandler$?ParseAuthAccount@CAuthClientDispatch@@AAE_NPAUPktAU@@@Z 0044730b f   authclientdispath.obj
 0001:00046320       $L38483                    00447320 f   authclientdispath.obj
 0001:0004632b       __ehhandler$?ParseCharCreate@CAuthClientDispatch@@AAE_NPAUPktCC@@@Z 0044732b f   authclientdispath.obj
 0001:00046340       $L38154                    00447340 f   authclientdispath.obj
 0001:00046340       $L38412                    00447340 f   authclientdispath.obj
 0001:00046340       $L38428                    00447340 f   authclientdispath.obj
 0001:00046340       $L38212                    00447340 f   authclientdispath.obj
 0001:00046340       $L38532                    00447340 f   authclientdispath.obj
 0001:00046340       $L38253                    00447340 f   authclientdispath.obj
 0001:00046348       __ehhandler$?ParseUserLogin@CAuthClientDispatch@@AAE_NPAUPktULi@@@Z 00447348 f   authclientdispath.obj
 0001:00046348       __ehhandler$?ParseServerZone@CAuthClientDispatch@@AAE_NPAUPktSZ@@@Z 00447348 f   authclientdispath.obj
 0001:00046348       __ehhandler$?UserMove@CAuthClientDispatch@@QAEXXZ 00447348 f   authclientdispath.obj
 0001:00046348       __ehhandler$?UserLogout@CAuthClientDispatch@@QAEXXZ 00447348 f   authclientdispath.obj
 0001:00046348       __ehhandler$?ParseCharSelect@CAuthClientDispatch@@AAE_NPAUPktCS@@@Z 00447348 f   authclientdispath.obj
 0001:00046348       __ehhandler$?ParseCharDelete@CAuthClientDispatch@@AAE_NPAUPktCD@@@Z 00447348 f   authclientdispath.obj
 0001:00046360       $L67165                    00447360 f   authorizethread.obj
 0001:0004636b       $L67166                    0044736b f   authorizethread.obj
 0001:00046376       __ehhandler$?Initialize@CAuthorizeThread@@QAE_NXZ 00447376 f   authorizethread.obj
 0001:00046380       $L67323                    00447380 f   authorizethread.obj
 0001:00046388       __ehhandler$??1CAuthorizeThread@@UAE@XZ 00447388 f   authorizethread.obj
 0001:000463a0       $L67446                    004473a0 f   authorizethread.obj
 0001:000463ae       __ehhandler$?GetInstance@?$CStaticSingleton@VCMasterPassword@@@@SAAAVCMasterPassword@@XZ 004473ae f   authorizethread.obj
 0001:000463c0       __ehhandler$?_Copy@?$basic_string@DU?$char_traits@D@std@@V?$allocator@D@2@@std@@IAEXII@Z 004473c0 f   authorizeuser.obj
 0001:000463d0       $L35988                    004473d0 f   authorizeuser.obj
 0001:000463d8       $L35989                    004473d8 f   authorizeuser.obj
 0001:000463e3       __ehhandler$??1CSyncronizedObjectQueue@@QAE@XZ 004473e3 f   authorizeuser.obj
 0001:000463f0       $L36286                    004473f0 f   authorizeuser.obj
 0001:000463f8       $L36287                    004473f8 f   authorizeuser.obj
 0001:00046403       __ehhandler$??1CAuthorizeUser@@AAE@XZ 00447403 f   authorizeuser.obj
 0001:00046410       $L36823                    00447410 f   authorizeuser.obj
 0001:00046418       __ehhandler$??0CSyncronizedObjectQueue@@QAE@XZ 00447418 f   authorizeuser.obj
 0001:00046430       $L37225                    00447430 f   authorizeuser.obj
 0001:0004643e       $L37227                    0044743e f   authorizeuser.obj
 0001:00046448       __ehhandler$?GetInstance@CAuthorizeUser@@SAAAV1@XZ 00447448 f   authorizeuser.obj
 0001:00046460       $L37318                    00447460 f   authorizeuser.obj
 0001:00046468       __ehhandler$?_Incsize@?$list@PAVCAuthInfo@@V?$allocator@PAVCAuthInfo@@@std@@@std@@IAEXI@Z 00447468 f   authorizeuser.obj
 0001:00046480       $L37455                    00447480 f   authorizeuser.obj
 0001:00046480       $L37006                    00447480 f   authorizeuser.obj
 0001:00046488       __ehhandler$??0logic_error@std@@QAE@ABV01@@Z 00447488 f   authorizeuser.obj
 0001:00046488       __ehhandler$??0logic_error@std@@QAE@ABV?$basic_string@DU?$char_traits@D@std@@V?$allocator@D@2@@1@@Z 00447488 f   authorizeuser.obj
 0001:000464a0       $L35233                    004474a0 f   authorizeuser.obj
 0001:000464a0       $L35017                    004474a0 f   authorizeuser.obj
 0001:000464a0       $L37696                    004474a0 f   authorizeuser.obj
 0001:000464a8       __ehhandler$?remove@CSyncronizedObjectQueue@@QAEXPBD@Z 004474a8 f   authorizeuser.obj
 0001:000464a8       __ehhandler$?clear@CSyncronizedObjectQueue@@QAEXXZ 004474a8 f   authorizeuser.obj
 0001:000464a8       __ehhandler$?enqueue@CSyncronizedObjectQueue@@QAE_NPAVCAuthInfo@@_N@Z 004474a8 f   authorizeuser.obj
 0001:000464c0       $L29382                    004474c0 f   itemcreator.obj
 0001:000464c0       $L29451                    004474c0 f   itemcreator.obj
 0001:000464c8       __ehhandler$?Create@CItemCreator@@QAEPAVCItem@Item@@G@Z 004474c8 f   itemcreator.obj
 0001:000464c8       __ehhandler$?Initialize@CItemCreator@@QAE_NXZ 004474c8 f   itemcreator.obj
 0001:000464e0       $L27412                    004474e0 f   masterpassword.obj
 0001:000464e8       __ehhandler$?CheckMasterPassword@CMasterPassword@@QAE_NPBD0ABUsockaddr_in@@@Z 004474e8 f   masterpassword.obj
 0001:00046500       $L28701                    00447500 f   masterpassword.obj
 0001:00046508       __ehhandler$?_Xlen@?$vector@KV?$allocator@K@std@@@std@@IBEXXZ 00447508 f   masterpassword.obj
 0001:00046520       $L29254                    00447520 f   masterpassword.obj
 0001:00046528       __ehhandler$??0CMasterPassword@@QAE@XZ 00447528 f   masterpassword.obj
 0001:00046540       $L29552                    00447540 f   masterpassword.obj
 0001:0004654b       __ehhandler$?LoadMasterPassword@CMasterPassword@@QAE_NPBD@Z 0044754b f   masterpassword.obj
 0001:00046560       $L41130                    00447560 f   rylauthserver.obj
 0001:00046568       __ehhandler$??1CRylAuthServerProcess@@UAE@XZ 00447568 f   rylauthserver.obj
 0001:00046580       $L41151                    00447580 f   rylauthserver.obj
 0001:00046588       $L41152                    00447588 f   rylauthserver.obj
 0001:00046593       __ehhandler$??0CRylAuthServer@@AAE@XZ 00447593 f   rylauthserver.obj
 0001:000465a0       $L41162                    004475a0 f   rylauthserver.obj
 0001:000465a8       __ehhandler$??1CRylAuthServer@@EAE@XZ 004475a8 f   rylauthserver.obj
 0001:000465c0       $L41458                    004475c0 f   rylauthserver.obj
 0001:000465ce       __ehhandler$?GetInstance@CRylAuthServer@@SAAAV1@XZ 004475ce f   rylauthserver.obj
 0001:000465e0       $L42727                    004475e0 f   rylauthserver.obj
 0001:000465e0       $L43107                    004475e0 f   rylauthserver.obj
 0001:000465f1       __ehhandler$?CreateDispatch@?$CPoolDispatchFactory@VCAuthClientDispatch@@@@UAEPAVCPacketDispatch@@AAVCSession@@@Z 004475f1 f   rylauthserver.obj
 0001:000465f1       __ehhandler$?CreateDispatch@?$CPoolDispatchFactory@VCAuthAgentDispatch@@@@UAEPAVCPacketDispatch@@AAVCSession@@@Z 004475f1 f   rylauthserver.obj
 0001:00046600       $L43482                    00447600 f   rylauthserver.obj
 0001:00046608       __ehhandler$?_Incsize@?$list@PAVCCommand@@V?$allocator@PAVCCommand@@@std@@@std@@IAEXI@Z 00447608 f   rylauthserver.obj
 0001:00046620       $L43752                    00447620 f   rylauthserver.obj
 0001:00046620       $L43831                    00447620 f   rylauthserver.obj
 0001:00046632       $L43753                    00447632 f   rylauthserver.obj
 0001:00046632       $L43832                    00447632 f   rylauthserver.obj
 0001:0004663d       $L43834                    0044763d f   rylauthserver.obj
 0001:0004663d       $L43755                    0044763d f   rylauthserver.obj
 0001:00046648       $L43835                    00447648 f   rylauthserver.obj
 0001:00046648       $L43756                    00447648 f   rylauthserver.obj
 0001:00046653       __ehhandler$??$Create@VCTCPFactory@@VCPoolBufferFactory@@V?$CPoolDispatchFactory@VCAuthClientDispatch@@@@VCStreamOverlappedFactory@@@CSessionPolicy@@SAPAV0@XZ 00447653 f   rylauthserver.obj
 0001:00046653       __ehhandler$??$Create@VCTCPFactory@@VCPoolBufferFactory@@V?$CPoolDispatchFactory@VCAuthAgentDispatch@@@@VCStreamOverlappedFactory@@@CSessionPolicy@@SAPAV0@XZ 00447653 f   rylauthserver.obj
 0001:00046660       $L43923                    00447660 f   rylauthserver.obj
 0001:00046668       __ehhandler$?ConnectToDBAgent@CRylAuthServer@@QAEXXZ 00447668 f   rylauthserver.obj
 0001:00046680       $L44006                    00447680 f   rylauthserver.obj
 0001:00046688       __ehhandler$?Add@CCommandProcess@@QAEXPAVCCommand@@@Z 00447688 f   rylauthserver.obj
 0001:000466a0       $L44112                    004476a0 f   rylauthserver.obj
 0001:000466ab       __ehhandler$?ApplicationSpecificInit@CRylAuthServer@@EAE_NPBD@Z 004476ab f   rylauthserver.obj
 0001:000466c0       $L34867                    004476c0 f   senduserloginout.obj
 0001:000466c0       $L34842                    004476c0 f   senduserloginout.obj
 0001:000466c8       __ehhandler$?SendUserLogout@AuthSendPacket@@YA_NKK@Z 004476c8 f   senduserloginout.obj
 0001:000466c8       __ehhandler$?SendUserMove@AuthSendPacket@@YA_NKK@Z 004476c8 f   senduserloginout.obj
 0001:000466e0       $L30946                    004476e0 f   rylgamelibrary:rylserverdispatch.obj
 0001:000466e8       $L30947                    004476e8 f   rylgamelibrary:rylserverdispatch.obj
 0001:000466f3       $L30948                    004476f3 f   rylgamelibrary:rylserverdispatch.obj
 0001:000466fe       __ehhandler$??0CRylServerDispatch@@IAE@AAVCSession@@K@Z 004476fe f   rylgamelibrary:rylserverdispatch.obj
 0001:00046710       $L31214                    00447710 f   rylgamelibrary:rylserverdispatch.obj
 0001:00046718       $L31215                    00447718 f   rylgamelibrary:rylserverdispatch.obj
 0001:00046723       $L31216                    00447723 f   rylgamelibrary:rylserverdispatch.obj
 0001:0004672e       $L31217                    0044772e f   rylgamelibrary:rylserverdispatch.obj
 0001:00046739       $L31218                    00447739 f   rylgamelibrary:rylserverdispatch.obj
 0001:00046741       __ehhandler$??1CRylServerDispatch@@MAE@XZ 00447741 f   rylgamelibrary:rylserverdispatch.obj
 0001:00046750       $L31306                    00447750 f   rylgamelibrary:rylserverdispatch.obj
 0001:00046758       $L31307                    00447758 f   rylgamelibrary:rylserverdispatch.obj
 0001:00046760       __ehhandler$?ParsePacket@CRylServerDispatch@@UAE_NQADPAK@Z 00447760 f   rylgamelibrary:rylserverdispatch.obj
 0001:00046770       $L31345                    00447770 f   rylgamelibrary:rylserverdispatch.obj
 0001:00046778       $L31346                    00447778 f   rylgamelibrary:rylserverdispatch.obj
 0001:00046780       $L31347                    00447780 f   rylgamelibrary:rylserverdispatch.obj
 0001:00046788       $L31348                    00447788 f   rylgamelibrary:rylserverdispatch.obj
 0001:00046790       $L31349                    00447790 f   rylgamelibrary:rylserverdispatch.obj
 0001:00046798       __ehhandler$?Dispatch@CRylServerDispatch@@MAE_NXZ 00447798 f   rylgamelibrary:rylserverdispatch.obj
 0001:000467b0       $L35851                    004477b0 f   rylgamelibrary:rylserverdispatch.obj
 0001:000467b8       __ehhandler$?_Xlen@?$vector@U?$pair@KK@std@@V?$allocator@U?$pair@KK@std@@@2@@std@@IBEXXZ 004477b8 f   rylgamelibrary:rylserverdispatch.obj
 0001:000467d0       __ehhandler$?_Insert_n@?$vector@U?$pair@KK@std@@V?$allocator@U?$pair@KK@std@@@2@@std@@IAEXViterator@12@IABU?$pair@KK@2@@Z 004477d0 f   rylgamelibrary:rylserverdispatch.obj
 0001:000467e0       __ehhandler$?reserve@?$vector@U?$pair@KK@std@@V?$allocator@U?$pair@KK@std@@@2@@std@@QAEXI@Z 004477e0 f   rylgamelibrary:rylserverdispatch.obj
 0001:000467f0       $L36761                    004477f0 f   rylgamelibrary:rylserverdispatch.obj
 0001:000467fb       __ehhandler$?ProcessTooManyPacket@CRylServerDispatch@@MAEXAAVCBufferQueue@@@Z 004477fb f   rylgamelibrary:rylserverdispatch.obj
 0001:00046810       $L21955                    00447810 f   rylgamelibrary:serverlog.obj
 0001:0004681b       __ehhandler$??0CServerLog@@QAE@PBD0@Z 0044781b f   rylgamelibrary:serverlog.obj
 0001:00046830       $L31018                    00447830 f   rylgamelibrary:serverrequest.obj
 0001:00046838       __ehhandler$?RemoveAllRequest@CServerRequest@@QAEXXZ 00447838 f   rylgamelibrary:serverrequest.obj
 0001:00046850       $L32966                    00447850 f   rylgamelibrary:serverrequest.obj
 0001:00046850       $L32338                    00447850 f   rylgamelibrary:serverrequest.obj
 0001:00046858       __ehhandler$?_Insert@?$_Tree@V?$_Tmap_traits@KURequestInfo@CServerRequest@@U?$less@K@std@@V?$allocator@U?$pair@$$CBKURequestInfo@CServerRequest@@@std@@@4@$0A@@std@@@std@@IAE?AViterator@12@_NPAU_Node@?$_Tree_nod@V?$_Tmap_traits@KURequestInfo@CServerRequest@@U?$less@K@std@@V?$allocator@U?$pair@$$CBKURequestInfo@CServerRequest@@@std@@@4@$0A@@std@@@2@ABU?$pair@$$CBKURequestInfo@CServerRequest@@@2@@Z 00447858 f   rylgamelibrary:serverrequest.obj
 0001:00046858       __ehhandler$?erase@?$_Tree@V?$_Tmap_traits@KURequestInfo@CServerRequest@@U?$less@K@std@@V?$allocator@U?$pair@$$CBKURequestInfo@CServerRequest@@@std@@@4@$0A@@std@@@std@@QAE?AViterator@12@V312@@Z 00447858 f   rylgamelibrary:serverrequest.obj
 0001:00046870       $L33811                    00447870 f   rylgamelibrary:serverrequest.obj
 0001:00046878       __ehhandler$?AddRequest@CServerRequest@@QAEKPAVCPacketDispatch@@0KP6AX0@Z@Z 00447878 f   rylgamelibrary:serverrequest.obj
 0001:00046890       $L34175                    00447890 f   rylgamelibrary:serverrequest.obj
 0001:00046898       __ehhandler$?RemoveTimeoutRequest@CServerRequest@@QAEXXZ 00447898 f   rylgamelibrary:serverrequest.obj
 0001:000468b0       $L34350                    004478b0 f   rylgamelibrary:serverrequest.obj
 0001:000468b8       __ehhandler$?PopRequest@CServerRequest@@AAEPAVCPacketDispatch@@K@Z 004478b8 f   rylgamelibrary:serverrequest.obj
 0001:000468d0       $L34762                    004478d0 f   rylgamelibrary:serverrequest.obj
 0001:000468d8       $L34763                    004478d8 f   rylgamelibrary:serverrequest.obj
 0001:000468e3       __ehhandler$??1CServerRequest@@AAE@XZ 004478e3 f   rylgamelibrary:serverrequest.obj
 0001:000468f0       $L35131                    004478f0 f   rylgamelibrary:serverrequest.obj
 0001:000468f8       __ehhandler$??0CServerRequest@@AAE@XZ 004478f8 f   rylgamelibrary:serverrequest.obj
 0001:00046910       $L35356                    00447910 f   rylgamelibrary:serverrequest.obj
 0001:0004691e       __ehhandler$?GetInstance@CServerRequest@@SAAAV1@XZ 0044791e f   rylgamelibrary:serverrequest.obj
 0001:00046930       $L28032                    00447930 f   rylgamelibrary:sendstream.obj
 0001:00046938       __ehhandler$?Send@CSession@@QAE_NXZ 00447938 f   rylgamelibrary:sendstream.obj
 0001:00046950       $L38747                    00447950 f   rylgamelibrary:serversetup.obj
 0001:00046968       __ehhandler$??0CServerSetup@@QAE@XZ 00447968 f   rylgamelibrary:serversetup.obj
 0001:00046980       $L39041                    00447980 f   rylgamelibrary:serversetup.obj
 0001:0004698e       __ehhandler$?GetInstance@CServerSetup@@SAAAV1@XZ 0044798e f   rylgamelibrary:serversetup.obj
 0001:000469a0       $L39320                    004479a0 f   rylgamelibrary:serversetup.obj
 0001:000469ab       __ehhandler$?InitGameServer@CServerSetup@@QAE_NXZ 004479ab f   rylgamelibrary:serversetup.obj
 0001:000469c0       $L33843                    004479c0 f   rylgamelibrary:multidispatchstorage.obj
 0001:000469c0       $L30389                    004479c0 f   rylgamelibrary:multidispatchstorage.obj
 0001:000469c8       __ehhandler$?RemoveDispatch@CMultiDispatch@@QAEXK@Z 004479c8 f   rylgamelibrary:multidispatchstorage.obj
 0001:000469c8       __ehhandler$?GetDispatch@CMultiDispatch@@AAEPAVCPacketDispatch@@K@Z 004479c8 f   rylgamelibrary:multidispatchstorage.obj
 0001:000469e0       $L31503                    004479e0 f   rylgamelibrary:multidispatchstorage.obj
 0001:000469e0       $L31994                    004479e0 f   rylgamelibrary:multidispatchstorage.obj
 0001:000469e8       __ehhandler$?_Insert@?$_Tree@V?$_Tmap_traits@KPAVCPacketDispatch@@U?$less@K@std@@V?$allocator@U?$pair@$$CBKPAVCPacketDispatch@@@std@@@3@$0A@@std@@@std@@IAE?AViterator@12@_NPAU_Node@?$_Tree_nod@V?$_Tmap_traits@KPAVCPacketDispatch@@U?$less@K@std@@V?$allocator@U?$pair@$$CBKPAVCPacketDispatch@@@std@@@3@$0A@@std@@@2@ABU?$pair@$$CBKPAVCPacketDispatch@@@2@@Z 004479e8 f   rylgamelibrary:multidispatchstorage.obj
 0001:000469e8       __ehhandler$?erase@?$_Tree@V?$_Tmap_traits@KPAVCPacketDispatch@@U?$less@K@std@@V?$allocator@U?$pair@$$CBKPAVCPacketDispatch@@@std@@@3@$0A@@std@@@std@@QAE?AViterator@12@V312@@Z 004479e8 f   rylgamelibrary:multidispatchstorage.obj
 0001:00046a00       $L33643                    00447a00 f   rylgamelibrary:multidispatchstorage.obj
 0001:00046a08       __ehhandler$?SetDispatch@CMultiDispatch@@QAE_NKPAVCPacketDispatch@@@Z 00447a08 f   rylgamelibrary:multidispatchstorage.obj
 0001:00046a20       $L34094                    00447a20 f   rylgamelibrary:multidispatchstorage.obj
 0001:00046a28       $L34095                    00447a28 f   rylgamelibrary:multidispatchstorage.obj
 0001:00046a33       $L34096                    00447a33 f   rylgamelibrary:multidispatchstorage.obj
 0001:00046a3b       __ehhandler$??1CMultiDispatch@@QAE@XZ 00447a3b f   rylgamelibrary:multidispatchstorage.obj
 0001:00046a50       $L34644                    00447a50 f   rylgamelibrary:multidispatchstorage.obj
 0001:00046a58       __ehhandler$??0CMultiDispatch@@QAE@XZ 00447a58 f   rylgamelibrary:multidispatchstorage.obj
 0001:00046a70       $L26808                    00447a70 f   rylgamelibrary:singledispatchstorage.obj
 0001:00046a78       __ehhandler$?SetDispatch@CSingleDispatch@@QAEXPAVCPacketDispatch@@@Z 00447a78 f   rylgamelibrary:singledispatchstorage.obj
 0001:00046a90       $L26852                    00447a90 f   rylgamelibrary:singledispatchstorage.obj
 0001:00046a90       $L26936                    00447a90 f   rylgamelibrary:singledispatchstorage.obj
 0001:00046a98       __ehhandler$?GetDispatch@CSingleDispatch@@AAEPAVCPacketDispatch@@XZ 00447a98 f   rylgamelibrary:singledispatchstorage.obj
 0001:00046a98       __ehhandler$?RemoveDispatch@CSingleDispatch@@QAEXPAVCPacketDispatch@@@Z 00447a98 f   rylgamelibrary:singledispatchstorage.obj
 0001:00046ab0       $L26903                    00447ab0 f   rylgamelibrary:singledispatchstorage.obj
 0001:00046ab8       $L26904                    00447ab8 f   rylgamelibrary:singledispatchstorage.obj
 0001:00046ac0       __ehhandler$??1CSingleDispatch@@QAE@XZ 00447ac0 f   rylgamelibrary:singledispatchstorage.obj
 0001:00046ad0       $L34103                    00447ad0 f   rylgamelibrary:session.obj
 0001:00046ad8       $L34104                    00447ad8 f   rylgamelibrary:session.obj
 0001:00046ae3       __ehhandler$??0CSession@@QAE@AAVCSessionPolicy@@@Z 00447ae3 f   rylgamelibrary:session.obj
 0001:00046af0       $L34806                    00447af0 f   rylgamelibrary:session.obj
 0001:00046af0       $L34856                    00447af0 f   rylgamelibrary:session.obj
 0001:00046af0       $L34312                    00447af0 f   rylgamelibrary:session.obj
 0001:00046af0       $L34560                    00447af0 f   rylgamelibrary:session.obj
 0001:00046af8       __ehhandler$?CloseSession@CSession@@QAEXXZ 00447af8 f   rylgamelibrary:session.obj
 0001:00046af8       __ehhandler$?SendCompleted@CSession@@QAEXHK@Z 00447af8 f   rylgamelibrary:session.obj
 0001:00046af8       __ehhandler$?SendPending@CSession@@QAE_NPAVCBuffer@@@Z 00447af8 f   rylgamelibrary:session.obj
 0001:00046af8       __ehhandler$?Dispatch@CSession@@QAE_NK@Z 00447af8 f   rylgamelibrary:session.obj
 0001:00046b10       $L34652                    00447b10 f   rylgamelibrary:session.obj
 0001:00046b18       $L34653                    00447b18 f   rylgamelibrary:session.obj
 0001:00046b23       $L34654                    00447b23 f   rylgamelibrary:session.obj
 0001:00046b2b       __ehhandler$??1CSession@@QAE@XZ 00447b2b f   rylgamelibrary:session.obj
 0001:00046b40       $L34700                    00447b40 f   rylgamelibrary:session.obj
 0001:00046b48       $L34701                    00447b48 f   rylgamelibrary:session.obj
 0001:00046b50       __ehhandler$?Process@CSession@@QAE_NXZ 00447b50 f   rylgamelibrary:session.obj
 0001:00046b60       $L34953                    00447b60 f   rylgamelibrary:session.obj
 0001:00046b60       $L35017                    00447b60 f   rylgamelibrary:session.obj
 0001:00046b68       __ehhandler$??0sentry@?$basic_ostream@DU?$char_traits@D@std@@@std@@QAE@AAV12@@Z 00447b68 f   rylgamelibrary:session.obj
 0001:00046b68       __ehhandler$??1sentry@?$basic_ostream@DU?$char_traits@D@std@@@std@@QAE@XZ 00447b68 f   rylgamelibrary:session.obj
 0001:00046b80       $L35068                    00447b80 f   rylgamelibrary:session.obj
 0001:00046b88       __ehhandler$??$?6U?$char_traits@D@std@@@std@@YAAAV?$basic_ostream@DU?$char_traits@D@std@@@0@AAV10@PBD@Z 00447b88 f   rylgamelibrary:session.obj
 0001:00046ba0       $L25288                    00447ba0 f   rylgamelibrary:threadmgr.obj
 0001:00046bae       __ehhandler$??1CThreadMgr@@UAE@XZ 00447bae f   rylgamelibrary:threadmgr.obj
 0001:00046bc0       $L98763                    00447bc0 f   rylgamelibrary:itemmgr.obj
 0001:00046bc0       $L98535                    00447bc0 f   rylgamelibrary:itemmgr.obj
 0001:00046bc8       __ehhandler$?_Xlen@?$vector@UItemInfo@Item@@V?$allocator@UItemInfo@Item@@@std@@@std@@IBEXXZ 00447bc8 f   rylgamelibrary:itemmgr.obj
 0001:00046bc8       __ehhandler$?_Xlen@?$vector@UParseData@ItemDataParser@@V?$allocator@UParseData@ItemDataParser@@@std@@@std@@IBEXXZ 00447bc8 f   rylgamelibrary:itemmgr.obj
 0001:00046be0       __ehhandler$?_Insert_n@?$vector@UItemInfo@Item@@V?$allocator@UItemInfo@Item@@@std@@@std@@IAEXViterator@12@IABUItemInfo@Item@@@Z 00447be0 f   rylgamelibrary:itemmgr.obj
 0001:00046bf0       $L100168                   00447bf0 f   rylgamelibrary:itemmgr.obj
 0001:00046bfb       $L100169                   00447bfb f   rylgamelibrary:itemmgr.obj
 0001:00046c06       $L100170                   00447c06 f   rylgamelibrary:itemmgr.obj
 0001:00046c11       $L100171                   00447c11 f   rylgamelibrary:itemmgr.obj
 0001:00046c1c       $L100172                   00447c1c f   rylgamelibrary:itemmgr.obj
 0001:00046c27       $L100173                   00447c27 f   rylgamelibrary:itemmgr.obj
 0001:00046c32       $L100174                   00447c32 f   rylgamelibrary:itemmgr.obj
 0001:00046c40       __ehhandler$?LoadItemProtoType@CItemMgr@Item@@QAE_NPBD@Z 00447c40 f   rylgamelibrary:itemmgr.obj
 0001:00046c50       $L84382                    00447c50 f   rylgamelibrary:itemfactory.obj
 0001:00046c5b       $L84383                    00447c5b f   rylgamelibrary:itemfactory.obj
 0001:00046c66       $L84384                    00447c66 f   rylgamelibrary:itemfactory.obj
 0001:00046c71       __ehhandler$?CreateItem@CItemFactory@Item@@QAEPAVCItem@2@ABUItemInfo@2@@Z 00447c71 f   rylgamelibrary:itemfactory.obj
 0001:00046c80       $L38684                    00447c80 f   rylgamelibrary:serverwindowframework.obj
 0001:00046c88       __ehhandler$??1CProcessThread@@UAE@XZ 00447c88 f   rylgamelibrary:serverwindowframework.obj
 0001:00046ca0       $L38859                    00447ca0 f   rylgamelibrary:serverwindowframework.obj
 0001:00046cab       $L38860                    00447cab f   rylgamelibrary:serverwindowframework.obj
 0001:00046cb6       __ehhandler$?InitializeFramework@CServerWindowFramework@@IAE_NPAUHINSTANCE__@@PBDHH@Z 00447cb6 f   rylgamelibrary:serverwindowframework.obj
 0001:00046cc0       $L40163                    00447cc0 f   rylgamelibrary:serverwindowframework.obj
 0001:00046ccb       __ehhandler$??1CServerWindowFramework@@MAE@XZ 00447ccb f   rylgamelibrary:serverwindowframework.obj
 0001:00046ce0       $L40707                    00447ce0 f   rylgamelibrary:serverwindowframework.obj
 0001:00046cf2       $L40708                    00447cf2 f   rylgamelibrary:serverwindowframework.obj
 0001:00046d04       $L40709                    00447d04 f   rylgamelibrary:serverwindowframework.obj
 0001:00046d16       $L40710                    00447d16 f   rylgamelibrary:serverwindowframework.obj
 0001:00046d28       $L40711                    00447d28 f   rylgamelibrary:serverwindowframework.obj
 0001:00046d3a       $L40712                    00447d3a f   rylgamelibrary:serverwindowframework.obj
 0001:00046d4c       __ehhandler$??0CServerWindowFramework@@IAE@XZ 00447d4c f   rylgamelibrary:serverwindowframework.obj
 0001:00046d60       $L41181                    00447d60 f   rylgamelibrary:serverwindowframework.obj
 0001:00046d68       __ehhandler$?_Incsize@?$list@PAVCThread@@V?$allocator@PAVCThread@@@std@@@std@@IAEXI@Z 00447d68 f   rylgamelibrary:serverwindowframework.obj
 0001:00046d80       __ehhandler$?reserve@?$vector@KV?$allocator@K@std@@@std@@QAEXI@Z 00447d80 f   rylgamelibrary:limituserbyip.obj
 0001:00046d90       $L36500                    00447d90 f   rylgamelibrary:limituserbyip.obj
 0001:00046d9b       __ehhandler$?LoadAllowIPList@CLimitUserByIP@@QAE_NPBD@Z 00447d9b f   rylgamelibrary:limituserbyip.obj
 0001:00046db0       $L36858                    00447db0 f   rylgamelibrary:limituserbyip.obj
 0001:00046db8       $L36859                    00447db8 f   rylgamelibrary:limituserbyip.obj
 0001:00046dc3       $L36860                    00447dc3 f   rylgamelibrary:limituserbyip.obj
 0001:00046dce       __ehhandler$??0CLimitUserByIP@@QAE@PBD@Z 00447dce f   rylgamelibrary:limituserbyip.obj
 0001:00046de0       $L37694                    00447de0 f   rylgamelibrary:listener.obj
 0001:00046deb       __ehhandler$??0CListener@@QAE@AAVCCompletionHandler@@AAVCSessionPolicy@@AAVCSessionMgr@@PAVCValidateConnection@@@Z 00447deb f   rylgamelibrary:listener.obj
 0001:00046e00       $L37763                    00447e00 f   rylgamelibrary:listener.obj
 0001:00046e08       __ehhandler$?PendingAccept@CListener@@QAE_NXZ 00447e08 f   rylgamelibrary:listener.obj
 0001:00046e20       $L37959                    00447e20 f   rylgamelibrary:listener.obj
 0001:00046e2b       $L37960                    00447e2b f   rylgamelibrary:listener.obj
 0001:00046e33       __ehhandler$??1CListener@@UAE@XZ 00447e33 f   rylgamelibrary:listener.obj
 0001:00046e40       $L38017                    00447e40 f   rylgamelibrary:listener.obj
 0001:00046e48       __ehhandler$?Initialize@CListener@@QAE_NAAVINET_Addr@@K@Z 00447e48 f   rylgamelibrary:listener.obj
 0001:00046e60       $L37365                    00447e60 f   rylgamelibrary:iocpnet.obj
 0001:00046e60       $L35934                    00447e60 f   rylgamelibrary:iocpnet.obj
 0001:00046e68       __ehhandler$?Process@CSessionMgr@@QAEXXZ 00447e68 f   rylgamelibrary:iocpnet.obj
 0001:00046e68       __ehhandler$?GetAcceptPendingNum@CIOCPNet@@QAEKXZ 00447e68 f   rylgamelibrary:iocpnet.obj
 0001:00046e80       $L35998                    00447e80 f   rylgamelibrary:iocpnet.obj
 0001:00046e92       __ehhandler$?Initialize@CIOCPNet@@QAE_NXZ 00447e92 f   rylgamelibrary:iocpnet.obj
 0001:00046ea0       __ehhandler$?_Copy@?$_Tree@V?$_Tmap_traits@PAVCSessionPolicy@@IU?$less@PAVCSessionPolicy@@@std@@V?$allocator@U?$pair@QAVCSessionPolicy@@I@std@@@3@$0A@@std@@@std@@IAEPAU_Node@?$_Tree_nod@V?$_Tmap_traits@PAVCSessionPolicy@@IU?$less@PAVCSessionPolicy@@@std@@V?$allocator@U?$pair@QAVCSessionPolicy@@I@std@@@3@$0A@@std@@@2@PAU342@0@Z 00447ea0 f   rylgamelibrary:iocpnet.obj
 0001:00046eb0       $L39910                    00447eb0 f   rylgamelibrary:iocpnet.obj
 0001:00046eb0       $L39307                    00447eb0 f   rylgamelibrary:iocpnet.obj
 0001:00046eb0       $L40397                    00447eb0 f   rylgamelibrary:iocpnet.obj
 0001:00046eb8       __ehhandler$?_Insert@?$_Tree@V?$_Tmap_traits@PAVCSessionPolicy@@IU?$less@PAVCSessionPolicy@@@std@@V?$allocator@U?$pair@QAVCSessionPolicy@@I@std@@@3@$0A@@std@@@std@@IAE?AViterator@12@_NPAU_Node@?$_Tree_nod@V?$_Tmap_traits@PAVCSessionPolicy@@IU?$less@PAVCSessionPolicy@@@std@@V?$allocator@U?$pair@QAVCSessionPolicy@@I@std@@@3@$0A@@std@@@2@ABU?$pair@QAVCSessionPolicy@@I@2@@Z 00447eb8 f   rylgamelibrary:iocpnet.obj
 0001:00046eb8       __ehhandler$?_Incsize@?$list@PAVCListener@@V?$allocator@PAVCListener@@@std@@@std@@IAEXI@Z 00447eb8 f   rylgamelibrary:iocpnet.obj
 0001:00046eb8       __ehhandler$?erase@?$_Tree@V?$_Tmap_traits@PAVCSessionPolicy@@IU?$less@PAVCSessionPolicy@@@std@@V?$allocator@U?$pair@QAVCSessionPolicy@@I@std@@@3@$0A@@std@@@std@@QAE?AViterator@12@V312@@Z 00447eb8 f   rylgamelibrary:iocpnet.obj
 0001:00046ed0       __ehhandler$??0?$_Tree@V?$_Tmap_traits@PAVCSessionPolicy@@IU?$less@PAVCSessionPolicy@@@std@@V?$allocator@U?$pair@QAVCSessionPolicy@@I@std@@@3@$0A@@std@@@std@@QAE@ABV01@@Z 00447ed0 f   rylgamelibrary:iocpnet.obj
 0001:00046ee0       $L42541                    00447ee0 f   rylgamelibrary:iocpnet.obj
 0001:00046eeb       $L42542                    00447eeb f   rylgamelibrary:iocpnet.obj
 0001:00046f00       $L42543                    00447f00 f   rylgamelibrary:iocpnet.obj
 0001:00046f15       $L42544                    00447f15 f   rylgamelibrary:iocpnet.obj
 0001:00046f2a       $L42545                    00447f2a f   rylgamelibrary:iocpnet.obj
 0001:00046f38       __ehhandler$??0CIOCPNet@@QAE@XZ 00447f38 f   rylgamelibrary:iocpnet.obj
 0001:00046f50       $L42867                    00447f50 f   rylgamelibrary:iocpnet.obj
 0001:00046f62       $L42868                    00447f62 f   rylgamelibrary:iocpnet.obj
 0001:00046f6a       __ehhandler$?AddListener@CIOCPNet@@QAE_NPAVCSessionPolicy@@PBDGKPAVCValidateConnection@@@Z 00447f6a f   rylgamelibrary:iocpnet.obj
 0001:00046f80       $L42900                    00447f80 f   rylgamelibrary:iocpnet.obj
 0001:00046f88       __ehhandler$?Connect@CIOCPNet@@QAE_NPAVCSessionPolicy@@PBDG@Z 00447f88 f   rylgamelibrary:iocpnet.obj
 0001:00046fa0       $L43001                    00447fa0 f   rylgamelibrary:iocpnet.obj
 0001:00046fa8       $L43002                    00447fa8 f   rylgamelibrary:iocpnet.obj
 0001:00046fb0       __ehhandler$?DestroyListener@CIOCPNet@@AAEXXZ 00447fb0 f   rylgamelibrary:iocpnet.obj
 0001:00046fc0       $L43389                    00447fc0 f   rylgamelibrary:iocpnet.obj
 0001:00046fc8       __ehhandler$?Destroy@CIOCPNet@@AAE_NXZ 00447fc8 f   rylgamelibrary:iocpnet.obj
 0001:00046fe0       $L43902                    00447fe0 f   rylgamelibrary:iocpnet.obj
 0001:00046fe8       $L43903                    00447fe8 f   rylgamelibrary:iocpnet.obj
 0001:00046ff3       $L43904                    00447ff3 f   rylgamelibrary:iocpnet.obj
 0001:00046ffe       __ehhandler$??1CIOCPNet@@QAE@XZ 00447ffe f   rylgamelibrary:iocpnet.obj
 0001:00047010       $L30277                    00448010 f   rylgamelibrary:performancecheck.obj
 0001:0004701b       __ehhandler$?PrintAllTime@CPerformanceCheck@@QAE_NPBD_N@Z 0044801b f   rylgamelibrary:performancecheck.obj
 0001:00047030       $L31547                    00448030 f   rylgamelibrary:performancecheck.obj
 0001:00047038       __ehhandler$?erase@?$_Tree@V?$_Tmap_traits@KUInstrument@CPerformanceCheck@@U?$less@K@std@@V?$allocator@U?$pair@$$CBKUInstrument@CPerformanceCheck@@@std@@@4@$00@std@@@std@@QAE?AViterator@12@V312@@Z 00448038 f   rylgamelibrary:performancecheck.obj
 0001:00047050       $L33302                    00448050 f   rylgamelibrary:performancecheck.obj
 0001:00047058       $L33303                    00448058 f   rylgamelibrary:performancecheck.obj
 0001:00047063       $L33304                    00448063 f   rylgamelibrary:performancecheck.obj
 0001:0004706b       __ehhandler$??1CPerformanceCheck@@AAE@XZ 0044806b f   rylgamelibrary:performancecheck.obj
 0001:00047080       $L33835                    00448080 f   rylgamelibrary:performancecheck.obj
 0001:00047088       __ehhandler$??0CPerformanceCheck@@AAE@XZ 00448088 f   rylgamelibrary:performancecheck.obj
 0001:000470a0       $L34060                    004480a0 f   rylgamelibrary:performancecheck.obj
 0001:000470ae       __ehhandler$?GetInstance@CPerformanceCheck@@SAAAV1@XZ 004480ae f   rylgamelibrary:performancecheck.obj
 0001:000470c0       $L88404                    004480c0 f   rylgamelibrary:gamelog.obj
 0001:000470c0       $L85631                    004480c0 f   rylgamelibrary:gamelog.obj
 0001:000470c0       $L88279                    004480c0 f   rylgamelibrary:gamelog.obj
 0001:000470c0       $L87674                    004480c0 f   rylgamelibrary:gamelog.obj
 0001:000470c8       __ehhandler$?SpliceOutFullBuffer@CGameLog@@AAEXAAV?$list@PAULogBuffer@@V?$allocator@PAULogBuffer@@@std@@@std@@@Z 004480c8 f   rylgamelibrary:gamelog.obj
 0001:000470c8       __ehhandler$?PushFullBuffer@CGameLog@@AAEXPAPAULogBuffer@@@Z 004480c8 f   rylgamelibrary:gamelog.obj
 0001:000470c8       __ehhandler$?GetBuffer@CGameLog@@AAEPAULogBuffer@@XZ 004480c8 f   rylgamelibrary:gamelog.obj
 0001:000470c8       __ehhandler$?SpliceInFreeBuffer@CGameLog@@AAEXAAV?$list@PAULogBuffer@@V?$allocator@PAULogBuffer@@@std@@@std@@@Z 004480c8 f   rylgamelibrary:gamelog.obj
 0001:000470e0       $L86363                    004480e0 f   rylgamelibrary:gamelog.obj
 0001:000470e8       __ehhandler$??0CLogSaveThread@@QAE@XZ 004480e8 f   rylgamelibrary:gamelog.obj
 0001:00047100       $L86466                    00448100 f   rylgamelibrary:gamelog.obj
 0001:00047108       $L86467                    00448108 f   rylgamelibrary:gamelog.obj
 0001:00047113       $L86468                    00448113 f   rylgamelibrary:gamelog.obj
 0001:0004711e       __ehhandler$??0CGameLog@@QAE@XZ 0044811e f   rylgamelibrary:gamelog.obj
 0001:00047130       $L87021                    00448130 f   rylgamelibrary:gamelog.obj
 0001:00047138       __ehhandler$?_Incsize@?$list@PAULogBuffer@@V?$allocator@PAULogBuffer@@@std@@@std@@IAEXI@Z 00448138 f   rylgamelibrary:gamelog.obj
 0001:00047150       $L88527                    00448150 f   rylgamelibrary:gamelog.obj
 0001:00047158       $L88528                    00448158 f   rylgamelibrary:gamelog.obj
 0001:00047163       $L88529                    00448163 f   rylgamelibrary:gamelog.obj
 0001:0004716e       $L88530                    0044816e f   rylgamelibrary:gamelog.obj
 0001:00047179       __ehhandler$??1CGameLog@@QAE@XZ 00448179 f   rylgamelibrary:gamelog.obj
 0001:00047190       $L88607                    00448190 f   rylgamelibrary:gamelog.obj
 0001:0004719e       __ehhandler$?GetInstance@CGameLog@@SAAAV1@XZ 0044819e f   rylgamelibrary:gamelog.obj
 0001:000471b0       $L30166                    004481b0 f   rylgamelibrary:bufferfactory.obj
 0001:000471b8       __ehhandler$?Release@CPoolBufferFactory@@UAEXPAVCBuffer@@@Z 004481b8 f   rylgamelibrary:bufferfactory.obj
 0001:000471d0       $L31285                    004481d0 f   rylgamelibrary:bufferfactory.obj
 0001:000471d8       $L31286                    004481d8 f   rylgamelibrary:bufferfactory.obj
 0001:000471e9       __ehhandler$?Create@CPoolBufferFactory@@UAEPAVCBuffer@@I@Z 004481e9 f   rylgamelibrary:bufferfactory.obj
 0001:00047200       $L32194                    00448200 f   rylgamelibrary:bufferfactory.obj
 0001:00047208       __ehhandler$?_Xlen@?$vector@PAV?$pool@Udefault_user_allocator_new_delete@boost@@@boost@@V?$allocator@PAV?$pool@Udefault_user_allocator_new_delete@boost@@@boost@@@std@@@std@@IBEXXZ 00448208 f   rylgamelibrary:bufferfactory.obj
 0001:00047220       $L32948                    00448220 f   rylgamelibrary:bufferfactory.obj
 0001:00047228       __ehhandler$?Initialize@CPoolBufferFactory@@IAE_NXZ 00448228 f   rylgamelibrary:bufferfactory.obj
 0001:00047240       $L33283                    00448240 f   rylgamelibrary:bufferfactory.obj
 0001:00047248       $L33284                    00448248 f   rylgamelibrary:bufferfactory.obj
 0001:00047253       $L33285                    00448253 f   rylgamelibrary:bufferfactory.obj
 0001:0004725e       __ehhandler$??0CPoolBufferFactory@@QAE@XZ 0044825e f   rylgamelibrary:bufferfactory.obj
 0001:00047270       $L30056                    00448270 f   rylgamelibrary:overlapped.obj
 0001:00047270       $L29646                    00448270 f   rylgamelibrary:overlapped.obj
 0001:00047278       __ehhandler$?Recv@CSession@@QAE_NXZ 00448278 f   rylgamelibrary:overlapped.obj
 0001:00047278       __ehhandler$?DeleteOverlapped@CStreamOverlappedFactory@@UAEXPAVCOverlapped@@@Z 00448278 f   rylgamelibrary:overlapped.obj
 0001:00047290       $L31954                    00448290 f   rylgamelibrary:consolecmdfactory.obj
 0001:00047298       __ehhandler$?_Xlen@?$vector@UStringCMD@CConsoleCMDFactory@@V?$allocator@UStringCMD@CConsoleCMDFactory@@@std@@@std@@IBEXXZ 00448298 f   rylgamelibrary:consolecmdfactory.obj
 0001:000472b0       __ehhandler$?_Insert_n@?$vector@UStringCMD@CConsoleCMDFactory@@V?$allocator@UStringCMD@CConsoleCMDFactory@@@std@@@std@@IAEXViterator@12@IABUStringCMD@CConsoleCMDFactory@@@Z 004482b0 f   rylgamelibrary:consolecmdfactory.obj
 0001:000472c0       $L24594                    004482c0 f   rylgamelibrary:exceptionreport.obj
 0001:000472cb       __ehhandler$??0CExceptionReport@@AAE@XZ 004482cb f   rylgamelibrary:exceptionreport.obj
 0001:000472e0       $L24651                    004482e0 f   rylgamelibrary:exceptionreport.obj
 0001:000472ee       __ehhandler$?GetInstance@CExceptionReport@@SAAAV1@XZ 004482ee f   rylgamelibrary:exceptionreport.obj
 0001:00047300       $L30367                    00448300 f   rylgamelibrary:msgproc.obj
 0001:00047300       $L31314                    00448300 f   rylgamelibrary:msgproc.obj
 0001:00047308       __ehhandler$?erase@?$_Tree@V?$_Tmap_traits@IPAVCMsgProc@@U?$less@I@std@@V?$allocator@U?$pair@$$CBIPAVCMsgProc@@@std@@@3@$0A@@std@@@std@@QAE?AViterator@12@V312@@Z 00448308 f   rylgamelibrary:msgproc.obj
 0001:00047308       __ehhandler$?_Insert@?$_Tree@V?$_Tmap_traits@IPAVCMsgProc@@U?$less@I@std@@V?$allocator@U?$pair@$$CBIPAVCMsgProc@@@std@@@3@$0A@@std@@@std@@IAE?AViterator@12@_NPAU_Node@?$_Tree_nod@V?$_Tmap_traits@IPAVCMsgProc@@U?$less@I@std@@V?$allocator@U?$pair@$$CBIPAVCMsgProc@@@std@@@3@$0A@@std@@@2@ABU?$pair@$$CBIPAVCMsgProc@@@2@@Z 00448308 f   rylgamelibrary:msgproc.obj
 0001:00047320       $L32123                    00448320 f   rylgamelibrary:msgproc.obj
 0001:00047328       __ehhandler$??1CMsgProcessMgr@@QAE@XZ 00448328 f   rylgamelibrary:msgproc.obj
 0001:00047340       $L29954                    00448340 f   rylgamelibrary:consolewindow.obj
 0001:0004734b       __ehhandler$??0CConsoleWindow@@QAE@PAUHINSTANCE__@@PAUHWND__@@AAVCConsoleCMDFactory@@AAVCCommandProcess@@@Z 0044834b f   rylgamelibrary:consolewindow.obj
 0001:00047360       $L33666                    00448360 f   rylgamelibrary:regfunctions.obj
 0001:0004736b       __ehhandler$??0?$ctype@D@std@@QAE@PBF_NI@Z 0044836b f   rylgamelibrary:regfunctions.obj
 0001:00047380       $L34752                    00448380 f   rylgamelibrary:regfunctions.obj
 0001:00047380       $L37406                    00448380 f   rylgamelibrary:regfunctions.obj
 0001:00047388       __ehhandler$??$use_facet@V?$codecvt@DDH@std@@@std@@YAABV?$codecvt@DDH@0@ABVlocale@0@@Z 00448388 f   rylgamelibrary:regfunctions.obj
 0001:00047388       __ehhandler$??$use_facet@V?$ctype@D@std@@@std@@YAABV?$ctype@D@0@ABVlocale@0@@Z 00448388 f   rylgamelibrary:regfunctions.obj
 0001:000473a0       $L34779                    004483a0 f   rylgamelibrary:regfunctions.obj
 0001:000473ab       __ehhandler$??0?$codecvt@DDH@std@@QAE@I@Z 004483ab f   rylgamelibrary:regfunctions.obj
 0001:000473c0       $L35997                    004483c0 f   rylgamelibrary:regfunctions.obj
 0001:000473cb       __ehhandler$??0?$basic_streambuf@DU?$char_traits@D@std@@@std@@IAE@XZ 004483cb f   rylgamelibrary:regfunctions.obj
 0001:000473e0       $L36185                    004483e0 f   rylgamelibrary:regfunctions.obj
 0001:000473e8       __ehhandler$?widen@?$basic_ios@DU?$char_traits@D@std@@@std@@QBEDD@Z 004483e8 f   rylgamelibrary:regfunctions.obj
 0001:00047400       $L36228                    00448400 f   rylgamelibrary:regfunctions.obj
 0001:00047400       $L33750                    00448400 f   rylgamelibrary:regfunctions.obj
 0001:0004740b       __ehhandler$?_Getcat@?$codecvt@DDH@std@@SAIPAPBVfacet@locale@2@@Z 0044840b f   rylgamelibrary:regfunctions.obj
 0001:0004740b       __ehhandler$?_Getcat@?$ctype@D@std@@SAIPAPBVfacet@locale@2@@Z 0044840b f   rylgamelibrary:regfunctions.obj
 0001:00047420       $L39753                    00448420 f   rylgamelibrary:regfunctions.obj
 0001:00047420       $L38655                    00448420 f   rylgamelibrary:regfunctions.obj
 0001:00047428       __ehhandler$?overflow@?$basic_filebuf@DU?$char_traits@D@std@@@std@@MAEHH@Z 00448428 f   rylgamelibrary:regfunctions.obj
 0001:00047428       __ehhandler$?_Endwrite@?$basic_filebuf@DU?$char_traits@D@std@@@std@@IAE_NXZ 00448428 f   rylgamelibrary:regfunctions.obj
 0001:00047440       $L39458                    00448440 f   rylgamelibrary:regfunctions.obj
 0001:0004745c       __ehhandler$??0?$basic_ostream@DU?$char_traits@D@std@@@std@@QAE@PAV?$basic_streambuf@DU?$char_traits@D@std@@@1@_N@Z 0044845c f   rylgamelibrary:regfunctions.obj
 0001:00047470       $L42332                    00448470 f   rylgamelibrary:regfunctions.obj
 0001:00047478       __ehhandler$??1?$basic_filebuf@DU?$char_traits@D@std@@@std@@UAE@XZ 00448478 f   rylgamelibrary:regfunctions.obj
 0001:00047490       $L90710                    00448490 f   rylgamelibrary:tokenlizedfile.obj
 0001:00047490       $L90938                    00448490 f   rylgamelibrary:tokenlizedfile.obj
 0001:00047498       __ehhandler$?_Xlen@?$vector@PADV?$allocator@PAD@std@@@std@@IBEXXZ 00448498 f   rylgamelibrary:tokenlizedfile.obj
 0001:00047498       __ehhandler$?_Xlen@?$vector@UColumnInfo@CTokenlizedFile@@V?$allocator@UColumnInfo@CTokenlizedFile@@@std@@@std@@IBEXXZ 00448498 f   rylgamelibrary:tokenlizedfile.obj
 0001:000474b0       __ehhandler$?_Insert_n@?$vector@UColumnInfo@CTokenlizedFile@@V?$allocator@UColumnInfo@CTokenlizedFile@@@std@@@std@@IAEXViterator@12@IABUColumnInfo@CTokenlizedFile@@@Z 004484b0 f   rylgamelibrary:tokenlizedfile.obj
 0001:000474c0       __ehhandler$?reserve@?$vector@UColumnInfo@CTokenlizedFile@@V?$allocator@UColumnInfo@CTokenlizedFile@@@std@@@std@@QAEXI@Z 004484c0 f   rylgamelibrary:tokenlizedfile.obj
 0001:000474d0       __ehhandler$?reserve@?$vector@PADV?$allocator@PAD@std@@@std@@QAEXI@Z 004484d0 f   rylgamelibrary:tokenlizedfile.obj
 0001:000474e0       $L92340                    004484e0 f   rylgamelibrary:tokenlizedfile.obj
 0001:000474ee       $L92341                    004484ee f   rylgamelibrary:tokenlizedfile.obj
 0001:000474fc       __ehhandler$??0CTokenlizedFile@@QAE@PBD@Z 004484fc f   rylgamelibrary:tokenlizedfile.obj
 0001:00047510       $L91864                    00448510 f   rylgamelibrary:itemconstants.obj
 0001:00047518       __ehhandler$??1CItemType@Item@@QAE@XZ 00448518 f   rylgamelibrary:itemconstants.obj
 0001:00047530       $L92451                    00448530 f   rylgamelibrary:itemconstants.obj
 0001:00047538       __ehhandler$?_Xlen@?$vector@W4Type@ItemType@Item@@V?$allocator@W4Type@ItemType@Item@@@std@@@std@@IBEXXZ 00448538 f   rylgamelibrary:itemconstants.obj
 0001:00047550       __ehhandler$?_Insert_n@?$vector@W4Type@ItemType@Item@@V?$allocator@W4Type@ItemType@Item@@@std@@@std@@IAEXViterator@12@IABW4Type@ItemType@Item@@@Z 00448550 f   rylgamelibrary:itemconstants.obj
 0001:00047560       __ehhandler$?reserve@?$vector@W4Type@ItemType@Item@@V?$allocator@W4Type@ItemType@Item@@@std@@@std@@QAEXI@Z 00448560 f   rylgamelibrary:itemconstants.obj
 0001:00047570       $L93574                    00448570 f   rylgamelibrary:itemconstants.obj
 0001:00047578       $L93575                    00448578 f   rylgamelibrary:itemconstants.obj
 0001:0004758b       __ehhandler$??0CItemType@Item@@AAE@XZ 0044858b f   rylgamelibrary:itemconstants.obj
 0001:000475a0       __ehhandler$?_Insert_n@?$vector@UParseData@ItemDataParser@@V?$allocator@UParseData@ItemDataParser@@@std@@@std@@IAEXViterator@12@IABUParseData@ItemDataParser@@@Z 004485a0 f   rylgamelibrary:itemdataparser.obj
 0001:000475b0       __ehhandler$?reserve@?$vector@UParseData@ItemDataParser@@V?$allocator@UParseData@ItemDataParser@@@std@@@std@@QAEXI@Z 004485b0 f   rylgamelibrary:itemdataparser.obj
 0001:000475c0       $L32808                    004485c0 f   rylgamelibrary:timerproc.obj
 0001:000475c8       __ehhandler$?erase@?$_Tree@V?$_Tmap_traits@IUInternalTimerData@CTimerProcMgr@@U?$less@I@std@@V?$allocator@U?$pair@$$CBIUInternalTimerData@CTimerProcMgr@@@std@@@4@$0A@@std@@@std@@QAE?AViterator@12@V312@@Z 004485c8 f   rylgamelibrary:timerproc.obj
 0001:000475e0       $L35285                    004485e0 f   rylgamelibrary:timerproc.obj
 0001:000475e8       __ehhandler$??1CTimerProcMgr@@QAE@XZ 004485e8 f   rylgamelibrary:timerproc.obj
 0001:00047600       $L28780                    00448600 f   rylgamelibrary:command.obj
 0001:00047608       __ehhandler$?ClearAll@CCommandProcess@@IAEXXZ 00448608 f   rylgamelibrary:command.obj
 0001:00047620       $L29489                    00448620 f   rylgamelibrary:command.obj
 0001:00047628       __ehhandler$??0CCommandProcess@@QAE@XZ 00448628 f   rylgamelibrary:command.obj
 0001:00047640       $L29588                    00448640 f   rylgamelibrary:command.obj
 0001:00047648       $L29589                    00448648 f   rylgamelibrary:command.obj
 0001:00047653       __ehhandler$??1CCommandProcess@@QAE@XZ 00448653 f   rylgamelibrary:command.obj
 0001:00047660       $L30558                    00448660 f   rylgamelibrary:command.obj
 0001:00047668       __ehhandler$?ProcessAll@CCommandProcess@@QAEXXZ 00448668 f   rylgamelibrary:command.obj
 0001:00047680       $L67629                    00448680 f   rylgamelibrary:sessionmgr.obj
 0001:00047680       $L65441                    00448680 f   rylgamelibrary:sessionmgr.obj
 0001:00047680       $L67879                    00448680 f   rylgamelibrary:sessionmgr.obj
 0001:00047688       __ehhandler$?Add@CSessionMgr@@QAEXPAVCSession@@@Z 00448688 f   rylgamelibrary:sessionmgr.obj
 0001:00047688       __ehhandler$?DeleteSession@CSessionMgr@@QAEXPAVCSession@@@Z 00448688 f   rylgamelibrary:sessionmgr.obj
 0001:00047688       __ehhandler$?InternalProcess@CSessionMgr@@AAEXXZ 00448688 f   rylgamelibrary:sessionmgr.obj
 0001:000476a0       $L66515                    004486a0 f   rylgamelibrary:sessionmgr.obj
 0001:000476a0       $L68410                    004486a0 f   rylgamelibrary:sessionmgr.obj
 0001:000476a8       $L66516                    004486a8 f   rylgamelibrary:sessionmgr.obj
 0001:000476a8       $L68411                    004486a8 f   rylgamelibrary:sessionmgr.obj
 0001:000476b3       $L68412                    004486b3 f   rylgamelibrary:sessionmgr.obj
 0001:000476b3       $L66517                    004486b3 f   rylgamelibrary:sessionmgr.obj
 0001:000476be       $L68413                    004486be f   rylgamelibrary:sessionmgr.obj
 0001:000476be       $L66518                    004486be f   rylgamelibrary:sessionmgr.obj
 0001:000476c9       $L66519                    004486c9 f   rylgamelibrary:sessionmgr.obj
 0001:000476c9       $L68414                    004486c9 f   rylgamelibrary:sessionmgr.obj
 0001:000476d4       __ehhandler$??0CSessionMgr@@QAE@XZ 004486d4 f   rylgamelibrary:sessionmgr.obj
 0001:000476d4       __ehhandler$??1CSessionMgr@@QAE@XZ 004486d4 f   rylgamelibrary:sessionmgr.obj
 0001:000476e0       $L66740                    004486e0 f   rylgamelibrary:sessionmgr.obj
 0001:000476e8       $L66741                    004486e8 f   rylgamelibrary:sessionmgr.obj
 0001:000476f9       __ehhandler$?CreateSession@CSessionMgr@@QAEPAVCSession@@AAVCSessionPolicy@@@Z 004486f9 f   rylgamelibrary:sessionmgr.obj
 0001:00047710       $L67177                    00448710 f   rylgamelibrary:sessionmgr.obj
 0001:00047718       __ehhandler$?_Incsize@?$list@PAVCSession@@V?$allocator@PAVCSession@@@std@@@std@@IAEXI@Z 00448718 f   rylgamelibrary:sessionmgr.obj
 0001:00047730       $L68155                    00448730 f   rylgamelibrary:sessionmgr.obj
 0001:00047738       $L68156                    00448738 f   rylgamelibrary:sessionmgr.obj
 0001:00047740       __ehhandler$?Destroy@CSessionMgr@@QAEXK@Z 00448740 f   rylgamelibrary:sessionmgr.obj
 0001:00047750       $L124450                   00448750 f   rylgamelibrary:cellmanager.obj
 0001:00047758       __ehhandler$?put@?$basic_ostream@DU?$char_traits@D@std@@@std@@QAEAAV12@D@Z 00448758 f   rylgamelibrary:cellmanager.obj
 0001:00047770       $L112561                   00448770 f   rylgamelibrary:partymgr.obj
 0001:00047770       $L113200                   00448770 f   rylgamelibrary:partymgr.obj
 0001:00047778       __ehhandler$?erase@?$_Tree@V?$_Tmap_traits@KPAVCCharacter@@U?$less@K@std@@V?$allocator@U?$pair@$$CBKPAVCCharacter@@@std@@@3@$0A@@std@@@std@@QAE?AViterator@12@V312@@Z 00448778 f   rylgamelibrary:partymgr.obj
 0001:00047778       __ehhandler$?erase@?$_Tree@V?$_Tmap_traits@KPAVCParty@@U?$less@K@std@@V?$allocator@U?$pair@$$CBKPAVCParty@@@std@@@3@$0A@@std@@@std@@QAE?AViterator@12@V312@@Z 00448778 f   rylgamelibrary:partymgr.obj
 0001:00047790       $L115240                   00448790 f   rylgamelibrary:partymgr.obj
 0001:00047798       $L115241                   00448798 f   rylgamelibrary:partymgr.obj
 0001:000477a0       $L115242                   004487a0 f   rylgamelibrary:partymgr.obj
 0001:000477ab       $L115243                   004487ab f   rylgamelibrary:partymgr.obj
 0001:000477b6       __ehhandler$??1CPartyMgr@@QAE@XZ 004487b6 f   rylgamelibrary:partymgr.obj
 0001:000477c0       $L116065                   004487c0 f   rylgamelibrary:partymgr.obj
 0001:000477c8       $L116066                   004487c8 f   rylgamelibrary:partymgr.obj
 0001:000477d0       $L116067                   004487d0 f   rylgamelibrary:partymgr.obj
 0001:000477db       __ehhandler$??0CPartyMgr@@QAE@XZ 004487db f   rylgamelibrary:partymgr.obj
 0001:000477f0       $L34185                    004487f0 f   rylgamelibrary:friendlist.obj
 0001:000477f8       __ehhandler$?erase@?$_Tree@V?$_Tmap_traits@KKU?$less@K@std@@V?$allocator@U?$pair@$$CBKK@std@@@2@$00@std@@@std@@QAE?AViterator@12@V312@@Z 004487f8 f   rylgamelibrary:friendlist.obj
 0001:00047810       $L36759                    00448810 f   rylgamelibrary:friendlist.obj
 0001:00047818       __ehhandler$??0CXRefFriends@@QAE@XZ 00448818 f   rylgamelibrary:friendlist.obj
 0001:00047830       $L36984                    00448830 f   rylgamelibrary:friendlist.obj
 0001:00047838       __ehhandler$??1CXRefFriends@@QAE@XZ 00448838 f   rylgamelibrary:friendlist.obj
 0001:00047850       $L116206                   00448850 f   rylgamelibrary:duelcellmanager.obj
 0001:00047858       __ehhandler$?erase@?$_Tree@V?$_Tmap_traits@KPAVCCell@@U?$less@K@std@@V?$allocator@U?$pair@$$CBKPAVCCell@@@std@@@3@$0A@@std@@@std@@QAE?AViterator@12@V312@@Z 00448858 f   rylgamelibrary:duelcellmanager.obj
 0001:00047870       $L120764                   00448870 f   rylgamelibrary:duelcellmanager.obj
 0001:00047878       __ehhandler$??1CDuelCellManager@@QAE@XZ 00448878 f   rylgamelibrary:duelcellmanager.obj
 0001:00047890       $L120937                   00448890 f   rylgamelibrary:duelcellmanager.obj
 0001:00047898       __ehhandler$??0CDuelCellManager@@AAE@XZ 00448898 f   rylgamelibrary:duelcellmanager.obj
 0001:000478b0       $L82267                    004488b0 f   rylgamelibrary:fsm.obj
 0001:000478b8       __ehhandler$??1CFSM@@QAE@XZ 004488b8 f   rylgamelibrary:fsm.obj
 0001:000478d0       $L94967                    004488d0 f   rylgamelibrary:questmgr.obj
 0001:000478d8       __ehhandler$??0CQuestMgr@@QAE@XZ 004488d8 f   rylgamelibrary:questmgr.obj
 0001:000478f0       $L73944                    004488f0 f   rylgamelibrary:reloctable.obj
 0001:000478f0       $L73719                    004488f0 f   rylgamelibrary:reloctable.obj
 0001:000478f8       __ehhandler$?_Xlen@?$vector@U?$pair@W4eStdFunc@@H@std@@V?$allocator@U?$pair@W4eStdFunc@@H@std@@@2@@std@@IBEXXZ 004488f8 f   rylgamelibrary:reloctable.obj
 0001:000478f8       __ehhandler$?_Xlen@?$vector@HV?$allocator@H@std@@@std@@IBEXXZ 004488f8 f   rylgamelibrary:reloctable.obj
 0001:00047910       __ehhandler$?_Insert_n@?$vector@U?$pair@W4eStdFunc@@H@std@@V?$allocator@U?$pair@W4eStdFunc@@H@std@@@2@@std@@IAEXViterator@12@IABU?$pair@W4eStdFunc@@H@2@@Z 00448910 f   rylgamelibrary:reloctable.obj
 0001:00047920       $L20838                    00448920 f   rylgamelibrary:imcodegen.obj
 0001:00047920       $L20355                    00448920 f   rylgamelibrary:imcodegen.obj
 0001:00047928       __ehhandler$?_Insert@?$_Tree@V?$_Tmap_traits@HPAV?$list@PAVIOPCode@@V?$allocator@PAVIOPCode@@@std@@@std@@U?$less@H@2@V?$allocator@U?$pair@$$CBHPAV?$list@PAVIOPCode@@V?$allocator@PAVIOPCode@@@std@@@std@@@std@@@2@$0A@@std@@@std@@IAE?AViterator@12@_NPAU_Node@?$_Tree_nod@V?$_Tmap_traits@HPAV?$list@PAVIOPCode@@V?$allocator@PAVIOPCode@@@std@@@std@@U?$less@H@2@V?$allocator@U?$pair@$$CBHPAV?$list@PAVIOPCode@@V?$allocator@PAVIOPCode@@@std@@@std@@@std@@@2@$0A@@std@@@2@ABU?$pair@$$CBHPAV?$list@PAVIOPCode@@V?$allocator@PAVIOPCode@@@std@@@std@@@2@@Z 00448928 f   rylgamelibrary:imcodegen.obj
 0001:00047928       __ehhandler$?_Incsize@?$list@PAVIOPCode@@V?$allocator@PAVIOPCode@@@std@@@std@@IAEXI@Z 00448928 f   rylgamelibrary:imcodegen.obj
 0001:00047940       $L21299                    00448940 f   rylgamelibrary:imcodegen.obj
 0001:0004794b       $L21300                    0044894b f   rylgamelibrary:imcodegen.obj
 0001:00047956       $L21301                    00448956 f   rylgamelibrary:imcodegen.obj
 0001:00047961       $L21302                    00448961 f   rylgamelibrary:imcodegen.obj
 0001:0004796c       $L21303                    0044896c f   rylgamelibrary:imcodegen.obj
 0001:00047977       $L21297                    00448977 f   rylgamelibrary:imcodegen.obj
 0001:00047982       $L21298                    00448982 f   rylgamelibrary:imcodegen.obj
 0001:0004798d       $L21304                    0044898d f   rylgamelibrary:imcodegen.obj
 0001:00047998       $L21305                    00448998 f   rylgamelibrary:imcodegen.obj
 0001:000479a3       $L21306                    004489a3 f   rylgamelibrary:imcodegen.obj
 0001:000479ae       $L21307                    004489ae f   rylgamelibrary:imcodegen.obj
 0001:000479b9       $L21308                    004489b9 f   rylgamelibrary:imcodegen.obj
 0001:000479c4       $L21309                    004489c4 f   rylgamelibrary:imcodegen.obj
 0001:000479cf       $L21310                    004489cf f   rylgamelibrary:imcodegen.obj
 0001:000479da       __ehhandler$?GenCode_DataTypeToString@@YAXW4eDataType@@W4eRegister@@@Z 004489da f   rylgamelibrary:imcodegen.obj
 0001:000479f0       $L22370                    004489f0 f   rylgamelibrary:imcodegen.obj
 0001:000479fb       $L22371                    004489fb f   rylgamelibrary:imcodegen.obj
 0001:00047a06       $L22372                    00448a06 f   rylgamelibrary:imcodegen.obj
 0001:00047a11       __ehhandler$?GenCode_If_Statement@@YAXPAUSNode@@W4eRegister@@@Z 00448a11 f   rylgamelibrary:imcodegen.obj
 0001:00047a20       $L22636                    00448a20 f   rylgamelibrary:imcodegen.obj
 0001:00047a2b       $L22637                    00448a2b f   rylgamelibrary:imcodegen.obj
 0001:00047a36       $L22638                    00448a36 f   rylgamelibrary:imcodegen.obj
 0001:00047a41       $L22639                    00448a41 f   rylgamelibrary:imcodegen.obj
 0001:00047a4c       $L22640                    00448a4c f   rylgamelibrary:imcodegen.obj
 0001:00047a57       __ehhandler$?GenCode_If_Else_Statement@@YAXPAUSNode@@W4eRegister@@@Z 00448a57 f   rylgamelibrary:imcodegen.obj
 0001:00047a70       $L23075                    00448a70 f   rylgamelibrary:imcodegen.obj
 0001:00047a7b       $L23076                    00448a7b f   rylgamelibrary:imcodegen.obj
 0001:00047a86       $L23077                    00448a86 f   rylgamelibrary:imcodegen.obj
 0001:00047a91       $L23078                    00448a91 f   rylgamelibrary:imcodegen.obj
 0001:00047a9c       $L23079                    00448a9c f   rylgamelibrary:imcodegen.obj
 0001:00047aa7       $L23080                    00448aa7 f   rylgamelibrary:imcodegen.obj
 0001:00047ab2       $L23081                    00448ab2 f   rylgamelibrary:imcodegen.obj
 0001:00047abd       __ehhandler$?GenCode_Switch_Statement@@YAXPAUSNode@@W4eRegister@@@Z 00448abd f   rylgamelibrary:imcodegen.obj
 0001:00047ad0       $L23798                    00448ad0 f   rylgamelibrary:imcodegen.obj
 0001:00047adb       $L23799                    00448adb f   rylgamelibrary:imcodegen.obj
 0001:00047ae6       $L23800                    00448ae6 f   rylgamelibrary:imcodegen.obj
 0001:00047af1       $L23801                    00448af1 f   rylgamelibrary:imcodegen.obj
 0001:00047afc       $L23802                    00448afc f   rylgamelibrary:imcodegen.obj
 0001:00047b07       $L23803                    00448b07 f   rylgamelibrary:imcodegen.obj
 0001:00047b12       $L23804                    00448b12 f   rylgamelibrary:imcodegen.obj
 0001:00047b1d       $L23805                    00448b1d f   rylgamelibrary:imcodegen.obj
 0001:00047b28       __ehhandler$?GenCode_For_Statement@@YAXPAUSNode@@W4eRegister@@@Z 00448b28 f   rylgamelibrary:imcodegen.obj
 0001:00047b40       $L24450                    00448b40 f   rylgamelibrary:imcodegen.obj
 0001:00047b4b       $L24451                    00448b4b f   rylgamelibrary:imcodegen.obj
 0001:00047b56       $L24452                    00448b56 f   rylgamelibrary:imcodegen.obj
 0001:00047b61       $L24453                    00448b61 f   rylgamelibrary:imcodegen.obj
 0001:00047b6c       $L24454                    00448b6c f   rylgamelibrary:imcodegen.obj
 0001:00047b77       __ehhandler$?GenCode_While_Statement@@YAXPAUSNode@@W4eRegister@@@Z 00448b77 f   rylgamelibrary:imcodegen.obj
 0001:00047b90       $L25154                    00448b90 f   rylgamelibrary:imcodegen.obj
 0001:00047b9b       __ehhandler$?GenCode_Variable@@YAXPAUSNode@@W4eRegister@@@Z 00448b9b f   rylgamelibrary:imcodegen.obj
 0001:00047bb0       $L25277                    00448bb0 f   rylgamelibrary:imcodegen.obj
 0001:00047bbb       $L25278                    00448bbb f   rylgamelibrary:imcodegen.obj
 0001:00047bc6       $L25279                    00448bc6 f   rylgamelibrary:imcodegen.obj
 0001:00047bd1       $L25280                    00448bd1 f   rylgamelibrary:imcodegen.obj
 0001:00047bdc       $L25281                    00448bdc f   rylgamelibrary:imcodegen.obj
 0001:00047be7       $L25282                    00448be7 f   rylgamelibrary:imcodegen.obj
 0001:00047bf2       $L25283                    00448bf2 f   rylgamelibrary:imcodegen.obj
 0001:00047bfd       $L25284                    00448bfd f   rylgamelibrary:imcodegen.obj
 0001:00047c08       __ehhandler$?GenCode_Init_Declaration@@YAXPAUSNode@@W4eRegister@@@Z 00448c08 f   rylgamelibrary:imcodegen.obj
 0001:00047c20       $L25895                    00448c20 f   rylgamelibrary:imcodegen.obj
 0001:00047c20       $L19154                    00448c20 f   rylgamelibrary:imcodegen.obj
 0001:00047c2b       __ehhandler$?HandleMARK@@YAXViterator@?$list@PAVIOPCode@@V?$allocator@PAVIOPCode@@@std@@@std@@0PAVIOPCode@@1@Z 00448c2b f   rylgamelibrary:imcodegen.obj
 0001:00047c2b       __ehhandler$?GenCode_Normal_Declaration@@YAXPAUSNode@@W4eRegister@@@Z 00448c2b f   rylgamelibrary:imcodegen.obj
 0001:00047c40       $L26019                    00448c40 f   rylgamelibrary:imcodegen.obj
 0001:00047c4b       $L26020                    00448c4b f   rylgamelibrary:imcodegen.obj
 0001:00047c56       $L26021                    00448c56 f   rylgamelibrary:imcodegen.obj
 0001:00047c61       $L26022                    00448c61 f   rylgamelibrary:imcodegen.obj
 0001:00047c6c       $L26023                    00448c6c f   rylgamelibrary:imcodegen.obj
 0001:00047c77       $L26024                    00448c77 f   rylgamelibrary:imcodegen.obj
 0001:00047c82       $L26025                    00448c82 f   rylgamelibrary:imcodegen.obj
 0001:00047c8d       $L26026                    00448c8d f   rylgamelibrary:imcodegen.obj
 0001:00047c98       __ehhandler$?GenCode_Array_Init@@YAXPAUSNode@@H@Z 00448c98 f   rylgamelibrary:imcodegen.obj
 0001:00047cb0       $L26673                    00448cb0 f   rylgamelibrary:imcodegen.obj
 0001:00047cbb       $L26674                    00448cbb f   rylgamelibrary:imcodegen.obj
 0001:00047cc6       $L26675                    00448cc6 f   rylgamelibrary:imcodegen.obj
 0001:00047cd1       $L26676                    00448cd1 f   rylgamelibrary:imcodegen.obj
 0001:00047cdc       $L26677                    00448cdc f   rylgamelibrary:imcodegen.obj
 0001:00047ce7       __ehhandler$?GenCode_Function_Declaration@@YAXPAUSNode@@W4eRegister@@@Z 00448ce7 f   rylgamelibrary:imcodegen.obj
 0001:00047d00       $L27278                    00448d00 f   rylgamelibrary:imcodegen.obj
 0001:00047d0b       $L27279                    00448d0b f   rylgamelibrary:imcodegen.obj
 0001:00047d16       $L27280                    00448d16 f   rylgamelibrary:imcodegen.obj
 0001:00047d21       $L27281                    00448d21 f   rylgamelibrary:imcodegen.obj
 0001:00047d2c       $L27282                    00448d2c f   rylgamelibrary:imcodegen.obj
 0001:00047d37       $L27283                    00448d37 f   rylgamelibrary:imcodegen.obj
 0001:00047d42       $L27284                    00448d42 f   rylgamelibrary:imcodegen.obj
 0001:00047d4d       __ehhandler$?GenCode_Function_Definition@@YAXPAUSNode@@W4eRegister@@@Z 00448d4d f   rylgamelibrary:imcodegen.obj
 0001:00047d60       $L27985                    00448d60 f   rylgamelibrary:imcodegen.obj
 0001:00047d6b       __ehhandler$?GenCode_Constant_Expression@@YAXPAUSNode@@W4eRegister@@@Z 00448d6b f   rylgamelibrary:imcodegen.obj
 0001:00047d80       $L28128                    00448d80 f   rylgamelibrary:imcodegen.obj
 0001:00047d8b       $L28129                    00448d8b f   rylgamelibrary:imcodegen.obj
 0001:00047d96       $L28130                    00448d96 f   rylgamelibrary:imcodegen.obj
 0001:00047da1       $L28131                    00448da1 f   rylgamelibrary:imcodegen.obj
 0001:00047dac       $L28132                    00448dac f   rylgamelibrary:imcodegen.obj
 0001:00047db7       $L28133                    00448db7 f   rylgamelibrary:imcodegen.obj
 0001:00047dc2       $L28134                    00448dc2 f   rylgamelibrary:imcodegen.obj
 0001:00047dcd       $L28135                    00448dcd f   rylgamelibrary:imcodegen.obj
 0001:00047dd8       $L28136                    00448dd8 f   rylgamelibrary:imcodegen.obj
 0001:00047de3       $L28137                    00448de3 f   rylgamelibrary:imcodegen.obj
 0001:00047dee       $L28138                    00448dee f   rylgamelibrary:imcodegen.obj
 0001:00047df9       $L28139                    00448df9 f   rylgamelibrary:imcodegen.obj
 0001:00047e04       __ehhandler$?GenCode_Assignment_Expression@@YAXPAUSNode@@W4eRegister@@@Z 00448e04 f   rylgamelibrary:imcodegen.obj
 0001:00047e10       $L28942                    00448e10 f   rylgamelibrary:imcodegen.obj
 0001:00047e10       $L29758                    00448e10 f   rylgamelibrary:imcodegen.obj
 0001:00047e1b       $L28943                    00448e1b f   rylgamelibrary:imcodegen.obj
 0001:00047e1b       $L29759                    00448e1b f   rylgamelibrary:imcodegen.obj
 0001:00047e26       $L28944                    00448e26 f   rylgamelibrary:imcodegen.obj
 0001:00047e26       $L29760                    00448e26 f   rylgamelibrary:imcodegen.obj
 0001:00047e31       $L29761                    00448e31 f   rylgamelibrary:imcodegen.obj
 0001:00047e31       $L28945                    00448e31 f   rylgamelibrary:imcodegen.obj
 0001:00047e3c       $L28946                    00448e3c f   rylgamelibrary:imcodegen.obj
 0001:00047e3c       $L29762                    00448e3c f   rylgamelibrary:imcodegen.obj
 0001:00047e47       $L29763                    00448e47 f   rylgamelibrary:imcodegen.obj
 0001:00047e47       $L28947                    00448e47 f   rylgamelibrary:imcodegen.obj
 0001:00047e52       $L29764                    00448e52 f   rylgamelibrary:imcodegen.obj
 0001:00047e52       $L28948                    00448e52 f   rylgamelibrary:imcodegen.obj
 0001:00047e5d       $L28949                    00448e5d f   rylgamelibrary:imcodegen.obj
 0001:00047e5d       $L29765                    00448e5d f   rylgamelibrary:imcodegen.obj
 0001:00047e68       $L29766                    00448e68 f   rylgamelibrary:imcodegen.obj
 0001:00047e68       $L28950                    00448e68 f   rylgamelibrary:imcodegen.obj
 0001:00047e73       $L29767                    00448e73 f   rylgamelibrary:imcodegen.obj
 0001:00047e73       $L28951                    00448e73 f   rylgamelibrary:imcodegen.obj
 0001:00047e7e       __ehhandler$?GenCode_AND_Expression@@YAXPAUSNode@@W4eRegister@@@Z 00448e7e f   rylgamelibrary:imcodegen.obj
 0001:00047e7e       __ehhandler$?GenCode_OR_Expression@@YAXPAUSNode@@W4eRegister@@@Z 00448e7e f   rylgamelibrary:imcodegen.obj
 0001:00047e90       $L30534                    00448e90 f   rylgamelibrary:imcodegen.obj
 0001:00047e90       $L37905                    00448e90 f   rylgamelibrary:imcodegen.obj
 0001:00047e9b       $L30535                    00448e9b f   rylgamelibrary:imcodegen.obj
 0001:00047e9b       $L37906                    00448e9b f   rylgamelibrary:imcodegen.obj
 0001:00047ea6       __ehhandler$?GenCode_NOT_Expression@@YAXPAUSNode@@W4eRegister@@@Z 00448ea6 f   rylgamelibrary:imcodegen.obj
 0001:00047ea6       __ehhandler$?GenCode_Reminder_Expression@@YAXPAUSNode@@W4eRegister@@@Z 00448ea6 f   rylgamelibrary:imcodegen.obj
 0001:00047eb0       $L31138                    00448eb0 f   rylgamelibrary:imcodegen.obj
 0001:00047eb0       $L30721                    00448eb0 f   rylgamelibrary:imcodegen.obj
 0001:00047ebb       $L30722                    00448ebb f   rylgamelibrary:imcodegen.obj
 0001:00047ebb       $L31139                    00448ebb f   rylgamelibrary:imcodegen.obj
 0001:00047ec6       $L31140                    00448ec6 f   rylgamelibrary:imcodegen.obj
 0001:00047ec6       $L30723                    00448ec6 f   rylgamelibrary:imcodegen.obj
 0001:00047ed1       $L30724                    00448ed1 f   rylgamelibrary:imcodegen.obj
 0001:00047ed1       $L31141                    00448ed1 f   rylgamelibrary:imcodegen.obj
 0001:00047edc       $L31142                    00448edc f   rylgamelibrary:imcodegen.obj
 0001:00047edc       $L30725                    00448edc f   rylgamelibrary:imcodegen.obj
 0001:00047ee7       __ehhandler$?GenCode_NotEqual_Expression@@YAXPAUSNode@@W4eRegister@@@Z 00448ee7 f   rylgamelibrary:imcodegen.obj
 0001:00047ee7       __ehhandler$?GenCode_Equality_Expression@@YAXPAUSNode@@W4eRegister@@@Z 00448ee7 f   rylgamelibrary:imcodegen.obj
 0001:00047f00       $L36189                    00448f00 f   rylgamelibrary:imcodegen.obj
 0001:00047f00       $L33058                    00448f00 f   rylgamelibrary:imcodegen.obj
 0001:00047f00       $L33800                    00448f00 f   rylgamelibrary:imcodegen.obj
 0001:00047f00       $L36771                    00448f00 f   rylgamelibrary:imcodegen.obj
 0001:00047f00       $L31574                    00448f00 f   rylgamelibrary:imcodegen.obj
 0001:00047f00       $L37353                    00448f00 f   rylgamelibrary:imcodegen.obj
 0001:00047f00       $L32316                    00448f00 f   rylgamelibrary:imcodegen.obj
 0001:00047f0b       $L36772                    00448f0b f   rylgamelibrary:imcodegen.obj
 0001:00047f0b       $L33801                    00448f0b f   rylgamelibrary:imcodegen.obj
 0001:00047f0b       $L36190                    00448f0b f   rylgamelibrary:imcodegen.obj
 0001:00047f0b       $L33059                    00448f0b f   rylgamelibrary:imcodegen.obj
 0001:00047f0b       $L37354                    00448f0b f   rylgamelibrary:imcodegen.obj
 0001:00047f0b       $L31575                    00448f0b f   rylgamelibrary:imcodegen.obj
 0001:00047f0b       $L32317                    00448f0b f   rylgamelibrary:imcodegen.obj
 0001:00047f16       $L32318                    00448f16 f   rylgamelibrary:imcodegen.obj
 0001:00047f16       $L37355                    00448f16 f   rylgamelibrary:imcodegen.obj
 0001:00047f16       $L31576                    00448f16 f   rylgamelibrary:imcodegen.obj
 0001:00047f16       $L36191                    00448f16 f   rylgamelibrary:imcodegen.obj
 0001:00047f16       $L33802                    00448f16 f   rylgamelibrary:imcodegen.obj
 0001:00047f16       $L36773                    00448f16 f   rylgamelibrary:imcodegen.obj
 0001:00047f16       $L33060                    00448f16 f   rylgamelibrary:imcodegen.obj
 0001:00047f21       $L33803                    00448f21 f   rylgamelibrary:imcodegen.obj
 0001:00047f21       $L33061                    00448f21 f   rylgamelibrary:imcodegen.obj
 0001:00047f21       $L37356                    00448f21 f   rylgamelibrary:imcodegen.obj
 0001:00047f21       $L32319                    00448f21 f   rylgamelibrary:imcodegen.obj
 0001:00047f21       $L31577                    00448f21 f   rylgamelibrary:imcodegen.obj
 0001:00047f21       $L36774                    00448f21 f   rylgamelibrary:imcodegen.obj
 0001:00047f21       $L36192                    00448f21 f   rylgamelibrary:imcodegen.obj
 0001:00047f2c       $L32320                    00448f2c f   rylgamelibrary:imcodegen.obj
 0001:00047f2c       $L33804                    00448f2c f   rylgamelibrary:imcodegen.obj
 0001:00047f2c       $L33062                    00448f2c f   rylgamelibrary:imcodegen.obj
 0001:00047f2c       $L36193                    00448f2c f   rylgamelibrary:imcodegen.obj
 0001:00047f2c       $L36775                    00448f2c f   rylgamelibrary:imcodegen.obj
 0001:00047f2c       $L31578                    00448f2c f   rylgamelibrary:imcodegen.obj
 0001:00047f2c       $L37357                    00448f2c f   rylgamelibrary:imcodegen.obj
 0001:00047f37       $L37358                    00448f37 f   rylgamelibrary:imcodegen.obj
 0001:00047f37       $L33805                    00448f37 f   rylgamelibrary:imcodegen.obj
 0001:00047f37       $L36194                    00448f37 f   rylgamelibrary:imcodegen.obj
 0001:00047f37       $L32321                    00448f37 f   rylgamelibrary:imcodegen.obj
 0001:00047f37       $L33063                    00448f37 f   rylgamelibrary:imcodegen.obj
 0001:00047f37       $L36776                    00448f37 f   rylgamelibrary:imcodegen.obj
 0001:00047f37       $L31579                    00448f37 f   rylgamelibrary:imcodegen.obj
 0001:00047f42       $L37359                    00448f42 f   rylgamelibrary:imcodegen.obj
 0001:00047f42       $L36195                    00448f42 f   rylgamelibrary:imcodegen.obj
 0001:00047f42       $L33064                    00448f42 f   rylgamelibrary:imcodegen.obj
 0001:00047f42       $L31580                    00448f42 f   rylgamelibrary:imcodegen.obj
 0001:00047f42       $L32322                    00448f42 f   rylgamelibrary:imcodegen.obj
 0001:00047f42       $L36777                    00448f42 f   rylgamelibrary:imcodegen.obj
 0001:00047f42       $L33806                    00448f42 f   rylgamelibrary:imcodegen.obj
 0001:00047f4d       $L33807                    00448f4d f   rylgamelibrary:imcodegen.obj
 0001:00047f4d       $L32323                    00448f4d f   rylgamelibrary:imcodegen.obj
 0001:00047f4d       $L36778                    00448f4d f   rylgamelibrary:imcodegen.obj
 0001:00047f4d       $L36196                    00448f4d f   rylgamelibrary:imcodegen.obj
 0001:00047f4d       $L31581                    00448f4d f   rylgamelibrary:imcodegen.obj
 0001:00047f4d       $L37360                    00448f4d f   rylgamelibrary:imcodegen.obj
 0001:00047f4d       $L33065                    00448f4d f   rylgamelibrary:imcodegen.obj
 0001:00047f58       __ehhandler$?GenCode_Division_Expression@@YAXPAUSNode@@W4eRegister@@@Z 00448f58 f   rylgamelibrary:imcodegen.obj
 0001:00047f58       __ehhandler$?GenCode_Multiplication_Expression@@YAXPAUSNode@@W4eRegister@@@Z 00448f58 f   rylgamelibrary:imcodegen.obj
 0001:00047f58       __ehhandler$?GenCode_LessThanEqual_Expression@@YAXPAUSNode@@W4eRegister@@@Z 00448f58 f   rylgamelibrary:imcodegen.obj
 0001:00047f58       __ehhandler$?GenCode_LessThan_Expression@@YAXPAUSNode@@W4eRegister@@@Z 00448f58 f   rylgamelibrary:imcodegen.obj
 0001:00047f58       __ehhandler$?GenCode_MoreThanEqual_Expression@@YAXPAUSNode@@W4eRegister@@@Z 00448f58 f   rylgamelibrary:imcodegen.obj
 0001:00047f58       __ehhandler$?GenCode_Subtraction_Expression@@YAXPAUSNode@@W4eRegister@@@Z 00448f58 f   rylgamelibrary:imcodegen.obj
 0001:00047f58       __ehhandler$?GenCode_MoreThan_Expression@@YAXPAUSNode@@W4eRegister@@@Z 00448f58 f   rylgamelibrary:imcodegen.obj
 0001:00047f70       $L34613                    00448f70 f   rylgamelibrary:imcodegen.obj
 0001:00047f7b       $L34614                    00448f7b f   rylgamelibrary:imcodegen.obj
 0001:00047f86       $L34615                    00448f86 f   rylgamelibrary:imcodegen.obj
 0001:00047f91       $L34616                    00448f91 f   rylgamelibrary:imcodegen.obj
 0001:00047f9c       $L34617                    00448f9c f   rylgamelibrary:imcodegen.obj
 0001:00047fa7       $L34618                    00448fa7 f   rylgamelibrary:imcodegen.obj
 0001:00047fb2       $L34619                    00448fb2 f   rylgamelibrary:imcodegen.obj
 0001:00047fbd       $L34620                    00448fbd f   rylgamelibrary:imcodegen.obj
 0001:00047fc8       $L34621                    00448fc8 f   rylgamelibrary:imcodegen.obj
 0001:00047fd3       $L34622                    00448fd3 f   rylgamelibrary:imcodegen.obj
 0001:00047fde       $L34623                    00448fde f   rylgamelibrary:imcodegen.obj
 0001:00047fe9       $L34624                    00448fe9 f   rylgamelibrary:imcodegen.obj
 0001:00047ff4       $L34625                    00448ff4 f   rylgamelibrary:imcodegen.obj
 0001:00047fff       $L34626                    00448fff f   rylgamelibrary:imcodegen.obj
 0001:0004800a       $L34627                    0044900a f   rylgamelibrary:imcodegen.obj
 0001:00048015       $L34628                    00449015 f   rylgamelibrary:imcodegen.obj
 0001:00048020       $L34629                    00449020 f   rylgamelibrary:imcodegen.obj
 0001:0004802b       $L34630                    0044902b f   rylgamelibrary:imcodegen.obj
 0001:00048036       $L34631                    00449036 f   rylgamelibrary:imcodegen.obj
 0001:00048041       $L34632                    00449041 f   rylgamelibrary:imcodegen.obj
 0001:0004804c       $L34633                    0044904c f   rylgamelibrary:imcodegen.obj
 0001:00048057       $L34634                    00449057 f   rylgamelibrary:imcodegen.obj
 0001:00048062       $L34635                    00449062 f   rylgamelibrary:imcodegen.obj
 0001:0004806d       __ehhandler$?GenCode_Addition_Expression@@YAXPAUSNode@@W4eRegister@@@Z 0044906d f   rylgamelibrary:imcodegen.obj
 0001:00048080       $L38196                    00449080 f   rylgamelibrary:imcodegen.obj
 0001:0004808b       $L38197                    0044908b f   rylgamelibrary:imcodegen.obj
 0001:00048096       $L38198                    00449096 f   rylgamelibrary:imcodegen.obj
 0001:000480a1       $L38199                    004490a1 f   rylgamelibrary:imcodegen.obj
 0001:000480ac       $L38200                    004490ac f   rylgamelibrary:imcodegen.obj
 0001:000480b7       $L38201                    004490b7 f   rylgamelibrary:imcodegen.obj
 0001:000480c2       $L38202                    004490c2 f   rylgamelibrary:imcodegen.obj
 0001:000480cd       $L38203                    004490cd f   rylgamelibrary:imcodegen.obj
 0001:000480d8       $L38204                    004490d8 f   rylgamelibrary:imcodegen.obj
 0001:000480e3       $L38205                    004490e3 f   rylgamelibrary:imcodegen.obj
 0001:000480ee       $L38206                    004490ee f   rylgamelibrary:imcodegen.obj
 0001:000480f9       $L38207                    004490f9 f   rylgamelibrary:imcodegen.obj
 0001:00048104       $L38208                    00449104 f   rylgamelibrary:imcodegen.obj
 0001:0004810f       $L38209                    0044910f f   rylgamelibrary:imcodegen.obj
 0001:0004811a       $L38210                    0044911a f   rylgamelibrary:imcodegen.obj
 0001:00048125       $L38211                    00449125 f   rylgamelibrary:imcodegen.obj
 0001:00048130       $L38212                    00449130 f   rylgamelibrary:imcodegen.obj
 0001:0004813b       $L38213                    0044913b f   rylgamelibrary:imcodegen.obj
 0001:00048146       $L38214                    00449146 f   rylgamelibrary:imcodegen.obj
 0001:00048151       $L38215                    00449151 f   rylgamelibrary:imcodegen.obj
 0001:0004815c       $L38216                    0044915c f   rylgamelibrary:imcodegen.obj
 0001:00048167       $L38217                    00449167 f   rylgamelibrary:imcodegen.obj
 0001:00048172       $L38218                    00449172 f   rylgamelibrary:imcodegen.obj
 0001:0004817d       $L38219                    0044917d f   rylgamelibrary:imcodegen.obj
 0001:00048188       $L38220                    00449188 f   rylgamelibrary:imcodegen.obj
 0001:00048193       __ehhandler$?GenCode_Compound_Addition@@YAXPAUSNode@@W4eRegister@@@Z 00449193 f   rylgamelibrary:imcodegen.obj
 0001:000481a0       $L40573                    004491a0 f   rylgamelibrary:imcodegen.obj
 0001:000481a0       $L39915                    004491a0 f   rylgamelibrary:imcodegen.obj
 0001:000481a0       $L41231                    004491a0 f   rylgamelibrary:imcodegen.obj
 0001:000481ab       $L40574                    004491ab f   rylgamelibrary:imcodegen.obj
 0001:000481ab       $L41232                    004491ab f   rylgamelibrary:imcodegen.obj
 0001:000481ab       $L39916                    004491ab f   rylgamelibrary:imcodegen.obj
 0001:000481b6       $L40575                    004491b6 f   rylgamelibrary:imcodegen.obj
 0001:000481b6       $L41233                    004491b6 f   rylgamelibrary:imcodegen.obj
 0001:000481b6       $L39917                    004491b6 f   rylgamelibrary:imcodegen.obj
 0001:000481c1       $L40576                    004491c1 f   rylgamelibrary:imcodegen.obj
 0001:000481c1       $L39918                    004491c1 f   rylgamelibrary:imcodegen.obj
 0001:000481c1       $L41234                    004491c1 f   rylgamelibrary:imcodegen.obj
 0001:000481cc       $L39919                    004491cc f   rylgamelibrary:imcodegen.obj
 0001:000481cc       $L40577                    004491cc f   rylgamelibrary:imcodegen.obj
 0001:000481cc       $L41235                    004491cc f   rylgamelibrary:imcodegen.obj
 0001:000481d7       $L40578                    004491d7 f   rylgamelibrary:imcodegen.obj
 0001:000481d7       $L39920                    004491d7 f   rylgamelibrary:imcodegen.obj
 0001:000481d7       $L41236                    004491d7 f   rylgamelibrary:imcodegen.obj
 0001:000481e2       $L41237                    004491e2 f   rylgamelibrary:imcodegen.obj
 0001:000481e2       $L39921                    004491e2 f   rylgamelibrary:imcodegen.obj
 0001:000481e2       $L40579                    004491e2 f   rylgamelibrary:imcodegen.obj
 0001:000481ed       $L39922                    004491ed f   rylgamelibrary:imcodegen.obj
 0001:000481ed       $L41238                    004491ed f   rylgamelibrary:imcodegen.obj
 0001:000481ed       $L40580                    004491ed f   rylgamelibrary:imcodegen.obj
 0001:000481f8       $L39923                    004491f8 f   rylgamelibrary:imcodegen.obj
 0001:000481f8       $L41239                    004491f8 f   rylgamelibrary:imcodegen.obj
 0001:000481f8       $L40581                    004491f8 f   rylgamelibrary:imcodegen.obj
 0001:00048203       __ehhandler$?GenCode_Compound_Division@@YAXPAUSNode@@W4eRegister@@@Z 00449203 f   rylgamelibrary:imcodegen.obj
 0001:00048203       __ehhandler$?GenCode_Compound_Multiplication@@YAXPAUSNode@@W4eRegister@@@Z 00449203 f   rylgamelibrary:imcodegen.obj
 0001:00048203       __ehhandler$?GenCode_Compound_Subtraction@@YAXPAUSNode@@W4eRegister@@@Z 00449203 f   rylgamelibrary:imcodegen.obj
 0001:00048210       $L41864                    00449210 f   rylgamelibrary:imcodegen.obj
 0001:0004821b       $L41865                    0044921b f   rylgamelibrary:imcodegen.obj
 0001:00048226       $L41866                    00449226 f   rylgamelibrary:imcodegen.obj
 0001:00048231       $L41867                    00449231 f   rylgamelibrary:imcodegen.obj
 0001:0004823c       __ehhandler$?GenCode_Compound_Reminder@@YAXPAUSNode@@W4eRegister@@@Z 0044923c f   rylgamelibrary:imcodegen.obj
 0001:00048250       $L42216                    00449250 f   rylgamelibrary:imcodegen.obj
 0001:00048250       $L42790                    00449250 f   rylgamelibrary:imcodegen.obj
 0001:0004825b       $L42791                    0044925b f   rylgamelibrary:imcodegen.obj
 0001:0004825b       $L42217                    0044925b f   rylgamelibrary:imcodegen.obj
 0001:00048266       $L42792                    00449266 f   rylgamelibrary:imcodegen.obj
 0001:00048266       $L42218                    00449266 f   rylgamelibrary:imcodegen.obj
 0001:00048271       $L42793                    00449271 f   rylgamelibrary:imcodegen.obj
 0001:00048271       $L42219                    00449271 f   rylgamelibrary:imcodegen.obj
 0001:0004827c       $L42220                    0044927c f   rylgamelibrary:imcodegen.obj
 0001:0004827c       $L42794                    0044927c f   rylgamelibrary:imcodegen.obj
 0001:00048287       $L42221                    00449287 f   rylgamelibrary:imcodegen.obj
 0001:00048287       $L42795                    00449287 f   rylgamelibrary:imcodegen.obj
 0001:00048292       $L42222                    00449292 f   rylgamelibrary:imcodegen.obj
 0001:00048292       $L42796                    00449292 f   rylgamelibrary:imcodegen.obj
 0001:0004829d       $L42797                    0044929d f   rylgamelibrary:imcodegen.obj
 0001:0004829d       $L42223                    0044929d f   rylgamelibrary:imcodegen.obj
 0001:000482a8       __ehhandler$?GenCode_PrefixDecrement@@YAXPAUSNode@@W4eRegister@@@Z 004492a8 f   rylgamelibrary:imcodegen.obj
 0001:000482a8       __ehhandler$?GenCode_PrefixIncrement@@YAXPAUSNode@@W4eRegister@@@Z 004492a8 f   rylgamelibrary:imcodegen.obj
 0001:000482c0       $L43339                    004492c0 f   rylgamelibrary:imcodegen.obj
 0001:000482cb       $L43340                    004492cb f   rylgamelibrary:imcodegen.obj
 0001:000482d6       $L43341                    004492d6 f   rylgamelibrary:imcodegen.obj
 0001:000482e1       __ehhandler$?GenCode_Array_Indexing@@YAXPAUSNode@@W4eRegister@@@Z 004492e1 f   rylgamelibrary:imcodegen.obj
 0001:000482f0       $L43601                    004492f0 f   rylgamelibrary:imcodegen.obj
 0001:000482fb       $L43603                    004492fb f   rylgamelibrary:imcodegen.obj
 0001:00048306       $L43602                    00449306 f   rylgamelibrary:imcodegen.obj
 0001:00048311       $L43604                    00449311 f   rylgamelibrary:imcodegen.obj
 0001:0004831c       $L43605                    0044931c f   rylgamelibrary:imcodegen.obj
 0001:00048327       __ehhandler$?GenCode_Function_Call@@YAXPAUSNode@@W4eRegister@@@Z 00449327 f   rylgamelibrary:imcodegen.obj
 0001:00048340       $L44767                    00449340 f   rylgamelibrary:imcodegen.obj
 0001:00048340       $L44039                    00449340 f   rylgamelibrary:imcodegen.obj
 0001:0004834b       $L44040                    0044934b f   rylgamelibrary:imcodegen.obj
 0001:0004834b       $L44768                    0044934b f   rylgamelibrary:imcodegen.obj
 0001:00048356       $L44041                    00449356 f   rylgamelibrary:imcodegen.obj
 0001:00048356       $L44769                    00449356 f   rylgamelibrary:imcodegen.obj
 0001:00048361       $L44042                    00449361 f   rylgamelibrary:imcodegen.obj
 0001:00048361       $L44770                    00449361 f   rylgamelibrary:imcodegen.obj
 0001:0004836c       $L44771                    0044936c f   rylgamelibrary:imcodegen.obj
 0001:0004836c       $L44043                    0044936c f   rylgamelibrary:imcodegen.obj
 0001:00048377       $L44044                    00449377 f   rylgamelibrary:imcodegen.obj
 0001:00048377       $L44772                    00449377 f   rylgamelibrary:imcodegen.obj
 0001:00048382       $L44045                    00449382 f   rylgamelibrary:imcodegen.obj
 0001:00048382       $L44773                    00449382 f   rylgamelibrary:imcodegen.obj
 0001:0004838d       $L44046                    0044938d f   rylgamelibrary:imcodegen.obj
 0001:0004838d       $L44774                    0044938d f   rylgamelibrary:imcodegen.obj
 0001:00048398       $L44047                    00449398 f   rylgamelibrary:imcodegen.obj
 0001:00048398       $L44775                    00449398 f   rylgamelibrary:imcodegen.obj
 0001:000483a3       __ehhandler$?GenCode_PostfixDecrement@@YAXPAUSNode@@W4eRegister@@@Z 004493a3 f   rylgamelibrary:imcodegen.obj
 0001:000483a3       __ehhandler$?GenCode_PostfixIncrement@@YAXPAUSNode@@W4eRegister@@@Z 004493a3 f   rylgamelibrary:imcodegen.obj
 0001:000483b0       $L17303                    004493b0 f   rylgamelibrary:imcodeunits.obj
 0001:000483b8       __ehhandler$??0COP_setcc@@QAE@W4eCondition@@W4eRegister@@@Z 004493b8 f   rylgamelibrary:imcodeunits.obj
 0001:000483c2       $L11664                    004493c2 f   libcpmt:string.obj
 0001:000483c2       $L11871                    004493c2 f   libcpmt:string.obj
 0001:000483ca       __ehhandler$?_Xran@_String_base@std@@QBEXXZ 004493ca f   libcpmt:string.obj
 0001:000483ca       __ehhandler$?_Xlen@_String_base@std@@QBEXXZ 004493ca f   libcpmt:string.obj
 0001:000483d4       $L8700                     004493d4 f   libcpmt:ios.obj
 0001:000483d4       $L8601                     004493d4 f   libcpmt:ios.obj
 0001:000483dc       __ehhandler$??0runtime_error@std@@QAE@ABV?$basic_string@DU?$char_traits@D@std@@V?$allocator@D@2@@1@@Z 004493dc f   libcpmt:ios.obj
 0001:000483dc       __ehhandler$??0runtime_error@std@@QAE@ABV01@@Z 004493dc f   libcpmt:ios.obj
 0001:000483e6       $L8663                     004493e6 f   libcpmt:ios.obj
 0001:000483ee       $L8664                     004493ee f   libcpmt:ios.obj
 0001:000483f6       $L8665                     004493f6 f   libcpmt:ios.obj
 0001:00048401       __ehhandler$?clear@ios_base@std@@QAEXH_N@Z 00449401 f   libcpmt:ios.obj
 0001:0004840b       $L12841                    0044940b f   libcpmt:locale0.obj
 0001:00048413       $L12842                    00449413 f   libcpmt:locale0.obj
 0001:0004841e       $L12843                    0044941e f   libcpmt:locale0.obj
 0001:00048426       __ehhandler$??1_Locimp@locale@std@@MAE@XZ 00449426 f   libcpmt:locale0.obj
 0001:00048430       $L13072                    00449430 f   libcpmt:locale0.obj
 0001:00048438       __ehhandler$??0_Locimp@locale@std@@AAE@_N@Z 00449438 f   libcpmt:locale0.obj
 0001:00048442       $L13087                    00449442 f   libcpmt:locale0.obj
 0001:0004844a       $L13088                    0044944a f   libcpmt:locale0.obj
 0001:00048455       $L13089                    00449455 f   libcpmt:locale0.obj
 0001:00048460       $L13090                    00449460 f   libcpmt:locale0.obj
 0001:0004846b       $L13091                    0044946b f   libcpmt:locale0.obj
 0001:00048476       __ehhandler$??0_Locinfo@std@@QAE@PBD@Z 00449476 f   libcpmt:locale0.obj
 0001:00048480       $L13116                    00449480 f   libcpmt:locale0.obj
 0001:00048488       $L13117                    00449488 f   libcpmt:locale0.obj
 0001:00048492       __ehhandler$?_Init@locale@std@@CAPAV_Locimp@12@XZ 00449492 f   libcpmt:locale0.obj
 0001:0004849c       __ehhandler$??2@YAPAXIABUnothrow_t@std@@@Z 0044949c f   LIBCMT:newopnt.obj
 0001:000484b0       _$E1                       004494b0 f   itemcreator.obj
 0001:000484d0       _$E1                       004494d0 f   rylgamelibrary:serverlog.obj
 0001:000484f0       _$E4                       004494f0 f   rylgamelibrary:serverlog.obj
 0001:00048510       _$E7                       00449510 f   rylgamelibrary:serverlog.obj
 0001:00048530       _$E5                       00449530 f   rylgamelibrary:itemmgr.obj
 0001:00048550       _$E5                       00449550 f   rylgamelibrary:itemfactory.obj
 0001:00048570       _$E1                       00449570 f   rylgamelibrary:serverwindowframework.obj
 0001:00048590       _$E1                       00449590 f   rylgamelibrary:consolewindow.obj
 0001:000485b0       _$E3                       004495b0 f   rylgamelibrary:consolewindow.obj
 0001:000485d0       _$E5                       004495d0 f   rylgamelibrary:consolewindow.obj
 0001:000485f0       _$E1                       004495f0 f   rylgamelibrary:xorcrypt.obj
 0001:00048610       _$E7                       00449610 f   rylgamelibrary:depositcontainer.obj
 0001:00048620       _$E5                       00449620 f   rylgamelibrary:itemconstants.obj
 0001:00048640       _$E5                       00449640 f   rylgamelibrary:item.obj
 0001:00048650       _$E5                       00449650 f   rylgamelibrary:itemcontainer.obj
 0001:00048660       _$E7                       00449660 f   rylgamelibrary:itemcontainer.obj
 0001:00048680       _$E5                       00449680 f   rylgamelibrary:skillmgr.obj
 0001:000486a0       _$E13                      004496a0 f   rylgamelibrary:creaturemanager.obj
 0001:000486b0       _$E17                      004496b0 f   rylgamelibrary:creaturemanager.obj
 0001:000486c0       _$E9                       004496c0 f   rylgamelibrary:cell.obj
 0001:000486d0       _$E5                       004496d0 f   rylgamelibrary:monstermgr.obj
 0001:000486f0       _$E5                       004496f0 f   rylgamelibrary:skilltable.obj
 0001:00048710       _$E8                       00449710 f   rylgamelibrary:skilltable.obj
 0001:00048720       _$E5                       00449720 f   rylgamelibrary:awardtable.obj
 0001:00048740       _$E5                       00449740 f   rylgamelibrary:rankingmgr.obj
 0001:00048760       _$E5                       00449760 f   rylgamelibrary:partymgr.obj
 0001:00048780       _$E1                       00449780 f   rylgamelibrary:friendlist.obj
 0001:000487a0       _$E5                       004497a0 f   rylgamelibrary:duelcellmanager.obj
 0001:000487c0       _$E5                       004497c0 f   rylgamelibrary:fsm.obj
 0001:000487e0       _$E5                       004497e0 f   rylgamelibrary:regularagentdispatch.obj
 0001:00048850       _$E5                       00449850 f   rylgamelibrary:questmgr.obj
 0001:00048866       _$E1                       00449866 f   libcpmt:xlock.obj
 0001:0004887c       _$E1                       0044987c f   libcpmt:locale0.obj
 0001:00048888       _$E1                       00449888 f   libcpmt:cout.obj
 0001:0004889e       _$E4                       0044989e f   libcpmt:cout.obj
 0001:000488bd       _$E7                       004498bd f   libcpmt:cout.obj
 0001:000488dc       _$E10                      004498dc f   libcpmt:cout.obj
 0001:000488e6       _$E1                       004498e6 f   libcpmt:iosptrs.obj
 0001:000488fc       _$E4                       004498fc f   libcpmt:iosptrs.obj
 0001:00048908       _$E5                       00449908 f   atls:atlbase.obj
 0001:00048920       _$E2                       00449920 f   authagentdispatch.obj
 0001:00048930       _$E2                       00449930 f   authagentservertable.obj
 0001:00048940       _$E2                       00449940 f   authclientdispath.obj
 0001:00048960       _$E2                       00449960 f   authorizeuser.obj
 0001:00048970       _$E2                       00449970 f   itemcreator.obj
 0001:00048980       _$E2                       00449980 f   rylauthserver.obj
 0001:00048990       _$E2                       00449990 f   rylgamelibrary:serverlog.obj
 0001:000489a0       _$E5                       004499a0 f   rylgamelibrary:serverlog.obj
 0001:000489b0       _$E8                       004499b0 f   rylgamelibrary:serverlog.obj
 0001:000489c0       _$E2                       004499c0 f   rylgamelibrary:serverrequest.obj
 0001:000489d0       _$E2                       004499d0 f   rylgamelibrary:serversetup.obj
 0001:000489e0       _$E6                       004499e0 f   rylgamelibrary:itemmgr.obj
 0001:000489f0       _$E6                       004499f0 f   rylgamelibrary:itemfactory.obj
 0001:00048a00       _$E2                       00449a00 f   rylgamelibrary:performancecheck.obj
 0001:00048a10       _$E6                       00449a10 f   rylgamelibrary:gamelog.obj
 0001:00048a20       _$E2                       00449a20 f   rylgamelibrary:packetstatistics.obj
 0001:00048a30       _$E2                       00449a30 f   rylgamelibrary:exceptionreport.obj
 0001:00048a40       _$E2                       00449a40 f   rylgamelibrary:xorcrypt.obj
 0001:00048a60       _$E6                       00449a60 f   rylgamelibrary:itemconstants.obj
 0001:00048a70       _$E2                       00449a70 f   rylgamelibrary:pulse.obj
 0001:00048a80       _$E8                       00449a80 f   rylgamelibrary:itemcontainer.obj
 0001:00048a90       _$E6                       00449a90 f   rylgamelibrary:skillmgr.obj
 0001:00048ad0       _$E6                       00449ad0 f   rylgamelibrary:monstermgr.obj
 0001:00048ae0       _$E6                       00449ae0 f   rylgamelibrary:skilltable.obj
 0001:00048af0       _$E6                       00449af0 f   rylgamelibrary:awardtable.obj
 0001:00048b00       _$E6                       00449b00 f   rylgamelibrary:rankingmgr.obj
 0001:00048b10       _$E6                       00449b10 f   rylgamelibrary:partymgr.obj
 0001:00048b20       _$E2                       00449b20 f   rylgamelibrary:friendlist.obj
 0001:00048b30       _$E6                       00449b30 f   rylgamelibrary:duelcellmanager.obj
 0001:00048b40       _$E6                       00449b40 f   rylgamelibrary:fsm.obj
 0001:00048b50       _$E6                       00449b50 f   rylgamelibrary:questmgr.obj
 0001:00048b5a       _$E2                       00449b5a f   libcpmt:xlock.obj
 0001:00048b64       _$E2                       00449b64 f   libcpmt:locale0.obj
 0001:00048b6e       _$E2                       00449b6e f   libcpmt:cout.obj
 0001:00048b78       _$E8                       00449b78 f   libcpmt:cout.obj
 0001:00048b94       _$E5                       00449b94 f   libcpmt:cout.obj
 0001:00048b9e       _$E2                       00449b9e f   libcpmt:nomemory.obj
 0001:00048ba8       _$E2                       00449ba8 f   libcpmt:iosptrs.obj
 0001:00048bb2       _$E5                       00449bb2 f   libcpmt:iosptrs.obj
 0001:00048bbc       _$E6                       00449bbc f   atls:atlbase.obj
